 CryAnimation

 Timestamp is 5036e49b (Fri Aug 24 04:19:07 2012)

 Preferred load address is 0000000031500000

 Start         Length     Name                   Class
 0001:00000000 0013fe2aH .text                   CODE
 0001:0013fe30 00000092H .text$x                 CODE
 0001:0013fed0 00000580H .text$yc                CODE
 0001:00140450 000006c5H .text$yd                CODE
 0002:00000000 00000298H .idata$5                DATA
 0002:00000298 00000008H .CRT$XCA                DATA
 0002:000002a0 000000d0H .CRT$XCU                DATA
 0002:00000370 00000008H .CRT$XCZ                DATA
 0002:00000378 00000008H .CRT$XIA                DATA
 0002:00000380 00000008H .CRT$XIAA               DATA
 0002:00000388 00000008H .CRT$XIZ                DATA
 0002:00000390 0000f788H .rdata                  DATA
 0002:0000fb18 00000057H .rdata$debug            DATA
 0002:0000fb70 00000008H .rtc$IAA                DATA
 0002:0000fb78 00000008H .rtc$IZZ                DATA
 0002:0000fb80 00000008H .rtc$TAA                DATA
 0002:0000fb88 00000008H .rtc$TZZ                DATA
 0002:0000fb90 00010dbcH .xdata                  DATA
 0002:0002094c 0000003cH .idata$2                DATA
 0002:00020988 00000014H .idata$3                DATA
 0002:000209a0 00000298H .idata$4                DATA
 0002:00020c38 00000490H .idata$6                DATA
 0002:000210d0 00000076H .edata                  DATA
 0003:00000000 00002758H .data                   DATA
 0003:00002760 0000af58H .bss                    DATA
 0004:00000000 0000de3cH .pdata                  DATA
 0005:00000000 00000008H .tls$                   DATA
 0006:00000000 00000058H .rsrc$01                DATA
 0006:00000060 00000248H .rsrc$02                DATA

  Address         Publics by Value              Rva+Base               Lib:Object

 0000:00000000       ___safe_se_handler_table   0000000000000000     <absolute>
 0000:00000000       ___safe_se_handler_count   0000000000000000     <absolute>
 0000:00000000       __ImageBase                0000000031500000     <linker-defined>
 0001:00000000       ??_EIMemReplay@@UEAAPEAXI@Z 0000000031501000 f i AnimEventList.obj
 0001:00000000       ??_GCDummyMemReplay@@UEAAPEAXI@Z 0000000031501000 f i AnimEventList.obj
 0001:00000000       ??_GIMemReplay@@UEAAPEAXI@Z 0000000031501000 f i AnimEventList.obj
 0001:00000000       ??_ECDummyMemReplay@@UEAAPEAXI@Z 0000000031501000 f i AnimEventList.obj
 0001:00000030       ?AddLabelFmt@CDummyMemReplay@@UEAAXPEBDZZ 0000000031501030 f i AnimEventList.obj
 0001:00000040       ?alloc@?$AllocPrefix@UStandardAlloc@NAlloc@@@NAlloc@@SAPEAXAEA_K_NHH@Z 0000000031501040 f i AnimEventList.obj
 0001:000000f0       ??0?$CryStringT@D@@QEAA@AEBV0@@Z 00000000315010f0 f i AnimEventList.obj
 0001:00000120       ?_Free@?$CryStringT@D@@IEAAXXZ 0000000031501120 f i AnimEventList.obj
 0001:00000170       ?GetByIndex@CAnimEventList@@UEAAAEAVCAnimEventData@@I@Z 0000000031501170 f   AnimEventList.obj
 0001:00000170       ?GetByIndex@CAnimEventList@@UEBAAEBVCAnimEventData@@I@Z 0000000031501170 f   AnimEventList.obj
 0001:00000180       ?CryGetIMemReplay@@YAPEAUIMemReplay@@XZ 0000000031501180 f i AnimEventList.obj
 0001:00000200       ?GetMemoryUsage@CAnimEventData@@QEBAXPEAVICrySizer@@@Z 0000000031501200 f i AnimEventList.obj
 0001:00000280       ??1?$CryStringT@D@@QEAA@XZ 0000000031501280 f i AnimEventList.obj
 0001:000002c0       ??4?$CryStringT@D@@QEAAAEAV0@AEBV0@@Z 00000000315012c0 f i AnimEventList.obj
 0001:00000370       ??0CAnimEventData@@QEAA@AEBV0@@Z 0000000031501370 f i AnimEventList.obj
 0001:00000410       ?set_size@?$SmallDynStorage@VCAnimEventData@@HUStandardAlloc@NAlloc@@@NArray@@QEAAXH@Z 0000000031501410 f i AnimEventList.obj
 0001:000004c0       ?get_alloc_size@?$SmallDynStorage@VCAnimEventData@@HUStandardAlloc@NAlloc@@@NArray@@QEBAHXZ 00000000315014c0 f i AnimEventList.obj
 0001:00000520       ??1CAnimEventData@@QEAA@XZ 0000000031501520 f i AnimEventList.obj
 0001:000005f0       ?GetAllocSize@CAnimEventList@@QEBA_KXZ 00000000315015f0 f   AnimEventList.obj
 0001:00000780       ??$AddObject@VCAnimEventData@@HU?$SmallDynStorage@VCAnimEventData@@HUStandardAlloc@NAlloc@@@NArray@@@ICrySizer@@QEAAXAEBU?$DynArray@VCAnimEventData@@HU?$SmallDynStorage@VCAnimEventData@@HUStandardAlloc@NAlloc@@@NArray@@@@@Z 0000000031501780 f i AnimEventList.obj
 0001:00000820       ??$move_init@VCAnimEventData@@@NArray@@YAXPEAVCAnimEventData@@0_K@Z 0000000031501820 f i AnimEventList.obj
 0001:00000880       ?GetMemoryUsage@CAnimEventList@@QEBAXPEAVICrySizer@@@Z 0000000031501880 f   AnimEventList.obj
 0001:00000890       ?pop_back@?$DynArray@VCAnimEventData@@HU?$SmallDynStorage@VCAnimEventData@@HUStandardAlloc@NAlloc@@@NArray@@@@QEAAXH@Z 0000000031501890 f i AnimEventList.obj
 0001:00000910       ?resize_raw@?$SmallDynStorage@VCAnimEventData@@HUStandardAlloc@NAlloc@@@NArray@@QEAAXHH_N@Z 0000000031501910 f i AnimEventList.obj
 0001:00000a90       ?clear@?$DynArray@VCAnimEventData@@HU?$SmallDynStorage@VCAnimEventData@@HUStandardAlloc@NAlloc@@@NArray@@@@QEAAXXZ 0000000031501a90 f i AnimEventList.obj
 0001:00000b30       ?erase@?$DynArray@VCAnimEventData@@HU?$SmallDynStorage@VCAnimEventData@@HUStandardAlloc@NAlloc@@@NArray@@@@QEAAPEAVCAnimEventData@@PEAV2@0@Z 0000000031501b30 f i AnimEventList.obj
 0001:00000c30       ??1?$DynArray@VCAnimEventData@@HU?$SmallDynStorage@VCAnimEventData@@HUStandardAlloc@NAlloc@@@NArray@@@@QEAA@XZ 0000000031501c30 f i AnimEventList.obj
 0001:00000cb0       ?expand_raw@?$DynArray@VCAnimEventData@@HU?$SmallDynStorage@VCAnimEventData@@HUStandardAlloc@NAlloc@@@NArray@@@@IEAAPEAVCAnimEventData@@PEAV2@H@Z 0000000031501cb0 f i AnimEventList.obj
 0001:00000d70       ??0CAnimEventList@@QEAA@XZ 0000000031501d70 f   AnimEventList.obj
 0001:00000de0       ??1CAnimEventList@@UEAA@XZ 0000000031501de0 f   AnimEventList.obj
 0001:00000e10       ?Clear@CAnimEventList@@UEAAXXZ 0000000031501e10 f   AnimEventList.obj
 0001:00000e20       ??_GCAnimEventList@@UEAAPEAXI@Z 0000000031501e20 f i AnimEventList.obj
 0001:00000e20       ??_ECAnimEventList@@UEAAPEAXI@Z 0000000031501e20 f i AnimEventList.obj
 0001:00000e70       ?Remove@CAnimEventList@@UEAAXI@Z 0000000031501e70 f   AnimEventList.obj
 0001:00000e90       ?grow@?$DynArray@VCAnimEventData@@HU?$SmallDynStorage@VCAnimEventData@@HUStandardAlloc@NAlloc@@@NArray@@@@QEAAPEAVCAnimEventData@@HAEBV2@@Z 0000000031501e90 f i AnimEventList.obj
 0001:00000f10       ?Append@CAnimEventList@@UEAAXAEBVCAnimEventData@@@Z 0000000031501f10 f   AnimEventList.obj
 0001:00000f30       ?ClearBinding@CAttachmentSKIN@@UEAAXXZ 0000000031501f30 f   Attachment.obj
 0001:00000f60       ?ClearBinding@CAttachmentFACE@@UEAAXXZ 0000000031501f60 f   Attachment.obj
 0001:00000f60       ?ClearBinding@CAttachmentBONE@@UEAAXXZ 0000000031501f60 f   Attachment.obj
 0001:00000fc0       ?GetPendulumParams2@SAttachmentPendulum@@QEAAXAEAHAEAC1AEAM22AEAU?$Vec3_tpl@M@@3@Z 0000000031501fc0 f   Attachment.obj
 0001:00001120       ?CryFatalError@@YAXPEBDZZ  0000000031502120 f i Attachment.obj
 0001:000011c0       ?CryLogAlways@@YAXPEBDZZ   00000000315021c0 f i Attachment.obj
 0001:00001220       ??_EIAttachment@@UEAAPEAXI@Z 0000000031502220 f i Attachment.obj
 0001:00001220       ??_GIAttachment@@UEAAPEAXI@Z 0000000031502220 f i Attachment.obj
 0001:00001250       ??_GIAttachmentSkin@@UEAAPEAXI@Z 0000000031502250 f i Attachment.obj
 0001:00001250       ??_EIAttachmentSkin@@UEAAPEAXI@Z 0000000031502250 f i Attachment.obj
 0001:00001280       ?SetBoneName@CAttachmentBONE@@UEAAIPEBD@Z 0000000031502280 f   Attachment.obj
 0001:00001320       ?AddBinding@CAttachmentBONE@@UEAAIPEAUIAttachmentObject@@V?$_smart_ptr@UISkin@@@@I@Z 0000000031502320 f   Attachment.obj
 0001:00001320       ?AddBinding@CAttachmentFACE@@UEAAIPEAUIAttachmentObject@@V?$_smart_ptr@UISkin@@@@I@Z 0000000031502320 f   Attachment.obj
 0001:000013c0       ?ToVec3@Vec3f16@@QEBA?AU?$Vec3_tpl@M@@XZ 00000000315023c0 f i Attachment.obj
 0001:00001510       ?ToVec2@Vec2f16@@QEBA?AU?$Vec2_tpl@M@@XZ 0000000031502510 f i Attachment.obj
 0001:00001600       ?Draw2dLabel@IRenderer@@QEAAXMMMPEBM_NPEBDZZ 0000000031502600 f i Attachment.obj
 0001:000016c0       ?GetAttWorldAbsolute@CAttachmentSKIN@@UEBA?BU?$QuatTS_tpl@M@@XZ 00000000315026c0 f   Attachment.obj
 0001:00001720       ?AlignBoneAttachment@CAttachmentBONE@@UEAAXXZ 0000000031502720 f   Attachment.obj
 0001:000017e0       ?Serialize@CAttachmentFACE@@UEAAXV?$CSerializeWrapper@UISerialize@@@@@Z 00000000315027e0 f   Attachment.obj
 0001:000017e0       ?Serialize@CAttachmentSKIN@@UEAAXV?$CSerializeWrapper@UISerialize@@@@@Z 00000000315027e0 f   Attachment.obj
 0001:000017e0       ?Serialize@CAttachmentBONE@@UEAAXV?$CSerializeWrapper@UISerialize@@@@@Z 00000000315027e0 f   Attachment.obj
 0001:00001880       ?GetAttWorldAbsolute@CAttachmentFACE@@UEBA?BU?$QuatTS_tpl@M@@XZ 0000000031502880 f   Attachment.obj
 0001:00001880       ?GetAttWorldAbsolute@CAttachmentBONE@@UEBA?BU?$QuatTS_tpl@M@@XZ 0000000031502880 f   Attachment.obj
 0001:00001b40       ?SetPendulumParams2@SAttachmentPendulum@@QEAAXHCCMMMU?$Vec3_tpl@M@@0@Z 0000000031502b40 f   Attachment.obj
 0001:00002120       ?DrawWireframeStatic@CAttachmentSKIN@@UEAAXAEBU?$Matrix34_tpl@M@@HI@Z 0000000031503120 f   Attachment.obj
 0001:000021a0       ?InitRenderMeshsSW@CAttachmentSKIN@@QEAAXXZ 00000000315031a0 f   Attachment.obj
 0001:00002930       ?ProjectAttachment@CAttachmentBONE@@UEAAIXZ 0000000031503930 f   Attachment.obj
 0001:00002e00       ?SizeOfThis@CAttachmentBONE@@UEAA_KXZ 0000000031503e00 f   Attachment.obj
 0001:00002e10       ?GetMemoryUsage@CAttachmentBONE@@UEBAXPEAVICrySizer@@@Z 0000000031503e10 f   Attachment.obj
 0001:00002e60       ?SizeOfThis@CAttachmentFACE@@UEAA_KXZ 0000000031503e60 f   Attachment.obj
 0001:00002e70       ?GetMemoryUsage@CAttachmentFACE@@UEBAXPEAVICrySizer@@@Z 0000000031503e70 f   Attachment.obj
 0001:00002ec0       ?UpdatePendulumPhysics@SAttachmentPendulum@@QEAAXXZ 0000000031503ec0 f   Attachment.obj
 0001:00005db0       ?set_size@?$SmallDynStorage@EHUStandardAlloc@NAlloc@@@NArray@@QEAAXH@Z 0000000031506db0 f i Attachment.obj
 0001:00005db0       ?set_size@?$SmallDynStorage@DHUStandardAlloc@NAlloc@@@NArray@@QEAAXH@Z 0000000031506db0 f i LoaderCHR.obj
 0001:00005db0       ?set_size@?$SmallDynStorage@_NHUStandardAlloc@NAlloc@@@NArray@@QEAAXH@Z 0000000031506db0 f i CharacterInstance.obj
 0001:00005e50       ?resize_raw@?$SmallDynStorage@EHUStandardAlloc@NAlloc@@@NArray@@QEAAXHH_N@Z 0000000031506e50 f i Attachment.obj
 0001:00005fd0       ?SizeOfThis@CAttachmentSKIN@@UEAA_KXZ 0000000031506fd0 f   Attachment.obj
 0001:00006040       ?UpdateLocation@CAttachmentBONE@@UEAAXXZ 0000000031507040 f   Attachment.obj
 0001:000063f0       ?DrawAttachment@CAttachmentBONE@@UEAAXAEAUSRendParams@@AEBUSRenderingPassInfo@@AEBU?$Matrix34_tpl@M@@M@Z 00000000315073f0 f   Attachment.obj
 0001:00007560       ?ProjectAttachment@CAttachmentFACE@@UEAAIXZ 0000000031508560 f   Attachment.obj
 0001:00008ba0       ?UpdateLocation@CAttachmentFACE@@UEAAXXZ 0000000031509ba0 f   Attachment.obj
 0001:0000a780       ?DrawAttachment@CAttachmentFACE@@UEAAXAEAUSRendParams@@AEBUSRenderingPassInfo@@AEBU?$Matrix34_tpl@M@@M@Z 000000003150b780 f   Attachment.obj
 0001:0000b8f0       ?GetMemoryUsage@CAttachmentSKIN@@UEBAXPEAVICrySizer@@@Z 000000003150c8f0 f   Attachment.obj
 0001:0000b9e0       ?append_raw@?$DynArray@EHU?$SmallDynStorage@EHUStandardAlloc@NAlloc@@@NArray@@@@QEAA?AU?$Array@EHU?$ArrayStorage@EH@NArray@@@@H@Z 000000003150c9e0 f i Attachment.obj
 0001:0000ba90       ??1CAttachmentSKIN@@UEAA@XZ 000000003150ca90 f   Attachment.obj
 0001:0000bc80       ?AddRef@CAttachmentSKIN@@UEAAXXZ 000000003150cc80 f i Attachment.obj
 0001:0000bc90       ?Release@CAttachmentSKIN@@UEAAXXZ 000000003150cc90 f i Attachment.obj
 0001:0000bcb0       ?IsAttachmentHidden@CAttachmentBONE@@UEAAIXZ 000000003150ccb0 f i AttachmentManager.obj
 0001:0000bcb0       ?IsAttachmentHidden@CAttachmentFACE@@UEAAIXZ 000000003150ccb0 f i AttachmentManager.obj
 0001:0000bcb0       ?IsAttachmentHidden@CAttachmentSKIN@@UEAAIXZ 000000003150ccb0 f i Attachment.obj
 0001:0000bcc0       ?HideInShadow@CAttachmentFACE@@UEAAXI@Z 000000003150ccc0 f i AttachmentManager.obj
 0001:0000bcc0       ?HideInShadow@CAttachmentSKIN@@UEAAXI@Z 000000003150ccc0 f i Attachment.obj
 0001:0000bcc0       ?HideInShadow@CAttachmentBONE@@UEAAXI@Z 000000003150ccc0 f i AttachmentManager.obj
 0001:0000bce0       ?GetAttRelativeDefault@CAttachmentSKIN@@UEBAAEBU?$QuatT_tpl@M@@XZ 000000003150cce0 f i Attachment.obj
 0001:0000bce0       ?GetAttAbsoluteDefault@CAttachmentSKIN@@UEBAAEBU?$QuatT_tpl@M@@XZ 000000003150cce0 f i Attachment.obj
 0001:0000bce0       ?GetAttModelRelative@CAttachmentSKIN@@UEBAAEBU?$QuatT_tpl@M@@XZ 000000003150cce0 f i Attachment.obj
 0001:0000bcf0       ?QueryComposite@CPoseBlenderLook@@MEBAPEAXPEBD@Z 000000003150ccf0 f i PoseBlenderLook.obj
 0001:0000bcf0       ?SetBoneName@CAttachmentSKIN@@UEAAIPEBD@Z 000000003150ccf0 f i Attachment.obj
 0001:0000bcf0       ?SetBoneName@CAttachmentFACE@@UEAAIPEBD@Z 000000003150ccf0 f i AttachmentManager.obj
 0001:0000bcf0       ?get_deleter@?$sp_counted_impl_p@VCOperatorQueue@@@detail@boost@@UEAAPEAXAEBVsp_typeinfo@23@@Z 000000003150ccf0 f i OperatorQueue.obj
 0001:0000bcf0       ?GetRelocateChain@?$CKeyTimesInformationStartStop@MUF32StartStopEncoder@@@@UEAAPEAVIControllerRelocatableChain@@XZ 000000003150ccf0 f i ControllerPQ.obj
 0001:0000bcf0       ?QueryComposite@CLimbIk@@MEBAPEAXPEBD@Z 000000003150ccf0 f i LimbIk.obj
 0001:0000bcf0       ?GetRelocateChain@?$CKeyTimesInformationStartStop@EUByteStartStopEncoder@@@@UEAAPEAVIControllerRelocatableChain@@XZ 000000003150ccf0 f i ControllerPQ.obj
 0001:0000bcf0       ?GetPositionKeysNum@CControllerPQLog@@UEBA_KXZ 000000003150ccf0 f i ControllerPQLog.obj
 0001:0000bcf0       ?GetType@CFacialEffector@@UEAA?AW4EFacialEffectorType@@XZ 000000003150ccf0 f i FaceEffector.obj
 0001:0000bcf0       ?get_deleter@?$sp_counted_impl_p@VCPoseBlenderLook@@@detail@boost@@UEAAPEAXAEBVsp_typeinfo@23@@Z 000000003150ccf0 f i PoseBlenderLook.obj
 0001:0000bcf0       ?GetRotationKeysNum@CControllerTCB@@UEBA_KXZ 000000003150ccf0 f i LoaderCGA.obj
 0001:0000bcf0       ?QueryComposite@COperatorQueue@@MEBAPEAXPEBD@Z 000000003150ccf0 f i OperatorQueue.obj
 0001:0000bcf0       ?get_deleter@?$sp_counted_impl_p@VCPoseAlignerChain@@@detail@boost@@UEAAPEAXAEBVsp_typeinfo@23@@Z 000000003150ccf0 f i PoseAlignerChain.obj
 0001:0000bcf0       ?QueryComposite@CEngineModule_CryAnimation@@MEBAPEAXPEBD@Z 000000003150ccf0 f i AnimationBase.obj
 0001:0000bcf0       ?get_deleter@?$sp_counted_impl_p@VCEngineModule_CryAnimation@@@detail@boost@@UEAAPEAXAEBVsp_typeinfo@23@@Z 000000003150ccf0 f i AnimationBase.obj
 0001:0000bcf0       ?get_deleter@?$sp_counted_impl_p@VCFeetPoseRestore@@@detail@boost@@UEAAPEAXAEBVsp_typeinfo@23@@Z 000000003150ccf0 f i FeetLock.obj
 0001:0000bcf0       ?QueryComposite@CFeetPoseStore@@MEBAPEAXPEBD@Z 000000003150ccf0 f i FeetLock.obj
 0001:0000bcf0       ?QueryComposite@CFeetPoseRestore@@MEBAPEAXPEBD@Z 000000003150ccf0 f i FeetLock.obj
 0001:0000bcf0       ?QueryComposite@CPoseAlignerChain@@MEBAPEAXPEBD@Z 000000003150ccf0 f i PoseAlignerChain.obj
 0001:0000bcf0       ?get_deleter@?$sp_counted_impl_p@VCRecoil@PoseModifier@@@detail@boost@@UEAAPEAXAEBVsp_typeinfo@23@@Z 000000003150ccf0 f i Recoil.obj
 0001:0000bcf0       ?ProjectAttachment@CAttachmentSKIN@@UEAAIXZ 000000003150ccf0 f i Attachment.obj
 0001:0000bcf0       ?get_deleter@?$sp_counted_impl_p@VCPoseMatching@@@detail@boost@@UEAAPEAXAEBVsp_typeinfo@23@@Z 000000003150ccf0 f i PoseMatching.obj
 0001:0000bcf0       ?get_deleter@?$sp_counted_impl_p@VCPoseBlenderAim@@@detail@boost@@UEAAPEAXAEBVsp_typeinfo@23@@Z 000000003150ccf0 f i PoseBlenderAim.obj
 0001:0000bcf0       ?GetRelocateChain@?$CKeyTimesInformationStartStop@GUUINT16StartStopEncoder@@@@UEAAPEAVIControllerRelocatableChain@@XZ 000000003150ccf0 f i ControllerPQ.obj
 0001:0000bcf0       ?get_deleter@?$sp_counted_impl_p@VCFeetPoseStore@@@detail@boost@@UEAAPEAXAEBVsp_typeinfo@23@@Z 000000003150ccf0 f i FeetLock.obj
 0001:0000bcf0       ?GetParamInt@CFacialEffector@@UEAAHW4EFacialEffectorParam@@@Z 000000003150ccf0 f i FaceEffector.obj
 0001:0000bcf0       ?get_deleter@?$sp_counted_impl_p@VCGroundAlignment@@@detail@boost@@UEAAPEAXAEBVsp_typeinfo@23@@Z 000000003150ccf0 f i GroundAlignment.obj
 0001:0000bcf0       ?GetAttachmentCRC@CFacialEffector@@UEAAIXZ 000000003150ccf0 f i FaceEffector.obj
 0001:0000bcf0       ?QueryComposite@CPoseMatching@@MEBAPEAXPEBD@Z 000000003150ccf0 f i PoseMatching.obj
 0001:0000bcf0       ?GetFormat@?$CKeyTimesInformation@MUF32Encoder@@@@UEAAIXZ 000000003150ccf0 f i ControllerPQ.obj
 0001:0000bcf0       ?GetRotationKeysNum@CControllerPQLog@@UEBA_KXZ 000000003150ccf0 f i ControllerPQLog.obj
 0001:0000bcf0       ?StreamOnNeedStorage@IStreamCallback@@UEAAPEAXPEAVIReadStream@@I@Z 000000003150ccf0 f i FaceAnimSequence.obj
 0001:0000bcf0       ?Allocate@CPool@Memory@@UEAAPEAXI@Z 000000003150ccf0 f i Pool.obj
 0001:0000bcf0       ?GetPositionKeysNum@CControllerTCB@@UEBA_KXZ 000000003150ccf0 f i LoaderCGA.obj
 0001:0000bcf0       ?QueryComposite@CGroundAlignment@@MEBAPEAXPEBD@Z 000000003150ccf0 f i GroundAlignment.obj
 0001:0000bcf0       ?get_deleter@?$sp_counted_impl_p@VCLimbIk@@@detail@boost@@UEAAPEAXAEBVsp_typeinfo@23@@Z 000000003150ccf0 f i LimbIk.obj
 0001:0000bcf0       ?GetIStatObj@IAttachmentObject@@UEBAPEAUIStatObj@@XZ 000000003150ccf0 f i AttachmentManager.obj
 0001:0000bcf0       ?QueryComposite@CPoseBlenderAim@@MEBAPEAXPEBD@Z 000000003150ccf0 f i PoseBlenderAim.obj
 0001:0000bcf0       ?GetRelocateChain@CKeyTimesInformationBitSet@@UEAAPEAVIControllerRelocatableChain@@XZ 000000003150ccf0 f i ControllerPQ.obj
 0001:0000bcf0       ?GetIAttachmentSkin@IAttachmentObject@@UEBAPEAUIAttachmentSkin@@XZ 000000003150ccf0 f i AttachmentManager.obj
 0001:0000bcf0       ?GetType@CAttachmentBONE@@UEBAIXZ 000000003150ccf0 f i AttachmentManager.obj
 0001:0000bcf0       ?GetICharacterInstance@IAttachmentObject@@UEBAPEAUICharacterInstance@@XZ 000000003150ccf0 f i AttachmentManager.obj
 0001:0000bcf0       ?QueryComposite@CRecoil@PoseModifier@@MEBAPEAXPEBD@Z 000000003150ccf0 f i Recoil.obj
 0001:0000bd00       ?GetIVertexAnimation@CAttachmentSKIN@@UEAAPEAUIVertexAnimation@@XZ 000000003150cd00 f i Attachment.obj
 0001:0000bd10       ?Release@CAttachmentSKIN@@W7EAAXXZ 000000003150cd10 f i Attachment.obj
 0001:0000bd20       ??_ECAttachmentSKIN@@W7EAAPEAXI@Z 000000003150cd20 f i Attachment.obj
 0001:0000bd30       ?AddRef@CAttachmentSKIN@@W7EAAXXZ 000000003150cd30 f i Attachment.obj
 0001:0000bd40       ?GetPendulumParams@CAttachmentSKIN@@UEAAXAEAHAEAC1AEAM22AEAU?$Vec3_tpl@M@@3@Z 000000003150cd40 f i Attachment.obj
 0001:0000bd80       ?GetParent@CFacialAnimChannel@@UEAAPEAUIFacialAnimChannel@@XZ 000000003150cd80 f i FaceAnimSequence.obj
 0001:0000bd80       ?GetFacialInstance@CCharInstance@@UEAAPEAUIFacialInstance@@XZ 000000003150cd80 f i CharacterInstance.obj
 0001:0000bd80       ?GetISkin@CAttachmentSKIN@@UEAAPEAUISkin@@XZ 000000003150cd80 f i Attachment.obj
 0001:0000bd90       ?_AllocData@?$CryStringT@D@@IEAAX_K@Z 000000003150cd90 f i Attachment.obj
 0001:0000be00       ?_Assign@?$CryStringT@D@@IEAAXPEBD_K@Z 000000003150ce00 f i Attachment.obj
 0001:0000bee0       ?_MakeUnique@?$CryStringT@D@@IEAAXXZ 000000003150cee0 f i Attachment.obj
 0001:0000bfa0       ??4?$CryStringT@D@@QEAAAEAV0@PEBD@Z 000000003150cfa0 f i Attachment.obj
 0001:0000bff0       ?append@?$CryStringT@D@@QEAAAEAV1@_KD@Z 000000003150cff0 f i Attachment.obj
 0001:0000c0e0       ?resize@?$CryStringT@D@@QEAAX_KD@Z 000000003150d0e0 f i Attachment.obj
 0001:0000c150       ?GetMemoryUsage@CAttachmentSKIN@@W7EBAXPEAVICrySizer@@@Z 000000003150d150 f i Attachment.obj
 0001:0000c160       ?clear@?$CryStringT@D@@QEAAXXZ 000000003150d160 f i Attachment.obj
 0001:0000c1d0       ??_GCAttachmentSKIN@@UEAAPEAXI@Z 000000003150d1d0 f i Attachment.obj
 0001:0000c1d0       ??_ECAttachmentSKIN@@UEAAPEAXI@Z 000000003150d1d0 f i Attachment.obj
 0001:0000c200       ?resize@?$DynArray@EHU?$SmallDynStorage@EHUStandardAlloc@NAlloc@@@NArray@@@@QEAAXH@Z 000000003150d200 f i Attachment.obj
 0001:0000c240       ?AddBinding@CAttachmentSKIN@@UEAAIPEAUIAttachmentObject@@V?$_smart_ptr@UISkin@@@@I@Z 000000003150d240 f   Attachment.obj
 0001:0000c560       ?GetStats@CControllerDefragHeap@@QEAA?AUStats@1@XZ 000000003150d560 f   ControllerDefragHeap.obj
 0001:0000c5e0       ?SyncCopy@CControllerDefragHeap@@EEAAXPEAX_K11@Z 000000003150d5e0 f   ControllerDefragHeap.obj
 0001:0000c5f0       ??_GIDefragAllocatorPolicy@@MEAAPEAXI@Z 000000003150d5f0 f i ControllerDefragHeap.obj
 0001:0000c5f0       ??_EIDefragAllocatorPolicy@@MEAAPEAXI@Z 000000003150d5f0 f i ControllerDefragHeap.obj
 0001:0000c620       ?UsableSize@CControllerDefragHeap@@QEAA_KVCControllerDefragHdl@@@Z 000000003150d620 f   ControllerDefragHeap.obj
 0001:0000c650       ?CancelCopy@CControllerDefragHeap@@EEAAXIPEAX_N@Z 000000003150d650 f   ControllerDefragHeap.obj
 0001:0000c6b0       ?Relocate@CControllerDefragHeap@@EEAAXIPEAX_K11@Z 000000003150d6b0 f   ControllerDefragHeap.obj
 0001:0000c7e0       ?allocate@?$_STLP_alloc_proxy@PEAHHV?$allocator@H@stlpmtx_std@@@priv@stlpmtx_std@@QEAAPEAH_KAEA_K@Z 000000003150d7e0 f i ControllerDefragHeap.obj
 0001:0000c850       ?IncreaseRange@CControllerDefragHeap@@AEAA_N_K0@Z 000000003150d850 f   ControllerDefragHeap.obj
 0001:0000c940       ?DecreaseRange@CControllerDefragHeap@@AEAAX_K0@Z 000000003150d940 f   ControllerDefragHeap.obj
 0001:0000c9c0       ?_M_insert_overflow@?$_Impl_vector@HV?$allocator@H@stlpmtx_std@@@priv@stlpmtx_std@@AEAAXPEAHAEBHAEBU__true_type@3@_K_N@Z 000000003150d9c0 f i ControllerDefragHeap.obj
 0001:0000c9c0       ?_M_insert_overflow@?$_Impl_vector@MV?$allocator@M@stlpmtx_std@@@priv@stlpmtx_std@@AEAAXPEAMAEBMAEBU__true_type@3@_K_N@Z 000000003150d9c0 f i FaceAnimation.obj
 0001:0000c9c0       ?_M_insert_overflow@?$_Impl_vector@IV?$allocator@I@stlpmtx_std@@@priv@stlpmtx_std@@AEAAXPEAIAEBIAEBU__true_type@3@_K_N@Z 000000003150d9c0 f i SkeletonPose_Process.obj
 0001:0000cb30       ?_M_fill_insert_aux@?$_Impl_vector@HV?$allocator@H@stlpmtx_std@@@priv@stlpmtx_std@@AEAAXPEAH_KAEBHAEBU__false_type@3@@Z 000000003150db30 f i ControllerDefragHeap.obj
 0001:0000cb30       ?_M_fill_insert_aux@?$_Impl_vector@IV?$allocator@I@stlpmtx_std@@@priv@stlpmtx_std@@AEAAXPEAI_KAEBIAEBU__false_type@3@@Z 000000003150db30 f i CharacterManager.obj
 0001:0000ccc0       ??$__insertion_sort@PEAIIU?$less@I@stlpmtx_std@@@priv@stlpmtx_std@@YAXPEAI00U?$less@I@1@@Z 000000003150dcc0 f i ControllerDefragHeap.obj
 0001:0000cd80       ??$__make_heap@PEAIU?$less@I@stlpmtx_std@@I_J@stlpmtx_std@@YAXPEAI0U?$less@I@0@0PEA_J@Z 000000003150dd80 f i ControllerDefragHeap.obj
 0001:0000ce60       ??1CControllerDefragHeap@@UEAA@XZ 000000003150de60 f   ControllerDefragHeap.obj
 0001:0000cee0       ?AllocPinned@CControllerDefragHeap@@QEAA?AVCControllerDefragHdl@@_KPEAVIControllerRelocatableChain@@@Z 000000003150dee0 f   ControllerDefragHeap.obj
 0001:0000d120       ?Free@CControllerDefragHeap@@QEAAXVCControllerDefragHdl@@@Z 000000003150e120 f   ControllerDefragHeap.obj
 0001:0000d250       ?BeginCopy@CControllerDefragHeap@@EEAAIPEAX_K11PEAUIDefragAllocatorCopyNotification@@@Z 000000003150e250 f   ControllerDefragHeap.obj
 0001:0000d3c0       ??$__final_insertion_sort@PEAIU?$less@I@stlpmtx_std@@@priv@stlpmtx_std@@YAXPEAI0U?$less@I@1@@Z 000000003150e3c0 f i ControllerDefragHeap.obj
 0001:0000d460       ??0CControllerDefragHeap@@QEAA@XZ 000000003150e460 f   ControllerDefragHeap.obj
 0001:0000d520       ??_ECControllerDefragHeap@@UEAAPEAXI@Z 000000003150e520 f i ControllerDefragHeap.obj
 0001:0000d520       ??_GCControllerDefragHeap@@UEAAPEAXI@Z 000000003150e520 f i ControllerDefragHeap.obj
 0001:0000d550       ??$sort_heap@PEAIU?$less@I@stlpmtx_std@@@stlpmtx_std@@YAXPEAI0U?$less@I@0@@Z 000000003150e550 f i ControllerDefragHeap.obj
 0001:0000d640       ??$__partial_sort@PEAIIU?$less@I@stlpmtx_std@@@priv@stlpmtx_std@@YAXPEAI000U?$less@I@1@@Z 000000003150e640 f i ControllerDefragHeap.obj
 0001:0000d740       ?Init@CControllerDefragHeap@@QEAAX_K@Z 000000003150e740 f   ControllerDefragHeap.obj
 0001:0000d890       ??$__introsort_loop@PEAII_JU?$less@I@stlpmtx_std@@@priv@stlpmtx_std@@YAXPEAI00_JU?$less@I@1@@Z 000000003150e890 f i ControllerDefragHeap.obj
 0001:0000d9c0       ??$sort@PEAI@stlpmtx_std@@YAXPEAI0@Z 000000003150e9c0 f i ControllerDefragHeap.obj
 0001:0000da30       ?UpdateInflight@CControllerDefragHeap@@AEAAXH@Z 000000003150ea30 f   ControllerDefragHeap.obj
 0001:0000dd00       ?Update@CControllerDefragHeap@@QEAAXXZ 000000003150ed00 f   ControllerDefragHeap.obj
 0001:0000de90       ?Draw@DrawHelper@@YAXAEBUSegment@1@@Z 000000003150ee90 f   DrawHelper.obj
 0001:0000ded0       ?Draw@DrawHelper@@YAXAEBUSphere@1@@Z 000000003150eed0 f   DrawHelper.obj
 0001:0000df00       ?Draw@DrawHelper@@YAXAEBUCylinder@1@@Z 000000003150ef00 f   DrawHelper.obj
 0001:0000df40       ??$?DMM@@YA?AU?$Vec3_tpl@M@@AEBU?$QuatT_tpl@M@@AEBU0@@Z 000000003150ef40 f i DrawHelper.obj
 0001:0000e090       ?DepthTest@DrawHelper@@YAX_N@Z 000000003150f090 f   DrawHelper.obj
 0001:0000e0f0       ?Frame@DrawHelper@@YAXAEBU?$Vec3_tpl@M@@000@Z 000000003150f0f0 f   DrawHelper.obj
 0001:0000e250       ?Frame@DrawHelper@@YAXAEBU?$Matrix34_tpl@M@@AEBU?$Vec3_tpl@M@@@Z 000000003150f250 f   DrawHelper.obj
 0001:0000e460       ?BonePrism@DrawHelper@@YAXAEBU?$Vec3_tpl@M@@00U?$Color_tpl@E@@@Z 000000003150f460 f   DrawHelper.obj
 0001:0000eb50       ?Frame@DrawHelper@@YAXAEBU?$QuatT_tpl@M@@AEBU?$Vec3_tpl@M@@@Z 000000003150fb50 f   DrawHelper.obj
 0001:0000ecf0       ?Arrow@DrawHelper@@YAXAEBU?$QuatT_tpl@M@@AEBU?$Vec3_tpl@M@@MU?$Color_tpl@E@@@Z 000000003150fcf0 f   DrawHelper.obj
 0001:0000f4f0       ?CurvedArrow@DrawHelper@@YAXAEBU?$QuatT_tpl@M@@MMMMU?$Color_tpl@E@@@Z 00000000315104f0 f   DrawHelper.obj
 0001:000109e0       ?BonePrism@DrawHelper@@YAMU?$QuatT_tpl@M@@AEBU?$Vec3_tpl@M@@U?$Color_tpl@E@@@Z 00000000315119e0 f   DrawHelper.obj
 0001:00011150       ?Pose@DrawHelper@@YAXAEBVCPoseData@Skeleton@@AEBU?$QuatT_tpl@M@@U?$Color_tpl@E@@@Z 0000000031512150 f   DrawHelper.obj
 0001:00011840       ??4?$_smart_ptr@UIRenderMesh@@@@QEAAAEAV0@PEAUIRenderMesh@@@Z 0000000031512840 f i LoaderSKIN.obj
 0001:00011880       ?CryLog@@YAXPEBDZZ         0000000031512880 f i LoaderSKIN.obj
 0001:000118e0       ?FixRanges@SMeshSubset@@QEAAXPEAG@Z 00000000315128e0 f i LoaderSKIN.obj
 0001:00011930       ?FindExtension@CryStringUtils@@YAPEBDPEBD@Z 0000000031512930 f i LoaderSKIN.obj
 0001:00011980       ?AddRef@?$_i_reference_target@H@@UEAAXXZ 0000000031512980 f i LoaderSKIN.obj
 0001:00011980       ?AddRef@CFacialEffectorsLibrary@@UEAAXXZ 0000000031512980 f i FaceEffectorLibrary.obj
 0001:00011980       ?AddRef@CPlaceholderCharacter@@UEAAXXZ 0000000031512980 f i PlaceholderCharacter.obj
 0001:00011990       ?Release@?$_i_reference_target@H@@UEAAXXZ 0000000031512990 f i LoaderSKIN.obj
 0001:000119c0       ??$move_init@UBoneWeights8@@@NArray@@YAXPEAUBoneWeights8@@0_K@Z 00000000315129c0 f i LoaderSKIN.obj
 0001:00011a20       ??$move_init@UExtSkinVertex@@@NArray@@YAXPEAUExtSkinVertex@@0_K@Z 0000000031512a20 f i LoaderSKIN.obj
 0001:00011a20       ??$move_init@UVirtualExample3D@@@NArray@@YAXPEAUVirtualExample3D@@0_K@Z 0000000031512a20 f i ParametricSampler.obj
 0001:00011a80       ?SetIMaterial@CSkin@@QEAAXPEAUIMaterial@@@Z 0000000031512a80 f i LoaderSKIN.obj
 0001:00011ad0       ?IsOrthonormalRH@?$Matrix34_tpl@M@@QEBAHM@Z 0000000031512ad0 f i LoaderSKIN.obj
 0001:00011ce0       ?_AllocData@?$CryStackStringT@D$0CAA@@@QEAAX_K@Z 0000000031512ce0 f i LoaderSKIN.obj
 0001:00011d60       ?_Concatenate@?$CryStackStringT@D$0CAA@@@QEAAXPEBD_K01@Z 0000000031512d60 f i LoaderSKIN.obj
 0001:00011e00       ??$move_init@U?$Quat_tpl@M@@@NArray@@YAXPEAU?$Quat_tpl@M@@0_K@Z 0000000031512e00 f i LoaderSKIN.obj
 0001:00011f50       ??0CMemStatContextFormat@@QEAA@W4Type@EMemStatContextTypes@@IPEBDZZ 0000000031512f50 f i LoaderSKIN.obj
 0001:00012280       ?resize_raw@?$SmallDynStorage@UExtSkinVertex@@HUStandardAlloc@NAlloc@@@NArray@@QEAAXHH_N@Z 0000000031513280 f i LoaderSKIN.obj
 0001:00012400       ?allocate@?$_STLP_alloc_proxy@PEAPEAXPEAXV?$allocator@PEAX@stlpmtx_std@@@priv@stlpmtx_std@@QEAAPEAPEAX_KAEA_K@Z 0000000031513400 f i LoaderSKIN.obj
 0001:00012400       ?allocate@?$_STLP_alloc_proxy@PEAV?$_smart_ptr@VCFacialEffector@@@@V1@V?$allocator@V?$_smart_ptr@VCFacialEffector@@@@@stlpmtx_std@@@priv@stlpmtx_std@@QEAAPEAV?$_smart_ptr@VCFacialEffector@@@@_KAEA_K@Z 0000000031513400 f i FaceEffectorLibrary.obj
 0001:00012470       ?GetCRC32Lowercase@Crc32Gen@@QEBAIPEBD@Z 0000000031513470 f i LoaderSKIN.obj
 0001:000124e0       ?_M_compute_next_size@?$_Impl_vector@U?$Vec3_tpl@M@@V?$allocator@U?$Vec3_tpl@M@@@stlpmtx_std@@@priv@stlpmtx_std@@AEAA_K_K@Z 00000000315134e0 f i LoaderSKIN.obj
 0001:00012570       ??0?$CryStackStringT@D$0CAA@@@QEAA@PEBD@Z 0000000031513570 f i LoaderSKIN.obj
 0001:00012600       ?_ConcatenateInPlace@?$CryStackStringT@D$0CAA@@@QEAAXPEBD_K@Z 0000000031513600 f i LoaderSKIN.obj
 0001:000126a0       ?_Assign@?$CryStackStringT@D$0CAA@@@QEAAXPEBD_K@Z 00000000315136a0 f i LoaderSKIN.obj
 0001:00012740       ?resize_raw@?$SmallDynStorage@U?$Vec3_tpl@M@@HUStandardAlloc@NAlloc@@@NArray@@QEAAXHH_N@Z 0000000031513740 f i LoaderSKIN.obj
 0001:000128f0       ?resize_raw@?$SmallDynStorage@U?$Quat_tpl@M@@HUStandardAlloc@NAlloc@@@NArray@@QEAAXHH_N@Z 00000000315138f0 f i LoaderSKIN.obj
 0001:00012a60       ?_Concatenate@?$CryStringT@D@@IEAAXPEBD_K01@Z 0000000031513a60 f i LoaderSKIN.obj
 0001:00012b10       ?set_size@?$SmallDynStorage@UMorphTargetVertex@@HUStandardAlloc@NAlloc@@@NArray@@QEAAXH@Z 0000000031513b10 f i LoaderSKIN.obj
 0001:00012bc0       ?resize_raw@?$SmallDynStorage@UBoneIndices8@@HUStandardAlloc@NAlloc@@@NArray@@QEAAXHH_N@Z 0000000031513bc0 f i LoaderSKIN.obj
 0001:00012d50       ?resize_raw@?$SmallDynStorage@UBoneWeights8@@HUStandardAlloc@NAlloc@@@NArray@@QEAAXHH_N@Z 0000000031513d50 f i LoaderSKIN.obj
 0001:00012ec0       ?expand_raw@?$DynArray@UExtSkinVertex@@HU?$SmallDynStorage@UExtSkinVertex@@HUStandardAlloc@NAlloc@@@NArray@@@@IEAAPEAUExtSkinVertex@@PEAU2@H@Z 0000000031513ec0 f i LoaderSKIN.obj
 0001:00012f80       ?resize_raw@?$SmallDynStorage@UMorphTargetVertex@@HUStandardAlloc@NAlloc@@@NArray@@QEAAXHH_N@Z 0000000031513f80 f i LoaderSKIN.obj
 0001:00013130       ??$move_init@V?$_smart_ptr@UCMorphTarget@@@@@NArray@@YAXPEAV?$_smart_ptr@UCMorphTarget@@@@0_K@Z 0000000031514130 f i LoaderSKIN.obj
 0001:00013130       ??$move_init@V?$_smart_ptr@VIController@@@@@NArray@@YAXPEAV?$_smart_ptr@VIController@@@@0_K@Z 0000000031514130 f i DirectionalBlender.obj
 0001:000131a0       ?_M_insert_overflow@?$_Impl_vector@U?$Vec3_tpl@M@@V?$allocator@U?$Vec3_tpl@M@@@stlpmtx_std@@@priv@stlpmtx_std@@AEAAXPEAU?$Vec3_tpl@M@@AEBU4@AEBU__true_type@3@_K_N@Z 00000000315141a0 f i LoaderSKIN.obj
 0001:000132e0       ??$__uninitialized_fill_n@PEAU?$Vec3_tpl@M@@_KU1@@priv@stlpmtx_std@@YAPEAU?$Vec3_tpl@M@@PEAU2@_KAEBU2@@Z 00000000315142e0 f i LoaderSKIN.obj
 0001:00013340       ??$__median@U?$pair@V?$CryStringT@D@@PEAUIFacialAnimChannel@@@stlpmtx_std@@VFirstLess@?$VectorMap@V?$CryStringT@D@@PEAUIFacialAnimChannel@@U?$less@V?$CryStringT@D@@@stlpmtx_std@@V?$allocator@U?$pair@V?$CryStringT@D@@PEAUIFacialAnimChannel@@@stlpmtx_std@@@4@@@@priv@stlpmtx_std@@YAAEBU?$pair@V?$CryStringT@D@@PEAUIFacialAnimChannel@@@1@AEBU21@00VFirstLess@?$VectorMap@V?$CryStringT@D@@PEAUIFacialAnimChannel@@U?$less@V?$CryStringT@D@@@stlpmtx_std@@V?$allocator@U?$pair@V?$CryStringT@D@@PEAUIFacialAnimChannel@@@stlpmtx_std@@@4@@@@Z 0000000031514340 f i FaceAnimation.obj
 0001:00013340       ??$__median@U?$pair@V?$CryStringT@D@@H@stlpmtx_std@@VFirstLess@?$VectorMap@V?$CryStringT@D@@HU?$less@V?$CryStringT@D@@@stlpmtx_std@@V?$allocator@U?$pair@V?$CryStringT@D@@H@stlpmtx_std@@@3@@@@priv@stlpmtx_std@@YAAEBU?$pair@V?$CryStringT@D@@H@1@AEBU21@00VFirstLess@?$VectorMap@V?$CryStringT@D@@HU?$less@V?$CryStringT@D@@@stlpmtx_std@@V?$allocator@U?$pair@V?$CryStringT@D@@H@stlpmtx_std@@@3@@@@Z 0000000031514340 f i LoaderSKIN.obj
 0001:00013440       ??$__unguarded_linear_insert@PEAU?$pair@V?$CryStringT@D@@H@stlpmtx_std@@U12@VFirstLess@?$VectorMap@V?$CryStringT@D@@HU?$less@V?$CryStringT@D@@@stlpmtx_std@@V?$allocator@U?$pair@V?$CryStringT@D@@H@stlpmtx_std@@@3@@@@priv@stlpmtx_std@@YAXPEAU?$pair@V?$CryStringT@D@@H@1@U21@VFirstLess@?$VectorMap@V?$CryStringT@D@@HU?$less@V?$CryStringT@D@@@stlpmtx_std@@V?$allocator@U?$pair@V?$CryStringT@D@@H@stlpmtx_std@@@3@@@@Z 0000000031514440 f i LoaderSKIN.obj
 0001:00013520       ??$swap@U?$pair@V?$CryStringT@D@@H@stlpmtx_std@@@stlpmtx_std@@YAXAEAU?$pair@V?$CryStringT@D@@H@0@0@Z 0000000031514520 f i LoaderSKIN.obj
 0001:00013600       ??$__push_heap@PEAU?$pair@V?$CryStringT@D@@H@stlpmtx_std@@_JU12@VFirstLess@?$VectorMap@V?$CryStringT@D@@HU?$less@V?$CryStringT@D@@@stlpmtx_std@@V?$allocator@U?$pair@V?$CryStringT@D@@H@stlpmtx_std@@@3@@@@stlpmtx_std@@YAXPEAU?$pair@V?$CryStringT@D@@H@0@_J1U10@VFirstLess@?$VectorMap@V?$CryStringT@D@@HU?$less@V?$CryStringT@D@@@stlpmtx_std@@V?$allocator@U?$pair@V?$CryStringT@D@@H@stlpmtx_std@@@3@@@@Z 0000000031514600 f i LoaderSKIN.obj
 0001:00013720       ??0?$CryStringT@D@@QEAA@PEBD@Z 0000000031514720 f i LoaderSKIN.obj
 0001:000137a0       ??0?$CryStringT@D@@QEAA@PEBD_K@Z 00000000315147a0 f i LoaderSKIN.obj
 0001:00013830       ?_ConcatenateInPlace@?$CryStringT@D@@IEAAXPEBD_K@Z 0000000031514830 f i LoaderSKIN.obj
 0001:000138f0       ?expand_raw@?$DynArray@U?$Vec3_tpl@M@@HU?$SmallDynStorage@U?$Vec3_tpl@M@@HUStandardAlloc@NAlloc@@@NArray@@@@IEAAPEAU?$Vec3_tpl@M@@PEAU2@H@Z 00000000315148f0 f i LoaderSKIN.obj
 0001:000139b0       ?pop_back@?$DynArray@V?$_smart_ptr@VIController@@@@HU?$SmallDynStorage@V?$_smart_ptr@VIController@@@@HUStandardAlloc@NAlloc@@@NArray@@@@QEAAXH@Z 00000000315149b0 f i LoaderDBA.obj
 0001:000139b0       ?pop_back@?$DynArray@V?$_smart_ptr@UCMorphTarget@@@@HU?$SmallDynStorage@V?$_smart_ptr@UCMorphTarget@@@@HUStandardAlloc@NAlloc@@@NArray@@@@QEAAXH@Z 00000000315149b0 f i LoaderSKIN.obj
 0001:00013a30       ?erase@?$DynArray@U?$Vec3_tpl@M@@HU?$SmallDynStorage@U?$Vec3_tpl@M@@HUStandardAlloc@NAlloc@@@NArray@@@@QEAAPEAU?$Vec3_tpl@M@@PEAU2@0@Z 0000000031514a30 f i LoaderSKIN.obj
 0001:00013ad0       ?erase@?$DynArray@U?$Quat_tpl@M@@HU?$SmallDynStorage@U?$Quat_tpl@M@@HUStandardAlloc@NAlloc@@@NArray@@@@QEAAPEAU?$Quat_tpl@M@@PEAU2@0@Z 0000000031514ad0 f i LoaderSKIN.obj
 0001:00013c10       ?erase@?$DynArray@UBoneIndices8@@HU?$SmallDynStorage@UBoneIndices8@@HUStandardAlloc@NAlloc@@@NArray@@@@QEAAPEAUBoneIndices8@@PEAU2@0@Z 0000000031514c10 f i LoaderSKIN.obj
 0001:00013c70       ?erase@?$DynArray@UBoneWeights8@@HU?$SmallDynStorage@UBoneWeights8@@HUStandardAlloc@NAlloc@@@NArray@@@@QEAAPEAUBoneWeights8@@PEAU2@0@Z 0000000031514c70 f i LoaderSKIN.obj
 0001:00013d10       ?resize_raw@?$SmallDynStorage@V?$_smart_ptr@UCMorphTarget@@@@HUStandardAlloc@NAlloc@@@NArray@@QEAAXHH_N@Z 0000000031514d10 f i LoaderSKIN.obj
 0001:00013e80       ?append_raw@?$DynArray@UBoneIndices8@@HU?$SmallDynStorage@UBoneIndices8@@HUStandardAlloc@NAlloc@@@NArray@@@@QEAA?AU?$Array@UBoneIndices8@@HU?$ArrayStorage@UBoneIndices8@@H@NArray@@@@H@Z 0000000031514e80 f i LoaderSKIN.obj
 0001:00013f40       ?append_raw@?$DynArray@UBoneWeights8@@HU?$SmallDynStorage@UBoneWeights8@@HUStandardAlloc@NAlloc@@@NArray@@@@QEAA?AU?$Array@UBoneWeights8@@HU?$ArrayStorage@UBoneWeights8@@H@NArray@@@@H@Z 0000000031514f40 f i LoaderSKIN.obj
 0001:00014000       ?_M_insert_overflow@?$_Impl_vector@PEAXV?$allocator@PEAX@stlpmtx_std@@@priv@stlpmtx_std@@AEAAXPEAPEAXAEBQEAXAEBU__true_type@3@_K_N@Z 0000000031515000 f i LoaderSKIN.obj
 0001:00014170       ??4?$_Impl_vector@PEAXV?$allocator@PEAX@stlpmtx_std@@@priv@stlpmtx_std@@QEAAAEAV012@AEBV012@@Z 0000000031515170 f i LoaderSKIN.obj
 0001:000142b0       ?_M_fill_insert_aux@?$_Impl_vector@U?$Vec3_tpl@M@@V?$allocator@U?$Vec3_tpl@M@@@stlpmtx_std@@@priv@stlpmtx_std@@AEAAXPEAU?$Vec3_tpl@M@@_KAEBU4@AEBU__false_type@3@@Z 00000000315152b0 f i LoaderSKIN.obj
 0001:000144a0       ?_M_fill_insert_aux@?$_Impl_vector@PEAXV?$allocator@PEAX@stlpmtx_std@@@priv@stlpmtx_std@@AEAAXPEAPEAX_KAEBQEAXAEBU__false_type@3@@Z 00000000315154a0 f i LoaderSKIN.obj
 0001:00014640       ??$__adjust_heap@PEAU?$pair@V?$CryStringT@D@@H@stlpmtx_std@@_JU12@VFirstLess@?$VectorMap@V?$CryStringT@D@@HU?$less@V?$CryStringT@D@@@stlpmtx_std@@V?$allocator@U?$pair@V?$CryStringT@D@@H@stlpmtx_std@@@3@@@@stlpmtx_std@@YAXPEAU?$pair@V?$CryStringT@D@@H@0@_J1U10@VFirstLess@?$VectorMap@V?$CryStringT@D@@HU?$less@V?$CryStringT@D@@@stlpmtx_std@@V?$allocator@U?$pair@V?$CryStringT@D@@H@stlpmtx_std@@@3@@@@Z 0000000031515640 f i LoaderSKIN.obj
 0001:000147b0       ??$?HD$0CAA@@@YA?AV?$CryStackStringT@D$0CAA@@@AEBV0@PEBD@Z 00000000315157b0 f i LoaderSKIN.obj
 0001:00014830       ?append_raw@?$DynArray@U?$Quat_tpl@M@@HU?$SmallDynStorage@U?$Quat_tpl@M@@HUStandardAlloc@NAlloc@@@NArray@@@@QEAA?AU?$Array@U?$Quat_tpl@M@@HU?$ArrayStorage@U?$Quat_tpl@M@@H@NArray@@@@H@Z 0000000031515830 f i LoaderSKIN.obj
 0001:000148f0       ??1?$DynArray@UExtSkinVertex@@HU?$SmallDynStorage@UExtSkinVertex@@HUStandardAlloc@NAlloc@@@NArray@@@@QEAA@XZ 00000000315158f0 f i LoaderSKIN.obj
 0001:00014930       ??4?$DynArray@U?$Vec3_tpl@M@@HU?$SmallDynStorage@U?$Vec3_tpl@M@@HUStandardAlloc@NAlloc@@@NArray@@@@QEAAAEAU0@U?$Array@$$CBU?$Vec3_tpl@M@@HU?$ArrayStorage@$$CBU?$Vec3_tpl@M@@H@NArray@@@@@Z 0000000031515930 f i LoaderSKIN.obj
 0001:00014a70       ??4?$DynArray@U?$Quat_tpl@M@@HU?$SmallDynStorage@U?$Quat_tpl@M@@HUStandardAlloc@NAlloc@@@NArray@@@@QEAAAEAU0@U?$Array@$$CBU?$Quat_tpl@M@@HU?$ArrayStorage@$$CBU?$Quat_tpl@M@@H@NArray@@@@@Z 0000000031515a70 f i LoaderSKIN.obj
 0001:00014bc0       ??4?$DynArray@UBoneIndices8@@HU?$SmallDynStorage@UBoneIndices8@@HUStandardAlloc@NAlloc@@@NArray@@@@QEAAAEAU0@U?$Array@$$CBUBoneIndices8@@HU?$ArrayStorage@$$CBUBoneIndices8@@H@NArray@@@@@Z 0000000031515bc0 f i LoaderSKIN.obj
 0001:00014cd0       ??4?$DynArray@UBoneWeights8@@HU?$SmallDynStorage@UBoneWeights8@@HUStandardAlloc@NAlloc@@@NArray@@@@QEAAAEAU0@U?$Array@$$CBUBoneWeights8@@HU?$ArrayStorage@$$CBUBoneWeights8@@H@NArray@@@@@Z 0000000031515cd0 f i LoaderSKIN.obj
 0001:00014e50       ??4?$DynArray@V?$_smart_ptr@UCMorphTarget@@@@HU?$SmallDynStorage@V?$_smart_ptr@UCMorphTarget@@@@HUStandardAlloc@NAlloc@@@NArray@@@@QEAAAEAU0@U?$Array@$$CBV?$_smart_ptr@UCMorphTarget@@@@HU?$ArrayStorage@$$CBV?$_smart_ptr@UCMorphTarget@@@@H@NArray@@@@@Z 0000000031515e50 f i LoaderSKIN.obj
 0001:00014fc0       ?GetPath@PathUtil@@YA?AV?$CryStringT@D@@PEBD@Z 0000000031515fc0 f i LoaderSKIN.obj
 0001:000150f0       ??4?$DynArray@EHU?$SmallDynStorage@EHUStandardAlloc@NAlloc@@@NArray@@@@QEAAAEAU0@U?$Array@$$CBEHU?$ArrayStorage@$$CBEH@NArray@@@@@Z 00000000315160f0 f i LoaderSKIN.obj
 0001:00015270       ??$move_init@USJointInfo@CSkin@@@NArray@@YAXPEAUSJointInfo@CSkin@@0_K@Z 0000000031516270 f i LoaderSKIN.obj
 0001:00015350       ??$__unguarded_insertion_sort@PEAU?$pair@V?$CryStringT@D@@H@stlpmtx_std@@VFirstLess@?$VectorMap@V?$CryStringT@D@@HU?$less@V?$CryStringT@D@@@stlpmtx_std@@V?$allocator@U?$pair@V?$CryStringT@D@@H@stlpmtx_std@@@3@@@@priv@stlpmtx_std@@YAXPEAU?$pair@V?$CryStringT@D@@H@1@0VFirstLess@?$VectorMap@V?$CryStringT@D@@HU?$less@V?$CryStringT@D@@@stlpmtx_std@@V?$allocator@U?$pair@V?$CryStringT@D@@H@stlpmtx_std@@@3@@@@Z 0000000031516350 f i LoaderSKIN.obj
 0001:000153d0       ??$__pop_heap@PEAU?$pair@V?$CryStringT@D@@H@stlpmtx_std@@U12@VFirstLess@?$VectorMap@V?$CryStringT@D@@HU?$less@V?$CryStringT@D@@@stlpmtx_std@@V?$allocator@U?$pair@V?$CryStringT@D@@H@stlpmtx_std@@@3@@@_J@stlpmtx_std@@YAXPEAU?$pair@V?$CryStringT@D@@H@0@00U10@VFirstLess@?$VectorMap@V?$CryStringT@D@@HU?$less@V?$CryStringT@D@@@stlpmtx_std@@V?$allocator@U?$pair@V?$CryStringT@D@@H@stlpmtx_std@@@3@@@PEA_J@Z 00000000315163d0 f i LoaderSKIN.obj
 0001:00015490       ??$__make_heap@PEAU?$pair@V?$CryStringT@D@@H@stlpmtx_std@@VFirstLess@?$VectorMap@V?$CryStringT@D@@HU?$less@V?$CryStringT@D@@@stlpmtx_std@@V?$allocator@U?$pair@V?$CryStringT@D@@H@stlpmtx_std@@@3@@@U12@_J@stlpmtx_std@@YAXPEAU?$pair@V?$CryStringT@D@@H@0@0VFirstLess@?$VectorMap@V?$CryStringT@D@@HU?$less@V?$CryStringT@D@@@stlpmtx_std@@V?$allocator@U?$pair@V?$CryStringT@D@@H@stlpmtx_std@@@3@@@0PEA_J@Z 0000000031516490 f i LoaderSKIN.obj
 0001:000162c0       ??0?$DynArray@UExtSkinVertex@@HU?$SmallDynStorage@UExtSkinVertex@@HUStandardAlloc@NAlloc@@@NArray@@@@QEAA@XZ 00000000315172c0 f i LoaderSKIN.obj
 0001:00016320       ?pop_back@?$DynArray@USJointInfo@CSkin@@HU?$SmallDynStorage@USJointInfo@CSkin@@HUStandardAlloc@NAlloc@@@NArray@@@@QEAAXH@Z 0000000031517320 f i LoaderSKIN.obj
 0001:00016320       ?pop_back@?$DynArray@USCRCName@@HU?$SmallDynStorage@USCRCName@@HUStandardAlloc@NAlloc@@@NArray@@@@QEAAXH@Z 0000000031517320 f i GlobalAnimationHeaderLMG.obj
 0001:000163d0       ?append_raw@?$DynArray@V?$_smart_ptr@UCMorphTarget@@@@HU?$SmallDynStorage@V?$_smart_ptr@UCMorphTarget@@@@HUStandardAlloc@NAlloc@@@NArray@@@@QEAA?AU?$Array@V?$_smart_ptr@UCMorphTarget@@@@HU?$ArrayStorage@V?$_smart_ptr@UCMorphTarget@@@@H@NArray@@@@H@Z 00000000315173d0 f i LoaderSKIN.obj
 0001:00016490       ??0?$DynArray@UBoneIndices8@@HU?$SmallDynStorage@UBoneIndices8@@HUStandardAlloc@NAlloc@@@NArray@@@@QEAA@AEBU0@@Z 0000000031517490 f i LoaderSKIN.obj
 0001:00016550       ??0?$DynArray@UBoneWeights8@@HU?$SmallDynStorage@UBoneWeights8@@HUStandardAlloc@NAlloc@@@NArray@@@@QEAA@AEBU0@@Z 0000000031517550 f i LoaderSKIN.obj
 0001:00016630       ??0?$DynArray@EHU?$SmallDynStorage@EHUStandardAlloc@NAlloc@@@NArray@@@@QEAA@AEBU0@@Z 0000000031517630 f i LoaderSKIN.obj
 0001:000166f0       ?resize_raw@?$SmallDynStorage@USJointInfo@CSkin@@HUStandardAlloc@NAlloc@@@NArray@@QEAAXHH_N@Z 00000000315176f0 f i LoaderSKIN.obj
 0001:00016860       ??$__unguarded_partition@PEAU?$pair@V?$CryStringT@D@@H@stlpmtx_std@@U12@VFirstLess@?$VectorMap@V?$CryStringT@D@@HU?$less@V?$CryStringT@D@@@stlpmtx_std@@V?$allocator@U?$pair@V?$CryStringT@D@@H@stlpmtx_std@@@3@@@@priv@stlpmtx_std@@YAPEAU?$pair@V?$CryStringT@D@@H@1@PEAU21@0U21@VFirstLess@?$VectorMap@V?$CryStringT@D@@HU?$less@V?$CryStringT@D@@@stlpmtx_std@@V?$allocator@U?$pair@V?$CryStringT@D@@H@stlpmtx_std@@@3@@@@Z 0000000031517860 f i LoaderSKIN.obj
 0001:00016990       ??$copy_backward@PEAU?$pair@V?$CryStringT@D@@H@stlpmtx_std@@PEAU12@@stlpmtx_std@@YAPEAU?$pair@V?$CryStringT@D@@H@0@PEAU10@00@Z 0000000031517990 f i LoaderSKIN.obj
 0001:00016a00       ??0?$DynArray@U?$Vec3_tpl@M@@HU?$SmallDynStorage@U?$Vec3_tpl@M@@HUStandardAlloc@NAlloc@@@NArray@@@@QEAA@AEBU0@@Z 0000000031517a00 f i LoaderSKIN.obj
 0001:00016ad0       ??0?$DynArray@U?$Quat_tpl@M@@HU?$SmallDynStorage@U?$Quat_tpl@M@@HUStandardAlloc@NAlloc@@@NArray@@@@QEAA@AEBU0@@Z 0000000031517ad0 f i LoaderSKIN.obj
 0001:000176c0       ??1CMorphTarget@@UEAA@XZ   00000000315186c0 f i LoaderSKIN.obj
 0001:00017740       ??_GCMorphTarget@@UEAAPEAXI@Z 0000000031518740 f i LoaderSKIN.obj
 0001:00017740       ??_ECMorphTarget@@UEAAPEAXI@Z 0000000031518740 f i LoaderSKIN.obj
 0001:00017770       ??0?$DynArray@V?$_smart_ptr@UCMorphTarget@@@@HU?$SmallDynStorage@V?$_smart_ptr@UCMorphTarget@@@@HUStandardAlloc@NAlloc@@@NArray@@@@QEAA@AEBU0@@Z 0000000031518770 f i LoaderSKIN.obj
 0001:00017850       ??$__linear_insert@PEAU?$pair@V?$CryStringT@D@@H@stlpmtx_std@@U12@VFirstLess@?$VectorMap@V?$CryStringT@D@@HU?$less@V?$CryStringT@D@@@stlpmtx_std@@V?$allocator@U?$pair@V?$CryStringT@D@@H@stlpmtx_std@@@3@@@@priv@stlpmtx_std@@YAXPEAU?$pair@V?$CryStringT@D@@H@1@0U21@VFirstLess@?$VectorMap@V?$CryStringT@D@@HU?$less@V?$CryStringT@D@@@stlpmtx_std@@V?$allocator@U?$pair@V?$CryStringT@D@@H@stlpmtx_std@@@3@@@@Z 0000000031518850 f i LoaderSKIN.obj
 0001:00017940       ??$sort_heap@PEAU?$pair@V?$CryStringT@D@@H@stlpmtx_std@@VFirstLess@?$VectorMap@V?$CryStringT@D@@HU?$less@V?$CryStringT@D@@@stlpmtx_std@@V?$allocator@U?$pair@V?$CryStringT@D@@H@stlpmtx_std@@@3@@@@stlpmtx_std@@YAXPEAU?$pair@V?$CryStringT@D@@H@0@0VFirstLess@?$VectorMap@V?$CryStringT@D@@HU?$less@V?$CryStringT@D@@@stlpmtx_std@@V?$allocator@U?$pair@V?$CryStringT@D@@H@stlpmtx_std@@@3@@@@Z 0000000031518940 f i LoaderSKIN.obj
 0001:00017a00       ?init@?$DynArray@URChunk@@HU?$SmallDynStorage@URChunk@@HUStandardAlloc@NAlloc@@@NArray@@@@KAPEAURChunk@@U?$Array@URChunk@@HU?$ArrayStorage@URChunk@@H@NArray@@@@@Z 0000000031518a00 f i LoaderSKIN.obj
 0001:00017b20       ?append_raw@?$DynArray@USJointInfo@CSkin@@HU?$SmallDynStorage@USJointInfo@CSkin@@HUStandardAlloc@NAlloc@@@NArray@@@@QEAA?AU?$Array@USJointInfo@CSkin@@HU?$ArrayStorage@USJointInfo@CSkin@@H@NArray@@@@H@Z 0000000031518b20 f i LoaderSKIN.obj
 0001:00017be0       ??$__insertion_sort@PEAU?$pair@V?$CryStringT@D@@H@stlpmtx_std@@U12@VFirstLess@?$VectorMap@V?$CryStringT@D@@HU?$less@V?$CryStringT@D@@@stlpmtx_std@@V?$allocator@U?$pair@V?$CryStringT@D@@H@stlpmtx_std@@@3@@@@priv@stlpmtx_std@@YAXPEAU?$pair@V?$CryStringT@D@@H@1@00VFirstLess@?$VectorMap@V?$CryStringT@D@@HU?$less@V?$CryStringT@D@@@stlpmtx_std@@V?$allocator@U?$pair@V?$CryStringT@D@@H@stlpmtx_std@@@3@@@@Z 0000000031518be0 f i LoaderSKIN.obj
 0001:00017c80       ??$__partial_sort@PEAU?$pair@V?$CryStringT@D@@H@stlpmtx_std@@U12@VFirstLess@?$VectorMap@V?$CryStringT@D@@HU?$less@V?$CryStringT@D@@@stlpmtx_std@@V?$allocator@U?$pair@V?$CryStringT@D@@H@stlpmtx_std@@@3@@@@priv@stlpmtx_std@@YAXPEAU?$pair@V?$CryStringT@D@@H@1@000VFirstLess@?$VectorMap@V?$CryStringT@D@@HU?$less@V?$CryStringT@D@@@stlpmtx_std@@V?$allocator@U?$pair@V?$CryStringT@D@@H@stlpmtx_std@@@3@@@@Z 0000000031518c80 f i LoaderSKIN.obj
 0001:00017d70       ?destroy@?$DynArray@URChunk@@HU?$SmallDynStorage@URChunk@@HUStandardAlloc@NAlloc@@@NArray@@@@KAXU?$Array@URChunk@@HU?$ArrayStorage@URChunk@@H@NArray@@@@@Z 0000000031518d70 f i LoaderSKIN.obj
 0001:00017e60       ?erase@?$DynArray@URChunk@@HU?$SmallDynStorage@URChunk@@HUStandardAlloc@NAlloc@@@NArray@@@@QEAAPEAURChunk@@PEAU2@0@Z 0000000031518e60 f i LoaderSKIN.obj
 0001:00017f50       ??$move_init@URChunk@@@NArray@@YAXPEAURChunk@@0_K@Z 0000000031518f50 f i LoaderSKIN.obj
 0001:00018070       ?resize@?$DynArray@USJointInfo@CSkin@@HU?$SmallDynStorage@USJointInfo@CSkin@@HUStandardAlloc@NAlloc@@@NArray@@@@QEAAXH@Z 0000000031519070 f i LoaderSKIN.obj
 0001:000180e0       ?resize_raw@?$SmallDynStorage@URChunk@@HUStandardAlloc@NAlloc@@@NArray@@QEAAXHH_N@Z 00000000315190e0 f i LoaderSKIN.obj
 0001:00018250       ??$__introsort_loop@PEAU?$pair@V?$CryStringT@D@@H@stlpmtx_std@@U12@_JVFirstLess@?$VectorMap@V?$CryStringT@D@@HU?$less@V?$CryStringT@D@@@stlpmtx_std@@V?$allocator@U?$pair@V?$CryStringT@D@@H@stlpmtx_std@@@3@@@@priv@stlpmtx_std@@YAXPEAU?$pair@V?$CryStringT@D@@H@1@00_JVFirstLess@?$VectorMap@V?$CryStringT@D@@HU?$less@V?$CryStringT@D@@@stlpmtx_std@@V?$allocator@U?$pair@V?$CryStringT@D@@H@stlpmtx_std@@@3@@@@Z 0000000031519250 f i LoaderSKIN.obj
 0001:00018650       ??4?$DynArray@URChunk@@HU?$SmallDynStorage@URChunk@@HUStandardAlloc@NAlloc@@@NArray@@@@QEAAAEAU0@U?$Array@$$CBURChunk@@HU?$ArrayStorage@$$CBURChunk@@H@NArray@@@@@Z 0000000031519650 f i LoaderSKIN.obj
 0001:000187e0       ??$sort@PEAU?$pair@V?$CryStringT@D@@H@stlpmtx_std@@VFirstLess@?$VectorMap@V?$CryStringT@D@@HU?$less@V?$CryStringT@D@@@stlpmtx_std@@V?$allocator@U?$pair@V?$CryStringT@D@@H@stlpmtx_std@@@3@@@@stlpmtx_std@@YAXPEAU?$pair@V?$CryStringT@D@@H@0@0VFirstLess@?$VectorMap@V?$CryStringT@D@@HU?$less@V?$CryStringT@D@@@stlpmtx_std@@V?$allocator@U?$pair@V?$CryStringT@D@@H@stlpmtx_std@@@3@@@@Z 00000000315197e0 f i LoaderSKIN.obj
 0001:00018890       ??0CModelMesh@@QEAA@XZ     0000000031519890 f i LoaderSKIN.obj
 0001:00018a80       ??1CModelMesh@@QEAA@XZ     0000000031519a80 f i LoaderSKIN.obj
 0001:00018ba0       ?append_raw@?$DynArray@URChunk@@HU?$SmallDynStorage@URChunk@@HUStandardAlloc@NAlloc@@@NArray@@@@QEAA?AU?$Array@URChunk@@HU?$ArrayStorage@URChunk@@H@NArray@@@@H@Z 0000000031519ba0 f i LoaderSKIN.obj
 0001:000194d0       ??4CModelMesh@@QEAAAEAV0@AEBV0@@Z 000000003151a4d0 f i LoaderSKIN.obj
 0001:00019600       ??0?$DynArray@URChunk@@HU?$SmallDynStorage@URChunk@@HUStandardAlloc@NAlloc@@@NArray@@@@QEAA@AEBU0@@Z 000000003151a600 f i LoaderSKIN.obj
 0001:000196f0       ?resize@?$DynArray@URChunk@@HU?$SmallDynStorage@URChunk@@HUStandardAlloc@NAlloc@@@NArray@@@@QEAAXH@Z 000000003151a6f0 f i LoaderSKIN.obj
 0001:00019790       ?pop_back@?$DynArray@VCModelMesh@@HU?$SmallDynStorage@VCModelMesh@@HUStandardAlloc@NAlloc@@@NArray@@@@QEAAXH@Z 000000003151a790 f i LoaderSKIN.obj
 0001:00019810       ?erase@?$DynArray@VCModelMesh@@HU?$SmallDynStorage@VCModelMesh@@HUStandardAlloc@NAlloc@@@NArray@@@@QEAAPEAVCModelMesh@@PEAV2@0@Z 000000003151a810 f i LoaderSKIN.obj
 0001:000198b0       ?init@?$DynArray@VCModelMesh@@HU?$SmallDynStorage@VCModelMesh@@HUStandardAlloc@NAlloc@@@NArray@@@@KAPEAVCModelMesh@@U?$Array@VCModelMesh@@HU?$ArrayStorage@VCModelMesh@@H@NArray@@@@AEBV2@@Z 000000003151a8b0 f i LoaderSKIN.obj
 0001:00019970       ??$move_init@VCModelMesh@@@NArray@@YAXPEAVCModelMesh@@0_K@Z 000000003151a970 f i LoaderSKIN.obj
 0001:00019a40       ?resize_raw@?$SmallDynStorage@VCModelMesh@@HUStandardAlloc@NAlloc@@@NArray@@QEAAXHH_N@Z 000000003151aa40 f i LoaderSKIN.obj
 0001:00019bd0       ?expand_raw@?$DynArray@VCModelMesh@@HU?$SmallDynStorage@VCModelMesh@@HUStandardAlloc@NAlloc@@@NArray@@@@IEAAPEAVCModelMesh@@PEAV2@H@Z 000000003151abd0 f i LoaderSKIN.obj
 0001:00019c90       ?resize@?$DynArray@VCModelMesh@@HU?$SmallDynStorage@VCModelMesh@@HUStandardAlloc@NAlloc@@@NArray@@@@QEAAXHAEBVCModelMesh@@@Z 000000003151ac90 f i LoaderSKIN.obj
 0001:00019d10       ?LoadNewSKIN@CryCHRLoader@@QEAAPEAVCSkin@@PEBDI@Z 000000003151ad10 f   LoaderSKIN.obj
 0001:0001bb80       ?DrawLabelEx@IRenderer@@QEAAXU?$Vec3_tpl@M@@MPEBM_N2PEBDZZ 000000003151cb80 f i ModelMesh_DebugPC.obj
 0001:0001bc50       ?erase@?$_Impl_vector@U?$Color_tpl@E@@V?$allocator@U?$Color_tpl@E@@@stlpmtx_std@@@priv@stlpmtx_std@@QEAAPEAU?$Color_tpl@E@@PEAU4@0@Z 000000003151cc50 f i ModelMesh_DebugPC.obj
 0001:0001bcf0       ?_M_insert_overflow_aux@?$_Impl_vector@U?$Color_tpl@E@@V?$allocator@U?$Color_tpl@E@@@stlpmtx_std@@@priv@stlpmtx_std@@AEAAXPEAU?$Color_tpl@E@@AEBU4@AEBU__false_type@3@_K_N@Z 000000003151ccf0 f i ModelMesh_DebugPC.obj
 0001:0001be90       ?_M_fill_insert_aux@?$_Impl_vector@U?$Color_tpl@E@@V?$allocator@U?$Color_tpl@E@@@stlpmtx_std@@@priv@stlpmtx_std@@AEAAXPEAU?$Color_tpl@E@@_KAEBU4@AEBU__false_type@3@@Z 000000003151ce90 f i ModelMesh_DebugPC.obj
 0001:0001c090       ?DrawDebugInfo@CModelMesh@@QEAAXPEAVCCharInstance@@HAEBU?$Matrix34_tpl@M@@HAEAPEBUIMaterial@@PEAVCRenderObject@@AEBUSRendParams@@@Z 000000003151d090 f   ModelMesh_DebugPC.obj
 0001:0001ce20       ?DrawWireframeStatic@CModelMesh@@QEAAXAEBU?$Matrix34_tpl@M@@PEAUIRenderMesh@@I@Z 000000003151de20 f   ModelMesh_DebugPC.obj
 0001:0001d6e0       ?SoftwareSkinningDQ@CModelMesh@@QEAAXPEAUIRenderMesh@@PEAVCCharInstance@@PEAVCAttachmentSKIN@@U?$Matrix34_tpl@M@@EEEEPEAU?$DualQuat_tpl@M@@@Z 000000003151e6e0 f   ModelMesh_DebugPC.obj
 0001:00020d10       ??_EISkin@@UEAAPEAXI@Z     0000000031521d10 f i ModelSkin.obj
 0001:00020d10       ??_EIFacialSentence@@UEAAPEAXI@Z 0000000031521d10 f i LipSync.obj
 0001:00020d10       ??_GIFacialSentence@@UEAAPEAXI@Z 0000000031521d10 f i LipSync.obj
 0001:00020d10       ??_GISkin@@UEAAPEAXI@Z     0000000031521d10 f i ModelSkin.obj
 0001:00020d40       ?GetTextureMemoryUsage@CSkin@@UEBAIPEAVICrySizer@@@Z 0000000031521d40 f   ModelSkin.obj
 0001:00020df0       ?GetMeshMemoryUsage@CSkin@@UEBAIPEAVICrySizer@@@Z 0000000031521df0 f   ModelSkin.obj
 0001:00020e40       ?GetIRenderMesh@CSkin@@UEAAPEAUIRenderMesh@@H@Z 0000000031521e40 f   ModelSkin.obj
 0001:00020e40       ?GetIRenderMesh@CSkin@@UEBAPEBUIRenderMesh@@H@Z 0000000031521e40 f   ModelSkin.obj
 0001:00020e60       ?resize_raw@?$SmallDynStorage@PEAVCAttachmentSKIN@@HUStandardAlloc@NAlloc@@@NArray@@QEAAXHH_N@Z 0000000031521e60 f i ModelSkin.obj
 0001:00020ff0       ?GetAttachmentTriangle@CSkin@@UEAA?AUClosestTri@@AEBU?$Vec3_tpl@M@@@Z 0000000031521ff0 f   ModelSkin.obj
 0001:00021060       ?SizeOfModelData@CSkin@@QEBAIXZ 0000000031522060 f   ModelSkin.obj
 0001:00021200       ??$AddObject@VCModelMesh@@HU?$SmallDynStorage@VCModelMesh@@HUStandardAlloc@NAlloc@@@NArray@@@ICrySizer@@QEAAXAEBU?$DynArray@VCModelMesh@@HU?$SmallDynStorage@VCModelMesh@@HUStandardAlloc@NAlloc@@@NArray@@@@@Z 0000000031522200 f i ModelSkin.obj
 0001:00021360       ?append_raw@?$DynArray@PEAVCAttachmentSKIN@@HU?$SmallDynStorage@PEAVCAttachmentSKIN@@HUStandardAlloc@NAlloc@@@NArray@@@@QEAA?AU?$Array@PEAVCAttachmentSKIN@@HU?$ArrayStorage@PEAVCAttachmentSKIN@@H@NArray@@@@H@Z 0000000031522360 f i ModelSkin.obj
 0001:00021420       ?destroy@?$DynArray@USCRCName@@HU?$SmallDynStorage@USCRCName@@HUStandardAlloc@NAlloc@@@NArray@@@@IEAAXXZ 0000000031522420 f i CharacterManager.obj
 0001:00021420       ?destroy@?$DynArray@USJointInfo@CSkin@@HU?$SmallDynStorage@USJointInfo@CSkin@@HUStandardAlloc@NAlloc@@@NArray@@@@IEAAXXZ 0000000031522420 f i ModelSkin.obj
 0001:000214a0       ?UnregisterInstance@CSkin@@QEAAXPEAVCAttachmentSKIN@@@Z 00000000315224a0 f   ModelSkin.obj
 0001:000214f0       ??$push_back_unique@U?$DynArray@PEAVCAttachmentSKIN@@HU?$SmallDynStorage@PEAVCAttachmentSKIN@@HUStandardAlloc@NAlloc@@@NArray@@@@PEAVCAttachmentSKIN@@@stl@@YA_NAEAU?$DynArray@PEAVCAttachmentSKIN@@HU?$SmallDynStorage@PEAVCAttachmentSKIN@@HUStandardAlloc@NAlloc@@@NArray@@@@AEBQEAVCAttachmentSKIN@@@Z 00000000315224f0 f i ModelSkin.obj
 0001:00021590       ?RegisterInstance@CSkin@@QEAAXPEAVCAttachmentSKIN@@@Z 0000000031522590 f   ModelSkin.obj
 0001:00021610       ??1?$DynArray@VCModelMesh@@HU?$SmallDynStorage@VCModelMesh@@HUStandardAlloc@NAlloc@@@NArray@@@@QEAA@XZ 0000000031522610 f i ModelSkin.obj
 0001:00021690       ??0CSkin@@QEAA@AEBV?$CryStringT@D@@@Z 0000000031522690 f   ModelSkin.obj
 0001:000218b0       ?AddRef@CSkin@@UEAAXXZ     00000000315228b0 f i ModelSkin.obj
 0001:000218c0       ?DecRef@CSkin@@UEAAXXZ     00000000315228c0 f i ModelSkin.obj
 0001:000218d0       ?Release@CSkin@@UEAAXXZ    00000000315228d0 f i ModelSkin.obj
 0001:00021900       ?GetModelFilePath@CSkin@@UEBAPEBDXZ 0000000031522900 f i ModelSkin.obj
 0001:00021900       ?GetFacialModel@CFacialInstance@@UEAAPEAUIFacialModel@@XZ 0000000031522900 f i FacialInstance.obj
 0001:00021910       ?GetIMaterial@CSkin@@UEBAPEAUIMaterial@@XZ 0000000031522910 f i ModelSkin.obj
 0001:00021920       ?GetNumInstances@CSkin@@UEBAIXZ 0000000031522920 f i ModelSkin.obj
 0001:00021930       ?GetNumLODs@CSkin@@UEBAIXZ 0000000031522930 f i ModelSkin.obj
 0001:00021940       ?GetNumMorphTargets@CSkin@@UEBAIXZ 0000000031522940 f i ModelSkin.obj
 0001:00021960       ?GetMorphTargetName@CSkin@@UEBAPEBDI@Z 0000000031522960 f i ModelSkin.obj
 0001:000219a0       ??1CSkin@@UEAA@XZ          00000000315229a0 f   ModelSkin.obj
 0001:00021b00       ??_ECSkin@@UEAAPEAXI@Z     0000000031522b00 f i ModelSkin.obj
 0001:00021b00       ??_GCSkin@@UEAAPEAXI@Z     0000000031522b00 f i ModelSkin.obj
 0001:00021b30       ?CryWarning@@YAXW4EValidatorModule@@W4EValidatorSeverity@@PEBDZZ 0000000031522b30 f i ParametricSampler.obj
 0001:00021ba0       ?DrawLabel@IRenderer@@QEAAXU?$Vec3_tpl@M@@MPEBDZZ 0000000031522ba0 f i ParametricSampler.obj
 0001:00021c10       ?InitRenderingFlags@SRenderingPassInfo@@AEAAXI@Z 0000000031522c10 f i ParametricSampler.obj
 0001:00022120       ?WeightTetrahedron@SParametricSamplerInternal@@QEAA?AUBC4@@AEBU?$Vec3_tpl@M@@0000@Z 0000000031523120 f   ParametricSampler.obj
 0001:00022590       ?WeightPyramid@SParametricSamplerInternal@@QEAA?AUBC5@@AEBU?$Vec3_tpl@M@@00000@Z 0000000031523590 f   ParametricSampler.obj
 0001:00022790       ?CreateGeneralPassRenderingInfo@SRenderingPassInfo@@SA?AU1@AEBVCCamera@@I@Z 0000000031523790 f i ParametricSampler.obj
 0001:000229e0       ?UpdateWeights@@YAXMIPEIAMAEBUGlobalAnimationHeaderLMG@@@Z 00000000315239e0 f   ParametricSampler.obj
 0001:00022ac0       ?GetWeights1D@SParametricSamplerInternal@@QEAAXMAEBUGlobalAnimationHeaderLMG@@QEAMI@Z 0000000031523ac0 f   ParametricSampler.obj
 0001:00022cf0       ?GetCRC32@Crc32Gen@@QEBAIPEBD@Z 0000000031523cf0 f i ParametricSampler.obj
 0001:00022d50       ?GetControllerByJointCRC32@GlobalAnimationHeaderCAF@@QEBAPEAVIController@@I@Z 0000000031523d50 f i ParametricSampler.obj
 0001:00022df0       ?set_size@?$SmallDynStorage@U?$Vec3_tpl@M@@HUStandardAlloc@NAlloc@@@NArray@@QEAAXH@Z 0000000031523df0 f i LoaderSKIN.obj
 0001:00022df0       ?set_size@?$SmallDynStorage@UVirtualExample1D@@HUStandardAlloc@NAlloc@@@NArray@@QEAAXH@Z 0000000031523df0 f i ParametricSampler.obj
 0001:00022df0       ?set_size@?$SmallDynStorage@UNodeDesc@@HUStandardAlloc@NAlloc@@@NArray@@QEAAXH@Z 0000000031523df0 f i LoaderCGA.obj
 0001:00022df0       ?set_size@?$SmallDynStorage@UBSBlendable@@HUStandardAlloc@NAlloc@@@NArray@@QEAAXH@Z 0000000031523df0 f i CharacterManager.obj
 0001:00022ea0       ?resize_raw@?$SmallDynStorage@UVirtualExample1D@@HUStandardAlloc@NAlloc@@@NArray@@QEAAXHH_N@Z 0000000031523ea0 f i ParametricSampler.obj
 0001:00023050       ?resize_raw@?$SmallDynStorage@UVirtualExample2D@@HUStandardAlloc@NAlloc@@@NArray@@QEAAXHH_N@Z 0000000031524050 f i ParametricSampler.obj
 0001:00023210       ?resize_raw@?$SmallDynStorage@UVirtualExample3D@@HUStandardAlloc@NAlloc@@@NArray@@QEAAXHH_N@Z 0000000031524210 f i ParametricSampler.obj
 0001:00023390       ?WeightPrism@SParametricSamplerInternal@@QEAA?AUBC6@@AEBU?$Vec3_tpl@M@@000000@Z 0000000031524390 f   ParametricSampler.obj
 0001:00023870       ?GetConvex8@SParametricSamplerInternal@@QEAA?AUBC8@@IAEBU?$Vec3_tpl@M@@AEBUGlobalAnimationHeaderLMG@@QEAMPEAEPEAU3@U?$Diag33_tpl@M@@U3@@Z 0000000031524870 f   ParametricSampler.obj
 0001:000257a0       ?expand_raw@?$DynArray@UVirtualExample1D@@HU?$SmallDynStorage@UVirtualExample1D@@HUStandardAlloc@NAlloc@@@NArray@@@@IEAAPEAUVirtualExample1D@@PEAU2@H@Z 00000000315267a0 f i ParametricSampler.obj
 0001:00025860       ?expand_raw@?$DynArray@UVirtualExample2D@@HU?$SmallDynStorage@UVirtualExample2D@@HUStandardAlloc@NAlloc@@@NArray@@@@IEAAPEAUVirtualExample2D@@PEAU2@H@Z 0000000031526860 f i ParametricSampler.obj
 0001:00025920       ?expand_raw@?$DynArray@UVirtualExample3D@@HU?$SmallDynStorage@UVirtualExample3D@@HUStandardAlloc@NAlloc@@@NArray@@@@IEAAPEAUVirtualExample3D@@PEAU2@H@Z 0000000031526920 f i ParametricSampler.obj
 0001:000259e0       ?GetWeights3D@SParametricSamplerInternal@@QEAAXAEBU?$Vec3_tpl@M@@AEBUGlobalAnimationHeaderLMG@@QEAMU?$Diag33_tpl@M@@U2@@Z 00000000315269e0 f   ParametricSampler.obj
 0001:00025d80       ?ComputeWeightExtrapolate4@SParametricSamplerInternal@@QEAAXAEAU?$Vec4_tpl@M@@AEBU?$Vec2_tpl@M@@1111@Z 0000000031526d80 f   ParametricSampler.obj
 0001:00026470       ?GetConvex4@SParametricSamplerInternal@@QEAA?AUBC4@@IAEBU?$Vec2_tpl@M@@AEBUGlobalAnimationHeaderLMG@@QEAMPEAEPEAU?$Vec3_tpl@M@@U?$Diag33_tpl@M@@U5@@Z 0000000031527470 f   ParametricSampler.obj
 0001:00027140       ?GetWeights2D@SParametricSamplerInternal@@QEAAXAEBU?$Vec2_tpl@M@@AEBUGlobalAnimationHeaderLMG@@QEAMU?$Diag33_tpl@M@@U?$Vec3_tpl@M@@@Z 0000000031528140 f   ParametricSampler.obj
 0001:00027420       ?VisualizeBlendSpace@SParametricSamplerInternal@@QEAAXPEBVCAnimationSet@@AEBVCAnimation@@MIAEBUGlobalAnimationHeaderLMG@@U?$Vec3_tpl@M@@@Z 0000000031528420 f   ParametricSampler.obj
 0001:00028420       ?resize@?$DynArray@UVirtualExample3D@@HU?$SmallDynStorage@UVirtualExample3D@@HUStandardAlloc@NAlloc@@@NArray@@@@QEAAXH@Z 0000000031529420 f i ParametricSampler.obj
 0001:00028460       ?BlendSpace1D@SParametricSamplerInternal@@QEAAXAEAUGlobalAnimationHeaderLMG@@PEBVCAnimationSet@@AEBVCAnimation@@MMU?$Vec3_tpl@M@@_NI@Z 0000000031529460 f   ParametricSampler.obj
 0001:000292d0       ?BlendSpace2D@SParametricSamplerInternal@@QEAAXAEAUGlobalAnimationHeaderLMG@@PEBVCAnimationSet@@AEBVCAnimation@@MMU?$Vec3_tpl@M@@_NI@Z 000000003152a2d0 f   ParametricSampler.obj
 0001:0002aab0       ?BlendSpace3D@SParametricSamplerInternal@@QEAAXAEAUGlobalAnimationHeaderLMG@@PEBVCAnimationSet@@AEBVCAnimation@@MMU?$Vec3_tpl@M@@_NI@Z 000000003152bab0 f   ParametricSampler.obj
 0001:0002c9e0       ?CombinedBlendSpaces@SParametricSamplerInternal@@QEAAXAEAUGlobalAnimationHeaderLMG@@PEBVCAnimationSet@@AEBVCAnimation@@MM_N@Z 000000003152d9e0 f   ParametricSampler.obj
 0001:0002d060       ?Parameterizer@SParametricSamplerInternal@@QEAAMPEBVCAnimationSet@@AEBVCAnimation@@MM_N@Z 000000003152e060 f   ParametricSampler.obj
 0001:0002d930       ?GetAllocatedObjects@CPlaceholderCharacter@@SAHXZ 000000003152e930 f   PlaceholderCharacter.obj
 0001:0002d940       ?Release@CPlaceholderCharacter@@UEAAXXZ 000000003152e940 f   PlaceholderCharacter.obj
 0001:0002d960       ?RequestHighPriorityMaterialsLoading@CPlaceholderCharacter@@UEAAXXZ 000000003152e960 f   PlaceholderCharacter.obj
 0001:0002d9d0       ?GenerateIdFromName@CPlaceholderCharacter@@SAIPEBD@Z 000000003152e9d0 f   PlaceholderCharacter.obj
 0001:0002da00       ??1CPlaceholderCharacter@@UEAA@XZ 000000003152ea00 f   PlaceholderCharacter.obj
 0001:0002dd30       ??0CPlaceholderCharacter@@QEAA@XZ 000000003152ed30 f   PlaceholderCharacter.obj
 0001:0002de00       ??_ECPlaceholderCharacter@@UEAAPEAXI@Z 000000003152ee00 f i PlaceholderCharacter.obj
 0001:0002de00       ??_GCPlaceholderCharacter@@UEAAPEAXI@Z 000000003152ee00 f i PlaceholderCharacter.obj
 0001:0002de30       ?RegisterUsedSkin@CPlaceholderCharacter@@QEAAXPEAUISkin@@@Z 000000003152ee30 f   PlaceholderCharacter.obj
 0001:0002dec0       ?RegisterUsedSkeleton@CPlaceholderCharacter@@QEAAXPEAUICharacterModel@@@Z 000000003152eec0 f   PlaceholderCharacter.obj
 0001:0002df50       ?RegisterUsedStaticObject@CPlaceholderCharacter@@QEAAXPEAUIStatObj@@@Z 000000003152ef50 f   PlaceholderCharacter.obj
 0001:0002dfe0       ?RegisterUsedMaterial@CPlaceholderCharacter@@QEAAXPEAUIMaterial@@@Z 000000003152efe0 f   PlaceholderCharacter.obj
 0001:0002e070       ?GetISkeletonPose@CCharInstance@@UEAAPEAUISkeletonPose@@XZ 000000003152f070 f i DirectionalBlender.obj
 0001:0002e080       ?AccumulateAimPoses@SDirectionalBlender@@QEAAXAEBUSAnimationPoseModifierParams@@AEAUGlobalAnimationHeaderAIM@@PEAU?$QuatT_tpl@M@@MAEBU?$Vec3_tpl@M@@HHPEAUSJointsAimIK_Rot@@IPEAUSJointsAimIK_Pos@@MIAEBU?$Color_tpl@E@@@Z 000000003152f080 f   DirectionalBlender.obj
 0001:0002f890       ?DebugVEGrid@SDirectionalBlender@@QEAAXAEBUSAnimationPoseModifierParams@@AEAUSDirInfo@@MMHPEAUSJointsAimIK_Rot@@IPEAUSJointsAimIK_Pos@@I@Z 0000000031530890 f   DirectionalBlender.obj
 0001:00032a60       ?resize_raw@?$SmallDynStorage@V?$_smart_ptr@VIController@@@@HUStandardAlloc@NAlloc@@@NArray@@QEAAXHH_N@Z 0000000031533a60 f i DirectionalBlender.obj
 0001:00032bd0       ?clear@?$DynArray@V?$_smart_ptr@VIController@@@@HU?$SmallDynStorage@V?$_smart_ptr@VIController@@@@HUStandardAlloc@NAlloc@@@NArray@@@@QEAAXXZ 0000000031533bd0 f i DirectionalBlender.obj
 0001:00032c70       ??1?$DynArray@V?$_smart_ptr@VIController@@@@HU?$SmallDynStorage@V?$_smart_ptr@VIController@@@@HUStandardAlloc@NAlloc@@@NArray@@@@QEAA@XZ 0000000031533c70 f i DirectionalBlender.obj
 0001:00032c70       ??1?$DynArray@V?$_smart_ptr@UCMorphTarget@@@@HU?$SmallDynStorage@V?$_smart_ptr@UCMorphTarget@@@@HUStandardAlloc@NAlloc@@@NArray@@@@QEAA@XZ 0000000031533c70 f i LoaderSKIN.obj
 0001:00032cf0       ?destroy@?$DynArray@UAimIKPose@@HU?$SmallDynStorage@UAimIKPose@@HUStandardAlloc@NAlloc@@@NArray@@@@KAXU?$Array@UAimIKPose@@HU?$ArrayStorage@UAimIKPose@@H@NArray@@@@@Z 0000000031533cf0 f i DirectionalBlender.obj
 0001:00032e60       ??0GlobalAnimationHeaderAIM@@QEAA@XZ 0000000031533e60 f i DirectionalBlender.obj
 0001:00032fa0       ??1GlobalAnimationHeaderAIM@@QEAA@XZ 0000000031533fa0 f i DirectionalBlender.obj
 0001:00033090       ?ExecuteDirectionalIK@SDirectionalBlender@@QEAA_NAEBUSAnimationPoseModifierParams@@PEAUDirectionalBlends@@IPEAUSJointsAimIK_Rot@@IPEAUSJointsAimIK_Pos@@IAEBU?$Color_tpl@E@@@Z 0000000031534090 f   DirectionalBlender.obj
 0001:00034760       ?Execute@COperatorQueue@@UEAA_NAEBUSAnimationPoseModifierParams@@@Z 0000000031535760 f   OperatorQueue.obj
 0001:000354a0       ?allocate@?$_STLP_alloc_proxy@PEAUSOp@COperatorQueue@@U12@V?$allocator@USOp@COperatorQueue@@@stlpmtx_std@@@priv@stlpmtx_std@@QEAAPEAUSOp@COperatorQueue@@_KAEA_K@Z 00000000315364a0 f i OperatorQueue.obj
 0001:00035510       ??$_M_allocate_and_copy@PEAUSOp@COperatorQueue@@@?$_Impl_vector@USOp@COperatorQueue@@V?$allocator@USOp@COperatorQueue@@@stlpmtx_std@@@priv@stlpmtx_std@@AEAAPEAUSOp@COperatorQueue@@AEA_KPEAU34@1@Z 0000000031536510 f i OperatorQueue.obj
 0001:000355c0       ??0CFactory@COperatorQueue@@AEAA@XZ 00000000315365c0 f i OperatorQueue.obj
 0001:00035660       ?GetClassName@CFactory@COperatorQueue@@UEBAPEBDXZ 0000000031536660 f i OperatorQueue.obj
 0001:00035670       ?GetClassID@CFactory@COperatorQueue@@UEBAAEBUCryGUID@@XZ 0000000031536670 f i OperatorQueue.obj
 0001:00035680       ??_Ebad_alloc@std@@UEAAPEAXI@Z 0000000031536680 f i OperatorQueue.obj
 0001:00035680       ??_Gbad_alloc@std@@UEAAPEAXI@Z 0000000031536680 f i OperatorQueue.obj
 0001:000356c0       ?sp_enable_shared_from_this@detail@boost@@YAXZZ 00000000315366c0 f i OperatorQueue.obj
 0001:000356e0       ??1COperatorQueue@@MEAA@XZ 00000000315366e0 f   OperatorQueue.obj
 0001:000357d0       ?GetFactory@COperatorQueue@@UEBAPEAUICryFactory@@XZ 00000000315367d0 f i OperatorQueue.obj
 0001:000357e0       ?QueryInterface@COperatorQueue@@MEBAPEAXAEBUCryGUID@@@Z 00000000315367e0 f i OperatorQueue.obj
 0001:00035850       ?reserve@?$_Impl_vector@USOp@COperatorQueue@@V?$allocator@USOp@COperatorQueue@@@stlpmtx_std@@@priv@stlpmtx_std@@QEAAX_K@Z 0000000031536850 f i OperatorQueue.obj
 0001:00035910       ??_GCOperatorQueue@@MEAAPEAXI@Z 0000000031536910 f i OperatorQueue.obj
 0001:00035910       ??_ECOperatorQueue@@MEAAPEAXI@Z 0000000031536910 f i OperatorQueue.obj
 0001:00035940       ??0COperatorQueue@@IEAA@XZ 0000000031536940 f   OperatorQueue.obj
 0001:00035a50       ?PushPosition@COperatorQueue@@UEAAXIW4EOp@IAnimationOperatorQueue@@AEBU?$Vec3_tpl@M@@@Z 0000000031536a50 f   OperatorQueue.obj
 0001:00035c10       ?PushOrientation@COperatorQueue@@UEAAXIW4EOp@IAnimationOperatorQueue@@AEBU?$Quat_tpl@M@@@Z 0000000031536c10 f   OperatorQueue.obj
 0001:00035dd0       ?PushStoreRelative@COperatorQueue@@UEAAXIAEAU?$QuatT_tpl@M@@@Z 0000000031536dd0 f   OperatorQueue.obj
 0001:00035f70       ?PushStoreAbsolute@COperatorQueue@@UEAAXIAEAU?$QuatT_tpl@M@@@Z 0000000031536f70 f   OperatorQueue.obj
 0001:00036110       ?PushComputeAbsolute@COperatorQueue@@UEAAXXZ 0000000031537110 f   OperatorQueue.obj
 0001:000362a0       ?Clear@COperatorQueue@@UEAAXXZ 00000000315372a0 f   OperatorQueue.obj
 0001:000362c0       ?Prepare@COperatorQueue@@UEAA_NAEBUSAnimationPoseModifierParams@@@Z 00000000315372c0 f   OperatorQueue.obj
 0001:000362f0       ?Synchronize@COperatorQueue@@UEAAXXZ 00000000315372f0 f   OperatorQueue.obj
 0001:00036310       ?CreateClassInstance@CFactory@COperatorQueue@@UEBA?AV?$shared_ptr@UICryUnknown@@@boost@@XZ 0000000031537310 f i OperatorQueue.obj
 0001:000363d0       ?Initialize@CPoseAlignerChain@@UEAAXW4EType@IAnimationPoseAlignerChain@@PEBDH@Z 00000000315373d0 f   PoseAlignerChain.obj
 0001:000363f0       ?Ray_Plane@Intersect@@YA_NAEBURay@@AEBU?$Plane_tpl@M@@AEAU?$Vec3_tpl@M@@_N@Z 00000000315373f0 f i PoseAlignerChain.obj
 0001:00036520       ?GetFactory@CPoseAlignerChain@@UEBAPEAUICryFactory@@XZ 0000000031537520 f i PoseAlignerChain.obj
 0001:00036530       ?SetTarget@CPoseAlignerChain@@UEAAXAEBU?$Plane_tpl@M@@MMMM@Z 0000000031537530 f i PoseAlignerChain.obj
 0001:00036570       ?GetMemoryUsage@CPoseAlignerChain@@UEBAXPEAVICrySizer@@@Z 0000000031537570 f i PoseAlignerChain.obj
 0001:00036590       ?AlignToTarget@CPoseAlignerChain@@AEAAXAEBUSAnimationPoseModifierParams@@@Z 0000000031537590 f   PoseAlignerChain.obj
 0001:00037550       ?MoveToTarget@CPoseAlignerChain@@AEAA_NAEBUSAnimationPoseModifierParams@@AEAU?$Vec3_tpl@M@@@Z 0000000031538550 f   PoseAlignerChain.obj
 0001:000379f0       ?Execute@CPoseAlignerChain@@UEAA_NAEBUSAnimationPoseModifierParams@@@Z 00000000315389f0 f   PoseAlignerChain.obj
 0001:000394a0       ?QueryInterface@CPoseAlignerChain@@MEBAPEAXAEBUCryGUID@@@Z 000000003153a4a0 f i PoseAlignerChain.obj
 0001:00039510       ?Prepare@CPoseAlignerChain@@UEAA_NAEBUSAnimationPoseModifierParams@@@Z 000000003153a510 f   PoseAlignerChain.obj
 0001:00039600       ??0CFactory@CPoseAlignerChain@@AEAA@XZ 000000003153a600 f i PoseAlignerChain.obj
 0001:000396a0       ?GetClassName@CFactory@CPoseAlignerChain@@UEBAPEBDXZ 000000003153a6a0 f i PoseAlignerChain.obj
 0001:000396b0       ?GetClassID@CFactory@CPoseAlignerChain@@UEBAAEBUCryGUID@@XZ 000000003153a6b0 f i PoseAlignerChain.obj
 0001:000396c0       ??$?0VCFeetPoseRestore@@@shared_count@detail@boost@@QEAA@PEAVCFeetPoseRestore@@@Z 000000003153a6c0 f i FeetLock.obj
 0001:000396c0       ??$?0VCPoseAlignerChain@@@shared_count@detail@boost@@QEAA@PEAVCPoseAlignerChain@@@Z 000000003153a6c0 f i PoseAlignerChain.obj
 0001:000396c0       ??$?0VCFeetPoseStore@@@shared_count@detail@boost@@QEAA@PEAVCFeetPoseStore@@@Z 000000003153a6c0 f i FeetLock.obj
 0001:000396c0       ??$?0VCPoseMatching@@@shared_count@detail@boost@@QEAA@PEAVCPoseMatching@@@Z 000000003153a6c0 f i PoseMatching.obj
 0001:000396c0       ??$?0VCLimbIk@@@shared_count@detail@boost@@QEAA@PEAVCLimbIk@@@Z 000000003153a6c0 f i LimbIk.obj
 0001:000396c0       ??$?0VCOperatorQueue@@@shared_count@detail@boost@@QEAA@PEAVCOperatorQueue@@@Z 000000003153a6c0 f i OperatorQueue.obj
 0001:000396c0       ??$?0VCPoseBlenderLook@@@shared_count@detail@boost@@QEAA@PEAVCPoseBlenderLook@@@Z 000000003153a6c0 f i PoseBlenderLook.obj
 0001:000396c0       ??$?0VCRecoil@PoseModifier@@@shared_count@detail@boost@@QEAA@PEAVCRecoil@PoseModifier@@@Z 000000003153a6c0 f i Recoil.obj
 0001:000396c0       ??$?0VCGroundAlignment@@@shared_count@detail@boost@@QEAA@PEAVCGroundAlignment@@@Z 000000003153a6c0 f i GroundAlignment.obj
 0001:000396c0       ??$?0VCPoseBlenderAim@@@shared_count@detail@boost@@QEAA@PEAVCPoseBlenderAim@@@Z 000000003153a6c0 f i PoseBlenderAim.obj
 0001:00039780       ?CreateClassInstance@CFactory@CPoseAlignerChain@@UEBA?AV?$shared_ptr@UICryUnknown@@@boost@@XZ 000000003153a780 f i PoseAlignerChain.obj
 0001:00039840       ?SetAnimations@CPoseMatching@@UEAAXPEBII@Z 000000003153a840 f   PoseMatching.obj
 0001:00039850       ?GetMatchingAnimation@CPoseMatching@@UEBA_NAEAI@Z 000000003153a850 f   PoseMatching.obj
 0001:00039860       ?Prepare@CPoseMatching@@UEAA_NAEBUSAnimationPoseModifierParams@@@Z 000000003153a860 f   PoseMatching.obj
 0001:00039870       ??$?0M@?$Ang3_tpl@M@@QEAA@AEBU?$Quat_tpl@M@@@Z 000000003153a870 f i PoseMatching.obj
 0001:00039a20       ?GetFactory@CPoseMatching@@UEBAPEAUICryFactory@@XZ 000000003153aa20 f i PoseMatching.obj
 0001:00039a30       ?Execute@CPoseMatching@@UEAA_NAEBUSAnimationPoseModifierParams@@@Z 000000003153aa30 f   PoseMatching.obj
 0001:0003a9d0       ?QueryInterface@CPoseMatching@@MEBAPEAXAEBUCryGUID@@@Z 000000003153b9d0 f i PoseMatching.obj
 0001:0003aa40       ??0CFactory@CPoseMatching@@AEAA@XZ 000000003153ba40 f i PoseMatching.obj
 0001:0003aae0       ?GetClassName@CFactory@CPoseMatching@@UEBAPEBDXZ 000000003153bae0 f i PoseMatching.obj
 0001:0003aaf0       ?GetClassID@CFactory@CPoseMatching@@UEBAAEBUCryGUID@@XZ 000000003153baf0 f i PoseMatching.obj
 0001:0003ab00       ?ClassSupports@CFactory@CPoseMatching@@UEBA_NAEBUCryGUID@@@Z 000000003153bb00 f i PoseMatching.obj
 0001:0003ab00       ?ClassSupports@CFactory@CLimbIk@@UEBA_NAEBUCryGUID@@@Z 000000003153bb00 f i LimbIk.obj
 0001:0003ab00       ?ClassSupports@CFactory@CPoseAlignerChain@@UEBA_NAEBUCryGUID@@@Z 000000003153bb00 f i PoseAlignerChain.obj
 0001:0003ab00       ?ClassSupports@CFactory@CPoseBlenderLook@@UEBA_NAEBUCryGUID@@@Z 000000003153bb00 f i PoseBlenderLook.obj
 0001:0003ab00       ?ClassSupports@CFactory@CFeetPoseRestore@@UEBA_NAEBUCryGUID@@@Z 000000003153bb00 f i FeetLock.obj
 0001:0003ab00       ?ClassSupports@CFactory@CRecoil@PoseModifier@@UEBA_NAEBUCryGUID@@@Z 000000003153bb00 f i Recoil.obj
 0001:0003ab00       ?ClassSupports@CFactory@COperatorQueue@@UEBA_NAEBUCryGUID@@@Z 000000003153bb00 f i OperatorQueue.obj
 0001:0003ab00       ?ClassSupports@CFactory@CGroundAlignment@@UEBA_NAEBUCryGUID@@@Z 000000003153bb00 f i GroundAlignment.obj
 0001:0003ab00       ?ClassSupports@CFactory@CEngineModule_CryAnimation@@UEBA_NAEBUCryGUID@@@Z 000000003153bb00 f i AnimationBase.obj
 0001:0003ab00       ?ClassSupports@CFactory@CPoseBlenderAim@@UEBA_NAEBUCryGUID@@@Z 000000003153bb00 f i PoseBlenderAim.obj
 0001:0003ab00       ?ClassSupports@CFactory@CFeetPoseStore@@UEBA_NAEBUCryGUID@@@Z 000000003153bb00 f i FeetLock.obj
 0001:0003ab40       ?CreateClassInstance@CFactory@CPoseMatching@@UEBA?AV?$shared_ptr@UICryUnknown@@@boost@@XZ 000000003153bb40 f i PoseMatching.obj
 0001:0003ac00       ?NTime2KTime@GlobalAnimationHeaderCAF@@QEAAMM@Z 000000003153bc00 f i SkeletonAnim_Locator.obj
 0001:0003ac40       ?ParseLayer0@CSkeletonAnim@@AEBAXAEBVCAnimation@@PEAUAnimInfo@@AEAIMI@Z 000000003153bc40 f   SkeletonAnim_Locator.obj
 0001:0003b2c0       ?GetRootController@CSkeletonAnim@@AEBAPEAVIController@@AEAUGlobalAnimationHeaderCAF@@@Z 000000003153c2c0 f   SkeletonAnim_Locator.obj
 0001:0003b3e0       ?Extract_DeltaMovement@CSkeletonAnim@@AEBAXPEAUAnimInfo@@AEAIPEAUSDeltaMotion@@M@Z 000000003153c3e0 f   SkeletonAnim_Locator.obj
 0001:0003ef00       ?CalculateRelativeMovement@CSkeletonAnim@@UEBA?AU?$QuatT_tpl@M@@M_N@Z 000000003153ff00 f   SkeletonAnim_Locator.obj
 0001:0003f980       ?GetJointCount@CSkeletonPhysics@@AEBAIXZ 0000000031540980 f   SkeletonPhysics.obj
 0001:0003f9a0       ?SetAuxParams@CSkeletonPhysics@@QEAAXPEAUpe_params@@@Z 00000000315409a0 f   SkeletonPhysics.obj
 0001:0003fa10       ?GetCharacterPhysics@CSkeletonPhysics@@QEAAPEAUIPhysicalEntity@@PEBD@Z 0000000031540a10 f   SkeletonPhysics.obj
 0001:0003faa0       ?GetCharacterPhysics@CSkeletonPhysics@@QEAAPEAUIPhysicalEntity@@H@Z 0000000031540aa0 f   SkeletonPhysics.obj
 0001:0003fad0       ??_GISplineBackup@@UEAAPEAXI@Z 0000000031540ad0 f i FaceAnimSequence.obj
 0001:0003fad0       ??_GIVertexAnimation@@UEAAPEAXI@Z 0000000031540ad0 f i VertexAnimation.obj
 0001:0003fad0       ??_GIFaceState@@UEAAPEAXI@Z 0000000031540ad0 f i FacialModel.obj
 0001:0003fad0       ??_EValidator@pe_action_batch_parts_update@@UEAAPEAXI@Z 0000000031540ad0 f i SkeletonPhysics.obj
 0001:0003fad0       ??_EISplineBackup@@UEAAPEAXI@Z 0000000031540ad0 f i FaceAnimSequence.obj
 0001:0003fad0       ??_GValidator@pe_action_batch_parts_update@@UEAAPEAXI@Z 0000000031540ad0 f i SkeletonPhysics.obj
 0001:0003fad0       ??_EIVertexAnimation@@UEAAPEAXI@Z 0000000031540ad0 f i VertexAnimation.obj
 0001:0003fad0       ??_EIFaceState@@UEAAPEAXI@Z 0000000031540ad0 f i FacialModel.obj
 0001:0003fb00       ??_ESBatchUpdateValidator@@UEAAPEAXI@Z 0000000031540b00 f i SkeletonPhysics.obj
 0001:0003fb00       ??_GSBatchUpdateValidator@@UEAAPEAXI@Z 0000000031540b00 f i SkeletonPhysics.obj
 0001:0003fb80       ?Initialize@CSkeletonPhysics@@QEAA_NAEAVCSkeletonPose@@@Z 0000000031540b80 f   SkeletonPhysics.obj
 0001:0003fbf0       ?GetPoseData@CSkeletonPhysics@@AEBAAEBVCPoseData@Skeleton@@XZ 0000000031540bf0 f   SkeletonPhysics.obj
 0001:0003fc00       ?SetPhysEntOnJoint@CSkeletonPhysics@@QEAAXHPEAUIPhysicalEntity@@@Z 0000000031540c00 f   SkeletonPhysics.obj
 0001:0003fd10       ?DestroyPhysics@CSkeletonPhysics@@QEAAXXZ 0000000031540d10 f   SkeletonPhysics.obj
 0001:0003fe50       ?getBonePhysParentOrSelfIndex@CSkeletonPhysics@@QEAAHHH@Z 0000000031540e50 f   SkeletonPhysics.obj
 0001:0003fee0       ?getBonePhysChildIndex@CSkeletonPhysics@@AEAAHHH@Z 0000000031540ee0 f   SkeletonPhysics.obj
 0001:0003ff90       ?GetBoneSurfaceTypeId@CSkeletonPhysics@@QEAAHHH@Z 0000000031540f90 f   SkeletonPhysics.obj
 0001:0003ffd0       ?TranslatePartIdToDeadBody@CSkeletonPhysics@@QEAAHH@Z 0000000031540fd0 f   SkeletonPhysics.obj
 0001:00040050       ?ParsePhysInfoProps@@YAXPEAVCModelJoint@@HAEAUpe_params_rope@@AEAUpe_simulation_params@@AEAUpe_params_flags@@@Z 0000000031541050 f   SkeletonPhysics.obj
 0001:000401e0       ??0?$Matrix34_tpl@M@@QEAA@AEBU?$Vec3_tpl@M@@AEBU?$Quat_tpl@M@@0@Z 00000000315411e0 f i SkeletonPhysics.obj
 0001:00040390       ??$?0M@?$Ang3_tpl@M@@QEAA@AEBU?$Matrix33_tpl@M@@@Z 0000000031541390 f i SkeletonPhysics.obj
 0001:00040490       ??0pe_params_part@@QEAA@XZ 0000000031541490 f i SkeletonPhysics.obj
 0001:000405a0       ??0pe_params_joint@@QEAA@XZ 00000000315415a0 f i SkeletonPhysics.obj
 0001:00040740       ??0pe_params_articulated_body@@QEAA@XZ 0000000031541740 f i SkeletonPhysics.obj
 0001:000408a0       ??0pe_params_rope@@QEAA@XZ 00000000315418a0 f i SkeletonPhysics.obj
 0001:00040b30       ??0pe_params_softbody@@QEAA@XZ 0000000031541b30 f i SkeletonPhysics.obj
 0001:00040cd0       ??0SBatchUpdateValidator@@QEAA@XZ 0000000031541cd0 f i SkeletonPhysics.obj
 0001:00040d40       ?Lock@SBatchUpdateValidator@@UEAA_NXZ 0000000031541d40 f i SkeletonPhysics.obj
 0001:00040d90       ?Unlock@SBatchUpdateValidator@@UEAAXXZ 0000000031541d90 f i SkeletonPhysics.obj
 0001:00040dd0       ?GetPhysIdOnJoint@CSkeletonPhysics@@QEAAHH@Z 0000000031541dd0 f   SkeletonPhysics.obj
 0001:00040e30       ?BuildPhysicalEntity@CSkeletonPhysics@@QEAAXPEAUIPhysicalEntity@@MHMHHAEBU?$Matrix34_tpl@M@@@Z 0000000031541e30 f   SkeletonPhysics.obj
 0001:00042680       ?DestroyCharacterPhysics@CSkeletonPhysics@@QEAAXH@Z 0000000031543680 f   SkeletonPhysics.obj
 0001:00042970       ?CreateCharacterPhysics@CSkeletonPhysics@@QEAAPEAUIPhysicalEntity@@PEAU2@MHMHAEBU?$Matrix34_tpl@M@@@Z 0000000031543970 f   SkeletonPhysics.obj
 0001:00042f20       ?AddImpact@CSkeletonPhysics@@QEAA_NHU?$Vec3_tpl@M@@0@Z 0000000031543f20 f   SkeletonPhysics.obj
 0001:00043190       ?Physics_SynchronizeToImpact@CSkeletonPhysics@@AEAAXM@Z 0000000031544190 f   SkeletonPhysics.obj
 0001:000434d0       ?SynchronizeWithPhysicsPost@CSkeletonPhysics@@QEAAXXZ 00000000315444d0 f   SkeletonPhysics.obj
 0001:00043750       ?FindSpineBones@CSkeletonPhysics@@AEAAXXZ 0000000031544750 f   SkeletonPhysics.obj
 0001:00043830       ?GoLimp@CSkeletonPhysics@@QEAAXXZ 0000000031544830 f   SkeletonPhysics.obj
 0001:00043940       ?GetFallingDir@CSkeletonPhysics@@QEAAHXZ 0000000031544940 f   SkeletonPhysics.obj
 0001:00044140       ?resize_raw@?$SmallDynStorage@HHUStandardAlloc@NAlloc@@@NArray@@QEAAXHH_N@Z 0000000031545140 f i SkeletonPhysics.obj
 0001:000442d0       ?CreateAuxilaryPhysics@CSkeletonPhysics@@QEAAHPEAUIPhysicalEntity@@AEBU?$Matrix34_tpl@M@@MU?$Vec3_tpl@M@@H@Z 00000000315452d0 f   SkeletonPhysics.obj
 0001:00046f20       ?Physics_SynchronizeToAux@CSkeletonPhysics@@AEAAXAEBVCPoseData@Skeleton@@@Z 0000000031547f20 f   SkeletonPhysics.obj
 0001:00047b40       ?Physics_SynchronizeToEntity@CSkeletonPhysics@@AEAAXAEAUIPhysicalEntity@@U?$QuatT_tpl@M@@@Z 0000000031548b40 f   SkeletonPhysics.obj
 0001:000482c0       ?Physics_SynchronizeToEntityArticulated@CSkeletonPhysics@@AEAAXM@Z 00000000315492c0 f   SkeletonPhysics.obj
 0001:000487a0       ?set_size@?$SmallDynStorage@UCPhysicsJoint@@HUStandardAlloc@NAlloc@@@NArray@@QEAAXH@Z 00000000315497a0 f i SkeletonPhysics.obj
 0001:00048850       ??$move_init@U?$QuatT_tpl@M@@@NArray@@YAXPEAU?$QuatT_tpl@M@@0_K@Z 0000000031549850 f i SkeletonPhysics.obj
 0001:00048a10       ?CreateAuxilaryPhysics@CSkeletonPhysics@@QEAAHPEAUIPhysicalEntity@@AEBU?$Matrix34_tpl@M@@H@Z 0000000031549a10 f   SkeletonPhysics.obj
 0001:00048a70       ?SynchronizeWithPhysicalEntity@CSkeletonPhysics@@QEAAXAEAVCPoseData@Skeleton@@PEAUIPhysicalEntity@@AEBU?$Vec3_tpl@M@@AEBU?$Quat_tpl@M@@U?$QuatT_tpl@M@@H@Z 0000000031549a70 f   SkeletonPhysics.obj
 0001:00048bb0       ?SynchronizeWithPhysicalEntity@CSkeletonPhysics@@QEAAXPEAUIPhysicalEntity@@AEBU?$Vec3_tpl@M@@AEBU?$Quat_tpl@M@@@Z 0000000031549bb0 f   SkeletonPhysics.obj
 0001:00048d10       ?ProcessPhysics@CSkeletonPhysics@@AEAAXAEAVCPoseData@Skeleton@@MPEAUSCharUpdateFeedback@@@Z 0000000031549d10 f   SkeletonPhysics.obj
 0001:00048e10       ?SynchronizeWithPhysics@CSkeletonPhysics@@QEAAXAEAVCPoseData@Skeleton@@@Z 0000000031549e10 f   SkeletonPhysics.obj
 0001:000490a0       ?append_raw@?$DynArray@HHU?$SmallDynStorage@HHUStandardAlloc@NAlloc@@@NArray@@@@QEAA?AU?$Array@HHU?$ArrayStorage@HH@NArray@@@@H@Z 000000003154a0a0 f i SkeletonPhysics.obj
 0001:00049160       ?resize_raw@?$SmallDynStorage@U?$QuatT_tpl@M@@HUStandardAlloc@NAlloc@@@NArray@@QEAAXHH_N@Z 000000003154a160 f i SkeletonPhysics.obj
 0001:000492f0       ??$move_init@UCPhysicsJoint@@@NArray@@YAXPEAUCPhysicsJoint@@0_K@Z 000000003154a2f0 f i SkeletonPhysics.obj
 0001:00049680       ?expand_raw@?$DynArray@U?$QuatT_tpl@M@@HU?$SmallDynStorage@U?$QuatT_tpl@M@@HUStandardAlloc@NAlloc@@@NArray@@@@IEAAPEAU?$QuatT_tpl@M@@PEAU2@H@Z 000000003154a680 f i SkeletonPhysics.obj
 0001:00049740       ?resize_raw@?$SmallDynStorage@UCPhysicsJoint@@HUStandardAlloc@NAlloc@@@NArray@@QEAAXHH_N@Z 000000003154a740 f i SkeletonPhysics.obj
 0001:000498c0       ??1CSkeletonPhysics@@QEAA@XZ 000000003154a8c0 f   SkeletonPhysics.obj
 0001:000499c0       ?resize@?$DynArray@HHU?$SmallDynStorage@HHUStandardAlloc@NAlloc@@@NArray@@@@QEAAXH@Z 000000003154a9c0 f i SkeletonPhysics.obj
 0001:00049a00       ?expand_raw@?$DynArray@UCPhysicsJoint@@HU?$SmallDynStorage@UCPhysicsJoint@@HUStandardAlloc@NAlloc@@@NArray@@@@IEAAPEAUCPhysicsJoint@@PEAU2@H@Z 000000003154aa00 f i SkeletonPhysics.obj
 0001:00049ac0       ??0CSkeletonPhysics@@QEAA@XZ 000000003154aac0 f   SkeletonPhysics.obj
 0001:00049d20       ?grow@?$DynArray@UCPhysicsJoint@@HU?$SmallDynStorage@UCPhysicsJoint@@HUStandardAlloc@NAlloc@@@NArray@@@@QEAAPEAUCPhysicsJoint@@H@Z 000000003154ad20 f i SkeletonPhysics.obj
 0001:00049dc0       ?InitializeAnimToPhysIndexArray@CSkeletonPhysics@@QEAAXXZ 000000003154adc0 f   SkeletonPhysics.obj
 0001:00049f00       ?InitPhysicsSkeleton@CSkeletonPhysics@@QEAAXXZ 000000003154af00 f   SkeletonPhysics.obj
 0001:0004a3c0       ?RelinquishCharacterPhysics@CSkeletonPhysics@@QEAAPEAUIPhysicalEntity@@AEBU?$Matrix34_tpl@M@@M_NAEBU?$Vec3_tpl@M@@@Z 000000003154b3c0 f   SkeletonPhysics.obj
 0001:0004ba90       ?BlendFromRagdoll@CSkeletonPhysics@@QEAA_NAEAU?$QuatTS_tpl@M@@AEAPEAUIPhysicalEntity@@_N@Z 000000003154ca90 f   SkeletonPhysics.obj
 0001:0004d020       ?GetParent@CModelJoint@@QEAAPEAV1@XZ 000000003154e020 f i SkeletonPhysics_SPU.obj
 0001:0004d050       ?getBoneParentIndex@CSkeletonPhysics@@AEAAII@Z 000000003154e050 f   SkeletonPhysics_SPU.obj
 0001:0004d090       ?ResetNonphysicalBoneRotations@CSkeletonPhysics@@AEAAXAEAVCPoseData@Skeleton@@HM@Z 000000003154e090 f   SkeletonPhysics_SPU.obj
 0001:0004d420       ?getBonePhysParentIndex@CSkeletonPhysics@@QEAAHHH@Z 000000003154e420 f   SkeletonPhysics_SPU.obj
 0001:0004d4b0       ?SPU_Physics_SynchronizeFromEntityPrepare@CSkeletonPhysics@@AEAAXAEAVCPool@Memory@@PEAUIPhysicalEntity@@@Z 000000003154e4b0 f   SkeletonPhysics_SPU.obj
 0001:0004da20       ?SPU_Physics_SynchronizeFromAuxPrepare@CSkeletonPhysics@@AEAAXAEAVCPool@Memory@@@Z 000000003154ea20 f   SkeletonPhysics_SPU.obj
 0001:0004e0a0       ?SPU_Physics_SynchronizeFromImpactPrepare@CSkeletonPhysics@@AEAAXAEAVCPool@Memory@@@Z 000000003154f0a0 f   SkeletonPhysics_SPU.obj
 0001:0004e230       ?SPU_SynchronizeWithPhysicsPrepare@CSkeletonPhysics@@QEAAXAEAVCPool@Memory@@@Z 000000003154f230 f   SkeletonPhysics_SPU.obj
 0001:0004e300       ?DoSetRagdollDefaultPose@CSkeletonPhysics@@AEAAXAEAVCPoseData@Skeleton@@@Z 000000003154f300 f   SkeletonPhysics_SPU.obj
 0001:0004ea30       ?UnconvertBoneGlobalFromRelativeForm@CSkeletonPhysics@@AEAAXAEAVCPoseData@Skeleton@@_NH1@Z 000000003154fa30 f   SkeletonPhysics_SPU.obj
 0001:0004ee20       ?SPU_Physics_SynchronizeFromEntity@CSkeletonPhysics@@AEAAXAEAVCPoseData@Skeleton@@PEAUIPhysicalEntity@@AEBU?$Vec3_tpl@M@@AEBU?$Quat_tpl@M@@U?$QuatT_tpl@M@@@Z 000000003154fe20 f   SkeletonPhysics_SPU.obj
 0001:0004f7f0       ?SPU_Physics_SynchronizeFromEntityArticulated@CSkeletonPhysics@@AEAAXAEAVCPoseData@Skeleton@@M@Z 00000000315507f0 f   SkeletonPhysics_SPU.obj
 0001:0004f880       ?SPU_Physics_SynchronizeFromAux@CSkeletonPhysics@@AEAAXAEAVCPoseData@Skeleton@@@Z 0000000031550880 f   SkeletonPhysics_SPU.obj
 0001:00051230       ?SPU_Physics_SynchronizeFromImpact@CSkeletonPhysics@@AEAAXAEAVCPoseData@Skeleton@@M@Z 0000000031552230 f   SkeletonPhysics_SPU.obj
 0001:00052290       ?SPU_Physics_BlendFromRagdoll@CSkeletonPhysics@@AEAAXAEAVCPoseData@Skeleton@@M@Z 0000000031553290 f   SkeletonPhysics_SPU.obj
 0001:00052890       ?SPU_Physics_SynchronizeFrom@CSkeletonPhysics@@QEAAXAEAVCPoseData@Skeleton@@M@Z 0000000031553890 f   SkeletonPhysics_SPU.obj
 0001:00052a60       ?SetFirstLayer@CTransitionQueue@@QEAAXXZ 0000000031553a60 f   TransitionQueue.obj
 0001:00052a70       ?IsAnimationLoaded@?A0x020955a7@@YA_NAEBVCAnimationSet@@AEBVCAnimation@@@Z 0000000031553a70 f   TransitionQueue.obj
 0001:00052c00       ?TriggerEvents@?A0x020955a7@@YAXPEBDIAEBUIAnimEventList@@MMAEAVCCharInstance@@@Z 0000000031553c00 f   TransitionQueue.obj
 0001:00052d90       ?GetAnimation@CTransitionQueue@@QEBAAEBVCAnimation@@I@Z 0000000031553d90 f   TransitionQueue.obj
 0001:00052d90       ?GetAnimation@CTransitionQueue@@QEAAAEAVCAnimation@@I@Z 0000000031553d90 f   TransitionQueue.obj
 0001:00052dc0       ?ApplyManualMixingWeight@CTransitionQueue@@QEAAXI@Z 0000000031553dc0 f   TransitionQueue.obj
 0001:00052e10       ?TransitionsBetweenSeveralAnimations@CTransitionQueue@@QEAAXI@Z 0000000031553e10 f   TransitionQueue.obj
 0001:00053140       ?AdjustTransitionWeights@CTransitionQueue@@QEAAXI@Z 0000000031554140 f   TransitionQueue.obj
 0001:00053590       ?UpdateTransitionTime@CTransitionQueue@@QEAAXIMMM@Z 0000000031554590 f   TransitionQueue.obj
 0001:00053810       ?AdjustAnimationTimeForTimeWarpedAnimations@CTransitionQueue@@QEAAXI@Z 0000000031554810 f   TransitionQueue.obj
 0001:00053a70       ??1?$shared_ptr@UIAnimationPoseModifier@@@boost@@QEAA@XZ 0000000031554a70 f i TransitionQueue.obj
 0001:00053ab0       ?Prepare@CPoseModifierQueue@@QEAAXAEBUSAnimationPoseModifierParams@@@Z 0000000031554ab0 f   TransitionQueue.obj
 0001:00053b30       ?Synchronize@CPoseModifierQueue@@QEAAXXZ 0000000031554b30 f   TransitionQueue.obj
 0001:00053b90       ??$move_init@VCAnimation@@@NArray@@YAXPEAVCAnimation@@0_K@Z 0000000031554b90 f i TransitionQueue.obj
 0001:00053c00       ?UnloadAnimationAssets@CTransitionQueue@@QEAAXH@Z 0000000031554c00 f   TransitionQueue.obj
 0001:00053e30       ?ManualSeekAnimation@CTransitionQueue@@QEAAXIM_NAEAVCCharInstance@@@Z 0000000031554e30 f   TransitionQueue.obj
 0001:00053f90       ?get_alloc_size@?$SmallDynStorage@USEntry@CPoseModifierQueue@@HUStandardAlloc@NAlloc@@@NArray@@QEBAHXZ 0000000031554f90 f i TransitionQueue.obj
 0001:00053ff0       ?resize_raw@?$SmallDynStorage@VCAnimation@@HUStandardAlloc@NAlloc@@@NArray@@QEAAXHH_N@Z 0000000031554ff0 f i TransitionQueue.obj
 0001:00054180       ??$move_init@USEntry@CPoseModifierQueue@@@NArray@@YAXPEAUSEntry@CPoseModifierQueue@@0_K@Z 0000000031555180 f i TransitionQueue.obj
 0001:00054240       ?GetSize@CPoseModifierQueue@@QEAAIXZ 0000000031555240 f   TransitionQueue.obj
 0001:00054310       ?erase@?$DynArray@VCAnimation@@HU?$SmallDynStorage@VCAnimation@@HUStandardAlloc@NAlloc@@@NArray@@@@QEAAPEAVCAnimation@@PEAV2@0@Z 0000000031555310 f i TransitionQueue.obj
 0001:000543d0       ?destroy@?$DynArray@USEntry@CPoseModifierQueue@@HU?$SmallDynStorage@USEntry@CPoseModifierQueue@@HUStandardAlloc@NAlloc@@@NArray@@@@IEAAXXZ 00000000315553d0 f i TransitionQueue.obj
 0001:00054440       ?resize_raw@?$SmallDynStorage@USEntry@CPoseModifierQueue@@HUStandardAlloc@NAlloc@@@NArray@@QEAAXHH_N@Z 0000000031555440 f i TransitionQueue.obj
 0001:000545c0       ?expand_raw@?$DynArray@VCAnimation@@HU?$SmallDynStorage@VCAnimation@@HUStandardAlloc@NAlloc@@@NArray@@@@IEAAPEAVCAnimation@@PEAV2@H@Z 00000000315555c0 f i TransitionQueue.obj
 0001:00054680       ?expand_raw@?$DynArray@USEntry@CPoseModifierQueue@@HU?$SmallDynStorage@USEntry@CPoseModifierQueue@@HUStandardAlloc@NAlloc@@@NArray@@@@IEAAPEAUSEntry@CPoseModifierQueue@@PEAU23@H@Z 0000000031555680 f i TransitionQueue.obj
 0001:00054740       ??$AddObject@USEntry@CPoseModifierQueue@@HU?$SmallDynStorage@USEntry@CPoseModifierQueue@@HUStandardAlloc@NAlloc@@@NArray@@@ICrySizer@@QEAAXAEBU?$DynArray@USEntry@CPoseModifierQueue@@HU?$SmallDynStorage@USEntry@CPoseModifierQueue@@HUStandardAlloc@NAlloc@@@NArray@@@@@Z 0000000031555740 f i TransitionQueue.obj
 0001:000547f0       ?AddToSizer@CPoseModifierQueue@@QEBAXPEAVICrySizer@@@Z 00000000315557f0 f   TransitionQueue.obj
 0001:00054830       ?clear@?$DynArray@USEntry@CPoseModifierQueue@@HU?$SmallDynStorage@USEntry@CPoseModifierQueue@@HUStandardAlloc@NAlloc@@@NArray@@@@QEAAXXZ 0000000031555830 f i TransitionQueue.obj
 0001:00054910       ?RemoveAnimation@CTransitionQueue@@QEAA_NI_N@Z 0000000031555910 f   TransitionQueue.obj
 0001:000549a0       ??1CPoseModifierQueue@@QEAA@XZ 00000000315559a0 f   TransitionQueue.obj
 0001:00054ae0       ?SwapBuffersAndClearActive@CPoseModifierQueue@@QEAAXXZ 0000000031555ae0 f   TransitionQueue.obj
 0001:00054b10       ?ClearAllPoseModifiers@CPoseModifierQueue@@QEAAXXZ 0000000031555b10 f   TransitionQueue.obj
 0001:00054b30       ?grow@?$DynArray@VCAnimation@@HU?$SmallDynStorage@VCAnimation@@HUStandardAlloc@NAlloc@@@NArray@@@@QEAAPEAVCAnimation@@H@Z 0000000031555b30 f i TransitionQueue.obj
 0001:00054bf0       ?grow@?$DynArray@VCAnimation@@HU?$SmallDynStorage@VCAnimation@@HUStandardAlloc@NAlloc@@@NArray@@@@QEAAPEAVCAnimation@@HAEBV2@@Z 0000000031555bf0 f i TransitionQueue.obj
 0001:00054c70       ??0CTransitionQueue@@QEAA@XZ 0000000031555c70 f   TransitionQueue.obj
 0001:00054d00       ?RemoveDelayConditions@CTransitionQueue@@QEAAXXZ 0000000031555d00 f   TransitionQueue.obj
 0001:00054e00       ??0CPoseModifierQueue@@QEAA@XZ 0000000031555e00 f   TransitionQueue.obj
 0001:00054f10       ?PushAnimation@CTransitionQueue@@QEAAXAEBVCAnimation@@@Z 0000000031555f10 f   TransitionQueue.obj
 0001:00055050       ?Clear@CTransitionQueue@@QEAAXXZ 0000000031556050 f   TransitionQueue.obj
 0001:000550d0       ?Push@CPoseModifierQueue@@QEAA_NV?$shared_ptr@UIAnimationPoseModifier@@@boost@@PEBD_N@Z 00000000315560d0 f   TransitionQueue.obj
 0001:00055260       ?Initialize@CVertexAnimation@@QEAA_NAEAVCSkin@@@Z 0000000031556260 f   VertexAnimation.obj
 0001:000552a0       ?FindMorphTarget@CModelMesh@@QEAAHPEBD@Z 00000000315562a0 f i VertexAnimation.obj
 0001:00055330       ?resize_raw@?$SmallDynStorage@USVertexFrameState@@HUStandardAlloc@NAlloc@@@NArray@@QEAAXHH_N@Z 0000000031556330 f i VertexAnimation.obj
 0001:000554d0       ?clear@?$DynArray@USVertexFrameState@@HU?$SmallDynStorage@USVertexFrameState@@HUStandardAlloc@NAlloc@@@NArray@@@@QEAAXXZ 00000000315564d0 f i VertexAnimation.obj
 0001:000555a0       ?ClearAllFramesWeight@CVertexAnimation@@UEAAXXZ 00000000315565a0 f   VertexAnimation.obj
 0001:000555b0       ??1CVertexAnimation@@UEAA@XZ 00000000315565b0 f   VertexAnimation.obj
 0001:00055620       ??0CVertexAnimation@@QEAA@XZ 0000000031556620 f   VertexAnimation.obj
 0001:000556a0       ??_GCVertexAnimation@@UEAAPEAXI@Z 00000000315566a0 f i VertexAnimation.obj
 0001:000556a0       ??_ECVertexAnimation@@UEAAPEAXI@Z 00000000315566a0 f i VertexAnimation.obj
 0001:00055730       ?SetFrameWeight@CVertexAnimation@@QEAAXAEBUCMorphTarget@@M@Z 0000000031556730 f   VertexAnimation.obj
 0001:00055860       ?SetFrameWeightByName@CVertexAnimation@@UEAAXPEBDM@Z 0000000031556860 f   VertexAnimation.obj
 0001:000558e0       ?Update@CVertexAnimation@@QEAA_NAEAVCVertexData@@@Z 00000000315568e0 f   VertexAnimation.obj
 0001:00055b60       ?Execute@VertexCommandAdd@@SAXAEAU1@PEAU?$Vec3_tpl@M@@@Z 0000000031556b60 f   VertexCommand.obj
 0001:00055ee0       ?Process@CVertexCommandBuffer@@QEAAXPEAU?$Vec3_tpl@M@@@Z 0000000031556ee0 f   VertexCommandBuffer.obj
 0001:00055f50       ?WriteBegin@CVertexData@@QEAAPEAUSVF_P3F@@XZ 0000000031556f50 f   VertexData.obj
 0001:00055f70       ?WriteEnd@CVertexData@@QEAAXXZ 0000000031556f70 f   VertexData.obj
 0001:00055fa0       ??0CVertexData@@QEAA@XZ    0000000031556fa0 f   VertexData.obj
 0001:00056030       ?ReleaseMemory@CVertexData@@QEAAXXZ 0000000031557030 f   VertexData.obj
 0001:00056120       ?Initialize@CVertexData@@QEAA_NI@Z 0000000031557120 f   VertexData.obj
 0001:00056160       ?AllocateMemoryFromRenderMesh@CVertexData@@QEAA_NAEAUIRenderMesh@@@Z 0000000031557160 f   VertexData.obj
 0001:00056230       ??0SRendParams@@QEAA@AEBU0@@Z 0000000031557230 f i _Render.obj
 0001:000563e0       ?MotionBlurMotionCheck@CCharInstance@@QEAA_NI@Z 00000000315573e0 f   _Render.obj
 0001:00056400       ?IsValid@?$Matrix34_tpl@M@@QEBA_NXZ 0000000031557400 f i _Render.obj
 0001:000564c0       ?RenderCGA@CCharInstance@@QEAAXAEBUSRendParams@@AEBU?$Matrix34_tpl@M@@AEBUSRenderingPassInfo@@@Z 00000000315574c0 f   _Render.obj
 0001:00056b00       ?GetSkinningData@CCharInstance@@QEAAPEAUSSkinningData@@PEAVCRenderObject@@AEBUSRenderingPassInfo@@@Z 0000000031557b00 f   _Render.obj
 0001:00056f30       ?RenderCHR@CCharInstance@@QEAAXAEBUSRendParams@@AEBU?$Matrix34_tpl@M@@AEBUSRenderingPassInfo@@@Z 0000000031557f30 f   _Render.obj
 0001:00057440       ?Render@CCharInstance@@UEAAXAEBUSRendParams@@AEBU?$QuatTS_tpl@M@@AEBUSRenderingPassInfo@@PEA_N@Z 0000000031558440 f   _Render.obj
 0001:00058490       ?GetSkinningData@CAttachmentSKIN@@QEAAPEAUSSkinningData@@PEAVCRenderObject@@AEBUSRenderingPassInfo@@_N@Z 0000000031559490 f   _RenderSkins.obj
 0001:00058a00       ?DrawAttachment@CAttachmentSKIN@@UEAAXAEAUSRendParams@@AEBUSRenderingPassInfo@@AEBU?$Matrix34_tpl@M@@M@Z 0000000031559a00 f   _RenderSkins.obj
 0001:0005a280       ?DephysicalizeAttachment@CAttachmentManager@@UEAAXHPEAUIPhysicalEntity@@@Z 000000003155b280 f   AttachmentManager.obj
 0001:0005a300       ?RemoveAttachmentByInterface@CAttachmentManager@@UEAAHPEBUIAttachment@@@Z 000000003155b300 f   AttachmentManager.obj
 0001:0005a330       ?GetInterfaceByName@CAttachmentManager@@UEBAPEAUIAttachment@@PEBD@Z 000000003155b330 f   AttachmentManager.obj
 0001:0005a360       ?GetIAttachmentSkinByName@CAttachmentManager@@UEBAPEAUIAttachmentSkin@@PEBD@Z 000000003155b360 f   AttachmentManager.obj
 0001:0005a390       ?GetIndexByName@CAttachmentManager@@UEBAHPEBD@Z 000000003155b390 f   AttachmentManager.obj
 0001:0005a410       ?GetInterfaceByNameCRC@CAttachmentManager@@UEBAPEAUIAttachment@@I@Z 000000003155b410 f   AttachmentManager.obj
 0001:0005a440       ?GetIndexByNameCRC@CAttachmentManager@@UEBAHI@Z 000000003155b440 f   AttachmentManager.obj
 0001:0005a4b0       ?GetExt@PathUtil@@YAPEBDPEBD@Z 000000003155b4b0 f i AttachmentManager.obj
 0001:0005a510       ??_EIAttachmentObject@@UEAAPEAXI@Z 000000003155b510 f i AttachmentManager.obj
 0001:0005a510       ??_GIAttachmentObject@@UEAAPEAXI@Z 000000003155b510 f i AttachmentManager.obj
 0001:0005a540       ?GetPoseData@CAttachmentManager@@QEAAAEBVCPoseData@Skeleton@@XZ 000000003155b540 f   AttachmentManager.obj
 0001:0005a560       ?Serialize@CAttachmentManager@@QEAAXV?$CSerializeWrapper@UISerialize@@@@@Z 000000003155b560 f   AttachmentManager.obj
 0001:0005a5f0       ??$move_init@V?$_smart_ptr@UIAttachment@@@@@NArray@@YAXPEAV?$_smart_ptr@UIAttachment@@@@0_K@Z 000000003155b5f0 f i AttachmentManager.obj
 0001:0005a660       ?RenderAttachment@CCGFAttachment@@UEAAXAEAUSRendParams@@AEBUSRenderingPassInfo@@@Z 000000003155b660 f i AttachmentManager.obj
 0001:0005a6d0       ?GetAABB@CCGFAttachment@@UEAA?AUAABB@@XZ 000000003155b6d0 f i AttachmentManager.obj
 0001:0005a6f0       ?GetRadiusSqr@CCGFAttachment@@UEAAMXZ 000000003155b6f0 f i AttachmentManager.obj
 0001:0005a710       ?GetBaseMaterial@CCGFAttachment@@UEBAPEAUIMaterial@@XZ 000000003155b710 f i AttachmentManager.obj
 0001:0005a730       ?SetReplacementMaterial@CSKINAttachment@@UEAAXPEAUIMaterial@@@Z 000000003155b730 f i AttachmentManager.obj
 0001:0005a730       ?SetReplacementMaterial@CCGFAttachment@@UEAAXPEAUIMaterial@@@Z 000000003155b730 f i AttachmentManager.obj
 0001:0005a730       ?SetReplacementMaterial@CSKELAttachment@@UEAAXPEAUIMaterial@@@Z 000000003155b730 f i AttachmentManager.obj
 0001:0005a770       ?ProcessAttachment@CSKELAttachment@@UEAAXPEAUIAttachment@@@Z 000000003155b770 f i AttachmentManager.obj
 0001:0005a780       ?GetRadiusSqr@CSKELAttachment@@UEAAMXZ 000000003155b780 f i AttachmentManager.obj
 0001:0005a7a0       ?Release@CSKELAttachment@@UEAAXXZ 000000003155b7a0 f i AttachmentManager.obj
 0001:0005a7d0       ?GetBaseMaterial@CSKELAttachment@@UEBAPEAUIMaterial@@XZ 000000003155b7d0 f i AttachmentManager.obj
 0001:0005a7f0       ?GetFormat@?$CKeyTimesInformationStartStop@MUF32StartStopEncoder@@@@UEAAIXZ 000000003155b7f0 f i ControllerPQ.obj
 0001:0005a7f0       ?GetSplineType@CFacialCameraPathOrientationInterpolator@@UEAA?AW4ESplineType@@XZ 000000003155b7f0 f i FaceAnimSequence.obj
 0001:0005a7f0       ?GetAttachmentType@CSKINAttachment@@UEAA?AW4EType@IAttachmentObject@@XZ 000000003155b7f0 f i AttachmentManager.obj
 0001:0005a7f0       ?GetType@CFacialEffectorBone@@UEAA?AW4EFacialEffectorType@@XZ 000000003155b7f0 f i FaceEffectorLibrary.obj
 0001:0005a7f0       ?GetNumDimensions@CFacialCameraPathPositionInterpolator@@UEAAHXZ 000000003155b7f0 f i FaceAnimSequence.obj
 0001:0005a7f0       ?GetSplineType@CFacialCameraPathPositionInterpolator@@UEAA?AW4ESplineType@@XZ 000000003155b7f0 f i FaceAnimSequence.obj
 0001:0005a800       ?GetRadiusSqr@CSKINAttachment@@UEAAMXZ 000000003155b800 f i AttachmentManager.obj
 0001:0005a800       ?GetStart@IAnimationSet@@UEAAMH@Z 000000003155b800 f i ModelAnimationSet.obj
 0001:0005a810       ?GetIAttachmentSkin@CSKINAttachment@@UEBAPEAUIAttachmentSkin@@XZ 000000003155b810 f i AttachmentManager.obj
 0001:0005a810       ?GetIMaterial_Instance@CCharInstance@@UEBAPEAUIMaterial@@XZ 000000003155b810 f i CharacterInstance.obj
 0001:0005a810       ?GetICharacterInstance@CSKELAttachment@@UEBAPEAUICharacterInstance@@XZ 000000003155b810 f i AttachmentManager.obj
 0001:0005a810       ?GetIStatObj@CCGFAttachment@@UEBAPEAUIStatObj@@XZ 000000003155b810 f i AttachmentManager.obj
 0001:0005a810       ?GetModelFilePath@CSkel@@UEBAPEBDXZ 000000003155b810 f i Model.obj
 0001:0005a810       ?GetTarget@CFacialJoystickChannel@@UEAAPEAXXZ 000000003155b810 f i FaceJoystick.obj
 0001:0005a810       ?GetName@CFacialAnimSkeletalAnimationEntry@@UEBAPEBDXZ 000000003155b810 f i FaceAnimSequence.obj
 0001:0005a810       ?GetSentence@CFacialAnimSoundEntry@@UEAAPEAUIFacialSentence@@XZ 000000003155b810 f i FaceAnimSequence.obj
 0001:0005a820       ?ProcessAttachment@CSKINAttachment@@UEAAXPEAUIAttachment@@@Z 000000003155b820 f i AttachmentManager.obj
 0001:0005a840       ?GetBaseMaterial@CSKINAttachment@@UEBAPEAUIMaterial@@XZ 000000003155b840 f i AttachmentManager.obj
 0001:0005a880       ??0ClosestTri@@QEAA@XZ     000000003155b880 f i AttachmentManager.obj
 0001:0005a940       ??_ECCGFAttachment@@UEAAPEAXI@Z 000000003155b940 f i AttachmentManager.obj
 0001:0005a940       ??_GCCGFAttachment@@UEAAPEAXI@Z 000000003155b940 f i AttachmentManager.obj
 0001:0005a9a0       ?ApplyVisibilityMask@CAttachmentManager@@UEAAXH@Z 000000003155b9a0 f   AttachmentManager.obj
 0001:0005aaa0       ?GetInterfaceByIndex@CAttachmentManager@@UEBAPEAUIAttachment@@I@Z 000000003155baa0 f   AttachmentManager.obj
 0001:0005aad0       ?GetIAttachmentSkinByIndex@CAttachmentManager@@UEBAPEAUIAttachmentSkin@@I@Z 000000003155bad0 f   AttachmentManager.obj
 0001:0005ab20       ?UpdateAllLocations@CAttachmentManager@@QEAAXXZ 000000003155bb20 f   AttachmentManager.obj
 0001:0005ab80       ?UpdateAllAttachedObjects@CAttachmentManager@@QEAAXXZ 000000003155bb80 f   AttachmentManager.obj
 0001:0005ac00       ?UpdateAllLocationsFast@CAttachmentManager@@QEAAXXZ 000000003155bc00 f   AttachmentManager.obj
 0001:0005acc0       ?ProcessAllAttachedObjectsFast@CAttachmentManager@@QEAAXXZ 000000003155bcc0 f   AttachmentManager.obj
 0001:0005ae50       ?DrawAttachments@CAttachmentManager@@QEAAXAEBUSRendParams@@AEBU?$Matrix34_tpl@M@@AEBUSRenderingPassInfo@@@Z 000000003155be50 f   AttachmentManager.obj
 0001:0005b120       ?resize_raw@?$SmallDynStorage@V?$_smart_ptr@UIAttachment@@@@HUStandardAlloc@NAlloc@@@NArray@@QEAAXHH_N@Z 000000003155c120 f i AttachmentManager.obj
 0001:0005b290       ?RenderAttachment@CSKELAttachment@@UEAAXAEAUSRendParams@@AEBUSRenderingPassInfo@@@Z 000000003155c290 f i AttachmentManager.obj
 0001:0005b370       ?GetAABB@CSKELAttachment@@UEAA?AUAABB@@XZ 000000003155c370 f i AttachmentManager.obj
 0001:0005b460       ??_GCSKELAttachment@@UEAAPEAXI@Z 000000003155c460 f i AttachmentManager.obj
 0001:0005b460       ??_ECSKELAttachment@@UEAAPEAXI@Z 000000003155c460 f i AttachmentManager.obj
 0001:0005b4c0       ?GetAABB@CSKINAttachment@@UEAA?AUAABB@@XZ 000000003155c4c0 f i AttachmentManager.obj
 0001:0005b530       ??_GCSKINAttachment@@UEAAPEAXI@Z 000000003155c530 f i AttachmentManager.obj
 0001:0005b530       ??_ECSKINAttachment@@UEAAPEAXI@Z 000000003155c530 f i AttachmentManager.obj
 0001:0005b590       ?set_size@?$SmallDynStorage@UCharacterAttachment@@HUStandardAlloc@NAlloc@@@NArray@@QEAAXH@Z 000000003155c590 f i AttachmentManager.obj
 0001:0005b650       ??0CharacterAttachment@@QEAA@AEBU0@@Z 000000003155c650 f i AttachmentManager.obj
 0001:0005b750       ?InitAttachmentList@CAttachmentManager@@QEAAXAEBU?$DynArray@UCharacterAttachment@@HU?$SmallDynStorage@UCharacterAttachment@@HUStandardAlloc@NAlloc@@@NArray@@@@V?$CryStringT@D@@I@Z 000000003155c750 f   AttachmentManager.obj
 0001:0005c0b0       ?PhysicalizeAttachment@CAttachmentManager@@QEAAXHHPEAUIPhysicalEntity@@AEBU?$Vec3_tpl@M@@@Z 000000003155d0b0 f   AttachmentManager.obj
 0001:0005c790       ?UpdatePhysicalizedAttachment@CAttachmentManager@@QEAAHHPEAUIPhysicalEntity@@AEBU?$QuatT_tpl@M@@@Z 000000003155d790 f   AttachmentManager.obj
 0001:0005cd50       ?pop_back@?$DynArray@V?$_smart_ptr@UIAttachment@@@@HU?$SmallDynStorage@V?$_smart_ptr@UIAttachment@@@@HUStandardAlloc@NAlloc@@@NArray@@@@QEAAXH@Z 000000003155dd50 f i AttachmentManager.obj
 0001:0005cdd0       ?init@?$DynArray@UCharacterAttachment@@HU?$SmallDynStorage@UCharacterAttachment@@HUStandardAlloc@NAlloc@@@NArray@@@@KAPEAUCharacterAttachment@@U?$Array@UCharacterAttachment@@HU?$ArrayStorage@UCharacterAttachment@@H@NArray@@@@AEBU2@@Z 000000003155ddd0 f i AttachmentManager.obj
 0001:0005cf40       ??$AddObject@V?$_smart_ptr@UIAttachment@@@@HU?$SmallDynStorage@V?$_smart_ptr@UIAttachment@@@@HUStandardAlloc@NAlloc@@@NArray@@@ICrySizer@@QEAAXAEBU?$DynArray@V?$_smart_ptr@UIAttachment@@@@HU?$SmallDynStorage@V?$_smart_ptr@UIAttachment@@@@HUStandardAlloc@NAlloc@@@NArray@@@@@Z 000000003155df40 f i AttachmentManager.obj
 0001:0005d090       ??1CharacterAttachment@@QEAA@XZ 000000003155e090 f i AttachmentManager.obj
 0001:0005d140       ??0CAttachmentBONE@@QEAA@XZ 000000003155e140 f i AttachmentManager.obj
 0001:0005d210       ?AddRef@CAttachmentFACE@@UEAAXXZ 000000003155e210 f i AttachmentManager.obj
 0001:0005d210       ?AddRef@CAttachmentBONE@@UEAAXXZ 000000003155e210 f i AttachmentManager.obj
 0001:0005d220       ?GetFlags@CAttachmentBONE@@UEAAIXZ 000000003155e220 f i AttachmentManager.obj
 0001:0005d220       ?GetFlags@CAttachmentFACE@@UEAAIXZ 000000003155e220 f i AttachmentManager.obj
 0001:0005d220       ?GetFlags@CAttachmentSKIN@@UEAAIXZ 000000003155e220 f i Attachment.obj
 0001:0005d230       ?SetFlags@CAttachmentBONE@@UEAAXI@Z 000000003155e230 f i AttachmentManager.obj
 0001:0005d230       ?SetFlags@CAttachmentSKIN@@UEAAXI@Z 000000003155e230 f i Attachment.obj
 0001:0005d230       ?SetForceSkeletonUpdate@CSkeletonPose@@UEAAXH@Z 000000003155e230 f i SkeletonPose.obj
 0001:0005d230       ?SetFlags@CAttachmentFACE@@UEAAXI@Z 000000003155e230 f i AttachmentManager.obj
 0001:0005d240       ?GetAttAbsoluteDefault@CAttachmentBONE@@UEBAAEBU?$QuatT_tpl@M@@XZ 000000003155e240 f i AttachmentManager.obj
 0001:0005d240       ?GetAttAbsoluteDefault@CAttachmentFACE@@UEBAAEBU?$QuatT_tpl@M@@XZ 000000003155e240 f i AttachmentManager.obj
 0001:0005d250       ?GetAttRelativeDefault@CAttachmentBONE@@UEBAAEBU?$QuatT_tpl@M@@XZ 000000003155e250 f i AttachmentManager.obj
 0001:0005d250       ?GetAttRelativeDefault@CAttachmentFACE@@UEBAAEBU?$QuatT_tpl@M@@XZ 000000003155e250 f i AttachmentManager.obj
 0001:0005d260       ?GetBoneID@CAttachmentBONE@@UEBAIXZ 000000003155e260 f i AttachmentManager.obj
 0001:0005d270       ?GetPendulumParams@CAttachmentFACE@@UEAAXAEAHAEAC1AEAM22AEAU?$Vec3_tpl@M@@3@Z 000000003155e270 f i AttachmentManager.obj
 0001:0005d270       ?GetPendulumParams@CAttachmentBONE@@UEAAXAEAHAEAC1AEAM22AEAU?$Vec3_tpl@M@@3@Z 000000003155e270 f i AttachmentManager.obj
 0001:0005d2d0       ?SetPendulumParams@CAttachmentFACE@@UEAAXHCCMMMU?$Vec3_tpl@M@@0@Z 000000003155e2d0 f i AttachmentManager.obj
 0001:0005d2d0       ?SetPendulumParams@CAttachmentBONE@@UEAAXHCCMMMU?$Vec3_tpl@M@@0@Z 000000003155e2d0 f i AttachmentManager.obj
 0001:0005d370       ??_ECAttachmentBONE@@UEAAPEAXI@Z 000000003155e370 f i AttachmentManager.obj
 0001:0005d370       ??_GCAttachmentBONE@@UEAAPEAXI@Z 000000003155e370 f i AttachmentManager.obj
 0001:0005d3e0       ??0CAttachmentFACE@@QEAA@XZ 000000003155e3e0 f i AttachmentManager.obj
 0001:0005d4d0       ?Release@CAttachmentBONE@@UEAAXXZ 000000003155e4d0 f i AttachmentManager.obj
 0001:0005d4d0       ?Release@CAttachmentFACE@@UEAAXXZ 000000003155e4d0 f i AttachmentManager.obj
 0001:0005d4f0       ?HideAttachment@CAttachmentBONE@@UEAAXI@Z 000000003155e4f0 f i AttachmentManager.obj
 0001:0005d4f0       ?HideAttachment@CAttachmentSKIN@@UEAAXI@Z 000000003155e4f0 f i Attachment.obj
 0001:0005d4f0       ?HideAttachment@CAttachmentFACE@@UEAAXI@Z 000000003155e4f0 f i AttachmentManager.obj
 0001:0005d510       ?HideInRecursion@CAttachmentBONE@@UEAAXI@Z 000000003155e510 f i AttachmentManager.obj
 0001:0005d510       ?HideInRecursion@CAttachmentFACE@@UEAAXI@Z 000000003155e510 f i AttachmentManager.obj
 0001:0005d510       ?HideInRecursion@CAttachmentSKIN@@UEAAXI@Z 000000003155e510 f i Attachment.obj
 0001:0005d530       ?IsAttachmentHiddenInRecursion@CAttachmentFACE@@UEAAIXZ 000000003155e530 f i AttachmentManager.obj
 0001:0005d530       ?IsAttachmentHiddenInRecursion@CAttachmentSKIN@@UEAAIXZ 000000003155e530 f i Attachment.obj
 0001:0005d530       ?IsAttachmentHiddenInRecursion@CAttachmentBONE@@UEAAIXZ 000000003155e530 f i AttachmentManager.obj
 0001:0005d540       ?IsAttachmentHiddenInShadow@CAttachmentFACE@@UEAAIXZ 000000003155e540 f i AttachmentManager.obj
 0001:0005d540       ?IsAttachmentHiddenInShadow@CAttachmentBONE@@UEAAIXZ 000000003155e540 f i AttachmentManager.obj
 0001:0005d540       ?IsAttachmentHiddenInShadow@CAttachmentSKIN@@UEAAIXZ 000000003155e540 f i Attachment.obj
 0001:0005d550       ?GetAttModelRelative@CAttachmentBONE@@UEBAAEBU?$QuatT_tpl@M@@XZ 000000003155e550 f i AttachmentManager.obj
 0001:0005d550       ?GetAttModelRelative@CAttachmentFACE@@UEBAAEBU?$QuatT_tpl@M@@XZ 000000003155e550 f i AttachmentManager.obj
 0001:0005d560       ?SetAttAbsoluteDefault@CAttachmentFACE@@UEAAXAEBU?$QuatT_tpl@M@@@Z 000000003155e560 f i AttachmentManager.obj
 0001:0005d560       ?SetAttAbsoluteDefault@CAttachmentBONE@@UEAAXAEBU?$QuatT_tpl@M@@@Z 000000003155e560 f i AttachmentManager.obj
 0001:0005d5a0       ?SetAttRelativeDefault@CAttachmentFACE@@UEAAXAEBU?$QuatT_tpl@M@@@Z 000000003155e5a0 f i AttachmentManager.obj
 0001:0005d5a0       ?SetAttRelativeDefault@CAttachmentBONE@@UEAAXAEBU?$QuatT_tpl@M@@@Z 000000003155e5a0 f i AttachmentManager.obj
 0001:0005d5e0       ??_ECAttachmentFACE@@UEAAPEAXI@Z 000000003155e5e0 f i AttachmentManager.obj
 0001:0005d5e0       ??_GCAttachmentFACE@@UEAAPEAXI@Z 000000003155e5e0 f i AttachmentManager.obj
 0001:0005d650       ?PhysicalizeAttachment@CAttachmentManager@@UEAAXHPEAUIPhysicalEntity@@H@Z 000000003155e650 f   AttachmentManager.obj
 0001:0005d6e0       ?ProjectAllAttachment@CAttachmentManager@@UEAAIXZ 000000003155e6e0 f   AttachmentManager.obj
 0001:0005e5c0       ?RemoveAttachmentByIndex@CAttachmentManager@@QEAAXI@Z 000000003155f5c0 f   AttachmentManager.obj
 0001:0005e6a0       ?RemoveAllAttachments@CAttachmentManager@@QEAAIXZ 000000003155f6a0 f   AttachmentManager.obj
 0001:0005e7b0       ?SizeOfAllAttachments@CAttachmentManager@@QEAA_KXZ 000000003155f7b0 f   AttachmentManager.obj
 0001:0005e880       ?GetMemoryUsage@CAttachmentManager@@QEBAXPEAVICrySizer@@@Z 000000003155f880 f   AttachmentManager.obj
 0001:0005e890       ?append_raw@?$DynArray@V?$_smart_ptr@UIAttachment@@@@HU?$SmallDynStorage@V?$_smart_ptr@UIAttachment@@@@HUStandardAlloc@NAlloc@@@NArray@@@@QEAA?AU?$Array@V?$_smart_ptr@UIAttachment@@@@HU?$ArrayStorage@V?$_smart_ptr@UIAttachment@@@@H@NArray@@@@H@Z 000000003155f890 f i AttachmentManager.obj
 0001:0005e950       ?RemoveAttachmentByName@CAttachmentManager@@UEAAHPEBD@Z 000000003155f950 f   AttachmentManager.obj
 0001:0005e990       ?RemoveAttachmentByNameCRC@CAttachmentManager@@UEAAHI@Z 000000003155f990 f   AttachmentManager.obj
 0001:0005e9d0       ??$move_init@UCharacterAttachment@@@NArray@@YAXPEAUCharacterAttachment@@0_K@Z 000000003155f9d0 f i AttachmentManager.obj
 0001:0005ea40       ?ReName@CAttachmentSKIN@@UEAAIPEBDI@Z 000000003155fa40 f i Attachment.obj
 0001:0005ea40       ?ReName@CAttachmentFACE@@UEAAIPEBDI@Z 000000003155fa40 f i AttachmentManager.obj
 0001:0005ea40       ?ReName@CAttachmentBONE@@UEAAIPEBDI@Z 000000003155fa40 f i AttachmentManager.obj
 0001:0005eb10       ?CreateXMLAttachmentList@CAttachmentManager@@QEAAIVXmlNodeRef@@@Z 000000003155fb10 f   AttachmentManager.obj
 0001:0005f450       ?resize_raw@?$SmallDynStorage@UCharacterAttachment@@HUStandardAlloc@NAlloc@@@NArray@@QEAAXHH_N@Z 0000000031560450 f i AttachmentManager.obj
 0001:0005f5e0       ??0CAttachmentSKIN@@QEAA@XZ 00000000315605e0 f i AttachmentManager.obj
 0001:0005f6f0       ?SaveAttachmentList@CAttachmentManager@@UEAAIPEBD@Z 00000000315606f0 f   AttachmentManager.obj
 0001:0005f780       ?CreateAttachment@CAttachmentManager@@UEAAPEAUIAttachment@@PEBDI0_N@Z 0000000031560780 f   AttachmentManager.obj
 0001:0005fb40       ?expand_raw@?$DynArray@UCharacterAttachment@@HU?$SmallDynStorage@UCharacterAttachment@@HUStandardAlloc@NAlloc@@@NArray@@@@IEAAPEAUCharacterAttachment@@PEAU2@H@Z 0000000031560b40 f i AttachmentManager.obj
 0001:0005fc00       ??1?$DynArray@UCharacterAttachment@@HU?$SmallDynStorage@UCharacterAttachment@@HUStandardAlloc@NAlloc@@@NArray@@@@QEAA@XZ 0000000031560c00 f i AttachmentManager.obj
 0001:0005fc80       ?ParseXMLAttachmentList@CAttachmentManager@@SAXAEAU?$DynArray@UCharacterAttachment@@HU?$SmallDynStorage@UCharacterAttachment@@HUStandardAlloc@NAlloc@@@NArray@@@@VXmlNodeRef@@@Z 0000000031560c80 f   AttachmentManager.obj
 0001:00060870       ?LoadAttachmentList@CAttachmentManager@@UEAAIPEBD@Z 0000000031561870 f   AttachmentManager.obj
 0001:00060a20       ?KillAllSkeletonEffects@CCharInstance@@UEAAXXZ 0000000031561a20 f i CharacterInstance.obj
 0001:00060a30       ?Release@CharacterManager@@UEAAXXZ 0000000031561a30 f   CharacterManager.obj
 0001:00060a30       ?DeleteThis@CCharInstance@@UEAAXXZ 0000000031561a30 f   CharacterInstance.obj
 0001:00060a30       ?destroy@sp_counted_base@detail@boost@@UEAAXXZ 0000000031561a30 f   OperatorQueue.obj
 0001:00060a30       ?Release@CCGFAttachment@@UEAAXXZ 0000000031561a30 f   AttachmentManager.obj
 0001:00060a30       ?Release@CSKINAttachment@@UEAAXXZ 0000000031561a30 f   AttachmentManager.obj
 0001:00060a50       ?LipSyncWithSound@CCharInstance@@UEAAXI_N@Z 0000000031561a50 f   CharacterInstance.obj
 0001:00060a90       ?EnableProceduralFacialAnimation@CCharInstance@@UEAAX_N@Z 0000000031561a90 f   CharacterInstance.obj
 0001:00060ac0       ??_GICharacterInstance@@UEAAPEAXI@Z 0000000031561ac0 f i CharacterInstance.obj
 0001:00060ac0       ??_EICharacterInstance@@UEAAPEAXI@Z 0000000031561ac0 f i CharacterInstance.obj
 0001:00060af0       ?GetFilePath@CCharInstance@@UEAAPEBDXZ 0000000031561af0 f i CharacterInstance.obj
 0001:00060b00       ?CopyPoseFrom@CCharInstance@@UEAAXAEBUICharacterInstance@@@Z 0000000031561b00 f   CharacterInstance.obj
 0001:00060b50       ?GetAABB@CCharInstance@@UEAAAEBUAABB@@XZ 0000000031561b50 f   CharacterInstance.obj
 0001:00060b60       ??$move_init@M@NArray@@YAXPEAM0_K@Z 0000000031561b60 f i CharacterInstance.obj
 0001:00060c00       ?GetRandomPart@GeomQuery@@QEBAHXZ 0000000031561c00 f i CharacterInstance.obj
 0001:00060d20       ?BoxRandomPos@@YAXAEAURandomPos@@W4EGeomForm@@AEBU?$Vec3_tpl@M@@@Z 0000000031561d20 f i CharacterInstance.obj
 0001:00061010       ?StartAnimationProcessing@CCharInstance@@UEAAXAEBUSAnimationProcessParams@@@Z 0000000031562010 f   CharacterInstance.obj
 0001:00061430       ?GetRadiusSqr@CCharInstance@@UEAAMXZ 0000000031562430 f   CharacterInstance.obj
 0001:000614a0       ?OnDetach@CCharInstance@@UEAAXXZ 00000000315624a0 f   CharacterInstance.obj
 0001:000614f0       ?Serialize@CCharInstance@@UEAAXV?$CSerializeWrapper@UISerialize@@@@@Z 00000000315624f0 f   CharacterInstance.obj
 0001:000615c0       ?EnableFacialAnimation@CCharInstance@@UEAAX_N@Z 00000000315625c0 f   CharacterInstance.obj
 0001:00061660       ?ProcessAttachment@CCharInstance@@UEAAXPEAUIAttachment@@@Z 0000000031562660 f   CharacterInstance.obj
 0001:00061940       ?resize_raw@?$SmallDynStorage@MHUStandardAlloc@NAlloc@@@NArray@@QEAAXHH_N@Z 0000000031562940 f i CharacterInstance.obj
 0001:00061ab0       ?set_size@?$SmallDynStorage@HHUStandardAlloc@NAlloc@@@NArray@@QEAAXH@Z 0000000031562ab0 f i SkeletonPhysics.obj
 0001:00061ab0       ?set_size@?$SmallDynStorage@IHUStandardAlloc@NAlloc@@@NArray@@QEAAXH@Z 0000000031562ab0 f i CharacterManager.obj
 0001:00061ab0       ?set_size@?$SmallDynStorage@MHUStandardAlloc@NAlloc@@@NArray@@QEAAXH@Z 0000000031562ab0 f i CharacterInstance.obj
 0001:00061ab0       ?set_size@?$SmallDynStorage@UCControllerType@@HUStandardAlloc@NAlloc@@@NArray@@QEAAXH@Z 0000000031562ab0 f i LoaderCGA.obj
 0001:00061b50       ?destroy@?$DynArray@UGeomQuery@@HU?$SmallDynStorage@UGeomQuery@@HUStandardAlloc@NAlloc@@@NArray@@@@KAXU?$Array@UGeomQuery@@HU?$ArrayStorage@UGeomQuery@@H@NArray@@@@@Z 0000000031562b50 f i CharacterInstance.obj
 0001:00061b90       ?resize_raw@?$SmallDynStorage@_NHUStandardAlloc@NAlloc@@@NArray@@QEAAXHH_N@Z 0000000031562b90 f i CharacterInstance.obj
 0001:00061d10       ?ApplyJointVelocitiesToPhysics@CCharInstance@@QEAAXPEAUIPhysicalEntity@@AEBU?$Quat_tpl@M@@AEBU?$Vec3_tpl@M@@@Z 0000000031562d10 f   CharacterInstance.obj
 0001:000629e0       ?SkinningTransformationsComputation@CCharInstance@@QEAAXPEAUSSkinningData@@PEAVCSkel@@HPEBVCPoseData@Skeleton@@PEAM@Z 00000000315639e0 f   CharacterInstance.obj
 0001:00063620       ?destroy@?$DynArray@UGeomQuery@@HU?$SmallDynStorage@UGeomQuery@@HUStandardAlloc@NAlloc@@@NArray@@@@IEAAXXZ 0000000031564620 f i CharacterInstance.obj
 0001:00063670       ?append_raw@?$DynArray@MHU?$SmallDynStorage@MHUStandardAlloc@NAlloc@@@NArray@@@@QEAA?AU?$Array@MHU?$ArrayStorage@MH@NArray@@@@H@Z 0000000031564670 f i CharacterInstance.obj
 0001:00063730       ?replace@?$CryStringT@D@@QEAAAEAV1@PEBD0@Z 0000000031564730 f i CharacterInstance.obj
 0001:00063960       ??$AddObject@V?$CryStringT@D@@HU?$SmallDynStorage@V?$CryStringT@D@@HUStandardAlloc@NAlloc@@@NArray@@@ICrySizer@@QEAAXAEBU?$DynArray@V?$CryStringT@D@@HU?$SmallDynStorage@V?$CryStringT@D@@HUStandardAlloc@NAlloc@@@NArray@@@@@Z 0000000031564960 f i CharacterInstance.obj
 0001:00063ab0       ?Invoke@?$SGenInvokerTSkinningTransformationsComputation@VCCharInstance@@PEAUSSkinningData@@PEAVCSkel@@HPEBVCPoseData@Skeleton@@PEAMUSNullType@Detail@JobManager@@U678@U678@U678@U678@U678@U678@@Detail@JobManager@@SAXPEAX@Z 0000000031564ab0 f i CharacterInstance.obj
 0001:00063ae0       ?SizeOfThis@CFacialInstance@@QEAAIXZ 0000000031564ae0 f i CharacterInstance.obj
 0001:00063b50       ?UpdatePhysicsCGA@CCharInstance@@QEAAXAEAVCPoseData@Skeleton@@MAEBU?$QuatTS_tpl@M@@@Z 0000000031564b50 f   CharacterInstance.obj
 0001:00064500       ?SizeOfCharInstance@CCharInstance@@UEAA_KXZ 0000000031565500 f   CharacterInstance.obj
 0001:00064780       ?clear@?$DynArray@MHU?$SmallDynStorage@MHUStandardAlloc@NAlloc@@@NArray@@@@QEAAXXZ 0000000031565780 f i CharacterInstance.obj
 0001:00064850       ?append_raw@?$DynArray@_NHU?$SmallDynStorage@_NHUStandardAlloc@NAlloc@@@NArray@@@@QEAA?AU?$Array@_NHU?$ArrayStorage@_NH@NArray@@@@H@Z 0000000031565850 f i CharacterInstance.obj
 0001:00064900       ?destroy@?$DynArray@V?$CryStringT@D@@HU?$SmallDynStorage@V?$CryStringT@D@@HUStandardAlloc@NAlloc@@@NArray@@@@KAXU?$Array@V?$CryStringT@D@@HU?$ArrayStorage@V?$CryStringT@D@@H@NArray@@@@@Z 0000000031565900 f i CharacterInstance.obj
 0001:00064970       ?GetMemoryUsage@CCharInstance@@UEBAXPEAVICrySizer@@@Z 0000000031565970 f   CharacterInstance.obj
 0001:00064c80       ??1?$DynArray@UGeomQuery@@HU?$SmallDynStorage@UGeomQuery@@HUStandardAlloc@NAlloc@@@NArray@@@@QEAA@XZ 0000000031565c80 f i CharacterInstance.obj
 0001:00064d00       ??1?$DynArray@V?$_smart_ptr@UIAttachment@@@@HU?$SmallDynStorage@V?$_smart_ptr@UIAttachment@@@@HUStandardAlloc@NAlloc@@@NArray@@@@QEAA@XZ 0000000031565d00 f i CharacterInstance.obj
 0001:00064d80       ?pop_back@?$DynArray@V?$CryStringT@D@@HU?$SmallDynStorage@V?$CryStringT@D@@HUStandardAlloc@NAlloc@@@NArray@@@@QEAAXH@Z 0000000031565d80 f i CharacterInstance.obj
 0001:00064e20       ??$move_init@V?$CryStringT@D@@@NArray@@YAXPEAV?$CryStringT@D@@0_K@Z 0000000031565e20 f i CharacterInstance.obj
 0001:00064ec0       ??0?$DynArray@MHU?$SmallDynStorage@MHUStandardAlloc@NAlloc@@@NArray@@@@QEAA@AEBU0@@Z 0000000031565ec0 f i CharacterInstance.obj
 0001:00064f80       ??1CryCHRLoader@@QEAA@XZ   0000000031565f80 f i CharacterInstance.obj
 0001:00065020       ?BeginSkinningTransformationsComputation@CCharInstance@@QEAAXPEAUSSkinningData@@@Z 0000000031566020 f   CharacterInstance.obj
 0001:00065180       ??_GGeomQuery@@QEAAPEAXI@Z 0000000031566180 f i CharacterInstance.obj
 0001:000651f0       ?resize_raw@?$SmallDynStorage@V?$CryStringT@D@@HUStandardAlloc@NAlloc@@@NArray@@QEAAXHH_N@Z 00000000315661f0 f i CharacterInstance.obj
 0001:00065360       ??1?$DynArray@V?$CryStringT@D@@HU?$SmallDynStorage@V?$CryStringT@D@@HUStandardAlloc@NAlloc@@@NArray@@@@QEAA@XZ 0000000031566360 f i CharacterInstance.obj
 0001:00065400       ??0GeomQuery@@QEAA@XZ      0000000031566400 f i CharacterInstance.obj
 0001:000654c0       ??0CAttachmentManager@@QEAA@XZ 00000000315664c0 f i CharacterInstance.obj
 0001:00065540       ?GetCount@CAnimEventList@@UEBAIXZ 0000000031566540 f i AnimEventList.obj
 0001:00065540       ?GetAttachmentCount@CAttachmentManager@@UEBAHXZ 0000000031566540 f i CharacterInstance.obj
 0001:00065550       ??_GCAttachmentManager@@UEAAPEAXI@Z 0000000031566550 f i CharacterInstance.obj
 0001:00065550       ??_ECAttachmentManager@@UEAAPEAXI@Z 0000000031566550 f i CharacterInstance.obj
 0001:00065590       ??0CryCHRLoader@@QEAA@XZ   0000000031566590 f i CharacterInstance.obj
 0001:00065660       ?ReloadCHRPARAMS@CCharInstance@@UEAAXXZ 0000000031566660 f   CharacterInstance.obj
 0001:00065a00       ??$move_init@UGeomQuery@@@NArray@@YAXPEAUGeomQuery@@0_K@Z 0000000031566a00 f i CharacterInstance.obj
 0001:00065be0       ??$__destroy_range_aux@V?$reverse_iterator@PEAVCAnimDecal@@@stlpmtx_std@@VCAnimDecal@@@stlpmtx_std@@YAXV?$reverse_iterator@PEAVCAnimDecal@@@0@0PEAVCAnimDecal@@AEBU__false_type@0@@Z 0000000031566be0 f i CharacterInstance.obj
 0001:00065d60       ?resize_raw@?$SmallDynStorage@UGeomQuery@@HUStandardAlloc@NAlloc@@@NArray@@QEAAXHH_N@Z 0000000031566d60 f i CharacterInstance.obj
 0001:00065ee0       ?append_raw@?$DynArray@V?$CryStringT@D@@HU?$SmallDynStorage@V?$CryStringT@D@@HUStandardAlloc@NAlloc@@@NArray@@@@QEAA?AU?$Array@V?$CryStringT@D@@HU?$ArrayStorage@V?$CryStringT@D@@H@NArray@@@@H@Z 0000000031566ee0 f i CharacterInstance.obj
 0001:00065fa0       ?expand_raw@?$DynArray@UGeomQuery@@HU?$SmallDynStorage@UGeomQuery@@HUStandardAlloc@NAlloc@@@NArray@@@@IEAAPEAUGeomQuery@@PEAU2@H@Z 0000000031566fa0 f i CharacterInstance.obj
 0001:00066060       ?clear@?$DynArray@UGeomQuery@@HU?$SmallDynStorage@UGeomQuery@@HUStandardAlloc@NAlloc@@@NArray@@@@QEAAXXZ 0000000031567060 f i CharacterInstance.obj
 0001:00066260       ?grow@?$DynArray@UGeomQuery@@HU?$SmallDynStorage@UGeomQuery@@HUStandardAlloc@NAlloc@@@NArray@@@@QEAAPEAUGeomQuery@@H@Z 0000000031567260 f i CharacterInstance.obj
 0001:000662d0       ??$GetExtent@UIStatObj@@@GeomQuery@@QEAAMPEAUIStatObj@@W4EGeomForm@@@Z 00000000315672d0 f i CharacterInstance.obj
 0001:00066350       ??$GetExtent@VCCharInstance@@@GeomQuery@@QEAAMPEAVCCharInstance@@W4EGeomForm@@@Z 0000000031567350 f i CharacterInstance.obj
 0001:000663d0       ??0?$DynArray@UGeomQuery@@HU?$SmallDynStorage@UGeomQuery@@HUStandardAlloc@NAlloc@@@NArray@@@@QEAA@AEBU0@@Z 00000000315673d0 f i CharacterInstance.obj
 0001:00066490       ?GetRandomPos@CCharInstance@@UEAAXAEAURandomPos@@AEAUGeomQuery@@W4EGeomForm@@@Z 0000000031567490 f   CharacterInstance.obj
 0001:00066780       ?resize@?$DynArray@UGeomQuery@@HU?$SmallDynStorage@UGeomQuery@@HUStandardAlloc@NAlloc@@@NArray@@@@QEAAXH@Z 0000000031567780 f i CharacterInstance.obj
 0001:00066970       ??0GeomQuery@@QEAA@AEBU0@@Z 0000000031567970 f i CharacterInstance.obj
 0001:000669c0       ?init@?$DynArray@UGeomQuery@@HU?$SmallDynStorage@UGeomQuery@@HUStandardAlloc@NAlloc@@@NArray@@@@KAPEAUGeomQuery@@U?$Array@UGeomQuery@@HU?$ArrayStorage@UGeomQuery@@H@NArray@@@@PEBU2@@Z 00000000315679c0 f i CharacterInstance.obj
 0001:00066a70       ??0CAnimDecalManager@@QEAA@XZ 0000000031567a70 f i CharacterInstance.obj
 0001:00066ae0       ??1CAnimDecalManager@@QEAA@XZ 0000000031567ae0 f i CharacterInstance.obj
 0001:00066b70       ??0CCharInstance@@QEAA@AEBV?$CryStringT@D@@PEAVCSkel@@@Z 0000000031567b70 f   CharacterInstance.obj
 0001:000674a0       ?GetIAttachmentManager@CCharInstance@@UEAAPEAUIAttachmentManager@@XZ 00000000315684a0 f i CharacterInstance.obj
 0001:000674b0       ?GetAverageFrameTime@CCharInstance@@UEAAMXZ 00000000315684b0 f i CharacterInstance.obj
 0001:000674c0       ?SetUniformScale@CCharInstance@@UEAAXAEBM@Z 00000000315684c0 f i CharacterInstance.obj
 0001:000674d0       ?GetUniformScale@CCharInstance@@UEBAMXZ 00000000315684d0 f i CharacterInstance.obj
 0001:000674e0       ?EnableDecals@CCharInstance@@UEAAXI@Z 00000000315684e0 f i CharacterInstance.obj
 0001:00067500       ?GetISkeletonAnim@CCharInstance@@UEAAPEAUISkeletonAnim@@XZ 0000000031568500 f i CharacterInstance.obj
 0001:00067510       ?FinishAnimationComputations@CCharInstance@@UEAAXXZ 0000000031568510 f i CharacterInstance.obj
 0001:00067520       ?EnableStartAnimation@CCharInstance@@UEAAX_N@Z 0000000031568520 f i CharacterInstance.obj
 0001:00067530       ?GetResetMode@CCharInstance@@UEAAIXZ 0000000031568530 f i CharacterInstance.obj
 0001:00067540       ?SetResetMode@CCharInstance@@UEAAXI@Z 0000000031568540 f i CharacterInstance.obj
 0001:00067550       ?SetCharEditMode@CCharInstance@@UEAAXI@Z 0000000031568550 f i CharacterInstance.obj
 0001:00067560       ?GetCharEditMode@CCharInstance@@UEBA_NXZ 0000000031568560 f i CharacterInstance.obj
 0001:00067570       ?HideMaster@CCharInstance@@UEAAXI@Z 0000000031568570 f i CharacterInstance.obj
 0001:00067590       ?IsCharacterVisible@CCharInstance@@UEAAIXZ 0000000031568590 f i CharacterInstance.obj
 0001:000675a0       ?IsAnimationGraphValid@CCharInstance@@UEAA_NXZ 00000000315685a0 f i CharacterInstance.obj
 0001:000675c0       ?SetForceLOD@CCharInstance@@UEAAX_N@Z 00000000315685c0 f i CharacterInstance.obj
 0001:000675d0       ?SetForceLODNum@CCharInstance@@UEAAXH@Z 00000000315685d0 f i CharacterInstance.obj
 0001:000675e0       ?GetPlaybackScale@CCharInstance@@UEAAMXZ 00000000315685e0 f i CharacterInstance.obj
 0001:000675f0       ?SpawnSkeletonEffect@CCharInstance@@UEAAXHPEBD00AEBU?$Vec3_tpl@M@@1AEBU?$Matrix34_tpl@M@@@Z 00000000315685f0 f i CharacterInstance.obj
 0001:00067680       ?SetFlags@CCharInstance@@UEAAXH@Z 0000000031568680 f i CharacterInstance.obj
 0001:00067690       ?GetFlags@CCharInstance@@UEAAHXZ 0000000031568690 f i CharacterInstance.obj
 0001:000676a0       ?AddRef@CCharInstance@@UEAAXXZ 00000000315686a0 f i CharacterInstance.obj
 0001:000676b0       ?GetRefCount@CCharInstance@@UEBAHXZ 00000000315686b0 f i CharacterInstance.obj
 0001:000676c0       ?GetIAnimationSet@CCharInstance@@UEAAPEAUIAnimationSet@@XZ 00000000315686c0 f i CharacterInstance.obj
 0001:000676d0       ?GetOjectType@CCharInstance@@UEAAHXZ 00000000315686d0 f i CharacterInstance.obj
 0001:000676e0       ?SetIMaterial_Instance@CCharInstance@@UEAAXPEAUIMaterial@@@Z 00000000315686e0 f i CharacterInstance.obj
 0001:00067720       ?SetPlaybackScale@CCharInstance@@UEAAXM@Z 0000000031568720 f i CharacterInstance.obj
 0001:00067740       ?Release@CCharInstance@@UEAAXXZ 0000000031568740 f i CharacterInstance.obj
 0001:00067790       ?GetModelAnimEventDatabase@CCharInstance@@UEAAPEBDXZ 0000000031568790 f i CharacterInstance.obj
 0001:000677a0       ?GetIMaterial@CCharInstance@@UEBAPEAUIMaterial@@XZ 00000000315687a0 f i CharacterInstance.obj
 0001:000677d0       ?SetAttachmentLocation_DEPRECATED@CCharInstance@@UEAAXAEBU?$QuatTS_tpl@M@@@Z 00000000315687d0 f i CharacterInstance.obj
 0001:00067820       ?GetIgnoreScaleForJoint@CCharInstance@@UEBA_NI@Z 0000000031568820 f i CharacterInstance.obj
 0001:00067830       ?GetIsCustomScaleForJoint@CCharInstance@@UEBA_NI@Z 0000000031568830 f i CharacterInstance.obj
 0001:00067840       ?GetCustomScaleForJoint@CCharInstance@@UEBAMI@Z 0000000031568840 f i CharacterInstance.obj
 0001:00067850       ?SetCustomScaleForJoint@CCharInstance@@UEAAXI_NM@Z 0000000031568850 f i CharacterInstance.obj
 0001:00067870       ?DrawWireframeStatic@CCharInstance@@UEAAXAEBU?$Matrix34_tpl@M@@HI@Z 0000000031568870 f i CharacterInstance.obj
 0001:000678f0       ??1CCharInstance@@MEAA@XZ  00000000315688f0 f   CharacterInstance.obj
 0001:00067ac0       ?ComputeExtent@CCharInstance@@UEAAMAEAUGeomQuery@@W4EGeomForm@@@Z 0000000031568ac0 f   CharacterInstance.obj
 0001:00067cb0       ??_ECCharInstance@@MEAAPEAXI@Z 0000000031568cb0 f i CharacterInstance.obj
 0001:00067cb0       ??_GCCharInstance@@MEAAPEAXI@Z 0000000031568cb0 f i CharacterInstance.obj
 0001:00067ce0       ??$AddObject@UTFace@@V?$allocator@UTFace@@@stlpmtx_std@@@ICrySizer@@QEAAXAEBV?$vector@UTFace@@V?$allocator@UTFace@@@stlpmtx_std@@@stlpmtx_std@@@Z 0000000031568ce0 f i DecalManager.obj
 0001:00067d70       ??$AddObject@UCDecalVertex@@V?$allocator@UCDecalVertex@@@stlpmtx_std@@@ICrySizer@@QEAAXAEBV?$vector@UCDecalVertex@@V?$allocator@UCDecalVertex@@@stlpmtx_std@@@stlpmtx_std@@@Z 0000000031568d70 f i DecalManager.obj
 0001:00067e10       ??$AddObject@UCryEngineDecalInfo@@V?$allocator@UCryEngineDecalInfo@@@stlpmtx_std@@@ICrySizer@@QEAAXAEBV?$vector@UCryEngineDecalInfo@@V?$allocator@UCryEngineDecalInfo@@@stlpmtx_std@@@stlpmtx_std@@@Z 0000000031568e10 f i DecalManager.obj
 0001:00067eb0       ?SizeOfThis@CAnimDecalManager@@QEAA_KXZ 0000000031568eb0 f   DecalManager.obj
 0001:00067f90       ??$AddObject@VCAnimDecal@@V?$allocator@VCAnimDecal@@@stlpmtx_std@@@ICrySizer@@QEAAXAEBV?$vector@VCAnimDecal@@V?$allocator@VCAnimDecal@@@stlpmtx_std@@@stlpmtx_std@@@Z 0000000031568f90 f i DecalManager.obj
 0001:00068060       ?GetMemoryUsage@CAnimDecalManager@@QEBAXPEAVICrySizer@@@Z 0000000031569060 f   DecalManager.obj
 0001:000680a0       ?SelectRandomPathExpansion@PathExpansion@@YAXPEBDPEAD@Z 00000000315690a0 f   PathExpansion.obj
 0001:00068210       ?EnumeratePathExpansions@PathExpansion@@YAXPEBDP6AXPEAX0@Z1@Z 0000000031569210 f   PathExpansion.obj
 0001:000685e0       ??0EffectEntry@CSkeletonEffectManager@@QEAA@V?$_smart_ptr@UIParticleEffect@@@@V?$_smart_ptr@UIParticleEmitter@@@@HAEBU?$Vec3_tpl@M@@2H@Z 00000000315695e0 f   SkeletonEffectManager.obj
 0001:000686c0       ?IsPlayingEffect@CSkeletonEffectManager@@AEAA_NPEBD@Z 00000000315696c0 f   SkeletonEffectManager.obj
 0001:00068750       ??0EffectEntry@CSkeletonEffectManager@@QEAA@AEBU01@@Z 0000000031569750 f i SkeletonEffectManager.obj
 0001:000687d0       ?Spawn@IParticleEffect@@QEAAPEAUIParticleEmitter@@_NAEBU?$Matrix34_tpl@M@@@Z 00000000315697d0 f i SkeletonEffectManager.obj
 0001:00068c00       ?GetEffectTM@CSkeletonEffectManager@@AEAAXPEAUISkeletonPose@@AEAU?$Matrix34_tpl@M@@HAEBU?$Vec3_tpl@M@@2AEBU3@@Z 0000000031569c00 f   SkeletonEffectManager.obj
 0001:00069450       ?init@?$DynArray@UEffectEntry@CSkeletonEffectManager@@HU?$SmallDynStorage@UEffectEntry@CSkeletonEffectManager@@HUStandardAlloc@NAlloc@@@NArray@@@@KAPEAUEffectEntry@CSkeletonEffectManager@@U?$Array@UEffectEntry@CSkeletonEffectManager@@HU?$ArrayStorage@UEffectEntry@CSkeletonEffectManager@@H@NArray@@@@AEBU23@@Z 000000003156a450 f i SkeletonEffectManager.obj
 0001:00069510       ??$move_init@UEffectEntry@CSkeletonEffectManager@@@NArray@@YAXPEAUEffectEntry@CSkeletonEffectManager@@0_K@Z 000000003156a510 f i SkeletonEffectManager.obj
 0001:000695c0       ?destroy@?$DynArray@UEffectEntry@CSkeletonEffectManager@@HU?$SmallDynStorage@UEffectEntry@CSkeletonEffectManager@@HUStandardAlloc@NAlloc@@@NArray@@@@IEAAXXZ 000000003156a5c0 f i SkeletonEffectManager.obj
 0001:00069660       ?resize_raw@?$SmallDynStorage@UEffectEntry@CSkeletonEffectManager@@HUStandardAlloc@NAlloc@@@NArray@@QEAAXHH_N@Z 000000003156a660 f i SkeletonEffectManager.obj
 0001:000697f0       ?pop_back@?$DynArray@UEffectEntry@CSkeletonEffectManager@@HU?$SmallDynStorage@UEffectEntry@CSkeletonEffectManager@@HUStandardAlloc@NAlloc@@@NArray@@@@QEAAXH@Z 000000003156a7f0 f i SkeletonEffectManager.obj
 0001:000698c0       ?expand_raw@?$DynArray@UEffectEntry@CSkeletonEffectManager@@HU?$SmallDynStorage@UEffectEntry@CSkeletonEffectManager@@HUStandardAlloc@NAlloc@@@NArray@@@@IEAAPEAUEffectEntry@CSkeletonEffectManager@@PEAU23@H@Z 000000003156a8c0 f i SkeletonEffectManager.obj
 0001:00069980       ?erase@?$DynArray@UEffectEntry@CSkeletonEffectManager@@HU?$SmallDynStorage@UEffectEntry@CSkeletonEffectManager@@HUStandardAlloc@NAlloc@@@NArray@@@@QEAAPEAUEffectEntry@CSkeletonEffectManager@@PEAU23@0@Z 000000003156a980 f i SkeletonEffectManager.obj
 0001:00069ae0       ?KillAllEffects@CSkeletonEffectManager@@QEAAXXZ 000000003156aae0 f   SkeletonEffectManager.obj
 0001:00069c70       ??0CSkeletonEffectManager@@QEAA@XZ 000000003156ac70 f   SkeletonEffectManager.obj
 0001:00069cd0       ??1CSkeletonEffectManager@@QEAA@XZ 000000003156acd0 f   SkeletonEffectManager.obj
 0001:00069d20       ?Update@CSkeletonEffectManager@@QEAAXPEAUISkeletonAnim@@PEAUISkeletonPose@@AEBU?$Matrix34_tpl@M@@@Z 000000003156ad20 f   SkeletonEffectManager.obj
 0001:00069f50       ?push_back@?$DynArray@UEffectEntry@CSkeletonEffectManager@@HU?$SmallDynStorage@UEffectEntry@CSkeletonEffectManager@@HUStandardAlloc@NAlloc@@@NArray@@@@QEAAPEAUEffectEntry@CSkeletonEffectManager@@AEBU23@@Z 000000003156af50 f i SkeletonEffectManager.obj
 0001:00069fb0       ?SpawnEffect@CSkeletonEffectManager@@QEAAXPEAUISkeletonPose@@HPEBD11AEBU?$Vec3_tpl@M@@2AEBU?$Matrix34_tpl@M@@@Z 000000003156afb0 f   SkeletonEffectManager.obj
 0001:0006a240       ?GetPoseDataWriteable@CSkeletonPose@@QEAAPEAVCPoseData@Skeleton@@XZ 000000003156b240 f   SkeletonPose.obj
 0001:0006a250       ?GetPoseDataForceWriteable@CSkeletonPose@@QEAAAEAVCPoseData@Skeleton@@XZ 000000003156b250 f   SkeletonPose.obj
 0001:0006a280       ?SynchronizePoseDataAndLocatorWriteables@CSkeletonPose@@QEAAXXZ 000000003156b280 f   SkeletonPose.obj
 0001:0006a2d0       ?SetDefaultPose@CSkeletonPose@@UEAAXXZ 000000003156b2d0 f   SkeletonPose.obj
 0001:0006a2e0       ??_GISkeletonPhysics@@UEAAPEAXI@Z 000000003156b2e0 f i SkeletonPose.obj
 0001:0006a2e0       ??_EISkeletonPhysics@@UEAAPEAXI@Z 000000003156b2e0 f i SkeletonPose.obj
 0001:0006a310       ?PreparePoseDataAndLocatorWriteables@CSkeletonPose@@QEAA_NAEAVCPool@Memory@@@Z 000000003156b310 f   SkeletonPose.obj
 0001:0006a3b0       ?GetJointCRC32@CSkeletonPose@@UEBAIH@Z 000000003156b3b0 f   SkeletonPose.obj
 0001:0006a410       ?Init@SDirectionalBlender@@QEAAXXZ 000000003156b410 f i SkeletonPose.obj
 0001:0006a5a0       ??1CFeetLock@@QEAA@XZ      000000003156b5a0 f i SkeletonPose.obj
 0001:0006a610       ?GetStatObjOnJoint@CSkeletonPose@@UEAAPEAUIStatObj@@H@Z 000000003156b610 f   SkeletonPose.obj
 0001:0006a670       ?SetStatObjOnJoint@CSkeletonPose@@UEAAXHPEAUIStatObj@@@Z 000000003156b670 f   SkeletonPose.obj
 0001:0006a700       ?GetInverted@?$QuatTS_tpl@M@@QEBA?AU1@XZ 000000003156b700 f i SkeletonPose.obj
 0001:0006a8c0       ??$move_init@USPostProcess@@@NArray@@YAXPEAUSPostProcess@@0_K@Z 000000003156b8c0 f i SkeletonPose.obj
 0001:0006aaa0       ??$move_init@UCCGAJoint@@@NArray@@YAXPEAUCCGAJoint@@0_K@Z 000000003156baa0 f i SkeletonPose.obj
 0001:0006ab90       ??4?$shared_ptr@UIAnimationPoseBlenderDir@@@boost@@QEAAAEAV01@AEBV01@@Z 000000003156bb90 f i SkeletonPose.obj
 0001:0006ab90       ??4?$shared_ptr@UIAnimationPoseModifier@@@boost@@QEAAAEAV01@AEBV01@@Z 000000003156bb90 f i TransitionQueue.obj
 0001:0006ac20       ?Op@?$cryinterface_cast_boost_helper@UIAnimationPoseBlenderDir@@UICryUnknown@@@Internal@InterfaceCastSemantics@@SA?AV?$shared_ptr@UIAnimationPoseBlenderDir@@@boost@@AEBV?$shared_ptr@UICryUnknown@@@5@@Z 000000003156bc20 f i SkeletonPose.obj
 0001:0006ad30       ?Op@?$cryinterface_cast_boost_helper@UIAnimationPoseModifier@@UICryUnknown@@@Internal@InterfaceCastSemantics@@SA?AV?$shared_ptr@UIAnimationPoseModifier@@@boost@@AEBV?$shared_ptr@UICryUnknown@@@5@@Z 000000003156bd30 f i SkeletonPose.obj
 0001:0006ae40       ?resize_raw@?$SmallDynStorage@USPostProcess@@HUStandardAlloc@NAlloc@@@NArray@@QEAAXHH_N@Z 000000003156be40 f i SkeletonPose.obj
 0001:0006afb0       ?pop_back@?$DynArray@UCCGAJoint@@HU?$SmallDynStorage@UCCGAJoint@@HUStandardAlloc@NAlloc@@@NArray@@@@QEAAXH@Z 000000003156bfb0 f i SkeletonPose.obj
 0001:0006b080       ?destroy@?$DynArray@UCCGAJoint@@HU?$SmallDynStorage@UCCGAJoint@@HUStandardAlloc@NAlloc@@@NArray@@@@IEAAXXZ 000000003156c080 f i SkeletonPose.obj
 0001:0006b120       ?resize_raw@?$SmallDynStorage@UCCGAJoint@@HUStandardAlloc@NAlloc@@@NArray@@QEAAXHH_N@Z 000000003156c120 f i SkeletonPose.obj
 0001:0006b2a0       ??$CryCreateClassInstance@UIAnimationPoseBlenderDir@@@@YA_NPEBDAEAV?$shared_ptr@UIAnimationPoseBlenderDir@@@boost@@@Z 000000003156c2a0 f i SkeletonPose.obj
 0001:0006b3f0       ??$CryCreateClassInstance@UIAnimationPoseModifier@@@@YA_NPEBDAEAV?$shared_ptr@UIAnimationPoseModifier@@@boost@@@Z 000000003156c3f0 f i SkeletonPose.obj
 0001:0006b540       ?append_raw@?$DynArray@USPostProcess@@HU?$SmallDynStorage@USPostProcess@@HUStandardAlloc@NAlloc@@@NArray@@@@QEAA?AU?$Array@USPostProcess@@HU?$ArrayStorage@USPostProcess@@H@NArray@@@@H@Z 000000003156c540 f i SkeletonPose.obj
 0001:0006b600       ??1CSkeletonPose@@UEAA@XZ  000000003156c600 f   SkeletonPose.obj
 0001:0006b7d0       ?GetJointCount@CSkeletonPose@@UEBAIXZ 000000003156c7d0 f i SkeletonPose.obj
 0001:0006b7f0       ?GetJointIDByName@CSkeletonPose@@UEBAFPEBD@Z 000000003156c7f0 f i SkeletonPose.obj
 0001:0006b800       ?GetJointIDByCRC32@CSkeletonPose@@UEBAFI@Z 000000003156c800 f i SkeletonPose.obj
 0001:0006b810       ?GetParentIDByID@CSkeletonPose@@UEBAFH@Z 000000003156c810 f i SkeletonPose.obj
 0001:0006b820       ?GetJointNameByID@CSkeletonPose@@UEBAPEBDH@Z 000000003156c820 f i SkeletonPose.obj
 0001:0006b830       ?SetPostProcessCallback@CSkeletonPose@@UEAAXP6AHPEAUICharacterInstance@@PEAX@Z1@Z 000000003156c830 f i SkeletonPose.obj
 0001:0006b840       ?GetPhysEntOnJoint@CSkeletonPose@@UEAAPEAUIPhysicalEntity@@H@Z 000000003156c840 f i SkeletonPose.obj
 0001:0006b860       ?SetPhysEntOnJoint@CSkeletonPose@@UEAAXHPEAUIPhysicalEntity@@@Z 000000003156c860 f i SkeletonPose.obj
 0001:0006b870       ?GetPhysIdOnJoint@CSkeletonPose@@UEAAHH@Z 000000003156c870 f i SkeletonPose.obj
 0001:0006b880       ?BuildPhysicalEntity@CSkeletonPose@@UEAAXPEAUIPhysicalEntity@@MHMHHAEBU?$Matrix34_tpl@M@@@Z 000000003156c880 f i SkeletonPose.obj
 0001:0006b8d0       ?CreateCharacterPhysics@CSkeletonPose@@UEAAPEAUIPhysicalEntity@@PEAU2@MHMHAEBU?$Matrix34_tpl@M@@@Z 000000003156c8d0 f i SkeletonPose.obj
 0001:0006b910       ?CreateAuxilaryPhysics@CSkeletonPose@@UEAAHPEAUIPhysicalEntity@@AEBU?$Matrix34_tpl@M@@H@Z 000000003156c910 f i SkeletonPose.obj
 0001:0006b920       ?GetCharacterPhysics@CSkeletonPose@@UEBAPEAUIPhysicalEntity@@XZ 000000003156c920 f i SkeletonPose.obj
 0001:0006b930       ?GetCharacterPhysics@CSkeletonPose@@UEAAPEAUIPhysicalEntity@@PEBD@Z 000000003156c930 f i SkeletonPose.obj
 0001:0006b940       ?GetCharacterPhysics@CSkeletonPose@@UEAAPEAUIPhysicalEntity@@H@Z 000000003156c940 f i SkeletonPose.obj
 0001:0006b950       ?SetCharacterPhysics@CSkeletonPose@@UEAAXPEAUIPhysicalEntity@@@Z 000000003156c950 f i SkeletonPose.obj
 0001:0006b970       ?SynchronizeWithPhysicalEntity@CSkeletonPose@@UEAAXPEAUIPhysicalEntity@@AEBU?$Vec3_tpl@M@@AEBU?$Quat_tpl@M@@@Z 000000003156c970 f i SkeletonPose.obj
 0001:0006b980       ?RelinquishCharacterPhysics@CSkeletonPose@@UEAAPEAUIPhysicalEntity@@AEBU?$Matrix34_tpl@M@@M_NAEBU?$Vec3_tpl@M@@@Z 000000003156c980 f i SkeletonPose.obj
 0001:0006b9a0       ?DestroyCharacterPhysics@CSkeletonPose@@UEAAXH@Z 000000003156c9a0 f i SkeletonPose.obj
 0001:0006b9b0       ?AddImpact@CSkeletonPose@@UEAA_NHU?$Vec3_tpl@M@@0@Z 000000003156c9b0 f i SkeletonPose.obj
 0001:0006ba00       ?TranslatePartIdToDeadBody@CSkeletonPose@@UEAAHH@Z 000000003156ca00 f i SkeletonPose.obj
 0001:0006ba10       ?GetAuxPhysicsBoneId@CSkeletonPose@@UEAAHHH@Z 000000003156ca10 f i SkeletonPose.obj
 0001:0006ba50       ?GoLimp@CSkeletonPose@@UEAAXXZ 000000003156ca50 f i SkeletonPose.obj
 0001:0006ba60       ?BlendFromRagdoll@CSkeletonPose@@UEAA_NAEAU?$QuatTS_tpl@M@@AEAPEAUIPhysicalEntity@@_N@Z 000000003156ca60 f i SkeletonPose.obj
 0001:0006ba70       ?GetFallingDir@CSkeletonPose@@UEAAHXZ 000000003156ca70 f i SkeletonPose.obj
 0001:0006ba80       ?getBonePhysParentOrSelfIndex@CSkeletonPose@@UEAAHHH@Z 000000003156ca80 f i SkeletonPose.obj
 0001:0006ba90       ?GetBoneSurfaceTypeId@CSkeletonPose@@UEAAHHH@Z 000000003156ca90 f i SkeletonPose.obj
 0001:0006baa0       ?SetRagdollDefaultPose@CSkeletonPose@@UEAAXXZ 000000003156caa0 f i SkeletonPose.obj
 0001:0006bab0       ?GetAbsJointByID@CSkeletonPose@@UEAAAEBU?$QuatT_tpl@M@@H@Z 000000003156cab0 f i SkeletonPose.obj
 0001:0006bb00       ?GetRelJointByID@CSkeletonPose@@UEAAAEBU?$QuatT_tpl@M@@H@Z 000000003156cb00 f i SkeletonPose.obj
 0001:0006bb50       ?GetDefaultAbsJointByID@CSkeletonPose@@UEAAAEBU?$QuatT_tpl@M@@H@Z 000000003156cb50 f i SkeletonPose.obj
 0001:0006bba0       ?GetDefaultRelJointByID@CSkeletonPose@@UEAAAEBU?$QuatT_tpl@M@@H@Z 000000003156cba0 f i SkeletonPose.obj
 0001:0006bbf0       ?GetIPoseBlenderLook@CSkeletonPose@@UEAAPEAUIAnimationPoseBlenderDir@@XZ 000000003156cbf0 f i SkeletonPose.obj
 0001:0006bc00       ?GetIPoseBlenderAim@CSkeletonPose@@UEAAPEAUIAnimationPoseBlenderDir@@XZ 000000003156cc00 f i SkeletonPose.obj
 0001:0006bc10       ?SetMaterialOnJoint@CSkeletonPose@@UEAAXHPEAUIMaterial@@@Z 000000003156cc10 f i SkeletonPose.obj
 0001:0006bc80       ?GetMaterialOnJoint@CSkeletonPose@@UEAAPEAUIMaterial@@H@Z 000000003156cc80 f i SkeletonPose.obj
 0001:0006bcb0       ?SetHumanLimbIK@CSkeletonPose@@UEAAIAEBU?$Vec3_tpl@M@@PEBD@Z 000000003156ccb0 f   SkeletonPose.obj
 0001:0006be80       ?ApplyRecoilAnimation@CSkeletonPose@@UEAAXMMMI@Z 000000003156ce80 f   SkeletonPose.obj
 0001:0006bf20       ?append_raw@?$DynArray@UCCGAJoint@@HU?$SmallDynStorage@UCCGAJoint@@HUStandardAlloc@NAlloc@@@NArray@@@@QEAA?AU?$Array@UCCGAJoint@@HU?$ArrayStorage@UCCGAJoint@@H@NArray@@@@H@Z 000000003156cf20 f i SkeletonPose.obj
 0001:0006bfe0       ??0CSkeletonPose@@QEAA@XZ  000000003156cfe0 f   SkeletonPose.obj
 0001:0006c1d0       ??_GCSkeletonPose@@UEAAPEAXI@Z 000000003156d1d0 f i SkeletonPose.obj
 0001:0006c1d0       ??_ECSkeletonPose@@UEAAPEAXI@Z 000000003156d1d0 f i SkeletonPose.obj
 0001:0006c200       ?SetDefaultPosePerInstance@CSkeletonPose@@QEAAX_N@Z 000000003156d200 f   SkeletonPose.obj
 0001:0006cc40       ?SetDefaultPoseExecute@CSkeletonPose@@QEAAX_N@Z 000000003156dc40 f   SkeletonPose.obj
 0001:0006cd20       ?resize@?$DynArray@UCCGAJoint@@HU?$SmallDynStorage@UCCGAJoint@@HUStandardAlloc@NAlloc@@@NArray@@@@QEAAXH@Z 000000003156dd20 f i SkeletonPose.obj
 0001:0006cda0       ?SetPostProcessQuat@CSkeletonPose@@UEAAXHAEBU?$QuatT_tpl@M@@@Z 000000003156dda0 f i SkeletonPose.obj
 0001:0006cea0       ?InitSkeletonPose@CSkeletonPose@@QEAAXPEAVCCharInstance@@PEAVCSkeletonAnim@@@Z 000000003156dea0 f   SkeletonPose.obj
 0001:0006d020       ?InitCGASkeleton@CSkeletonPose@@QEAAXXZ 000000003156e020 f   SkeletonPose.obj
 0001:0006d1a0       ?DrawBBox@CSkeletonPose@@QEAAXAEBU?$Matrix34_tpl@M@@@Z 000000003156e1a0 f   SkeletonPose_Debug.obj
 0001:0006d360       ??$AddObject@UCCGAJoint@@HU?$SmallDynStorage@UCCGAJoint@@HUStandardAlloc@NAlloc@@@NArray@@@ICrySizer@@QEAAXAEBU?$DynArray@UCCGAJoint@@HU?$SmallDynStorage@UCCGAJoint@@HUStandardAlloc@NAlloc@@@NArray@@@@@Z 000000003156e360 f i SkeletonPose_Debug.obj
 0001:0006d3d0       ?get_alloc_size@?$SmallDynStorage@U?$Vec3_tpl@M@@HUStandardAlloc@NAlloc@@@NArray@@QEBAHXZ 000000003156e3d0 f i SkeletonPose_Debug.obj
 0001:0006d430       ??$AddObject@UCPhysicsJoint@@HU?$SmallDynStorage@UCPhysicsJoint@@HUStandardAlloc@NAlloc@@@NArray@@@ICrySizer@@QEAAXAEBU?$DynArray@UCPhysicsJoint@@HU?$SmallDynStorage@UCPhysicsJoint@@HUStandardAlloc@NAlloc@@@NArray@@@@@Z 000000003156e430 f i SkeletonPose_Debug.obj
 0001:0006d4a0       ?DrawPose@CSkeletonPose@@QEAAXAEBVCPoseData@Skeleton@@AEBU?$Matrix34_tpl@M@@@Z 000000003156e4a0 f   SkeletonPose_Debug.obj
 0001:0006e210       ?DrawSkeleton@CSkeletonPose@@UEAAXAEBU?$Matrix34_tpl@M@@I@Z 000000003156f210 f   SkeletonPose_Debug.obj
 0001:0006e220       ?SizeOfThis@CSkeletonPhysics@@QEAA_KXZ 000000003156f220 f i SkeletonPose_Debug.obj
 0001:0006e2c0       ?SizeOfThis@CSkeletonPose@@QEAA_KXZ 000000003156f2c0 f   SkeletonPose_Debug.obj
 0001:0006e4b0       ?GetMemoryUsage@CSkeletonPose@@QEBAXPEAVICrySizer@@@Z 000000003156f4b0 f   SkeletonPose_Debug.obj
 0001:0006e5f0       ?_M_set@?$_Impl_vector@USFacialEffectorChannel@@V?$allocator@USFacialEffectorChannel@@@stlpmtx_std@@@priv@stlpmtx_std@@AEAAXPEAUSFacialEffectorChannel@@00@Z 000000003156f5f0 f i FaceAnimation.obj
 0001:0006e5f0       ?_M_set@?$_Impl_vector@U?$TCoeffBasis@M@spline@@V?$allocator@U?$TCoeffBasis@M@spline@@@stlpmtx_std@@@priv@stlpmtx_std@@AEAAXPEAU?$TCoeffBasis@M@spline@@00@Z 000000003156f5f0 f i FaceEffector.obj
 0001:0006e5f0       ?_M_set@?$_Impl_vector@UWordRec@CFacialSentence@@V?$allocator@UWordRec@CFacialSentence@@@stlpmtx_std@@@priv@stlpmtx_std@@AEAAXPEAUWordRec@CFacialSentence@@00@Z 000000003156f5f0 f i LipSync.obj
 0001:0006e5f0       ?_M_set@?$_Impl_vector@UPhoneme@IFacialSentence@@V?$allocator@UPhoneme@IFacialSentence@@@stlpmtx_std@@@priv@stlpmtx_std@@AEAAXPEAUPhoneme@IFacialSentence@@00@Z 000000003156f5f0 f i LipSync.obj
 0001:0006e5f0       ?_M_set@?$_Impl_vector@UBalanceChannelEntry@CFacialAnimSequenceInstance@@V?$allocator@UBalanceChannelEntry@CFacialAnimSequenceInstance@@@stlpmtx_std@@@priv@stlpmtx_std@@AEAAXPEAUBalanceChannelEntry@CFacialAnimSequenceInstance@@00@Z 000000003156f5f0 f i FaceAnimSequence.obj
 0001:0006e5f0       ?_M_set@?$_Impl_vector@V?$_smart_ptr@VCFacialEffCtrl@@@@V?$allocator@V?$_smart_ptr@VCFacialEffCtrl@@@@@stlpmtx_std@@@priv@stlpmtx_std@@AEAAXPEAV?$_smart_ptr@VCFacialEffCtrl@@@@00@Z 000000003156f5f0 f i FaceEffector.obj
 0001:0006e5f0       ?_M_set@?$_Impl_vector@MV?$allocator@M@stlpmtx_std@@@priv@stlpmtx_std@@AEAAXPEAM00@Z 000000003156f5f0 f i FaceAnimation.obj
 0001:0006e5f0       ?_M_set@?$_Impl_vector@USPlayingSequence@CFacialAnimationContext@@V?$allocator@USPlayingSequence@CFacialAnimationContext@@@stlpmtx_std@@@priv@stlpmtx_std@@AEAAXPEAUSPlayingSequence@CFacialAnimationContext@@00@Z 000000003156f5f0 f i FaceAnimation.obj
 0001:0006e5f0       ?_M_set@?$_Impl_vector@USPhoneme@@V?$allocator@USPhoneme@@@stlpmtx_std@@@priv@stlpmtx_std@@AEAAXPEAUSPhoneme@@00@Z 000000003156f5f0 f i LipSync.obj
 0001:0006e5f0       ?_M_set@?$_Impl_vector@VCFacialAnimSoundEntry@@V?$allocator@VCFacialAnimSoundEntry@@@stlpmtx_std@@@priv@stlpmtx_std@@AEAAXPEAVCFacialAnimSoundEntry@@00@Z 000000003156f5f0 f i FaceAnimSequence.obj
 0001:0006e5f0       ?_M_set@?$_Impl_vector@V?$_smart_ptr@VCFacialEffector@@@@V?$allocator@V?$_smart_ptr@VCFacialEffector@@@@@stlpmtx_std@@@priv@stlpmtx_std@@AEAAXPEAV?$_smart_ptr@VCFacialEffector@@@@00@Z 000000003156f5f0 f i FaceEffectorLibrary.obj
 0001:0006e5f0       ?_M_set@?$_Impl_vector@UChannelInfo@CFacialAnimSequenceInstance@@V?$allocator@UChannelInfo@CFacialAnimSequenceInstance@@@stlpmtx_std@@@priv@stlpmtx_std@@AEAAXPEAUChannelInfo@CFacialAnimSequenceInstance@@00@Z 000000003156f5f0 f i FaceAnimSequence.obj
 0001:0006e5f0       ?_M_set@?$_Impl_vector@V?$CryStringT@D@@V?$allocator@V?$CryStringT@D@@@stlpmtx_std@@@priv@stlpmtx_std@@AEAAXPEAV?$CryStringT@D@@00@Z 000000003156f5f0 f i SkeletonPose_Process.obj
 0001:0006e5f0       ?_M_set@?$_Impl_vector@U?$Vec3_tpl@M@@V?$allocator@U?$Vec3_tpl@M@@@stlpmtx_std@@@priv@stlpmtx_std@@AEAAXPEAU?$Vec3_tpl@M@@00@Z 000000003156f5f0 f i LoaderSKIN.obj
 0001:0006e5f0       ?_M_set@?$_Impl_vector@U?$pair@V?$CryStringT@D@@PEAUIFacialAnimChannel@@@stlpmtx_std@@V?$allocator@U?$pair@V?$CryStringT@D@@PEAUIFacialAnimChannel@@@stlpmtx_std@@@2@@priv@stlpmtx_std@@AEAAXPEAU?$pair@V?$CryStringT@D@@PEAUIFacialAnimChannel@@@3@00@Z 000000003156f5f0 f i FaceAnimation.obj
 0001:0006e5f0       ?_M_set@?$_Impl_vector@HV?$allocator@H@stlpmtx_std@@@priv@stlpmtx_std@@AEAAXPEAH00@Z 000000003156f5f0 f i ControllerDefragHeap.obj
 0001:0006e5f0       ?_M_set@?$_Impl_vector@USOp@COperatorQueue@@V?$allocator@USOp@COperatorQueue@@@stlpmtx_std@@@priv@stlpmtx_std@@AEAAXPEAUSOp@COperatorQueue@@00@Z 000000003156f5f0 f i OperatorQueue.obj
 0001:0006e5f0       ?_M_set@?$_Impl_vector@VCFacialAnimSkeletalAnimationEntry@@V?$allocator@VCFacialAnimSkeletalAnimationEntry@@@stlpmtx_std@@@priv@stlpmtx_std@@AEAAXPEAVCFacialAnimSkeletalAnimationEntry@@00@Z 000000003156f5f0 f i FaceAnimSequence.obj
 0001:0006e5f0       ?_M_set@?$_Impl_vector@U?$DynArray@U?$QuatT_tpl@M@@HU?$SmallDynStorage@U?$QuatT_tpl@M@@HUStandardAlloc@NAlloc@@@NArray@@@@V?$allocator@U?$DynArray@U?$QuatT_tpl@M@@HU?$SmallDynStorage@U?$QuatT_tpl@M@@HUStandardAlloc@NAlloc@@@NArray@@@@@stlpmtx_std@@@priv@stlpmtx_std@@AEAAXPEAU?$DynArray@U?$QuatT_tpl@M@@HU?$SmallDynStorage@U?$QuatT_tpl@M@@HUStandardAlloc@NAlloc@@@NArray@@@@00@Z 000000003156f5f0 f i GlobalAnimationHeaderCAF.obj
 0001:0006e5f0       ?_M_set@?$_Impl_vector@U?$pair@PEAUIFacialAnimChannel@@H@stlpmtx_std@@V?$allocator@U?$pair@PEAUIFacialAnimChannel@@H@stlpmtx_std@@@2@@priv@stlpmtx_std@@AEAAXPEAU?$pair@PEAUIFacialAnimChannel@@H@3@00@Z 000000003156f5f0 f i FaceAnimSequence.obj
 0001:0006e5f0       ?_M_set@?$_Impl_vector@USMorphTargetInfo@CFacialModel@@V?$allocator@USMorphTargetInfo@CFacialModel@@@stlpmtx_std@@@priv@stlpmtx_std@@AEAAXPEAUSMorphTargetInfo@CFacialModel@@00@Z 000000003156f5f0 f i FacialModel.obj
 0001:0006e5f0       ?_M_set@?$_Impl_vector@UFacialAnimationEntry@CAnimationSet@@V?$allocator@UFacialAnimationEntry@CAnimationSet@@@stlpmtx_std@@@priv@stlpmtx_std@@AEAAXPEAUFacialAnimationEntry@CAnimationSet@@00@Z 000000003156f5f0 f i LoaderCHR.obj
 0001:0006e5f0       ?_M_set@?$_Impl_vector@IV?$allocator@I@stlpmtx_std@@@priv@stlpmtx_std@@AEAAXPEAI00@Z 000000003156f5f0 f i SkeletonPose_Process.obj
 0001:0006e5f0       ?_M_set@?$_Impl_vector@V?$_smart_ptr@VCFacialJoystick@@@@V?$allocator@V?$_smart_ptr@VCFacialJoystick@@@@@stlpmtx_std@@@priv@stlpmtx_std@@AEAAXPEAV?$_smart_ptr@VCFacialJoystick@@@@00@Z 000000003156f5f0 f i FaceJoystick.obj
 0001:0006e5f0       ?_M_set@?$_Impl_vector@V?$_smart_ptr@VCFacialAnimChannel@@@@V?$allocator@V?$_smart_ptr@VCFacialAnimChannel@@@@@stlpmtx_std@@@priv@stlpmtx_std@@AEAAXPEAV?$_smart_ptr@VCFacialAnimChannel@@@@00@Z 000000003156f5f0 f i FaceAnimSequence.obj
 0001:0006e5f0       ?_M_set@?$_Impl_vector@U?$Color_tpl@E@@V?$allocator@U?$Color_tpl@E@@@stlpmtx_std@@@priv@stlpmtx_std@@AEAAXPEAU?$Color_tpl@E@@00@Z 000000003156f5f0 f i ModelMesh_DebugPC.obj
 0001:0006e5f0       ?_M_set@?$_Impl_vector@UCharacterDefinition@@V?$allocator@UCharacterDefinition@@@stlpmtx_std@@@priv@stlpmtx_std@@AEAAXPEAUCharacterDefinition@@00@Z 000000003156f5f0 f i CharacterManager.obj
 0001:0006e5f0       ?_M_set@?$_Impl_vector@PEAXV?$allocator@PEAX@stlpmtx_std@@@priv@stlpmtx_std@@AEAAXPEAPEAX00@Z 000000003156f5f0 f i LoaderSKIN.obj
 0001:0006e5f0       ?_M_set@?$_Impl_vector@USEffectorInfo@CFacialModel@@V?$allocator@USEffectorInfo@CFacialModel@@@stlpmtx_std@@@priv@stlpmtx_std@@AEAAXPEAUSEffectorInfo@CFacialModel@@00@Z 000000003156f5f0 f i FacialModel.obj
 0001:0006e680       ?UpdateBBox@CSkeletonPose@@QEAAXI@Z 000000003156f680 f   SkeletonPose_Process.obj
 0001:0006fbc0       ?UpdateAttachments@CSkeletonPose@@QEAAXAEAVCPoseData@Skeleton@@@Z 0000000031570bc0 f   SkeletonPose_Process.obj
 0001:0006fd80       ?_M_clear_after_move@?$_Impl_vector@V?$CryStringT@D@@V?$allocator@V?$CryStringT@D@@@stlpmtx_std@@@priv@stlpmtx_std@@AEAAXXZ 0000000031570d80 f i SkeletonPose_Process.obj
 0001:0006fe00       ?_M_insert_overflow_aux@?$_Impl_vector@V?$CryStringT@D@@V?$allocator@V?$CryStringT@D@@@stlpmtx_std@@@priv@stlpmtx_std@@AEAAXPEAV?$CryStringT@D@@AEBV4@AEBU__false_type@3@_K_N@Z 0000000031570e00 f i SkeletonPose_Process.obj
 0001:0006fff0       ?SkeletonPostProcess@CSkeletonPose@@QEAAXAEAVCPoseData@Skeleton@@@Z 0000000031570ff0 f   SkeletonPose_Process.obj
 0001:00070d40       ?SetDebugging@CSkeletonAnim@@UEAAXI@Z 0000000031571d40 f   SkeletonAnim.obj
 0001:00070d50       ?SetTrackViewExclusive@CSkeletonAnim@@UEAAXI@Z 0000000031571d50 f   SkeletonAnim.obj
 0001:00070d80       ??_EISkeletonAnim@@UEAAPEAXI@Z 0000000031571d80 f i SkeletonAnim.obj
 0001:00070d80       ??_GISkeletonAnim@@UEAAPEAXI@Z 0000000031571d80 f i SkeletonAnim.obj
 0001:00070db0       ?Initialize@CSkeletonAnimTask@@SA_NXZ 0000000031571db0 f   SkeletonAnim.obj
 0001:00070e00       ??_ECSkeletonAnimTask@@UEAAPEAXI@Z 0000000031571e00 f i SkeletonAnim.obj
 0001:00070e00       ??_GCSkeletonAnimTask@@UEAAPEAXI@Z 0000000031571e00 f i SkeletonAnim.obj
 0001:00070e40       ?Execute@CSkeletonAnimTask@@UEAAXXZ 0000000031571e40 f   SkeletonAnim.obj
 0001:00070ea0       ?InitSkeletonAnim@CSkeletonAnim@@QEAAXPEAVCCharInstance@@PEAVCSkeletonPose@@@Z 0000000031571ea0 f   SkeletonAnim.obj
 0001:00070f90       ?PoseModifiersSynchronize@CSkeletonAnim@@QEAAXXZ 0000000031571f90 f   SkeletonAnim.obj
 0001:00071010       ?GetCurrentVelocity@CSkeletonAnim@@UEAA?AU?$Vec3_tpl@M@@XZ 0000000031572010 f   SkeletonAnim.obj
 0001:000710a0       ?SetTrackViewMixingWeight@CSkeletonAnim@@UEAAXIM@Z 00000000315720a0 f   SkeletonAnim.obj
 0001:000710e0       ?AllocateRuntimeParametric@CSkeletonAnim@@QEAAPEAUSParametricSamplerInternal@@XZ 00000000315720e0 f   SkeletonAnim.obj
 0001:000711a0       ?Invoke@?$SGenInvokerTCommandBufferExecuteJob@VCSkeletonAnimTask@@HUSNullType@Detail@JobManager@@U234@U234@U234@U234@U234@U234@U234@U234@U234@U234@@Detail@JobManager@@SAXPEAX@Z 00000000315721a0 f i SkeletonAnim.obj
 0001:00071200       ?Serialize@SParametricSamplerInternal@@QEAAXV?$CSerializeWrapper@UISerialize@@@@@Z 0000000031572200 f i SkeletonAnim.obj
 0001:00071480       ?Wait@CSkeletonAnimTask@@QEAAXXZ 0000000031572480 f   SkeletonAnim.obj
 0001:000715f0       ?PoseModifiersExecutePost@CSkeletonAnim@@QEAAXAEAVCPoseData@Skeleton@@AEBU?$QuatTS_tpl@M@@@Z 00000000315725f0 f   SkeletonAnim.obj
 0001:00071690       ?ProcessAnimationUpdate@CSkeletonAnim@@QEAAXU?$QuatTS_tpl@M@@@Z 0000000031572690 f   SkeletonAnim.obj
 0001:000719a0       ?FinishAnimationComputations@CSkeletonAnim@@AEAAXW4FinishAnimationComputationCallMethod@1@@Z 00000000315729a0 f   SkeletonAnim.obj
 0001:00071e70       ?PushPoseModifier@CSkeletonAnim@@UEAA_NIV?$shared_ptr@UIAnimationPoseModifier@@@boost@@PEBD@Z 0000000031572e70 f   SkeletonAnim.obj
 0001:00071fd0       ?PoseModifiersPrepare@CSkeletonAnim@@QEAAXAEBU?$QuatTS_tpl@M@@@Z 0000000031572fd0 f   SkeletonAnim.obj
 0001:00072270       ?SizeOfThis@CSkeletonAnim@@QEAA_KXZ 0000000031573270 f   SkeletonAnim.obj
 0001:00072310       ?Prepare@CSkeletonAnimTask@@QEAAXXZ 0000000031573310 f   SkeletonAnim.obj
 0001:00072420       ?FinishAnimationComputations@CSkeletonAnim@@QEAAXXZ 0000000031573420 f   SkeletonAnim.obj
 0001:00072430       ?GetMemoryUsage@CSkeletonAnim@@QEBAXPEAVICrySizer@@@Z 0000000031573430 f   SkeletonAnim.obj
 0001:00072520       ?Format@?$CryStringT@D@@QEAAAEAV1@PEBDZZ 0000000031573520 f i SkeletonAnim.obj
 0001:000725b0       ?Begin@CSkeletonAnimTask@@QEAAXAEBU?$QuatTS_tpl@M@@_N@Z 00000000315735b0 f   SkeletonAnim.obj
 0001:00072740       ?ProcessAnimations@CSkeletonAnim@@QEAAXAEBU?$QuatTS_tpl@M@@_N@Z 0000000031573740 f   SkeletonAnim.obj
 0001:00072970       ?Serialize@CAnimation@@QEAAXV?$CSerializeWrapper@UISerialize@@@@@Z 0000000031573970 f i SkeletonAnim.obj
 0001:00072c50       ??1CSkeletonAnim@@UEAA@XZ  0000000031573c50 f   SkeletonAnim.obj
 0001:00072dc0       ?GetAnimationDrivenMotion@CSkeletonAnim@@UEAAIXZ 0000000031573dc0 f i SkeletonAnim.obj
 0001:00072dd0       ?GetTrackViewStatus@CSkeletonAnim@@UEAAIXZ 0000000031573dd0 f i SkeletonAnim.obj
 0001:00072de0       ?GetLayerPlaybackScale@CSkeletonAnim@@UEAAMI@Z 0000000031573de0 f i SkeletonAnim.obj
 0001:00072e00       ?SetEventCallback@CSkeletonAnim@@UEAAXP6AHPEAUICharacterInstance@@PEAX@Z1@Z 0000000031573e00 f i SkeletonAnim.obj
 0001:00072e10       ?GetLastAnimEvent@CSkeletonAnim@@UEAA?AUAnimEventInstance@@XZ 0000000031573e10 f i SkeletonAnim.obj
 0001:00072e40       ?GetUserData@CSkeletonAnim@@UEAAMH@Z 0000000031573e40 f i SkeletonAnim.obj
 0001:00072e50       ?GetAnimFromFIFO@CSkeletonAnim@@UEBAAEBVCAnimation@@II@Z 0000000031573e50 f i SkeletonAnim.obj
 0001:00072e50       ?GetAnimFromFIFO@CSkeletonAnim@@UEAAAEAVCAnimation@@II@Z 0000000031573e50 f i SkeletonAnim.obj
 0001:00072e70       ?RemoveAnimFromFIFO@CSkeletonAnim@@UEAA_NII_N@Z 0000000031573e70 f i SkeletonAnim.obj
 0001:00072e90       ?ClearFIFOLayer@CSkeletonAnim@@UEAAXI@Z 0000000031573e90 f i SkeletonAnim.obj
 0001:00072ea0       ?RemoveTransitionDelayConditions@CSkeletonAnim@@UEAAXI@Z 0000000031573ea0 f i SkeletonAnim.obj
 0001:00072eb0       ?ManualSeekAnimationInFIFO@CSkeletonAnim@@UEAAXIIM_N@Z 0000000031573eb0 f i SkeletonAnim.obj
 0001:00072ef0       ?GetNumAnimsInFIFO@CSkeletonAnim@@UEBAHI@Z 0000000031573ef0 f i SkeletonAnim.obj
 0001:00072f10       ??0CSkeletonAnim@@QEAA@XZ  0000000031573f10 f   SkeletonAnim.obj
 0001:000730b0       ??_GCSkeletonAnim@@UEAAPEAXI@Z 00000000315740b0 f i SkeletonAnim.obj
 0001:000730b0       ??_ECSkeletonAnim@@UEAAPEAXI@Z 00000000315740b0 f i SkeletonAnim.obj
 0001:000730e0       ?Serialize@CSkeletonAnim@@QEAAXV?$CSerializeWrapper@UISerialize@@@@@Z 00000000315740e0 f   SkeletonAnim.obj
 0001:00073520       ?AnimFlags@@YAPEBDI@Z      0000000031574520 f   SkeletonAnim_BlendMan.obj
 0001:000735b0       ?GetAnimationNormalizedTime@CSkeletonAnim@@UEBAMII@Z 00000000315745b0 f   SkeletonAnim_BlendMan.obj
 0001:000735f0       ?SetAnimationDrivenMotion@CSkeletonAnim@@UEAAXI@Z 00000000315745f0 f   SkeletonAnim_BlendMan.obj
 0001:00073600       ?SetMirrorAnimation@CSkeletonAnim@@UEAAXI@Z 0000000031574600 f   SkeletonAnim_BlendMan.obj
 0001:00073610       ?SetLayerBlendWeight@CSkeletonAnim@@UEAAXHM@Z 0000000031574610 f   SkeletonAnim_BlendMan.obj
 0001:00073640       ?SetLayerPlaybackScale@CSkeletonAnim@@UEAAXHM@Z 0000000031574640 f   SkeletonAnim_BlendMan.obj
 0001:00073680       ?Draw2dLabel@IRenderer@@QEAAXMMMAEBU?$Color_tpl@M@@_NPEBDZZ 0000000031574680 f i SkeletonAnim_BlendMan.obj
 0001:00073730       ?UpdateParameters@CSkeletonAnim@@AEAAXPEAVCAnimation@@IIM@Z 0000000031574730 f   SkeletonAnim_BlendMan.obj
 0001:00073b70       ?GetMaxSegments@CSkeletonAnim@@AEBAIAEBVCAnimation@@@Z 0000000031574b70 f   SkeletonAnim_BlendMan.obj
 0001:00073cc0       ?AnimCallback@CSkeletonAnim@@QEAAXPEAVCAnimation@@II@Z 0000000031574cc0 f   SkeletonAnim_BlendMan.obj
 0001:00074020       ?SetLayerNormalizedTimeAndSegment@CSkeletonAnim@@QEAAXIMEH@Z 0000000031575020 f   SkeletonAnim_BlendMan.obj
 0001:000740c0       ?SetLayerNormalizedTime@CSkeletonAnim@@UEAAXIM@Z 00000000315750c0 f   SkeletonAnim_BlendMan.obj
 0001:00074120       ?GetLayerNormalizedTime@CSkeletonAnim@@UEBAMI@Z 0000000031575120 f   SkeletonAnim_BlendMan.obj
 0001:00074150       ?SetAnimationNormalizedTime@CSkeletonAnim@@UEAAXPEAVCAnimation@@M@Z 0000000031575150 f   SkeletonAnim_BlendMan.obj
 0001:00074260       ?GetAnimationNormalizedTime@CSkeletonAnim@@UEBAMPEBVCAnimation@@@Z 0000000031575260 f   SkeletonAnim_BlendMan.obj
 0001:00074310       ?LayerBlendManager@CSkeletonAnim@@QEAAXMI@Z 0000000031575310 f   SkeletonAnim_BlendMan.obj
 0001:000743c0       ?GetRelMovement@CSkeletonAnim@@UEBAAEBU?$QuatT_tpl@M@@XZ 00000000315753c0 f   SkeletonAnim_BlendMan.obj
 0001:00074460       ?CheckIsCAFLoaded@CSkeletonAnim@@AEAAIPEAVCAnimationSet@@H@Z 0000000031575460 f   SkeletonAnim_BlendMan.obj
 0001:00074520       ?UpdateAnimationTime@CSkeletonAnim@@AEAAXAEAVCAnimation@@IIII@Z 0000000031575520 f   SkeletonAnim_BlendMan.obj
 0001:00074990       ?IsAnimationInMemory@CSkeletonAnim@@AEAAIPEAVCAnimationSet@@PEAVCAnimation@@@Z 0000000031575990 f   SkeletonAnim_BlendMan.obj
 0001:00074af0       ?BlendManagerDebug@CSkeletonAnim@@QEAAIAEAU?$DynArray@VCAnimation@@HU?$SmallDynStorage@VCAnimation@@HUStandardAlloc@NAlloc@@@NArray@@@@I@Z 0000000031575af0 f   SkeletonAnim_BlendMan.obj
 0001:00075450       ?EvaluateTransitionFlags@CSkeletonAnim@@AEAAIPEAVCAnimation@@I@Z 0000000031576450 f   SkeletonAnim_BlendMan.obj
 0001:000758a0       ?BlendManager@CSkeletonAnim@@QEAAIMAEAU?$DynArray@VCAnimation@@HU?$SmallDynStorage@VCAnimation@@HUStandardAlloc@NAlloc@@@NArray@@@@I@Z 00000000315768a0 f   SkeletonAnim_BlendMan.obj
 0001:00075d60       ?Commands_BasePlayback@CSkeletonAnim@@AEAAXAEBVCAnimation@@AEAVCBuffer@Command@@@Z 0000000031576d60 f   SkeletonAnim_Commands.obj
 0001:00075f90       ?Commands_LPlayback@CSkeletonAnim@@AEAAXAEBVCAnimation@@IIAEAVCBuffer@Command@@@Z 0000000031576f90 f   SkeletonAnim_Commands.obj
 0001:00076170       ?Commands_BaseEvaluationLMG@CSkeletonAnim@@AEAAXAEBVCAnimation@@IAEAVCBuffer@Command@@@Z 0000000031577170 f   SkeletonAnim_Commands.obj
 0001:00076a60       ?Commands_Create@CSkeletonAnim@@AEAAXAEBU?$QuatTS_tpl@M@@AEAVCBuffer@Command@@@Z 0000000031577a60 f   SkeletonAnim_Commands.obj
 0001:00077210       ?SetDesiredMotionParam@CSkeletonAnim@@UEAAXW4EMotionParamID@@MM@Z 0000000031578210 f   SkeletonAnim_Params.obj
 0001:000772e0       ?GetDesiredMotionParam@CSkeletonAnim@@UEBA_NW4EMotionParamID@@AEAM@Z 00000000315782e0 f   SkeletonAnim_Params.obj
 0001:000773f0       ?StopAnimationsAllLayers@CSkeletonAnim@@UEAA_NXZ 00000000315783f0 f   SkeletonAnim_Queue.obj
 0001:00077430       ?StartAnimation@CSkeletonAnim@@UEAA_NPEBDAEBUCryCharAnimationParams@@@Z 0000000031578430 f   SkeletonAnim_Queue.obj
 0001:00077560       ?StopAnimationInLayer@CSkeletonAnim@@UEAA_NHM@Z 0000000031578560 f   SkeletonAnim_Queue.obj
 0001:00077600       ?FindAnimInFIFO@CSkeletonAnim@@UEAAPEAVCAnimation@@IH@Z 0000000031578600 f   SkeletonAnim_Queue.obj
 0001:00077680       ?AnimationToQueue@CSkeletonAnim@@AEAAIPEBUModelAnimationHeader@@HMAEBUCryCharAnimationParams@@@Z 0000000031578680 f   SkeletonAnim_Queue.obj
 0001:00077e30       ?StartAnimationById@CSkeletonAnim@@UEAA_NHAEBUCryCharAnimationParams@@@Z 0000000031578e30 f   SkeletonAnim_Queue.obj
 0001:000786a0       ?RetrieveEffectorIdentifiers@CEyeMovementFaceAnim@@AEBAPEBVCFaceIdentifierHandle@@XZ 00000000315796a0 f   EyeMovementFaceAnim.obj
 0001:00078870       ?InitialiseBoneIDs@CEyeMovementFaceAnim@@AEAAXXZ 0000000031579870 f   EyeMovementFaceAnim.obj
 0001:00078900       ??4?$_smart_ptr@VCFacialEffector@@@@QEAAAEAV0@PEAVCFacialEffector@@@Z 0000000031579900 f i EyeMovementFaceAnim.obj
 0001:00078950       ?CreateChannelForEffector@CEyeMovementFaceAnim@@AEAAIW4EffectorID@1@@Z 0000000031579950 f   EyeMovementFaceAnim.obj
 0001:00078aa0       ?DisplayDebugInfoForEye@CEyeMovementFaceAnim@@AEAAXAEBU?$QuatTS_tpl@M@@W4EyeID@1@AEBV?$CryStringT@D@@@Z 0000000031579aa0 f   EyeMovementFaceAnim.obj
 0001:00078c10       ?GetMemoryUsage@CEyeMovementFaceAnim@@QEBAXPEAVICrySizer@@@Z 0000000031579c10 f   EyeMovementFaceAnim.obj
 0001:00078c90       ??0CEyeMovementFaceAnim@@QEAA@PEAVCFacialInstance@@@Z 0000000031579c90 f   EyeMovementFaceAnim.obj
 0001:00078d10       ??_G?$_i_reference_target@H@@UEAAPEAXI@Z 0000000031579d10 f i LoaderSKIN.obj
 0001:00078d10       ??_GCEyeMovementFaceAnim@@UEAAPEAXI@Z 0000000031579d10 f i EyeMovementFaceAnim.obj
 0001:00078d10       ??_EIController@@UEAAPEAXI@Z 0000000031579d10 f i LoaderCGA.obj
 0001:00078d10       ??_GCControllerOptNonVirtual@@UEAAPEAXI@Z 0000000031579d10 f i LoaderDBA.obj
 0001:00078d10       ??_GIController@@UEAAPEAXI@Z 0000000031579d10 f i LoaderCGA.obj
 0001:00078d10       ??_E?$_i_reference_target@H@@UEAAPEAXI@Z 0000000031579d10 f i LoaderSKIN.obj
 0001:00078d10       ??_ECControllerOptNonVirtual@@UEAAPEAXI@Z 0000000031579d10 f i LoaderDBA.obj
 0001:00078d10       ??_ECEyeMovementFaceAnim@@UEAAPEAXI@Z 0000000031579d10 f i EyeMovementFaceAnim.obj
 0001:00078d40       ?OnExpressionLibraryLoad@CEyeMovementFaceAnim@@QEAAXXZ 0000000031579d40 f   EyeMovementFaceAnim.obj
 0001:00078d80       ?FindLookAngleAndStrength@CEyeMovementFaceAnim@@AEAAXW4EyeID@1@AEAM1AEBU?$QuatT_tpl@M@@@Z 0000000031579d80 f   EyeMovementFaceAnim.obj
 0001:000790a0       ?CalculateEyeAdditionalRotation@CEyeMovementFaceAnim@@AEAAXPEAVCCharInstance@@PEAVCFaceState@@PEAVCFacialEffectorsLibrary@@QEAU?$QuatT_tpl@M@@@Z 000000003157a0a0 f   EyeMovementFaceAnim.obj
 0001:000795f0       ?Format@?$CryStackStringT@D$0CAA@@@QEAAAEAV1@PEBDZZ 000000003157a5f0 f i EyeMovementFaceAnim.obj
 0001:000796e0       ?UpdateEye@CEyeMovementFaceAnim@@AEAAXAEBU?$QuatTS_tpl@M@@W4EyeID@1@AEBU?$QuatT_tpl@M@@@Z 000000003157a6e0 f   EyeMovementFaceAnim.obj
 0001:00079aa0       ?Update@CEyeMovementFaceAnim@@QEAAXMAEBU?$QuatTS_tpl@M@@PEAVCCharInstance@@PEAVCFacialEffectorsLibrary@@PEAVCFaceState@@@Z 000000003157aaa0 f   EyeMovementFaceAnim.obj
 0001:00079b40       ?GetPhonemeLibrary@CFacialAnimation@@UEAAPEAUIPhonemeLibrary@@XZ 000000003157ab40 f   FaceAnimation.obj
 0001:00079b50       ?CreateEffectorsLibrary@CFacialAnimation@@UEAAPEAUIFacialEffectorsLibrary@@XZ 000000003157ab50 f   FaceAnimation.obj
 0001:00079b80       ?CreateSequence@CFacialAnimation@@UEAAPEAUIFacialAnimSequence@@XZ 000000003157ab80 f   FaceAnimation.obj
 0001:00079bd0       ?GetJoystickContext@CFacialAnimation@@UEAAPEAVIJoystickContext@@XZ 000000003157abd0 f   FaceAnimation.obj
 0001:00079be0       ?CreateJoystick@CFacialAnimation@@UEAAPEAVIJoystick@@_K@Z 000000003157abe0 f   FaceAnimation.obj
 0001:00079c10       ?CreateJoystickSet@CFacialAnimation@@UEAAPEAVIJoystickSet@@XZ 000000003157ac10 f   FaceAnimation.obj
 0001:00079c40       ?CreateJoystickChannel@CFacialAnimation@@UEAAPEAVIJoystickChannel@@PEAUIFacialAnimChannel@@@Z 000000003157ac40 f   FaceAnimation.obj
 0001:00079c70       ?TemporarilyEnableAdditionalBoneRotationSmoothing@CFacialAnimationContext@@QEAAXXZ 000000003157ac70 f   FaceAnimation.obj
 0001:00079c80       ?IsBoneRotationSmoothingRequired@CFacialAnimationContext@@QEAA_NXZ 000000003157ac80 f   FaceAnimation.obj
 0001:00079ca0       ??0SFacialEffectorChannel@@QEAA@AEBU0@@Z 000000003157aca0 f i FaceAnimation.obj
 0001:00079d60       ?_Rotate_left@?$_Rb_global@_N@priv@stlpmtx_std@@SAXPEAU_Rb_tree_node_base@23@AEAPEAU423@@Z 000000003157ad60 f i FaceAnimation.obj
 0001:00079dc0       ?_Rotate_right@?$_Rb_global@_N@priv@stlpmtx_std@@SAXPEAU_Rb_tree_node_base@23@AEAPEAU423@@Z 000000003157adc0 f i FaceAnimation.obj
 0001:00079e20       ?_Rebalance_for_erase@?$_Rb_global@_N@priv@stlpmtx_std@@SAPEAU_Rb_tree_node_base@23@PEAU423@AEAPEAU423@11@Z 000000003157ae20 f i FaceAnimation.obj
 0001:0007a170       ??$find@PEAPEAVCAttachmentSKIN@@PEAV1@@stlpmtx_std@@YAPEAPEAVCAttachmentSKIN@@PEAPEAV1@0AEBQEAV1@@Z 000000003157b170 f i ModelSkin.obj
 0001:0007a170       ??$find@PEAPEAVCCharInstance@@PEAV1@@stlpmtx_std@@YAPEAPEAVCCharInstance@@PEAPEAV1@0AEBQEAV1@@Z 000000003157b170 f i Model.obj
 0001:0007a170       ??$find@PEAV?$_smart_ptr@VCFacialJoystick@@@@PEAVIJoystick@@@stlpmtx_std@@YAPEAV?$_smart_ptr@VCFacialJoystick@@@@PEAV1@0AEBQEAVIJoystick@@@Z 000000003157b170 f i FaceJoystick.obj
 0001:0007a170       ??$find@PEAPEAVCFacialEffectorsLibrary@@PEAV1@@stlpmtx_std@@YAPEAPEAVCFacialEffectorsLibrary@@PEAPEAV1@0AEBQEAV1@@Z 000000003157b170 f i FaceAnimation.obj
 0001:0007a200       ??0SPlayingSequence@CFacialAnimationContext@@QEAA@AEBU01@@Z 000000003157b200 f i FaceAnimation.obj
 0001:0007a280       ??$fill@PEAMM@stlpmtx_std@@YAXPEAM0AEBM@Z 000000003157b280 f i FaceAnimation.obj
 0001:0007a2f0       ?_Rebalance@?$_Rb_global@_N@priv@stlpmtx_std@@SAXPEAU_Rb_tree_node_base@23@AEAPEAU423@@Z 000000003157b2f0 f i FaceAnimation.obj
 0001:0007a4e0       ?GetChannel@CFacialAnimationContext@@QEAAPEAUSFacialEffectorChannel@@I@Z 000000003157b4e0 f   FaceAnimation.obj
 0001:0007a540       ?SetChannelWeight@CFacialAnimationContext@@QEAAXIM@Z 000000003157b540 f   FaceAnimation.obj
 0001:0007a5a0       ?AverageFaceState@CFacialAnimationContext@@AEAAXAEAVCFaceState@@@Z 000000003157b5a0 f   FaceAnimation.obj
 0001:0007a6c0       ?AnimatePlayingSequences@CFacialAnimationContext@@AEAAXAEBU?$QuatTS_tpl@M@@@Z 000000003157b6c0 f   FaceAnimation.obj
 0001:0007a760       ?SeekSequence@CFacialAnimationContext@@QEAAXPEAUIFacialAnimSequence@@M@Z 000000003157b760 f   FaceAnimation.obj
 0001:0007a7e0       ?PauseSequence@CFacialAnimationContext@@QEAAXPEAVCFacialAnimSequence@@_N@Z 000000003157b7e0 f   FaceAnimation.obj
 0001:0007a870       ?IsPlayingSequence@CFacialAnimationContext@@QEAA_NPEAVCFacialAnimSequence@@@Z 000000003157b870 f   FaceAnimation.obj
 0001:0007a8d0       ??$AddObject@USFacialEffectorChannel@@V?$allocator@USFacialEffectorChannel@@@stlpmtx_std@@@ICrySizer@@QEAAXAEBV?$vector@USFacialEffectorChannel@@V?$allocator@USFacialEffectorChannel@@@stlpmtx_std@@@stlpmtx_std@@@Z 000000003157b8d0 f i FaceAnimation.obj
 0001:0007a9a0       ?_M_compute_next_size@?$_Impl_vector@USFacialEffectorChannel@@V?$allocator@USFacialEffectorChannel@@@stlpmtx_std@@@priv@stlpmtx_std@@AEAA_K_K@Z 000000003157b9a0 f i FaceAnimation.obj
 0001:0007a9a0       ?_M_compute_next_size@?$_Impl_vector@USPlayingSequence@CFacialAnimationContext@@V?$allocator@USPlayingSequence@CFacialAnimationContext@@@stlpmtx_std@@@priv@stlpmtx_std@@AEAA_K_K@Z 000000003157b9a0 f i FaceAnimation.obj
 0001:0007aa30       ??$_M_find@V?$CryStringT@D@@@?$_Rb_tree@V?$CryStringT@D@@U?$less_stricmp@V?$CryStringT@D@@@stl@@U?$pair@$$CBV?$CryStringT@D@@V?$_smart_ptr@UIFacialAnimSequence@@@@@stlpmtx_std@@U?$_Select1st@U?$pair@$$CBV?$CryStringT@D@@V?$_smart_ptr@UIFacialAnimSequence@@@@@stlpmtx_std@@@priv@5@U?$_MapTraitsT@U?$pair@$$CBV?$CryStringT@D@@V?$_smart_ptr@UIFacialAnimSequence@@@@@stlpmtx_std@@@75@V?$allocator@U?$pair@$$CBV?$CryStringT@D@@V?$_smart_ptr@UIFacialAnimSequence@@@@@stlpmtx_std@@@5@@priv@stlpmtx_std@@AEBAPEAU_Rb_tree_node_base@12@AEBV?$CryStringT@D@@@Z 000000003157ba30 f i FaceAnimation.obj
 0001:0007aac0       ??$__copy@PEAUSFacialEffectorChannel@@PEAU1@_J@priv@stlpmtx_std@@YAPEAUSFacialEffectorChannel@@PEAU2@00AEBUrandom_access_iterator_tag@1@PEA_J@Z 000000003157bac0 f i FaceAnimation.obj
 0001:0007abe0       ??$__copy@PEAUSPlayingSequence@CFacialAnimationContext@@PEAU12@_J@priv@stlpmtx_std@@YAPEAUSPlayingSequence@CFacialAnimationContext@@PEAU23@00AEBUrandom_access_iterator_tag@1@PEA_J@Z 000000003157bbe0 f i FaceAnimation.obj
 0001:0007acd0       ?LoadEffectorsLibrary@CFacialAnimation@@UEAAPEAUIFacialEffectorsLibrary@@PEBD@Z 000000003157bcd0 f   FaceAnimation.obj
 0001:0007af20       ?CreateIdentifierHandle@CFacialAnimation@@UEAA?AVCFaceIdentifierHandle@@PEBD@Z 000000003157bf20 f   FaceAnimation.obj
 0001:0007af70       ??$AddObject@V?$CryStringT@D@@V?$_smart_ptr@UIFacialAnimSequence@@@@U?$less_stricmp@V?$CryStringT@D@@@stl@@V?$allocator@U?$pair@$$CBV?$CryStringT@D@@V?$_smart_ptr@UIFacialAnimSequence@@@@@stlpmtx_std@@@stlpmtx_std@@@ICrySizer@@QEAAXAEBV?$map@V?$CryStringT@D@@V?$_smart_ptr@UIFacialAnimSequence@@@@U?$less_stricmp@V?$CryStringT@D@@@stl@@V?$allocator@U?$pair@$$CBV?$CryStringT@D@@V?$_smart_ptr@UIFacialAnimSequence@@@@@stlpmtx_std@@@stlpmtx_std@@@stlpmtx_std@@@Z 000000003157bf70 f i FaceAnimation.obj
 0001:0007b060       ??$AddObject@PEAVCFacialEffectorsLibrary@@V?$allocator@PEAVCFacialEffectorsLibrary@@@stlpmtx_std@@@ICrySizer@@QEAAXAEBV?$vector@PEAVCFacialEffectorsLibrary@@V?$allocator@PEAVCFacialEffectorsLibrary@@@stlpmtx_std@@@stlpmtx_std@@@Z 000000003157c060 f i FaceAnimation.obj
 0001:0007b0e0       ??$__uninitialized_fill_n@PEAUSFacialEffectorChannel@@_KU1@@priv@stlpmtx_std@@YAPEAUSFacialEffectorChannel@@PEAU2@_KAEBU2@@Z 000000003157c0e0 f i FaceAnimation.obj
 0001:0007b170       ??$__ucopy@PEAUSPlayingSequence@CFacialAnimationContext@@PEAU12@_J@priv@stlpmtx_std@@YAPEAUSPlayingSequence@CFacialAnimationContext@@PEAU23@00AEBUrandom_access_iterator_tag@1@PEA_J@Z 000000003157c170 f i FaceAnimation.obj
 0001:0007b230       ??$__unguarded_linear_insert@PEAU?$pair@V?$CryStringT@D@@PEAUIFacialAnimChannel@@@stlpmtx_std@@U12@VFirstLess@?$VectorMap@V?$CryStringT@D@@PEAUIFacialAnimChannel@@U?$less@V?$CryStringT@D@@@stlpmtx_std@@V?$allocator@U?$pair@V?$CryStringT@D@@PEAUIFacialAnimChannel@@@stlpmtx_std@@@4@@@@priv@stlpmtx_std@@YAXPEAU?$pair@V?$CryStringT@D@@PEAUIFacialAnimChannel@@@1@U21@VFirstLess@?$VectorMap@V?$CryStringT@D@@PEAUIFacialAnimChannel@@U?$less@V?$CryStringT@D@@@stlpmtx_std@@V?$allocator@U?$pair@V?$CryStringT@D@@PEAUIFacialAnimChannel@@@stlpmtx_std@@@4@@@@Z 000000003157c230 f i FaceAnimation.obj
 0001:0007b310       ??$swap@U?$pair@V?$CryStringT@D@@PEAUIFacialAnimChannel@@@stlpmtx_std@@@stlpmtx_std@@YAXAEAU?$pair@V?$CryStringT@D@@PEAUIFacialAnimChannel@@@0@0@Z 000000003157c310 f i FaceAnimation.obj
 0001:0007b3f0       ??$__push_heap@PEAU?$pair@V?$CryStringT@D@@PEAUIFacialAnimChannel@@@stlpmtx_std@@_JU12@VFirstLess@?$VectorMap@V?$CryStringT@D@@PEAUIFacialAnimChannel@@U?$less@V?$CryStringT@D@@@stlpmtx_std@@V?$allocator@U?$pair@V?$CryStringT@D@@PEAUIFacialAnimChannel@@@stlpmtx_std@@@4@@@@stlpmtx_std@@YAXPEAU?$pair@V?$CryStringT@D@@PEAUIFacialAnimChannel@@@0@_J1U10@VFirstLess@?$VectorMap@V?$CryStringT@D@@PEAUIFacialAnimChannel@@U?$less@V?$CryStringT@D@@@stlpmtx_std@@V?$allocator@U?$pair@V?$CryStringT@D@@PEAUIFacialAnimChannel@@@stlpmtx_std@@@4@@@@Z 000000003157c3f0 f i FaceAnimation.obj
 0001:0007b670       ?ToUnixPath@PathUtil@@YA?AV?$CryStringT@D@@AEBV2@@Z 000000003157c670 f i FaceAnimation.obj
 0001:0007b7a0       ??$AddObject@USPhoneme@@V?$allocator@USPhoneme@@@stlpmtx_std@@@ICrySizer@@QEAAXAEBV?$vector@USPhoneme@@V?$allocator@USPhoneme@@@stlpmtx_std@@@stlpmtx_std@@@Z 000000003157c7a0 f i FaceAnimation.obj
 0001:0007b830       ??$AddObject@USPlayingSequence@CFacialAnimationContext@@V?$allocator@USPlayingSequence@CFacialAnimationContext@@@stlpmtx_std@@@ICrySizer@@QEAAXAEBV?$vector@USPlayingSequence@CFacialAnimationContext@@V?$allocator@USPlayingSequence@CFacialAnimationContext@@@stlpmtx_std@@@stlpmtx_std@@@Z 000000003157c830 f i FaceAnimation.obj
 0001:0007b930       ?_M_fill_insert_aux@?$_Impl_vector@MV?$allocator@M@stlpmtx_std@@@priv@stlpmtx_std@@AEAAXPEAM_KAEBMAEBU__false_type@3@@Z 000000003157c930 f i FaceAnimation.obj
 0001:0007ba80       ??$__adjust_heap@PEAU?$pair@V?$CryStringT@D@@PEAUIFacialAnimChannel@@@stlpmtx_std@@_JU12@VFirstLess@?$VectorMap@V?$CryStringT@D@@PEAUIFacialAnimChannel@@U?$less@V?$CryStringT@D@@@stlpmtx_std@@V?$allocator@U?$pair@V?$CryStringT@D@@PEAUIFacialAnimChannel@@@stlpmtx_std@@@4@@@@stlpmtx_std@@YAXPEAU?$pair@V?$CryStringT@D@@PEAUIFacialAnimChannel@@@0@_J1U10@VFirstLess@?$VectorMap@V?$CryStringT@D@@PEAUIFacialAnimChannel@@U?$less@V?$CryStringT@D@@@stlpmtx_std@@V?$allocator@U?$pair@V?$CryStringT@D@@PEAUIFacialAnimChannel@@@stlpmtx_std@@@4@@@@Z 000000003157ca80 f i FaceAnimation.obj
 0001:0007bbf0       ?ApplyEffector@CFacialAnimationContext@@QEAAXAEAVCFaceState@@PEAVCFacialEffector@@MM_N@Z 000000003157cbf0 f   FaceAnimation.obj
 0001:0007be60       ?ClearEffectorsLibraryFromCache@CFacialAnimation@@UEAAXPEBD@Z 000000003157ce60 f   FaceAnimation.obj
 0001:0007c090       ?UnregisterLib@CFacialAnimation@@QEAAXPEAVCFacialEffectorsLibrary@@@Z 000000003157d090 f   FaceAnimation.obj
 0001:0007c110       ?OnSequenceStreamed@CFacialAnimation@@QEAAXPEAUIFacialAnimSequence@@_N@Z 000000003157d110 f   FaceAnimation.obj
 0001:0007c1d0       ?GetMemoryUsage@CFacialAnimationContext@@QEBAXPEAVICrySizer@@@Z 000000003157d1d0 f   FaceAnimation.obj
 0001:0007c290       ?erase@?$_Impl_vector@USFacialEffectorChannel@@V?$allocator@USFacialEffectorChannel@@@stlpmtx_std@@@priv@stlpmtx_std@@QEAAPEAUSFacialEffectorChannel@@PEAU4@@Z 000000003157d290 f i FaceAnimation.obj
 0001:0007c310       ?erase@?$_Impl_vector@USPlayingSequence@CFacialAnimationContext@@V?$allocator@USPlayingSequence@CFacialAnimationContext@@@stlpmtx_std@@@priv@stlpmtx_std@@QEAAPEAUSPlayingSequence@CFacialAnimationContext@@PEAU45@@Z 000000003157d310 f i FaceAnimation.obj
 0001:0007c3a0       ?RemoveExtension@PathUtil@@YAXAEAV?$CryStringT@D@@@Z 000000003157d3a0 f i FaceAnimation.obj
 0001:0007c4d0       ?ReplaceExtension@PathUtil@@YA?AV?$CryStringT@D@@AEBV2@PEBD@Z 000000003157d4d0 f i FaceAnimation.obj
 0001:0007c560       ?ReplaceExtension@PathUtil@@YA?AV?$CryStringT@D@@PEBD0@Z 000000003157d560 f i FaceAnimation.obj
 0001:0007c6a0       ?_M_clear_after_move@?$_Impl_vector@USFacialEffectorChannel@@V?$allocator@USFacialEffectorChannel@@@stlpmtx_std@@@priv@stlpmtx_std@@AEAAXXZ 000000003157d6a0 f i FaceAnimation.obj
 0001:0007c710       ?_M_clear_after_move@?$_Impl_vector@USPlayingSequence@CFacialAnimationContext@@V?$allocator@USPlayingSequence@CFacialAnimationContext@@@stlpmtx_std@@@priv@stlpmtx_std@@AEAAXXZ 000000003157d710 f i FaceAnimation.obj
 0001:0007c790       ??$__unguarded_insertion_sort@PEAU?$pair@V?$CryStringT@D@@PEAUIFacialAnimChannel@@@stlpmtx_std@@VFirstLess@?$VectorMap@V?$CryStringT@D@@PEAUIFacialAnimChannel@@U?$less@V?$CryStringT@D@@@stlpmtx_std@@V?$allocator@U?$pair@V?$CryStringT@D@@PEAUIFacialAnimChannel@@@stlpmtx_std@@@4@@@@priv@stlpmtx_std@@YAXPEAU?$pair@V?$CryStringT@D@@PEAUIFacialAnimChannel@@@1@0VFirstLess@?$VectorMap@V?$CryStringT@D@@PEAUIFacialAnimChannel@@U?$less@V?$CryStringT@D@@@stlpmtx_std@@V?$allocator@U?$pair@V?$CryStringT@D@@PEAUIFacialAnimChannel@@@stlpmtx_std@@@4@@@@Z 000000003157d790 f i FaceAnimation.obj
 0001:0007c810       ??$__pop_heap@PEAU?$pair@V?$CryStringT@D@@PEAUIFacialAnimChannel@@@stlpmtx_std@@U12@VFirstLess@?$VectorMap@V?$CryStringT@D@@PEAUIFacialAnimChannel@@U?$less@V?$CryStringT@D@@@stlpmtx_std@@V?$allocator@U?$pair@V?$CryStringT@D@@PEAUIFacialAnimChannel@@@stlpmtx_std@@@4@@@_J@stlpmtx_std@@YAXPEAU?$pair@V?$CryStringT@D@@PEAUIFacialAnimChannel@@@0@00U10@VFirstLess@?$VectorMap@V?$CryStringT@D@@PEAUIFacialAnimChannel@@U?$less@V?$CryStringT@D@@@stlpmtx_std@@V?$allocator@U?$pair@V?$CryStringT@D@@PEAUIFacialAnimChannel@@@stlpmtx_std@@@4@@@PEA_J@Z 000000003157d810 f i FaceAnimation.obj
 0001:0007c8d0       ??$__make_heap@PEAU?$pair@V?$CryStringT@D@@PEAUIFacialAnimChannel@@@stlpmtx_std@@VFirstLess@?$VectorMap@V?$CryStringT@D@@PEAUIFacialAnimChannel@@U?$less@V?$CryStringT@D@@@stlpmtx_std@@V?$allocator@U?$pair@V?$CryStringT@D@@PEAUIFacialAnimChannel@@@stlpmtx_std@@@4@@@U12@_J@stlpmtx_std@@YAXPEAU?$pair@V?$CryStringT@D@@PEAUIFacialAnimChannel@@@0@0VFirstLess@?$VectorMap@V?$CryStringT@D@@PEAUIFacialAnimChannel@@U?$less@V?$CryStringT@D@@@stlpmtx_std@@V?$allocator@U?$pair@V?$CryStringT@D@@PEAUIFacialAnimChannel@@@stlpmtx_std@@@4@@@0PEA_J@Z 000000003157d8d0 f i FaceAnimation.obj
 0001:0007c990       ?LoadJoystickSet@CFacialAnimation@@UEAAPEAVIJoystickSet@@PEBD_N@Z 000000003157d990 f   FaceAnimation.obj
 0001:0007cc00       ??1?$_Impl_vector@UChannelInfo@CFacialAnimSequenceInstance@@V?$allocator@UChannelInfo@CFacialAnimSequenceInstance@@@stlpmtx_std@@@priv@stlpmtx_std@@QEAA@XZ 000000003157dc00 f i FaceAnimation.obj
 0001:0007cc80       ??1?$_Impl_vector@USFacialEffectorChannel@@V?$allocator@USFacialEffectorChannel@@@stlpmtx_std@@@priv@stlpmtx_std@@QEAA@XZ 000000003157dc80 f i FaceAnimation.obj
 0001:0007cd00       ??1?$_Impl_vector@USPlayingSequence@CFacialAnimationContext@@V?$allocator@USPlayingSequence@CFacialAnimationContext@@@stlpmtx_std@@@priv@stlpmtx_std@@QEAA@XZ 000000003157dd00 f i FaceAnimation.obj
 0001:0007cd80       ?erase@?$_Impl_vector@USPlayingSequence@CFacialAnimationContext@@V?$allocator@USPlayingSequence@CFacialAnimationContext@@@stlpmtx_std@@@priv@stlpmtx_std@@QEAAPEAUSPlayingSequence@CFacialAnimationContext@@PEAU45@0@Z 000000003157dd80 f i FaceAnimation.obj
 0001:0007ce40       ?erase@?$_Rb_tree@V?$CryStringT@D@@U?$less_stricmp@V?$CryStringT@D@@@stl@@U?$pair@$$CBV?$CryStringT@D@@V?$_smart_ptr@UIFacialAnimSequence@@@@@stlpmtx_std@@U?$_Select1st@U?$pair@$$CBV?$CryStringT@D@@V?$_smart_ptr@UIFacialAnimSequence@@@@@stlpmtx_std@@@priv@5@U?$_MapTraitsT@U?$pair@$$CBV?$CryStringT@D@@V?$_smart_ptr@UIFacialAnimSequence@@@@@stlpmtx_std@@@75@V?$allocator@U?$pair@$$CBV?$CryStringT@D@@V?$_smart_ptr@UIFacialAnimSequence@@@@@stlpmtx_std@@@5@@priv@stlpmtx_std@@QEAAXU?$_Rb_tree_iterator@U?$pair@$$CBV?$CryStringT@D@@V?$_smart_ptr@UIFacialAnimSequence@@@@@stlpmtx_std@@U?$_MapTraitsT@U?$pair@$$CBV?$CryStringT@D@@V?$_smart_ptr@UIFacialAnimSequence@@@@@stlpmtx_std@@@priv@2@@23@@Z 000000003157de40 f i FaceAnimation.obj
 0001:0007cec0       ?_M_insert_overflow_aux@?$_Impl_vector@USFacialEffectorChannel@@V?$allocator@USFacialEffectorChannel@@@stlpmtx_std@@@priv@stlpmtx_std@@AEAAXPEAUSFacialEffectorChannel@@AEBU4@AEBU__false_type@3@_K_N@Z 000000003157dec0 f i FaceAnimation.obj
 0001:0007d070       ?_M_erase@?$_Rb_tree@V?$CryStringT@D@@U?$less_stricmp@V?$CryStringT@D@@@stl@@U?$pair@$$CBV?$CryStringT@D@@V?$_smart_ptr@UIFacialAnimSequence@@@@@stlpmtx_std@@U?$_Select1st@U?$pair@$$CBV?$CryStringT@D@@V?$_smart_ptr@UIFacialAnimSequence@@@@@stlpmtx_std@@@priv@5@U?$_MapTraitsT@U?$pair@$$CBV?$CryStringT@D@@V?$_smart_ptr@UIFacialAnimSequence@@@@@stlpmtx_std@@@75@V?$allocator@U?$pair@$$CBV?$CryStringT@D@@V?$_smart_ptr@UIFacialAnimSequence@@@@@stlpmtx_std@@@5@@priv@stlpmtx_std@@AEAAXPEAU_Rb_tree_node_base@23@@Z 000000003157e070 f i FaceAnimation.obj
 0001:0007d100       ??$push_back_unique@V?$vector@PEAVCFacialEffectorsLibrary@@V?$allocator@PEAVCFacialEffectorsLibrary@@@stlpmtx_std@@@stlpmtx_std@@PEAVCFacialEffectorsLibrary@@@stl@@YA_NAEAV?$vector@PEAVCFacialEffectorsLibrary@@V?$allocator@PEAVCFacialEffectorsLibrary@@@stlpmtx_std@@@stlpmtx_std@@AEBQEAVCFacialEffectorsLibrary@@@Z 000000003157e100 f i FaceAnimation.obj
 0001:0007d1b0       ?_M_create_node@?$_Rb_tree@V?$CryStringT@D@@U?$less_stricmp@V?$CryStringT@D@@@stl@@U?$pair@$$CBV?$CryStringT@D@@V?$_smart_ptr@UIFacialAnimSequence@@@@@stlpmtx_std@@U?$_Select1st@U?$pair@$$CBV?$CryStringT@D@@V?$_smart_ptr@UIFacialAnimSequence@@@@@stlpmtx_std@@@priv@5@U?$_MapTraitsT@U?$pair@$$CBV?$CryStringT@D@@V?$_smart_ptr@UIFacialAnimSequence@@@@@stlpmtx_std@@@75@V?$allocator@U?$pair@$$CBV?$CryStringT@D@@V?$_smart_ptr@UIFacialAnimSequence@@@@@stlpmtx_std@@@5@@priv@stlpmtx_std@@IEAAPEAU_Rb_tree_node_base@23@AEBU?$pair@$$CBV?$CryStringT@D@@V?$_smart_ptr@UIFacialAnimSequence@@@@@3@@Z 000000003157e1b0 f i FaceAnimation.obj
 0001:0007d250       ??$__unguarded_partition@PEAU?$pair@V?$CryStringT@D@@PEAUIFacialAnimChannel@@@stlpmtx_std@@U12@VFirstLess@?$VectorMap@V?$CryStringT@D@@PEAUIFacialAnimChannel@@U?$less@V?$CryStringT@D@@@stlpmtx_std@@V?$allocator@U?$pair@V?$CryStringT@D@@PEAUIFacialAnimChannel@@@stlpmtx_std@@@4@@@@priv@stlpmtx_std@@YAPEAU?$pair@V?$CryStringT@D@@PEAUIFacialAnimChannel@@@1@PEAU21@0U21@VFirstLess@?$VectorMap@V?$CryStringT@D@@PEAUIFacialAnimChannel@@U?$less@V?$CryStringT@D@@@stlpmtx_std@@V?$allocator@U?$pair@V?$CryStringT@D@@PEAUIFacialAnimChannel@@@stlpmtx_std@@@4@@@@Z 000000003157e250 f i FaceAnimation.obj
 0001:0007d380       ??$copy_backward@PEAU?$pair@V?$CryStringT@D@@PEAUIFacialAnimChannel@@@stlpmtx_std@@PEAU12@@stlpmtx_std@@YAPEAU?$pair@V?$CryStringT@D@@PEAUIFacialAnimChannel@@@0@PEAU10@00@Z 000000003157e380 f i FaceAnimation.obj
 0001:0007d3f0       ?StopChannel@CFacialAnimationContext@@QEAAXIM@Z 000000003157e3f0 f   FaceAnimation.obj
 0001:0007d4d0       ?RemoveChannel@CFacialAnimationContext@@QEAAXI@Z 000000003157e4d0 f   FaceAnimation.obj
 0001:0007d600       ?RemoveAllPreviewChannels@CFacialAnimationContext@@QEAAXXZ 000000003157e600 f   FaceAnimation.obj
 0001:0007d6b0       ?StopSequence@CFacialAnimationContext@@QEAAXPEAVCFacialAnimSequence@@@Z 000000003157e6b0 f   FaceAnimation.obj
 0001:0007d790       ?RegisterLib@CFacialAnimation@@QEAAXPEAVCFacialEffectorsLibrary@@@Z 000000003157e790 f   FaceAnimation.obj
 0001:0007d7b0       ?GetMemoryUsage@CFacialAnimation@@QEBAXPEAVICrySizer@@@Z 000000003157e7b0 f   FaceAnimation.obj
 0001:0007d810       ?_M_clear_after_move@?$_Impl_vector@U?$pair@V?$CryStringT@D@@PEAUIFacialAnimChannel@@@stlpmtx_std@@V?$allocator@U?$pair@V?$CryStringT@D@@PEAUIFacialAnimChannel@@@stlpmtx_std@@@2@@priv@stlpmtx_std@@AEAAXXZ 000000003157e810 f i FaceAnimation.obj
 0001:0007d810       ?_M_clear@?$_Impl_vector@U?$pair@V?$CryStringT@D@@PEAUIFacialAnimChannel@@@stlpmtx_std@@V?$allocator@U?$pair@V?$CryStringT@D@@PEAUIFacialAnimChannel@@@stlpmtx_std@@@2@@priv@stlpmtx_std@@AEAAXXZ 000000003157e810 f i FaceAnimation.obj
 0001:0007d890       ?_M_insert@?$_Rb_tree@V?$CryStringT@D@@U?$less_stricmp@V?$CryStringT@D@@@stl@@U?$pair@$$CBV?$CryStringT@D@@V?$_smart_ptr@UIFacialAnimSequence@@@@@stlpmtx_std@@U?$_Select1st@U?$pair@$$CBV?$CryStringT@D@@V?$_smart_ptr@UIFacialAnimSequence@@@@@stlpmtx_std@@@priv@5@U?$_MapTraitsT@U?$pair@$$CBV?$CryStringT@D@@V?$_smart_ptr@UIFacialAnimSequence@@@@@stlpmtx_std@@@75@V?$allocator@U?$pair@$$CBV?$CryStringT@D@@V?$_smart_ptr@UIFacialAnimSequence@@@@@stlpmtx_std@@@5@@priv@stlpmtx_std@@AEAA?AU?$_Rb_tree_iterator@U?$pair@$$CBV?$CryStringT@D@@V?$_smart_ptr@UIFacialAnimSequence@@@@@stlpmtx_std@@U?$_MapTraitsT@U?$pair@$$CBV?$CryStringT@D@@V?$_smart_ptr@UIFacialAnimSequence@@@@@stlpmtx_std@@@priv@2@@23@PEAU_Rb_tree_node_base@23@AEBU?$pair@$$CBV?$CryStringT@D@@V?$_smart_ptr@UIFacialAnimSequence@@@@@3@00@Z 000000003157e890 f i FaceAnimation.obj
 0001:0007d960       ?insert_unique@?$_Rb_tree@V?$CryStringT@D@@U?$less_stricmp@V?$CryStringT@D@@@stl@@U?$pair@$$CBV?$CryStringT@D@@V?$_smart_ptr@UIFacialAnimSequence@@@@@stlpmtx_std@@U?$_Select1st@U?$pair@$$CBV?$CryStringT@D@@V?$_smart_ptr@UIFacialAnimSequence@@@@@stlpmtx_std@@@priv@5@U?$_MapTraitsT@U?$pair@$$CBV?$CryStringT@D@@V?$_smart_ptr@UIFacialAnimSequence@@@@@stlpmtx_std@@@75@V?$allocator@U?$pair@$$CBV?$CryStringT@D@@V?$_smart_ptr@UIFacialAnimSequence@@@@@stlpmtx_std@@@5@@priv@stlpmtx_std@@QEAA?AU?$pair@U?$_Rb_tree_iterator@U?$pair@$$CBV?$CryStringT@D@@V?$_smart_ptr@UIFacialAnimSequence@@@@@stlpmtx_std@@U?$_MapTraitsT@U?$pair@$$CBV?$CryStringT@D@@V?$_smart_ptr@UIFacialAnimSequence@@@@@stlpmtx_std@@@priv@2@@priv@stlpmtx_std@@_N@3@AEBU?$pair@$$CBV?$CryStringT@D@@V?$_smart_ptr@UIFacialAnimSequence@@@@@3@@Z 000000003157e960 f i FaceAnimation.obj
 0001:0007db90       ??$__linear_insert@PEAU?$pair@V?$CryStringT@D@@PEAUIFacialAnimChannel@@@stlpmtx_std@@U12@VFirstLess@?$VectorMap@V?$CryStringT@D@@PEAUIFacialAnimChannel@@U?$less@V?$CryStringT@D@@@stlpmtx_std@@V?$allocator@U?$pair@V?$CryStringT@D@@PEAUIFacialAnimChannel@@@stlpmtx_std@@@4@@@@priv@stlpmtx_std@@YAXPEAU?$pair@V?$CryStringT@D@@PEAUIFacialAnimChannel@@@1@0U21@VFirstLess@?$VectorMap@V?$CryStringT@D@@PEAUIFacialAnimChannel@@U?$less@V?$CryStringT@D@@@stlpmtx_std@@V?$allocator@U?$pair@V?$CryStringT@D@@PEAUIFacialAnimChannel@@@stlpmtx_std@@@4@@@@Z 000000003157eb90 f i FaceAnimation.obj
 0001:0007dc80       ??$sort_heap@PEAU?$pair@V?$CryStringT@D@@PEAUIFacialAnimChannel@@@stlpmtx_std@@VFirstLess@?$VectorMap@V?$CryStringT@D@@PEAUIFacialAnimChannel@@U?$less@V?$CryStringT@D@@@stlpmtx_std@@V?$allocator@U?$pair@V?$CryStringT@D@@PEAUIFacialAnimChannel@@@stlpmtx_std@@@4@@@@stlpmtx_std@@YAXPEAU?$pair@V?$CryStringT@D@@PEAUIFacialAnimChannel@@@0@0VFirstLess@?$VectorMap@V?$CryStringT@D@@PEAUIFacialAnimChannel@@U?$less@V?$CryStringT@D@@@stlpmtx_std@@V?$allocator@U?$pair@V?$CryStringT@D@@PEAUIFacialAnimChannel@@@stlpmtx_std@@@4@@@@Z 000000003157ec80 f i FaceAnimation.obj
 0001:0007dd50       ??0CFacialAnimSequenceInstance@@QEAA@XZ 000000003157ed50 f i FaceAnimation.obj
 0001:0007de30       ??1CFacialAnimSequenceInstance@@UEAA@XZ 000000003157ee30 f i FaceAnimation.obj
 0001:0007ded0       ??_GCFacialAnimSequenceInstance@@UEAAPEAXI@Z 000000003157eed0 f i FaceAnimation.obj
 0001:0007ded0       ??_ECFacialAnimSequenceInstance@@UEAAPEAXI@Z 000000003157eed0 f i FaceAnimation.obj
 0001:0007df00       ??0CFacialAnimationContext@@QEAA@PEAVCFacialInstance@@@Z 000000003157ef00 f   FaceAnimation.obj
 0001:0007e020       ??1CFacialAnimationContext@@UEAA@XZ 000000003157f020 f i FaceAnimation.obj
 0001:0007e0d0       ??_GCFacialAnimationContext@@UEAAPEAXI@Z 000000003157f0d0 f i FaceAnimation.obj
 0001:0007e0d0       ??_ECFacialAnimationContext@@UEAAPEAXI@Z 000000003157f0d0 f i FaceAnimation.obj
 0001:0007e100       ?UpdatePlayingSequences@CFacialAnimationContext@@QEAAXAEBU?$QuatTS_tpl@M@@@Z 000000003157f100 f   FaceAnimation.obj
 0001:0007e640       ??1?$_Impl_vector@U?$pair@V?$CryStringT@D@@PEAUIFacialAnimChannel@@@stlpmtx_std@@V?$allocator@U?$pair@V?$CryStringT@D@@PEAUIFacialAnimChannel@@@stlpmtx_std@@@2@@priv@stlpmtx_std@@QEAA@XZ 000000003157f640 f i FaceAnimation.obj
 0001:0007e640       ??1?$_Impl_vector@U?$pair@V?$CryStringT@D@@H@stlpmtx_std@@V?$allocator@U?$pair@V?$CryStringT@D@@H@stlpmtx_std@@@2@@priv@stlpmtx_std@@QEAA@XZ 000000003157f640 f i LoaderSKIN.obj
 0001:0007e6d0       ?push_back@?$_Impl_vector@USPlayingSequence@CFacialAnimationContext@@V?$allocator@USPlayingSequence@CFacialAnimationContext@@@stlpmtx_std@@@priv@stlpmtx_std@@QEAAXAEBUSPlayingSequence@CFacialAnimationContext@@@Z 000000003157f6d0 f i FaceAnimation.obj
 0001:0007e7f0       ?_M_insert_overflow_aux@?$_Impl_vector@U?$pair@V?$CryStringT@D@@PEAUIFacialAnimChannel@@@stlpmtx_std@@V?$allocator@U?$pair@V?$CryStringT@D@@PEAUIFacialAnimChannel@@@stlpmtx_std@@@2@@priv@stlpmtx_std@@AEAAXPEAU?$pair@V?$CryStringT@D@@PEAUIFacialAnimChannel@@@3@AEBU43@AEBU__false_type@3@_K_N@Z 000000003157f7f0 f i FaceAnimation.obj
 0001:0007ea10       ?insert_unique@?$_Rb_tree@V?$CryStringT@D@@U?$less_stricmp@V?$CryStringT@D@@@stl@@U?$pair@$$CBV?$CryStringT@D@@V?$_smart_ptr@UIFacialAnimSequence@@@@@stlpmtx_std@@U?$_Select1st@U?$pair@$$CBV?$CryStringT@D@@V?$_smart_ptr@UIFacialAnimSequence@@@@@stlpmtx_std@@@priv@5@U?$_MapTraitsT@U?$pair@$$CBV?$CryStringT@D@@V?$_smart_ptr@UIFacialAnimSequence@@@@@stlpmtx_std@@@75@V?$allocator@U?$pair@$$CBV?$CryStringT@D@@V?$_smart_ptr@UIFacialAnimSequence@@@@@stlpmtx_std@@@5@@priv@stlpmtx_std@@QEAA?AU?$_Rb_tree_iterator@U?$pair@$$CBV?$CryStringT@D@@V?$_smart_ptr@UIFacialAnimSequence@@@@@stlpmtx_std@@U?$_MapTraitsT@U?$pair@$$CBV?$CryStringT@D@@V?$_smart_ptr@UIFacialAnimSequence@@@@@stlpmtx_std@@@priv@2@@23@U423@AEBU?$pair@$$CBV?$CryStringT@D@@V?$_smart_ptr@UIFacialAnimSequence@@@@@3@@Z 000000003157fa10 f i FaceAnimation.obj
 0001:0007ef10       ??$_M_allocate_and_copy@PEAU?$pair@V?$CryStringT@D@@PEAUIFacialAnimChannel@@@stlpmtx_std@@@?$_Impl_vector@U?$pair@V?$CryStringT@D@@PEAUIFacialAnimChannel@@@stlpmtx_std@@V?$allocator@U?$pair@V?$CryStringT@D@@PEAUIFacialAnimChannel@@@stlpmtx_std@@@2@@priv@stlpmtx_std@@AEAAPEAU?$pair@V?$CryStringT@D@@PEAUIFacialAnimChannel@@@2@AEA_KPEAU32@1@Z 000000003157ff10 f i FaceAnimation.obj
 0001:0007efe0       ??$__insertion_sort@PEAU?$pair@V?$CryStringT@D@@PEAUIFacialAnimChannel@@@stlpmtx_std@@U12@VFirstLess@?$VectorMap@V?$CryStringT@D@@PEAUIFacialAnimChannel@@U?$less@V?$CryStringT@D@@@stlpmtx_std@@V?$allocator@U?$pair@V?$CryStringT@D@@PEAUIFacialAnimChannel@@@stlpmtx_std@@@4@@@@priv@stlpmtx_std@@YAXPEAU?$pair@V?$CryStringT@D@@PEAUIFacialAnimChannel@@@1@00VFirstLess@?$VectorMap@V?$CryStringT@D@@PEAUIFacialAnimChannel@@U?$less@V?$CryStringT@D@@@stlpmtx_std@@V?$allocator@U?$pair@V?$CryStringT@D@@PEAUIFacialAnimChannel@@@stlpmtx_std@@@4@@@@Z 000000003157ffe0 f i FaceAnimation.obj
 0001:0007f080       ??$__partial_sort@PEAU?$pair@V?$CryStringT@D@@PEAUIFacialAnimChannel@@@stlpmtx_std@@U12@VFirstLess@?$VectorMap@V?$CryStringT@D@@PEAUIFacialAnimChannel@@U?$less@V?$CryStringT@D@@@stlpmtx_std@@V?$allocator@U?$pair@V?$CryStringT@D@@PEAUIFacialAnimChannel@@@stlpmtx_std@@@4@@@@priv@stlpmtx_std@@YAXPEAU?$pair@V?$CryStringT@D@@PEAUIFacialAnimChannel@@@1@000VFirstLess@?$VectorMap@V?$CryStringT@D@@PEAUIFacialAnimChannel@@U?$less@V?$CryStringT@D@@@stlpmtx_std@@V?$allocator@U?$pair@V?$CryStringT@D@@PEAUIFacialAnimChannel@@@stlpmtx_std@@@4@@@@Z 0000000031580080 f i FaceAnimation.obj
 0001:0007f170       ?ResetFaceState@CFacialAnimationContext@@AEAAXAEAVCFaceState@@@Z 0000000031580170 f   FaceAnimation.obj
 0001:0007f320       ?StopAllSequences@CFacialAnimationContext@@QEAAXXZ 0000000031580320 f   FaceAnimation.obj
 0001:0007f3c0       ??1CFacialAnimation@@UEAA@XZ 00000000315803c0 f   FaceAnimation.obj
 0001:0007f480       ??_ECFacialAnimation@@W7EAAPEAXI@Z 0000000031580480 f i FaceAnimation.obj
 0001:0007f490       ?ClearAllCaches@CFacialAnimation@@UEAAXXZ 0000000031580490 f   FaceAnimation.obj
 0001:0007f4f0       ?ClearSequenceFromCache@CFacialAnimation@@UEAAXPEBD@Z 00000000315804f0 f   FaceAnimation.obj
 0001:0007f610       ?reserve@?$_Impl_vector@U?$pair@V?$CryStringT@D@@PEAUIFacialAnimChannel@@@stlpmtx_std@@V?$allocator@U?$pair@V?$CryStringT@D@@PEAUIFacialAnimChannel@@@stlpmtx_std@@@2@@priv@stlpmtx_std@@QEAAX_K@Z 0000000031580610 f i FaceAnimation.obj
 0001:0007f6d0       ?StartChannel@CFacialAnimationContext@@QEAAIAEAUSFacialEffectorChannel@@@Z 00000000315806d0 f   FaceAnimation.obj
 0001:0007f770       ?FadeInChannel@CFacialAnimationContext@@QEAAIPEAUIFacialEffector@@MMMH@Z 0000000031580770 f   FaceAnimation.obj
 0001:0007f9c0       ?Update@CFacialAnimationContext@@QEAA_NAEAVCFaceState@@AEBU?$QuatTS_tpl@M@@@Z 00000000315809c0 f   FaceAnimation.obj
 0001:000800a0       ?PlaySequence@CFacialAnimationContext@@QEAAXPEAVCFacialAnimSequence@@_N1@Z 00000000315810a0 f   FaceAnimation.obj
 0001:00080270       ??0CFacialAnimation@@QEAA@XZ 0000000031581270 f   FaceAnimation.obj
 0001:00080340       ??_ECFacialAnimation@@UEAAPEAXI@Z 0000000031581340 f i FaceAnimation.obj
 0001:00080340       ??_GCFacialAnimation@@UEAAPEAXI@Z 0000000031581340 f i FaceAnimation.obj
 0001:00080370       ??$?AV?$CryStringT@D@@@?$map@V?$CryStringT@D@@V?$_smart_ptr@UIFacialAnimSequence@@@@U?$less_stricmp@V?$CryStringT@D@@@stl@@V?$allocator@U?$pair@$$CBV?$CryStringT@D@@V?$_smart_ptr@UIFacialAnimSequence@@@@@stlpmtx_std@@@stlpmtx_std@@@stlpmtx_std@@QEAAAEAV?$_smart_ptr@UIFacialAnimSequence@@@@AEBV?$CryStringT@D@@@Z 0000000031581370 f i FaceAnimation.obj
 0001:00080460       ??$__introsort_loop@PEAU?$pair@V?$CryStringT@D@@PEAUIFacialAnimChannel@@@stlpmtx_std@@U12@_JVFirstLess@?$VectorMap@V?$CryStringT@D@@PEAUIFacialAnimChannel@@U?$less@V?$CryStringT@D@@@stlpmtx_std@@V?$allocator@U?$pair@V?$CryStringT@D@@PEAUIFacialAnimChannel@@@stlpmtx_std@@@4@@@@priv@stlpmtx_std@@YAXPEAU?$pair@V?$CryStringT@D@@PEAUIFacialAnimChannel@@@1@00_JVFirstLess@?$VectorMap@V?$CryStringT@D@@PEAUIFacialAnimChannel@@U?$less@V?$CryStringT@D@@@stlpmtx_std@@V?$allocator@U?$pair@V?$CryStringT@D@@PEAUIFacialAnimChannel@@@stlpmtx_std@@@4@@@@Z 0000000031581460 f i FaceAnimation.obj
 0001:00080570       ?RenameAnimSequence@CFacialAnimation@@QEAAXPEAVCFacialAnimSequence@@PEBD_N@Z 0000000031581570 f   FaceAnimation.obj
 0001:00080700       ?LoadSequence@CFacialAnimation@@UEAAPEAUIFacialAnimSequence@@PEBD_N1@Z 0000000031581700 f   FaceAnimation.obj
 0001:00080b90       ?StartStreamingSequence@CFacialAnimation@@UEAAPEAUIFacialAnimSequence@@PEBD@Z 0000000031581b90 f   FaceAnimation.obj
 0001:00080f30       ??$sort@PEAU?$pair@V?$CryStringT@D@@PEAUIFacialAnimChannel@@@stlpmtx_std@@VFirstLess@?$VectorMap@V?$CryStringT@D@@PEAUIFacialAnimChannel@@U?$less@V?$CryStringT@D@@@stlpmtx_std@@V?$allocator@U?$pair@V?$CryStringT@D@@PEAUIFacialAnimChannel@@@stlpmtx_std@@@4@@@@stlpmtx_std@@YAXPEAU?$pair@V?$CryStringT@D@@PEAUIFacialAnimChannel@@@0@0VFirstLess@?$VectorMap@V?$CryStringT@D@@PEAUIFacialAnimChannel@@U?$less@V?$CryStringT@D@@@stlpmtx_std@@V?$allocator@U?$pair@V?$CryStringT@D@@PEAUIFacialAnimChannel@@@stlpmtx_std@@@4@@@@Z 0000000031581f30 f i FaceAnimation.obj
 0001:00080fe0       ?BindJoystickSetToSequence@CFacialAnimation@@UEAAXPEAVIJoystickSet@@PEAUIFacialAnimSequence@@@Z 0000000031581fe0 f   FaceAnimation.obj
 0001:00081ac0       ??_GIFacialAnimChannel@@UEAAPEAXI@Z 0000000031582ac0 f i FaceAnimSequence.obj
 0001:00081ac0       ??_EISplineInterpolator@@UEAAPEAXI@Z 0000000031582ac0 f i FaceAnimSequence.obj
 0001:00081ac0       ??_GISplineInterpolator@@UEAAPEAXI@Z 0000000031582ac0 f i FaceAnimSequence.obj
 0001:00081ac0       ??_EIFacialAnimChannel@@UEAAPEAXI@Z 0000000031582ac0 f i FaceAnimSequence.obj
 0001:00081af0       ??_EIFacialAnimSoundEntry@@UEAAPEAXI@Z 0000000031582af0 f i FaceAnimSequence.obj
 0001:00081af0       ??_GIFacialAnimSoundEntry@@UEAAPEAXI@Z 0000000031582af0 f i FaceAnimSequence.obj
 0001:00081b20       ??_GIFacialAnimSequence@@UEAAPEAXI@Z 0000000031582b20 f i FaceAnimSequence.obj
 0001:00081b20       ??_EIFacialAnimSequence@@UEAAPEAXI@Z 0000000031582b20 f i FaceAnimSequence.obj
 0001:00081b50       ?Release@CFacialAnimSequence@@UEAAXXZ 0000000031582b50 f   FaceAnimSequence.obj
 0001:00081b70       ?SetName@CFacialAnimSequence@@UEAAXPEBD@Z 0000000031582b70 f   FaceAnimSequence.obj
 0001:00081b90       ?GetStartTime@CFacialAnimSoundEntry@@UEAAMXZ 0000000031582b90 f   FaceAnimSequence.obj
 0001:00081ba0       ?SetStartTime@CFacialAnimSoundEntry@@UEAAXM@Z 0000000031582ba0 f   FaceAnimSequence.obj
 0001:00081bb0       ?SetStartTime@CFacialAnimSkeletalAnimationEntry@@UEAAXM@Z 0000000031582bb0 f   FaceAnimSequence.obj
 0001:00081bc0       ?GetStartTime@CFacialAnimSkeletalAnimationEntry@@UEBAMXZ 0000000031582bc0 f   FaceAnimSequence.obj
 0001:00081bd0       ?SetEndTime@CFacialAnimSkeletalAnimationEntry@@UEAAXM@Z 0000000031582bd0 f   FaceAnimSequence.obj
 0001:00081be0       ?GetEndTime@CFacialAnimSkeletalAnimationEntry@@UEBAMXZ 0000000031582be0 f   FaceAnimSequence.obj
 0001:00081bf0       ??_EIStreamCallback@@UEAAPEAXI@Z 0000000031582bf0 f i FaceAnimSequence.obj
 0001:00081bf0       ??_GIStreamCallback@@UEAAPEAXI@Z 0000000031582bf0 f i FaceAnimSequence.obj
 0001:00081c20       ?GetJoystickFile@CFacialAnimSequence@@UEBAPEBDXZ 0000000031582c20 f   FaceAnimSequence.obj
 0001:00081c20       ?GetName@CFacialJoystick@@UEAAPEBDXZ 0000000031582c20 f   FaceJoystick.obj
 0001:00081c30       ??$move_init@U?$TCBSplineKey@U?$Vec3_tpl@M@@@spline@@@NArray@@YAXPEAU?$TCBSplineKey@U?$Vec3_tpl@M@@@spline@@0_K@Z 0000000031582c30 f i FaceAnimSequence.obj
 0001:00081ca0       ??$__copy_backward_ptrs@PEAUChannelInfo@CFacialAnimSequenceInstance@@PEAU12@@priv@stlpmtx_std@@YAPEAUChannelInfo@CFacialAnimSequenceInstance@@PEAU23@00AEBU__false_type@1@@Z 0000000031582ca0 f i FaceAnimSequence.obj
 0001:00081d60       ??$fill@PEAUChannelInfo@CFacialAnimSequenceInstance@@U12@@stlpmtx_std@@YAXPEAUChannelInfo@CFacialAnimSequenceInstance@@0AEBU12@@Z 0000000031582d60 f i FaceAnimSequence.obj
 0001:00081e00       ??$__push_heap@PEAU?$SplineKey@M@spline@@_JU12@U?$less@U?$SplineKey@M@spline@@@stlpmtx_std@@@stlpmtx_std@@YAXPEAU?$SplineKey@M@spline@@_J1U12@U?$less@U?$SplineKey@M@spline@@@0@@Z 0000000031582e00 f i FaceAnimSequence.obj
 0001:00081ed0       ??$__push_heap@PEAU?$pair@PEAUIFacialAnimChannel@@H@stlpmtx_std@@_JU12@VFirstLess@?$VectorMap@PEAUIFacialAnimChannel@@HU?$less@PEAUIFacialAnimChannel@@@stlpmtx_std@@V?$allocator@U?$pair@PEAUIFacialAnimChannel@@H@stlpmtx_std@@@3@@@@stlpmtx_std@@YAXPEAU?$pair@PEAUIFacialAnimChannel@@H@0@_J1U10@VFirstLess@?$VectorMap@PEAUIFacialAnimChannel@@HU?$less@PEAUIFacialAnimChannel@@@stlpmtx_std@@V?$allocator@U?$pair@PEAUIFacialAnimChannel@@H@stlpmtx_std@@@3@@@@Z 0000000031582ed0 f i FaceAnimSequence.obj
 0001:00081f60       ?GetMemoryUsage@CFacialSentence@@QEBAXPEAVICrySizer@@@Z 0000000031582f60 f i FaceAnimSequence.obj
 0001:00082000       ?GetChannel@CFacialAnimSequence@@UEAAPEAUIFacialAnimChannel@@H@Z 0000000031583000 f   FaceAnimSequence.obj
 0001:00082010       ?GetSoundEntryCount@CFacialAnimSequence@@UEAAHXZ 0000000031583010 f   FaceAnimSequence.obj
 0001:00082020       ?GetSoundEntry@CFacialAnimSequence@@UEAAPEAUIFacialAnimSoundEntry@@H@Z 0000000031583020 f   FaceAnimSequence.obj
 0001:00082050       ?SerializeChannelSave@CFacialAnimSequence@@AEAAXPEAUIFacialAnimChannel@@AEAVXmlNodeRef@@@Z 0000000031583050 f   FaceAnimSequence.obj
 0001:000821e0       ?GetSkeletonAnimationEntryCount@CFacialAnimSequence@@UEAAHXZ 00000000315831e0 f   FaceAnimSequence.obj
 0001:00082210       ?GetSkeletonAnimationEntry@CFacialAnimSequence@@UEAAPEAUIFacialAnimSkeletonAnimationEntry@@H@Z 0000000031583210 f   FaceAnimSequence.obj
 0001:00082280       ?GenerateProceduralChannels@CFacialAnimSequence@@AEAAXAEAUData@1@@Z 0000000031583280 f   FaceAnimSequence.obj
 0001:00082720       ??4?$_smart_ptr@VIReadStream@@@@QEAAAEAV0@AEBV0@@Z 0000000031583720 f i FaceAnimSequence.obj
 0001:000827a0       ?resize_raw@?$SmallDynStorage@U?$SplineKey@M@spline@@HUStandardAlloc@NAlloc@@@NArray@@QEAAXHH_N@Z 00000000315837a0 f i FaceAnimSequence.obj
 0001:00082960       ?set_size@?$SmallDynStorage@VCModelMesh@@HUStandardAlloc@NAlloc@@@NArray@@QEAAXH@Z 0000000031583960 f i LoaderSKIN.obj
 0001:00082960       ?set_size@?$SmallDynStorage@U?$SplineKey@U?$Quat_tpl@M@@@spline@@HUStandardAlloc@NAlloc@@@NArray@@QEAAXH@Z 0000000031583960 f i FaceAnimSequence.obj
 0001:00082a10       ?expand_raw@?$DynArray@U?$SplineKey@M@spline@@HU?$SmallDynStorage@U?$SplineKey@M@spline@@HUStandardAlloc@NAlloc@@@NArray@@@@IEAAPEAU?$SplineKey@M@spline@@PEAU23@H@Z 0000000031583a10 f i FaceAnimSequence.obj
 0001:00082ad0       ??$AddObject@V?$_smart_ptr@VCFacialAnimChannel@@@@V?$allocator@V?$_smart_ptr@VCFacialAnimChannel@@@@@stlpmtx_std@@@ICrySizer@@QEAAXAEBV?$vector@V?$_smart_ptr@VCFacialAnimChannel@@@@V?$allocator@V?$_smart_ptr@VCFacialAnimChannel@@@@@stlpmtx_std@@@stlpmtx_std@@@Z 0000000031583ad0 f i FaceAnimSequence.obj
 0001:00082b50       ??$AddObject@UBalanceChannelEntry@CFacialAnimSequenceInstance@@V?$allocator@UBalanceChannelEntry@CFacialAnimSequenceInstance@@@stlpmtx_std@@@ICrySizer@@QEAAXAEBV?$vector@UBalanceChannelEntry@CFacialAnimSequenceInstance@@V?$allocator@UBalanceChannelEntry@CFacialAnimSequenceInstance@@@stlpmtx_std@@@stlpmtx_std@@@Z 0000000031583b50 f i FaceAnimSequence.obj
 0001:00082be0       ??$move_init@U?$SplineKey@U?$Quat_tpl@M@@@spline@@@NArray@@YAXPEAU?$SplineKey@U?$Quat_tpl@M@@@spline@@0_K@Z 0000000031583be0 f i FaceAnimSequence.obj
 0001:00082e90       ??$__copy_ptrs@PEAUChannelInfo@CFacialAnimSequenceInstance@@PEAU12@@priv@stlpmtx_std@@YAPEAUChannelInfo@CFacialAnimSequenceInstance@@PEAU23@00AEBU__false_type@1@@Z 0000000031583e90 f i FaceAnimSequence.obj
 0001:00082f50       ??$__equal_range@PEAVEffectorChannelPair@@V1@U?$__less_2@VEffectorChannelPair@@V1@@priv@stlpmtx_std@@U234@_J@priv@stlpmtx_std@@YA?AU?$pair@PEAVEffectorChannelPair@@PEAV1@@1@PEAVEffectorChannelPair@@0AEBV3@U?$__less_2@VEffectorChannelPair@@V1@@01@2PEA_J@Z 0000000031583f50 f i FaceAnimSequence.obj
 0001:00083070       ??$__adjust_heap@PEAVEffectorChannelPair@@_JV1@U?$less@VEffectorChannelPair@@@stlpmtx_std@@@stlpmtx_std@@YAXPEAVEffectorChannelPair@@_J1V1@U?$less@VEffectorChannelPair@@@0@@Z 0000000031584070 f i FaceAnimSequence.obj
 0001:00083170       ??$__adjust_heap@PEAU?$SplineKey@M@spline@@_JU12@U?$less@U?$SplineKey@M@spline@@@stlpmtx_std@@@stlpmtx_std@@YAXPEAU?$SplineKey@M@spline@@_J1U12@U?$less@U?$SplineKey@M@spline@@@0@@Z 0000000031584170 f i FaceAnimSequence.obj
 0001:00083270       ??$__adjust_heap@PEAVCFaceIdentifierHandle@@_JV1@USFaceIdentifierHandleLess@CFacialSentence@@@stlpmtx_std@@YAXPEAVCFaceIdentifierHandle@@_J1V1@USFaceIdentifierHandleLess@CFacialSentence@@@Z 0000000031584270 f i FaceAnimSequence.obj
 0001:00083380       ??$__adjust_heap@PEAU?$pair@PEAUIFacialAnimChannel@@H@stlpmtx_std@@_JU12@VFirstLess@?$VectorMap@PEAUIFacialAnimChannel@@HU?$less@PEAUIFacialAnimChannel@@@stlpmtx_std@@V?$allocator@U?$pair@PEAUIFacialAnimChannel@@H@stlpmtx_std@@@3@@@@stlpmtx_std@@YAXPEAU?$pair@PEAUIFacialAnimChannel@@H@0@_J1U10@VFirstLess@?$VectorMap@PEAUIFacialAnimChannel@@HU?$less@PEAUIFacialAnimChannel@@@stlpmtx_std@@V?$allocator@U?$pair@PEAUIFacialAnimChannel@@H@stlpmtx_std@@@3@@@@Z 0000000031584380 f i FaceAnimSequence.obj
 0001:00083440       ?CleanupKeys@CFacialAnimChannel@@UEAAXM@Z 0000000031584440 f   FaceAnimSequence.obj
 0001:00083460       ?SmoothKeys@CFacialAnimChannel@@UEAAXM@Z 0000000031584460 f   FaceAnimSequence.obj
 0001:00083480       ?RemoveNoise@CFacialAnimChannel@@UEAAXMM@Z 0000000031584480 f   FaceAnimSequence.obj
 0001:000834a0       ??1CFacialAnimSoundEntry@@UEAA@XZ 00000000315844a0 f i FaceAnimSequence.obj
 0001:00083530       ?UpdateProceduralChannels@CFacialAnimSequence@@AEAAXXZ 0000000031584530 f   FaceAnimSequence.obj
 0001:000835a0       ??_GCFacialAnimSoundEntry@@UEAAPEAXI@Z 00000000315845a0 f i FaceAnimSequence.obj
 0001:000835a0       ??_ECFacialAnimSoundEntry@@UEAAPEAXI@Z 00000000315845a0 f i FaceAnimSequence.obj
 0001:000835d0       ??_ECFacialAnimSkeletalAnimationEntry@@UEAAPEAXI@Z 00000000315845d0 f i FaceAnimSequence.obj
 0001:000835d0       ??_GCFacialAnimSkeletalAnimationEntry@@UEAAPEAXI@Z 00000000315845d0 f i FaceAnimSequence.obj
 0001:00083640       ?swap@?$TSpline@U?$TCBSplineKey@U?$Vec3_tpl@M@@@spline@@VHermitBasis@2@@spline@@QEAAXAEAV12@@Z 0000000031584640 f i FaceAnimSequence.obj
 0001:00083640       ?swap@?$TSpline@U?$SplineKey@M@spline@@VHermitBasis@2@@spline@@QEAAXAEAV12@@Z 0000000031584640 f i FaceAnimSequence.obj
 0001:00083640       ?swap@?$TSpline@U?$SplineKey@U?$Quat_tpl@M@@@spline@@VHermitBasis@2@@spline@@QEAAXAEAV12@@Z 0000000031584640 f i FaceAnimSequence.obj
 0001:000836f0       ?erase@?$vector@_NV?$allocator@_N@stlpmtx_std@@@stlpmtx_std@@QEAA?AU?$_Bit_iter@U_Bit_reference@priv@stlpmtx_std@@PEAU123@@priv@2@U342@0@Z 00000000315846f0 f i FaceAnimSequence.obj
 0001:000837e0       ?resize_raw@?$SmallDynStorage@U?$TCBSplineKey@U?$Vec3_tpl@M@@@spline@@HUStandardAlloc@NAlloc@@@NArray@@QEAAXHH_N@Z 00000000315847e0 f i FaceAnimSequence.obj
 0001:00083950       ?resize_raw@?$SmallDynStorage@U?$SplineKey@U?$Quat_tpl@M@@@spline@@HUStandardAlloc@NAlloc@@@NArray@@QEAAXHH_N@Z 0000000031584950 f i FaceAnimSequence.obj
 0001:00083ae0       ?_M_erase@?$_Impl_vector@V?$_smart_ptr@VCFacialEffCtrl@@@@V?$allocator@V?$_smart_ptr@VCFacialEffCtrl@@@@@stlpmtx_std@@@priv@stlpmtx_std@@AEAAPEAV?$_smart_ptr@VCFacialEffCtrl@@@@PEAV4@AEBU__false_type@3@@Z 0000000031584ae0 f i FaceEffector.obj
 0001:00083ae0       ?_M_erase@?$_Impl_vector@V?$_smart_ptr@VCFacialAnimChannel@@@@V?$allocator@V?$_smart_ptr@VCFacialAnimChannel@@@@@stlpmtx_std@@@priv@stlpmtx_std@@AEAAPEAV?$_smart_ptr@VCFacialAnimChannel@@@@PEAV4@AEBU__false_type@3@@Z 0000000031584ae0 f i FaceAnimSequence.obj
 0001:00083bc0       ?set_size@?$SmallDynStorage@U?$TCBSplineKey@U?$Vec3_tpl@M@@@spline@@HUStandardAlloc@NAlloc@@@NArray@@QEAAXH@Z 0000000031584bc0 f i FaceAnimSequence.obj
 0001:00083bc0       ?set_size@?$SmallDynStorage@UBSParameter@@HUStandardAlloc@NAlloc@@@NArray@@QEAAXH@Z 0000000031584bc0 f i CharacterManager.obj
 0001:00083bc0       ?set_size@?$SmallDynStorage@USMeshSubset@@HUStandardAlloc@NAlloc@@@NArray@@QEAAXH@Z 0000000031584bc0 f i LoaderCGA.obj
 0001:00083bc0       ?set_size@?$SmallDynStorage@UDirectionalBlends@@HUStandardAlloc@NAlloc@@@NArray@@QEAAXH@Z 0000000031584bc0 f i ParamLoader.obj
 0001:00083c70       ?expand_raw@?$DynArray@U?$TCBSplineKey@U?$Vec3_tpl@M@@@spline@@HU?$SmallDynStorage@U?$TCBSplineKey@U?$Vec3_tpl@M@@@spline@@HUStandardAlloc@NAlloc@@@NArray@@@@IEAAPEAU?$TCBSplineKey@U?$Vec3_tpl@M@@@spline@@PEAU23@H@Z 0000000031584c70 f i FaceAnimSequence.obj
 0001:00083d10       ?expand_raw@?$DynArray@U?$SplineKey@U?$Quat_tpl@M@@@spline@@HU?$SmallDynStorage@U?$SplineKey@U?$Quat_tpl@M@@@spline@@HUStandardAlloc@NAlloc@@@NArray@@@@IEAAPEAU?$SplineKey@U?$Quat_tpl@M@@@spline@@PEAU23@H@Z 0000000031584d10 f i FaceAnimSequence.obj
 0001:00083dd0       ??$AddObject@PEAVCFacialAnimChannelInterpolator@@V?$allocator@PEAVCFacialAnimChannelInterpolator@@@stlpmtx_std@@@ICrySizer@@QEAAXAEBV?$vector@PEAVCFacialAnimChannelInterpolator@@V?$allocator@PEAVCFacialAnimChannelInterpolator@@@stlpmtx_std@@@stlpmtx_std@@@Z 0000000031584dd0 f i FaceAnimSequence.obj
 0001:00083e60       ?_M_insert_overflow@?$_Impl_vector@U?$pair@PEAUIFacialAnimChannel@@H@stlpmtx_std@@V?$allocator@U?$pair@PEAUIFacialAnimChannel@@H@stlpmtx_std@@@2@@priv@stlpmtx_std@@AEAAXPEAU?$pair@PEAUIFacialAnimChannel@@H@3@AEBU43@AEBU__true_type@3@_K_N@Z 0000000031584e60 f i FaceAnimSequence.obj
 0001:00083fe0       ??$_M_allocate_and_copy@PEAH@?$_Impl_vector@HV?$allocator@H@stlpmtx_std@@@priv@stlpmtx_std@@AEAAPEAHAEA_KPEAH1@Z 0000000031584fe0 f i FaceAnimSequence.obj
 0001:00084090       ??$__copy@PEAV?$CryStringT@D@@PEAV1@_J@priv@stlpmtx_std@@YAPEAV?$CryStringT@D@@PEAV2@00AEBUrandom_access_iterator_tag@1@PEA_J@Z 0000000031585090 f i FaceAnimSequence.obj
 0001:00084180       ??$__uninitialized_fill_n@PEAUChannelInfo@CFacialAnimSequenceInstance@@_KU12@@priv@stlpmtx_std@@YAPEAUChannelInfo@CFacialAnimSequenceInstance@@PEAU23@_KAEBU23@@Z 0000000031585180 f i FaceAnimSequence.obj
 0001:00084230       ??$__ucopy_ptrs@PEAUChannelInfo@CFacialAnimSequenceInstance@@PEAU12@@priv@stlpmtx_std@@YAPEAUChannelInfo@CFacialAnimSequenceInstance@@PEAU23@00AEBU__false_type@1@@Z 0000000031585230 f i FaceAnimSequence.obj
 0001:000842d0       ??$__unguarded_insertion_sort@PEAU?$SplineKey@M@spline@@U?$less@U?$SplineKey@M@spline@@@stlpmtx_std@@@priv@stlpmtx_std@@YAXPEAU?$SplineKey@M@spline@@0U?$less@U?$SplineKey@M@spline@@@1@@Z 00000000315852d0 f i FaceAnimSequence.obj
 0001:00084340       ??$__copy_backward@PEAV?$CryStringT@D@@PEAV1@_J@priv@stlpmtx_std@@YAPEAV?$CryStringT@D@@PEAV2@00AEBUrandom_access_iterator_tag@1@PEA_J@Z 0000000031585340 f i FaceAnimSequence.obj
 0001:00084430       ??$__fill@PEAV?$CryStringT@D@@V1@_J@priv@stlpmtx_std@@YAXPEAV?$CryStringT@D@@0AEBV2@AEBUrandom_access_iterator_tag@1@PEA_J@Z 0000000031585430 f i FaceAnimSequence.obj
 0001:00084510       ??$__unguarded_insertion_sort@PEAU?$pair@PEAUIFacialAnimChannel@@H@stlpmtx_std@@VFirstLess@?$VectorMap@PEAUIFacialAnimChannel@@HU?$less@PEAUIFacialAnimChannel@@@stlpmtx_std@@V?$allocator@U?$pair@PEAUIFacialAnimChannel@@H@stlpmtx_std@@@3@@@@priv@stlpmtx_std@@YAXPEAU?$pair@PEAUIFacialAnimChannel@@H@1@0VFirstLess@?$VectorMap@PEAUIFacialAnimChannel@@HU?$less@PEAUIFacialAnimChannel@@@stlpmtx_std@@V?$allocator@U?$pair@PEAUIFacialAnimChannel@@H@stlpmtx_std@@@3@@@@Z 0000000031585510 f i FaceAnimSequence.obj
 0001:00084580       ??$__make_heap@PEAVEffectorChannelPair@@U?$less@VEffectorChannelPair@@@stlpmtx_std@@V1@_J@stlpmtx_std@@YAXPEAVEffectorChannelPair@@0U?$less@VEffectorChannelPair@@@0@0PEA_J@Z 0000000031585580 f i FaceAnimSequence.obj
 0001:000846e0       ??$__make_heap@PEAU?$SplineKey@M@spline@@U?$less@U?$SplineKey@M@spline@@@stlpmtx_std@@U12@_J@stlpmtx_std@@YAXPEAU?$SplineKey@M@spline@@0U?$less@U?$SplineKey@M@spline@@@0@0PEA_J@Z 00000000315856e0 f i FaceAnimSequence.obj
 0001:000848b0       ??$__make_heap@PEAVCFaceIdentifierHandle@@USFaceIdentifierHandleLess@CFacialSentence@@V1@_J@stlpmtx_std@@YAXPEAVCFaceIdentifierHandle@@0USFaceIdentifierHandleLess@CFacialSentence@@0PEA_J@Z 00000000315858b0 f i FaceAnimSequence.obj
 0001:00084a10       ??$__make_heap@PEAU?$pair@PEAUIFacialAnimChannel@@H@stlpmtx_std@@VFirstLess@?$VectorMap@PEAUIFacialAnimChannel@@HU?$less@PEAUIFacialAnimChannel@@@stlpmtx_std@@V?$allocator@U?$pair@PEAUIFacialAnimChannel@@H@stlpmtx_std@@@3@@@U12@_J@stlpmtx_std@@YAXPEAU?$pair@PEAUIFacialAnimChannel@@H@0@0VFirstLess@?$VectorMap@PEAUIFacialAnimChannel@@HU?$less@PEAUIFacialAnimChannel@@@stlpmtx_std@@V?$allocator@U?$pair@PEAUIFacialAnimChannel@@H@stlpmtx_std@@@3@@@0PEA_J@Z 0000000031585a10 f i FaceAnimSequence.obj
 0001:00084b70       ?GetMemoryUsage@CFacialAnimChannel@@QEBAXPEAVICrySizer@@@Z 0000000031585b70 f i FaceAnimSequence.obj
 0001:00084bf0       ?swap@CProceduralChannelSet@@QEAAXAEAV1@@Z 0000000031585bf0 f i FaceAnimSequence.obj
 0001:00084c80       ??1CFacialAnimChannel@@UEAA@XZ 0000000031585c80 f   FaceAnimSequence.obj
 0001:00084df0       ?SetEffectorIdentifier@CFacialAnimChannel@@UEAAXVCFaceIdentifierHandle@@@Z 0000000031585df0 f i FaceAnimSequence.obj
 0001:00084e00       ?GetEffectorIdentifier@CFacialAnimChannel@@UEAA?BVCFaceIdentifierHandle@@XZ 0000000031585e00 f i FaceAnimSequence.obj
 0001:00084e20       ?SetFlags@CFacialAnimChannel@@UEAAXI@Z 0000000031585e20 f i FaceAnimSequence.obj
 0001:00084e30       ??_ECFacialAnimChannel@@W7EAAPEAXI@Z 0000000031585e30 f i FaceAnimSequence.obj
 0001:00084e40       ?SetParent@CFacialAnimChannel@@UEAAXPEAUIFacialAnimChannel@@@Z 0000000031585e40 f i FaceAnimSequence.obj
 0001:00084e90       ?GetEffector@CFacialAnimChannel@@UEAAPEAUIFacialEffector@@XZ 0000000031585e90 f i FaceAnimSequence.obj
 0001:00084ea0       ?GetInterpolatorCount@CFacialAnimChannel@@UEBAHXZ 0000000031585ea0 f i FaceAnimSequence.obj
 0001:00084eb0       ?GetInterpolator@CFacialAnimChannel@@UEAAPEAUISplineInterpolator@@H@Z 0000000031585eb0 f i FaceAnimSequence.obj
 0001:00084ec0       ?GetLastInterpolator@CFacialAnimChannel@@UEAAPEAUISplineInterpolator@@XZ 0000000031585ec0 f i FaceAnimSequence.obj
 0001:00084ee0       ?GetName@CFacialAnimChannel@@UEBAPEBDXZ 0000000031585ee0 f i FaceAnimSequence.obj
 0001:00084f30       ?SetIdentifier@CFacialAnimChannel@@UEAAXVCFaceIdentifierHandle@@@Z 0000000031585f30 f   FaceAnimSequence.obj
 0001:00085070       ?GetIdentifier@CFacialAnimChannel@@UEAA?BVCFaceIdentifierHandle@@XZ 0000000031586070 f   FaceAnimSequence.obj
 0001:000851e0       ?SetEffector@CFacialAnimChannel@@UEAAXPEAUIFacialEffector@@@Z 00000000315861e0 f   FaceAnimSequence.obj
 0001:00085360       ?SetName@CFacialAnimChannel@@UEAAXPEBD@Z 0000000031586360 f   FaceAnimSequence.obj
 0001:000854a0       ?SetSoundFile@CFacialAnimSoundEntry@@UEAAXPEBD@Z 00000000315864a0 f   FaceAnimSequence.obj
 0001:000854a0       ?SetName@CFacialEffectorsLibrary@@UEAAXPEBD@Z 00000000315864a0 f   FaceEffectorLibrary.obj
 0001:000854f0       ?SetName@CFacialAnimSkeletalAnimationEntry@@UEAAXPEBD@Z 00000000315864f0 f   FaceAnimSequence.obj
 0001:00085540       ?clear@?$DynArray@U?$TCBSplineKey@U?$Vec3_tpl@M@@@spline@@HU?$SmallDynStorage@U?$TCBSplineKey@U?$Vec3_tpl@M@@@spline@@HUStandardAlloc@NAlloc@@@NArray@@@@QEAAXXZ 0000000031586540 f i FaceAnimSequence.obj
 0001:00085620       ?clear@?$DynArray@U?$SplineKey@M@spline@@HU?$SmallDynStorage@U?$SplineKey@M@spline@@HUStandardAlloc@NAlloc@@@NArray@@@@QEAAXXZ 0000000031586620 f i FaceAnimSequence.obj
 0001:00085700       ?clear@?$DynArray@U?$SplineKey@U?$Quat_tpl@M@@@spline@@HU?$SmallDynStorage@U?$SplineKey@U?$Quat_tpl@M@@@spline@@HUStandardAlloc@NAlloc@@@NArray@@@@QEAAXXZ 0000000031586700 f i FaceAnimSequence.obj
 0001:000857e0       ?_M_fill_insert@?$vector@_NV?$allocator@_N@stlpmtx_std@@@stlpmtx_std@@QEAAXU?$_Bit_iter@U_Bit_reference@priv@stlpmtx_std@@PEAU123@@priv@2@_K_N@Z 00000000315867e0 f i FaceAnimSequence.obj
 0001:00085cc0       ?append_raw@?$DynArray@U?$TCBSplineKey@U?$Vec3_tpl@M@@@spline@@HU?$SmallDynStorage@U?$TCBSplineKey@U?$Vec3_tpl@M@@@spline@@HUStandardAlloc@NAlloc@@@NArray@@@@QEAA?AU?$Array@U?$TCBSplineKey@U?$Vec3_tpl@M@@@spline@@HU?$ArrayStorage@U?$TCBSplineKey@U?$Vec3_tpl@M@@@spline@@H@NArray@@@@H@Z 0000000031586cc0 f i FaceAnimSequence.obj
 0001:00085d80       ?_M_erase@?$_Impl_vector@V?$_smart_ptr@VCFacialAnimChannel@@@@V?$allocator@V?$_smart_ptr@VCFacialAnimChannel@@@@@stlpmtx_std@@@priv@stlpmtx_std@@AEAAPEAV?$_smart_ptr@VCFacialAnimChannel@@@@PEAV4@0AEBU__false_type@3@@Z 0000000031586d80 f i FaceAnimSequence.obj
 0001:00085d80       ?_M_erase@?$_Impl_vector@V?$_smart_ptr@VCFacialEffCtrl@@@@V?$allocator@V?$_smart_ptr@VCFacialEffCtrl@@@@@stlpmtx_std@@@priv@stlpmtx_std@@AEAAPEAV?$_smart_ptr@VCFacialEffCtrl@@@@PEAV4@0AEBU__false_type@3@@Z 0000000031586d80 f i FaceEffector.obj
 0001:00085d80       ?_M_erase@?$_Impl_vector@V?$_smart_ptr@VCFacialEffector@@@@V?$allocator@V?$_smart_ptr@VCFacialEffector@@@@@stlpmtx_std@@@priv@stlpmtx_std@@AEAAPEAV?$_smart_ptr@VCFacialEffector@@@@PEAV4@0AEBU__false_type@3@@Z 0000000031586d80 f i FaceEffectorLibrary.obj
 0001:00085e70       ?reserve@?$_Impl_vector@HV?$allocator@H@stlpmtx_std@@@priv@stlpmtx_std@@QEAAX_K@Z 0000000031586e70 f i FaceAnimSequence.obj
 0001:00085f30       ??$make_pair@V?$CryStringT@D@@V?$_smart_ptr@VCFacialAnimChannel@@@@@stlpmtx_std@@YA?AU?$pair@V?$CryStringT@D@@V?$_smart_ptr@VCFacialAnimChannel@@@@@0@V?$CryStringT@D@@V?$_smart_ptr@VCFacialAnimChannel@@@@@Z 0000000031586f30 f i FaceAnimSequence.obj
 0001:00085fd0       ?reserve@?$_Impl_vector@U?$pair@PEAUIFacialAnimChannel@@H@stlpmtx_std@@V?$allocator@U?$pair@PEAUIFacialAnimChannel@@H@stlpmtx_std@@@2@@priv@stlpmtx_std@@QEAAX_K@Z 0000000031586fd0 f i FaceAnimSequence.obj
 0001:00086090       ??$AddObject@VCFacialAnimSkeletalAnimationEntry@@V?$allocator@VCFacialAnimSkeletalAnimationEntry@@@stlpmtx_std@@@ICrySizer@@QEAAXAEBV?$vector@VCFacialAnimSkeletalAnimationEntry@@V?$allocator@VCFacialAnimSkeletalAnimationEntry@@@stlpmtx_std@@@stlpmtx_std@@@Z 0000000031587090 f i FaceAnimSequence.obj
 0001:00086180       ??$AddObject@UChannelInfo@CFacialAnimSequenceInstance@@V?$allocator@UChannelInfo@CFacialAnimSequenceInstance@@@stlpmtx_std@@@ICrySizer@@QEAAXAEBV?$vector@UChannelInfo@CFacialAnimSequenceInstance@@V?$allocator@UChannelInfo@CFacialAnimSequenceInstance@@@stlpmtx_std@@@stlpmtx_std@@@Z 0000000031587180 f i FaceAnimSequence.obj
 0001:00086250       ?_M_fill_insert_aux@?$_Impl_vector@UChannelInfo@CFacialAnimSequenceInstance@@V?$allocator@UChannelInfo@CFacialAnimSequenceInstance@@@stlpmtx_std@@@priv@stlpmtx_std@@AEAAXPEAUChannelInfo@CFacialAnimSequenceInstance@@_KAEBU45@AEBU__false_type@3@@Z 0000000031587250 f i FaceAnimSequence.obj
 0001:00086400       ??$__copy_backward_ptrs@PEAVCFacialAnimSkeletalAnimationEntry@@PEAV1@@priv@stlpmtx_std@@YAPEAVCFacialAnimSkeletalAnimationEntry@@PEAV2@00AEBU__false_type@1@@Z 0000000031587400 f i FaceAnimSequence.obj
 0001:000864a0       ??$fill@PEAVCFacialAnimSkeletalAnimationEntry@@V1@@stlpmtx_std@@YAXPEAVCFacialAnimSkeletalAnimationEntry@@0AEBV1@@Z 00000000315874a0 f i FaceAnimSequence.obj
 0001:00086520       ??$__copy_backward_ptrs@PEAVCFacialAnimSoundEntry@@PEAV1@@priv@stlpmtx_std@@YAPEAVCFacialAnimSoundEntry@@PEAV2@00AEBU__false_type@1@@Z 0000000031587520 f i FaceAnimSequence.obj
 0001:000865f0       ??$fill@PEAVCFacialAnimSoundEntry@@V1@@stlpmtx_std@@YAXPEAVCFacialAnimSoundEntry@@0AEBV1@@Z 00000000315875f0 f i FaceAnimSequence.obj
 0001:000866a0       ??$__insertion_sort@PEAVEffectorChannelPair@@V1@U?$less@VEffectorChannelPair@@@stlpmtx_std@@@priv@stlpmtx_std@@YAXPEAVEffectorChannelPair@@00U?$less@VEffectorChannelPair@@@1@@Z 00000000315876a0 f i FaceAnimSequence.obj
 0001:00086770       ??$__insertion_sort@PEAVCFaceIdentifierHandle@@V1@USFaceIdentifierHandleLess@CFacialSentence@@@priv@stlpmtx_std@@YAXPEAVCFaceIdentifierHandle@@00USFaceIdentifierHandleLess@CFacialSentence@@@Z 0000000031587770 f i FaceAnimSequence.obj
 0001:00086850       ??$__insertion_sort@PEAU?$pair@PEAUIFacialAnimChannel@@H@stlpmtx_std@@U12@VFirstLess@?$VectorMap@PEAUIFacialAnimChannel@@HU?$less@PEAUIFacialAnimChannel@@@stlpmtx_std@@V?$allocator@U?$pair@PEAUIFacialAnimChannel@@H@stlpmtx_std@@@3@@@@priv@stlpmtx_std@@YAXPEAU?$pair@PEAUIFacialAnimChannel@@H@1@00VFirstLess@?$VectorMap@PEAUIFacialAnimChannel@@HU?$less@PEAUIFacialAnimChannel@@@stlpmtx_std@@V?$allocator@U?$pair@PEAUIFacialAnimChannel@@H@stlpmtx_std@@@3@@@@Z 0000000031587850 f i FaceAnimSequence.obj
 0001:00086920       ?swap@@YAXAEAUData@CFacialAnimSequence@@0@Z 0000000031587920 f i FaceAnimSequence.obj
 0001:00086b00       ??_ECFacialAnimChannel@@UEAAPEAXI@Z 0000000031587b00 f i FaceAnimSequence.obj
 0001:00086b00       ??_GCFacialAnimChannel@@UEAAPEAXI@Z 0000000031587b00 f i FaceAnimSequence.obj
 0001:00086b30       ?DeleteInterpolator@CFacialAnimChannel@@UEAAXH@Z 0000000031587b30 f   FaceAnimSequence.obj
 0001:00086ba0       ?GetMemoryUsage@CFacialAnimSequenceInstance@@QEBAXPEAVICrySizer@@@Z 0000000031587ba0 f   FaceAnimSequence.obj
 0001:00086c20       ?grow@?$DynArray@U?$TCBSplineKey@U?$Vec3_tpl@M@@@spline@@HU?$SmallDynStorage@U?$TCBSplineKey@U?$Vec3_tpl@M@@@spline@@HUStandardAlloc@NAlloc@@@NArray@@@@QEAAPEAU?$TCBSplineKey@U?$Vec3_tpl@M@@@spline@@H@Z 0000000031587c20 f i FaceAnimSequence.obj
 0001:00086cb0       ?grow@?$DynArray@U?$SplineKey@U?$Quat_tpl@M@@@spline@@HU?$SmallDynStorage@U?$SplineKey@U?$Quat_tpl@M@@@spline@@HUStandardAlloc@NAlloc@@@NArray@@@@QEAAPEAU?$SplineKey@U?$Quat_tpl@M@@@spline@@H@Z 0000000031587cb0 f i FaceAnimSequence.obj
 0001:00086d20       ??$__copy_ptrs@PEAVCFacialAnimSoundEntry@@PEAV1@@priv@stlpmtx_std@@YAPEAVCFacialAnimSoundEntry@@PEAV2@00AEBU__false_type@1@@Z 0000000031587d20 f i FaceAnimSequence.obj
 0001:00086df0       ?_M_clear_after_move@?$_Impl_vector@V?$_smart_ptr@VCFacialEffCtrl@@@@V?$allocator@V?$_smart_ptr@VCFacialEffCtrl@@@@@stlpmtx_std@@@priv@stlpmtx_std@@AEAAXXZ 0000000031587df0 f i FaceEffector.obj
 0001:00086df0       ?_M_clear_after_move@?$_Impl_vector@V?$_smart_ptr@VCFacialAnimChannel@@@@V?$allocator@V?$_smart_ptr@VCFacialAnimChannel@@@@@stlpmtx_std@@@priv@stlpmtx_std@@AEAAXXZ 0000000031587df0 f i FaceAnimSequence.obj
 0001:00086df0       ?_M_clear_after_move@?$_Impl_vector@V?$_smart_ptr@VCFacialEffector@@@@V?$allocator@V?$_smart_ptr@VCFacialEffector@@@@@stlpmtx_std@@@priv@stlpmtx_std@@AEAAXXZ 0000000031587df0 f i FaceEffectorLibrary.obj
 0001:00086df0       ?_M_clear@?$_Impl_vector@V?$_smart_ptr@VCFacialEffector@@@@V?$allocator@V?$_smart_ptr@VCFacialEffector@@@@@stlpmtx_std@@@priv@stlpmtx_std@@AEAAXXZ 0000000031587df0 f i FaceEffectorLibrary.obj
 0001:00086e60       ?_M_fill_insert_aux@?$_Impl_vector@V?$CryStringT@D@@V?$allocator@V?$CryStringT@D@@@stlpmtx_std@@@priv@stlpmtx_std@@AEAAXPEAV?$CryStringT@D@@_KAEBV4@AEBU__false_type@3@@Z 0000000031587e60 f i FaceAnimSequence.obj
 0001:00087090       ??$__final_insertion_sort@PEAVEffectorChannelPair@@U?$less@VEffectorChannelPair@@@stlpmtx_std@@@priv@stlpmtx_std@@YAXPEAVEffectorChannelPair@@0U?$less@VEffectorChannelPair@@@1@@Z 0000000031588090 f i FaceAnimSequence.obj
 0001:00087130       ?_M_clear_after_move@?$_Impl_vector@UChannelInfo@CFacialAnimSequenceInstance@@V?$allocator@UChannelInfo@CFacialAnimSequenceInstance@@@stlpmtx_std@@@priv@stlpmtx_std@@AEAAXXZ 0000000031588130 f i FaceAnimSequence.obj
 0001:000871a0       ??$__final_insertion_sort@PEAVCFaceIdentifierHandle@@USFaceIdentifierHandleLess@CFacialSentence@@@priv@stlpmtx_std@@YAXPEAVCFaceIdentifierHandle@@0USFaceIdentifierHandleLess@CFacialSentence@@@Z 00000000315881a0 f i FaceAnimSequence.obj
 0001:00087240       ??$__insertion_sort@PEAU?$SplineKey@M@spline@@U12@U?$less@U?$SplineKey@M@spline@@@stlpmtx_std@@@priv@stlpmtx_std@@YAXPEAU?$SplineKey@M@spline@@00U?$less@U?$SplineKey@M@spline@@@1@@Z 0000000031588240 f i FaceAnimSequence.obj
 0001:00087360       ??$sort_heap@PEAVEffectorChannelPair@@U?$less@VEffectorChannelPair@@@stlpmtx_std@@@stlpmtx_std@@YAXPEAVEffectorChannelPair@@0U?$less@VEffectorChannelPair@@@0@@Z 0000000031588360 f i FaceAnimSequence.obj
 0001:000873f0       ??$sort_heap@PEAU?$SplineKey@M@spline@@U?$less@U?$SplineKey@M@spline@@@stlpmtx_std@@@stlpmtx_std@@YAXPEAU?$SplineKey@M@spline@@0U?$less@U?$SplineKey@M@spline@@@0@@Z 00000000315883f0 f i FaceAnimSequence.obj
 0001:000874e0       ??$sort_heap@PEAVCFaceIdentifierHandle@@USFaceIdentifierHandleLess@CFacialSentence@@@stlpmtx_std@@YAXPEAVCFaceIdentifierHandle@@0USFaceIdentifierHandleLess@CFacialSentence@@@Z 00000000315884e0 f i FaceAnimSequence.obj
 0001:00087570       ??$sort_heap@PEAU?$pair@PEAUIFacialAnimChannel@@H@stlpmtx_std@@VFirstLess@?$VectorMap@PEAUIFacialAnimChannel@@HU?$less@PEAUIFacialAnimChannel@@@stlpmtx_std@@V?$allocator@U?$pair@PEAUIFacialAnimChannel@@H@stlpmtx_std@@@3@@@@stlpmtx_std@@YAXPEAU?$pair@PEAUIFacialAnimChannel@@H@0@0VFirstLess@?$VectorMap@PEAUIFacialAnimChannel@@HU?$less@PEAUIFacialAnimChannel@@@stlpmtx_std@@V?$allocator@U?$pair@PEAUIFacialAnimChannel@@H@stlpmtx_std@@@3@@@@Z 0000000031588570 f i FaceAnimSequence.obj
 0001:00087610       ??0CFacialAnimChannel@@QEAA@H@Z 0000000031588610 f   FaceAnimSequence.obj
 0001:00087930       ??$AddContainer@U?$DynArray@U?$SplineKey@M@spline@@HU?$SmallDynStorage@U?$SplineKey@M@spline@@HUStandardAlloc@NAlloc@@@NArray@@@@@ICrySizer@@QEAA_NAEBU?$DynArray@U?$SplineKey@M@spline@@HU?$SmallDynStorage@U?$SplineKey@M@spline@@HUStandardAlloc@NAlloc@@@NArray@@@@@Z 0000000031588930 f i FaceAnimSequence.obj
 0001:000879d0       ?GetMemoryUsage@?$TSpline@U?$SplineKey@M@spline@@U?$TCoeffBasis@M@2@@spline@@UEBAXPEAVICrySizer@@_N@Z 00000000315889d0 f i FaceEffector.obj
 0001:000879d0       ?GetMemoryUsage@?$TSpline@U?$SplineKey@M@spline@@VHermitBasis@2@@spline@@UEBAXPEAVICrySizer@@_N@Z 00000000315889d0 f i FaceAnimSequence.obj
 0001:00087a20       ??$AddContainer@U?$DynArray@U?$SplineKey@U?$Quat_tpl@M@@@spline@@HU?$SmallDynStorage@U?$SplineKey@U?$Quat_tpl@M@@@spline@@HUStandardAlloc@NAlloc@@@NArray@@@@@ICrySizer@@QEAA_NAEBU?$DynArray@U?$SplineKey@U?$Quat_tpl@M@@@spline@@HU?$SmallDynStorage@U?$SplineKey@U?$Quat_tpl@M@@@spline@@HUStandardAlloc@NAlloc@@@NArray@@@@@Z 0000000031588a20 f i FaceAnimSequence.obj
 0001:00087ab0       ?GetMemoryUsage@?$TSpline@U?$SplineKey@U?$Quat_tpl@M@@@spline@@VHermitBasis@2@@spline@@UEBAXPEAVICrySizer@@_N@Z 0000000031588ab0 f i FaceAnimSequence.obj
 0001:00087b00       ??1?$_Impl_vector@VCFacialAnimSkeletalAnimationEntry@@V?$allocator@VCFacialAnimSkeletalAnimationEntry@@@stlpmtx_std@@@priv@stlpmtx_std@@QEAA@XZ 0000000031588b00 f i FaceAnimSequence.obj
 0001:00087b70       ??1?$_Impl_vector@V?$_smart_ptr@VCFacialAnimChannel@@@@V?$allocator@V?$_smart_ptr@VCFacialAnimChannel@@@@@stlpmtx_std@@@priv@stlpmtx_std@@QEAA@XZ 0000000031588b70 f i FaceAnimSequence.obj
 0001:00087b70       ??1?$_Impl_vector@V?$_smart_ptr@VCFacialEffector@@@@V?$allocator@V?$_smart_ptr@VCFacialEffector@@@@@stlpmtx_std@@@priv@stlpmtx_std@@QEAA@XZ 0000000031588b70 f i FaceEffectorLibrary.obj
 0001:00087b70       ??1?$_Impl_vector@V?$_smart_ptr@VCFacialEffCtrl@@@@V?$allocator@V?$_smart_ptr@VCFacialEffCtrl@@@@@stlpmtx_std@@@priv@stlpmtx_std@@QEAA@XZ 0000000031588b70 f i FaceEffector.obj
 0001:00087bf0       ??1?$_Impl_vector@VCFacialAnimSoundEntry@@V?$allocator@VCFacialAnimSoundEntry@@@stlpmtx_std@@@priv@stlpmtx_std@@QEAA@XZ 0000000031588bf0 f i FaceAnimSequence.obj
 0001:00087c60       ?resize@?$vector@_NV?$allocator@_N@stlpmtx_std@@@stlpmtx_std@@QEAAX_K_N@Z 0000000031588c60 f i FaceAnimSequence.obj
 0001:00087d50       ??_E?$TSpline@U?$SplineKey@U?$Quat_tpl@M@@@spline@@VHermitBasis@2@@spline@@UEAAPEAXI@Z 0000000031588d50 f i FaceAnimSequence.obj
 0001:00087d50       ??_G?$TSpline@U?$SplineKey@U?$Quat_tpl@M@@@spline@@VHermitBasis@2@@spline@@UEAAPEAXI@Z 0000000031588d50 f i FaceAnimSequence.obj
 0001:00087dc0       ?_M_erase@?$_Impl_vector@VCFacialAnimSkeletalAnimationEntry@@V?$allocator@VCFacialAnimSkeletalAnimationEntry@@@stlpmtx_std@@@priv@stlpmtx_std@@AEAAPEAVCFacialAnimSkeletalAnimationEntry@@PEAV4@AEBU__false_type@3@@Z 0000000031588dc0 f i FaceAnimSequence.obj
 0001:00087e80       ?_M_erase@?$_Impl_vector@VCFacialAnimSkeletalAnimationEntry@@V?$allocator@VCFacialAnimSkeletalAnimationEntry@@@stlpmtx_std@@@priv@stlpmtx_std@@AEAAPEAVCFacialAnimSkeletalAnimationEntry@@PEAV4@0AEBU__false_type@3@@Z 0000000031588e80 f i FaceAnimSequence.obj
 0001:00087f70       ??$AddObject@VCFacialAnimSoundEntry@@V?$allocator@VCFacialAnimSoundEntry@@@stlpmtx_std@@@ICrySizer@@QEAAXAEBV?$vector@VCFacialAnimSoundEntry@@V?$allocator@VCFacialAnimSoundEntry@@@stlpmtx_std@@@stlpmtx_std@@@Z 0000000031588f70 f i FaceAnimSequence.obj
 0001:00088010       ?_M_insert_overflow_aux@?$_Impl_vector@UChannelInfo@CFacialAnimSequenceInstance@@V?$allocator@UChannelInfo@CFacialAnimSequenceInstance@@@stlpmtx_std@@@priv@stlpmtx_std@@AEAAXPEAUChannelInfo@CFacialAnimSequenceInstance@@AEBU45@AEBU__false_type@3@_K_N@Z 0000000031589010 f i FaceAnimSequence.obj
 0001:00088150       ??$__final_insertion_sort@PEAU?$SplineKey@M@spline@@U?$less@U?$SplineKey@M@spline@@@stlpmtx_std@@@priv@stlpmtx_std@@YAXPEAU?$SplineKey@M@spline@@0U?$less@U?$SplineKey@M@spline@@@1@@Z 0000000031589150 f i FaceAnimSequence.obj
 0001:000881d0       ??$__uninitialized_fill_n@PEAVCFacialAnimSkeletalAnimationEntry@@_KV1@@priv@stlpmtx_std@@YAPEAVCFacialAnimSkeletalAnimationEntry@@PEAV2@_KAEBV2@@Z 00000000315891d0 f i FaceAnimSequence.obj
 0001:00088250       ??$__uninitialized_fill_n@PEAVCFacialAnimSoundEntry@@_KV1@@priv@stlpmtx_std@@YAPEAVCFacialAnimSoundEntry@@PEAV2@_KAEBV2@@Z 0000000031589250 f i FaceAnimSequence.obj
 0001:000882d0       ??$__partial_sort@PEAVEffectorChannelPair@@V1@U?$less@VEffectorChannelPair@@@stlpmtx_std@@@priv@stlpmtx_std@@YAXPEAVEffectorChannelPair@@000U?$less@VEffectorChannelPair@@@1@@Z 00000000315892d0 f i FaceAnimSequence.obj
 0001:00088390       ??$__partial_sort@PEAU?$SplineKey@M@spline@@U12@U?$less@U?$SplineKey@M@spline@@@stlpmtx_std@@@priv@stlpmtx_std@@YAXPEAU?$SplineKey@M@spline@@000U?$less@U?$SplineKey@M@spline@@@1@@Z 0000000031589390 f i FaceAnimSequence.obj
 0001:00088480       ??$__partial_sort@PEAVCFaceIdentifierHandle@@V1@USFaceIdentifierHandleLess@CFacialSentence@@@priv@stlpmtx_std@@YAXPEAVCFaceIdentifierHandle@@000USFaceIdentifierHandleLess@CFacialSentence@@@Z 0000000031589480 f i FaceAnimSequence.obj
 0001:00088540       ??$__partial_sort@PEAU?$pair@PEAUIFacialAnimChannel@@H@stlpmtx_std@@U12@VFirstLess@?$VectorMap@PEAUIFacialAnimChannel@@HU?$less@PEAUIFacialAnimChannel@@@stlpmtx_std@@V?$allocator@U?$pair@PEAUIFacialAnimChannel@@H@stlpmtx_std@@@3@@@@priv@stlpmtx_std@@YAXPEAU?$pair@PEAUIFacialAnimChannel@@H@1@000VFirstLess@?$VectorMap@PEAUIFacialAnimChannel@@HU?$less@PEAUIFacialAnimChannel@@@stlpmtx_std@@V?$allocator@U?$pair@PEAUIFacialAnimChannel@@H@stlpmtx_std@@@3@@@@Z 0000000031589540 f i FaceAnimSequence.obj
 0001:00088600       ??$AddContainer@U?$DynArray@U?$TCBSplineKey@U?$Vec3_tpl@M@@@spline@@HU?$SmallDynStorage@U?$TCBSplineKey@U?$Vec3_tpl@M@@@spline@@HUStandardAlloc@NAlloc@@@NArray@@@@@ICrySizer@@QEAA_NAEBU?$DynArray@U?$TCBSplineKey@U?$Vec3_tpl@M@@@spline@@HU?$SmallDynStorage@U?$TCBSplineKey@U?$Vec3_tpl@M@@@spline@@HUStandardAlloc@NAlloc@@@NArray@@@@@Z 0000000031589600 f i FaceAnimSequence.obj
 0001:00088690       ?GetMemoryUsage@?$TSpline@U?$TCBSplineKey@U?$Vec3_tpl@M@@@spline@@VHermitBasis@2@@spline@@UEBAXPEAVICrySizer@@_N@Z 0000000031589690 f i FaceAnimSequence.obj
 0001:000886e0       ?SerializeSpline@CFacialAnimChannelInterpolator@@UEAAXAEAVXmlNodeRef@@_N@Z 00000000315896e0 f   FaceAnimSequence.obj
 0001:00088d30       ?RemoveChannel@CFacialAnimSequence@@UEAAXPEAUIFacialAnimChannel@@@Z 0000000031589d30 f   FaceAnimSequence.obj
 0001:00088f50       ?GetMemoryUsage@CFacialAnimSequence@@UEBAXPEAVICrySizer@@@Z 0000000031589f50 f   FaceAnimSequence.obj
 0001:00089040       ??0?$TSpline@U?$SplineKey@M@spline@@U?$TCoeffBasis@M@2@@spline@@QEAA@XZ 000000003158a040 f i FaceEffector.obj
 0001:00089040       ??0?$TSpline@U?$SplineKey@M@spline@@VHermitBasis@2@@spline@@QEAA@XZ 000000003158a040 f i FaceAnimSequence.obj
 0001:000890c0       ??0?$TSpline@U?$SplineKey@U?$Quat_tpl@M@@@spline@@VHermitBasis@2@@spline@@QEAA@XZ 000000003158a0c0 f i FaceAnimSequence.obj
 0001:00089140       ?erase@?$_Impl_vector@UChannelInfo@CFacialAnimSequenceInstance@@V?$allocator@UChannelInfo@CFacialAnimSequenceInstance@@@stlpmtx_std@@@priv@stlpmtx_std@@QEAAPEAUChannelInfo@CFacialAnimSequenceInstance@@PEAU45@0@Z 000000003158a140 f i FaceAnimSequence.obj
 0001:000891f0       ?erase@?$_Impl_vector@VCFacialAnimSoundEntry@@V?$allocator@VCFacialAnimSoundEntry@@@stlpmtx_std@@@priv@stlpmtx_std@@QEAAPEAVCFacialAnimSoundEntry@@PEAV4@0@Z 000000003158a1f0 f i FaceAnimSequence.obj
 0001:00089290       ?_M_erase@?$_Impl_vector@V?$CryStringT@D@@V?$allocator@V?$CryStringT@D@@@stlpmtx_std@@@priv@stlpmtx_std@@AEAAPEAV?$CryStringT@D@@PEAV4@0AEBU__false_type@3@@Z 000000003158a290 f i FaceAnimSequence.obj
 0001:00089350       ?_M_fill_insert_aux@?$_Impl_vector@VCFacialAnimSkeletalAnimationEntry@@V?$allocator@VCFacialAnimSkeletalAnimationEntry@@@stlpmtx_std@@@priv@stlpmtx_std@@AEAAXPEAVCFacialAnimSkeletalAnimationEntry@@_KAEBV4@AEBU__false_type@3@@Z 000000003158a350 f i FaceAnimSequence.obj
 0001:000895f0       ?_M_fill_insert_aux@?$_Impl_vector@VCFacialAnimSoundEntry@@V?$allocator@VCFacialAnimSoundEntry@@@stlpmtx_std@@@priv@stlpmtx_std@@AEAAXPEAVCFacialAnimSoundEntry@@_KAEBV4@AEBU__false_type@3@@Z 000000003158a5f0 f i FaceAnimSequence.obj
 0001:000898b0       ??1?$_Impl_vector@V?$CryStringT@D@@V?$allocator@V?$CryStringT@D@@@stlpmtx_std@@@priv@stlpmtx_std@@QEAA@XZ 000000003158a8b0 f i FaceAnimSequence.obj
 0001:00089940       ??0?$TSpline@U?$TCBSplineKey@U?$Vec3_tpl@M@@@spline@@VHermitBasis@2@@spline@@QEAA@XZ 000000003158a940 f i FaceAnimSequence.obj
 0001:000899c0       ?comp_deriv@?$HermitSplineEx@U?$Quat_tpl@M@@U?$SplineKey@U?$Quat_tpl@M@@@spline@@@spline@@UEAAXXZ 000000003158a9c0 f i FaceAnimSequence.obj
 0001:00089e40       ?interp_keys@?$HermitSplineEx@U?$Quat_tpl@M@@U?$SplineKey@U?$Quat_tpl@M@@@spline@@@spline@@MEAAXHHMAEAU?$Quat_tpl@M@@@Z 000000003158ae40 f i FaceAnimSequence.obj
 0001:0008a070       ?comp_deriv@?$HermitSplineEx@MU?$SplineKey@M@spline@@@spline@@UEAAXXZ 000000003158b070 f i FaceAnimSequence.obj
 0001:0008a1c0       ?interp_keys@?$HermitSplineEx@MU?$SplineKey@M@spline@@@spline@@MEAAXHHMAEAM@Z 000000003158b1c0 f i FaceAnimSequence.obj
 0001:0008a2a0       ?SerializeSpline@CFacialCameraPathPositionInterpolator@@UEAAXAEAVXmlNodeRef@@_N@Z 000000003158b2a0 f   FaceAnimSequence.obj
 0001:0008a8f0       ?SerializeSpline@CFacialCameraPathOrientationInterpolator@@UEAAXAEAVXmlNodeRef@@_N@Z 000000003158b8f0 f   FaceAnimSequence.obj
 0001:0008af70       ?_M_insert_overflow_aux@?$_Impl_vector@VCFacialAnimSkeletalAnimationEntry@@V?$allocator@VCFacialAnimSkeletalAnimationEntry@@@stlpmtx_std@@@priv@stlpmtx_std@@AEAAXPEAVCFacialAnimSkeletalAnimationEntry@@AEBV4@AEBU__false_type@3@_K_N@Z 000000003158bf70 f i FaceAnimSequence.obj
 0001:0008b1c0       ?_M_insert_overflow_aux@?$_Impl_vector@VCFacialAnimSoundEntry@@V?$allocator@VCFacialAnimSoundEntry@@@stlpmtx_std@@@priv@stlpmtx_std@@AEAAXPEAVCFacialAnimSoundEntry@@AEBV4@AEBU__false_type@3@_K_N@Z 000000003158c1c0 f i FaceAnimSequence.obj
 0001:0008b440       ??$__introsort_loop@PEAVEffectorChannelPair@@V1@_JU?$less@VEffectorChannelPair@@@stlpmtx_std@@@priv@stlpmtx_std@@YAXPEAVEffectorChannelPair@@00_JU?$less@VEffectorChannelPair@@@1@@Z 000000003158c440 f i FaceAnimSequence.obj
 0001:0008b590       ??$__introsort_loop@PEAU?$SplineKey@M@spline@@U12@_JU?$less@U?$SplineKey@M@spline@@@stlpmtx_std@@@priv@stlpmtx_std@@YAXPEAU?$SplineKey@M@spline@@00_JU?$less@U?$SplineKey@M@spline@@@1@@Z 000000003158c590 f i FaceAnimSequence.obj
 0001:0008b750       ??$__introsort_loop@PEAVCFaceIdentifierHandle@@V1@_JUSFaceIdentifierHandleLess@CFacialSentence@@@priv@stlpmtx_std@@YAXPEAVCFaceIdentifierHandle@@00_JUSFaceIdentifierHandleLess@CFacialSentence@@@Z 000000003158c750 f i FaceAnimSequence.obj
 0001:0008b8b0       ??$__introsort_loop@PEAU?$pair@PEAUIFacialAnimChannel@@H@stlpmtx_std@@U12@_JVFirstLess@?$VectorMap@PEAUIFacialAnimChannel@@HU?$less@PEAUIFacialAnimChannel@@@stlpmtx_std@@V?$allocator@U?$pair@PEAUIFacialAnimChannel@@H@stlpmtx_std@@@3@@@@priv@stlpmtx_std@@YAXPEAU?$pair@PEAUIFacialAnimChannel@@H@1@00_JVFirstLess@?$VectorMap@PEAUIFacialAnimChannel@@HU?$less@PEAUIFacialAnimChannel@@@stlpmtx_std@@V?$allocator@U?$pair@PEAUIFacialAnimChannel@@H@stlpmtx_std@@@3@@@@Z 000000003158c8b0 f i FaceAnimSequence.obj
 0001:0008ba00       ?compMiddleDeriv@?$TCBSpline@U?$Vec3_tpl@M@@U?$TCBSplineKey@U?$Vec3_tpl@M@@@spline@@@spline@@AEAAXH@Z 000000003158ca00 f i FaceAnimSequence.obj
 0001:0008bdb0       ?compFirstDeriv@?$TCBSpline@U?$Vec3_tpl@M@@U?$TCBSplineKey@U?$Vec3_tpl@M@@@spline@@@spline@@AEAAXXZ 000000003158cdb0 f i FaceAnimSequence.obj
 0001:0008be70       ?compLastDeriv@?$TCBSpline@U?$Vec3_tpl@M@@U?$TCBSplineKey@U?$Vec3_tpl@M@@@spline@@@spline@@AEAAXXZ 000000003158ce70 f i FaceAnimSequence.obj
 0001:0008bf60       ?comp2KeyDeriv@?$TCBSpline@U?$Vec3_tpl@M@@U?$TCBSplineKey@U?$Vec3_tpl@M@@@spline@@@spline@@AEAAXXZ 000000003158cf60 f i FaceAnimSequence.obj
 0001:0008c070       ?comp_deriv@?$TCBSpline@U?$Vec3_tpl@M@@U?$TCBSplineKey@U?$Vec3_tpl@M@@@spline@@@spline@@UEAAXXZ 000000003158d070 f i FaceAnimSequence.obj
 0001:0008c140       ?interp_keys@?$TCBSpline@U?$Vec3_tpl@M@@U?$TCBSplineKey@U?$Vec3_tpl@M@@@spline@@@spline@@MEAAXHHMAEAU?$Vec3_tpl@M@@@Z 000000003158d140 f i FaceAnimSequence.obj
 0001:0008c2f0       ??_E?$TSpline@U?$TCBSplineKey@U?$Vec3_tpl@M@@@spline@@VHermitBasis@2@@spline@@UEAAPEAXI@Z 000000003158d2f0 f i FaceAnimSequence.obj
 0001:0008c2f0       ??_E?$TCBSpline@U?$Vec3_tpl@M@@U?$TCBSplineKey@U?$Vec3_tpl@M@@@spline@@@spline@@UEAAPEAXI@Z 000000003158d2f0 f i FaceAnimSequence.obj
 0001:0008c2f0       ??_G?$TSpline@U?$TCBSplineKey@U?$Vec3_tpl@M@@@spline@@VHermitBasis@2@@spline@@UEAAPEAXI@Z 000000003158d2f0 f i FaceAnimSequence.obj
 0001:0008c2f0       ??_G?$TCBSpline@U?$Vec3_tpl@M@@U?$TCBSplineKey@U?$Vec3_tpl@M@@@spline@@@spline@@UEAAPEAXI@Z 000000003158d2f0 f i FaceAnimSequence.obj
 0001:0008c360       ??$__push_heap@PEAU?$TCBSplineKey@U?$Vec3_tpl@M@@@spline@@_JU12@U?$less@U?$TCBSplineKey@U?$Vec3_tpl@M@@@spline@@@stlpmtx_std@@@stlpmtx_std@@YAXPEAU?$TCBSplineKey@U?$Vec3_tpl@M@@@spline@@_J1U12@U?$less@U?$TCBSplineKey@U?$Vec3_tpl@M@@@spline@@@0@@Z 000000003158d360 f i FaceAnimSequence.obj
 0001:0008c460       ??$__copy_backward@PEAU?$TCBSplineKey@U?$Vec3_tpl@M@@@spline@@PEAU12@_J@priv@stlpmtx_std@@YAPEAU?$TCBSplineKey@U?$Vec3_tpl@M@@@spline@@PEAU23@00AEBUrandom_access_iterator_tag@1@PEA_J@Z 000000003158d460 f i FaceAnimSequence.obj
 0001:0008c640       ?GetKeyTime@?$CBaseSplineInterpolator@U?$Vec3_tpl@M@@V?$TCBSpline@U?$Vec3_tpl@M@@U?$TCBSplineKey@U?$Vec3_tpl@M@@@spline@@@spline@@@spline@@UEAAMH@Z 000000003158d640 f i FaceAnimSequence.obj
 0001:0008c670       ?GetKeyValue@?$CBaseSplineInterpolator@U?$Vec3_tpl@M@@V?$TCBSpline@U?$Vec3_tpl@M@@U?$TCBSplineKey@U?$Vec3_tpl@M@@@spline@@@spline@@@spline@@UEAA_NHAEAY03M@Z 000000003158d670 f i FaceAnimSequence.obj
 0001:0008c6b0       ?SetKeyValue@?$CBaseSplineInterpolator@U?$Vec3_tpl@M@@V?$TCBSpline@U?$Vec3_tpl@M@@U?$TCBSplineKey@U?$Vec3_tpl@M@@@spline@@@spline@@@spline@@UEAAXHQEAM@Z 000000003158d6b0 f i FaceAnimSequence.obj
 0001:0008c700       ?SetKeyTime@?$CBaseSplineInterpolator@U?$Vec3_tpl@M@@V?$TCBSpline@U?$Vec3_tpl@M@@U?$TCBSplineKey@U?$Vec3_tpl@M@@@spline@@@spline@@@spline@@UEAAXHM@Z 000000003158d700 f i FaceAnimSequence.obj
 0001:0008c730       ?SetKeyInTangent@?$CBaseSplineInterpolator@U?$Vec3_tpl@M@@V?$TCBSpline@U?$Vec3_tpl@M@@U?$TCBSplineKey@U?$Vec3_tpl@M@@@spline@@@spline@@@spline@@UEAAXHQEAM@Z 000000003158d730 f i FaceAnimSequence.obj
 0001:0008c780       ?SetKeyOutTangent@?$CBaseSplineInterpolator@U?$Vec3_tpl@M@@V?$TCBSpline@U?$Vec3_tpl@M@@U?$TCBSplineKey@U?$Vec3_tpl@M@@@spline@@@spline@@@spline@@UEAAXHQEAM@Z 000000003158d780 f i FaceAnimSequence.obj
 0001:0008c7d0       ?SetKeyTangents@?$CBaseSplineInterpolator@U?$Vec3_tpl@M@@V?$TCBSpline@U?$Vec3_tpl@M@@U?$TCBSplineKey@U?$Vec3_tpl@M@@@spline@@@spline@@@spline@@UEAAXHQEAM0@Z 000000003158d7d0 f i FaceAnimSequence.obj
 0001:0008c830       ?GetKeyTangents@?$CBaseSplineInterpolator@U?$Vec3_tpl@M@@V?$TCBSpline@U?$Vec3_tpl@M@@U?$TCBSplineKey@U?$Vec3_tpl@M@@@spline@@@spline@@@spline@@UEAA_NHAEAY03M0@Z 000000003158d830 f i FaceAnimSequence.obj
 0001:0008c890       ?SetKeyFlags@?$CBaseSplineInterpolator@U?$Vec3_tpl@M@@V?$TCBSpline@U?$Vec3_tpl@M@@U?$TCBSplineKey@U?$Vec3_tpl@M@@@spline@@@spline@@@spline@@UEAAXHH@Z 000000003158d890 f i FaceAnimSequence.obj
 0001:0008c8c0       ?GetKeyFlags@?$CBaseSplineInterpolator@U?$Vec3_tpl@M@@V?$TCBSpline@U?$Vec3_tpl@M@@U?$TCBSplineKey@U?$Vec3_tpl@M@@@spline@@@spline@@@spline@@UEAAHH@Z 000000003158d8c0 f i FaceAnimSequence.obj
 0001:0008c8f0       ?seek_key@?$TSpline@U?$TCBSplineKey@U?$Vec3_tpl@M@@@spline@@VHermitBasis@2@@spline@@IEAAHM@Z 000000003158d8f0 f i FaceAnimSequence.obj
 0001:0008c970       ??$__unguarded_insertion_sort_aux@PEAU?$TCBSplineKey@U?$Vec3_tpl@M@@@spline@@U12@U?$less@U?$TCBSplineKey@U?$Vec3_tpl@M@@@spline@@@stlpmtx_std@@@priv@stlpmtx_std@@YAXPEAU?$TCBSplineKey@U?$Vec3_tpl@M@@@spline@@00U?$less@U?$TCBSplineKey@U?$Vec3_tpl@M@@@spline@@@1@@Z 000000003158d970 f i FaceAnimSequence.obj
 0001:0008cac0       ??$__adjust_heap@PEAU?$TCBSplineKey@U?$Vec3_tpl@M@@@spline@@_JU12@U?$less@U?$TCBSplineKey@U?$Vec3_tpl@M@@@spline@@@stlpmtx_std@@@stlpmtx_std@@YAXPEAU?$TCBSplineKey@U?$Vec3_tpl@M@@@spline@@_J1U12@U?$less@U?$TCBSplineKey@U?$Vec3_tpl@M@@@spline@@@0@@Z 000000003158dac0 f i FaceAnimSequence.obj
 0001:0008cc10       ?FindKeysInRange@?$CBaseSplineInterpolator@U?$Vec3_tpl@M@@V?$TCBSpline@U?$Vec3_tpl@M@@U?$TCBSplineKey@U?$Vec3_tpl@M@@@spline@@@spline@@@spline@@UEAAXMMAEAH0@Z 000000003158dc10 f i FaceAnimSequence.obj
 0001:0008cd50       ??$__make_heap@PEAU?$TCBSplineKey@U?$Vec3_tpl@M@@@spline@@U?$less@U?$TCBSplineKey@U?$Vec3_tpl@M@@@spline@@@stlpmtx_std@@U12@_J@stlpmtx_std@@YAXPEAU?$TCBSplineKey@U?$Vec3_tpl@M@@@spline@@0U?$less@U?$TCBSplineKey@U?$Vec3_tpl@M@@@spline@@@0@0PEA_J@Z 000000003158dd50 f i FaceAnimSequence.obj
 0001:0008cf50       ??$__pop_heap_aux@PEAU?$TCBSplineKey@U?$Vec3_tpl@M@@@spline@@U12@U?$less@U?$TCBSplineKey@U?$Vec3_tpl@M@@@spline@@@stlpmtx_std@@@stlpmtx_std@@YAXPEAU?$TCBSplineKey@U?$Vec3_tpl@M@@@spline@@00U?$less@U?$TCBSplineKey@U?$Vec3_tpl@M@@@spline@@@0@@Z 000000003158df50 f i FaceAnimSequence.obj
 0001:0008d030       ?erase@?$DynArray@U?$TCBSplineKey@U?$Vec3_tpl@M@@@spline@@HU?$SmallDynStorage@U?$TCBSplineKey@U?$Vec3_tpl@M@@@spline@@HUStandardAlloc@NAlloc@@@NArray@@@@QEAAPEAU?$TCBSplineKey@U?$Vec3_tpl@M@@@spline@@PEAU23@0@Z 000000003158e030 f i FaceAnimSequence.obj
 0001:0008d240       ?insert_raw@?$DynArray@U?$TCBSplineKey@U?$Vec3_tpl@M@@@spline@@HU?$SmallDynStorage@U?$TCBSplineKey@U?$Vec3_tpl@M@@@spline@@HUStandardAlloc@NAlloc@@@NArray@@@@QEAA?AU?$Array@U?$TCBSplineKey@U?$Vec3_tpl@M@@@spline@@HU?$ArrayStorage@U?$TCBSplineKey@U?$Vec3_tpl@M@@@spline@@H@NArray@@@@PEAU?$TCBSplineKey@U?$Vec3_tpl@M@@@spline@@H@Z 000000003158e240 f i FaceAnimSequence.obj
 0001:0008d360       ??4?$DynArray@U?$TCBSplineKey@U?$Vec3_tpl@M@@@spline@@HU?$SmallDynStorage@U?$TCBSplineKey@U?$Vec3_tpl@M@@@spline@@HUStandardAlloc@NAlloc@@@NArray@@@@QEAAAEAU0@U?$Array@$$CBU?$TCBSplineKey@U?$Vec3_tpl@M@@@spline@@HU?$ArrayStorage@$$CBU?$TCBSplineKey@U?$Vec3_tpl@M@@@spline@@H@NArray@@@@@Z 000000003158e360 f i FaceAnimSequence.obj
 0001:0008d4e0       ?RemoveKey@?$CBaseSplineInterpolator@U?$Vec3_tpl@M@@V?$TCBSpline@U?$Vec3_tpl@M@@U?$TCBSplineKey@U?$Vec3_tpl@M@@@spline@@@spline@@@spline@@UEAAXH@Z 000000003158e4e0 f i FaceAnimSequence.obj
 0001:0008d530       ?RemoveKeysInRange@?$CBaseSplineInterpolator@U?$Vec3_tpl@M@@V?$TCBSpline@U?$Vec3_tpl@M@@U?$TCBSplineKey@U?$Vec3_tpl@M@@@spline@@@spline@@@spline@@UEAAXMM@Z 000000003158e530 f i FaceAnimSequence.obj
 0001:0008d6a0       ??0?$DynArray@U?$TCBSplineKey@U?$Vec3_tpl@M@@@spline@@HU?$SmallDynStorage@U?$TCBSplineKey@U?$Vec3_tpl@M@@@spline@@HUStandardAlloc@NAlloc@@@NArray@@@@QEAA@AEBU0@@Z 000000003158e6a0 f i FaceAnimSequence.obj
 0001:0008d780       ??$__insertion_sort@PEAU?$TCBSplineKey@U?$Vec3_tpl@M@@@spline@@U12@U?$less@U?$TCBSplineKey@U?$Vec3_tpl@M@@@spline@@@stlpmtx_std@@@priv@stlpmtx_std@@YAXPEAU?$TCBSplineKey@U?$Vec3_tpl@M@@@spline@@00U?$less@U?$TCBSplineKey@U?$Vec3_tpl@M@@@spline@@@1@@Z 000000003158e780 f i FaceAnimSequence.obj
 0001:0008d980       ??$__partial_sort@PEAU?$TCBSplineKey@U?$Vec3_tpl@M@@@spline@@U12@U?$less@U?$TCBSplineKey@U?$Vec3_tpl@M@@@spline@@@stlpmtx_std@@@priv@stlpmtx_std@@YAXPEAU?$TCBSplineKey@U?$Vec3_tpl@M@@@spline@@000U?$less@U?$TCBSplineKey@U?$Vec3_tpl@M@@@spline@@@1@@Z 000000003158e980 f i FaceAnimSequence.obj
 0001:0008db00       ??4?$TSpline@U?$TCBSplineKey@U?$Vec3_tpl@M@@@spline@@VHermitBasis@2@@spline@@QEAAAEAV01@AEBV01@@Z 000000003158eb00 f i FaceAnimSequence.obj
 0001:0008db80       ??$__final_insertion_sort@PEAU?$TCBSplineKey@U?$Vec3_tpl@M@@@spline@@U?$less@U?$TCBSplineKey@U?$Vec3_tpl@M@@@spline@@@stlpmtx_std@@@priv@stlpmtx_std@@YAXPEAU?$TCBSplineKey@U?$Vec3_tpl@M@@@spline@@0U?$less@U?$TCBSplineKey@U?$Vec3_tpl@M@@@spline@@@1@@Z 000000003158eb80 f i FaceAnimSequence.obj
 0001:0008dbf0       ?InsertKey@?$CBaseSplineInterpolator@U?$Vec3_tpl@M@@V?$TCBSpline@U?$Vec3_tpl@M@@U?$TCBSplineKey@U?$Vec3_tpl@M@@@spline@@@spline@@@spline@@UEAAHMQEAM@Z 000000003158ebf0 f i FaceAnimSequence.obj
 0001:0008de50       ??$__introsort_loop@PEAU?$TCBSplineKey@U?$Vec3_tpl@M@@@spline@@U12@_JU?$less@U?$TCBSplineKey@U?$Vec3_tpl@M@@@spline@@@stlpmtx_std@@@priv@stlpmtx_std@@YAXPEAU?$TCBSplineKey@U?$Vec3_tpl@M@@@spline@@00_JU?$less@U?$TCBSplineKey@U?$Vec3_tpl@M@@@spline@@@1@@Z 000000003158ee50 f i FaceAnimSequence.obj
 0001:0008e090       ??$__push_heap@PEAU?$SplineKey@U?$Quat_tpl@M@@@spline@@_JU12@U?$less@U?$SplineKey@U?$Quat_tpl@M@@@spline@@@stlpmtx_std@@@stlpmtx_std@@YAXPEAU?$SplineKey@U?$Quat_tpl@M@@@spline@@_J1U12@U?$less@U?$SplineKey@U?$Quat_tpl@M@@@spline@@@0@@Z 000000003158f090 f i FaceAnimSequence.obj
 0001:0008e140       ?seek_key@?$TSpline@U?$SplineKey@U?$Quat_tpl@M@@@spline@@VHermitBasis@2@@spline@@IEAAHM@Z 000000003158f140 f i FaceAnimSequence.obj
 0001:0008e1c0       ?init@?$DynArray@U?$SplineKey@U?$Quat_tpl@M@@@spline@@HU?$SmallDynStorage@U?$SplineKey@U?$Quat_tpl@M@@@spline@@HUStandardAlloc@NAlloc@@@NArray@@@@KAPEAU?$SplineKey@U?$Quat_tpl@M@@@spline@@U?$Array@U?$SplineKey@U?$Quat_tpl@M@@@spline@@HU?$ArrayStorage@U?$SplineKey@U?$Quat_tpl@M@@@spline@@H@NArray@@@@PEBU23@@Z 000000003158f1c0 f i FaceAnimSequence.obj
 0001:0008e270       ??$__unguarded_insertion_sort_aux@PEAU?$SplineKey@U?$Quat_tpl@M@@@spline@@U12@U?$less@U?$SplineKey@U?$Quat_tpl@M@@@spline@@@stlpmtx_std@@@priv@stlpmtx_std@@YAXPEAU?$SplineKey@U?$Quat_tpl@M@@@spline@@00U?$less@U?$SplineKey@U?$Quat_tpl@M@@@spline@@@1@@Z 000000003158f270 f i FaceAnimSequence.obj
 0001:0008e3a0       ??$__adjust_heap@PEAU?$SplineKey@U?$Quat_tpl@M@@@spline@@_JU12@U?$less@U?$SplineKey@U?$Quat_tpl@M@@@spline@@@stlpmtx_std@@@stlpmtx_std@@YAXPEAU?$SplineKey@U?$Quat_tpl@M@@@spline@@_J1U12@U?$less@U?$SplineKey@U?$Quat_tpl@M@@@spline@@@0@@Z 000000003158f3a0 f i FaceAnimSequence.obj
 0001:0008e510       ?FindKeysInRange@?$CBaseSplineInterpolator@U?$Quat_tpl@M@@V?$HermitSplineEx@U?$Quat_tpl@M@@U?$SplineKey@U?$Quat_tpl@M@@@spline@@@spline@@@spline@@UEAAXMMAEAH0@Z 000000003158f510 f i FaceAnimSequence.obj
 0001:0008e650       ?GetKeyTime@?$CBaseSplineInterpolator@U?$Quat_tpl@M@@V?$HermitSplineEx@U?$Quat_tpl@M@@U?$SplineKey@U?$Quat_tpl@M@@@spline@@@spline@@@spline@@UEAAMH@Z 000000003158f650 f i FaceAnimSequence.obj
 0001:0008e680       ?GetKeyValue@?$CBaseSplineInterpolator@U?$Quat_tpl@M@@V?$HermitSplineEx@U?$Quat_tpl@M@@U?$SplineKey@U?$Quat_tpl@M@@@spline@@@spline@@@spline@@UEAA_NHAEAY03M@Z 000000003158f680 f i FaceAnimSequence.obj
 0001:0008e6d0       ?SetKeyValue@?$CBaseSplineInterpolator@U?$Quat_tpl@M@@V?$HermitSplineEx@U?$Quat_tpl@M@@U?$SplineKey@U?$Quat_tpl@M@@@spline@@@spline@@@spline@@UEAAXHQEAM@Z 000000003158f6d0 f i FaceAnimSequence.obj
 0001:0008e720       ?SetKeyTime@?$CBaseSplineInterpolator@U?$Quat_tpl@M@@V?$HermitSplineEx@U?$Quat_tpl@M@@U?$SplineKey@U?$Quat_tpl@M@@@spline@@@spline@@@spline@@UEAAXHM@Z 000000003158f720 f i FaceAnimSequence.obj
 0001:0008e750       ?SetKeyInTangent@?$CBaseSplineInterpolator@U?$Quat_tpl@M@@V?$HermitSplineEx@U?$Quat_tpl@M@@U?$SplineKey@U?$Quat_tpl@M@@@spline@@@spline@@@spline@@UEAAXHQEAM@Z 000000003158f750 f i FaceAnimSequence.obj
 0001:0008e7a0       ?SetKeyOutTangent@?$CBaseSplineInterpolator@U?$Quat_tpl@M@@V?$HermitSplineEx@U?$Quat_tpl@M@@U?$SplineKey@U?$Quat_tpl@M@@@spline@@@spline@@@spline@@UEAAXHQEAM@Z 000000003158f7a0 f i FaceAnimSequence.obj
 0001:0008e7f0       ?SetKeyTangents@?$CBaseSplineInterpolator@U?$Quat_tpl@M@@V?$HermitSplineEx@U?$Quat_tpl@M@@U?$SplineKey@U?$Quat_tpl@M@@@spline@@@spline@@@spline@@UEAAXHQEAM0@Z 000000003158f7f0 f i FaceAnimSequence.obj
 0001:0008e870       ?GetKeyTangents@?$CBaseSplineInterpolator@U?$Quat_tpl@M@@V?$HermitSplineEx@U?$Quat_tpl@M@@U?$SplineKey@U?$Quat_tpl@M@@@spline@@@spline@@@spline@@UEAA_NHAEAY03M0@Z 000000003158f870 f i FaceAnimSequence.obj
 0001:0008e8e0       ?SetKeyFlags@?$CBaseSplineInterpolator@U?$Quat_tpl@M@@V?$HermitSplineEx@U?$Quat_tpl@M@@U?$SplineKey@U?$Quat_tpl@M@@@spline@@@spline@@@spline@@UEAAXHH@Z 000000003158f8e0 f i FaceAnimSequence.obj
 0001:0008e910       ?GetKeyFlags@?$CBaseSplineInterpolator@U?$Quat_tpl@M@@V?$HermitSplineEx@U?$Quat_tpl@M@@U?$SplineKey@U?$Quat_tpl@M@@@spline@@@spline@@@spline@@UEAAHH@Z 000000003158f910 f i FaceAnimSequence.obj
 0001:0008e940       ?erase@?$DynArray@U?$SplineKey@U?$Quat_tpl@M@@@spline@@HU?$SmallDynStorage@U?$SplineKey@U?$Quat_tpl@M@@@spline@@HUStandardAlloc@NAlloc@@@NArray@@@@QEAAPEAU?$SplineKey@U?$Quat_tpl@M@@@spline@@PEAU23@0@Z 000000003158f940 f i FaceAnimSequence.obj
 0001:0008ea00       ??$__pop_heap@PEAU?$SplineKey@U?$Quat_tpl@M@@@spline@@U12@U?$less@U?$SplineKey@U?$Quat_tpl@M@@@spline@@@stlpmtx_std@@_J@stlpmtx_std@@YAXPEAU?$SplineKey@U?$Quat_tpl@M@@@spline@@00U12@U?$less@U?$SplineKey@U?$Quat_tpl@M@@@spline@@@0@PEA_J@Z 000000003158fa00 f i FaceAnimSequence.obj
 0001:0008eb10       ??$copy_backward@PEAU?$SplineKey@U?$Quat_tpl@M@@@spline@@PEAU12@@stlpmtx_std@@YAPEAU?$SplineKey@U?$Quat_tpl@M@@@spline@@PEAU12@00@Z 000000003158fb10 f i FaceAnimSequence.obj
 0001:0008eb90       ??$__make_heap@PEAU?$SplineKey@U?$Quat_tpl@M@@@spline@@U?$less@U?$SplineKey@U?$Quat_tpl@M@@@spline@@@stlpmtx_std@@U12@_J@stlpmtx_std@@YAXPEAU?$SplineKey@U?$Quat_tpl@M@@@spline@@0U?$less@U?$SplineKey@U?$Quat_tpl@M@@@spline@@@0@0PEA_J@Z 000000003158fb90 f i FaceAnimSequence.obj
 0001:0008ed80       ??$__pop_heap_aux@PEAU?$SplineKey@U?$Quat_tpl@M@@@spline@@U12@U?$less@U?$SplineKey@U?$Quat_tpl@M@@@spline@@@stlpmtx_std@@@stlpmtx_std@@YAXPEAU?$SplineKey@U?$Quat_tpl@M@@@spline@@00U?$less@U?$SplineKey@U?$Quat_tpl@M@@@spline@@@0@@Z 000000003158fd80 f i FaceAnimSequence.obj
 0001:0008ee40       ??4?$DynArray@U?$SplineKey@U?$Quat_tpl@M@@@spline@@HU?$SmallDynStorage@U?$SplineKey@U?$Quat_tpl@M@@@spline@@HUStandardAlloc@NAlloc@@@NArray@@@@QEAAAEAU0@U?$Array@$$CBU?$SplineKey@U?$Quat_tpl@M@@@spline@@HU?$ArrayStorage@$$CBU?$SplineKey@U?$Quat_tpl@M@@@spline@@H@NArray@@@@@Z 000000003158fe40 f i FaceAnimSequence.obj
 0001:0008ef60       ?push_back@?$DynArray@U?$SplineKey@U?$Quat_tpl@M@@@spline@@HU?$SmallDynStorage@U?$SplineKey@U?$Quat_tpl@M@@@spline@@HUStandardAlloc@NAlloc@@@NArray@@@@QEAAPEAU?$SplineKey@U?$Quat_tpl@M@@@spline@@U?$Array@$$CBU?$SplineKey@U?$Quat_tpl@M@@@spline@@HU?$ArrayStorage@$$CBU?$SplineKey@U?$Quat_tpl@M@@@spline@@H@NArray@@@@@Z 000000003158ff60 f i FaceAnimSequence.obj
 0001:0008f040       ?insert_raw@?$DynArray@U?$SplineKey@U?$Quat_tpl@M@@@spline@@HU?$SmallDynStorage@U?$SplineKey@U?$Quat_tpl@M@@@spline@@HUStandardAlloc@NAlloc@@@NArray@@@@QEAA?AU?$Array@U?$SplineKey@U?$Quat_tpl@M@@@spline@@HU?$ArrayStorage@U?$SplineKey@U?$Quat_tpl@M@@@spline@@H@NArray@@@@PEAU?$SplineKey@U?$Quat_tpl@M@@@spline@@H@Z 0000000031590040 f i FaceAnimSequence.obj
 0001:0008f180       ??$__unguarded_partition@PEAU?$SplineKey@U?$Quat_tpl@M@@@spline@@U12@U?$less@U?$SplineKey@U?$Quat_tpl@M@@@spline@@@stlpmtx_std@@@priv@stlpmtx_std@@YAPEAU?$SplineKey@U?$Quat_tpl@M@@@spline@@PEAU23@0U23@U?$less@U?$SplineKey@U?$Quat_tpl@M@@@spline@@@1@@Z 0000000031590180 f i FaceAnimSequence.obj
 0001:0008f2a0       ??$__linear_insert@PEAU?$SplineKey@U?$Quat_tpl@M@@@spline@@U12@U?$less@U?$SplineKey@U?$Quat_tpl@M@@@spline@@@stlpmtx_std@@@priv@stlpmtx_std@@YAXPEAU?$SplineKey@U?$Quat_tpl@M@@@spline@@0U23@U?$less@U?$SplineKey@U?$Quat_tpl@M@@@spline@@@1@@Z 00000000315902a0 f i FaceAnimSequence.obj
 0001:0008f3c0       ?RemoveKey@?$CBaseSplineInterpolator@U?$Quat_tpl@M@@V?$HermitSplineEx@U?$Quat_tpl@M@@U?$SplineKey@U?$Quat_tpl@M@@@spline@@@spline@@@spline@@UEAAXH@Z 00000000315903c0 f i FaceAnimSequence.obj
 0001:0008f410       ?RemoveKeysInRange@?$CBaseSplineInterpolator@U?$Quat_tpl@M@@V?$HermitSplineEx@U?$Quat_tpl@M@@U?$SplineKey@U?$Quat_tpl@M@@@spline@@@spline@@@spline@@UEAAXMM@Z 0000000031590410 f i FaceAnimSequence.obj
 0001:0008f580       ??0?$DynArray@U?$SplineKey@U?$Quat_tpl@M@@@spline@@HU?$SmallDynStorage@U?$SplineKey@U?$Quat_tpl@M@@@spline@@HUStandardAlloc@NAlloc@@@NArray@@@@QEAA@AEBU0@@Z 0000000031590580 f i FaceAnimSequence.obj
 0001:0008f620       ??$__insertion_sort@PEAU?$SplineKey@U?$Quat_tpl@M@@@spline@@U12@U?$less@U?$SplineKey@U?$Quat_tpl@M@@@spline@@@stlpmtx_std@@@priv@stlpmtx_std@@YAXPEAU?$SplineKey@U?$Quat_tpl@M@@@spline@@00U?$less@U?$SplineKey@U?$Quat_tpl@M@@@spline@@@1@@Z 0000000031590620 f i FaceAnimSequence.obj
 0001:0008f740       ??$sort_heap@PEAU?$SplineKey@U?$Quat_tpl@M@@@spline@@U?$less@U?$SplineKey@U?$Quat_tpl@M@@@spline@@@stlpmtx_std@@@stlpmtx_std@@YAXPEAU?$SplineKey@U?$Quat_tpl@M@@@spline@@0U?$less@U?$SplineKey@U?$Quat_tpl@M@@@spline@@@0@@Z 0000000031590740 f i FaceAnimSequence.obj
 0001:0008f7f0       ??4?$TSpline@U?$SplineKey@U?$Quat_tpl@M@@@spline@@VHermitBasis@2@@spline@@QEAAAEAV01@AEBV01@@Z 00000000315907f0 f i FaceAnimSequence.obj
 0001:0008f870       ??$__final_insertion_sort@PEAU?$SplineKey@U?$Quat_tpl@M@@@spline@@U?$less@U?$SplineKey@U?$Quat_tpl@M@@@spline@@@stlpmtx_std@@@priv@stlpmtx_std@@YAXPEAU?$SplineKey@U?$Quat_tpl@M@@@spline@@0U?$less@U?$SplineKey@U?$Quat_tpl@M@@@spline@@@1@@Z 0000000031590870 f i FaceAnimSequence.obj
 0001:0008f8f0       ??$__partial_sort@PEAU?$SplineKey@U?$Quat_tpl@M@@@spline@@U12@U?$less@U?$SplineKey@U?$Quat_tpl@M@@@spline@@@stlpmtx_std@@@priv@stlpmtx_std@@YAXPEAU?$SplineKey@U?$Quat_tpl@M@@@spline@@000U?$less@U?$SplineKey@U?$Quat_tpl@M@@@spline@@@1@@Z 00000000315908f0 f i FaceAnimSequence.obj
 0001:0008fa50       ?InsertKey@?$CBaseSplineInterpolator@U?$Quat_tpl@M@@V?$HermitSplineEx@U?$Quat_tpl@M@@U?$SplineKey@U?$Quat_tpl@M@@@spline@@@spline@@@spline@@UEAAHMQEAM@Z 0000000031590a50 f i FaceAnimSequence.obj
 0001:0008fcd0       ?Restore@?$CBaseSplineInterpolator@U?$Quat_tpl@M@@V?$HermitSplineEx@U?$Quat_tpl@M@@U?$SplineKey@U?$Quat_tpl@M@@@spline@@@spline@@@spline@@UEAAXPEAUISplineBackup@@@Z 0000000031590cd0 f i FaceAnimSequence.obj
 0001:0008fd00       ??0?$SSplineBackup@V?$HermitSplineEx@U?$Quat_tpl@M@@U?$SplineKey@U?$Quat_tpl@M@@@spline@@@spline@@@spline@@QEAA@AEBV?$HermitSplineEx@U?$Quat_tpl@M@@U?$SplineKey@U?$Quat_tpl@M@@@spline@@@1@@Z 0000000031590d00 f i FaceAnimSequence.obj
 0001:0008fd80       ??_E?$SSplineBackup@V?$HermitSplineEx@U?$Quat_tpl@M@@U?$SplineKey@U?$Quat_tpl@M@@@spline@@@spline@@@spline@@W7EAAPEAXI@Z 0000000031590d80 f i FaceAnimSequence.obj
 0001:0008fd90       ??_G?$SSplineBackup@V?$HermitSplineEx@U?$Quat_tpl@M@@U?$SplineKey@U?$Quat_tpl@M@@@spline@@@spline@@@spline@@UEAAPEAXI@Z 0000000031590d90 f i FaceAnimSequence.obj
 0001:0008fd90       ??_E?$SSplineBackup@V?$HermitSplineEx@U?$Quat_tpl@M@@U?$SplineKey@U?$Quat_tpl@M@@@spline@@@spline@@@spline@@UEAAPEAXI@Z 0000000031590d90 f i FaceAnimSequence.obj
 0001:0008fe10       ??$__introsort_loop@PEAU?$SplineKey@U?$Quat_tpl@M@@@spline@@U12@_JU?$less@U?$SplineKey@U?$Quat_tpl@M@@@spline@@@stlpmtx_std@@@priv@stlpmtx_std@@YAXPEAU?$SplineKey@U?$Quat_tpl@M@@@spline@@00_JU?$less@U?$SplineKey@U?$Quat_tpl@M@@@spline@@@1@@Z 0000000031590e10 f i FaceAnimSequence.obj
 0001:00090000       ?GetAnimationCount@CAnimationSet@@UEBAIXZ 0000000031591000 f i ModelAnimationSet.obj
 0001:00090000       ?GetKeyCount@?$CBaseSplineInterpolator@MV?$CatmullRomSpline@MU?$SplineKey@M@spline@@$0A@@spline@@@spline@@UEAAHXZ 0000000031591000 f i FaceEffector.obj
 0001:00090000       ?GetKeyCount@?$CBaseSplineInterpolator@U?$Quat_tpl@M@@V?$HermitSplineEx@U?$Quat_tpl@M@@U?$SplineKey@U?$Quat_tpl@M@@@spline@@@spline@@@spline@@UEAAHXZ 0000000031591000 f i FaceAnimSequence.obj
 0001:00090000       ?GetKeyCount@?$CBaseSplineInterpolator@MV?$HermitSplineEx@MU?$SplineKey@M@spline@@@spline@@@spline@@UEAAHXZ 0000000031591000 f i FaceAnimSequence.obj
 0001:00090000       ?GetKeyCount@?$CBaseSplineInterpolator@U?$Vec3_tpl@M@@V?$TCBSpline@U?$Vec3_tpl@M@@U?$TCBSplineKey@U?$Vec3_tpl@M@@@spline@@@spline@@@spline@@UEAAHXZ 0000000031591000 f i FaceAnimSequence.obj
 0001:00090010       ?GetKeyValue@?$CBaseSplineInterpolator@MV?$HermitSplineEx@MU?$SplineKey@M@spline@@@spline@@@spline@@UEAA_NHAEAY03M@Z 0000000031591010 f i FaceAnimSequence.obj
 0001:00090010       ?GetKeyValue@?$CBaseSplineInterpolator@MV?$CatmullRomSpline@MU?$SplineKey@M@spline@@$0A@@spline@@@spline@@UEAA_NHAEAY03M@Z 0000000031591010 f i FaceEffector.obj
 0001:00090040       ?SetKeyOutTangent@?$CBaseSplineInterpolator@MV?$HermitSplineEx@MU?$SplineKey@M@spline@@@spline@@@spline@@UEAAXHQEAM@Z 0000000031591040 f i FaceAnimSequence.obj
 0001:00090040       ?SetKeyOutTangent@?$CBaseSplineInterpolator@MV?$CatmullRomSpline@MU?$SplineKey@M@spline@@$0A@@spline@@@spline@@UEAAXHQEAM@Z 0000000031591040 f i FaceEffector.obj
 0001:00090070       ?GetKeyTangents@?$CBaseSplineInterpolator@MV?$HermitSplineEx@MU?$SplineKey@M@spline@@@spline@@@spline@@UEAA_NHAEAY03M0@Z 0000000031591070 f i FaceAnimSequence.obj
 0001:00090070       ?GetKeyTangents@?$CBaseSplineInterpolator@MV?$CatmullRomSpline@MU?$SplineKey@M@spline@@$0A@@spline@@@spline@@UEAA_NHAEAY03M0@Z 0000000031591070 f i FaceEffector.obj
 0001:000900b0       ?GetKeyFlags@?$CBaseSplineInterpolator@MV?$HermitSplineEx@MU?$SplineKey@M@spline@@@spline@@@spline@@UEAAHH@Z 00000000315910b0 f i FaceAnimSequence.obj
 0001:000900b0       ?GetKeyFlags@?$CBaseSplineInterpolator@MV?$CatmullRomSpline@MU?$SplineKey@M@spline@@$0A@@spline@@@spline@@UEAAHH@Z 00000000315910b0 f i FaceEffector.obj
 0001:000900e0       ?FindKeysInRange@?$CBaseSplineInterpolator@MV?$HermitSplineEx@MU?$SplineKey@M@spline@@@spline@@@spline@@UEAAXMMAEAH0@Z 00000000315910e0 f i FaceAnimSequence.obj
 0001:000900e0       ?FindKeysInRange@?$CBaseSplineInterpolator@MV?$CatmullRomSpline@MU?$SplineKey@M@spline@@$0A@@spline@@@spline@@UEAAXMMAEAH0@Z 00000000315910e0 f i FaceEffector.obj
 0001:00090220       ?erase@?$DynArray@U?$SplineKey@M@spline@@HU?$SmallDynStorage@U?$SplineKey@M@spline@@HUStandardAlloc@NAlloc@@@NArray@@@@QEAAPEAU?$SplineKey@M@spline@@PEAU23@0@Z 0000000031591220 f i FaceAnimSequence.obj
 0001:000902d0       ?insert_raw@?$DynArray@U?$SplineKey@M@spline@@HU?$SmallDynStorage@U?$SplineKey@M@spline@@HUStandardAlloc@NAlloc@@@NArray@@@@QEAA?AU?$Array@U?$SplineKey@M@spline@@HU?$ArrayStorage@U?$SplineKey@M@spline@@H@NArray@@@@PEAU?$SplineKey@M@spline@@H@Z 00000000315912d0 f i FaceAnimSequence.obj
 0001:000903f0       ??4?$DynArray@U?$SplineKey@M@spline@@HU?$SmallDynStorage@U?$SplineKey@M@spline@@HUStandardAlloc@NAlloc@@@NArray@@@@QEAAAEAU0@U?$Array@$$CBU?$SplineKey@M@spline@@HU?$ArrayStorage@$$CBU?$SplineKey@M@spline@@H@NArray@@@@@Z 00000000315913f0 f i FaceAnimSequence.obj
 0001:00090550       ??0?$DynArray@U?$SplineKey@M@spline@@HU?$SmallDynStorage@U?$SplineKey@M@spline@@HUStandardAlloc@NAlloc@@@NArray@@@@QEAA@AEBU0@@Z 0000000031591550 f i FaceAnimSequence.obj
 0001:00090630       ?Restore@?$CBaseSplineInterpolator@MV?$HermitSplineEx@MU?$SplineKey@M@spline@@@spline@@@spline@@UEAAXPEAUISplineBackup@@@Z 0000000031591630 f i FaceAnimSequence.obj
 0001:00090660       ??0?$SSplineBackup@V?$HermitSplineEx@MU?$SplineKey@M@spline@@@spline@@@spline@@QEAA@AEBV?$HermitSplineEx@MU?$SplineKey@M@spline@@@1@@Z 0000000031591660 f i FaceAnimSequence.obj
 0001:000906e0       ??_E?$SSplineBackup@V?$HermitSplineEx@MU?$SplineKey@M@spline@@@spline@@@spline@@W7EAAPEAXI@Z 00000000315916e0 f i FaceAnimSequence.obj
 0001:000906f0       ??_G?$SSplineBackup@V?$HermitSplineEx@MU?$SplineKey@M@spline@@@spline@@@spline@@UEAAPEAXI@Z 00000000315916f0 f i FaceAnimSequence.obj
 0001:000906f0       ??_E?$SSplineBackup@V?$HermitSplineEx@MU?$SplineKey@M@spline@@@spline@@@spline@@UEAAPEAXI@Z 00000000315916f0 f i FaceAnimSequence.obj
 0001:00090770       ?DeleteSoundEntry@CFacialAnimSequence@@UEAAXH@Z 0000000031591770 f   FaceAnimSequence.obj
 0001:00090810       ?DeleteSkeletonAnimationEntry@CFacialAnimSequence@@UEAAXH@Z 0000000031591810 f   FaceAnimSequence.obj
 0001:00090870       ?Backup@?$CBaseSplineInterpolator@MV?$HermitSplineEx@MU?$SplineKey@M@spline@@@spline@@@spline@@UEAAPEAUISplineBackup@@XZ 0000000031591870 f i FaceAnimSequence.obj
 0001:000908c0       ?Restore@?$CBaseSplineInterpolator@U?$Vec3_tpl@M@@V?$TCBSpline@U?$Vec3_tpl@M@@U?$TCBSplineKey@U?$Vec3_tpl@M@@@spline@@@spline@@@spline@@UEAAXPEAUISplineBackup@@@Z 00000000315918c0 f i FaceAnimSequence.obj
 0001:000908f0       ?Backup@?$CBaseSplineInterpolator@U?$Quat_tpl@M@@V?$HermitSplineEx@U?$Quat_tpl@M@@U?$SplineKey@U?$Quat_tpl@M@@@spline@@@spline@@@spline@@UEAAPEAUISplineBackup@@XZ 00000000315918f0 f i FaceAnimSequence.obj
 0001:00090940       ??0?$SSplineBackup@V?$TCBSpline@U?$Vec3_tpl@M@@U?$TCBSplineKey@U?$Vec3_tpl@M@@@spline@@@spline@@@spline@@QEAA@AEBV?$TCBSpline@U?$Vec3_tpl@M@@U?$TCBSplineKey@U?$Vec3_tpl@M@@@spline@@@1@@Z 0000000031591940 f i FaceAnimSequence.obj
 0001:000909c0       ?AddRef@?$SSplineBackup@V?$HermitSplineEx@MU?$SplineKey@M@spline@@@spline@@@spline@@UEAAXXZ 00000000315919c0 f i FaceAnimSequence.obj
 0001:000909c0       ?AddRef@?$SSplineBackup@V?$HermitSplineEx@U?$Quat_tpl@M@@U?$SplineKey@U?$Quat_tpl@M@@@spline@@@spline@@@spline@@UEAAXXZ 00000000315919c0 f i FaceAnimSequence.obj
 0001:000909c0       ?AddRef@?$SSplineBackup@V?$TCBSpline@U?$Vec3_tpl@M@@U?$TCBSplineKey@U?$Vec3_tpl@M@@@spline@@@spline@@@spline@@UEAAXXZ 00000000315919c0 f i FaceAnimSequence.obj
 0001:000909d0       ?Release@?$SSplineBackup@V?$HermitSplineEx@MU?$SplineKey@M@spline@@@spline@@@spline@@UEAAXXZ 00000000315919d0 f i FaceAnimSequence.obj
 0001:000909d0       ?Release@?$SSplineBackup@V?$HermitSplineEx@U?$Quat_tpl@M@@U?$SplineKey@U?$Quat_tpl@M@@@spline@@@spline@@@spline@@UEAAXXZ 00000000315919d0 f i FaceAnimSequence.obj
 0001:000909d0       ?Release@?$SSplineBackup@V?$TCBSpline@U?$Vec3_tpl@M@@U?$TCBSplineKey@U?$Vec3_tpl@M@@@spline@@@spline@@@spline@@UEAAXXZ 00000000315919d0 f i FaceAnimSequence.obj
 0001:000909f0       ??_E?$SSplineBackup@V?$TCBSpline@U?$Vec3_tpl@M@@U?$TCBSplineKey@U?$Vec3_tpl@M@@@spline@@@spline@@@spline@@W7EAAPEAXI@Z 00000000315919f0 f i FaceAnimSequence.obj
 0001:00090a00       ??_G?$SSplineBackup@V?$TCBSpline@U?$Vec3_tpl@M@@U?$TCBSplineKey@U?$Vec3_tpl@M@@@spline@@@spline@@@spline@@UEAAPEAXI@Z 0000000031591a00 f i FaceAnimSequence.obj
 0001:00090a00       ??_E?$SSplineBackup@V?$TCBSpline@U?$Vec3_tpl@M@@U?$TCBSplineKey@U?$Vec3_tpl@M@@@spline@@@spline@@@spline@@UEAAPEAXI@Z 0000000031591a00 f i FaceAnimSequence.obj
 0001:00090a80       ??$sort@PEAU?$TCBSplineKey@U?$Vec3_tpl@M@@@spline@@@stlpmtx_std@@YAXPEAU?$TCBSplineKey@U?$Vec3_tpl@M@@@spline@@0@Z 0000000031591a80 f i FaceAnimSequence.obj
 0001:00090af0       ??$sort@PEAU?$SplineKey@M@spline@@@stlpmtx_std@@YAXPEAU?$SplineKey@M@spline@@0@Z 0000000031591af0 f i FaceAnimSequence.obj
 0001:00090b70       ??$sort@PEAU?$SplineKey@U?$Quat_tpl@M@@@spline@@@stlpmtx_std@@YAXPEAU?$SplineKey@U?$Quat_tpl@M@@@spline@@0@Z 0000000031591b70 f i FaceAnimSequence.obj
 0001:00090bf0       ??$sort@PEAU?$pair@PEAUIFacialAnimChannel@@H@stlpmtx_std@@VFirstLess@?$VectorMap@PEAUIFacialAnimChannel@@HU?$less@PEAUIFacialAnimChannel@@@stlpmtx_std@@V?$allocator@U?$pair@PEAUIFacialAnimChannel@@H@stlpmtx_std@@@3@@@@stlpmtx_std@@YAXPEAU?$pair@PEAUIFacialAnimChannel@@H@0@0VFirstLess@?$VectorMap@PEAUIFacialAnimChannel@@HU?$less@PEAUIFacialAnimChannel@@@stlpmtx_std@@V?$allocator@U?$pair@PEAUIFacialAnimChannel@@H@stlpmtx_std@@@3@@@@Z 0000000031591bf0 f i FaceAnimSequence.obj
 0001:00090ca0       ?CreateChannelGroup@Data@CFacialAnimSequence@@QEAAPEAUIFacialAnimChannel@@XZ 0000000031591ca0 f i FaceAnimSequence.obj
 0001:00090e90       ??1CProceduralChannelSet@@QEAA@XZ 0000000031591e90 f i FaceAnimSequence.obj
 0001:00090fa0       ??_ECFacialCameraPathPositionInterpolator@@W7EAAPEAXI@Z 0000000031591fa0 f i FaceAnimSequence.obj
 0001:00090fb0       ??_ECFacialCameraPathPositionInterpolator@@UEAAPEAXI@Z 0000000031591fb0 f i FaceAnimSequence.obj
 0001:00090fb0       ??_GCFacialCameraPathPositionInterpolator@@UEAAPEAXI@Z 0000000031591fb0 f i FaceAnimSequence.obj
 0001:00091030       ??_ECFacialCameraPathOrientationInterpolator@@W7EAAPEAXI@Z 0000000031592030 f i FaceAnimSequence.obj
 0001:00091040       ??_GCFacialCameraPathOrientationInterpolator@@UEAAPEAXI@Z 0000000031592040 f i FaceAnimSequence.obj
 0001:00091040       ??_ECFacialCameraPathOrientationInterpolator@@UEAAPEAXI@Z 0000000031592040 f i FaceAnimSequence.obj
 0001:000910c0       ??_ECFacialAnimChannelInterpolator@@W7EAAPEAXI@Z 00000000315920c0 f i FaceAnimSequence.obj
 0001:000910d0       ??_GCFacialAnimChannelInterpolator@@UEAAPEAXI@Z 00000000315920d0 f i FaceAnimSequence.obj
 0001:000910d0       ??_ECFacialAnimChannelInterpolator@@UEAAPEAXI@Z 00000000315920d0 f i FaceAnimSequence.obj
 0001:00091150       ?CreateInterpolator@CFacialAnimChannel@@QEAAXXZ 0000000031592150 f   FaceAnimSequence.obj
 0001:00091390       ?AddInterpolator@CFacialAnimChannel@@UEAAXXZ 0000000031592390 f   FaceAnimSequence.obj
 0001:00091520       ??1Data@CFacialAnimSequence@@QEAA@XZ 0000000031592520 f i FaceAnimSequence.obj
 0001:00091670       ??1CFacialAnimSequence@@UEAA@XZ 0000000031592670 f   FaceAnimSequence.obj
 0001:00091740       ?AddRef@CFacialAnimSequence@@UEAAXXZ 0000000031592740 f i FaceAnimSequence.obj
 0001:00091750       ?SetFlags@CFacialAnimSequence@@UEAAXH@Z 0000000031592750 f i FaceAnimSequence.obj
 0001:00091760       ?GetFlags@CFacialAnimSequence@@UEAAHXZ 0000000031592760 f i FaceAnimSequence.obj
 0001:00091770       ?GetCameraPathPosition@CFacialAnimSequence@@UEAAPEAUISplineInterpolator@@XZ 0000000031592770 f i FaceAnimSequence.obj
 0001:00091780       ?GetCameraPathOrientation@CFacialAnimSequence@@UEAAPEAUISplineInterpolator@@XZ 0000000031592780 f i FaceAnimSequence.obj
 0001:00091790       ?GetCameraPathFOV@CFacialAnimSequence@@UEAAPEAUISplineInterpolator@@XZ 0000000031592790 f i FaceAnimSequence.obj
 0001:000917a0       ?IsInMemory@CFacialAnimSequence@@UEBA_NXZ 00000000315927a0 f i FaceAnimSequence.obj
 0001:000917b0       ?SetInMemory@CFacialAnimSequence@@UEAAX_N@Z 00000000315927b0 f i FaceAnimSequence.obj
 0001:000917c0       ??_ECFacialAnimSequence@@W7EAAPEAXI@Z 00000000315927c0 f i FaceAnimSequence.obj
 0001:000917d0       ?GetName@CFacialAnimSequence@@UEAAPEBDXZ 00000000315927d0 f i FaceAnimSequence.obj
 0001:000917d0       ?GetID@CFacialJoystick@@UEBA_KXZ 00000000315927d0 f i FaceJoystick.obj
 0001:000917d0       ?GetText@CFacialSentence@@UEAAPEBDXZ 00000000315927d0 f i LipSync.obj
 0001:000917e0       ?GetTimeRange@CFacialAnimSequence@@UEAA?AV?$TRange@M@@XZ 00000000315927e0 f i FaceAnimSequence.obj
 0001:000917f0       ?SetTimeRange@CFacialAnimSequence@@UEAAXV?$TRange@M@@@Z 00000000315927f0 f i FaceAnimSequence.obj
 0001:00091800       ?GetChannelCount@CFacialAnimSequence@@UEAAHXZ 0000000031592800 f i FaceAnimSequence.obj
 0001:00091810       ?CreateChannelGroup@CFacialAnimSequence@@UEAAPEAUIFacialAnimChannel@@XZ 0000000031592810 f   FaceAnimSequence.obj
 0001:00091820       ?StreamOnComplete@CFacialAnimSequence@@UEAAXPEAVIReadStream@@I@Z 0000000031592820 f   FaceAnimSequence.obj
 0001:00091a70       ?UnbindProceduralChannels@CFacialAnimSequenceInstance@@AEAAXXZ 0000000031592a70 f   FaceAnimSequence.obj
 0001:00091b10       ?Backup@?$CBaseSplineInterpolator@U?$Vec3_tpl@M@@V?$TCBSpline@U?$Vec3_tpl@M@@U?$TCBSplineKey@U?$Vec3_tpl@M@@@spline@@@spline@@@spline@@UEAAPEAUISplineBackup@@XZ 0000000031592b10 f i FaceAnimSequence.obj
 0001:00091b60       ?CreateChannel@Data@CFacialAnimSequence@@QEAAPEAUIFacialAnimChannel@@XZ 0000000031592b60 f i FaceAnimSequence.obj
 0001:00091d50       ??_ECFacialAnimSequence@@UEAAPEAXI@Z 0000000031592d50 f i FaceAnimSequence.obj
 0001:00091d50       ??_GCFacialAnimSequence@@UEAAPEAXI@Z 0000000031592d50 f i FaceAnimSequence.obj
 0001:00091d80       ?CreateChannel@CFacialAnimSequence@@UEAAPEAUIFacialAnimChannel@@XZ 0000000031592d80 f   FaceAnimSequence.obj
 0001:00091d90       ?SerializeChannelLoad@CFacialAnimSequence@@AEAAXAEAUData@1@PEAUIFacialAnimChannel@@AEAVXmlNodeRef@@@Z 0000000031592d90 f   FaceAnimSequence.obj
 0001:00092030       ?UnbindChannels@CFacialAnimSequenceInstance@@QEAAXXZ 0000000031593030 f   FaceAnimSequence.obj
 0001:00092140       ??0CProceduralChannelSet@@QEAA@XZ 0000000031593140 f   FaceAnimSequence.obj
 0001:000922f0       ??0Data@CFacialAnimSequence@@QEAA@XZ 00000000315932f0 f i FaceAnimSequence.obj
 0001:00092450       ??0CFacialAnimSequence@@QEAA@PEAVCFacialAnimation@@@Z 0000000031593450 f   FaceAnimSequence.obj
 0001:000924e0       ?StartStreaming@CFacialAnimSequence@@UEAA_NPEBD@Z 00000000315934e0 f   FaceAnimSequence.obj
 0001:00092680       ?BindProceduralChannels@CFacialAnimSequenceInstance@@AEAAXPEAVCFacialAnimationContext@@PEAVCFacialAnimSequence@@@Z 0000000031593680 f   FaceAnimSequence.obj
 0001:00092910       ?interpolate@?$TSpline@U?$TCBSplineKey@U?$Vec3_tpl@M@@@spline@@VHermitBasis@2@@spline@@QEAA_NMAEAU?$Vec3_tpl@M@@@Z 0000000031593910 f i FaceAnimSequence.obj
 0001:00092a70       ?interpolate@?$TSpline@U?$SplineKey@U?$Quat_tpl@M@@@spline@@VHermitBasis@2@@spline@@QEAA_NMAEAU?$Quat_tpl@M@@@Z 0000000031593a70 f i FaceAnimSequence.obj
 0001:00092bd0       ?Interpolate@CFacialAnimChannelInterpolator@@UEAAXMAEAY03M@Z 0000000031593bd0 f i FaceAnimSequence.obj
 0001:00092c00       ?Interpolate@CFacialCameraPathPositionInterpolator@@UEAAXMAEAY03M@Z 0000000031593c00 f i FaceAnimSequence.obj
 0001:00092c50       ?Interpolate@CFacialCameraPathOrientationInterpolator@@UEAAXMAEAY03M@Z 0000000031593c50 f i FaceAnimSequence.obj
 0001:00092cc0       ?Evaluate@CFacialAnimChannel@@QEAAMM@Z 0000000031593cc0 f   FaceAnimSequence.obj
 0001:00092f70       ?InsertSoundEntry@CFacialAnimSequence@@UEAAXH@Z 0000000031593f70 f   FaceAnimSequence.obj
 0001:000930e0       ?InsertSkeletonAnimationEntry@CFacialAnimSequence@@UEAAXH@Z 00000000315940e0 f   FaceAnimSequence.obj
 0001:00093200       ?MergeSequence@CFacialAnimSequence@@UEAAXPEAUIFacialAnimSequence@@AEBV?$Functor1wRet@PEBDW4MergeCollisionAction@@@@@Z 0000000031594200 f   FaceAnimSequence.obj
 0001:00094840       ?BindChannels@CFacialAnimSequenceInstance@@QEAAXPEAVCFacialAnimationContext@@PEAVCFacialAnimSequence@@@Z 0000000031595840 f   FaceAnimSequence.obj
 0001:00095680       ?Animate@CFacialAnimSequence@@UEAAXAEBU?$QuatTS_tpl@M@@PEAVCFacialAnimSequenceInstance@@M@Z 0000000031596680 f   FaceAnimSequence.obj
 0001:000964a0       ?SerializeLoad@CFacialAnimSequence@@AEAAXAEAUData@1@AEAVXmlNodeRef@@W4ESerializationFlags@IFacialAnimSequence@@@Z 00000000315974a0 f   FaceAnimSequence.obj
 0001:00096ee0       ?Serialize@CFacialAnimSequence@@UEAAXAEAVXmlNodeRef@@_NW4ESerializationFlags@IFacialAnimSequence@@@Z 0000000031597ee0 f   FaceAnimSequence.obj
 0001:00097290       ?StreamAsyncOnComplete@CFacialAnimSequence@@UEAAXPEAVIReadStream@@I@Z 0000000031598290 f   FaceAnimSequence.obj
 0001:00097370       ??$fill@PEAVFaceChannelCleanupKeysKeyEntry@@V1@@stlpmtx_std@@YAXPEAVFaceChannelCleanupKeysKeyEntry@@0AEBV1@@Z 0000000031598370 f i FaceChannelKeyCleanup.obj
 0001:000973e0       ??$__uninitialized_fill_n@PEAVFaceChannelCleanupKeysKeyEntry@@_KV1@@priv@stlpmtx_std@@YAPEAVFaceChannelCleanupKeysKeyEntry@@PEAV2@_KAEBV2@@Z 00000000315983e0 f i FaceChannelKeyCleanup.obj
 0001:00097480       ?_M_fill_insert_aux@?$_Impl_vector@VFaceChannelCleanupKeysKeyEntry@@V?$allocator@VFaceChannelCleanupKeysKeyEntry@@@stlpmtx_std@@@priv@stlpmtx_std@@AEAAXPEAVFaceChannelCleanupKeysKeyEntry@@_KAEBV4@AEBU__false_type@3@@Z 0000000031598480 f i FaceChannelKeyCleanup.obj
 0001:00097610       ?CleanupKeys@FaceChannel@@YAXPEAVCFacialAnimChannelInterpolator@@M@Z 0000000031598610 f   FaceChannelKeyCleanup.obj
 0001:000986d0       ??0GaussianKernel@FaceChannel@@QEAA@M_N@Z 00000000315996d0 f   FaceChannelSmoothing.obj
 0001:00098800       ?ApplyKernel@FaceChannel@@YAXPEAVCFacialAnimChannelInterpolator@@0HPEBM@Z 0000000031599800 f   FaceChannelSmoothing.obj
 0001:000989e0       ?ApplyKernelNoiseFilter@FaceChannel@@YAXPEAVCFacialAnimChannelInterpolator@@0HPEBMM@Z 00000000315999e0 f   FaceChannelSmoothing.obj
 0001:00098c40       ?RemoveNoise@FaceChannel@@YAXPEAVCFacialAnimChannelInterpolator@@MM@Z 0000000031599c40 f   FaceChannelSmoothing.obj
 0001:00098d60       ?GaussianBlurKeys@FaceChannel@@YAXPEAVCFacialAnimChannelInterpolator@@M@Z 0000000031599d60 f   FaceChannelSmoothing.obj
 0001:00098f50       ??_GIFacialEffector@@UEAAPEAXI@Z 0000000031599f50 f i FaceEffector.obj
 0001:00098f50       ??_EIFacialEffector@@UEAAPEAXI@Z 0000000031599f50 f i FaceEffector.obj
 0001:00098f80       ??_GIJoystickSet@@UEAAPEAXI@Z 0000000031599f80 f i FaceJoystick.obj
 0001:00098f80       ??_EIFacialEffCtrl@@UEAAPEAXI@Z 0000000031599f80 f i FaceEffector.obj
 0001:00098f80       ??_GIFacialEffCtrl@@UEAAPEAXI@Z 0000000031599f80 f i FaceEffector.obj
 0001:00098f80       ??_EIJoystickSet@@UEAAPEAXI@Z 0000000031599f80 f i FaceJoystick.obj
 0001:00098fb0       ?GetParamString@CFacialEffector@@UEAAPEBDW4EFacialEffectorParam@@@Z 0000000031599fb0 f i FaceEffector.obj
 0001:00098fc0       ?Interpolate@CFacialEffCtrlSplineInterpolator@@UEAAXMAEAY03M@Z 0000000031599fc0 f   FaceEffector.obj
 0001:00098fe0       ?GetParamString@CFacialEffectorAttachment@@UEAAPEBDW4EFacialEffectorParam@@@Z 0000000031599fe0 f   FaceEffector.obj
 0001:00099000       ?GetParamVec3@CFacialEffectorAttachment@@UEAA?AU?$Vec3_tpl@M@@W4EFacialEffectorParam@@@Z 000000003159a000 f   FaceEffector.obj
 0001:00099040       ?GetSubEffector@CFacialEffector@@UEAAPEAUIFacialEffector@@H@Z 000000003159a040 f   FaceEffector.obj
 0001:00099060       ?GetSubEffCtrl@CFacialEffector@@UEAAPEAUIFacialEffCtrl@@H@Z 000000003159a060 f   FaceEffector.obj
 0001:00099070       ?SetParamVec3@CFacialEffectorAttachment@@UEAAXW4EFacialEffectorParam@@U?$Vec3_tpl@M@@@Z 000000003159a070 f   FaceEffector.obj
 0001:00099230       ?GetQuatT@CFacialEffectorAttachment@@UEAA?AU?$QuatT_tpl@M@@XZ 000000003159a230 f   FaceEffector.obj
 0001:00099270       ?seek_key@?$TSpline@U?$SplineKey@M@spline@@VHermitBasis@2@@spline@@IEAAHM@Z 000000003159a270 f i FaceAnimSequence.obj
 0001:00099270       ?seek_key@?$TSpline@U?$SplineKey@M@spline@@U?$TCoeffBasis@M@2@@spline@@IEAAHM@Z 000000003159a270 f i FaceEffector.obj
 0001:000992e0       ?Set@CFacialEffectorAttachment@@UEAAXQEBV1@@Z 000000003159a2e0 f   FaceEffector.obj
 0001:00099380       ?SetIdentifier@CFacialEffector@@UEAAXVCFaceIdentifierHandle@@@Z 000000003159a380 f   FaceEffector.obj
 0001:000994d0       ?GetMemoryUsage@CFacialEffector@@UEBAXPEAVICrySizer@@@Z 000000003159a4d0 f   FaceEffector.obj
 0001:000995b0       ?SetParamString@CFacialEffectorAttachment@@UEAAXW4EFacialEffectorParam@@PEBD@Z 000000003159a5b0 f   FaceEffector.obj
 0001:00099620       ?Serialize@CFacialEffectorAttachment@@UEAAXAEAVXmlNodeRef@@_N@Z 000000003159a620 f   FaceEffector.obj
 0001:00099950       ?SerializeSpline@CFacialEffCtrlSplineInterpolator@@UEAAXAEAVXmlNodeRef@@_N@Z 000000003159a950 f   FaceEffector.obj
 0001:00099ce0       ?RemoveSubEffector@CFacialEffector@@UEAAXPEAUIFacialEffector@@@Z 000000003159ace0 f   FaceEffector.obj
 0001:00099d50       ??_E?$TSpline@U?$SplineKey@M@spline@@U?$TCoeffBasis@M@2@@spline@@UEAAPEAXI@Z 000000003159ad50 f i FaceEffector.obj
 0001:00099d50       ??_G?$TSpline@U?$SplineKey@M@spline@@VHermitBasis@2@@spline@@UEAAPEAXI@Z 000000003159ad50 f i FaceAnimSequence.obj
 0001:00099d50       ??_G?$TSpline@U?$SplineKey@M@spline@@U?$TCoeffBasis@M@2@@spline@@UEAAPEAXI@Z 000000003159ad50 f i FaceEffector.obj
 0001:00099d50       ??_E?$TSpline@U?$SplineKey@M@spline@@VHermitBasis@2@@spline@@UEAAPEAXI@Z 000000003159ad50 f i FaceAnimSequence.obj
 0001:00099dc0       ??0CFacialEffector@@QEAA@XZ 000000003159adc0 f i FaceEffector.obj
 0001:00099e40       ?SetFlags@CFacialEffector@@UEAAXI@Z 000000003159ae40 f i FaceEffector.obj
 0001:00099e50       ?GetFlags@CFacialEffector@@UEAAIXZ 000000003159ae50 f i FaceEffector.obj
 0001:00099e60       ?GetIndexInState@CFacialEffector@@UEAAHXZ 000000003159ae60 f i FaceEffector.obj
 0001:00099e70       ?GetIdentifier@CFacialEffector@@UEAA?AVCFaceIdentifierHandle@@XZ 000000003159ae70 f i FaceEffector.obj
 0001:00099e90       ?GetParamVec3@CFacialEffector@@UEAA?AU?$Vec3_tpl@M@@W4EFacialEffectorParam@@@Z 000000003159ae90 f i FaceEffector.obj
 0001:00099ea0       ?GetQuatT@CFacialEffector@@UEAA?AU?$QuatT_tpl@M@@XZ 000000003159aea0 f i FaceEffector.obj
 0001:00099ec0       ?GetSubEffectorCount@CFacialEffector@@UEAAHXZ 000000003159aec0 f i FaceEffector.obj
 0001:00099ed0       ?SetName@CFacialEffector@@UEAAXPEBD@Z 000000003159aed0 f i FaceEffector.obj
 0001:0009a080       ?GetName@CFacialEffector@@UEBAPEBDXZ 000000003159b080 f i FaceEffector.obj
 0001:0009a0d0       ??1?$CatmullRomSpline@MU?$SplineKey@M@spline@@$0A@@spline@@UEAA@XZ 000000003159b0d0 f i FaceEffector.obj
 0001:0009a140       ?set@?$TCoeffBasis@M@spline@@QEAAXMMMMMM@Z 000000003159b140 f i FaceEffector.obj
 0001:0009a210       ?comp_deriv@?$TSplineSlopes@MU?$SplineKey@M@spline@@$0A@@spline@@UEAAXXZ 000000003159b210 f i FaceEffector.obj
 0001:0009a300       ?RemoveAllSubEffectors@CFacialEffector@@UEAAXXZ 000000003159b300 f   FaceEffector.obj
 0001:0009a330       ??0CFacialEffectorAttachment@@QEAA@XZ 000000003159b330 f   FaceEffector.obj
 0001:0009a380       ?GetFormat@?$CKeyTimesInformationStartStop@EUByteStartStopEncoder@@@@UEAAIXZ 000000003159b380 f i ControllerPQ.obj
 0001:0009a380       ?GetFormat@?$CTrackDataStorageInt@U?$Quat_tpl@M@@USmallTree48BitQuat@@VITrackRotationStorage@@@@UEAAIXZ 000000003159b380 f i ControllerPQ.obj
 0001:0009a380       ?GetType@CFacialEffectorAttachment@@UEAA?AW4EFacialEffectorType@@XZ 000000003159b380 f i FaceEffector.obj
 0001:0009a390       ?SetAttachmentCRC@CFacialEffectorAttachment@@UEAAXI@Z 000000003159b390 f i FaceEffector.obj
 0001:0009a3a0       ?GetAttachmentCRC@CFacialEffectorAttachment@@UEAAIXZ 000000003159b3a0 f i FaceEffector.obj
 0001:0009a3b0       ??_ECFacialEffectorAttachment@@W7EAAPEAXI@Z 000000003159b3b0 f i FaceEffector.obj
 0001:0009a3b0       ??_ECFacialEffectorBone@@W7EAAPEAXI@Z 000000003159b3b0 f i FaceEffectorLibrary.obj
 0001:0009a3c0       ?SetQuatT@CFacialEffectorAttachment@@UEAAXU?$QuatT_tpl@M@@@Z 000000003159b3c0 f i FaceEffector.obj
 0001:0009a400       ?GetMemoryUsage@CFacialEffectorAttachment@@UEBAXPEAVICrySizer@@@Z 000000003159b400 f i FaceEffector.obj
 0001:0009a440       ??1CFacialEffectorAttachment@@UEAA@XZ 000000003159b440 f i FaceEffector.obj
 0001:0009a4d0       ??_GCFacialEffectorBone@@UEAAPEAXI@Z 000000003159b4d0 f i FaceEffectorLibrary.obj
 0001:0009a4d0       ??_ECFacialEffectorBone@@UEAAPEAXI@Z 000000003159b4d0 f i FaceEffectorLibrary.obj
 0001:0009a4d0       ??_GCFacialEffectorAttachment@@UEAAPEAXI@Z 000000003159b4d0 f i FaceEffector.obj
 0001:0009a4d0       ??_ECFacialEffectorAttachment@@UEAAPEAXI@Z 000000003159b4d0 f i FaceEffector.obj
 0001:0009a500       ?interp_keys@?$CatmullRomSpline@MU?$SplineKey@M@spline@@$0A@@spline@@MEAAXHHMAEAM@Z 000000003159b500 f i FaceEffector.obj
 0001:0009a560       ?_M_insert_overflow@?$_Impl_vector@U?$TCoeffBasis@M@spline@@V?$allocator@U?$TCoeffBasis@M@spline@@@stlpmtx_std@@@priv@stlpmtx_std@@AEAAXPEAU?$TCoeffBasis@M@spline@@AEBU45@AEBU__true_type@3@_K_N@Z 000000003159b560 f i FaceEffector.obj
 0001:0009a560       ?_M_insert_overflow@?$_Impl_vector@UBalanceChannelEntry@CFacialAnimSequenceInstance@@V?$allocator@UBalanceChannelEntry@CFacialAnimSequenceInstance@@@stlpmtx_std@@@priv@stlpmtx_std@@AEAAXPEAUBalanceChannelEntry@CFacialAnimSequenceInstance@@AEBU45@AEBU__true_type@3@_K_N@Z 000000003159b560 f i FaceAnimSequence.obj
 0001:0009a560       ?_M_insert_overflow@?$_Impl_vector@UPhoneme@IFacialSentence@@V?$allocator@UPhoneme@IFacialSentence@@@stlpmtx_std@@@priv@stlpmtx_std@@AEAAXPEAUPhoneme@IFacialSentence@@AEBU45@AEBU__true_type@3@_K_N@Z 000000003159b560 f i LipSync.obj
 0001:0009a6f0       ??$__uninitialized_fill_n@PEAUBalanceChannelEntry@CFacialAnimSequenceInstance@@_KU12@@priv@stlpmtx_std@@YAPEAUBalanceChannelEntry@CFacialAnimSequenceInstance@@PEAU23@_KAEBU23@@Z 000000003159b6f0 f i FaceAnimSequence.obj
 0001:0009a6f0       ??$__uninitialized_fill_n@PEAU?$TCoeffBasis@M@spline@@_KU12@@priv@stlpmtx_std@@YAPEAU?$TCoeffBasis@M@spline@@PEAU23@_KAEBU23@@Z 000000003159b6f0 f i FaceEffector.obj
 0001:0009a750       ?GetMemoryUsage@?$CatmullRomSpline@MU?$SplineKey@M@spline@@$0A@@spline@@UEBAXPEAVICrySizer@@_N@Z 000000003159b750 f i FaceEffector.obj
 0001:0009a7c0       ?erase@?$_Impl_vector@HV?$allocator@H@stlpmtx_std@@@priv@stlpmtx_std@@QEAAPEAHPEAH0@Z 000000003159b7c0 f i ControllerDefragHeap.obj
 0001:0009a7c0       ?erase@?$_Impl_vector@PEAXV?$allocator@PEAX@stlpmtx_std@@@priv@stlpmtx_std@@QEAAPEAPEAXPEAPEAX0@Z 000000003159b7c0 f i LoaderSKIN.obj
 0001:0009a7c0       ?erase@?$_Impl_vector@IV?$allocator@I@stlpmtx_std@@@priv@stlpmtx_std@@QEAAPEAIPEAI0@Z 000000003159b7c0 f i CharacterManager.obj
 0001:0009a7c0       ?erase@?$_Impl_vector@U?$TCoeffBasis@M@spline@@V?$allocator@U?$TCoeffBasis@M@spline@@@stlpmtx_std@@@priv@stlpmtx_std@@QEAAPEAU?$TCoeffBasis@M@spline@@PEAU45@0@Z 000000003159b7c0 f i FaceEffector.obj
 0001:0009a7c0       ?erase@?$_Impl_vector@MV?$allocator@M@stlpmtx_std@@@priv@stlpmtx_std@@QEAAPEAMPEAM0@Z 000000003159b7c0 f i FaceAnimation.obj
 0001:0009a7c0       ?erase@?$_Impl_vector@UPhoneme@IFacialSentence@@V?$allocator@UPhoneme@IFacialSentence@@@stlpmtx_std@@@priv@stlpmtx_std@@QEAAPEAUPhoneme@IFacialSentence@@PEAU45@0@Z 000000003159b7c0 f i LipSync.obj
 0001:0009a7c0       ?erase@?$_Impl_vector@USOp@COperatorQueue@@V?$allocator@USOp@COperatorQueue@@@stlpmtx_std@@@priv@stlpmtx_std@@QEAAPEAUSOp@COperatorQueue@@PEAU45@0@Z 000000003159b7c0 f i OperatorQueue.obj
 0001:0009a840       ?_M_fill_insert_aux@?$_Impl_vector@U?$TCoeffBasis@M@spline@@V?$allocator@U?$TCoeffBasis@M@spline@@@stlpmtx_std@@@priv@stlpmtx_std@@AEAAXPEAU?$TCoeffBasis@M@spline@@_KAEBU45@AEBU__false_type@3@@Z 000000003159b840 f i FaceEffector.obj
 0001:0009a840       ?_M_fill_insert_aux@?$_Impl_vector@UBalanceChannelEntry@CFacialAnimSequenceInstance@@V?$allocator@UBalanceChannelEntry@CFacialAnimSequenceInstance@@@stlpmtx_std@@@priv@stlpmtx_std@@AEAAXPEAUBalanceChannelEntry@CFacialAnimSequenceInstance@@_KAEBU45@AEBU__false_type@3@@Z 000000003159b840 f i FaceAnimSequence.obj
 0001:0009a9f0       ??_G?$CatmullRomSpline@MU?$SplineKey@M@spline@@$0A@@spline@@UEAAPEAXI@Z 000000003159b9f0 f i FaceEffector.obj
 0001:0009a9f0       ??_E?$CatmullRomSpline@MU?$SplineKey@M@spline@@$0A@@spline@@UEAAPEAXI@Z 000000003159b9f0 f i FaceEffector.obj
 0001:0009aa20       ?comp_deriv@?$CatmullRomSpline@MU?$SplineKey@M@spline@@$0A@@spline@@MEAAXXZ 000000003159ba20 f i FaceEffector.obj
 0001:0009abe0       ??0?$CBaseSplineInterpolator@MV?$CatmullRomSpline@MU?$SplineKey@M@spline@@$0A@@spline@@@spline@@QEAA@XZ 000000003159bbe0 f i FaceEffector.obj
 0001:0009ac60       ?GetNumDimensions@CFacialEffCtrlSplineInterpolator@@UEAAHXZ 000000003159bc60 f i FaceEffector.obj
 0001:0009ac60       ?GetType@CFacialEffectorExpression@@UEAA?AW4EFacialEffectorType@@XZ 000000003159bc60 f i FaceEffectorLibrary.obj
 0001:0009ac60       ?GetAttachmentType@CCGFAttachment@@UEAA?AW4EType@IAttachmentObject@@XZ 000000003159bc60 f i AttachmentManager.obj
 0001:0009ac60       ?GetSplineType@CFacialEffCtrl@@UEAA?AW4ESplineType@@XZ 000000003159bc60 f i FaceEffector.obj
 0001:0009ac60       ?GetFormat@?$CKeyTimesInformation@GUUINT16Encoder@@@@UEAAIXZ 000000003159bc60 f i ControllerPQ.obj
 0001:0009ac60       ?GetSplineType@?$CBaseSplineInterpolator@MV?$CatmullRomSpline@MU?$SplineKey@M@spline@@$0A@@spline@@@spline@@UEAA?AW4ESplineType@@XZ 000000003159bc60 f i FaceEffector.obj
 0001:0009ac60       ?GetNumDimensions@?$CBaseSplineInterpolator@MV?$CatmullRomSpline@MU?$SplineKey@M@spline@@$0A@@spline@@@spline@@UEAAHXZ 000000003159bc60 f i FaceEffector.obj
 0001:0009ac60       ?GetNumDimensions@CFacialAnimChannelInterpolator@@UEAAHXZ 000000003159bc60 f i FaceAnimSequence.obj
 0001:0009ac60       ?GetFormat@?$CTrackDataStorageInt@U?$Quat_tpl@M@@UNoCompressQuat@@VITrackRotationStorage@@@@UEAAIXZ 000000003159bc60 f i ControllerPQ.obj
 0001:0009ac60       ?GetType@CAttachmentFACE@@UEBAIXZ 000000003159bc60 f i AttachmentManager.obj
 0001:0009ac70       ?GetKeyTime@?$CBaseSplineInterpolator@MV?$HermitSplineEx@MU?$SplineKey@M@spline@@@spline@@@spline@@UEAAMH@Z 000000003159bc70 f i FaceAnimSequence.obj
 0001:0009ac70       ?GetKeyTime@?$CBaseSplineInterpolator@MV?$CatmullRomSpline@MU?$SplineKey@M@spline@@$0A@@spline@@@spline@@UEAAMH@Z 000000003159bc70 f i FaceEffector.obj
 0001:0009aca0       ?SetKeyValue@?$CBaseSplineInterpolator@MV?$CatmullRomSpline@MU?$SplineKey@M@spline@@$0A@@spline@@@spline@@UEAAXHQEAM@Z 000000003159bca0 f i FaceEffector.obj
 0001:0009aca0       ?SetKeyValue@?$CBaseSplineInterpolator@MV?$HermitSplineEx@MU?$SplineKey@M@spline@@@spline@@@spline@@UEAAXHQEAM@Z 000000003159bca0 f i FaceAnimSequence.obj
 0001:0009acd0       ?SetKeyTime@?$CBaseSplineInterpolator@MV?$HermitSplineEx@MU?$SplineKey@M@spline@@@spline@@@spline@@UEAAXHM@Z 000000003159bcd0 f i FaceAnimSequence.obj
 0001:0009acd0       ?SetKeyTime@?$CBaseSplineInterpolator@MV?$CatmullRomSpline@MU?$SplineKey@M@spline@@$0A@@spline@@@spline@@UEAAXHM@Z 000000003159bcd0 f i FaceEffector.obj
 0001:0009ad00       ?SetKeyInTangent@?$CBaseSplineInterpolator@MV?$HermitSplineEx@MU?$SplineKey@M@spline@@@spline@@@spline@@UEAAXHQEAM@Z 000000003159bd00 f i FaceAnimSequence.obj
 0001:0009ad00       ?SetKeyInTangent@?$CBaseSplineInterpolator@MV?$CatmullRomSpline@MU?$SplineKey@M@spline@@$0A@@spline@@@spline@@UEAAXHQEAM@Z 000000003159bd00 f i FaceEffector.obj
 0001:0009ad30       ?SetKeyTangents@?$CBaseSplineInterpolator@MV?$CatmullRomSpline@MU?$SplineKey@M@spline@@$0A@@spline@@@spline@@UEAAXHQEAM0@Z 000000003159bd30 f i FaceEffector.obj
 0001:0009ad30       ?SetKeyTangents@?$CBaseSplineInterpolator@MV?$HermitSplineEx@MU?$SplineKey@M@spline@@@spline@@@spline@@UEAAXHQEAM0@Z 000000003159bd30 f i FaceAnimSequence.obj
 0001:0009ad70       ?SetKeyFlags@?$CBaseSplineInterpolator@MV?$CatmullRomSpline@MU?$SplineKey@M@spline@@$0A@@spline@@@spline@@UEAAXHH@Z 000000003159bd70 f i FaceEffector.obj
 0001:0009ad70       ?SetKeyFlags@?$CBaseSplineInterpolator@MV?$HermitSplineEx@MU?$SplineKey@M@spline@@@spline@@@spline@@UEAAXHH@Z 000000003159bd70 f i FaceAnimSequence.obj
 0001:0009ada0       ??0?$_Vector_base@U?$TCoeffBasis@M@spline@@V?$allocator@U?$TCoeffBasis@M@spline@@@stlpmtx_std@@@priv@stlpmtx_std@@QEAA@_KAEBV?$allocator@U?$TCoeffBasis@M@spline@@@2@@Z 000000003159bda0 f i FaceEffector.obj
 0001:0009ada0       ??0?$_Vector_base@UPhoneme@IFacialSentence@@V?$allocator@UPhoneme@IFacialSentence@@@stlpmtx_std@@@priv@stlpmtx_std@@QEAA@_KAEBV?$allocator@UPhoneme@IFacialSentence@@@2@@Z 000000003159bda0 f i LipSync.obj
 0001:0009ae70       ??0?$_Impl_vector@U?$TCoeffBasis@M@spline@@V?$allocator@U?$TCoeffBasis@M@spline@@@stlpmtx_std@@@priv@stlpmtx_std@@QEAA@AEBV012@@Z 000000003159be70 f i FaceEffector.obj
 0001:0009ae70       ??0?$_Impl_vector@UPhoneme@IFacialSentence@@V?$allocator@UPhoneme@IFacialSentence@@@stlpmtx_std@@@priv@stlpmtx_std@@QEAA@AEBV012@@Z 000000003159be70 f i LipSync.obj
 0001:0009aef0       ?RemoveKey@?$CBaseSplineInterpolator@MV?$HermitSplineEx@MU?$SplineKey@M@spline@@@spline@@@spline@@UEAAXH@Z 000000003159bef0 f i FaceAnimSequence.obj
 0001:0009aef0       ?RemoveKey@?$CBaseSplineInterpolator@MV?$CatmullRomSpline@MU?$SplineKey@M@spline@@$0A@@spline@@@spline@@UEAAXH@Z 000000003159bef0 f i FaceEffector.obj
 0001:0009af40       ?RemoveKeysInRange@?$CBaseSplineInterpolator@MV?$CatmullRomSpline@MU?$SplineKey@M@spline@@$0A@@spline@@@spline@@UEAAXMM@Z 000000003159bf40 f i FaceEffector.obj
 0001:0009af40       ?RemoveKeysInRange@?$CBaseSplineInterpolator@MV?$HermitSplineEx@MU?$SplineKey@M@spline@@@spline@@@spline@@UEAAXMM@Z 000000003159bf40 f i FaceAnimSequence.obj
 0001:0009b0a0       ?InsertKey@?$CBaseSplineInterpolator@MV?$CatmullRomSpline@MU?$SplineKey@M@spline@@$0A@@spline@@@spline@@UEAAHMQEAM@Z 000000003159c0a0 f i FaceEffector.obj
 0001:0009b0a0       ?InsertKey@?$CBaseSplineInterpolator@MV?$HermitSplineEx@MU?$SplineKey@M@spline@@@spline@@@spline@@UEAAHMQEAM@Z 000000003159c0a0 f i FaceAnimSequence.obj
 0001:0009b2a0       ??4?$TSpline@U?$SplineKey@M@spline@@VHermitBasis@2@@spline@@QEAAAEAV01@AEBV01@@Z 000000003159c2a0 f i FaceAnimSequence.obj
 0001:0009b2a0       ??4?$TSpline@U?$SplineKey@M@spline@@U?$TCoeffBasis@M@2@@spline@@QEAAAEAV01@AEBV01@@Z 000000003159c2a0 f i FaceEffector.obj
 0001:0009b320       ??0?$CatmullRomSpline@MU?$SplineKey@M@spline@@$0A@@spline@@QEAA@AEBV01@@Z 000000003159c320 f i FaceEffector.obj
 0001:0009b390       ?AddRef@?$SSplineBackup@V?$CatmullRomSpline@MU?$SplineKey@M@spline@@$0A@@spline@@@spline@@UEAAXXZ 000000003159c390 f i FaceEffector.obj
 0001:0009b3a0       ?Release@?$SSplineBackup@V?$CatmullRomSpline@MU?$SplineKey@M@spline@@$0A@@spline@@@spline@@UEAAXXZ 000000003159c3a0 f i FaceEffector.obj
 0001:0009b3c0       ??_E?$SSplineBackup@V?$CatmullRomSpline@MU?$SplineKey@M@spline@@$0A@@spline@@@spline@@W7EAAPEAXI@Z 000000003159c3c0 f i FaceEffector.obj
 0001:0009b3d0       ??_G?$SSplineBackup@V?$CatmullRomSpline@MU?$SplineKey@M@spline@@$0A@@spline@@@spline@@UEAAPEAXI@Z 000000003159c3d0 f i FaceEffector.obj
 0001:0009b3d0       ??_E?$SSplineBackup@V?$CatmullRomSpline@MU?$SplineKey@M@spline@@$0A@@spline@@@spline@@UEAAPEAXI@Z 000000003159c3d0 f i FaceEffector.obj
 0001:0009b410       ?Backup@?$CBaseSplineInterpolator@MV?$CatmullRomSpline@MU?$SplineKey@M@spline@@$0A@@spline@@@spline@@UEAAPEAUISplineBackup@@XZ 000000003159c410 f i FaceEffector.obj
 0001:0009b490       ?Restore@?$CBaseSplineInterpolator@MV?$CatmullRomSpline@MU?$SplineKey@M@spline@@$0A@@spline@@@spline@@UEAAXPEAUISplineBackup@@@Z 000000003159c490 f i FaceEffector.obj
 0001:0009b4e0       ??0CFacialEffCtrlSplineInterpolator@@QEAA@PEAVCFacialEffCtrl@@@Z 000000003159c4e0 f i FaceEffector.obj
 0001:0009b520       ??_E?$CBaseSplineInterpolator@MV?$CatmullRomSpline@MU?$SplineKey@M@spline@@$0A@@spline@@@spline@@W7EAAPEAXI@Z 000000003159c520 f i FaceEffector.obj
 0001:0009b520       ??_ECFacialEffCtrlSplineInterpolator@@W7EAAPEAXI@Z 000000003159c520 f i FaceEffector.obj
 0001:0009b530       ??_ECFacialEffCtrlSplineInterpolator@@UEAAPEAXI@Z 000000003159c530 f i FaceEffector.obj
 0001:0009b530       ??_E?$CBaseSplineInterpolator@MV?$CatmullRomSpline@MU?$SplineKey@M@spline@@$0A@@spline@@@spline@@UEAAPEAXI@Z 000000003159c530 f i FaceEffector.obj
 0001:0009b530       ??_G?$CBaseSplineInterpolator@MV?$CatmullRomSpline@MU?$SplineKey@M@spline@@$0A@@spline@@@spline@@UEAAPEAXI@Z 000000003159c530 f i FaceEffector.obj
 0001:0009b530       ??_GCFacialEffCtrlSplineInterpolator@@UEAAPEAXI@Z 000000003159c530 f i FaceEffector.obj
 0001:0009b570       ?SetType@CFacialEffCtrl@@UEAAXW4ControlType@IFacialEffCtrl@@@Z 000000003159c570 f   FaceEffector.obj
 0001:0009b690       ?SetConstantWeight@CFacialEffCtrl@@UEAAXM@Z 000000003159c690 f   FaceEffector.obj
 0001:0009b780       ??0CFacialEffCtrl@@QEAA@XZ 000000003159c780 f   FaceEffector.obj
 0001:0009b840       ?GetFlags@CFacialAnimChannel@@UEAAIXZ 000000003159c840 f i FaceAnimSequence.obj
 0001:0009b840       ?GetType@CFacialEffCtrl@@UEAA?AW4ControlType@IFacialEffCtrl@@XZ 000000003159c840 f i FaceEffector.obj
 0001:0009b840       ?GetNameCRC@CAttachmentFACE@@UEBAIXZ 000000003159c840 f i AttachmentManager.obj
 0001:0009b840       ?GetNameCRC@CAttachmentBONE@@UEBAIXZ 000000003159c840 f i AttachmentManager.obj
 0001:0009b840       ?GetNameCRC@CAttachmentSKIN@@UEBAIXZ 000000003159c840 f i Attachment.obj
 0001:0009b850       ?GetVideoMarkerScale@CFacialJoystickChannel@@UEBAMXZ 000000003159c850 f i FaceJoystick.obj
 0001:0009b850       ?GetConstantBalance@CFacialEffCtrl@@UEAAMXZ 000000003159c850 f i FaceEffector.obj
 0001:0009b860       ?GetFlags@CFacialEffCtrl@@UEAAHXZ 000000003159c860 f i FaceEffector.obj
 0001:0009b870       ?SetFlags@CFacialEffCtrl@@UEAAXH@Z 000000003159c870 f i FaceEffector.obj
 0001:0009b880       ?SerializeSpline@CFacialEffCtrl@@UEAAXAEAVXmlNodeRef@@_N@Z 000000003159c880 f i FaceEffector.obj
 0001:0009b8a0       ??_ECFacialEffCtrl@@W7EAAPEAXI@Z 000000003159c8a0 f i FaceEffector.obj
 0001:0009b8b0       ??_GCFacialEffCtrl@@UEAAPEAXI@Z 000000003159c8b0 f i FaceEffector.obj
 0001:0009b8b0       ??_ECFacialEffCtrl@@UEAAPEAXI@Z 000000003159c8b0 f i FaceEffector.obj
 0001:0009b930       ?AddSubEffector@CFacialEffector@@UEAAPEAUIFacialEffCtrl@@PEAUIFacialEffector@@@Z 000000003159c930 f   FaceEffector.obj
 0001:0009bb30       ?interpolate@?$TSpline@U?$SplineKey@M@spline@@U?$TCoeffBasis@M@2@@spline@@QEAA_NMAEAM@Z 000000003159cb30 f i FaceEffector.obj
 0001:0009bb30       ?interpolate@?$TSpline@U?$SplineKey@M@spline@@VHermitBasis@2@@spline@@QEAA_NMAEAM@Z 000000003159cb30 f i FaceAnimSequence.obj
 0001:0009bc80       ?Evaluate@CFacialEffCtrl@@UEAAMM@Z 000000003159cc80 f   FaceEffector.obj
 0001:0009bcd0       ?Interpolate@?$CBaseSplineInterpolator@MV?$CatmullRomSpline@MU?$SplineKey@M@spline@@$0A@@spline@@@spline@@UEAAXMAEAY03M@Z 000000003159ccd0 f i FaceEffector.obj
 0001:0009bd00       ?EffectorTypeToName@@YAPEBDW4EFacialEffectorType@@@Z 000000003159cd00 f i FaceEffectorLibrary.obj
 0001:0009bd70       ?NameToEffectorType@@YA?AW4EFacialEffectorType@@PEBD@Z 000000003159cd70 f i FaceEffectorLibrary.obj
 0001:0009c070       ?Find@CFacialEffectorsLibrary@@UEAAPEAUIFacialEffector@@PEBD@Z 000000003159d070 f   FaceEffectorLibrary.obj
 0001:0009c0c0       ?GetRoot@CFacialEffectorsLibrary@@UEAAPEAUIFacialEffector@@XZ 000000003159d0c0 f   FaceEffectorLibrary.obj
 0001:0009c0d0       ?CreateEffector@CFacialEffectorsLibrary@@UEAAPEAUIFacialEffector@@W4EFacialEffectorType@@PEBD@Z 000000003159d0d0 f   FaceEffectorLibrary.obj
 0001:0009c1f0       ??$fill@PEAV?$_smart_ptr@VCFacialEffector@@@@V1@@stlpmtx_std@@YAXPEAV?$_smart_ptr@VCFacialEffector@@@@0AEBV1@@Z 000000003159d1f0 f i FaceEffectorLibrary.obj
 0001:0009c260       ??$AddObject@V?$_smart_ptr@VCFacialEffector@@@@V?$allocator@V?$_smart_ptr@VCFacialEffector@@@@@stlpmtx_std@@@ICrySizer@@QEAAXAEBV?$vector@V?$_smart_ptr@VCFacialEffector@@@@V?$allocator@V?$_smart_ptr@VCFacialEffector@@@@@stlpmtx_std@@@stlpmtx_std@@@Z 000000003159d260 f i FaceEffectorLibrary.obj
 0001:0009c2f0       ?VisitEffectors@CFacialEffectorsLibrary@@UEAAXPEAUIFacialEffectorsLibraryEffectorVisitor@@@Z 000000003159d2f0 f   FaceEffectorLibrary.obj
 0001:0009c390       ?GetEffectorFromIndex@CFacialEffectorsLibrary@@QEAAPEAVCFacialEffector@@H@Z 000000003159d390 f   FaceEffectorLibrary.obj
 0001:0009c3c0       ?SerializeEffectorSubCtrls@CFacialEffectorsLibrary@@AEAAXPEAVCFacialEffector@@AEAVXmlNodeRef@@_N@Z 000000003159d3c0 f   FaceEffectorLibrary.obj
 0001:0009c630       ?_M_erase@?$_Rb_tree@IU?$less@I@stlpmtx_std@@U?$pair@$$CBIV?$_smart_ptr@VCFacialEffector@@@@@2@U?$_Select1st@U?$pair@$$CBIV?$_smart_ptr@VCFacialEffector@@@@@stlpmtx_std@@@priv@2@U?$_MapTraitsT@U?$pair@$$CBIV?$_smart_ptr@VCFacialEffector@@@@@stlpmtx_std@@@52@V?$allocator@U?$pair@$$CBIV?$_smart_ptr@VCFacialEffector@@@@@stlpmtx_std@@@2@@priv@stlpmtx_std@@AEAAXPEAU_Rb_tree_node_base@23@@Z 000000003159d630 f i FaceEffectorLibrary.obj
 0001:0009c6a0       ??$AddObject@IV?$_smart_ptr@VCFacialEffector@@@@U?$less@I@stlpmtx_std@@V?$allocator@U?$pair@$$CBIV?$_smart_ptr@VCFacialEffector@@@@@stlpmtx_std@@@3@@ICrySizer@@QEAAXAEBV?$map@IV?$_smart_ptr@VCFacialEffector@@@@U?$less@I@stlpmtx_std@@V?$allocator@U?$pair@$$CBIV?$_smart_ptr@VCFacialEffector@@@@@stlpmtx_std@@@3@@stlpmtx_std@@@Z 000000003159d6a0 f i FaceEffectorLibrary.obj
 0001:0009c770       ?_M_create_node@?$_Rb_tree@_JU?$less@_J@stlpmtx_std@@U?$pair@$$CB_JPEAUphys_geometry@@@2@U?$_Select1st@U?$pair@$$CB_JPEAUphys_geometry@@@stlpmtx_std@@@priv@2@U?$_MapTraitsT@U?$pair@$$CB_JPEAUphys_geometry@@@stlpmtx_std@@@52@V?$allocator@U?$pair@$$CB_JPEAUphys_geometry@@@stlpmtx_std@@@2@@priv@stlpmtx_std@@IEAAPEAU_Rb_tree_node_base@23@AEBU?$pair@$$CB_JPEAUphys_geometry@@@3@@Z 000000003159d770 f i LoaderCHR.obj
 0001:0009c770       ?_M_create_node@?$_Rb_tree@PEAUIFacialEffector@@U?$less@PEAUIFacialEffector@@@stlpmtx_std@@U?$pair@QEAUIFacialEffector@@PEAU1@@3@U?$_Select1st@U?$pair@QEAUIFacialEffector@@PEAU1@@stlpmtx_std@@@priv@3@U?$_MapTraitsT@U?$pair@QEAUIFacialEffector@@PEAU1@@stlpmtx_std@@@63@V?$allocator@U?$pair@QEAUIFacialEffector@@PEAU1@@stlpmtx_std@@@3@@priv@stlpmtx_std@@IEAAPEAU_Rb_tree_node_base@23@AEBU?$pair@QEAUIFacialEffector@@PEAU1@@3@@Z 000000003159d770 f i FaceEffectorLibrary.obj
 0001:0009c7e0       ??$__uninitialized_fill_n@PEAV?$_smart_ptr@VCFacialEffector@@@@_KV1@@priv@stlpmtx_std@@YAPEAV?$_smart_ptr@VCFacialEffector@@@@PEAV2@_KAEBV2@@Z 000000003159d7e0 f i FaceEffectorLibrary.obj
 0001:0009c850       ?_M_create_node@?$_Rb_tree@IU?$less@I@stlpmtx_std@@U?$pair@$$CBIV?$_smart_ptr@VCFacialEffector@@@@@2@U?$_Select1st@U?$pair@$$CBIV?$_smart_ptr@VCFacialEffector@@@@@stlpmtx_std@@@priv@2@U?$_MapTraitsT@U?$pair@$$CBIV?$_smart_ptr@VCFacialEffector@@@@@stlpmtx_std@@@52@V?$allocator@U?$pair@$$CBIV?$_smart_ptr@VCFacialEffector@@@@@stlpmtx_std@@@2@@priv@stlpmtx_std@@IEAAPEAU_Rb_tree_node_base@23@AEBU?$pair@$$CBIV?$_smart_ptr@VCFacialEffector@@@@@3@@Z 000000003159d850 f i FaceEffectorLibrary.obj
 0001:0009c8d0       ?SetIdentifierByLibrary@CFacialEffector@@QEAAXVCFaceIdentifierHandle@@@Z 000000003159d8d0 f i FaceEffectorLibrary.obj
 0001:0009c9f0       ?GetMemoryUsage@CFacialEffectorsLibrary@@QEBAXPEAVICrySizer@@@Z 000000003159d9f0 f   FaceEffectorLibrary.obj
 0001:0009ca80       ?erase@?$map@IV?$_smart_ptr@VCFacialEffector@@@@U?$less@I@stlpmtx_std@@V?$allocator@U?$pair@$$CBIV?$_smart_ptr@VCFacialEffector@@@@@stlpmtx_std@@@3@@stlpmtx_std@@QEAAXU?$_Rb_tree_iterator@U?$pair@$$CBIV?$_smart_ptr@VCFacialEffector@@@@@stlpmtx_std@@U?$_MapTraitsT@U?$pair@$$CBIV?$_smart_ptr@VCFacialEffector@@@@@stlpmtx_std@@@priv@2@@priv@2@@Z 000000003159da80 f i FaceEffectorLibrary.obj
 0001:0009cae0       ?_M_fill_insert_aux@?$_Impl_vector@V?$_smart_ptr@VCFacialEffector@@@@V?$allocator@V?$_smart_ptr@VCFacialEffector@@@@@stlpmtx_std@@@priv@stlpmtx_std@@AEAAXPEAV?$_smart_ptr@VCFacialEffector@@@@_KAEBV4@AEBU__false_type@3@@Z 000000003159dae0 f i FaceEffectorLibrary.obj
 0001:0009cd40       ?_M_insert@?$_Rb_tree@IU?$less@I@stlpmtx_std@@U?$pair@$$CBIV?$_smart_ptr@VCFacialEffector@@@@@2@U?$_Select1st@U?$pair@$$CBIV?$_smart_ptr@VCFacialEffector@@@@@stlpmtx_std@@@priv@2@U?$_MapTraitsT@U?$pair@$$CBIV?$_smart_ptr@VCFacialEffector@@@@@stlpmtx_std@@@52@V?$allocator@U?$pair@$$CBIV?$_smart_ptr@VCFacialEffector@@@@@stlpmtx_std@@@2@@priv@stlpmtx_std@@AEAA?AU?$_Rb_tree_iterator@U?$pair@$$CBIV?$_smart_ptr@VCFacialEffector@@@@@stlpmtx_std@@U?$_MapTraitsT@U?$pair@$$CBIV?$_smart_ptr@VCFacialEffector@@@@@stlpmtx_std@@@priv@2@@23@PEAU_Rb_tree_node_base@23@AEBU?$pair@$$CBIV?$_smart_ptr@VCFacialEffector@@@@@3@00@Z 000000003159dd40 f i FaceEffectorLibrary.obj
 0001:0009ce00       ?insert_unique@?$_Rb_tree@IU?$less@I@stlpmtx_std@@U?$pair@$$CBIV?$_smart_ptr@VCFacialEffector@@@@@2@U?$_Select1st@U?$pair@$$CBIV?$_smart_ptr@VCFacialEffector@@@@@stlpmtx_std@@@priv@2@U?$_MapTraitsT@U?$pair@$$CBIV?$_smart_ptr@VCFacialEffector@@@@@stlpmtx_std@@@52@V?$allocator@U?$pair@$$CBIV?$_smart_ptr@VCFacialEffector@@@@@stlpmtx_std@@@2@@priv@stlpmtx_std@@QEAA?AU?$pair@U?$_Rb_tree_iterator@U?$pair@$$CBIV?$_smart_ptr@VCFacialEffector@@@@@stlpmtx_std@@U?$_MapTraitsT@U?$pair@$$CBIV?$_smart_ptr@VCFacialEffector@@@@@stlpmtx_std@@@priv@2@@priv@stlpmtx_std@@_N@3@AEBU?$pair@$$CBIV?$_smart_ptr@VCFacialEffector@@@@@3@@Z 000000003159de00 f i FaceEffectorLibrary.obj
 0001:0009d000       ?Find@CFacialEffectorsLibrary@@UEAAPEAUIFacialEffector@@VCFaceIdentifierHandle@@@Z 000000003159e000 f   FaceEffectorLibrary.obj
 0001:0009d090       ?RemoveEffector@CFacialEffectorsLibrary@@UEAAXPEAUIFacialEffector@@@Z 000000003159e090 f   FaceEffectorLibrary.obj
 0001:0009d240       ?ReplaceEffector@CFacialEffectorsLibrary@@AEAAXPEAVCFacialEffector@@0@Z 000000003159e240 f   FaceEffectorLibrary.obj
 0001:0009d3c0       ?insert_unique@?$_Rb_tree@PEAUIFacialEffector@@U?$less@PEAUIFacialEffector@@@stlpmtx_std@@U?$pair@QEAUIFacialEffector@@PEAU1@@3@U?$_Select1st@U?$pair@QEAUIFacialEffector@@PEAU1@@stlpmtx_std@@@priv@3@U?$_MapTraitsT@U?$pair@QEAUIFacialEffector@@PEAU1@@stlpmtx_std@@@63@V?$allocator@U?$pair@QEAUIFacialEffector@@PEAU1@@stlpmtx_std@@@3@@priv@stlpmtx_std@@QEAA?AU?$pair@U?$_Rb_tree_iterator@U?$pair@QEAUIFacialEffector@@PEAU1@@stlpmtx_std@@U?$_MapTraitsT@U?$pair@QEAUIFacialEffector@@PEAU1@@stlpmtx_std@@@priv@2@@priv@stlpmtx_std@@_N@3@AEBU?$pair@QEAUIFacialEffector@@PEAU1@@3@@Z 000000003159e3c0 f i FaceEffectorLibrary.obj
 0001:0009d5c0       ?insert_unique@?$_Rb_tree@IU?$less@I@stlpmtx_std@@U?$pair@$$CBIV?$_smart_ptr@VCFacialEffector@@@@@2@U?$_Select1st@U?$pair@$$CBIV?$_smart_ptr@VCFacialEffector@@@@@stlpmtx_std@@@priv@2@U?$_MapTraitsT@U?$pair@$$CBIV?$_smart_ptr@VCFacialEffector@@@@@stlpmtx_std@@@52@V?$allocator@U?$pair@$$CBIV?$_smart_ptr@VCFacialEffector@@@@@stlpmtx_std@@@2@@priv@stlpmtx_std@@QEAA?AU?$_Rb_tree_iterator@U?$pair@$$CBIV?$_smart_ptr@VCFacialEffector@@@@@stlpmtx_std@@U?$_MapTraitsT@U?$pair@$$CBIV?$_smart_ptr@VCFacialEffector@@@@@stlpmtx_std@@@priv@2@@23@U423@AEBU?$pair@$$CBIV?$_smart_ptr@VCFacialEffector@@@@@3@@Z 000000003159e5c0 f i FaceEffectorLibrary.obj
 0001:0009da00       ??$_M_allocate_and_copy@PEAV?$_smart_ptr@VCFacialEffector@@@@@?$_Impl_vector@V?$_smart_ptr@VCFacialEffector@@@@V?$allocator@V?$_smart_ptr@VCFacialEffector@@@@@stlpmtx_std@@@priv@stlpmtx_std@@AEAAPEAV?$_smart_ptr@VCFacialEffector@@@@AEA_KPEAV3@1@Z 000000003159ea00 f i FaceEffectorLibrary.obj
 0001:0009dad0       ?_M_insert_overflow_aux@?$_Impl_vector@V?$_smart_ptr@VCFacialEffector@@@@V?$allocator@V?$_smart_ptr@VCFacialEffector@@@@@stlpmtx_std@@@priv@stlpmtx_std@@AEAAXPEAV?$_smart_ptr@VCFacialEffector@@@@AEBV4@AEBU__false_type@3@_K_N@Z 000000003159ead0 f i FaceEffectorLibrary.obj
 0001:0009dcb0       ??1CFacialEffectorsLibrary@@UEAA@XZ 000000003159ecb0 f   FaceEffectorLibrary.obj
 0001:0009dd70       ?Release@CFacialEffectorsLibrary@@UEAAXXZ 000000003159ed70 f i FaceEffectorLibrary.obj
 0001:0009e1b0       ??0CFacialMorphTarget@@QEAA@I@Z 000000003159f1b0 f i FaceEffectorLibrary.obj
 0001:0009e1f0       ??_ECFacialEffector@@W7EAAPEAXI@Z 000000003159f1f0 f i FaceEffector.obj
 0001:0009e1f0       ??_ECFacialMorphTarget@@W7EAAPEAXI@Z 000000003159f1f0 f i FaceEffectorLibrary.obj
 0001:0009e1f0       ??_ECFacialEffectorExpression@@W7EAAPEAXI@Z 000000003159f1f0 f i FaceEffectorLibrary.obj
 0001:0009e200       ??_GCFacialMorphTarget@@UEAAPEAXI@Z 000000003159f200 f i FaceEffectorLibrary.obj
 0001:0009e200       ??_ECFacialEffector@@UEAAPEAXI@Z 000000003159f200 f i FaceEffector.obj
 0001:0009e200       ??_ECFacialMorphTarget@@UEAAPEAXI@Z 000000003159f200 f i FaceEffectorLibrary.obj
 0001:0009e200       ??_GCFacialEffector@@UEAAPEAXI@Z 000000003159f200 f i FaceEffector.obj
 0001:0009e200       ??_ECFacialEffectorExpression@@UEAAPEAXI@Z 000000003159f200 f i FaceEffectorLibrary.obj
 0001:0009e200       ??_GCFacialEffectorExpression@@UEAAPEAXI@Z 000000003159f200 f i FaceEffectorLibrary.obj
 0001:0009e280       ??_ECFacialEffectorsLibrary@@UEAAPEAXI@Z 000000003159f280 f i FaceEffectorLibrary.obj
 0001:0009e280       ??_GCFacialEffectorsLibrary@@UEAAPEAXI@Z 000000003159f280 f i FaceEffectorLibrary.obj
 0001:0009e2b0       ?NewRoot@CFacialEffectorsLibrary@@AEAAXXZ 000000003159f2b0 f   FaceEffectorLibrary.obj
 0001:0009e410       ??0CFacialEffectorExpression@@QEAA@XZ 000000003159f410 f i FaceEffectorLibrary.obj
 0001:0009e440       ??0CFacialEffectorBone@@QEAA@XZ 000000003159f440 f i FaceEffectorLibrary.obj
 0001:0009e470       ?RenameEffector@CFacialEffectorsLibrary@@QEAAXPEAVCFacialEffector@@VCFaceIdentifierHandle@@@Z 000000003159f470 f   FaceEffectorLibrary.obj
 0001:0009e5e0       ?SerializeEffectorSelf@CFacialEffectorsLibrary@@AEAAXPEAVCFacialEffector@@AEAVXmlNodeRef@@_N@Z 000000003159f5e0 f   FaceEffectorLibrary.obj
 0001:0009e750       ?SerializeEffector@CFacialEffectorsLibrary@@UEAAXPEAUIFacialEffector@@AEAVXmlNodeRef@@_N@Z 000000003159f750 f   FaceEffectorLibrary.obj
 0001:0009e7a0       ??0CFacialEffectorsLibrary@@QEAA@PEAVCFacialAnimation@@@Z 000000003159f7a0 f   FaceEffectorLibrary.obj
 0001:0009e900       ?MergeLibrary@CFacialEffectorsLibrary@@UEAAXPEAUIFacialEffectorsLibrary@@AEBV?$Functor1wRet@PEBDW4MergeCollisionAction@@@@@Z 000000003159f900 f   FaceEffectorLibrary.obj
 0001:0009e9e0       ?Serialize@CFacialEffectorsLibrary@@UEAAXAEAVXmlNodeRef@@_N@Z 000000003159f9e0 f   FaceEffectorLibrary.obj
 0001:0009eeb0       ?SetEffectorIndex@CFacialEffectorsLibrary@@AEAAXPEAVCFacialEffector@@@Z 000000003159feb0 f   FaceEffectorLibrary.obj
 0001:0009efa0       ?CreateEffector@CFacialEffectorsLibrary@@UEAAPEAUIFacialEffector@@W4EFacialEffectorType@@VCFaceIdentifierHandle@@@Z 000000003159ffa0 f   FaceEffectorLibrary.obj
 0001:0009f1b0       ??_GIJoystick@@UEAAPEAXI@Z 00000000315a01b0 f i FaceJoystick.obj
 0001:0009f1b0       ??_GIFacialEffectorsLibrary@@UEAAPEAXI@Z 00000000315a01b0 f i FaceEffectorLibrary.obj
 0001:0009f1b0       ??_GIJoystickChannel@@UEAAPEAXI@Z 00000000315a01b0 f i FaceJoystick.obj
 0001:0009f1b0       ??_EIJoystick@@UEAAPEAXI@Z 00000000315a01b0 f i FaceJoystick.obj
 0001:0009f1b0       ??_GIFacialAnimation@@UEAAPEAXI@Z 00000000315a01b0 f i FaceAnimation.obj
 0001:0009f1b0       ??_EIFacialEffectorsLibrary@@UEAAPEAXI@Z 00000000315a01b0 f i FaceEffectorLibrary.obj
 0001:0009f1b0       ??_EIFacialAnimation@@UEAAPEAXI@Z 00000000315a01b0 f i FaceAnimation.obj
 0001:0009f1b0       ??_EIJoystickChannel@@UEAAPEAXI@Z 00000000315a01b0 f i FaceJoystick.obj
 0001:0009f1e0       ?AddRef@CFacialJoystickChannel@@UEAAXXZ 00000000315a01e0 f   FaceJoystick.obj
 0001:0009f1f0       ?Release@CFacialJoystickChannel@@UEAAXXZ 00000000315a01f0 f   FaceJoystick.obj
 0001:0009f210       ?GetName@CFacialJoystickChannel@@UEBAPEBDXZ 00000000315a0210 f   FaceJoystick.obj
 0001:0009f240       ?GetSplineCount@CFacialJoystickChannel@@UEAAHXZ 00000000315a0240 f   FaceJoystick.obj
 0001:0009f260       ?GetSpline@CFacialJoystickChannel@@UEAAPEAUISplineInterpolator@@H@Z 00000000315a0260 f   FaceJoystick.obj
 0001:0009f2b0       ?SetFlipped@CFacialJoystickChannel@@UEAAX_N@Z 00000000315a02b0 f   FaceJoystick.obj
 0001:0009f2c0       ?GetFlipped@CFacialJoystickChannel@@UEBA_NXZ 00000000315a02c0 f   FaceJoystick.obj
 0001:0009f2d0       ?GetConstantWeight@CFacialEffCtrl@@UEAAMXZ 00000000315a02d0 f   FaceEffector.obj
 0001:0009f2d0       ?GetVideoMarkerOffset@CFacialJoystickChannel@@UEBAMXZ 00000000315a02d0 f   FaceJoystick.obj
 0001:0009f2e0       ?SetVideoMarkerScale@CFacialJoystickChannel@@UEAAXM@Z 00000000315a02e0 f   FaceJoystick.obj
 0001:0009f2e0       ?SetConstantBalance@CFacialEffCtrl@@UEAAXM@Z 00000000315a02e0 f   FaceEffector.obj
 0001:0009f2f0       ?CleanupKeys@CFacialJoystickChannel@@UEAAXM@Z 00000000315a02f0 f   FaceJoystick.obj
 0001:0009f310       ?AddRef@CFacialJoystick@@UEAAXXZ 00000000315a0310 f   FaceJoystick.obj
 0001:0009f320       ?Release@CFacialJoystick@@UEAAXXZ 00000000315a0320 f   FaceJoystick.obj
 0001:0009f340       ?GetCentre@CFacialJoystick@@UEBAAEBU?$Vec2_tpl@M@@XZ 00000000315a0340 f   FaceJoystick.obj
 0001:0009f350       ?GetDimensions@CFacialJoystick@@UEBAAEBU?$Vec2_tpl@M@@XZ 00000000315a0350 f   FaceJoystick.obj
 0001:0009f360       ?SetColor@CFacialJoystick@@UEAAXAEBU?$Vec3_tpl@E@@@Z 00000000315a0360 f   FaceJoystick.obj
 0001:0009f370       ?GetColor@CFacialJoystick@@UEBA?AU?$Vec3_tpl@E@@XZ 00000000315a0370 f   FaceJoystick.obj
 0001:0009f390       ?Release@CFacialJoystickSet@@UEAAXXZ 00000000315a0390 f   FaceJoystick.obj
 0001:0009f3b0       ??_9CFacialJoystick@@$BEI@AA 00000000315a03b0 f i FaceJoystick.obj
 0001:0009f3c0       ??_9CFacialJoystick@@$BFI@AA 00000000315a03c0 f i FaceJoystick.obj
 0001:0009f3d0       ??_9CFacialJoystick@@$BEA@AA 00000000315a03d0 f i FaceJoystick.obj
 0001:0009f3e0       ??_9CFacialJoystick@@$BFA@AA 00000000315a03e0 f i FaceJoystick.obj
 0001:0009f3f0       ?GetChannel@CFacialJoystick@@UEAAPEAVIJoystickChannel@@W4ChannelType@IJoystick@@@Z 00000000315a03f0 f   FaceJoystick.obj
 0001:0009f410       ?SetChannel@CFacialJoystick@@UEAAXW4ChannelType@IJoystick@@PEAVIJoystickChannel@@@Z 00000000315a0410 f   FaceJoystick.obj
 0001:0009f470       ?SetCentre@CFacialJoystick@@UEAAXAEBU?$Vec2_tpl@M@@@Z 00000000315a0470 f   FaceJoystick.obj
 0001:0009f480       ?SetDimensions@CFacialJoystick@@UEAAXAEBU?$Vec2_tpl@M@@@Z 00000000315a0480 f   FaceJoystick.obj
 0001:0009f490       ?GetName@CFacialJoystickSet@@UEBAPEBDXZ 00000000315a0490 f   FaceJoystick.obj
 0001:0009f490       ?GetSpline@CFacialEffCtrl@@UEAAPEAUISplineInterpolator@@XZ 00000000315a0490 f   FaceEffector.obj
 0001:0009f4a0       ?GetJoystickCount@CFacialJoystickSet@@UEBAHXZ 00000000315a04a0 f   FaceJoystick.obj
 0001:0009f4b0       ?GetJoystick@CFacialJoystickSet@@UEAAPEAVIJoystick@@H@Z 00000000315a04b0 f   FaceJoystick.obj
 0001:0009f4c0       ?GetJoystickAtPoint@CFacialJoystickSet@@UEAAPEAVIJoystick@@AEBU?$Vec2_tpl@M@@@Z 00000000315a04c0 f   FaceJoystick.obj
 0001:0009f580       ?GetJoystickByID@CFacialJoystickSet@@UEAAPEAVIJoystick@@_K@Z 00000000315a0580 f   FaceJoystick.obj
 0001:0009f5f0       ?Bind@CFacialJoystickSet@@QEAAXPEAVIFacialJoystickSerializeContext@@@Z 00000000315a05f0 f   FaceJoystick.obj
 0001:0009f6a0       ??0CFacialJoystick@@QEAA@_K@Z 00000000315a06a0 f   FaceJoystick.obj
 0001:0009f6e0       ??1CFacialJoystick@@UEAA@XZ 00000000315a06e0 f i FaceJoystick.obj
 0001:0009f770       ?_M_erase@?$_Impl_vector@V?$_smart_ptr@VCFacialJoystick@@@@V?$allocator@V?$_smart_ptr@VCFacialJoystick@@@@@stlpmtx_std@@@priv@stlpmtx_std@@AEAAPEAV?$_smart_ptr@VCFacialJoystick@@@@PEAV4@AEBU__false_type@3@@Z 00000000315a0770 f i FaceJoystick.obj
 0001:0009f840       ??$__uninitialized_fill_n@PEAV?$_smart_ptr@VCFacialJoystick@@@@_KV1@@priv@stlpmtx_std@@YAPEAV?$_smart_ptr@VCFacialJoystick@@@@PEAV2@_KAEBV2@@Z 00000000315a0840 f i FaceJoystick.obj
 0001:0009f8b0       ??_ECFacialJoystickChannel@@UEAAPEAXI@Z 00000000315a08b0 f i FaceJoystick.obj
 0001:0009f8b0       ??_GCFacialJoystickChannel@@UEAAPEAXI@Z 00000000315a08b0 f i FaceJoystick.obj
 0001:0009f920       ??_GCFacialJoystick@@UEAAPEAXI@Z 00000000315a0920 f i FaceJoystick.obj
 0001:0009f920       ??_ECFacialJoystick@@UEAAPEAXI@Z 00000000315a0920 f i FaceJoystick.obj
 0001:0009f950       ?SetJoystickFile@CFacialAnimSequence@@UEAAXPEBD@Z 00000000315a0950 f   FaceAnimSequence.obj
 0001:0009f950       ?SetName@CFacialJoystick@@UEAAXPEBD@Z 00000000315a0950 f   FaceJoystick.obj
 0001:0009f9a0       ?SetName@CFacialJoystickSet@@UEAAXPEBD@Z 00000000315a09a0 f   FaceJoystick.obj
 0001:0009f9f0       ?_M_erase@?$_Impl_vector@V?$_smart_ptr@VCFacialJoystick@@@@V?$allocator@V?$_smart_ptr@VCFacialJoystick@@@@@stlpmtx_std@@@priv@stlpmtx_std@@AEAAPEAV?$_smart_ptr@VCFacialJoystick@@@@PEAV4@0AEBU__false_type@3@@Z 00000000315a09f0 f i FaceJoystick.obj
 0001:0009fad0       ??0CFacialJoystickChannel@@QEAA@PEAUIFacialAnimChannel@@@Z 00000000315a0ad0 f   FaceJoystick.obj
 0001:000a0010       ?RemoveJoystick@CFacialJoystickSet@@UEAAXPEAVIJoystick@@@Z 00000000315a1010 f   FaceJoystick.obj
 0001:000a00b0       ??1?$_Impl_vector@V?$_smart_ptr@VCFacialJoystick@@@@V?$allocator@V?$_smart_ptr@VCFacialJoystick@@@@@stlpmtx_std@@@priv@stlpmtx_std@@QEAA@XZ 00000000315a10b0 f i FaceJoystick.obj
 0001:000a0120       ?_M_insert_overflow_aux@?$_Impl_vector@V?$_smart_ptr@VCFacialJoystick@@@@V?$allocator@V?$_smart_ptr@VCFacialJoystick@@@@@stlpmtx_std@@@priv@stlpmtx_std@@AEAAXPEAV?$_smart_ptr@VCFacialJoystick@@@@AEBV4@AEBU__false_type@3@_K_N@Z 00000000315a1120 f i FaceJoystick.obj
 0001:000a0310       ??0CFacialJoystickSet@@QEAA@XZ 00000000315a1310 f   FaceJoystick.obj
 0001:000a0380       ??_ECFacialJoystickSet@@UEAAPEAXI@Z 00000000315a1380 f i FaceJoystick.obj
 0001:000a0380       ??_GCFacialJoystickSet@@UEAAPEAXI@Z 00000000315a1380 f i FaceJoystick.obj
 0001:000a03f0       ?AddJoystick@CFacialJoystickSet@@UEAAXPEAVIJoystick@@@Z 00000000315a13f0 f   FaceJoystick.obj
 0001:000a0490       ?Serialize@CFacialJoystickSet@@UEAAXAEAVXmlNodeRef@@_N@Z 00000000315a1490 f   FaceJoystick.obj
 0001:000a10a0       ?Reset@CFaceState@@QEAAXXZ 00000000315a20a0 f   FaceState.obj
 0001:000a10f0       ?SetNumWeights@CFaceState@@QEAAXH@Z 00000000315a20f0 f   FaceState.obj
 0001:000a1280       ??_EIAttachmentManager@@UEAAPEAXI@Z 00000000315a2280 f i CharacterInstance.obj
 0001:000a1280       ??_EIFacialInstance@@UEAAPEAXI@Z 00000000315a2280 f i FacialInstance.obj
 0001:000a1280       ??_GIFacialInstance@@UEAAPEAXI@Z 00000000315a2280 f i FacialInstance.obj
 0001:000a1280       ??_GIAttachmentManager@@UEAAPEAXI@Z 00000000315a2280 f i CharacterInstance.obj
 0001:000a12b0       ?LoadSequence@CFacialInstance@@UEAAPEAUIFacialAnimSequence@@PEBD_N@Z 00000000315a22b0 f   FacialInstance.obj
 0001:000a13d0       ?PrecacheFacialExpressionCallback@@YAXPEAXPEBD@Z 00000000315a23d0 f   FacialInstance.obj
 0001:000a1410       ?PrecacheFacialExpression@CFacialInstance@@UEAAXPEBD@Z 00000000315a2410 f   FacialInstance.obj
 0001:000a14d0       ?EnableProceduralFacialAnimation@CFacialInstance@@UEAAX_N@Z 00000000315a24d0 f   FacialInstance.obj
 0001:000a14e0       ?SetMasterCharacter@CFacialInstance@@UEAAXPEAUICharacterInstance@@@Z 00000000315a24e0 f   FacialInstance.obj
 0001:000a14f0       ?StartWaiting@CLipSync@CFacialInstance@@QEAAXPEAUIFacialAnimSequence@@H@Z 00000000315a24f0 f i FacialInstance.obj
 0001:000a1540       ?Done@CLipSync@CFacialInstance@@QEAAXXZ 00000000315a2540 f i FacialInstance.obj
 0001:000a1570       ?GetFaceState@CFacialInstance@@UEAAPEAUIFaceState@@XZ 00000000315a2570 f   FacialInstance.obj
 0001:000a1580       ?StartEffectorChannel@CFacialInstance@@UEAAIPEAUIFacialEffector@@MMMH@Z 00000000315a2580 f   FacialInstance.obj
 0001:000a15c0       ?StopEffectorChannel@CFacialInstance@@UEAAXIM@Z 00000000315a25c0 f   FacialInstance.obj
 0001:000a15e0       ?FindEffector@CFacialInstance@@QEAAPEAUIFacialEffector@@VCFaceIdentifierHandle@@@Z 00000000315a25e0 f   FacialInstance.obj
 0001:000a1620       ?SeekSequence@CFacialInstance@@UEAAXW4EFacialSequenceLayer@@M@Z 00000000315a2620 f   FacialInstance.obj
 0001:000a1650       ?IsPlaySequence@CFacialInstance@@UEAA_NPEAUIFacialAnimSequence@@W4EFacialSequenceLayer@@@Z 00000000315a2650 f   FacialInstance.obj
 0001:000a1690       ?PauseSequence@CFacialInstance@@UEAAXW4EFacialSequenceLayer@@_N@Z 00000000315a2690 f   FacialInstance.obj
 0001:000a16c0       ?ProcessWaitingLipSync@CFacialInstance@@QEAAXXZ 00000000315a26c0 f   FacialInstance.obj
 0001:000a17b0       ?OnExpressionLibraryLoad@CFacialInstance@@UEAAXXZ 00000000315a27b0 f   FacialInstance.obj
 0001:000a17c0       ?ApplyProceduralFaceBehaviour@CFacialInstance@@QEAAXAEAU?$Vec3_tpl@M@@@Z 00000000315a27c0 f   FacialInstance.obj
 0001:000a1930       ?TemporarilyEnableBoneRotationSmoothing@CFacialInstance@@UEAAXXZ 00000000315a2930 f   FacialInstance.obj
 0001:000a1970       ?UpdateCurrentSequence@CFacialInstance@@AEAAXPEAUIFacialAnimSequence@@@Z 00000000315a2970 f   FacialInstance.obj
 0001:000a1b20       ?UpdateDue@CConstantFrameRateSkipper@@QEAA_NXZ 00000000315a2b20 f i FacialInstance.obj
 0001:000a1bc0       ?UpdatePlayingSequences@CFacialInstance@@QEAAXMAEBU?$QuatTS_tpl@M@@@Z 00000000315a2bc0 f   FacialInstance.obj
 0001:000a1d70       ?PreviewEffector@CFacialInstance@@UEAAXPEAUIFacialEffector@@MM@Z 00000000315a2d70 f   FacialInstance.obj
 0001:000a1e80       ?PreviewEffectors@CFacialInstance@@UEAAXPEAPEAUIFacialEffector@@PEAM1H@Z 00000000315a2e80 f   FacialInstance.obj
 0001:000a1fe0       ?PlaySequence@CFacialInstance@@UEAAXPEAUIFacialAnimSequence@@W4EFacialSequenceLayer@@_N2@Z 00000000315a2fe0 f   FacialInstance.obj
 0001:000a2150       ?StopSequence@CFacialInstance@@UEAAXW4EFacialSequenceLayer@@@Z 00000000315a3150 f   FacialInstance.obj
 0001:000a2280       ?UpdateProceduralFaceBehaviour@CFacialInstance@@QEAAXXZ 00000000315a3280 f   FacialInstance.obj
 0001:000a2440       ?Reset@CFacialInstance@@AEAAXXZ 00000000315a3440 f   FacialInstance.obj
 0001:000a2540       ?set_size@?$SmallDynStorage@VCFacialAnimForcedRotationEntry@@HUStandardAlloc@NAlloc@@@NArray@@QEAAXH@Z 00000000315a3540 f i FacialInstance.obj
 0001:000a2540       ?set_size@?$SmallDynStorage@UVirtualExample2D@@HUStandardAlloc@NAlloc@@@NArray@@QEAAXH@Z 00000000315a3540 f i ParametricSampler.obj
 0001:000a2540       ?set_size@?$SmallDynStorage@U?$SplineKey@M@spline@@HUStandardAlloc@NAlloc@@@NArray@@QEAAXH@Z 00000000315a3540 f i FaceAnimSequence.obj
 0001:000a25f0       ?replace@?$CryStackStringT@D$0CAA@@@QEAAAEAV1@PEBD0@Z 00000000315a35f0 f i FacialInstance.obj
 0001:000a27d0       ??Y?$CryStackStringT@D$0CAA@@@QEAAAEAV0@AEBV0@@Z 00000000315a37d0 f i FacialInstance.obj
 0001:000a2890       ??$move_init@VCFacialAnimForcedRotationEntry@@@NArray@@YAXPEAVCFacialAnimForcedRotationEntry@@0_K@Z 00000000315a3890 f i FacialInstance.obj
 0001:000a2a10       ?GetMemoryUsage@CFacialInstance@@QEBAXPEAVICrySizer@@@Z 00000000315a3a10 f   FacialInstance.obj
 0001:000a2b20       ?resize_raw@?$SmallDynStorage@VCFacialAnimForcedRotationEntry@@HUStandardAlloc@NAlloc@@@NArray@@QEAAXHH_N@Z 00000000315a3b20 f i FacialInstance.obj
 0001:000a2ca0       ?GetPath@PathUtil@@YA?AV?$CryStackStringT@D$0CAA@@@AEBV2@@Z 00000000315a3ca0 f i FacialInstance.obj
 0001:000a2d70       ?Update@CFacialInstance@@QEAAXAEAV?$map@IUSFacialDisplaceInfo@CFacialModel@@U?$less@I@stlpmtx_std@@V?$allocator@U?$pair@$$CBIUSFacialDisplaceInfo@CFacialModel@@@stlpmtx_std@@@4@@stlpmtx_std@@MAEBU?$QuatTS_tpl@M@@@Z 00000000315a3d70 f   FacialInstance.obj
 0001:000a2ef0       ?expand_raw@?$DynArray@VCFacialAnimForcedRotationEntry@@HU?$SmallDynStorage@VCFacialAnimForcedRotationEntry@@HUStandardAlloc@NAlloc@@@NArray@@@@IEAAPEAVCFacialAnimForcedRotationEntry@@PEAV2@H@Z 00000000315a3ef0 f i FacialInstance.obj
 0001:000a2fb0       ?GetFileName@PathUtil@@YA?AV?$CryStringT@D@@AEBV2@@Z 00000000315a3fb0 f i FacialInstance.obj
 0001:000a3090       ?AddSlash@PathUtil@@YA?AV?$CryStackStringT@D$0CAA@@@AEBV2@@Z 00000000315a4090 f i FacialInstance.obj
 0001:000a3210       ?LipSyncWithSound@CFacialInstance@@UEAAXI_N@Z 00000000315a4210 f   FacialInstance.obj
 0001:000a4810       ??0CFacialInstance@@QEAA@PEAVCFacialModel@@PEAVCCharInstance@@@Z 00000000315a5810 f   FacialInstance.obj
 0001:000a4b70       ??_ECFacialInstance@@W7EAAPEAXI@Z 00000000315a5b70 f i FacialInstance.obj
 0001:000a4b80       ??1CFacialInstance@@UEAA@XZ 00000000315a5b80 f i FacialInstance.obj
 0001:000a4c90       ??_GCFacialInstance@@UEAAPEAXI@Z 00000000315a5c90 f i FacialInstance.obj
 0001:000a4c90       ??_ECFacialInstance@@UEAAPEAXI@Z 00000000315a5c90 f i FacialInstance.obj
 0001:000a4cc0       ?SetForcedRotations@CFacialInstance@@UEAAXHPEAVCFacialAnimForcedRotationEntry@@@Z 00000000315a5cc0 f   FacialInstance.obj
 0001:000a4d40       ?GetEffectorName@CFacialAnimChannel@@UEAAPEBDXZ 00000000315a5d40 f   FaceAnimSequence.obj
 0001:000a4d40       ?GetEffector@CFacialEffCtrl@@UEAAPEAUIFacialEffector@@XZ 00000000315a5d40 f   FaceEffector.obj
 0001:000a4d40       ?GetLibrary@CFacialModel@@UEAAPEAUIFacialEffectorsLibrary@@XZ 00000000315a5d40 f   FacialModel.obj
 0001:000a4d50       ?GetMorphTargetCount@CFacialModel@@UEBAHXZ 00000000315a5d50 f   FacialModel.obj
 0001:000a4d80       ?ApplyBoneEffector@CFacialModel@@AEAAHPEAVCSkeletonPose@@PEAVCFacialEffector@@MAEAU?$QuatT_tpl@M@@@Z 00000000315a5d80 f   FacialModel.obj
 0001:000a4f40       ?TransformTranslations@CFacialModel@@AEAAXAEAV?$map@IUSFacialDisplaceInfo@CFacialModel@@U?$less@I@stlpmtx_std@@V?$allocator@U?$pair@$$CBIUSFacialDisplaceInfo@CFacialModel@@@stlpmtx_std@@@4@@stlpmtx_std@@QEBVCSkeletonPose@@@Z 00000000315a5f40 f   FacialModel.obj
 0001:000a5160       ?SetAffectedJointsToDefaultPose@CFacialModel@@SAXAEBV?$map@IUSFacialDisplaceInfo@CFacialModel@@U?$less@I@stlpmtx_std@@V?$allocator@U?$pair@$$CBIUSFacialDisplaceInfo@CFacialModel@@@stlpmtx_std@@@4@@stlpmtx_std@@QEAU?$QuatT_tpl@M@@QEBU4@@Z 00000000315a6160 f   FacialModel.obj
 0001:000a5230       ?ApplyDisplaceInfoToJoints@CFacialModel@@SAXAEBV?$map@IUSFacialDisplaceInfo@CFacialModel@@U?$less@I@stlpmtx_std@@V?$allocator@U?$pair@$$CBIUSFacialDisplaceInfo@CFacialModel@@@stlpmtx_std@@@4@@stlpmtx_std@@QEBVCModelSkeleton@@QEAVCPoseData@Skeleton@@@Z 00000000315a6230 f   FacialModel.obj
 0001:000a5810       ?SizeOfThis@CFacialModel@@QEAA_KXZ 00000000315a6810 f   FacialModel.obj
 0001:000a5880       ??$__unguarded_linear_insert@PEAUSMorphTargetInfo@CFacialModel@@U12@U?$less@USMorphTargetInfo@CFacialModel@@@stlpmtx_std@@@priv@stlpmtx_std@@YAXPEAUSMorphTargetInfo@CFacialModel@@U23@U?$less@USMorphTargetInfo@CFacialModel@@@1@@Z 00000000315a6880 f i FacialModel.obj
 0001:000a5920       ??$__push_heap@PEAUSMorphTargetInfo@CFacialModel@@_JU12@U?$less@USMorphTargetInfo@CFacialModel@@@stlpmtx_std@@@stlpmtx_std@@YAXPEAUSMorphTargetInfo@CFacialModel@@_J1U12@U?$less@USMorphTargetInfo@CFacialModel@@@0@@Z 00000000315a6920 f i FacialModel.obj
 0001:000a5a30       ?GetMorphTargetName@CFacialModel@@UEBAPEBDH@Z 00000000315a6a30 f   FacialModel.obj
 0001:000a5ae0       ??$AddObject@USEffectorInfo@CFacialModel@@V?$allocator@USEffectorInfo@CFacialModel@@@stlpmtx_std@@@ICrySizer@@QEAAXAEBV?$vector@USEffectorInfo@CFacialModel@@V?$allocator@USEffectorInfo@CFacialModel@@@stlpmtx_std@@@stlpmtx_std@@@Z 00000000315a6ae0 f i FacialModel.obj
 0001:000a5bc0       ??$__adjust_heap@PEAUSMorphTargetInfo@CFacialModel@@_JU12@U?$less@USMorphTargetInfo@CFacialModel@@@stlpmtx_std@@@stlpmtx_std@@YAXPEAUSMorphTargetInfo@CFacialModel@@_J1U12@U?$less@USMorphTargetInfo@CFacialModel@@@0@@Z 00000000315a6bc0 f i FacialModel.obj
 0001:000a5d30       ??$swap@USMorphTargetInfo@CFacialModel@@@stlpmtx_std@@YAXAEAUSMorphTargetInfo@CFacialModel@@0@Z 00000000315a6d30 f i FacialModel.obj
 0001:000a5e20       ??$AddObject@USMorphTargetInfo@CFacialModel@@V?$allocator@USMorphTargetInfo@CFacialModel@@@stlpmtx_std@@@ICrySizer@@QEAAXAEBV?$vector@USMorphTargetInfo@CFacialModel@@V?$allocator@USMorphTargetInfo@CFacialModel@@@stlpmtx_std@@@stlpmtx_std@@@Z 00000000315a6e20 f i FacialModel.obj
 0001:000a5ef0       ??$_Copy_Construct@USEffectorInfo@CFacialModel@@@stlpmtx_std@@YAXPEAUSEffectorInfo@CFacialModel@@AEBU12@@Z 00000000315a6ef0 f i FacialModel.obj
 0001:000a5f60       ?_M_create_node@?$_Rb_tree@IU?$less@I@stlpmtx_std@@U?$pair@$$CBIUSFacialDisplaceInfo@CFacialModel@@@2@U?$_Select1st@U?$pair@$$CBIUSFacialDisplaceInfo@CFacialModel@@@stlpmtx_std@@@priv@2@U?$_MapTraitsT@U?$pair@$$CBIUSFacialDisplaceInfo@CFacialModel@@@stlpmtx_std@@@52@V?$allocator@U?$pair@$$CBIUSFacialDisplaceInfo@CFacialModel@@@stlpmtx_std@@@2@@priv@stlpmtx_std@@IEAAPEAU_Rb_tree_node_base@23@AEBU?$pair@$$CBIUSFacialDisplaceInfo@CFacialModel@@@3@@Z 00000000315a6f60 f i FacialModel.obj
 0001:000a6000       ??$__pop_heap@PEAUSMorphTargetInfo@CFacialModel@@U12@U?$less@USMorphTargetInfo@CFacialModel@@@stlpmtx_std@@_J@stlpmtx_std@@YAXPEAUSMorphTargetInfo@CFacialModel@@00U12@U?$less@USMorphTargetInfo@CFacialModel@@@0@PEA_J@Z 00000000315a7000 f i FacialModel.obj
 0001:000a60e0       ??$__make_heap@PEAUSMorphTargetInfo@CFacialModel@@U?$less@USMorphTargetInfo@CFacialModel@@@stlpmtx_std@@U12@_J@stlpmtx_std@@YAXPEAUSMorphTargetInfo@CFacialModel@@0U?$less@USMorphTargetInfo@CFacialModel@@@0@0PEA_J@Z 00000000315a70e0 f i FacialModel.obj
 0001:000a61b0       ??0CFaceState@@QEAA@PEAVCFacialModel@@@Z 00000000315a71b0 f i FacialModel.obj
 0001:000a6250       ??_ECFaceState@@W7EAAPEAXI@Z 00000000315a7250 f i FacialModel.obj
 0001:000a6260       ?SetEffectorWeight@CFaceState@@UEAAXHM@Z 00000000315a7260 f i FacialModel.obj
 0001:000a6290       ?GetEffectorWeight@CFaceState@@UEAAMH@Z 00000000315a7290 f i FacialModel.obj
 0001:000a62c0       ??1CFaceState@@UEAA@XZ     00000000315a72c0 f i FacialModel.obj
 0001:000a6340       ??_ECFaceState@@UEAAPEAXI@Z 00000000315a7340 f i FacialModel.obj
 0001:000a6340       ??_GCFaceState@@UEAAPEAXI@Z 00000000315a7340 f i FacialModel.obj
 0001:000a6370       ?CreateState@CFacialModel@@QEAAPEAVCFaceState@@XZ 00000000315a7370 f   FacialModel.obj
 0001:000a63d0       ?GetMemoryUsage@CFacialModel@@QEBAXPEAVICrySizer@@@Z 00000000315a73d0 f   FacialModel.obj
 0001:000a6460       ??$__destroy_mv_srcs@V?$reverse_iterator@PEAUSEffectorInfo@CFacialModel@@@stlpmtx_std@@USEffectorInfo@CFacialModel@@@stlpmtx_std@@YAXV?$reverse_iterator@PEAUSEffectorInfo@CFacialModel@@@0@0PEAUSEffectorInfo@CFacialModel@@@Z 00000000315a7460 f i FacialModel.obj
 0001:000a6460       ??$__destroy_range@V?$reverse_iterator@PEAUSEffectorInfo@CFacialModel@@@stlpmtx_std@@USEffectorInfo@CFacialModel@@@stlpmtx_std@@YAXV?$reverse_iterator@PEAUSEffectorInfo@CFacialModel@@@0@0PEAUSEffectorInfo@CFacialModel@@@Z 00000000315a7460 f i FacialModel.obj
 0001:000a64e0       ??$__ucopy_ptrs@PEAUSEffectorInfo@CFacialModel@@PEAU12@@priv@stlpmtx_std@@YAPEAUSEffectorInfo@CFacialModel@@PEAU23@00AEBU__false_type@1@@Z 00000000315a74e0 f i FacialModel.obj
 0001:000a65a0       ?_M_insert@?$_Rb_tree@IU?$less@I@stlpmtx_std@@U?$pair@$$CBIUSFacialDisplaceInfo@CFacialModel@@@2@U?$_Select1st@U?$pair@$$CBIUSFacialDisplaceInfo@CFacialModel@@@stlpmtx_std@@@priv@2@U?$_MapTraitsT@U?$pair@$$CBIUSFacialDisplaceInfo@CFacialModel@@@stlpmtx_std@@@52@V?$allocator@U?$pair@$$CBIUSFacialDisplaceInfo@CFacialModel@@@stlpmtx_std@@@2@@priv@stlpmtx_std@@AEAA?AU?$_Rb_tree_iterator@U?$pair@$$CBIUSFacialDisplaceInfo@CFacialModel@@@stlpmtx_std@@U?$_MapTraitsT@U?$pair@$$CBIUSFacialDisplaceInfo@CFacialModel@@@stlpmtx_std@@@priv@2@@23@PEAU_Rb_tree_node_base@23@AEBU?$pair@$$CBIUSFacialDisplaceInfo@CFacialModel@@@3@00@Z 00000000315a75a0 f i FacialModel.obj
 0001:000a6660       ?insert_unique@?$_Rb_tree@IU?$less@I@stlpmtx_std@@U?$pair@$$CBIUSFacialDisplaceInfo@CFacialModel@@@2@U?$_Select1st@U?$pair@$$CBIUSFacialDisplaceInfo@CFacialModel@@@stlpmtx_std@@@priv@2@U?$_MapTraitsT@U?$pair@$$CBIUSFacialDisplaceInfo@CFacialModel@@@stlpmtx_std@@@52@V?$allocator@U?$pair@$$CBIUSFacialDisplaceInfo@CFacialModel@@@stlpmtx_std@@@2@@priv@stlpmtx_std@@QEAA?AU?$pair@U?$_Rb_tree_iterator@U?$pair@$$CBIUSFacialDisplaceInfo@CFacialModel@@@stlpmtx_std@@U?$_MapTraitsT@U?$pair@$$CBIUSFacialDisplaceInfo@CFacialModel@@@stlpmtx_std@@@priv@2@@priv@stlpmtx_std@@_N@3@AEBU?$pair@$$CBIUSFacialDisplaceInfo@CFacialModel@@@3@@Z 00000000315a7660 f i FacialModel.obj
 0001:000a6860       ??$copy_backward@PEAUSMorphTargetInfo@CFacialModel@@PEAU12@@stlpmtx_std@@YAPEAUSMorphTargetInfo@CFacialModel@@PEAU12@00@Z 00000000315a7860 f i FacialModel.obj
 0001:000a6900       ?_M_clear@?$_Impl_vector@USEffectorInfo@CFacialModel@@V?$allocator@USEffectorInfo@CFacialModel@@@stlpmtx_std@@@priv@stlpmtx_std@@AEAAXXZ 00000000315a7900 f i FacialModel.obj
 0001:000a6940       ?_M_clear_after_move@?$_Impl_vector@USMorphTargetInfo@CFacialModel@@V?$allocator@USMorphTargetInfo@CFacialModel@@@stlpmtx_std@@@priv@stlpmtx_std@@AEAAXXZ 00000000315a7940 f i FacialModel.obj
 0001:000a6940       ?_M_clear@?$_Impl_vector@USMorphTargetInfo@CFacialModel@@V?$allocator@USMorphTargetInfo@CFacialModel@@@stlpmtx_std@@@priv@stlpmtx_std@@AEAAXXZ 00000000315a7940 f i FacialModel.obj
 0001:000a69c0       ?insert_unique@?$_Rb_tree@IU?$less@I@stlpmtx_std@@U?$pair@$$CBIUSFacialDisplaceInfo@CFacialModel@@@2@U?$_Select1st@U?$pair@$$CBIUSFacialDisplaceInfo@CFacialModel@@@stlpmtx_std@@@priv@2@U?$_MapTraitsT@U?$pair@$$CBIUSFacialDisplaceInfo@CFacialModel@@@stlpmtx_std@@@52@V?$allocator@U?$pair@$$CBIUSFacialDisplaceInfo@CFacialModel@@@stlpmtx_std@@@2@@priv@stlpmtx_std@@QEAA?AU?$_Rb_tree_iterator@U?$pair@$$CBIUSFacialDisplaceInfo@CFacialModel@@@stlpmtx_std@@U?$_MapTraitsT@U?$pair@$$CBIUSFacialDisplaceInfo@CFacialModel@@@stlpmtx_std@@@priv@2@@23@U423@AEBU?$pair@$$CBIUSFacialDisplaceInfo@CFacialModel@@@3@@Z 00000000315a79c0 f i FacialModel.obj
 0001:000a6e00       ??$__linear_insert@PEAUSMorphTargetInfo@CFacialModel@@U12@U?$less@USMorphTargetInfo@CFacialModel@@@stlpmtx_std@@@priv@stlpmtx_std@@YAXPEAUSMorphTargetInfo@CFacialModel@@0U23@U?$less@USMorphTargetInfo@CFacialModel@@@1@@Z 00000000315a7e00 f i FacialModel.obj
 0001:000a6ec0       ??$sort_heap@PEAUSMorphTargetInfo@CFacialModel@@U?$less@USMorphTargetInfo@CFacialModel@@@stlpmtx_std@@@stlpmtx_std@@YAXPEAUSMorphTargetInfo@CFacialModel@@0U?$less@USMorphTargetInfo@CFacialModel@@@0@@Z 00000000315a7ec0 f i FacialModel.obj
 0001:000a6fb0       ??1?$_Impl_vector@USMorphTargetInfo@CFacialModel@@V?$allocator@USMorphTargetInfo@CFacialModel@@@stlpmtx_std@@@priv@stlpmtx_std@@QEAA@XZ 00000000315a7fb0 f i FacialModel.obj
 0001:000a7040       ??$uninitialized_copy@PEAUSMorphTargetInfo@CFacialModel@@PEAU12@@stlpmtx_std@@YAPEAUSMorphTargetInfo@CFacialModel@@PEAU12@00@Z 00000000315a8040 f i FacialModel.obj
 0001:000a70b0       ??$__insertion_sort@PEAUSMorphTargetInfo@CFacialModel@@U12@U?$less@USMorphTargetInfo@CFacialModel@@@stlpmtx_std@@@priv@stlpmtx_std@@YAXPEAUSMorphTargetInfo@CFacialModel@@00U?$less@USMorphTargetInfo@CFacialModel@@@1@@Z 00000000315a80b0 f i FacialModel.obj
 0001:000a7150       ??$__partial_sort@PEAUSMorphTargetInfo@CFacialModel@@U12@U?$less@USMorphTargetInfo@CFacialModel@@@stlpmtx_std@@@priv@stlpmtx_std@@YAXPEAUSMorphTargetInfo@CFacialModel@@000U?$less@USMorphTargetInfo@CFacialModel@@@1@@Z 00000000315a8150 f i FacialModel.obj
 0001:000a7220       ?AssignLibrary@CFacialModel@@UEAAXPEAUIFacialEffectorsLibrary@@@Z 00000000315a8220 f   FacialModel.obj
 0001:000a76d0       ?reserve@?$_Impl_vector@USEffectorInfo@CFacialModel@@V?$allocator@USEffectorInfo@CFacialModel@@@stlpmtx_std@@@priv@stlpmtx_std@@QEAAX_K@Z 00000000315a86d0 f i FacialModel.obj
 0001:000a7850       ??$?AH@?$map@IUSFacialDisplaceInfo@CFacialModel@@U?$less@I@stlpmtx_std@@V?$allocator@U?$pair@$$CBIUSFacialDisplaceInfo@CFacialModel@@@stlpmtx_std@@@4@@stlpmtx_std@@QEAAAEAUSFacialDisplaceInfo@CFacialModel@@AEBH@Z 00000000315a8850 f i FacialModel.obj
 0001:000a7930       ?FillInfoMapFromFaceState@CFacialModel@@QEAAXAEAV?$map@IUSFacialDisplaceInfo@CFacialModel@@U?$less@I@stlpmtx_std@@V?$allocator@U?$pair@$$CBIUSFacialDisplaceInfo@CFacialModel@@@stlpmtx_std@@@4@@stlpmtx_std@@QEAVCFaceState@@QEAVCSkeletonPose@@HQEBVCFacialAnimForcedRotationEntry@@_N@Z 00000000315a8930 f   FacialModel.obj
 0001:000a80b0       ?push_back@?$_Impl_vector@USEffectorInfo@CFacialModel@@V?$allocator@USEffectorInfo@CFacialModel@@@stlpmtx_std@@@priv@stlpmtx_std@@QEAAXAEBUSEffectorInfo@CFacialModel@@@Z 00000000315a90b0 f i FacialModel.obj
 0001:000a81e0       ?reserve@?$_Impl_vector@USMorphTargetInfo@CFacialModel@@V?$allocator@USMorphTargetInfo@CFacialModel@@@stlpmtx_std@@@priv@stlpmtx_std@@QEAAX_K@Z 00000000315a91e0 f i FacialModel.obj
 0001:000a8360       ??$__introsort_loop@PEAUSMorphTargetInfo@CFacialModel@@U12@_JU?$less@USMorphTargetInfo@CFacialModel@@@stlpmtx_std@@@priv@stlpmtx_std@@YAXPEAUSMorphTargetInfo@CFacialModel@@00_JU?$less@USMorphTargetInfo@CFacialModel@@@1@@Z 00000000315a9360 f i FacialModel.obj
 0001:000a8530       ?InitMorphTargets@CFacialModel@@AEAAXXZ 00000000315a9530 f   FacialModel.obj
 0001:000a8c50       ??0CFacialModel@@QEAA@PEAVCSkel@@@Z 00000000315a9c50 f   FacialModel.obj
 0001:000a8d20       ??_ECFacialModel@@W7EAAPEAXI@Z 00000000315a9d20 f i FacialModel.obj
 0001:000a8d30       ?GetEffector@CFacialModel@@UEBAPEAVCFacialEffector@@H@Z 00000000315a9d30 f i FacialModel.obj
 0001:000a8d40       ??1CFacialModel@@UEAA@XZ   00000000315a9d40 f i FacialModel.obj
 0001:000a8e00       ??_GCFacialModel@@UEAAPEAXI@Z 00000000315a9e00 f i FacialModel.obj
 0001:000a8e00       ??_ECFacialModel@@UEAAPEAXI@Z 00000000315a9e00 f i FacialModel.obj
 0001:000a8e30       ??_EIPlaceholderCharacter@@UEAAPEAXI@Z 00000000315a9e30 f i PlaceholderCharacter.obj
 0001:000a8e30       ??_GCPoseAlignerChain@@MEAAPEAXI@Z 00000000315a9e30 f i PoseAlignerChain.obj
 0001:000a8e30       ??_ECPoseBlenderLook@@MEAAPEAXI@Z 00000000315a9e30 f i PoseBlenderLook.obj
 0001:000a8e30       ??_GICryUnknown@@MEAAPEAXI@Z 00000000315a9e30 f i OperatorQueue.obj
 0001:000a8e30       ??_GIPlaceholderCharacter@@UEAAPEAXI@Z 00000000315a9e30 f i PlaceholderCharacter.obj
 0001:000a8e30       ??_GIJoystickContext@@UEAAPEAXI@Z 00000000315a9e30 f i FaceAnimation.obj
 0001:000a8e30       ??_EIJoystickContext@@UEAAPEAXI@Z 00000000315a9e30 f i FaceAnimation.obj
 0001:000a8e30       ??_ECPoseAlignerChain@@MEAAPEAXI@Z 00000000315a9e30 f i PoseAlignerChain.obj
 0001:000a8e30       ??_GCPoseBlenderLook@@MEAAPEAXI@Z 00000000315a9e30 f i PoseBlenderLook.obj
 0001:000a8e30       ??_ECGroundAlignment@@MEAAPEAXI@Z 00000000315a9e30 f i GroundAlignment.obj
 0001:000a8e30       ??_GIPhonemeLibrary@@UEAAPEAXI@Z 00000000315a9e30 f i LipSync.obj
 0001:000a8e30       ??_ECFeetPoseStore@@MEAAPEAXI@Z 00000000315a9e30 f i FeetLock.obj
 0001:000a8e30       ??_GCGroundAlignment@@MEAAPEAXI@Z 00000000315a9e30 f i GroundAlignment.obj
 0001:000a8e30       ??_EICryUnknown@@MEAAPEAXI@Z 00000000315a9e30 f i OperatorQueue.obj
 0001:000a8e30       ??_EIPhonemeLibrary@@UEAAPEAXI@Z 00000000315a9e30 f i LipSync.obj
 0001:000a8e30       ??_GCFeetPoseStore@@MEAAPEAXI@Z 00000000315a9e30 f i FeetLock.obj
 0001:000a8e60       ?phoneme_less@@YA_NAEBUSPhoneme@@0@Z 00000000315a9e60 f i LipSync.obj
 0001:000a8e80       ?GetPhonemeLib@CFacialSentence@@UEAAPEAUIPhonemeLibrary@@XZ 00000000315a9e80 f   LipSync.obj
 0001:000a8eb0       ??_G?$_reference_target@H@@UEAAPEAXI@Z 00000000315a9eb0 f i LipSync.obj
 0001:000a8eb0       ??_E?$_reference_target@H@@UEAAPEAXI@Z 00000000315a9eb0 f i LipSync.obj
 0001:000a8ee0       ?GetPhonemeCount@CPhonemesLibrary@@UEBAHXZ 00000000315a9ee0 f   LipSync.obj
 0001:000a8ef0       ?GetPhonemeInfo@CPhonemesLibrary@@UEAA_NHAEAUSPhonemeInfo@@@Z 00000000315a9ef0 f   LipSync.obj
 0001:000a8f40       ?allocate@?$_STLP_alloc_proxy@PEAU?$pair@PEAUIFacialAnimChannel@@H@stlpmtx_std@@U12@V?$allocator@U?$pair@PEAUIFacialAnimChannel@@H@stlpmtx_std@@@2@@priv@stlpmtx_std@@QEAAPEAU?$pair@PEAUIFacialAnimChannel@@H@3@_KAEA_K@Z 00000000315a9f40 f i FaceAnimSequence.obj
 0001:000a8f40       ?allocate@?$_STLP_alloc_proxy@PEAU?$pair@V?$CryStringT@D@@PEAUIFacialAnimChannel@@@stlpmtx_std@@U12@V?$allocator@U?$pair@V?$CryStringT@D@@PEAUIFacialAnimChannel@@@stlpmtx_std@@@2@@priv@stlpmtx_std@@QEAAPEAU?$pair@V?$CryStringT@D@@PEAUIFacialAnimChannel@@@3@_KAEA_K@Z 00000000315a9f40 f i FaceAnimation.obj
 0001:000a8f40       ?allocate@?$_STLP_alloc_proxy@PEAUSPhoneme@@U1@V?$allocator@USPhoneme@@@stlpmtx_std@@@priv@stlpmtx_std@@QEAAPEAUSPhoneme@@_KAEA_K@Z 00000000315a9f40 f i LipSync.obj
 0001:000a8fb0       ?_M_compute_next_size@?$_Impl_vector@UWordRec@CFacialSentence@@V?$allocator@UWordRec@CFacialSentence@@@stlpmtx_std@@@priv@stlpmtx_std@@AEAA_K_K@Z 00000000315a9fb0 f i LipSync.obj
 0001:000a9040       ?GetPhoneme@CFacialSentence@@UEAA_NHAEAUPhoneme@IFacialSentence@@@Z 00000000315aa040 f   LipSync.obj
 0001:000a9090       ?GetWord@CFacialSentence@@UEAA_NHAEAUWord@IFacialSentence@@@Z 00000000315aa090 f   LipSync.obj
 0001:000a90f0       ?Evaluate@CFacialSentence@@UEAAHMMHPEAUChannelSample@IFacialSentence@@@Z 00000000315aa0f0 f   LipSync.obj
 0001:000a9310       ??$_M_allocate_and_copy@PEBU?$TCoeffBasis@M@spline@@@?$_Impl_vector@U?$TCoeffBasis@M@spline@@V?$allocator@U?$TCoeffBasis@M@spline@@@stlpmtx_std@@@priv@stlpmtx_std@@AEAAPEAU?$TCoeffBasis@M@spline@@AEA_KPEBU34@1@Z 00000000315aa310 f i FaceEffector.obj
 0001:000a9310       ??$_M_allocate_and_copy@PEBUPhoneme@IFacialSentence@@@?$_Impl_vector@UPhoneme@IFacialSentence@@V?$allocator@UPhoneme@IFacialSentence@@@stlpmtx_std@@@priv@stlpmtx_std@@AEAAPEAUPhoneme@IFacialSentence@@AEA_KPEBU34@1@Z 00000000315aa310 f i LipSync.obj
 0001:000a9310       ??$_M_allocate_and_copy@PEAU?$pair@PEAUIFacialAnimChannel@@H@stlpmtx_std@@@?$_Impl_vector@U?$pair@PEAUIFacialAnimChannel@@H@stlpmtx_std@@V?$allocator@U?$pair@PEAUIFacialAnimChannel@@H@stlpmtx_std@@@2@@priv@stlpmtx_std@@AEAAPEAU?$pair@PEAUIFacialAnimChannel@@H@2@AEA_KPEAU32@1@Z 00000000315aa310 f i FaceAnimSequence.obj
 0001:000a93c0       ??4SPhoneme@@QEAAAEAU0@AEBU0@@Z 00000000315aa3c0 f i LipSync.obj
 0001:000a94b0       ??$__unguarded_linear_insert@PEAUSPhoneme@@U1@P6A_NAEBU1@0@Z@priv@stlpmtx_std@@YAXPEAUSPhoneme@@U2@P6A_NAEBU2@2@Z@Z 00000000315aa4b0 f i LipSync.obj
 0001:000a9550       ??$__push_heap@PEAUSPhoneme@@_JU1@P6A_NAEBU1@0@Z@stlpmtx_std@@YAXPEAUSPhoneme@@_J1U1@P6A_NAEBU1@3@Z@Z 00000000315aa550 f i LipSync.obj
 0001:000a9650       ?FindPhonemeByName@CPhonemesLibrary@@UEAAHPEBD@Z 00000000315aa650 f   LipSync.obj
 0001:000a9780       ?push_back@?$_Impl_vector@UPhoneme@IFacialSentence@@V?$allocator@UPhoneme@IFacialSentence@@@stlpmtx_std@@@priv@stlpmtx_std@@QEAAXAEBUPhoneme@IFacialSentence@@@Z 00000000315aa780 f i LipSync.obj
 0001:000a9800       ??4?$_Impl_vector@UPhoneme@IFacialSentence@@V?$allocator@UPhoneme@IFacialSentence@@@stlpmtx_std@@@priv@stlpmtx_std@@QEAAAEAV012@AEBV012@@Z 00000000315aa800 f i LipSync.obj
 0001:000a9800       ??4?$_Impl_vector@U?$TCoeffBasis@M@spline@@V?$allocator@U?$TCoeffBasis@M@spline@@@stlpmtx_std@@@priv@stlpmtx_std@@QEAAAEAV012@AEBV012@@Z 00000000315aa800 f i FaceEffector.obj
 0001:000a9950       ??$__adjust_heap@PEAUSPhoneme@@_JU1@P6A_NAEBU1@0@Z@stlpmtx_std@@YAXPEAUSPhoneme@@_J1U1@P6A_NAEBU1@3@Z@Z 00000000315aa950 f i LipSync.obj
 0001:000a9a90       ??$__pop_heap@PEAUSPhoneme@@U1@P6A_NAEBU1@0@Z_J@stlpmtx_std@@YAXPEAUSPhoneme@@00U1@P6A_NAEBU1@2@ZPEA_J@Z 00000000315aaa90 f i LipSync.obj
 0001:000a9b40       ??$__make_heap@PEAUSPhoneme@@P6A_NAEBU1@0@ZU1@_J@stlpmtx_std@@YAXPEAUSPhoneme@@0P6A_NAEBU1@1@Z0PEA_J@Z 00000000315aab40 f i LipSync.obj
 0001:000a9c10       ?AddPhoneme@CFacialSentence@@UEAAHAEBUPhoneme@IFacialSentence@@@Z 00000000315aac10 f   LipSync.obj
 0001:000a9c50       ?Animate@CFacialSentence@@QEAAXAEBU?$QuatTS_tpl@M@@PEAVCFacialAnimationContext@@MMAEBV?$VectorSet@VCFaceIdentifierHandle@@USFaceIdentifierHandleLess@CFacialSentence@@V?$allocator@VCFaceIdentifierHandle@@@stlpmtx_std@@@@@Z 00000000315aac50 f   LipSync.obj
 0001:000aa170       ??$__unguarded_partition@PEAUSPhoneme@@U1@P6A_NAEBU1@0@Z@priv@stlpmtx_std@@YAPEAUSPhoneme@@PEAU2@0U2@P6A_NAEBU2@2@Z@Z 00000000315ab170 f i LipSync.obj
 0001:000aa2a0       ??$__destroy_range_aux@V?$reverse_iterator@PEAUWordRec@CFacialSentence@@@stlpmtx_std@@UWordRec@CFacialSentence@@@stlpmtx_std@@YAXV?$reverse_iterator@PEAUWordRec@CFacialSentence@@@0@0PEAUWordRec@CFacialSentence@@AEBU__false_type@0@@Z 00000000315ab2a0 f i LipSync.obj
 0001:000aa3c0       ??$__destroy_range_aux@PEAUWordRec@CFacialSentence@@U12@@stlpmtx_std@@YAXPEAUWordRec@CFacialSentence@@00AEBU__false_type@0@@Z 00000000315ab3c0 f i LipSync.obj
 0001:000aa4d0       ?_M_clear@?$_Impl_vector@USPhoneme@@V?$allocator@USPhoneme@@@stlpmtx_std@@@priv@stlpmtx_std@@AEAAXXZ 00000000315ab4d0 f i LipSync.obj
 0001:000aa550       ??$__ucopy@PEAUWordRec@CFacialSentence@@PEAU12@_J@priv@stlpmtx_std@@YAPEAUWordRec@CFacialSentence@@PEAU23@00AEBUrandom_access_iterator_tag@1@PEA_J@Z 00000000315ab550 f i LipSync.obj
 0001:000aa8b0       ??$__linear_insert@PEAUSPhoneme@@U1@P6A_NAEBU1@0@Z@priv@stlpmtx_std@@YAXPEAUSPhoneme@@0U2@P6A_NAEBU2@2@Z@Z 00000000315ab8b0 f i LipSync.obj
 0001:000aa9b0       ??$sort_heap@PEAUSPhoneme@@P6A_NAEBU1@0@Z@stlpmtx_std@@YAXPEAUSPhoneme@@0P6A_NAEBU1@1@Z@Z 00000000315ab9b0 f i LipSync.obj
 0001:000aaaf0       ??1?$_Impl_vector@USPhoneme@@V?$allocator@USPhoneme@@@stlpmtx_std@@@priv@stlpmtx_std@@QEAA@XZ 00000000315abaf0 f i LipSync.obj
 0001:000aab80       ??$_M_allocate_and_copy@PEAUSPhoneme@@@?$_Impl_vector@USPhoneme@@V?$allocator@USPhoneme@@@stlpmtx_std@@@priv@stlpmtx_std@@AEAAPEAUSPhoneme@@AEA_KPEAU3@1@Z 00000000315abb80 f i LipSync.obj
 0001:000aac60       ??$__insertion_sort@PEAUSPhoneme@@U1@P6A_NAEBU1@0@Z@priv@stlpmtx_std@@YAXPEAUSPhoneme@@00P6A_NAEBU2@1@Z@Z 00000000315abc60 f i LipSync.obj
 0001:000aad00       ??$__partial_sort@PEAUSPhoneme@@U1@P6A_NAEBU1@0@Z@priv@stlpmtx_std@@YAXPEAUSPhoneme@@000P6A_NAEBU2@1@Z@Z 00000000315abd00 f i LipSync.obj
 0001:000aade0       ?_M_erase@?$_Impl_vector@UWordRec@CFacialSentence@@V?$allocator@UWordRec@CFacialSentence@@@stlpmtx_std@@@priv@stlpmtx_std@@AEAAPEAUWordRec@CFacialSentence@@PEAU45@0AEBU__false_type@3@@Z 00000000315abde0 f i LipSync.obj
 0001:000aaed0       ?reserve@?$_Impl_vector@USPhoneme@@V?$allocator@USPhoneme@@@stlpmtx_std@@@priv@stlpmtx_std@@QEAAX_K@Z 00000000315abed0 f i LipSync.obj
 0001:000aaf90       ??$__introsort_loop@PEAUSPhoneme@@U1@_JP6A_NAEBU1@0@Z@priv@stlpmtx_std@@YAXPEAUSPhoneme@@00_JP6A_NAEBU2@2@Z@Z 00000000315abf90 f i LipSync.obj
 0001:000ab0f0       ??0CFacialSentence@@QEAA@XZ 00000000315ac0f0 f   LipSync.obj
 0001:000ab190       ??_ECFacialSentence@@W7EAAPEAXI@Z 00000000315ac190 f i LipSync.obj
 0001:000ab1a0       ?GetPhonemeCount@CFacialSentence@@UEAAHXZ 00000000315ac1a0 f i LipSync.obj
 0001:000ab1b0       ?GetWordCount@CFacialSentence@@UEAAHXZ 00000000315ac1b0 f i LipSync.obj
 0001:000ab1e0       ?SetText@CFacialSentence@@UEAAXPEBD@Z 00000000315ac1e0 f i LipSync.obj
 0001:000ab230       ??1CFacialSentence@@UEAA@XZ 00000000315ac230 f i LipSync.obj
 0001:000ab300       ??_GCFacialSentence@@UEAAPEAXI@Z 00000000315ac300 f i LipSync.obj
 0001:000ab300       ??_ECFacialSentence@@UEAAPEAXI@Z 00000000315ac300 f i LipSync.obj
 0001:000ab330       ??0CPhonemesLibrary@@QEAA@XZ 00000000315ac330 f   LipSync.obj
 0001:000ab9b0       ??_ECPhonemesLibrary@@UEAAPEAXI@Z 00000000315ac9b0 f i LipSync.obj
 0001:000ab9b0       ??_GCPhonemesLibrary@@UEAAPEAXI@Z 00000000315ac9b0 f i LipSync.obj
 0001:000ab9f0       ?ClearAllPhonemes@CFacialSentence@@UEAAXXZ 00000000315ac9f0 f i LipSync.obj
 0001:000aba30       ?ClearAllWords@CFacialSentence@@UEAAXXZ 00000000315aca30 f i LipSync.obj
 0001:000aba60       ?AddWord@CFacialSentence@@UEAAXAEBUWord@IFacialSentence@@@Z 00000000315aca60 f   LipSync.obj
 0001:000abcd0       ?Serialize@CFacialSentence@@QEAAXAEAVXmlNodeRef@@_N@Z 00000000315accd0 f   LipSync.obj
 0001:000acc20       ?GetFactory@CFeetPoseRestore@@UEBAPEAUICryFactory@@XZ 00000000315adc20 f i FeetLock.obj
 0001:000acc30       ?GetFactory@CFeetPoseStore@@UEBAPEAUICryFactory@@XZ 00000000315adc30 f i FeetLock.obj
 0001:000acc40       ?Prepare@CFeetPoseStore@@UEAA_NAEBUSAnimationPoseModifierParams@@@Z 00000000315adc40 f i FeetLock.obj
 0001:000acc40       ?Prepare@CFeetPoseRestore@@UEAA_NAEBUSAnimationPoseModifierParams@@@Z 00000000315adc40 f i FeetLock.obj
 0001:000acc50       ?GetMemoryUsage@CFeetPoseStore@@UEBAXPEAVICrySizer@@@Z 00000000315adc50 f i FeetLock.obj
 0001:000acc50       ?GetMemoryUsage@CFeetPoseRestore@@UEBAXPEAVICrySizer@@@Z 00000000315adc50 f i FeetLock.obj
 0001:000acca0       ?Execute@CFeetPoseStore@@UEAA_NAEBUSAnimationPoseModifierParams@@@Z 00000000315adca0 f   FeetLock.obj
 0001:000ad0e0       ?Execute@CFeetPoseRestore@@UEAA_NAEBUSAnimationPoseModifierParams@@@Z 00000000315ae0e0 f   FeetLock.obj
 0001:000ad660       ?GetClassName@CFactory@CFeetPoseStore@@UEBAPEBDXZ 00000000315ae660 f i FeetLock.obj
 0001:000ad670       ?GetClassID@CFactory@CFeetPoseStore@@UEBAAEBUCryGUID@@XZ 00000000315ae670 f i FeetLock.obj
 0001:000ad680       ??_E?$sp_counted_impl_p@VCEngineModule_CryAnimation@@@detail@boost@@UEAAPEAXI@Z 00000000315ae680 f i AnimationBase.obj
 0001:000ad680       ??_E?$sp_counted_impl_p@VCOperatorQueue@@@detail@boost@@UEAAPEAXI@Z 00000000315ae680 f i OperatorQueue.obj
 0001:000ad680       ??_E?$sp_counted_impl_p@VCPoseBlenderAim@@@detail@boost@@UEAAPEAXI@Z 00000000315ae680 f i PoseBlenderAim.obj
 0001:000ad680       ??_E?$sp_counted_impl_p@VCFeetPoseRestore@@@detail@boost@@UEAAPEAXI@Z 00000000315ae680 f i FeetLock.obj
 0001:000ad680       ??_G?$sp_counted_impl_p@VCPoseBlenderLook@@@detail@boost@@UEAAPEAXI@Z 00000000315ae680 f i PoseBlenderLook.obj
 0001:000ad680       ??_Gsp_counted_base@detail@boost@@UEAAPEAXI@Z 00000000315ae680 f i OperatorQueue.obj
 0001:000ad680       ??_G?$sp_counted_impl_p@VCLimbIk@@@detail@boost@@UEAAPEAXI@Z 00000000315ae680 f i LimbIk.obj
 0001:000ad680       ??_E?$sp_counted_impl_p@VCPoseBlenderLook@@@detail@boost@@UEAAPEAXI@Z 00000000315ae680 f i PoseBlenderLook.obj
 0001:000ad680       ??_E?$sp_counted_impl_p@VCLimbIk@@@detail@boost@@UEAAPEAXI@Z 00000000315ae680 f i LimbIk.obj
 0001:000ad680       ??_G?$sp_counted_impl_p@VCPoseMatching@@@detail@boost@@UEAAPEAXI@Z 00000000315ae680 f i PoseMatching.obj
 0001:000ad680       ??_E?$sp_counted_impl_p@VCPoseMatching@@@detail@boost@@UEAAPEAXI@Z 00000000315ae680 f i PoseMatching.obj
 0001:000ad680       ??_G?$sp_counted_impl_p@VCOperatorQueue@@@detail@boost@@UEAAPEAXI@Z 00000000315ae680 f i OperatorQueue.obj
 0001:000ad680       ??_E?$sp_counted_impl_p@VCRecoil@PoseModifier@@@detail@boost@@UEAAPEAXI@Z 00000000315ae680 f i Recoil.obj
 0001:000ad680       ??_G?$sp_counted_impl_p@VCFeetPoseStore@@@detail@boost@@UEAAPEAXI@Z 00000000315ae680 f i FeetLock.obj
 0001:000ad680       ??_G?$sp_counted_impl_p@VCPoseAlignerChain@@@detail@boost@@UEAAPEAXI@Z 00000000315ae680 f i PoseAlignerChain.obj
 0001:000ad680       ??_E?$sp_counted_impl_p@VCFeetPoseStore@@@detail@boost@@UEAAPEAXI@Z 00000000315ae680 f i FeetLock.obj
 0001:000ad680       ??_G?$sp_counted_impl_p@VCPoseBlenderAim@@@detail@boost@@UEAAPEAXI@Z 00000000315ae680 f i PoseBlenderAim.obj
 0001:000ad680       ??_G?$sp_counted_impl_p@VCEngineModule_CryAnimation@@@detail@boost@@UEAAPEAXI@Z 00000000315ae680 f i AnimationBase.obj
 0001:000ad680       ??_G?$sp_counted_impl_p@VCRecoil@PoseModifier@@@detail@boost@@UEAAPEAXI@Z 00000000315ae680 f i Recoil.obj
 0001:000ad680       ??_Esp_counted_base@detail@boost@@UEAAPEAXI@Z 00000000315ae680 f i OperatorQueue.obj
 0001:000ad680       ??_E?$sp_counted_impl_p@VCGroundAlignment@@@detail@boost@@UEAAPEAXI@Z 00000000315ae680 f i GroundAlignment.obj
 0001:000ad680       ??_G?$sp_counted_impl_p@VCFeetPoseRestore@@@detail@boost@@UEAAPEAXI@Z 00000000315ae680 f i FeetLock.obj
 0001:000ad680       ??_G?$sp_counted_impl_p@VCGroundAlignment@@@detail@boost@@UEAAPEAXI@Z 00000000315ae680 f i GroundAlignment.obj
 0001:000ad680       ??_E?$sp_counted_impl_p@VCPoseAlignerChain@@@detail@boost@@UEAAPEAXI@Z 00000000315ae680 f i PoseAlignerChain.obj
 0001:000ad6b0       ?CreateClassInstance@CFactory@CFeetPoseStore@@UEBA?AV?$shared_ptr@UICryUnknown@@@boost@@XZ 00000000315ae6b0 f i FeetLock.obj
 0001:000ad770       ?GetClassName@CFactory@CFeetPoseRestore@@UEBAPEBDXZ 00000000315ae770 f i FeetLock.obj
 0001:000ad780       ?GetClassID@CFactory@CFeetPoseRestore@@UEBAAEBUCryGUID@@XZ 00000000315ae780 f i FeetLock.obj
 0001:000ad790       ?dispose@?$sp_counted_impl_p@VCPoseBlenderAim@@@detail@boost@@UEAAXXZ 00000000315ae790 f i PoseBlenderAim.obj
 0001:000ad790       ?dispose@?$sp_counted_impl_p@VCPoseAlignerChain@@@detail@boost@@UEAAXXZ 00000000315ae790 f i PoseAlignerChain.obj
 0001:000ad790       ?dispose@?$sp_counted_impl_p@VCGroundAlignment@@@detail@boost@@UEAAXXZ 00000000315ae790 f i GroundAlignment.obj
 0001:000ad790       ?dispose@?$sp_counted_impl_p@VCRecoil@PoseModifier@@@detail@boost@@UEAAXXZ 00000000315ae790 f i Recoil.obj
 0001:000ad790       ?dispose@?$sp_counted_impl_p@VCLimbIk@@@detail@boost@@UEAAXXZ 00000000315ae790 f i LimbIk.obj
 0001:000ad790       ?dispose@?$sp_counted_impl_p@VCPoseMatching@@@detail@boost@@UEAAXXZ 00000000315ae790 f i PoseMatching.obj
 0001:000ad790       ?dispose@?$sp_counted_impl_p@VCEngineModule_CryAnimation@@@detail@boost@@UEAAXXZ 00000000315ae790 f i AnimationBase.obj
 0001:000ad790       ?dispose@?$sp_counted_impl_p@VCOperatorQueue@@@detail@boost@@UEAAXXZ 00000000315ae790 f i OperatorQueue.obj
 0001:000ad790       ?dispose@?$sp_counted_impl_p@VCPoseBlenderLook@@@detail@boost@@UEAAXXZ 00000000315ae790 f i PoseBlenderLook.obj
 0001:000ad790       ?dispose@?$sp_counted_impl_p@VCFeetPoseStore@@@detail@boost@@UEAAXXZ 00000000315ae790 f i FeetLock.obj
 0001:000ad790       ?dispose@?$sp_counted_impl_p@VCFeetPoseRestore@@@detail@boost@@UEAAXXZ 00000000315ae790 f i FeetLock.obj
 0001:000ad7b0       ?CreateClassInstance@CFactory@CFeetPoseRestore@@UEBA?AV?$shared_ptr@UICryUnknown@@@boost@@XZ 00000000315ae7b0 f i FeetLock.obj
 0001:000ad870       ?QueryInterface@CRecoil@PoseModifier@@MEBAPEAXAEBUCryGUID@@@Z 00000000315ae870 f i Recoil.obj
 0001:000ad870       ?QueryInterface@CFeetPoseRestore@@MEBAPEAXAEBUCryGUID@@@Z 00000000315ae870 f i FeetLock.obj
 0001:000ad870       ?QueryInterface@CFeetPoseStore@@MEBAPEAXAEBUCryGUID@@@Z 00000000315ae870 f i FeetLock.obj
 0001:000ad870       ?QueryInterface@CLimbIk@@MEBAPEAXAEBUCryGUID@@@Z 00000000315ae870 f i LimbIk.obj
 0001:000ad8c0       ??0CFeetLock@@QEAA@XZ      00000000315ae8c0 f   FeetLock.obj
 0001:000ad930       ?Prepare@CGroundAlignment@@UEAA_NAEBUSAnimationPoseModifierParams@@@Z 00000000315ae930 f   GroundAlignment.obj
 0001:000ad9c0       ??0CGroundAlignment@@IEAA@XZ 00000000315ae9c0 f   GroundAlignment.obj
 0001:000ada70       ?GetFactory@CGroundAlignment@@UEBAPEAUICryFactory@@XZ 00000000315aea70 f i GroundAlignment.obj
 0001:000ada80       ?SetData@CGroundAlignment@@UEAAX_NMAEBU?$Plane_tpl@M@@1@Z 00000000315aea80 f i GroundAlignment.obj
 0001:000adad0       ?GetMemoryUsage@CGroundAlignment@@UEBAXPEAVICrySizer@@@Z 00000000315aead0 f i GroundAlignment.obj
 0001:000adaf0       ?SetFootGroundAlignment@CGroundAlignment@@AEAAIAEBUSAnimationPoseModifierParams@@AEBU?$Vec3_tpl@M@@HHHH@Z 00000000315aeaf0 f   GroundAlignment.obj
 0001:000ae9b0       ?PerformGroundAlignmentCCD@CGroundAlignment@@AEAAIAEBUSAnimationPoseModifierParams@@PEBDAEBU?$Plane_tpl@M@@@Z 00000000315af9b0 f   GroundAlignment.obj
 0001:000af9f0       ?MoveSkeletonVertical@CGroundAlignment@@AEAAXAEBUSAnimationPoseModifierParams@@M@Z 00000000315b09f0 f   GroundAlignment.obj
 0001:000afe90       ?AlignJointToPlane@@YA_NAEBUSAnimationPoseModifierParams@@IAEBU?$Vec3_tpl@M@@1@Z 00000000315b0e90 f   GroundAlignment.obj
 0001:000b0730       ?QueryInterface@CGroundAlignment@@MEBAPEAXAEBUCryGUID@@@Z 00000000315b1730 f i GroundAlignment.obj
 0001:000b07a0       ?LimbAlign@CGroundAlignment@@AEAA_NAEBUSAnimationPoseModifierParams@@IPEBDAEBU?$Plane_tpl@M@@@Z 00000000315b17a0 f   GroundAlignment.obj
 0001:000b0b10       ?ExecuteNew@CGroundAlignment@@AEAA_NAEBUSAnimationPoseModifierParams@@@Z 00000000315b1b10 f   GroundAlignment.obj
 0001:000b0b80       ?Execute@CGroundAlignment@@UEAA_NAEBUSAnimationPoseModifierParams@@@Z 00000000315b1b80 f   GroundAlignment.obj
 0001:000b0bf0       ??0CFactory@CGroundAlignment@@AEAA@XZ 00000000315b1bf0 f i GroundAlignment.obj
 0001:000b0c90       ?GetClassName@CFactory@CGroundAlignment@@UEBAPEBDXZ 00000000315b1c90 f i GroundAlignment.obj
 0001:000b0ca0       ?GetClassID@CFactory@CGroundAlignment@@UEBAAEBUCryGUID@@XZ 00000000315b1ca0 f i GroundAlignment.obj
 0001:000b0cb0       ?ClassSupports@CFactory@CPoseMatching@@UEBAXAEAPEBUCryGUID@@AEA_K@Z 00000000315b1cb0 f i PoseMatching.obj
 0001:000b0cb0       ?ClassSupports@CFactory@CFeetPoseStore@@UEBAXAEAPEBUCryGUID@@AEA_K@Z 00000000315b1cb0 f i FeetLock.obj
 0001:000b0cb0       ?ClassSupports@CFactory@CPoseBlenderLook@@UEBAXAEAPEBUCryGUID@@AEA_K@Z 00000000315b1cb0 f i PoseBlenderLook.obj
 0001:000b0cb0       ?ClassSupports@CFactory@CRecoil@PoseModifier@@UEBAXAEAPEBUCryGUID@@AEA_K@Z 00000000315b1cb0 f i Recoil.obj
 0001:000b0cb0       ?ClassSupports@CFactory@CPoseBlenderAim@@UEBAXAEAPEBUCryGUID@@AEA_K@Z 00000000315b1cb0 f i PoseBlenderAim.obj
 0001:000b0cb0       ?ClassSupports@CFactory@COperatorQueue@@UEBAXAEAPEBUCryGUID@@AEA_K@Z 00000000315b1cb0 f i OperatorQueue.obj
 0001:000b0cb0       ?ClassSupports@CFactory@CLimbIk@@UEBAXAEAPEBUCryGUID@@AEA_K@Z 00000000315b1cb0 f i LimbIk.obj
 0001:000b0cb0       ?ClassSupports@CFactory@CPoseAlignerChain@@UEBAXAEAPEBUCryGUID@@AEA_K@Z 00000000315b1cb0 f i PoseAlignerChain.obj
 0001:000b0cb0       ?ClassSupports@CFactory@CFeetPoseRestore@@UEBAXAEAPEBUCryGUID@@AEA_K@Z 00000000315b1cb0 f i FeetLock.obj
 0001:000b0cb0       ?ClassSupports@CFactory@CEngineModule_CryAnimation@@UEBAXAEAPEBUCryGUID@@AEA_K@Z 00000000315b1cb0 f i AnimationBase.obj
 0001:000b0cb0       ?ClassSupports@CFactory@CGroundAlignment@@UEBAXAEAPEBUCryGUID@@AEA_K@Z 00000000315b1cb0 f i GroundAlignment.obj
 0001:000b0cc0       ?CreateClassInstance@CFactory@CGroundAlignment@@UEBA?AV?$shared_ptr@UICryUnknown@@@boost@@XZ 00000000315b1cc0 f i GroundAlignment.obj
 0001:000b0d80       ?AddSetup@CLimbIk@@QEAAX_KAEBU?$Vec3_tpl@M@@@Z 00000000315b1d80 f   LimbIk.obj
 0001:000b0e20       ?Prepare@CLimbIk@@UEAA_NAEBUSAnimationPoseModifierParams@@@Z 00000000315b1e20 f   LimbIk.obj
 0001:000b0e60       ?Execute@CLimbIk@@UEAA_NAEBUSAnimationPoseModifierParams@@@Z 00000000315b1e60 f   LimbIk.obj
 0001:000b0ee0       ?GetFactory@CLimbIk@@UEBAPEAUICryFactory@@XZ 00000000315b1ee0 f i LimbIk.obj
 0001:000b0ef0       ?GetMemoryUsage@CLimbIk@@UEBAXPEAVICrySizer@@@Z 00000000315b1ef0 f i LimbIk.obj
 0001:000b0f10       ?GetClassName@CFactory@CLimbIk@@UEBAPEBDXZ 00000000315b1f10 f i LimbIk.obj
 0001:000b0f20       ?GetClassID@CFactory@CLimbIk@@UEBAAEBUCryGUID@@XZ 00000000315b1f20 f i LimbIk.obj
 0001:000b0f30       ?CreateClassInstance@CFactory@CLimbIk@@UEBA?AV?$shared_ptr@UICryUnknown@@@boost@@XZ 00000000315b1f30 f i LimbIk.obj
 0001:000b1020       ??0SDirectionalBlender@@QEAA@XZ 00000000315b2020 f i PoseBlenderAim.obj
 0001:000b1090       ?GetFactory@CPoseBlenderAim@@UEBAPEAUICryFactory@@XZ 00000000315b2090 f i PoseBlenderAim.obj
 0001:000b10a0       ?SetState@CPoseBlenderAim@@UEAAX_N@Z 00000000315b20a0 f i PoseBlenderAim.obj
 0001:000b10b0       ?SetLayer@CPoseBlenderAim@@UEAAXI@Z 00000000315b20b0 f i PoseBlenderAim.obj
 0001:000b10d0       ?SetFadeoutAngle@CPoseBlenderAim@@UEAAXM@Z 00000000315b20d0 f i PoseBlenderAim.obj
 0001:000b10d0       ?SetVideoMarkerOffset@CFacialJoystickChannel@@UEAAXM@Z 00000000315b20d0 f i FaceJoystick.obj
 0001:000b10e0       ?SetFadeOutSpeed@CPoseBlenderAim@@UEAAXM@Z 00000000315b20e0 f i PoseBlenderAim.obj
 0001:000b1110       ?SetFadeInSpeed@CPoseBlenderAim@@UEAAXM@Z 00000000315b2110 f i PoseBlenderAim.obj
 0001:000b1140       ?SetTargetSmoothTime@CPoseBlenderAim@@UEAAXM@Z 00000000315b2140 f i PoseBlenderAim.obj
 0001:000b1150       ?GetBlend@CPoseBlenderAim@@UEAAMXZ 00000000315b2150 f i PoseBlenderAim.obj
 0001:000b1160       ?Synchronize@CPoseBlenderAim@@UEAAXXZ 00000000315b2160 f i PoseBlenderAim.obj
 0001:000b1170       ?GetMemoryUsage@CPoseBlenderAim@@UEBAXPEAVICrySizer@@@Z 00000000315b2170 f i PoseBlenderAim.obj
 0001:000b1190       ?SetPolarCoordinates@CPoseBlenderAim@@UEAAXAEBU?$Vec2_tpl@M@@@Z 00000000315b2190 f i PoseBlenderAim.obj
 0001:000b11a0       ?SetTarget@CPoseBlenderAim@@UEAAXAEBU?$Vec3_tpl@M@@@Z 00000000315b21a0 f i PoseBlenderAim.obj
 0001:000b11e0       ?Prepare@CPoseBlenderAim@@UEAA_NAEBUSAnimationPoseModifierParams@@@Z 00000000315b21e0 f   PoseBlenderAim.obj
 0001:000b1bd0       ?Execute@CPoseBlenderAim@@UEAA_NAEBUSAnimationPoseModifierParams@@@Z 00000000315b2bd0 f   PoseBlenderAim.obj
 0001:000b2a00       ??0CFactory@CPoseBlenderAim@@AEAA@XZ 00000000315b3a00 f i PoseBlenderAim.obj
 0001:000b2aa0       ?GetClassName@CFactory@CPoseBlenderAim@@UEBAPEBDXZ 00000000315b3aa0 f i PoseBlenderAim.obj
 0001:000b2ab0       ?GetClassID@CFactory@CPoseBlenderAim@@UEBAAEBUCryGUID@@XZ 00000000315b3ab0 f i PoseBlenderAim.obj
 0001:000b2ac0       ??_GCFactory@CGroundAlignment@@UEAAPEAXI@Z 00000000315b3ac0 f i GroundAlignment.obj
 0001:000b2ac0       ??_GCFactory@COperatorQueue@@UEAAPEAXI@Z 00000000315b3ac0 f i OperatorQueue.obj
 0001:000b2ac0       ??_ECFactory@CGroundAlignment@@UEAAPEAXI@Z 00000000315b3ac0 f i GroundAlignment.obj
 0001:000b2ac0       ??_ECFactory@CPoseBlenderAim@@UEAAPEAXI@Z 00000000315b3ac0 f i PoseBlenderAim.obj
 0001:000b2ac0       ??_ECFactory@CPoseAlignerChain@@UEAAPEAXI@Z 00000000315b3ac0 f i PoseAlignerChain.obj
 0001:000b2ac0       ??_ECFactory@CPoseMatching@@UEAAPEAXI@Z 00000000315b3ac0 f i PoseMatching.obj
 0001:000b2ac0       ??_GCFactory@CPoseMatching@@UEAAPEAXI@Z 00000000315b3ac0 f i PoseMatching.obj
 0001:000b2ac0       ??_GCFactory@CRecoil@PoseModifier@@UEAAPEAXI@Z 00000000315b3ac0 f i Recoil.obj
 0001:000b2ac0       ??_ECFactory@COperatorQueue@@UEAAPEAXI@Z 00000000315b3ac0 f i OperatorQueue.obj
 0001:000b2ac0       ??_ECFactory@CFeetPoseStore@@UEAAPEAXI@Z 00000000315b3ac0 f i FeetLock.obj
 0001:000b2ac0       ??_EICryFactory@@MEAAPEAXI@Z 00000000315b3ac0 f i OperatorQueue.obj
 0001:000b2ac0       ??_GCFactory@CPoseAlignerChain@@UEAAPEAXI@Z 00000000315b3ac0 f i PoseAlignerChain.obj
 0001:000b2ac0       ??_GCFactory@CFeetPoseRestore@@UEAAPEAXI@Z 00000000315b3ac0 f i FeetLock.obj
 0001:000b2ac0       ??_ECFactory@CFeetPoseRestore@@UEAAPEAXI@Z 00000000315b3ac0 f i FeetLock.obj
 0001:000b2ac0       ??_GCFactory@CPoseBlenderAim@@UEAAPEAXI@Z 00000000315b3ac0 f i PoseBlenderAim.obj
 0001:000b2ac0       ??_GCFactory@CLimbIk@@UEAAPEAXI@Z 00000000315b3ac0 f i LimbIk.obj
 0001:000b2ac0       ??_ECFactory@CPoseBlenderLook@@UEAAPEAXI@Z 00000000315b3ac0 f i PoseBlenderLook.obj
 0001:000b2ac0       ??_GCFactory@CPoseBlenderLook@@UEAAPEAXI@Z 00000000315b3ac0 f i PoseBlenderLook.obj
 0001:000b2ac0       ??_GCFactory@CFeetPoseStore@@UEAAPEAXI@Z 00000000315b3ac0 f i FeetLock.obj
 0001:000b2ac0       ??_GICryFactory@@MEAAPEAXI@Z 00000000315b3ac0 f i OperatorQueue.obj
 0001:000b2ac0       ??_ECFactory@CLimbIk@@UEAAPEAXI@Z 00000000315b3ac0 f i LimbIk.obj
 0001:000b2ac0       ??_ECFactory@CRecoil@PoseModifier@@UEAAPEAXI@Z 00000000315b3ac0 f i Recoil.obj
 0001:000b2af0       ?CreateClassInstance@CFactory@CPoseBlenderAim@@UEBA?AV?$shared_ptr@UICryUnknown@@@boost@@XZ 00000000315b3af0 f i PoseBlenderAim.obj
 0001:000b2bb0       ?QueryInterface@CPoseBlenderAim@@MEBAPEAXAEBUCryGUID@@@Z 00000000315b3bb0 f i PoseBlenderAim.obj
 0001:000b2bb0       ?QueryInterface@CPoseBlenderLook@@MEBAPEAXAEBUCryGUID@@@Z 00000000315b3bb0 f i PoseBlenderLook.obj
 0001:000b2c20       ?Synchronize@CPoseBlenderLook@@UEAAXXZ 00000000315b3c20 f   PoseBlenderLook.obj
 0001:000b2f60       ??0CPoseBlenderLook@@IEAA@XZ 00000000315b3f60 f   PoseBlenderLook.obj
 0001:000b3010       ?GetFactory@CPoseBlenderLook@@UEBAPEAUICryFactory@@XZ 00000000315b4010 f i PoseBlenderLook.obj
 0001:000b3020       ?SetState@CPoseBlenderLook@@UEAAX_N@Z 00000000315b4020 f i PoseBlenderLook.obj
 0001:000b3030       ?SetLayer@CPoseBlenderLook@@UEAAXI@Z 00000000315b4030 f i PoseBlenderLook.obj
 0001:000b3050       ?SetFadeoutAngle@CPoseBlenderLook@@UEAAXM@Z 00000000315b4050 f i PoseBlenderLook.obj
 0001:000b3060       ?SetFadeOutSpeed@CPoseBlenderLook@@UEAAXM@Z 00000000315b4060 f i PoseBlenderLook.obj
 0001:000b3090       ?SetFadeInSpeed@CPoseBlenderLook@@UEAAXM@Z 00000000315b4090 f i PoseBlenderLook.obj
 0001:000b30c0       ?SetTargetSmoothTime@CPoseBlenderLook@@UEAAXM@Z 00000000315b40c0 f i PoseBlenderLook.obj
 0001:000b30d0       ?GetBlend@CPoseBlenderLook@@UEAAMXZ 00000000315b40d0 f i PoseBlenderLook.obj
 0001:000b30e0       ?GetMemoryUsage@CPoseBlenderLook@@UEBAXPEAVICrySizer@@@Z 00000000315b40e0 f i PoseBlenderLook.obj
 0001:000b3100       ?SetPolarCoordinates@CPoseBlenderLook@@UEAAXAEBU?$Vec2_tpl@M@@@Z 00000000315b4100 f i PoseBlenderLook.obj
 0001:000b3120       ?SetTarget@CPoseBlenderLook@@UEAAXAEBU?$Vec3_tpl@M@@@Z 00000000315b4120 f i PoseBlenderLook.obj
 0001:000b3170       ?Prepare@CPoseBlenderLook@@UEAA_NAEBUSAnimationPoseModifierParams@@@Z 00000000315b4170 f   PoseBlenderLook.obj
 0001:000b3e10       ?Execute@CPoseBlenderLook@@UEAA_NAEBUSAnimationPoseModifierParams@@@Z 00000000315b4e10 f   PoseBlenderLook.obj
 0001:000b5e70       ??0CFactory@CPoseBlenderLook@@AEAA@XZ 00000000315b6e70 f i PoseBlenderLook.obj
 0001:000b5f10       ?GetClassName@CFactory@CPoseBlenderLook@@UEBAPEBDXZ 00000000315b6f10 f i PoseBlenderLook.obj
 0001:000b5f20       ?GetClassID@CFactory@CPoseBlenderLook@@UEBAAEBUCryGUID@@XZ 00000000315b6f20 f i PoseBlenderLook.obj
 0001:000b5f30       ?CreateClassInstance@CFactory@CPoseBlenderLook@@UEBA?AV?$shared_ptr@UICryUnknown@@@boost@@XZ 00000000315b6f30 f i PoseBlenderLook.obj
 0001:000b5ff0       ?IK_Solver2Bones@PoseModifierHelper@@YAXAEBU?$Vec3_tpl@M@@AEBUIKLimbType@@AEAVCPoseData@Skeleton@@@Z 00000000315b6ff0 f   PoseModifierHelper.obj
 0001:000b6ee0       ?IK_Solver3Bones@PoseModifierHelper@@YAXAEBU?$Vec3_tpl@M@@AEBUIKLimbType@@AEAVCPoseData@Skeleton@@@Z 00000000315b7ee0 f   PoseModifierHelper.obj
 0001:000b95e0       ?IK_SolverCCD@PoseModifierHelper@@YAXAEBU?$Vec3_tpl@M@@AEBUIKLimbType@@AEAVCPoseData@Skeleton@@@Z 00000000315ba5e0 f   PoseModifierHelper.obj
 0001:000ba7b0       ?IK_Solver@PoseModifierHelper@@YA_NPEIBVCModelSkeleton@@PEBDAEBU?$Vec3_tpl@M@@AEAVCPoseData@Skeleton@@@Z 00000000315bb7b0 f   PoseModifierHelper.obj
 0001:000bad70       ?Prepare@CRecoil@PoseModifier@@UEAA_NAEBUSAnimationPoseModifierParams@@@Z 00000000315bbd70 f   Recoil.obj
 0001:000bada0       ?RecoilEffect@CRecoil@PoseModifier@@AEAAMM@Z 00000000315bbda0 f   Recoil.obj
 0001:000bae20       ?GetFactory@CRecoil@PoseModifier@@UEBAPEAUICryFactory@@XZ 00000000315bbe20 f i Recoil.obj
 0001:000bae30       ?GetMemoryUsage@CRecoil@PoseModifier@@UEBAXPEAVICrySizer@@@Z 00000000315bbe30 f i Recoil.obj
 0001:000bae50       ?GetClassName@CFactory@CRecoil@PoseModifier@@UEBAPEBDXZ 00000000315bbe50 f i Recoil.obj
 0001:000bae60       ?GetClassID@CFactory@CRecoil@PoseModifier@@UEBAAEBUCryGUID@@XZ 00000000315bbe60 f i Recoil.obj
 0001:000bae70       ?Execute@CRecoil@PoseModifier@@UEAA_NAEBUSAnimationPoseModifierParams@@@Z 00000000315bbe70 f   Recoil.obj
 0001:000bbfd0       ?CreateClassInstance@CFactory@CRecoil@PoseModifier@@UEBA?AV?$shared_ptr@UICryUnknown@@@boost@@XZ 00000000315bcfd0 f i Recoil.obj
 0001:000bc0f0       ?Initialize@CState@Command@@QEAA_NPEAVCCharInstance@@AEBU?$QuatTS_tpl@M@@@Z 00000000315bd0f0 f   Command_Buffer.obj
 0001:000bc190       ?Initialize@CBuffer@Command@@QEAA_NPEAVCCharInstance@@AEBU?$QuatTS_tpl@M@@@Z 00000000315bd190 f   Command_Buffer.obj
 0001:000bc1d0       ?DebugDraw@CBuffer@Command@@AEAAXXZ 00000000315bd1d0 f   Command_Buffer.obj
 0001:000bc6c0       ?ProcessAnimationDrivenIk@@YAXAEAVCCharInstance@@AEBUSAnimationPoseModifierParams@@@Z 00000000315bd6c0 f   Command_Buffer.obj
 0001:000bd880       ?Execute@CBuffer@Command@@QEAAXXZ 00000000315be880 f   Command_Buffer.obj
 0001:000bdda0       ?Execute@ClearFull@Command@@QEBAXAEBVCState@2@QEAPEAX@Z 00000000315beda0 f   Command_Commands.obj
 0001:000bdde0       ?Execute@ClearSingle@Command@@QEBAXAEBVCState@2@QEAPEAX@Z 00000000315bede0 f   Command_Commands.obj
 0001:000bde00       ?Execute@NormalizeFull@Command@@QEBAXAEBVCState@2@QEAPEAX@Z 00000000315bee00 f   Command_Commands.obj
 0001:000be1a0       ?Execute@ScaleUniformFull@Command@@QEBAXAEBVCState@2@QEAPEAX@Z 00000000315bf1a0 f   Command_Commands.obj
 0001:000be320       ?Execute@CopyAddAnimFull@Command@@QEBAXAEBVCState@2@QEAPEAX@Z 00000000315bf320 f   Command_Commands.obj
 0001:000be810       ?Execute@SampleAddPoseFull@Command@@QEBAXAEBVCState@2@QEAPEAX@Z 00000000315bf810 f   Command_Commands.obj
 0001:000bec30       ?Execute@SamplePosePart@Command@@QEBAXAEBVCState@2@QEAPEAX@Z 00000000315bfc30 f   Command_Commands.obj
 0001:000bf040       ?Execute@PoseModifier@Command@@QEBAXAEBVCState@2@QEAPEAX@Z 00000000315c0040 f   Command_Commands.obj
 0001:000bf0d0       ?LoadControllers@Command@@YAXAEAUGlobalAnimationHeaderCAF@@AEBVCState@1@PEAPEAVIController@@@Z 00000000315c00d0 f   Command_Commands.obj
 0001:000bf360       ?Execute@SampleAddAnimFull@Command@@QEBAXAEBVCState@2@QEAPEAX@Z 00000000315c0360 f   Command_Commands.obj
 0001:000bfc80       ?Execute@SampleAnimPart@Command@@QEBAXAEBVCState@2@QEAPEAX@Z 00000000315c0c80 f   Command_Commands.obj
 0001:000c02f0       ?AllocationRelease@CPoseData@Skeleton@@QEAAXXZ 00000000315c12f0 f   Skeleton.obj
 0001:000c0340       ?GetAllocationLength@CPoseData@Skeleton@@QEBAIXZ 00000000315c1340 f   Skeleton.obj
 0001:000c0350       ?GetJointCount@CPoseData@Skeleton@@UEBAIXZ 00000000315c1350 f   Skeleton.obj
 0001:000c0360       ?SetJointRelativeP@CPoseData@Skeleton@@UEAAXIAEBU?$Vec3_tpl@M@@@Z 00000000315c1360 f   Skeleton.obj
 0001:000c0390       ?GetJointRelative@CPoseData@Skeleton@@UEBAAEBU?$QuatT_tpl@M@@I@Z 00000000315c1390 f   Skeleton.obj
 0001:000c03a0       ?SetJointAbsoluteP@CPoseData@Skeleton@@UEAAXIAEBU?$Vec3_tpl@M@@@Z 00000000315c13a0 f   Skeleton.obj
 0001:000c03d0       ?GetJointAbsolute@CPoseData@Skeleton@@UEBAAEBU?$QuatT_tpl@M@@I@Z 00000000315c13d0 f   Skeleton.obj
 0001:000c03e0       ?GetParentIndex@CPoseData@Skeleton@@QEBAHI@Z 00000000315c13e0 f   Skeleton.obj
 0001:000c03f0       ??_GIAnimationPoseData@@UEAAPEAXI@Z 00000000315c13f0 f i Skeleton.obj
 0001:000c03f0       ??_EIAnimationPoseData@@UEAAPEAXI@Z 00000000315c13f0 f i Skeleton.obj
 0001:000c0420       ??0CPoseData@Skeleton@@QEAA@XZ 00000000315c1420 f   Skeleton.obj
 0001:000c0450       ??1CPoseData@Skeleton@@UEAA@XZ 00000000315c1450 f   Skeleton.obj
 0001:000c04b0       ?AllocateData@CPoseData@Skeleton@@QEAA_NI@Z 00000000315c14b0 f   Skeleton.obj
 0001:000c05c0       ?Initialize@CPoseData@Skeleton@@QEAA_NAEBVCModelSkeleton@@I@Z 00000000315c15c0 f   Skeleton.obj
 0001:000c05e0       ?SetJointRelativeO@CPoseData@Skeleton@@UEAAXIAEBU?$Quat_tpl@M@@@Z 00000000315c15e0 f   Skeleton.obj
 0001:000c0610       ?SetJointAbsoluteO@CPoseData@Skeleton@@UEAAXIAEBU?$Quat_tpl@M@@@Z 00000000315c1610 f   Skeleton.obj
 0001:000c0640       ??_ECPoseData@Skeleton@@UEAAPEAXI@Z 00000000315c1640 f i Skeleton.obj
 0001:000c0640       ??_GCPoseData@Skeleton@@UEAAPEAXI@Z 00000000315c1640 f i Skeleton.obj
 0001:000c06c0       ?SetJointRelative@CPoseData@Skeleton@@UEAAXIAEBU?$QuatT_tpl@M@@@Z 00000000315c16c0 f   Skeleton.obj
 0001:000c0710       ?SetJointAbsolute@CPoseData@Skeleton@@UEAAXIAEBU?$QuatT_tpl@M@@@Z 00000000315c1710 f   Skeleton.obj
 0001:000c0760       ?Initialize@CPoseData@Skeleton@@QEAA_NAEBVCModelSkeleton@@@Z 00000000315c1760 f   Skeleton.obj
 0001:000c0820       ?Initialize@CPoseData@Skeleton@@QEAA_NAEBV12@@Z 00000000315c1820 f   Skeleton.obj
 0001:000c0930       ?ComputeAbsolutePose@CPoseData@Skeleton@@QEAAX_N@Z 00000000315c1930 f   Skeleton.obj
 0001:000c0f10       ?ComputeRelativePose@CPoseData@Skeleton@@QEAAX_N@Z 00000000315c1f10 f   Skeleton.obj
 0001:000c1690       ?ValidateRelative@CPoseData@Skeleton@@QEBAXXZ 00000000315c2690 f   Skeleton.obj
 0001:000c1bf0       ?ValidateAbsolute@CPoseData@Skeleton@@QEBAXXZ 00000000315c2bf0 f   Skeleton.obj
 0001:000c2470       ?Validate@CPoseData@Skeleton@@QEBAXXZ 00000000315c3470 f   Skeleton.obj
 0001:000c2490       ?SetPreLoadParticleEffects@AnimEventLoader@@YAX_N@Z 00000000315c3490 f   AnimEventLoader.obj
 0001:000c24a0       ?DoAdditionalAnimEventInitialization@AnimEventLoader@@YAXPEBDAEAVCAnimEventData@@@Z 00000000315c34a0 f   AnimEventLoader.obj
 0001:000c2560       ?LoadAnimationEventDatabase@AnimEventLoader@@YA_NPEAVCSkel@@PEBD@Z 00000000315c3560 f   AnimEventLoader.obj
 0001:000c29a0       ?GetIFacialAnimation@CharacterManager@@UEAAPEAUIFacialAnimation@@XZ 00000000315c39a0 f   CharacterManager.obj
 0001:000c29b0       ?GetRendererMainThreadId@CharacterManager@@SAIXZ 00000000315c39b0 f   CharacterManager.obj
 0001:000c2a10       ?UpdateRendererFrame@CharacterManager@@UEAAXXZ 00000000315c3a10 f   CharacterManager.obj
 0001:000c2a20       ?DummyUpdate@CharacterManager@@UEAAXXZ 00000000315c3a20 f   CharacterManager.obj
 0001:000c2a30       ?AlignBoneAttachment@CAttachmentFACE@@UEAAXXZ 00000000315c3a30 f   AttachmentManager.obj
 0001:000c2a30       ?AddRef@CControllerOptNonVirtual@@UEAAXXZ 00000000315c3a30 f   LoaderDBA.obj
 0001:000c2a30       ?AddRef@?$CTrackDataStorage@U?$Quat_tpl@M@@USmallTree64BitExtQuat@@VITrackRotationStorage@@@@UEAAXXZ 00000000315c3a30 f   ControllerPQ.obj
 0001:000c2a30       ?ExitScope_Free@CDummyMemReplay@@UEAAX_K@Z 00000000315c3a30 f   AnimEventList.obj
 0001:000c2a30       ?UnMarkPool@CDummyMemReplay@@UEAAXHPEAX@Z 00000000315c3a30 f   AnimEventList.obj
 0001:000c2a30       ?DumpSymbols@CDummyMemReplay@@UEAAXXZ 00000000315c3a30 f   AnimEventList.obj
 0001:000c2a30       ?AllocUsage@CDummyMemReplay@@UEAAXW4Class@EMemReplayAllocClass@@_K1@Z 00000000315c3a30 f   AnimEventList.obj
 0001:000c2a30       ?MarkBucket@CDummyMemReplay@@UEAAXH_KPEAX0@Z 00000000315c3a30 f   AnimEventList.obj
 0001:000c2a30       ?Flush@CDummyMemReplay@@UEAAXXZ 00000000315c3a30 f   AnimEventList.obj
 0001:000c2a30       ?AddSizerTree@CDummyMemReplay@@UEAAXPEBD@Z 00000000315c3a30 f   AnimEventList.obj
 0001:000c2a30       ?SetPendulumParams@CAttachmentSKIN@@UEAAXHCCMMMU?$Vec3_tpl@M@@0@Z 00000000315c3a30 f   Attachment.obj
 0001:000c2a30       ?Synchronize@CLimbIk@@UEAAXXZ 00000000315c3a30 f   LimbIk.obj
 0001:000c2a30       ?DumpStats@CDummyMemReplay@@UEAAXXZ 00000000315c3a30 f   AnimEventList.obj
 0001:000c2a30       ?BindToContainer@CDummyMemReplay@@UEAAXPEBX0@Z 00000000315c3a30 f   AnimEventList.obj
 0001:000c2a30       ?AddRef@?$CTrackDataStorage@U?$Quat_tpl@M@@USmallTree48BitQuat@@VITrackRotationStorage@@@@UEAAXXZ 00000000315c3a30 f   ControllerPQ.obj
 0001:000c2a30       ?UpdateLocation@CAttachmentSKIN@@UEAAXXZ 00000000315c3a30 f   Attachment.obj
 0001:000c2a30       ?SetParamString@CFacialEffector@@UEAAXW4EFacialEffectorParam@@PEBD@Z 00000000315c3a30 f   FaceEffector.obj
 0001:000c2a30       ?AddFrameStart@CDummyMemReplay@@UEAAXXZ 00000000315c3a30 f   AnimEventList.obj
 0001:000c2a30       ?GetRandomPos@CModelMesh@@QEAAXPEAUIRenderMesh@@PEAU?$DualQuat_tpl@M@@AEAURandomPos@@AEAUGeomQuery@@W4EGeomForm@@@Z 00000000315c3a30 f   ModelMesh.obj
 0001:000c2a30       ?AddScreenshot@CDummyMemReplay@@UEAAXXZ 00000000315c3a30 f   AnimEventList.obj
 0001:000c2a30       ?LockResources@CharacterManager@@UEAAXXZ 00000000315c3a30 f   CharacterManager.obj
 0001:000c2a30       ?ProcessAttachment@CAttachmentSKIN@@UEAAXPEAUIAttachment@@@Z 00000000315c3a30 f   Attachment.obj
 0001:000c2a30       ?SetAttAbsoluteDefault@CAttachmentSKIN@@UEAAXAEBU?$QuatT_tpl@M@@@Z 00000000315c3a30 f   Attachment.obj
 0001:000c2a30       ?UnregisterContainer@CDummyMemReplay@@UEAAXPEBX@Z 00000000315c3a30 f   AnimEventList.obj
 0001:000c2a30       ?GetMemoryUsage@CControllerOptNonVirtual@@UEBAXPEAVICrySizer@@@Z 00000000315c3a30 f   LoaderDBA.obj
 0001:000c2a30       ?SetDefaultAbsInvJointByID@CSkeletonPose@@UEAAXHAEBU?$QuatT_tpl@M@@@Z 00000000315c3a30 f   SkeletonPose.obj
 0001:000c2a30       ?GetMemoryUsage@IPositionController@@UEBAXPEAVICrySizer@@@Z 00000000315c3a30 f   LoaderTCB.obj
 0001:000c2a30       ?UnMarkBucket@CDummyMemReplay@@UEAAXHPEAX@Z 00000000315c3a30 f   AnimEventList.obj
 0001:000c2a30       ?Synchronize@CPoseAlignerChain@@UEAAXXZ 00000000315c3a30 f   PoseAlignerChain.obj
 0001:000c2a30       ?AddRef@?$CTrackDataStorage@U?$Vec3_tpl@M@@UNoCompressVec3@@VITrackPositionStorage@@@@UEAAXXZ 00000000315c3a30 f   ControllerPQ.obj
 0001:000c2a30       ?Synchronize@CPoseMatching@@UEAAXXZ 00000000315c3a30 f   PoseMatching.obj
 0001:000c2a30       ?ExitScope@CDummyMemReplay@@UEAAXXZ 00000000315c3a30 f   AnimEventList.obj
 0001:000c2a30       ?Synchronize@CRecoil@PoseModifier@@UEAAXXZ 00000000315c3a30 f   Recoil.obj
 0001:000c2a30       ?MarkPool@CDummyMemReplay@@UEAAXH_KPEAX0PEBD@Z 00000000315c3a30 f   AnimEventList.obj
 0001:000c2a30       ?AddRef@?$CTrackDataStorage@U?$Quat_tpl@M@@UNoCompressQuat@@VITrackRotationStorage@@@@UEAAXXZ 00000000315c3a30 f   ControllerPQ.obj
 0001:000c2a30       ?ProcessAttachment@CAttachmentBONE@@UEAAXPEAUIAttachment@@@Z 00000000315c3a30 f   AttachmentManager.obj
 0001:000c2a30       ?OnRemoveAttachment@IAttachmentObject@@UEAAXPEAUIAttachmentManager@@H@Z 00000000315c3a30 f   AttachmentManager.obj
 0001:000c2a30       ?AddContext@CDummyMemReplay@@UEAAXHIPEBD@Z 00000000315c3a30 f   AnimEventList.obj
 0001:000c2a30       ?Free@CPool@Memory@@UEAAXPEAX@Z 00000000315c3a30 f   Pool.obj
 0001:000c2a30       ?AddTexturePoolContext@CDummyMemReplay@@UEAAXPEAXHHHPEBDI@Z 00000000315c3a30 f   AnimEventList.obj
 0001:000c2a30       ?SwapContainers@CDummyMemReplay@@UEAAXPEBX0@Z 00000000315c3a30 f   AnimEventList.obj
 0001:000c2a30       ?Stop@CDummyMemReplay@@UEAAXXZ 00000000315c3a30 f   AnimEventList.obj
 0001:000c2a30       ?GetMemoryUsage@IRotationController@@UEBAXPEAVICrySizer@@@Z 00000000315c3a30 f   LoaderTCB.obj
 0001:000c2a30       ?BucketEnableCleanups@CDummyMemReplay@@UEAAXPEAX_N@Z 00000000315c3a30 f   AnimEventList.obj
 0001:000c2a30       ?GetInfo@CDummyMemReplay@@UEAAXAEAUCryReplayInfo@@@Z 00000000315c3a30 f   AnimEventList.obj
 0001:000c2a30       ?ProcessAttachment@CAttachmentFACE@@UEAAXPEAUIAttachment@@@Z 00000000315c3a30 f   AttachmentManager.obj
 0001:000c2a30       ?Release@CControllerOptNonVirtual@@UEAAXXZ 00000000315c3a30 f   LoaderDBA.obj
 0001:000c2a30       ?UnlockResources@CharacterManager@@UEAAXXZ 00000000315c3a30 f   CharacterManager.obj
 0001:000c2a30       ?SetParamInt@CFacialEffector@@UEAAXW4EFacialEffectorParam@@H@Z 00000000315c3a30 f   FaceEffector.obj
 0001:000c2a30       ?UnMapPage@CDummyMemReplay@@UEAAXPEAX_K@Z 00000000315c3a30 f   AnimEventList.obj
 0001:000c2a30       ?RenderAttachment@IAttachmentObject@@UEAAXAEAUSRendParams@@AEBUSRenderingPassInfo@@@Z 00000000315c3a30 f   AttachmentManager.obj
 0001:000c2a30       ?StreamAsyncOnComplete@IStreamCallback@@UEAAXPEAVIReadStream@@I@Z 00000000315c3a30 f   FaceAnimSequence.obj
 0001:000c2a30       ?SetParamVec3@CFacialEffector@@UEAAXW4EFacialEffectorParam@@U?$Vec3_tpl@M@@@Z 00000000315c3a30 f   FaceEffector.obj
 0001:000c2a30       ?UnbindFromContainer@CDummyMemReplay@@UEAAXPEBX0@Z 00000000315c3a30 f   AnimEventList.obj
 0001:000c2a30       ?CreateDecal@CCharInstance@@UEAAXAEAUCryEngineDecalInfo@@@Z 00000000315c3a30 f   CharacterInstance.obj
 0001:000c2a30       ?Synchronize@CFeetPoseRestore@@UEAAXXZ 00000000315c3a30 f   FeetLock.obj
 0001:000c2a30       ?Serialize@CFacialEffector@@UEAAXAEAVXmlNodeRef@@_N@Z 00000000315c3a30 f   FaceEffector.obj
 0001:000c2a30       ?ExitScope_Realloc@CDummyMemReplay@@UEAAX_K000@Z 00000000315c3a30 f   AnimEventList.obj
 0001:000c2a30       ?SetAttRelativeDefault@CAttachmentSKIN@@UEAAXAEBU?$QuatT_tpl@M@@@Z 00000000315c3a30 f   Attachment.obj
 0001:000c2a30       ?Synchronize@CFeetPoseStore@@UEAAXXZ 00000000315c3a30 f   FeetLock.obj
 0001:000c2a30       ?AddContextV@CDummyMemReplay@@UEAAXHIPEBDPEAD@Z 00000000315c3a30 f   AnimEventList.obj
 0001:000c2a30       ?AddLabel@CDummyMemReplay@@UEAAXPEBD@Z 00000000315c3a30 f   AnimEventList.obj
 0001:000c2a30       ?ExitScope_Alloc@CDummyMemReplay@@UEAAX_K00@Z 00000000315c3a30 f   AnimEventList.obj
 0001:000c2a30       ?ProcessAttachment@CCGFAttachment@@UEAAXPEAUIAttachment@@@Z 00000000315c3a30 f   AttachmentManager.obj
 0001:000c2a30       ?InitSpuControllerLookupTable@@YAXAEBU?$DynArray@IHU?$SmallDynStorage@IHUStandardAlloc@NAlloc@@@NArray@@@@@Z 00000000315c3a30 f   SkeletonAnim.obj
 0001:000c2a30       ?RemoveAllocReference@CDummyMemReplay@@UEAAXPEAX@Z 00000000315c3a30 f   AnimEventList.obj
 0001:000c2a30       ?Update@CPool@Memory@@UEAAXXZ 00000000315c3a30 f   Pool.obj
 0001:000c2a30       ?Start@CDummyMemReplay@@UEAAX_NPEBD@Z 00000000315c3a30 f   AnimEventList.obj
 0001:000c2a30       ?MapPage@CDummyMemReplay@@UEAAXPEAX_K@Z 00000000315c3a30 f   AnimEventList.obj
 0001:000c2a30       ?RegisterFixedAddressRange@CDummyMemReplay@@UEAAXPEAX_KPEBD@Z 00000000315c3a30 f   AnimEventList.obj
 0001:000c2a30       ?ReloadAllModels@CharacterManager@@UEAAXXZ 00000000315c3a30 f   CharacterManager.obj
 0001:000c2a30       ?RemoveContext@CDummyMemReplay@@UEAAXXZ 00000000315c3a30 f   AnimEventList.obj
 0001:000c2a30       ?StartOnCommandLine@CDummyMemReplay@@UEAAXPEBD@Z 00000000315c3a30 f   AnimEventList.obj
 0001:000c2a30       ?StreamOnComplete@IStreamCallback@@UEAAXPEAVIReadStream@@I@Z 00000000315c3a30 f   FaceAnimSequence.obj
 0001:000c2a30       ?RegisterContainer@CDummyMemReplay@@UEAAXPEBXH@Z 00000000315c3a30 f   AnimEventList.obj
 0001:000c2a30       ?Synchronize@CGroundAlignment@@UEAAXXZ 00000000315c3a30 f   GroundAlignment.obj
 0001:000c2a30       ?AddAllocReference@CDummyMemReplay@@UEAAXPEAX0@Z 00000000315c3a30 f   AnimEventList.obj
 0001:000c2a30       ?AddRef@?$CTrackDataStorage@U?$Quat_tpl@M@@USmallTree64BitQuat@@VITrackRotationStorage@@@@UEAAXXZ 00000000315c3a30 f   ControllerPQ.obj
 0001:000c2a30       ?AlignBoneAttachment@CAttachmentSKIN@@UEAAXXZ 00000000315c3a30 f   Attachment.obj
 0001:000c2a40       ?fxopen@@YAPEAU_iobuf@@PEBD0_N@Z 00000000315c3a40 f i CharacterManager.obj
 0001:000c2b50       ??_EICharacterManager@@UEAAPEAXI@Z 00000000315c3b50 f i CharacterManager.obj
 0001:000c2b50       ??_GICharacterManager@@UEAAPEAXI@Z 00000000315c3b50 f i CharacterManager.obj
 0001:000c2b80       ?SaveCharacterDefinition@CharacterManager@@UEAAIPEAUICharacterInstance@@PEBD@Z 00000000315c3b80 f   CharacterManager.obj
 0001:000c2d30       ?DBA_PreLoad@CharacterManager@@UEAA_NPEBDW4EStreamingDBAPriority@ICharacterManager@@@Z 00000000315c3d30 f   CharacterManager.obj
 0001:000c2d50       ?DBA_LockStatus@CharacterManager@@UEAA_NPEBDIW4EStreamingDBAPriority@ICharacterManager@@@Z 00000000315c3d50 f   CharacterManager.obj
 0001:000c2d70       ?DBA_Unload@CharacterManager@@UEAA_NPEBD@Z 00000000315c3d70 f   CharacterManager.obj
 0001:000c2db0       ??$move_init@UVirtualExampleInit2@CHUNK_GAHAIM_INFO@@@NArray@@YAXPEAUVirtualExampleInit2@CHUNK_GAHAIM_INFO@@0_K@Z 00000000315c3db0 f i CharacterManager.obj
 0001:000c2e00       ?DeleteDebugInstances@CharacterManager@@UEAAXXZ 00000000315c3e00 f   CharacterManager.obj
 0001:000c2e80       ?GetAverageFrameTime@CharacterManager@@AEAAMMMMM@Z 00000000315c3e80 f   CharacterManager.obj
 0001:000c2ff0       ?GetDBAFilePathByGlobalID@CharacterManager@@UEAAPEBDH@Z 00000000315c3ff0 f   CharacterManager.obj
 0001:000c3050       ?_M_compute_next_size@?$_Impl_vector@UCharacterDefinition@@V?$allocator@UCharacterDefinition@@@stlpmtx_std@@@priv@stlpmtx_std@@AEAA_K_K@Z 00000000315c4050 f i CharacterManager.obj
 0001:000c30e0       ?resize_raw@?$SmallDynStorage@IHUStandardAlloc@NAlloc@@@NArray@@QEAAXHH_N@Z 00000000315c40e0 f i CharacterManager.obj
 0001:000c3270       ??4CharacterAttachment@@QEAAAEAU0@AEBU0@@Z 00000000315c4270 f i CharacterManager.obj
 0001:000c3380       ?resize_raw@?$SmallDynStorage@UBSBlendable@@HUStandardAlloc@NAlloc@@@NArray@@QEAAXHH_N@Z 00000000315c4380 f i CharacterManager.obj
 0001:000c3530       ?set_size@?$SmallDynStorage@UVirtualExampleInit2@CHUNK_GAHAIM_INFO@@HUStandardAlloc@NAlloc@@@NArray@@QEAAXH@Z 00000000315c4530 f i CharacterManager.obj
 0001:000c3530       ?set_size@?$SmallDynStorage@U?$QuatT_tpl@M@@HUStandardAlloc@NAlloc@@@NArray@@QEAAXH@Z 00000000315c4530 f i SkeletonPhysics.obj
 0001:000c35e0       ?resize_raw@?$SmallDynStorage@UVirtualExampleInit2@CHUNK_GAHAIM_INFO@@HUStandardAlloc@NAlloc@@@NArray@@QEAAXHH_N@Z 00000000315c45e0 f i CharacterManager.obj
 0001:000c3770       ?CheckIfModelSKELLoaded@CharacterManager@@QEAAPEAVCSkel@@AEBV?$CryStringT@D@@I@Z 00000000315c4770 f   CharacterManager.obj
 0001:000c3860       ?CheckIfModelSKINLoaded@CharacterManager@@QEAAPEAVCSkin@@AEBV?$CryStringT@D@@I@Z 00000000315c4860 f   CharacterManager.obj
 0001:000c3950       ?GetStatistics@CharacterManager@@UEAAXAEAUStatistics@ICharacterManager@@@Z 00000000315c4950 f   CharacterManager.obj
 0001:000c39d0       ?GetCharacterInstancesSize@CharacterManager@@QEBAXPEAVICrySizer@@@Z 00000000315c49d0 f   CharacterManager.obj
 0001:000c3ac0       ?GetModelByAimPoseID@CharacterManager@@QEAAPEAVCSkel@@I@Z 00000000315c4ac0 f   CharacterManager.obj
 0001:000c3d10       ?TrackSkinTransMemory@CharacterManager@@AEAAIAEAV?$vector@PEAVCSkel@@V?$allocator@PEAVCSkel@@@stlpmtx_std@@@stlpmtx_std@@AEAV?$vector@PEAVCSkin@@V?$allocator@PEAVCSkin@@@stlpmtx_std@@@3@@Z 00000000315c4d10 f   CharacterManager.obj
 0001:000c3e70       ?DebugModelCache@CharacterManager@@AEAAXIAEAV?$vector@PEAVCSkel@@V?$allocator@PEAVCSkel@@@stlpmtx_std@@@stlpmtx_std@@AEAV?$vector@PEAVCSkin@@V?$allocator@PEAVCSkin@@@stlpmtx_std@@@3@@Z 00000000315c4e70 f   CharacterManager.obj
 0001:000c4b40       ?GetAnimationSetUsedInCharEdit@CharacterManager@@QEAAPEAVCAnimationSet@@XZ 00000000315c5b40 f   CharacterManager.obj
 0001:000c4ca0       ?DatabaseUnloading@CharacterManager@@QEAAXXZ 00000000315c5ca0 f   CharacterManager.obj
 0001:000c5090       ?SaveCAF@CAnimationStatsResourceList@@QEAAXXZ 00000000315c6090 f i CharacterManager.obj
 0001:000c5270       ?SaveLMG@CAnimationStatsResourceList@@QEAAXXZ 00000000315c6270 f i CharacterManager.obj
 0001:000c5400       ?GetLoadedModels@CharacterManager@@UEAAXPEAPEAUICharacterModel@@AEAH@Z 00000000315c6400 f   CharacterManager.obj
 0001:000c5450       ?set_size@?$SmallDynStorage@UGlobalAnimationHeaderCAF@@HUStandardAlloc@NAlloc@@@NArray@@QEAAXH@Z 00000000315c6450 f i CharacterManager.obj
 0001:000c5500       ?set_size@?$SmallDynStorage@UGlobalAnimationHeaderAIM@@HUStandardAlloc@NAlloc@@@NArray@@QEAAXH@Z 00000000315c6500 f i CharacterManager.obj
 0001:000c55c0       ??$AddObject@PEAVCSkel@@V?$allocator@PEAVCSkel@@@stlpmtx_std@@@ICrySizer@@QEAAXAEBV?$vector@PEAVCSkel@@V?$allocator@PEAVCSkel@@@stlpmtx_std@@@stlpmtx_std@@@Z 00000000315c65c0 f i CharacterManager.obj
 0001:000c5640       ??$_M_allocate_and_copy@PEAPEAX@?$_Impl_vector@PEAXV?$allocator@PEAX@stlpmtx_std@@@priv@stlpmtx_std@@AEAAPEAPEAXAEA_KPEAPEAX1@Z 00000000315c6640 f i CharacterManager.obj
 0001:000c5640       ??$_M_allocate_and_copy@PEBQEAX@?$_Impl_vector@PEAXV?$allocator@PEAX@stlpmtx_std@@@priv@stlpmtx_std@@AEAAPEAPEAXAEA_KPEBQEAX1@Z 00000000315c6640 f i LoaderSKIN.obj
 0001:000c56f0       ?_M_create_node@?$_Rb_tree@IU?$less@I@stlpmtx_std@@U?$pair@$$CBIV?$_smart_ptr@UIPlaceholderCharacter@@@@@2@U?$_Select1st@U?$pair@$$CBIV?$_smart_ptr@UIPlaceholderCharacter@@@@@stlpmtx_std@@@priv@2@U?$_MapTraitsT@U?$pair@$$CBIV?$_smart_ptr@UIPlaceholderCharacter@@@@@stlpmtx_std@@@52@V?$allocator@U?$pair@$$CBIV?$_smart_ptr@UIPlaceholderCharacter@@@@@stlpmtx_std@@@2@@priv@stlpmtx_std@@IEAAPEAU_Rb_tree_node_base@23@AEBU?$pair@$$CBIV?$_smart_ptr@UIPlaceholderCharacter@@@@@3@@Z 00000000315c66f0 f i CharacterManager.obj
 0001:000c5770       ?_M_create_node@?$_Rb_tree@V?$CryStringT@D@@U?$less@V?$CryStringT@D@@@stlpmtx_std@@V1@U?$_Identity@V?$CryStringT@D@@@priv@3@U?$_SetTraitsT@V?$CryStringT@D@@@53@V?$allocator@V?$CryStringT@D@@@3@@priv@stlpmtx_std@@IEAAPEAU_Rb_tree_node_base@23@AEBV?$CryStringT@D@@@Z 00000000315c6770 f i CharacterManager.obj
 0001:000c57f0       ?GetMemoryUsage@CharacterAttachment@@QEBAXPEAVICrySizer@@@Z 00000000315c67f0 f i CharacterManager.obj
 0001:000c5870       ?clear@?$_Rb_tree@IU?$less@I@stlpmtx_std@@U?$pair@$$CBIUSFacialDisplaceInfo@CFacialModel@@@2@U?$_Select1st@U?$pair@$$CBIUSFacialDisplaceInfo@CFacialModel@@@stlpmtx_std@@@priv@2@U?$_MapTraitsT@U?$pair@$$CBIUSFacialDisplaceInfo@CFacialModel@@@stlpmtx_std@@@52@V?$allocator@U?$pair@$$CBIUSFacialDisplaceInfo@CFacialModel@@@stlpmtx_std@@@2@@priv@stlpmtx_std@@QEAAXXZ 00000000315c6870 f i SkeletonAnim.obj
 0001:000c5870       ?clear@?$_Rb_tree@IU?$less@I@stlpmtx_std@@U?$pair@$$CBI_K@2@U?$_Select1st@U?$pair@$$CBI_K@stlpmtx_std@@@priv@2@U?$_MapTraitsT@U?$pair@$$CBI_K@stlpmtx_std@@@52@V?$allocator@U?$pair@$$CBI_K@stlpmtx_std@@@2@@priv@stlpmtx_std@@QEAAXXZ 00000000315c6870 f i CharacterManager.obj
 0001:000c5870       ?clear@?$_Rb_tree@IU?$less@I@stlpmtx_std@@U?$pair@$$CBIPEAV?$vector@HV?$allocator@H@stlpmtx_std@@@stlpmtx_std@@@2@U?$_Select1st@U?$pair@$$CBIPEAV?$vector@HV?$allocator@H@stlpmtx_std@@@stlpmtx_std@@@stlpmtx_std@@@priv@2@U?$_MapTraitsT@U?$pair@$$CBIPEAV?$vector@HV?$allocator@H@stlpmtx_std@@@stlpmtx_std@@@stlpmtx_std@@@52@V?$allocator@U?$pair@$$CBIPEAV?$vector@HV?$allocator@H@stlpmtx_std@@@stlpmtx_std@@@stlpmtx_std@@@2@@priv@stlpmtx_std@@QEAAXXZ 00000000315c6870 f i CharacterManager.obj
 0001:000c5870       ?clear@?$_Rb_tree@PEAUIFacialEffector@@U?$less@PEAUIFacialEffector@@@stlpmtx_std@@U?$pair@QEAUIFacialEffector@@PEAU1@@3@U?$_Select1st@U?$pair@QEAUIFacialEffector@@PEAU1@@stlpmtx_std@@@priv@3@U?$_MapTraitsT@U?$pair@QEAUIFacialEffector@@PEAU1@@stlpmtx_std@@@63@V?$allocator@U?$pair@QEAUIFacialEffector@@PEAU1@@stlpmtx_std@@@3@@priv@stlpmtx_std@@QEAAXXZ 00000000315c6870 f i FaceEffectorLibrary.obj
 0001:000c5870       ?clear@?$_Rb_tree@IU?$less@I@stlpmtx_std@@U?$pair@$$CBIPEAV?$vector@IV?$allocator@I@stlpmtx_std@@@stlpmtx_std@@@2@U?$_Select1st@U?$pair@$$CBIPEAV?$vector@IV?$allocator@I@stlpmtx_std@@@stlpmtx_std@@@stlpmtx_std@@@priv@2@U?$_MapTraitsT@U?$pair@$$CBIPEAV?$vector@IV?$allocator@I@stlpmtx_std@@@stlpmtx_std@@@stlpmtx_std@@@52@V?$allocator@U?$pair@$$CBIPEAV?$vector@IV?$allocator@I@stlpmtx_std@@@stlpmtx_std@@@stlpmtx_std@@@2@@priv@stlpmtx_std@@QEAAXXZ 00000000315c6870 f i CharacterManager.obj
 0001:000c58e0       ?expand_raw@?$DynArray@IHU?$SmallDynStorage@IHUStandardAlloc@NAlloc@@@NArray@@@@IEAAPEAIPEAIH@Z 00000000315c68e0 f i CharacterManager.obj
 0001:000c5980       ?get_alloc_size@?$SmallDynStorage@UCharacterAttachment@@HUStandardAlloc@NAlloc@@@NArray@@QEBAHXZ 00000000315c6980 f i CharacterManager.obj
 0001:000c59e0       ?init@?$DynArray@UCharacterAttachment@@HU?$SmallDynStorage@UCharacterAttachment@@HUStandardAlloc@NAlloc@@@NArray@@@@KAPEAUCharacterAttachment@@U?$Array@UCharacterAttachment@@HU?$ArrayStorage@UCharacterAttachment@@H@NArray@@@@PEBU2@@Z 00000000315c69e0 f i CharacterManager.obj
 0001:000c5b70       ?expand_raw@?$DynArray@UBSBlendable@@HU?$SmallDynStorage@UBSBlendable@@HUStandardAlloc@NAlloc@@@NArray@@@@IEAAPEAUBSBlendable@@PEAU2@H@Z 00000000315c6b70 f i CharacterManager.obj
 0001:000c5c30       ?expand_raw@?$DynArray@UVirtualExampleInit2@CHUNK_GAHAIM_INFO@@HU?$SmallDynStorage@UVirtualExampleInit2@CHUNK_GAHAIM_INFO@@HUStandardAlloc@NAlloc@@@NArray@@@@IEAAPEAUVirtualExampleInit2@CHUNK_GAHAIM_INFO@@PEAU23@H@Z 00000000315c6c30 f i CharacterManager.obj
 0001:000c5cf0       ?CheckIfPlaceholderCharacterLoaded@CharacterManager@@QEBA?AV?$_smart_ptr@UIPlaceholderCharacter@@@@PEBD@Z 00000000315c6cf0 f   CharacterManager.obj
 0001:000c5df0       ?UnregisterModelSKEL@CharacterManager@@QEAAXPEAVCSkel@@@Z 00000000315c6df0 f   CharacterManager.obj
 0001:000c6020       ?UnregisterModelSKIN@CharacterManager@@QEAAXPEAVCSkin@@@Z 00000000315c7020 f   CharacterManager.obj
 0001:000c6250       ?TrackMemoryOfModels@CharacterManager@@QEAAXXZ 00000000315c7250 f   CharacterManager.obj
 0001:000c6290       ?ClearPoseModifiersFromSynchQueue@CharacterManager@@AEAAXXZ 00000000315c7290 f   CharacterManager.obj
 0001:000c63a0       ?PreloadModelsCHR@CharacterManager@@AEAAXXZ 00000000315c73a0 f   CharacterManager.obj
 0001:000c6920       ?Enable@CLogIndenter@@QEAAX_NPEBDZZ 00000000315c7920 f i CharacterManager.obj
 0001:000c6a10       ?pop_back@?$DynArray@UDebugInstances@@HU?$SmallDynStorage@UDebugInstances@@HUStandardAlloc@NAlloc@@@NArray@@@@QEAAXH@Z 00000000315c7a10 f i CharacterManager.obj
 0001:000c6aa0       ?reserve@?$_Impl_vector@PEAXV?$allocator@PEAX@stlpmtx_std@@@priv@stlpmtx_std@@QEAAX_K@Z 00000000315c7aa0 f i CharacterManager.obj
 0001:000c6b60       ?_M_erase@?$_Rb_tree@IU?$less@I@stlpmtx_std@@U?$pair@$$CBIV?$_smart_ptr@UIPlaceholderCharacter@@@@@2@U?$_Select1st@U?$pair@$$CBIV?$_smart_ptr@UIPlaceholderCharacter@@@@@stlpmtx_std@@@priv@2@U?$_MapTraitsT@U?$pair@$$CBIV?$_smart_ptr@UIPlaceholderCharacter@@@@@stlpmtx_std@@@52@V?$allocator@U?$pair@$$CBIV?$_smart_ptr@UIPlaceholderCharacter@@@@@stlpmtx_std@@@2@@priv@stlpmtx_std@@AEAAXPEAU_Rb_tree_node_base@23@@Z 00000000315c7b60 f i CharacterManager.obj
 0001:000c6bc0       ??$move_init@UDebugInstances@@@NArray@@YAXPEAUDebugInstances@@0_K@Z 00000000315c7bc0 f i CharacterManager.obj
 0001:000c6c90       ??$_M_find@V?$CryStackStringT@D$0CAA@@@@?$_Rb_tree@V?$CryStringT@D@@U?$less@V?$CryStringT@D@@@stlpmtx_std@@V1@U?$_Identity@V?$CryStringT@D@@@priv@3@U?$_SetTraitsT@V?$CryStringT@D@@@53@V?$allocator@V?$CryStringT@D@@@3@@priv@stlpmtx_std@@AEBAPEAU_Rb_tree_node_base@12@AEBV?$CryStackStringT@D$0CAA@@@@Z 00000000315c7c90 f i CharacterManager.obj
 0001:000c6e60       ?append_raw@?$DynArray@IHU?$SmallDynStorage@IHUStandardAlloc@NAlloc@@@NArray@@@@QEAA?AU?$Array@IHU?$ArrayStorage@IH@NArray@@@@H@Z 00000000315c7e60 f i CharacterManager.obj
 0001:000c6f20       ??$AddObject@UCharacterAttachment@@HU?$SmallDynStorage@UCharacterAttachment@@HUStandardAlloc@NAlloc@@@NArray@@@ICrySizer@@QEAAXAEBU?$DynArray@UCharacterAttachment@@HU?$SmallDynStorage@UCharacterAttachment@@HUStandardAlloc@NAlloc@@@NArray@@@@@Z 00000000315c7f20 f i CharacterManager.obj
 0001:000c6fd0       ?init@?$DynArray@UBSParameter@@HU?$SmallDynStorage@UBSParameter@@HUStandardAlloc@NAlloc@@@NArray@@@@KAPEAUBSParameter@@U?$Array@UBSParameter@@HU?$ArrayStorage@UBSParameter@@H@NArray@@@@PEBU2@@Z 00000000315c7fd0 f i CharacterManager.obj
 0001:000c7090       ?append_raw@?$DynArray@V?$_smart_ptr@VIController@@@@HU?$SmallDynStorage@V?$_smart_ptr@VIController@@@@HUStandardAlloc@NAlloc@@@NArray@@@@QEAA?AU?$Array@V?$_smart_ptr@VIController@@@@HU?$ArrayStorage@V?$_smart_ptr@VIController@@@@H@NArray@@@@H@Z 00000000315c8090 f i CharacterManager.obj
 0001:000c7150       ??$move_init@USCRCName@@@NArray@@YAXPEAUSCRCName@@0_K@Z 00000000315c8150 f i CharacterManager.obj
 0001:000c7220       ?StopAnimationsOnAllInstances@CharacterManager@@QEAAXXZ 00000000315c8220 f   CharacterManager.obj
 0001:000c74d0       ?RemoveAnimationToSyncQueue@CharacterManager@@UEAAXPEAUICharacterInstance@@@Z 00000000315c84d0 f   CharacterManager.obj
 0001:000c75f0       ?DBA_Unload_All@CharacterManager@@UEAA_NXZ 00000000315c85f0 f   CharacterManager.obj
 0001:000c7630       ?CAF_AddRef@CharacterManager@@UEAA_NI@Z 00000000315c8630 f   CharacterManager.obj
 0001:000c76e0       ?CAF_IsLoaded@CharacterManager@@UEBA_NI@Z 00000000315c86e0 f   CharacterManager.obj
 0001:000c7770       ?CAF_Release@CharacterManager@@UEAA_NI@Z 00000000315c8770 f   CharacterManager.obj
 0001:000c77f0       ?CAF_LoadSynchronously@CharacterManager@@UEAA_NI@Z 00000000315c87f0 f   CharacterManager.obj
 0001:000c78f0       ??1?$DynArray@UDebugInstances@@HU?$SmallDynStorage@UDebugInstances@@HUStandardAlloc@NAlloc@@@NArray@@@@QEAA@XZ 00000000315c88f0 f i CharacterManager.obj
 0001:000c7970       ??1?$DynArray@V?$TCBSpline@U?$Vec3_tpl@M@@U?$TCBSplineKey@U?$Vec3_tpl@M@@@spline@@@spline@@HU?$SmallDynStorage@V?$TCBSpline@U?$Vec3_tpl@M@@U?$TCBSplineKey@U?$Vec3_tpl@M@@@spline@@@spline@@HUStandardAlloc@NAlloc@@@NArray@@@@QEAA@XZ 00000000315c8970 f i CharacterManager.obj
 0001:000c7970       ??1?$DynArray@VTCBAngleAxisSpline@spline@@HU?$SmallDynStorage@VTCBAngleAxisSpline@spline@@HUStandardAlloc@NAlloc@@@NArray@@@@QEAA@XZ 00000000315c8970 f i CharacterManager.obj
 0001:000c79f0       ??1?$DynArray@UCControllerTCB@@HU?$SmallDynStorage@UCControllerTCB@@HUStandardAlloc@NAlloc@@@NArray@@@@QEAA@XZ 00000000315c89f0 f i CharacterManager.obj
 0001:000c7a70       ?erase@?$_Rb_tree@V?$CryStringT@D@@U?$less@V?$CryStringT@D@@@stlpmtx_std@@V1@U?$_Identity@V?$CryStringT@D@@@priv@3@U?$_SetTraitsT@V?$CryStringT@D@@@53@V?$allocator@V?$CryStringT@D@@@3@@priv@stlpmtx_std@@QEAAXU?$_Rb_tree_iterator@V?$CryStringT@D@@U?$_SetTraitsT@V?$CryStringT@D@@@priv@stlpmtx_std@@@23@@Z 00000000315c8a70 f i CharacterManager.obj
 0001:000c7ae0       ?resize_raw@?$SmallDynStorage@UDebugInstances@@HUStandardAlloc@NAlloc@@@NArray@@QEAAXHH_N@Z 00000000315c8ae0 f i CharacterManager.obj
 0001:000c7c60       ?_M_erase@?$_Rb_tree@V?$CryStringT@D@@U?$less@V?$CryStringT@D@@@stlpmtx_std@@V1@U?$_Identity@V?$CryStringT@D@@@priv@3@U?$_SetTraitsT@V?$CryStringT@D@@@53@V?$allocator@V?$CryStringT@D@@@3@@priv@stlpmtx_std@@AEAAXPEAU_Rb_tree_node_base@23@@Z 00000000315c8c60 f i CharacterManager.obj
 0001:000c7ce0       ?insert_unique@?$_Rb_tree@V?$CryStringT@D@@U?$less@V?$CryStringT@D@@@stlpmtx_std@@V1@U?$_Identity@V?$CryStringT@D@@@priv@3@U?$_SetTraitsT@V?$CryStringT@D@@@53@V?$allocator@V?$CryStringT@D@@@3@@priv@stlpmtx_std@@QEAA?AU?$pair@U?$_Rb_tree_iterator@V?$CryStringT@D@@U?$_SetTraitsT@V?$CryStringT@D@@@priv@stlpmtx_std@@@priv@stlpmtx_std@@_N@3@AEBV?$CryStringT@D@@@Z 00000000315c8ce0 f i CharacterManager.obj
 0001:000c7f70       ?insert_unique@?$_Rb_tree@IU?$less@I@stlpmtx_std@@U?$pair@$$CBIV?$_smart_ptr@UIPlaceholderCharacter@@@@@2@U?$_Select1st@U?$pair@$$CBIV?$_smart_ptr@UIPlaceholderCharacter@@@@@stlpmtx_std@@@priv@2@U?$_MapTraitsT@U?$pair@$$CBIV?$_smart_ptr@UIPlaceholderCharacter@@@@@stlpmtx_std@@@52@V?$allocator@U?$pair@$$CBIV?$_smart_ptr@UIPlaceholderCharacter@@@@@stlpmtx_std@@@2@@priv@stlpmtx_std@@QEAA?AU?$pair@U?$_Rb_tree_iterator@U?$pair@$$CBIV?$_smart_ptr@UIPlaceholderCharacter@@@@@stlpmtx_std@@U?$_MapTraitsT@U?$pair@$$CBIV?$_smart_ptr@UIPlaceholderCharacter@@@@@stlpmtx_std@@@priv@2@@priv@stlpmtx_std@@_N@3@AEBU?$pair@$$CBIV?$_smart_ptr@UIPlaceholderCharacter@@@@@3@@Z 00000000315c8f70 f i CharacterManager.obj
 0001:000c8170       ?_M_clear@?$_Impl_vector@UCharacterDefinition@@V?$allocator@UCharacterDefinition@@@stlpmtx_std@@@priv@stlpmtx_std@@AEAAXXZ 00000000315c9170 f i CharacterManager.obj
 0001:000c81d0       ??1?$DynArray@UCGlobalHeaderDBA@@HU?$SmallDynStorage@UCGlobalHeaderDBA@@HUStandardAlloc@NAlloc@@@NArray@@@@QEAA@XZ 00000000315c91d0 f i CharacterManager.obj
 0001:000c8250       ?resize_raw@?$SmallDynStorage@UCGlobalHeaderDBA@@HUStandardAlloc@NAlloc@@@NArray@@QEAAXHH_N@Z 00000000315c9250 f i CharacterManager.obj
 0001:000c83e0       ??0?$DynArray@IHU?$SmallDynStorage@IHUStandardAlloc@NAlloc@@@NArray@@@@QEAA@AEBU0@@Z 00000000315c93e0 f i CharacterManager.obj
 0001:000c84a0       ?pop_back@?$DynArray@UCharacterAttachment@@HU?$SmallDynStorage@UCharacterAttachment@@HUStandardAlloc@NAlloc@@@NArray@@@@QEAAXH@Z 00000000315c94a0 f i CharacterManager.obj
 0001:000c8530       ?resize_raw@?$SmallDynStorage@USCRCName@@HUStandardAlloc@NAlloc@@@NArray@@QEAAXHH_N@Z 00000000315c9530 f i CharacterManager.obj
 0001:000c86a0       ??$move_init@UBSParameter@@@NArray@@YAXPEAUBSParameter@@0_K@Z 00000000315c96a0 f i CharacterManager.obj
 0001:000c87c0       ??$move_init@UBlendSpaceInfo@@@NArray@@YAXPEAUBlendSpaceInfo@@0_K@Z 00000000315c97c0 f i CharacterManager.obj
 0001:000c8880       ??1CryCGALoader@@QEAA@XZ   00000000315c9880 f i CharacterManager.obj
 0001:000c8930       ??1?$_Impl_vector@UCharacterDefinition@@V?$allocator@UCharacterDefinition@@@stlpmtx_std@@@priv@stlpmtx_std@@QEAA@XZ 00000000315c9930 f i CharacterManager.obj
 0001:000c89a0       ?expand_raw@?$DynArray@UDebugInstances@@HU?$SmallDynStorage@UDebugInstances@@HUStandardAlloc@NAlloc@@@NArray@@@@IEAAPEAUDebugInstances@@PEAU2@H@Z 00000000315c99a0 f i CharacterManager.obj
 0001:000c8a60       ??1GlobalAnimationHeaderCAF@@QEAA@XZ 00000000315c9a60 f i CharacterManager.obj
 0001:000c8b20       ??0AnimSearchHelper@@QEAA@XZ 00000000315c9b20 f i CharacterManager.obj
 0001:000c8bc0       ?destroy@?$DynArray@UBSParameter@@HU?$SmallDynStorage@UBSParameter@@HUStandardAlloc@NAlloc@@@NArray@@@@IEAAXXZ 00000000315c9bc0 f i CharacterManager.obj
 0001:000c8c40       ??0?$DynArray@UBSBlendable@@HU?$SmallDynStorage@UBSBlendable@@HUStandardAlloc@NAlloc@@@NArray@@@@QEAA@AEBU0@@Z 00000000315c9c40 f i CharacterManager.obj
 0001:000c8d10       ??0?$DynArray@UVirtualExample1D@@HU?$SmallDynStorage@UVirtualExample1D@@HUStandardAlloc@NAlloc@@@NArray@@@@QEAA@AEBU0@@Z 00000000315c9d10 f i CharacterManager.obj
 0001:000c8de0       ??0?$DynArray@UVirtualExample2D@@HU?$SmallDynStorage@UVirtualExample2D@@HUStandardAlloc@NAlloc@@@NArray@@@@QEAA@AEBU0@@Z 00000000315c9de0 f i CharacterManager.obj
 0001:000c8ec0       ??0?$DynArray@UVirtualExample3D@@HU?$SmallDynStorage@UVirtualExample3D@@HUStandardAlloc@NAlloc@@@NArray@@@@QEAA@AEBU0@@Z 00000000315c9ec0 f i CharacterManager.obj
 0001:000c8fa0       ??0?$DynArray@V?$_smart_ptr@VIController@@@@HU?$SmallDynStorage@V?$_smart_ptr@VIController@@@@HUStandardAlloc@NAlloc@@@NArray@@@@QEAA@AEBU0@@Z 00000000315c9fa0 f i CharacterManager.obj
 0001:000c9080       ??0?$DynArray@UVirtualExampleInit2@CHUNK_GAHAIM_INFO@@HU?$SmallDynStorage@UVirtualExampleInit2@CHUNK_GAHAIM_INFO@@HUStandardAlloc@NAlloc@@@NArray@@@@QEAA@AEBU0@@Z 00000000315ca080 f i CharacterManager.obj
 0001:000c9170       ?erase@?$DynArray@UCharacterAttachment@@HU?$SmallDynStorage@UCharacterAttachment@@HUStandardAlloc@NAlloc@@@NArray@@@@QEAAPEAUCharacterAttachment@@PEAU2@0@Z 00000000315ca170 f i CharacterManager.obj
 0001:000c9220       ?resize_raw@?$SmallDynStorage@UBSParameter@@HUStandardAlloc@NAlloc@@@NArray@@QEAAXHH_N@Z 00000000315ca220 f i CharacterManager.obj
 0001:000c93a0       ?resize_raw@?$SmallDynStorage@UBlendSpaceInfo@@HUStandardAlloc@NAlloc@@@NArray@@QEAAXHH_N@Z 00000000315ca3a0 f i CharacterManager.obj
 0001:000c9510       ??0CryCGALoader@@QEAA@XZ   00000000315ca510 f i CharacterManager.obj
 0001:000c96c0       ?RegisterModelSKEL@CharacterManager@@QEAAXPEAVCSkel@@I@Z 00000000315ca6c0 f   CharacterManager.obj
 0001:000c9800       ?RegisterModelSKIN@CharacterManager@@QEAAXPEAVCSkin@@I@Z 00000000315ca800 f   CharacterManager.obj
 0001:000c9940       ?ReloadAllCHRPARAMS@CharacterManager@@AEAAXXZ 00000000315ca940 f   CharacterManager.obj
 0001:000ca040       ?Add@CAnimationStatsResourceList@@QEAAXPEBD@Z 00000000315cb040 f i CharacterManager.obj
 0001:000ca250       ?IsExist@CAnimationStatsResourceList@@QEAA_NPEBD@Z 00000000315cb250 f i CharacterManager.obj
 0001:000ca3f0       ?LoadCAF@CAnimationStatsResourceList@@QEAAXPEBD@Z 00000000315cb3f0 f i CharacterManager.obj
 0001:000ca510       ?LoadLMG@CAnimationStatsResourceList@@QEAAXPEBD@Z 00000000315cb510 f i CharacterManager.obj
 0001:000ca630       ?SyncAllAnimations@CharacterManager@@UEAAXXZ 00000000315cb630 f   CharacterManager.obj
 0001:000ca7d0       ?AddAnimationToSyncQueue@CharacterManager@@UEAAXPEAUICharacterInstance@@@Z 00000000315cb7d0 f   CharacterManager.obj
 0001:000ca840       ?PreloadModelsCGA@CharacterManager@@AEAAXXZ 00000000315cb840 f   CharacterManager.obj
 0001:000cac60       ??$AddObject@UCharacterDefinition@@V?$allocator@UCharacterDefinition@@@stlpmtx_std@@@ICrySizer@@QEAAXAEBV?$vector@UCharacterDefinition@@V?$allocator@UCharacterDefinition@@@stlpmtx_std@@@stlpmtx_std@@@Z 00000000315cbc60 f i CharacterManager.obj
 0001:000cad70       ??0GlobalAnimationHeaderCAF@@QEAA@XZ 00000000315cbd70 f i CharacterManager.obj
 0001:000caec0       ??4?$DynArray@UCharacterAttachment@@HU?$SmallDynStorage@UCharacterAttachment@@HUStandardAlloc@NAlloc@@@NArray@@@@QEAAAEAU0@U?$Array@$$CBUCharacterAttachment@@HU?$ArrayStorage@$$CBUCharacterAttachment@@H@NArray@@@@@Z 00000000315cbec0 f i CharacterManager.obj
 0001:000cb020       ?append_raw@?$DynArray@USCRCName@@HU?$SmallDynStorage@USCRCName@@HUStandardAlloc@NAlloc@@@NArray@@@@QEAA?AU?$Array@USCRCName@@HU?$ArrayStorage@USCRCName@@H@NArray@@@@H@Z 00000000315cc020 f i CharacterManager.obj
 0001:000cb0e0       ?FetchModelSKIN@CharacterManager@@QEAA?AV?$_smart_ptr@VCSkin@@@@PEBDI@Z 00000000315cc0e0 f   CharacterManager.obj
 0001:000cb1f0       ?GetMemoryUsage@CharacterManager@@UEBAXPEAVICrySizer@@@Z 00000000315cc1f0 f   CharacterManager.obj
 0001:000cb370       ?Remove@CAnimationStatsResourceList@@QEAAXPEBD@Z 00000000315cc370 f i CharacterManager.obj
 0001:000cb600       ?init@?$DynArray@UAimIKPose@@HU?$SmallDynStorage@UAimIKPose@@HUStandardAlloc@NAlloc@@@NArray@@@@KAPEAUAimIKPose@@U?$Array@UAimIKPose@@HU?$ArrayStorage@UAimIKPose@@H@NArray@@@@@Z 00000000315cc600 f i CharacterManager.obj
 0001:000cb7f0       ??$reconstruct@V?$map@IV?$_smart_ptr@UIPlaceholderCharacter@@@@U?$less@I@stlpmtx_std@@V?$allocator@U?$pair@$$CBIV?$_smart_ptr@UIPlaceholderCharacter@@@@@stlpmtx_std@@@3@@stlpmtx_std@@@stl@@YAXAEAV?$map@IV?$_smart_ptr@UIPlaceholderCharacter@@@@U?$less@I@stlpmtx_std@@V?$allocator@U?$pair@$$CBIV?$_smart_ptr@UIPlaceholderCharacter@@@@@stlpmtx_std@@@3@@stlpmtx_std@@@Z 00000000315cc7f0 f i CharacterManager.obj
 0001:000cb880       ?InsertValue@CNameCRCMap@@QEAA_NI_K@Z 00000000315cc880 f i CharacterManager.obj
 0001:000cb950       ??1GlobalAnimationHeaderLMG@@QEAA@XZ 00000000315cc950 f i CharacterManager.obj
 0001:000cbc40       ??1CharacterDefinition@@UEAA@XZ 00000000315ccc40 f i CharacterManager.obj
 0001:000cbce0       ?AddRef@CFacialJoystickSet@@UEAAXXZ 00000000315ccce0 f i FaceJoystick.obj
 0001:000cbce0       ?AddRef@CharacterDefinition@@UEAAXXZ 00000000315ccce0 f i CharacterManager.obj
 0001:000cbcf0       ??_GCharacterDefinition@@UEAAPEAXI@Z 00000000315cccf0 f i CharacterManager.obj
 0001:000cbcf0       ??_ECharacterDefinition@@UEAAPEAXI@Z 00000000315cccf0 f i CharacterManager.obj
 0001:000cbd20       ?append_raw@?$DynArray@UBSParameter@@HU?$SmallDynStorage@UBSParameter@@HUStandardAlloc@NAlloc@@@NArray@@@@QEAA?AU?$Array@UBSParameter@@HU?$ArrayStorage@UBSParameter@@H@NArray@@@@H@Z 00000000315ccd20 f i CharacterManager.obj
 0001:000cbde0       ?append_raw@?$DynArray@UBlendSpaceInfo@@HU?$SmallDynStorage@UBlendSpaceInfo@@HUStandardAlloc@NAlloc@@@NArray@@@@QEAA?AU?$Array@UBlendSpaceInfo@@HU?$ArrayStorage@UBlendSpaceInfo@@H@NArray@@@@H@Z 00000000315ccde0 f i CharacterManager.obj
 0001:000cbea0       ??$move_init@UAimIKPose@@@NArray@@YAXPEAUAimIKPose@@0_K@Z 00000000315ccea0 f i CharacterManager.obj
 0001:000cc030       ?LoadModelSKIN@CharacterManager@@UEAA?AV?$_smart_ptr@UISkin@@@@PEBDI@Z 00000000315cd030 f   CharacterManager.obj
 0001:000cc450       ??1?$DynArray@UGlobalAnimationHeaderCAF@@HU?$SmallDynStorage@UGlobalAnimationHeaderCAF@@HUStandardAlloc@NAlloc@@@NArray@@@@QEAA@XZ 00000000315cd450 f i CharacterManager.obj
 0001:000cc4d0       ??0?$DynArray@VCAnimEventData@@HU?$SmallDynStorage@VCAnimEventData@@HUStandardAlloc@NAlloc@@@NArray@@@@QEAA@AEBU0@@Z 00000000315cd4d0 f i CharacterManager.obj
 0001:000cc5b0       ??0?$DynArray@USCRCName@@HU?$SmallDynStorage@USCRCName@@HUStandardAlloc@NAlloc@@@NArray@@@@QEAA@AEBU0@@Z 00000000315cd5b0 f i CharacterManager.obj
 0001:000cc690       ?resize_raw@?$SmallDynStorage@UAimIKPose@@HUStandardAlloc@NAlloc@@@NArray@@QEAAXHH_N@Z 00000000315cd690 f i CharacterManager.obj
 0001:000cc800       ?CreateDebugInstances@CharacterManager@@UEAAXPEBD@Z 00000000315cd800 f   CharacterManager.obj
 0001:000cc9a0       ?DumpAssetStatistics@CharacterManager@@AEAAXXZ 00000000315cd9a0 f   CharacterManager.obj
 0001:000cd1b0       ?ReleaseCDF@CharacterManager@@QEAAXPEBD@Z 00000000315ce1b0 f   CharacterManager.obj
 0001:000cd3d0       ??0?$DynArray@UCharacterAttachment@@HU?$SmallDynStorage@UCharacterAttachment@@HUStandardAlloc@NAlloc@@@NArray@@@@QEAA@AEBU0@@Z 00000000315ce3d0 f i CharacterManager.obj
 0001:000cd490       ??$__copy@PEAUCharacterDefinition@@PEAU1@_J@priv@stlpmtx_std@@YAPEAUCharacterDefinition@@PEAU2@00AEBUrandom_access_iterator_tag@1@PEA_J@Z 00000000315ce490 f i CharacterManager.obj
 0001:000cd590       ??0?$DynArray@UBSParameter@@HU?$SmallDynStorage@UBSParameter@@HUStandardAlloc@NAlloc@@@NArray@@@@QEAA@AEBU0@@Z 00000000315ce590 f i CharacterManager.obj
 0001:000cd630       ??0?$DynArray@UBlendSpaceInfo@@HU?$SmallDynStorage@UBlendSpaceInfo@@HUStandardAlloc@NAlloc@@@NArray@@@@QEAA@AEBU0@@Z 00000000315ce630 f i CharacterManager.obj
 0001:000cd710       ?init@?$DynArray@UGlobalAnimationHeaderAIM@@HU?$SmallDynStorage@UGlobalAnimationHeaderAIM@@HUStandardAlloc@NAlloc@@@NArray@@@@KAPEAUGlobalAnimationHeaderAIM@@U?$Array@UGlobalAnimationHeaderAIM@@HU?$ArrayStorage@UGlobalAnimationHeaderAIM@@H@NArray@@@@@Z 00000000315ce710 f i CharacterManager.obj
 0001:000cd9f0       ??1?$DynArray@UGlobalAnimationHeaderLMG@@HU?$SmallDynStorage@UGlobalAnimationHeaderLMG@@HUStandardAlloc@NAlloc@@@NArray@@@@QEAA@XZ 00000000315ce9f0 f i CharacterManager.obj
 0001:000cda70       ??0GlobalAnimationHeaderLMG@@QEAA@AEBU0@@Z 00000000315cea70 f i CharacterManager.obj
 0001:000cdef0       ?append_raw@?$DynArray@UAimIKPose@@HU?$SmallDynStorage@UAimIKPose@@HUStandardAlloc@NAlloc@@@NArray@@@@QEAA?AU?$Array@UAimIKPose@@HU?$ArrayStorage@UAimIKPose@@H@NArray@@@@H@Z 00000000315ceef0 f i CharacterManager.obj
 0001:000cdfb0       ?pop_back@?$DynArray@UGlobalAnimationHeaderAIM@@HU?$SmallDynStorage@UGlobalAnimationHeaderAIM@@HUStandardAlloc@NAlloc@@@NArray@@@@QEAAXH@Z 00000000315cefb0 f i CharacterManager.obj
 0001:000ce040       ?Update@CharacterManager@@UEAAX_N@Z 00000000315cf040 f   CharacterManager.obj
 0001:000cea90       ?resize@?$DynArray@UAimIKPose@@HU?$SmallDynStorage@UAimIKPose@@HUStandardAlloc@NAlloc@@@NArray@@@@QEAAXH@Z 00000000315cfa90 f i CharacterManager.obj
 0001:000ceb30       ??$__ucopy@PEAUCharacterDefinition@@PEAU1@_J@priv@stlpmtx_std@@YAPEAUCharacterDefinition@@PEAU2@00AEBUrandom_access_iterator_tag@1@PEA_J@Z 00000000315cfb30 f i CharacterManager.obj
 0001:000cec10       ??1?$DynArray@UGlobalAnimationHeaderAIM@@HU?$SmallDynStorage@UGlobalAnimationHeaderAIM@@HUStandardAlloc@NAlloc@@@NArray@@@@QEAA@XZ 00000000315cfc10 f i CharacterManager.obj
 0001:000cec90       ?erase@?$_Impl_vector@UCharacterDefinition@@V?$allocator@UCharacterDefinition@@@stlpmtx_std@@@priv@stlpmtx_std@@QEAAPEAUCharacterDefinition@@PEAU4@0@Z 00000000315cfc90 f i CharacterManager.obj
 0001:000ced40       ??$move_init@UGlobalAnimationHeaderLMG@@@NArray@@YAXPEAUGlobalAnimationHeaderLMG@@0_K@Z 00000000315cfd40 f i CharacterManager.obj
 0001:000cedb0       ??0?$DynArray@UAimIKPose@@HU?$SmallDynStorage@UAimIKPose@@HUStandardAlloc@NAlloc@@@NArray@@@@QEAA@AEBU0@@Z 00000000315cfdb0 f i CharacterManager.obj
 0001:000ceea0       ??1CAnimationManager@@UEAA@XZ 00000000315cfea0 f i CharacterManager.obj
 0001:000cefa0       ?GetGlobalAnimCount@CAnimationManager@@UEAA_KXZ 00000000315cffa0 f i CharacterManager.obj
 0001:000cefb0       ??_ECAnimationManager@@UEAAPEAXI@Z 00000000315cffb0 f i CharacterManager.obj
 0001:000cefb0       ??_GCAnimationManager@@UEAAPEAXI@Z 00000000315cffb0 f i CharacterManager.obj
 0001:000cefe0       ?resize_raw@?$SmallDynStorage@UGlobalAnimationHeaderCAF@@HUStandardAlloc@NAlloc@@@NArray@@QEAAXHH_N@Z 00000000315cffe0 f i CharacterManager.obj
 0001:000cf170       ?resize_raw@?$SmallDynStorage@UGlobalAnimationHeaderLMG@@HUStandardAlloc@NAlloc@@@NArray@@QEAAXHH_N@Z 00000000315d0170 f i CharacterManager.obj
 0001:000cf300       ??0GlobalAnimationHeaderAIM@@QEAA@AEBU0@@Z 00000000315d0300 f i CharacterManager.obj
 0001:000cf400       ?clear@?$DynArray@UGlobalAnimationHeaderCAF@@HU?$SmallDynStorage@UGlobalAnimationHeaderCAF@@HUStandardAlloc@NAlloc@@@NArray@@@@QEAAXXZ 00000000315d0400 f i CharacterManager.obj
 0001:000cf4b0       ?expand_raw@?$DynArray@UGlobalAnimationHeaderCAF@@HU?$SmallDynStorage@UGlobalAnimationHeaderCAF@@HUStandardAlloc@NAlloc@@@NArray@@@@IEAAPEAUGlobalAnimationHeaderCAF@@PEAU2@H@Z 00000000315d04b0 f i CharacterManager.obj
 0001:000cf570       ?reserve@?$DynArray@UGlobalAnimationHeaderCAF@@HU?$SmallDynStorage@UGlobalAnimationHeaderCAF@@HUStandardAlloc@NAlloc@@@NArray@@@@QEAAXH@Z 00000000315d0570 f i CharacterManager.obj
 0001:000cf5d0       ?CleanupModelCache@CharacterManager@@QEAAX_N@Z 00000000315d05d0 f   CharacterManager.obj
 0001:000cf700       ?ClearResources@CharacterManager@@UEAAX_N@Z 00000000315d0700 f   CharacterManager.obj
 0001:000cf780       ??1CharacterManager@@UEAA@XZ 00000000315d0780 f   CharacterManager.obj
 0001:000cf9f0       ?SetAnimMemoryTracker@CharacterManager@@UEAAXAEBUSAnimMemoryTracker@@@Z 00000000315d09f0 f i CharacterManager.obj
 0001:000cfa50       ?GetAnimMemoryTracker@CharacterManager@@UEAA?AUSAnimMemoryTracker@@XZ 00000000315d0a50 f i CharacterManager.obj
 0001:000cfac0       ?ReloadCAF@CharacterManager@@UEAAHPEBD@Z 00000000315d0ac0 f i CharacterManager.obj
 0001:000cfae0       ?ReloadLMG@CharacterManager@@UEAAHPEBD@Z 00000000315d0ae0 f i CharacterManager.obj
 0001:000cfb00       ?SetStreamingListener@CharacterManager@@UEAAXPEAUIAnimationStreamingListener@@@Z 00000000315d0b00 f i CharacterManager.obj
 0001:000cfb10       ?AddFrameTicks@CharacterManager@@UEAAX_K@Z 00000000315d0b10 f i CharacterManager.obj
 0001:000cfb20       ?AddFrameSyncTicks@CharacterManager@@UEAAX_K@Z 00000000315d0b20 f i CharacterManager.obj
 0001:000cfb30       ?ResetFrameTicks@CharacterManager@@UEAAXXZ 00000000315d0b30 f i CharacterManager.obj
 0001:000cfb50       ?GetNamePART@CSkel@@UEBAPEBDXZ 00000000315d0b50 f i Model.obj
 0001:000cfb50       ?NumFrameTicks@CharacterManager@@UEBA_KXZ 00000000315d0b50 f i CharacterManager.obj
 0001:000cfb60       ?NumFrameSyncTicks@CharacterManager@@UEBA_KXZ 00000000315d0b60 f i CharacterManager.obj
 0001:000cfb70       ?NumCharacters@CharacterManager@@UEBAIXZ 00000000315d0b70 f i CharacterManager.obj
 0001:000cfb80       ?GetIAnimEvents@CharacterManager@@UEAAPEAUIAnimEvents@@XZ 00000000315d0b80 f i CharacterManager.obj
 0001:000cfb90       ?ClearCDFCache@CharacterManager@@EEAAXXZ 00000000315d0b90 f i CharacterManager.obj
 0001:000cfbb0       ??$move_init@UGlobalAnimationHeaderAIM@@@NArray@@YAXPEAUGlobalAnimationHeaderAIM@@0_K@Z 00000000315d0bb0 f i CharacterManager.obj
 0001:000cfc20       ??_GCharacterManager@@UEAAPEAXI@Z 00000000315d0c20 f i CharacterManager.obj
 0001:000cfc20       ??_ECharacterManager@@UEAAPEAXI@Z 00000000315d0c20 f i CharacterManager.obj
 0001:000cfc50       ?grow@?$DynArray@UGlobalAnimationHeaderCAF@@HU?$SmallDynStorage@UGlobalAnimationHeaderCAF@@HUStandardAlloc@NAlloc@@@NArray@@@@QEAAPEAUGlobalAnimationHeaderCAF@@H@Z 00000000315d0c50 f i CharacterManager.obj
 0001:000cfcd0       ?reserve@?$_Impl_vector@UCharacterDefinition@@V?$allocator@UCharacterDefinition@@@stlpmtx_std@@@priv@stlpmtx_std@@QEAAX_K@Z 00000000315d0cd0 f i CharacterManager.obj
 0001:000cfe60       ?resize_raw@?$SmallDynStorage@UGlobalAnimationHeaderAIM@@HUStandardAlloc@NAlloc@@@NArray@@QEAAXHH_N@Z 00000000315d0e60 f i CharacterManager.obj
 0001:000cfff0       ?resize@?$DynArray@UGlobalAnimationHeaderCAF@@HU?$SmallDynStorage@UGlobalAnimationHeaderCAF@@HUStandardAlloc@NAlloc@@@NArray@@@@QEAAXH@Z 00000000315d0ff0 f i CharacterManager.obj
 0001:000d00a0       ?clear@?$DynArray@UGlobalAnimationHeaderAIM@@HU?$SmallDynStorage@UGlobalAnimationHeaderAIM@@HUStandardAlloc@NAlloc@@@NArray@@@@QEAAXXZ 00000000315d10a0 f i CharacterManager.obj
 0001:000d0140       ?expand_raw@?$DynArray@UGlobalAnimationHeaderAIM@@HU?$SmallDynStorage@UGlobalAnimationHeaderAIM@@HUStandardAlloc@NAlloc@@@NArray@@@@IEAAPEAUGlobalAnimationHeaderAIM@@PEAU2@H@Z 00000000315d1140 f i CharacterManager.obj
 0001:000d0200       ?LoadAnimationImageFileCAF@CharacterManager@@AEAA_NPEBDPEAUIChunkFile@@@Z 00000000315d1200 f   CharacterManager.obj
 0001:000d08f0       ??0CAnimationManager@@QEAA@XZ 00000000315d18f0 f i CharacterManager.obj
 0001:000d0e10       ?LoadCDF@CharacterManager@@QEAAHPEBD@Z 00000000315d1e10 f   CharacterManager.obj
 0001:000d14d0       ?GetOrLoadCDFId@CharacterManager@@QEAAIAEBV?$CryStringT@D@@@Z 00000000315d24d0 f   CharacterManager.obj
 0001:000d1590       ??0CharacterManager@@QEAA@XZ 00000000315d2590 f   CharacterManager.obj
 0001:000d1b50       ?PreloadModelsCDF@CharacterManager@@AEAAXXZ 00000000315d2b50 f   CharacterManager.obj
 0001:000d1e80       ?LoadCharacterDefinition@CharacterManager@@QEAAPEAUICharacterInstance@@V?$CryStringT@D@@I@Z 00000000315d2e80 f   CharacterManager.obj
 0001:000d21e0       ?PreloadLevelModels@CharacterManager@@UEAAXXZ 00000000315d31e0 f   CharacterManager.obj
 0001:000d22a0       ?resize@?$DynArray@UGlobalAnimationHeaderAIM@@HU?$SmallDynStorage@UGlobalAnimationHeaderAIM@@HUStandardAlloc@NAlloc@@@NArray@@@@QEAAXH@Z 00000000315d32a0 f i CharacterManager.obj
 0001:000d2310       ?LoadAnimationImageFileAIM@CharacterManager@@AEAA_NPEBDPEAUIChunkFile@@@Z 00000000315d3310 f   CharacterManager.obj
 0001:000d2b00       ?LoadAnimationImageFile@CharacterManager@@AEAAXPEBD0@Z 00000000315d3b00 f   CharacterManager.obj
 0001:000d2c40       ?FetchModelSKEL@CharacterManager@@QEAA?AV?$_smart_ptr@VCSkel@@@@PEBDI@Z 00000000315d3c40 f   CharacterManager.obj
 0001:000d2d60       ?FetchModelSKELForGCA@CharacterManager@@QEAA?AV?$_smart_ptr@VCSkel@@@@PEBDI@Z 00000000315d3d60 f   CharacterManager.obj
 0001:000d2e00       ?FetchPlaceHolderCharacterFromCDFInternal@CharacterManager@@QEAA_NAEAVCPlaceholderCharacter@@PEBDI@Z 00000000315d3e00 f   CharacterManager.obj
 0001:000d38c0       ?CreateCGAInstance@CharacterManager@@QEAAPEAUICharacterInstance@@PEBDI@Z 00000000315d48c0 f   CharacterManager.obj
 0001:000d3cf0       ?CreateSKELInstance@CharacterManager@@QEAAPEAUICharacterInstance@@PEBDI@Z 00000000315d4cf0 f   CharacterManager.obj
 0001:000d4350       ?LoadModelSKEL@CharacterManager@@UEAA?AV?$_smart_ptr@UICharacterModel@@@@PEBDI@Z 00000000315d5350 f   CharacterManager.obj
 0001:000d4770       ?FetchPlaceHolderCharacterFromCDF@CharacterManager@@QEAA?AV?$_smart_ptr@UIPlaceholderCharacter@@@@PEBDI@Z 00000000315d5770 f   CharacterManager.obj
 0001:000d4870       ?CreateCPFInstance@CharacterManager@@QEAAPEAUICharacterInstance@@PEBD0@Z 00000000315d5870 f   CharacterManager.obj
 0001:000d4c60       ?CreateInstance@CharacterManager@@UEAAPEAUICharacterInstance@@PEBDI@Z 00000000315d5c60 f   CharacterManager.obj
 0001:000d5020       ?PrefetchCharacterResources@CharacterManager@@UEAA?AV?$_smart_ptr@UIPlaceholderCharacter@@@@PEBDI@Z 00000000315d6020 f   CharacterManager.obj
 0001:000d5780       ?LoadANM@CryCGALoader@@QEAAIPEAVCSkel@@PEBD1AEAU?$DynArray@UCControllerTCB@@HU?$SmallDynStorage@UCControllerTCB@@HUStandardAlloc@NAlloc@@@NArray@@@@@Z 00000000315d6780 f   LoaderCGA.obj
 0001:000d5840       ?GetStreamInfo@CMesh@@QEBAXHAEAPEAXAEAH@Z 00000000315d6840 f i LoaderCGA.obj
 0001:000d59b0       ?stristr@CryStringUtils@@YAPEBDPEBD0@Z 00000000315d69b0 f i LoaderCGA.obj
 0001:000d5a50       ?GetP_numKey@IController@@UEBAHXZ 00000000315d6a50 f i LoaderCGA.obj
 0001:000d5a50       ?FindMorphTarget@IAnimationSet@@UEAAHPEBD@Z 00000000315d6a50 f i ModelAnimationSet.obj
 0001:000d5a50       ?GetO_numKey@IController@@UEBAHXZ 00000000315d6a50 f i LoaderCGA.obj
 0001:000d5a50       ?GetBoneID@CAttachmentFACE@@UEBAIXZ 00000000315d6a50 f i AttachmentManager.obj
 0001:000d5a50       ?GetBoneID@CAttachmentSKIN@@UEBAIXZ 00000000315d6a50 f i Attachment.obj
 0001:000d5a60       ?SetStreamData@CMesh@@AEAAXHPEAXH@Z 00000000315d6a60 f i LoaderCGA.obj
 0001:000d5c50       ??0?$CInt32HashMap@E$0CAA@@@QEAA@F@Z 00000000315d6c50 f i LoaderCGA.obj
 0001:000d5ce0       ?Insert@?$CInt32HashMap@E$0CAA@@@QEAAXIE@Z 00000000315d6ce0 f i LoaderCGA.obj
 0001:000d5df0       ??$find@PEAHH@stlpmtx_std@@YAPEAHPEAH0AEBH@Z 00000000315d6df0 f i LoaderCGA.obj
 0001:000d5e80       ??$ComputeTexMappingAreas@U?$Vec3_tpl@M@@USMeshTexCoord@@@CMeshHelpers@@SA_N_KPEBG0PEBU?$Vec3_tpl@M@@0PEBUSMeshTexCoord@@0AEAM4AEAPEBD@Z 00000000315d6e80 f i LoaderCGA.obj
 0001:000d6280       ?CryModuleCRTRealloc@@YAPEAXPEAX_K@Z 00000000315d7280 f i LoaderCGA.obj
 0001:000d6310       ?set_size@?$SmallDynStorage@USPostProcess@@HUStandardAlloc@NAlloc@@@NArray@@QEAAXH@Z 00000000315d7310 f i SkeletonPose.obj
 0001:000d6310       ?set_size@?$SmallDynStorage@UBoneWeights8@@HUStandardAlloc@NAlloc@@@NArray@@QEAAXH@Z 00000000315d7310 f i LoaderSKIN.obj
 0001:000d6310       ?set_size@?$SmallDynStorage@VTCBAngleAxisSpline@spline@@HUStandardAlloc@NAlloc@@@NArray@@QEAAXH@Z 00000000315d7310 f i LoaderCGA.obj
 0001:000d6310       ?set_size@?$SmallDynStorage@V?$TCBSpline@U?$Vec3_tpl@M@@U?$TCBSplineKey@U?$Vec3_tpl@M@@@spline@@@spline@@HUStandardAlloc@NAlloc@@@NArray@@QEAAXH@Z 00000000315d7310 f i LoaderCGA.obj
 0001:000d6310       ?set_size@?$SmallDynStorage@UCCGAJoint@@HUStandardAlloc@NAlloc@@@NArray@@QEAAXH@Z 00000000315d7310 f i SkeletonPose.obj
 0001:000d63c0       ?set_size@?$SmallDynStorage@UCControllerTCB@@HUStandardAlloc@NAlloc@@@NArray@@QEAAXH@Z 00000000315d73c0 f i LoaderCGA.obj
 0001:000d6470       ?set_size@?$SmallDynStorage@VCModelJoint@@HUStandardAlloc@NAlloc@@@NArray@@QEAAXH@Z 00000000315d7470 f i LoaderCGA.obj
 0001:000d6520       ?resize_raw@?$SmallDynStorage@UNodeDesc@@HUStandardAlloc@NAlloc@@@NArray@@QEAAXHH_N@Z 00000000315d7520 f i LoaderCGA.obj
 0001:000d66d0       ?ReallocStream@CMesh@@QEAAXHH@Z 00000000315d76d0 f i LoaderCGA.obj
 0001:000d67b0       ?Append@CMesh@@QEAAXAEAV1@HHHHPEAV?$vector@HV?$allocator@H@stlpmtx_std@@@stlpmtx_std@@@Z 00000000315d77b0 f i LoaderCGA.obj
 0001:000d6c80       ?PrepareJointIDHash@CModelSkeleton@@QEAAXXZ 00000000315d7c80 f i LoaderCGA.obj
 0001:000d6d30       ??$ComputeTexMappingAreas@UVec3f16@@USMeshTexCoord@@@CMeshHelpers@@SA_N_KPEBG0PEBUVec3f16@@0PEBUSMeshTexCoord@@0AEAM4AEAPEBD@Z 00000000315d7d30 f i LoaderCGA.obj
 0001:000d7160       ?pop_back@?$DynArray@V?$TCBSpline@U?$Vec3_tpl@M@@U?$TCBSplineKey@U?$Vec3_tpl@M@@@spline@@@spline@@HU?$SmallDynStorage@V?$TCBSpline@U?$Vec3_tpl@M@@U?$TCBSplineKey@U?$Vec3_tpl@M@@@spline@@@spline@@HUStandardAlloc@NAlloc@@@NArray@@@@QEAAXH@Z 00000000315d8160 f i LoaderCGA.obj
 0001:000d7160       ?pop_back@?$DynArray@VTCBAngleAxisSpline@spline@@HU?$SmallDynStorage@VTCBAngleAxisSpline@spline@@HUStandardAlloc@NAlloc@@@NArray@@@@QEAAXH@Z 00000000315d8160 f i LoaderCGA.obj
 0001:000d71f0       ?pop_back@?$DynArray@UCControllerTCB@@HU?$SmallDynStorage@UCControllerTCB@@HUStandardAlloc@NAlloc@@@NArray@@@@QEAAXH@Z 00000000315d81f0 f i LoaderCGA.obj
 0001:000d7280       ?assign@?$Array@UTCBAngAxisKey@spline@@HU?$SmallDynStorage@UTCBAngAxisKey@spline@@HUStandardAlloc@NAlloc@@@NArray@@@@QEAAXU?$Array@$$CBUTCBAngAxisKey@spline@@HU?$ArrayStorage@$$CBUTCBAngAxisKey@spline@@H@NArray@@@@@Z 00000000315d8280 f i LoaderCGA.obj
 0001:000d7330       ?set_size@?$SmallDynStorage@UTCBAngAxisKey@spline@@HUStandardAlloc@NAlloc@@@NArray@@QEAAXH@Z 00000000315d8330 f i LoaderCGA.obj
 0001:000d73e0       ?resize_raw@?$SmallDynStorage@UCControllerType@@HUStandardAlloc@NAlloc@@@NArray@@QEAAXHH_N@Z 00000000315d83e0 f i LoaderCGA.obj
 0001:000d7570       ??0CModelJoint@@QEAA@AEBV0@@Z 00000000315d8570 f i LoaderCGA.obj
 0001:000d7690       ?expand_raw@?$DynArray@UNodeDesc@@HU?$SmallDynStorage@UNodeDesc@@HUStandardAlloc@NAlloc@@@NArray@@@@IEAAPEAUNodeDesc@@PEAU2@H@Z 00000000315d8690 f i LoaderCGA.obj
 0001:000d7750       ?_M_create_node@?$_Rb_tree@HU?$less@H@stlpmtx_std@@HU?$_Identity@H@priv@2@U?$_SetTraitsT@H@42@V?$allocator@H@2@@priv@stlpmtx_std@@IEAAPEAU_Rb_tree_node_base@23@AEBH@Z 00000000315d8750 f i LoaderCGA.obj
 0001:000d77b0       ?SetVertexCount@CMesh@@QEAAXH@Z 00000000315d87b0 f i LoaderCGA.obj
 0001:000d7850       ?ComputeSubsetTexMappingAreas@CMesh@@QEAA_N_KAEAM1AEAPEBD@Z 00000000315d8850 f i LoaderCGA.obj
 0001:000d79e0       ?RecomputeTexMappingDensity@CMesh@@QEAA_NXZ 00000000315d89e0 f i LoaderCGA.obj
 0001:000d7ad0       ?comp_deriv@TCBAngleAxisSpline@spline@@UEAAXXZ 00000000315d8ad0 f i LoaderCGA.obj
 0001:000d7de0       ??0CModelJoint@@QEAA@XZ    00000000315d8de0 f i LoaderCGA.obj
 0001:000d7e90       ?AddList@?$PodArray@G$0A@@@QEAAXAEBV1@@Z 00000000315d8e90 f i LoaderCGA.obj
 0001:000d7f70       ?erase@?$DynArray@UTCBAngAxisKey@spline@@HU?$SmallDynStorage@UTCBAngAxisKey@spline@@HUStandardAlloc@NAlloc@@@NArray@@@@QEAAPEAUTCBAngAxisKey@spline@@PEAU23@0@Z 00000000315d8f70 f i LoaderCGA.obj
 0001:000d8280       ?init@?$DynArray@UTCBAngAxisKey@spline@@HU?$SmallDynStorage@UTCBAngAxisKey@spline@@HUStandardAlloc@NAlloc@@@NArray@@@@KAPEAUTCBAngAxisKey@spline@@U?$Array@UTCBAngAxisKey@spline@@HU?$ArrayStorage@UTCBAngAxisKey@spline@@H@NArray@@@@PEBU23@@Z 00000000315d9280 f i LoaderCGA.obj
 0001:000d8370       ?append_raw@?$DynArray@UCControllerType@@HU?$SmallDynStorage@UCControllerType@@HUStandardAlloc@NAlloc@@@NArray@@@@QEAA?AU?$Array@UCControllerType@@HU?$ArrayStorage@UCControllerType@@H@NArray@@@@H@Z 00000000315d9370 f i LoaderCGA.obj
 0001:000d8430       ??$move_init@UTCBAngAxisKey@spline@@@NArray@@YAXPEAUTCBAngAxisKey@spline@@0_K@Z 00000000315d9430 f i LoaderCGA.obj
 0001:000d88b0       ??$move_init@VCModelJoint@@@NArray@@YAXPEAVCModelJoint@@0_K@Z 00000000315d98b0 f i LoaderCGA.obj
 0001:000d8920       ?SetNameChar@CModelJoint@@QEAAXPEBD@Z 00000000315d9920 f i LoaderCGA.obj
 0001:000d8a30       ?SetJointName@CModelJoint@@QEAAXPEBD@Z 00000000315d9a30 f i LoaderCGA.obj
 0001:000d8aa0       ?SetAnimName@ModelAnimationHeader@@QEAAXPEBD@Z 00000000315d9aa0 f i LoaderCGA.obj
 0001:000d8ba0       ?destroy@?$DynArray@USMeshSubset@@HU?$SmallDynStorage@USMeshSubset@@HUStandardAlloc@NAlloc@@@NArray@@@@KAXU?$Array@USMeshSubset@@HU?$ArrayStorage@USMeshSubset@@H@NArray@@@@@Z 00000000315d9ba0 f i LoaderCGA.obj
 0001:000d8ca0       ??4?$DynArray@UCControllerType@@HU?$SmallDynStorage@UCControllerType@@HUStandardAlloc@NAlloc@@@NArray@@@@QEAAAEAU0@U?$Array@$$CBUCControllerType@@HU?$ArrayStorage@$$CBUCControllerType@@H@NArray@@@@@Z 00000000315d9ca0 f i LoaderCGA.obj
 0001:000d8db0       ?grow@?$DynArray@UNodeDesc@@HU?$SmallDynStorage@UNodeDesc@@HUStandardAlloc@NAlloc@@@NArray@@@@QEAAPEAUNodeDesc@@H@Z 00000000315d9db0 f i LoaderCGA.obj
 0001:000d8e30       ?init@?$DynArray@USMeshSubset@@HU?$SmallDynStorage@USMeshSubset@@HUStandardAlloc@NAlloc@@@NArray@@@@KAPEAUSMeshSubset@@U?$Array@USMeshSubset@@HU?$ArrayStorage@USMeshSubset@@H@NArray@@@@@Z 00000000315d9e30 f i LoaderCGA.obj
 0001:000d8f70       ?resize_raw@?$SmallDynStorage@UTCBAngAxisKey@spline@@HUStandardAlloc@NAlloc@@@NArray@@QEAAXHH_N@Z 00000000315d9f70 f i LoaderCGA.obj
 0001:000d9100       ?expand_raw@?$DynArray@UTCBAngAxisKey@spline@@HU?$SmallDynStorage@UTCBAngAxisKey@spline@@HUStandardAlloc@NAlloc@@@NArray@@@@IEAAPEAUTCBAngAxisKey@spline@@PEAU23@H@Z 00000000315da100 f i LoaderCGA.obj
 0001:000d91c0       ?resize_raw@?$SmallDynStorage@VCModelJoint@@HUStandardAlloc@NAlloc@@@NArray@@QEAAXHH_N@Z 00000000315da1c0 f i LoaderCGA.obj
 0001:000d9350       ?insert_unique@?$_Rb_tree@HU?$less@H@stlpmtx_std@@HU?$_Identity@H@priv@2@U?$_SetTraitsT@H@42@V?$allocator@H@2@@priv@stlpmtx_std@@QEAA?AU?$pair@U?$_Rb_tree_iterator@HU?$_SetTraitsT@H@priv@stlpmtx_std@@@priv@stlpmtx_std@@_N@3@AEBH@Z 00000000315da350 f i LoaderCGA.obj
 0001:000d95c0       ??0SMeshSubset@@QEAA@AEBU0@@Z 00000000315da5c0 f i LoaderCGA.obj
 0001:000d9660       ??4?$DynArray@UTCBAngAxisKey@spline@@HU?$SmallDynStorage@UTCBAngAxisKey@spline@@HUStandardAlloc@NAlloc@@@NArray@@@@QEAAAEAU0@U?$Array@$$CBUTCBAngAxisKey@spline@@HU?$ArrayStorage@$$CBUTCBAngAxisKey@spline@@H@NArray@@@@@Z 00000000315da660 f i LoaderCGA.obj
 0001:000d9740       ?init@?$DynArray@USMeshSubset@@HU?$SmallDynStorage@USMeshSubset@@HUStandardAlloc@NAlloc@@@NArray@@@@KAPEAUSMeshSubset@@U?$Array@USMeshSubset@@HU?$ArrayStorage@USMeshSubset@@H@NArray@@@@AEBU2@@Z 00000000315da740 f i LoaderCGA.obj
 0001:000d98b0       ?expand_raw@?$DynArray@VCModelJoint@@HU?$SmallDynStorage@VCModelJoint@@HUStandardAlloc@NAlloc@@@NArray@@@@IEAAPEAVCModelJoint@@PEAV2@H@Z 00000000315da8b0 f i LoaderCGA.obj
 0001:000d9970       ??$AddContainer@U?$DynArray@UTCBAngAxisKey@spline@@HU?$SmallDynStorage@UTCBAngAxisKey@spline@@HUStandardAlloc@NAlloc@@@NArray@@@@@ICrySizer@@QEAA_NAEBU?$DynArray@UTCBAngAxisKey@spline@@HU?$SmallDynStorage@UTCBAngAxisKey@spline@@HUStandardAlloc@NAlloc@@@NArray@@@@@Z 00000000315da970 f i LoaderCGA.obj
 0001:000d9a00       ?GetMemoryUsage@?$TSpline@UTCBAngAxisKey@spline@@VHermitBasis@2@@spline@@UEBAXPEAVICrySizer@@_N@Z 00000000315daa00 f i LoaderCGA.obj
 0001:000d9a50       ??$move_init@USMeshSubset@@@NArray@@YAXPEAUSMeshSubset@@0_K@Z 00000000315daa50 f i LoaderCGA.obj
 0001:000d9b70       ?grow@?$DynArray@UTCBAngAxisKey@spline@@HU?$SmallDynStorage@UTCBAngAxisKey@spline@@HUStandardAlloc@NAlloc@@@NArray@@@@QEAAPEAUTCBAngAxisKey@spline@@H@Z 00000000315dab70 f i LoaderCGA.obj
 0001:000d9c10       ??0?$DynArray@UTCBAngAxisKey@spline@@HU?$SmallDynStorage@UTCBAngAxisKey@spline@@HUStandardAlloc@NAlloc@@@NArray@@@@QEAA@AEBU0@@Z 00000000315dac10 f i LoaderCGA.obj
 0001:000d9cd0       ??0CMesh@@QEAA@XZ          00000000315dacd0 f i LoaderCGA.obj
 0001:000d9e20       ?resize_raw@?$SmallDynStorage@USMeshSubset@@HUStandardAlloc@NAlloc@@@NArray@@QEAAXHH_N@Z 00000000315dae20 f i LoaderCGA.obj
 0001:000d9fa0       ??4?$TSpline@UTCBAngAxisKey@spline@@VHermitBasis@2@@spline@@QEAAAEAV01@AEBV01@@Z 00000000315dafa0 f i LoaderCGA.obj
 0001:000da020       ?calc_ease@?$TCBSpline@U?$Vec3_tpl@M@@U?$TCBSplineKey@U?$Vec3_tpl@M@@@spline@@@spline@@IEAAMMMM@Z 00000000315db020 f i FaceAnimSequence.obj
 0001:000da020       ?calc_ease@?$TCBSpline@U?$Quat_tpl@M@@UTCBAngAxisKey@spline@@@spline@@IEAAMMMM@Z 00000000315db020 f i LoaderCGA.obj
 0001:000da0f0       ?append_raw@?$DynArray@USMeshSubset@@HU?$SmallDynStorage@USMeshSubset@@HUStandardAlloc@NAlloc@@@NArray@@@@QEAA?AU?$Array@USMeshSubset@@HU?$ArrayStorage@USMeshSubset@@H@NArray@@@@H@Z 00000000315db0f0 f i LoaderCGA.obj
 0001:000da1b0       ?init@?$DynArray@V?$TCBSpline@U?$Vec3_tpl@M@@U?$TCBSplineKey@U?$Vec3_tpl@M@@@spline@@@spline@@HU?$SmallDynStorage@V?$TCBSpline@U?$Vec3_tpl@M@@U?$TCBSplineKey@U?$Vec3_tpl@M@@@spline@@@spline@@HUStandardAlloc@NAlloc@@@NArray@@@@KAPEAV?$TCBSpline@U?$Vec3_tpl@M@@U?$TCBSplineKey@U?$Vec3_tpl@M@@@spline@@@spline@@U?$Array@V?$TCBSpline@U?$Vec3_tpl@M@@U?$TCBSplineKey@U?$Vec3_tpl@M@@@spline@@@spline@@HU?$ArrayStorage@V?$TCBSpline@U?$Vec3_tpl@M@@U?$TCBSplineKey@U?$Vec3_tpl@M@@@spline@@@spline@@H@NArray@@@@@Z 00000000315db1b0 f i LoaderCGA.obj
 0001:000da320       ??$move_init@V?$TCBSpline@U?$Vec3_tpl@M@@U?$TCBSplineKey@U?$Vec3_tpl@M@@@spline@@@spline@@@NArray@@YAXPEAV?$TCBSpline@U?$Vec3_tpl@M@@U?$TCBSplineKey@U?$Vec3_tpl@M@@@spline@@@spline@@0_K@Z 00000000315db320 f i LoaderCGA.obj
 0001:000da410       ?compKeyDeriv@TCBAngleAxisSpline@spline@@EEAAXH@Z 00000000315db410 f i LoaderCGA.obj
 0001:000dafb0       ?interp_keys@TCBAngleAxisSpline@spline@@MEAAXHHMAEAU?$Quat_tpl@M@@@Z 00000000315dbfb0 f i LoaderCGA.obj
 0001:000dcee0       ??_GTCBAngleAxisSpline@spline@@UEAAPEAXI@Z 00000000315ddee0 f i LoaderCGA.obj
 0001:000dcee0       ??_E?$TSpline@UTCBAngAxisKey@spline@@VHermitBasis@2@@spline@@UEAAPEAXI@Z 00000000315ddee0 f i LoaderCGA.obj
 0001:000dcee0       ??_G?$TSpline@UTCBAngAxisKey@spline@@VHermitBasis@2@@spline@@UEAAPEAXI@Z 00000000315ddee0 f i LoaderCGA.obj
 0001:000dcee0       ??_ETCBAngleAxisSpline@spline@@UEAAPEAXI@Z 00000000315ddee0 f i LoaderCGA.obj
 0001:000dcf50       ?resize_raw@?$SmallDynStorage@V?$TCBSpline@U?$Vec3_tpl@M@@U?$TCBSplineKey@U?$Vec3_tpl@M@@@spline@@@spline@@HUStandardAlloc@NAlloc@@@NArray@@QEAAXHH_N@Z 00000000315ddf50 f i LoaderCGA.obj
 0001:000dd0d0       ?init@?$DynArray@VTCBAngleAxisSpline@spline@@HU?$SmallDynStorage@VTCBAngleAxisSpline@spline@@HUStandardAlloc@NAlloc@@@NArray@@@@KAPEAVTCBAngleAxisSpline@spline@@U?$Array@VTCBAngleAxisSpline@spline@@HU?$ArrayStorage@VTCBAngleAxisSpline@spline@@H@NArray@@@@@Z 00000000315de0d0 f i LoaderCGA.obj
 0001:000dd240       ??0CControllerTCB@@QEAA@AEBU0@@Z 00000000315de240 f i LoaderCGA.obj
 0001:000dd370       ?GetMemoryUsage@CControllerTCB@@UEBAXPEAVICrySizer@@@Z 00000000315de370 f i LoaderCGA.obj
 0001:000dd3e0       ?SizeOfController@CControllerTCB@@UEBA_KXZ 00000000315de3e0 f i LoaderCGA.obj
 0001:000dd4a0       ??1CControllerTCB@@UEAA@XZ 00000000315de4a0 f i LoaderCGA.obj
 0001:000dd560       ??_GCControllerTCB@@UEAAPEAXI@Z 00000000315de560 f i LoaderCGA.obj
 0001:000dd560       ??_ECControllerTCB@@UEAAPEAXI@Z 00000000315de560 f i LoaderCGA.obj
 0001:000dd590       ?resize@?$DynArray@USMeshSubset@@HU?$SmallDynStorage@USMeshSubset@@HUStandardAlloc@NAlloc@@@NArray@@@@QEAAXH@Z 00000000315de590 f i LoaderCGA.obj
 0001:000dd630       ?clear@?$DynArray@V?$TCBSpline@U?$Vec3_tpl@M@@U?$TCBSplineKey@U?$Vec3_tpl@M@@@spline@@@spline@@HU?$SmallDynStorage@V?$TCBSpline@U?$Vec3_tpl@M@@U?$TCBSplineKey@U?$Vec3_tpl@M@@@spline@@@spline@@HUStandardAlloc@NAlloc@@@NArray@@@@QEAAXXZ 00000000315de630 f i LoaderCGA.obj
 0001:000dd6d0       ?append_raw@?$DynArray@V?$TCBSpline@U?$Vec3_tpl@M@@U?$TCBSplineKey@U?$Vec3_tpl@M@@@spline@@@spline@@HU?$SmallDynStorage@V?$TCBSpline@U?$Vec3_tpl@M@@U?$TCBSplineKey@U?$Vec3_tpl@M@@@spline@@@spline@@HUStandardAlloc@NAlloc@@@NArray@@@@QEAA?AU?$Array@V?$TCBSpline@U?$Vec3_tpl@M@@U?$TCBSplineKey@U?$Vec3_tpl@M@@@spline@@@spline@@HU?$ArrayStorage@V?$TCBSpline@U?$Vec3_tpl@M@@U?$TCBSplineKey@U?$Vec3_tpl@M@@@spline@@@spline@@H@NArray@@@@H@Z 00000000315de6d0 f i LoaderCGA.obj
 0001:000dd790       ?init@?$DynArray@UCControllerTCB@@HU?$SmallDynStorage@UCControllerTCB@@HUStandardAlloc@NAlloc@@@NArray@@@@KAPEAUCControllerTCB@@U?$Array@UCControllerTCB@@HU?$ArrayStorage@UCControllerTCB@@H@NArray@@@@@Z 00000000315de790 f i LoaderCGA.obj
 0001:000ddac0       ??$move_init@VTCBAngleAxisSpline@spline@@@NArray@@YAXPEAVTCBAngleAxisSpline@spline@@0_K@Z 00000000315deac0 f i LoaderCGA.obj
 0001:000ddbb0       ?resize_raw@?$SmallDynStorage@VTCBAngleAxisSpline@spline@@HUStandardAlloc@NAlloc@@@NArray@@QEAAXHH_N@Z 00000000315debb0 f i LoaderCGA.obj
 0001:000ddd30       ?init@?$DynArray@VCModelMesh@@HU?$SmallDynStorage@VCModelMesh@@HUStandardAlloc@NAlloc@@@NArray@@@@KAPEAVCModelMesh@@U?$Array@VCModelMesh@@HU?$ArrayStorage@VCModelMesh@@H@NArray@@@@@Z 00000000315ded30 f i LoaderCGA.obj
 0001:000de1d0       ??$move_init@UCControllerTCB@@@NArray@@YAXPEAUCControllerTCB@@0_K@Z 00000000315df1d0 f i LoaderCGA.obj
 0001:000de240       ?clear@?$DynArray@VTCBAngleAxisSpline@spline@@HU?$SmallDynStorage@VTCBAngleAxisSpline@spline@@HUStandardAlloc@NAlloc@@@NArray@@@@QEAAXXZ 00000000315df240 f i LoaderCGA.obj
 0001:000de2e0       ?resize_raw@?$SmallDynStorage@UCControllerTCB@@HUStandardAlloc@NAlloc@@@NArray@@QEAAXHH_N@Z 00000000315df2e0 f i LoaderCGA.obj
 0001:000de460       ?append_raw@?$DynArray@VTCBAngleAxisSpline@spline@@HU?$SmallDynStorage@VTCBAngleAxisSpline@spline@@HUStandardAlloc@NAlloc@@@NArray@@@@QEAA?AU?$Array@VTCBAngleAxisSpline@spline@@HU?$ArrayStorage@VTCBAngleAxisSpline@spline@@H@NArray@@@@H@Z 00000000315df460 f i LoaderCGA.obj
 0001:000de520       ?clear@?$DynArray@UCControllerTCB@@HU?$SmallDynStorage@UCControllerTCB@@HUStandardAlloc@NAlloc@@@NArray@@@@QEAAXXZ 00000000315df520 f i LoaderCGA.obj
 0001:000de5c0       ?append_raw@?$DynArray@UCControllerTCB@@HU?$SmallDynStorage@UCControllerTCB@@HUStandardAlloc@NAlloc@@@NArray@@@@QEAA?AU?$Array@UCControllerTCB@@HU?$ArrayStorage@UCControllerTCB@@H@NArray@@@@H@Z 00000000315df5c0 f i LoaderCGA.obj
 0001:000de680       ?Reset@CryCGALoader@@QEAAXXZ 00000000315df680 f   LoaderCGA.obj
 0001:000de7c0       ?InitNodes@CryCGALoader@@QEAAXPEAUCHeaderTCB@@PEAVCSkel@@PEBDAEBV?$CryStringT@D@@_NII@Z 00000000315df7c0 f   LoaderCGA.obj
 0001:000e1f80       ?LoadAnimationANM@CryCGALoader@@QEAA_NPEBDPEAVCSkel@@II@Z 00000000315e2f80 f   LoaderCGA.obj
 0001:000e2200       ?LoadAnimations@CryCGALoader@@QEAAXPEBDPEAVCSkel@@II@Z 00000000315e3200 f   LoaderCGA.obj
 0001:000e2d20       ?LoadNewCGA@CryCGALoader@@QEAAPEAVCSkel@@PEBDPEAVCharacterManager@@I@Z 00000000315e3d20 f   LoaderCGA.obj
 0001:000e33c0       ?SetIMaterial@CSkel@@QEAAXPEAUIMaterial@@@Z 00000000315e43c0 f i LoaderCHR.obj
 0001:000e3410       ??$move_init@USAnimFile@@@NArray@@YAXPEAUSAnimFile@@0_K@Z 00000000315e4410 f i LoaderCHR.obj
 0001:000e3480       ?resize_raw@?$SmallDynStorage@DHUStandardAlloc@NAlloc@@@NArray@@QEAAXHH_N@Z 00000000315e4480 f i LoaderCHR.obj
 0001:000e3600       ?_M_erase@?$_Rb_tree@_JU?$less@_J@stlpmtx_std@@U?$pair@$$CB_JPEAUphys_geometry@@@2@U?$_Select1st@U?$pair@$$CB_JPEAUphys_geometry@@@stlpmtx_std@@@priv@2@U?$_MapTraitsT@U?$pair@$$CB_JPEAUphys_geometry@@@stlpmtx_std@@@52@V?$allocator@U?$pair@$$CB_JPEAUphys_geometry@@@stlpmtx_std@@@2@@priv@stlpmtx_std@@AEAAXPEAU_Rb_tree_node_base@23@@Z 00000000315e4600 f i LoaderCHR.obj
 0001:000e3600       ?_M_erase@?$_Rb_tree@PEAUIFacialEffector@@U?$less@PEAUIFacialEffector@@@stlpmtx_std@@U?$pair@QEAUIFacialEffector@@PEAU1@@3@U?$_Select1st@U?$pair@QEAUIFacialEffector@@PEAU1@@stlpmtx_std@@@priv@3@U?$_MapTraitsT@U?$pair@QEAUIFacialEffector@@PEAU1@@stlpmtx_std@@@63@V?$allocator@U?$pair@QEAUIFacialEffector@@PEAU1@@stlpmtx_std@@@3@@priv@stlpmtx_std@@AEAAXPEAU_Rb_tree_node_base@23@@Z 00000000315e4600 f i FaceEffectorLibrary.obj
 0001:000e3600       ?_M_erase@?$_Rb_tree@IU?$less@I@stlpmtx_std@@U?$pair@$$CBIPEAV?$vector@IV?$allocator@I@stlpmtx_std@@@stlpmtx_std@@@2@U?$_Select1st@U?$pair@$$CBIPEAV?$vector@IV?$allocator@I@stlpmtx_std@@@stlpmtx_std@@@stlpmtx_std@@@priv@2@U?$_MapTraitsT@U?$pair@$$CBIPEAV?$vector@IV?$allocator@I@stlpmtx_std@@@stlpmtx_std@@@stlpmtx_std@@@52@V?$allocator@U?$pair@$$CBIPEAV?$vector@IV?$allocator@I@stlpmtx_std@@@stlpmtx_std@@@stlpmtx_std@@@2@@priv@stlpmtx_std@@AEAAXPEAU_Rb_tree_node_base@23@@Z 00000000315e4600 f i CharacterManager.obj
 0001:000e3600       ?_M_erase@?$_Rb_tree@IU?$less@I@stlpmtx_std@@U?$pair@$$CBIPEAV?$vector@HV?$allocator@H@stlpmtx_std@@@stlpmtx_std@@@2@U?$_Select1st@U?$pair@$$CBIPEAV?$vector@HV?$allocator@H@stlpmtx_std@@@stlpmtx_std@@@stlpmtx_std@@@priv@2@U?$_MapTraitsT@U?$pair@$$CBIPEAV?$vector@HV?$allocator@H@stlpmtx_std@@@stlpmtx_std@@@stlpmtx_std@@@52@V?$allocator@U?$pair@$$CBIPEAV?$vector@HV?$allocator@H@stlpmtx_std@@@stlpmtx_std@@@stlpmtx_std@@@2@@priv@stlpmtx_std@@AEAAXPEAU_Rb_tree_node_base@23@@Z 00000000315e4600 f i CharacterManager.obj
 0001:000e3600       ?_M_erase@?$_Rb_tree@IU?$less@I@stlpmtx_std@@U?$pair@$$CBI_K@2@U?$_Select1st@U?$pair@$$CBI_K@stlpmtx_std@@@priv@2@U?$_MapTraitsT@U?$pair@$$CBI_K@stlpmtx_std@@@52@V?$allocator@U?$pair@$$CBI_K@stlpmtx_std@@@2@@priv@stlpmtx_std@@AEAAXPEAU_Rb_tree_node_base@23@@Z 00000000315e4600 f i CharacterManager.obj
 0001:000e3600       ?_M_erase@?$_Rb_tree@HU?$less@H@stlpmtx_std@@HU?$_Identity@H@priv@2@U?$_SetTraitsT@H@42@V?$allocator@H@2@@priv@stlpmtx_std@@AEAAXPEAU_Rb_tree_node_base@23@@Z 00000000315e4600 f i LoaderCGA.obj
 0001:000e3600       ?_M_erase@?$_Rb_tree@IU?$less@I@stlpmtx_std@@U?$pair@$$CBIPEAVCModelJoint@@@2@U?$_Select1st@U?$pair@$$CBIPEAVCModelJoint@@@stlpmtx_std@@@priv@2@U?$_MapTraitsT@U?$pair@$$CBIPEAVCModelJoint@@@stlpmtx_std@@@52@V?$allocator@U?$pair@$$CBIPEAVCModelJoint@@@stlpmtx_std@@@2@@priv@stlpmtx_std@@AEAAXPEAU_Rb_tree_node_base@23@@Z 00000000315e4600 f i Model.obj
 0001:000e3600       ?_M_erase@?$_Rb_tree@IU?$less@I@stlpmtx_std@@U?$pair@$$CBIUSFacialDisplaceInfo@CFacialModel@@@2@U?$_Select1st@U?$pair@$$CBIUSFacialDisplaceInfo@CFacialModel@@@stlpmtx_std@@@priv@2@U?$_MapTraitsT@U?$pair@$$CBIUSFacialDisplaceInfo@CFacialModel@@@stlpmtx_std@@@52@V?$allocator@U?$pair@$$CBIUSFacialDisplaceInfo@CFacialModel@@@stlpmtx_std@@@2@@priv@stlpmtx_std@@AEAAXPEAU_Rb_tree_node_base@23@@Z 00000000315e4600 f i SkeletonAnim.obj
 0001:000e3660       ?_M_compute_next_size@?$_Impl_vector@USEffectorInfo@CFacialModel@@V?$allocator@USEffectorInfo@CFacialModel@@@stlpmtx_std@@@priv@stlpmtx_std@@AEAA_K_K@Z 00000000315e4660 f i FacialModel.obj
 0001:000e3660       ?_M_compute_next_size@?$_Impl_vector@UChannelInfo@CFacialAnimSequenceInstance@@V?$allocator@UChannelInfo@CFacialAnimSequenceInstance@@@stlpmtx_std@@@priv@stlpmtx_std@@AEAA_K_K@Z 00000000315e4660 f i FaceAnimSequence.obj
 0001:000e3660       ?_M_compute_next_size@?$_Impl_vector@UFacialAnimationEntry@CAnimationSet@@V?$allocator@UFacialAnimationEntry@CAnimationSet@@@stlpmtx_std@@@priv@stlpmtx_std@@AEAA_K_K@Z 00000000315e4660 f i LoaderCHR.obj
 0001:000e3660       ?_M_compute_next_size@?$_Impl_vector@USMorphTargetInfo@CFacialModel@@V?$allocator@USMorphTargetInfo@CFacialModel@@@stlpmtx_std@@@priv@stlpmtx_std@@AEAA_K_K@Z 00000000315e4660 f i FacialModel.obj
 0001:000e3660       ?_M_compute_next_size@?$_Impl_vector@VCFacialAnimSkeletalAnimationEntry@@V?$allocator@VCFacialAnimSkeletalAnimationEntry@@@stlpmtx_std@@@priv@stlpmtx_std@@AEAA_K_K@Z 00000000315e4660 f i FaceAnimSequence.obj
 0001:000e36f0       ?resize_raw@?$SmallDynStorage@USAnimFile@@HUStandardAlloc@NAlloc@@@NArray@@QEAAXHH_N@Z 00000000315e46f0 f i LoaderCHR.obj
 0001:000e3880       ?resize_raw@?$SmallDynStorage@GHUStandardAlloc@NAlloc@@@NArray@@QEAAXHH_N@Z 00000000315e4880 f i LoaderCHR.obj
 0001:000e3a10       ??1FacialAnimationEntry@CAnimationSet@@QEAA@XZ 00000000315e4a10 f i LoaderCHR.obj
 0001:000e3a80       ?ReuseAnimationFiles@CryCHRLoader@@AEAAIAEAVCParamLoader@@IPEAVCSkel@@@Z 00000000315e4a80 f   LoaderCHR.obj
 0001:000e3b70       ??$__unguarded_linear_insert@PEAUFacialAnimationEntry@CAnimationSet@@U12@U?$less_stricmp@UFacialAnimationEntry@CAnimationSet@@@stl@@@priv@stlpmtx_std@@YAXPEAUFacialAnimationEntry@CAnimationSet@@U23@U?$less_stricmp@UFacialAnimationEntry@CAnimationSet@@@stl@@@Z 00000000315e4b70 f i LoaderCHR.obj
 0001:000e3c10       ??$swap@UFacialAnimationEntry@CAnimationSet@@@stlpmtx_std@@YAXAEAUFacialAnimationEntry@CAnimationSet@@0@Z 00000000315e4c10 f i LoaderCHR.obj
 0001:000e3d70       ??$__push_heap@PEAUFacialAnimationEntry@CAnimationSet@@_JU12@U?$less_stricmp@UFacialAnimationEntry@CAnimationSet@@@stl@@@stlpmtx_std@@YAXPEAUFacialAnimationEntry@CAnimationSet@@_J1U12@U?$less_stricmp@UFacialAnimationEntry@CAnimationSet@@@stl@@@Z 00000000315e4d70 f i LoaderCHR.obj
 0001:000e3e60       ?expand_raw@?$DynArray@GHU?$SmallDynStorage@GHUStandardAlloc@NAlloc@@@NArray@@@@IEAAPEAGPEAGH@Z 00000000315e4e60 f i LoaderCHR.obj
 0001:000e3f00       ??0?$CryStringT@D@@QEAA@PEBD0@Z 00000000315e4f00 f i LoaderCHR.obj
 0001:000e3f90       ?clear@?$DynArray@IHU?$SmallDynStorage@IHUStandardAlloc@NAlloc@@@NArray@@@@QEAAXXZ 00000000315e4f90 f i LoaderCHR.obj
 0001:000e4060       ?append_raw@?$DynArray@DHU?$SmallDynStorage@DHUStandardAlloc@NAlloc@@@NArray@@@@QEAA?AU?$Array@DHU?$ArrayStorage@DH@NArray@@@@H@Z 00000000315e5060 f i LoaderCHR.obj
 0001:000e4110       ?append_raw@?$DynArray@GHU?$SmallDynStorage@GHUStandardAlloc@NAlloc@@@NArray@@@@QEAA?AU?$Array@GHU?$ArrayStorage@GH@NArray@@@@H@Z 00000000315e5110 f i LoaderCHR.obj
 0001:000e41d0       ?_M_insert@?$_Rb_tree@_JU?$less@_J@stlpmtx_std@@U?$pair@$$CB_JPEAUphys_geometry@@@2@U?$_Select1st@U?$pair@$$CB_JPEAUphys_geometry@@@stlpmtx_std@@@priv@2@U?$_MapTraitsT@U?$pair@$$CB_JPEAUphys_geometry@@@stlpmtx_std@@@52@V?$allocator@U?$pair@$$CB_JPEAUphys_geometry@@@stlpmtx_std@@@2@@priv@stlpmtx_std@@AEAA?AU?$_Rb_tree_iterator@U?$pair@$$CB_JPEAUphys_geometry@@@stlpmtx_std@@U?$_MapTraitsT@U?$pair@$$CB_JPEAUphys_geometry@@@stlpmtx_std@@@priv@2@@23@PEAU_Rb_tree_node_base@23@AEBU?$pair@$$CB_JPEAUphys_geometry@@@3@00@Z 00000000315e51d0 f i LoaderCHR.obj
 0001:000e4290       ?insert_unique@?$_Rb_tree@_JU?$less@_J@stlpmtx_std@@U?$pair@$$CB_JPEAUphys_geometry@@@2@U?$_Select1st@U?$pair@$$CB_JPEAUphys_geometry@@@stlpmtx_std@@@priv@2@U?$_MapTraitsT@U?$pair@$$CB_JPEAUphys_geometry@@@stlpmtx_std@@@52@V?$allocator@U?$pair@$$CB_JPEAUphys_geometry@@@stlpmtx_std@@@2@@priv@stlpmtx_std@@QEAA?AU?$pair@U?$_Rb_tree_iterator@U?$pair@$$CB_JPEAUphys_geometry@@@stlpmtx_std@@U?$_MapTraitsT@U?$pair@$$CB_JPEAUphys_geometry@@@stlpmtx_std@@@priv@2@@priv@stlpmtx_std@@_N@3@AEBU?$pair@$$CB_JPEAUphys_geometry@@@3@@Z 00000000315e5290 f i LoaderCHR.obj
 0001:000e4490       ??$__adjust_heap@PEAUFacialAnimationEntry@CAnimationSet@@_JU12@U?$less_stricmp@UFacialAnimationEntry@CAnimationSet@@@stl@@@stlpmtx_std@@YAXPEAUFacialAnimationEntry@CAnimationSet@@_J1U12@U?$less_stricmp@UFacialAnimationEntry@CAnimationSet@@@stl@@@Z 00000000315e5490 f i LoaderCHR.obj
 0001:000e4600       ?clear@?$DynArray@USAnimFile@@HU?$SmallDynStorage@USAnimFile@@HUStandardAlloc@NAlloc@@@NArray@@@@QEAAXXZ 00000000315e5600 f i LoaderCHR.obj
 0001:000e46e0       ??$move_init@UModelAnimationHeader@@@NArray@@YAXPEAUModelAnimationHeader@@0_K@Z 00000000315e56e0 f i LoaderCHR.obj
 0001:000e47a0       ?ClearModel@CryCHRLoader@@AEAAXXZ 00000000315e57a0 f   LoaderCHR.obj
 0001:000e47d0       ?GetDefaultAnimDir@CryCHRLoader@@AEAA?BV?$CryStringT@D@@XZ 00000000315e57d0 f   LoaderCHR.obj
 0001:000e4bf0       ?insert_unique@?$_Rb_tree@_JU?$less@_J@stlpmtx_std@@U?$pair@$$CB_JPEAUphys_geometry@@@2@U?$_Select1st@U?$pair@$$CB_JPEAUphys_geometry@@@stlpmtx_std@@@priv@2@U?$_MapTraitsT@U?$pair@$$CB_JPEAUphys_geometry@@@stlpmtx_std@@@52@V?$allocator@U?$pair@$$CB_JPEAUphys_geometry@@@stlpmtx_std@@@2@@priv@stlpmtx_std@@QEAA?AU?$_Rb_tree_iterator@U?$pair@$$CB_JPEAUphys_geometry@@@stlpmtx_std@@U?$_MapTraitsT@U?$pair@$$CB_JPEAUphys_geometry@@@stlpmtx_std@@@priv@2@@23@U423@AEBU?$pair@$$CB_JPEAUphys_geometry@@@3@@Z 00000000315e5bf0 f i LoaderCHR.obj
 0001:000e5040       ??$__pop_heap@PEAUFacialAnimationEntry@CAnimationSet@@U12@U?$less_stricmp@UFacialAnimationEntry@CAnimationSet@@@stl@@_J@stlpmtx_std@@YAXPEAUFacialAnimationEntry@CAnimationSet@@00U12@U?$less_stricmp@UFacialAnimationEntry@CAnimationSet@@@stl@@PEA_J@Z 00000000315e6040 f i LoaderCHR.obj
 0001:000e5120       ??$copy_backward@PEAUFacialAnimationEntry@CAnimationSet@@PEAU12@@stlpmtx_std@@YAPEAUFacialAnimationEntry@CAnimationSet@@PEAU12@00@Z 00000000315e6120 f i LoaderCHR.obj
 0001:000e51c0       ??$__make_heap@PEAUFacialAnimationEntry@CAnimationSet@@U?$less_stricmp@UFacialAnimationEntry@CAnimationSet@@@stl@@U12@_J@stlpmtx_std@@YAXPEAUFacialAnimationEntry@CAnimationSet@@0U?$less_stricmp@UFacialAnimationEntry@CAnimationSet@@@stl@@0PEA_J@Z 00000000315e61c0 f i LoaderCHR.obj
 0001:000e52b0       ?resize_raw@?$SmallDynStorage@UModelAnimationHeader@@HUStandardAlloc@NAlloc@@@NArray@@QEAAXHH_N@Z 00000000315e62b0 f i LoaderCHR.obj
 0001:000e5c00       ??0?$DynArray@DHU?$SmallDynStorage@DHUStandardAlloc@NAlloc@@@NArray@@@@QEAA@AEBU0@@Z 00000000315e6c00 f i LoaderCHR.obj
 0001:000e5cc0       ??0?$DynArray@GHU?$SmallDynStorage@GHUStandardAlloc@NAlloc@@@NArray@@@@QEAA@AEBU0@@Z 00000000315e6cc0 f i LoaderCHR.obj
 0001:000e5d80       ?AddSlash@PathUtil@@YA?AV?$CryStringT@D@@AEBV2@@Z 00000000315e6d80 f i LoaderCHR.obj
 0001:000e5f20       ?Make@PathUtil@@YA?AV?$CryStringT@D@@AEBV2@PEBD@Z 00000000315e6f20 f i LoaderCHR.obj
 0001:000e6060       ?Make@PathUtil@@YA?AV?$CryStringT@D@@QEBD0@Z 00000000315e7060 f i LoaderCHR.obj
 0001:000e6230       ??$__unguarded_partition@PEAUFacialAnimationEntry@CAnimationSet@@U12@U?$less_stricmp@UFacialAnimationEntry@CAnimationSet@@@stl@@@priv@stlpmtx_std@@YAPEAUFacialAnimationEntry@CAnimationSet@@PEAU23@0U23@U?$less_stricmp@UFacialAnimationEntry@CAnimationSet@@@stl@@@Z 00000000315e7230 f i LoaderCHR.obj
 0001:000e62e0       ??$__linear_insert@PEAUFacialAnimationEntry@CAnimationSet@@U12@U?$less_stricmp@UFacialAnimationEntry@CAnimationSet@@@stl@@@priv@stlpmtx_std@@YAXPEAUFacialAnimationEntry@CAnimationSet@@0U23@U?$less_stricmp@UFacialAnimationEntry@CAnimationSet@@@stl@@@Z 00000000315e72e0 f i LoaderCHR.obj
 0001:000e63b0       ??$copy@PEBUFacialAnimationEntry@CAnimationSet@@PEAU12@@stlpmtx_std@@YAPEAUFacialAnimationEntry@CAnimationSet@@PEBU12@0PEAU12@@Z 00000000315e73b0 f i LoaderCHR.obj
 0001:000e6450       ??$__destroy_range@V?$reverse_iterator@PEAUFacialAnimationEntry@CAnimationSet@@@stlpmtx_std@@UFacialAnimationEntry@CAnimationSet@@@stlpmtx_std@@YAXV?$reverse_iterator@PEAUFacialAnimationEntry@CAnimationSet@@@0@0PEAUFacialAnimationEntry@CAnimationSet@@@Z 00000000315e7450 f i LoaderCHR.obj
 0001:000e6450       ??$__destroy_mv_srcs@V?$reverse_iterator@PEAUFacialAnimationEntry@CAnimationSet@@@stlpmtx_std@@UFacialAnimationEntry@CAnimationSet@@@stlpmtx_std@@YAXV?$reverse_iterator@PEAUFacialAnimationEntry@CAnimationSet@@@0@0PEAUFacialAnimationEntry@CAnimationSet@@@Z 00000000315e7450 f i LoaderCHR.obj
 0001:000e64e0       ?append_raw@?$DynArray@UModelAnimationHeader@@HU?$SmallDynStorage@UModelAnimationHeader@@HUStandardAlloc@NAlloc@@@NArray@@@@QEAA?AU?$Array@UModelAnimationHeader@@HU?$ArrayStorage@UModelAnimationHeader@@H@NArray@@@@H@Z 00000000315e74e0 f i LoaderCHR.obj
 0001:000e6810       ?LoadFaceLib@CryCHRLoader@@AEAAXPEBD0PEAVCSkel@@@Z 00000000315e7810 f   LoaderCHR.obj
 0001:000e6b30       ??$__insertion_sort@PEAUFacialAnimationEntry@CAnimationSet@@U12@U?$less_stricmp@UFacialAnimationEntry@CAnimationSet@@@stl@@@priv@stlpmtx_std@@YAXPEAUFacialAnimationEntry@CAnimationSet@@00U?$less_stricmp@UFacialAnimationEntry@CAnimationSet@@@stl@@@Z 00000000315e7b30 f i LoaderCHR.obj
 0001:000e6be0       ??$uninitialized_copy@PEBUFacialAnimationEntry@CAnimationSet@@PEAU12@@stlpmtx_std@@YAPEAUFacialAnimationEntry@CAnimationSet@@PEBU12@0PEAU12@@Z 00000000315e7be0 f i LoaderCHR.obj
 0001:000e6c60       ??$sort_heap@PEAUFacialAnimationEntry@CAnimationSet@@U?$less_stricmp@UFacialAnimationEntry@CAnimationSet@@@stl@@@stlpmtx_std@@YAXPEAUFacialAnimationEntry@CAnimationSet@@0U?$less_stricmp@UFacialAnimationEntry@CAnimationSet@@@stl@@@Z 00000000315e7c60 f i LoaderCHR.obj
 0001:000e6d70       ?grow@?$DynArray@UModelAnimationHeader@@HU?$SmallDynStorage@UModelAnimationHeader@@HUStandardAlloc@NAlloc@@@NArray@@@@QEAAPEAUModelAnimationHeader@@HAEBU2@@Z 00000000315e7d70 f i LoaderCHR.obj
 0001:000e77c0       ??$_M_range_insert_aux@PEBUFacialAnimationEntry@CAnimationSet@@@?$_Impl_vector@UFacialAnimationEntry@CAnimationSet@@V?$allocator@UFacialAnimationEntry@CAnimationSet@@@stlpmtx_std@@@priv@stlpmtx_std@@AEAAXPEAUFacialAnimationEntry@CAnimationSet@@PEBU34@1_KAEBU__false_type@2@@Z 00000000315e87c0 f i LoaderCHR.obj
 0001:000e7a30       ??$__partial_sort@PEAUFacialAnimationEntry@CAnimationSet@@U12@U?$less_stricmp@UFacialAnimationEntry@CAnimationSet@@@stl@@@priv@stlpmtx_std@@YAXPEAUFacialAnimationEntry@CAnimationSet@@000U?$less_stricmp@UFacialAnimationEntry@CAnimationSet@@@stl@@@Z 00000000315e8a30 f i LoaderCHR.obj
 0001:000e8ca0       ?grow@?$DynArray@VCModelJoint@@HU?$SmallDynStorage@VCModelJoint@@HUStandardAlloc@NAlloc@@@NArray@@@@QEAAPEAVCModelJoint@@H@Z 00000000315e9ca0 f i LoaderCHR.obj
 0001:000e8d20       ??$_M_range_insert_realloc@PEBUFacialAnimationEntry@CAnimationSet@@@?$_Impl_vector@UFacialAnimationEntry@CAnimationSet@@V?$allocator@UFacialAnimationEntry@CAnimationSet@@@stlpmtx_std@@@priv@stlpmtx_std@@AEAAXPEAUFacialAnimationEntry@CAnimationSet@@PEBU34@1_K@Z 00000000315e9d20 f i LoaderCHR.obj
 0001:000e8f10       ?LoadAnimationFiles@CryCHRLoader@@AEAAIAEAVCParamLoader@@IPEAVCSkel@@@Z 00000000315e9f10 f   LoaderCHR.obj
 0001:000e9440       ?resize@?$DynArray@VCModelJoint@@HU?$SmallDynStorage@VCModelJoint@@HUStandardAlloc@NAlloc@@@NArray@@@@QEAAXH@Z 00000000315ea440 f i LoaderCHR.obj
 0001:000e94f0       ??$__introsort_loop@PEAUFacialAnimationEntry@CAnimationSet@@U12@_JU?$less_stricmp@UFacialAnimationEntry@CAnimationSet@@@stl@@@priv@stlpmtx_std@@YAXPEAUFacialAnimationEntry@CAnimationSet@@00_JU?$less_stricmp@UFacialAnimationEntry@CAnimationSet@@@stl@@@Z 00000000315ea4f0 f i LoaderCHR.obj
 0001:000ea0d0       ?LoadAnimations@CryCHRLoader@@AEAA_NAEAVCParamLoader@@PEAVCSkel@@@Z 00000000315eb0d0 f   LoaderCHR.obj
 0001:000eb1f0       ?LoadCHRPARAMS@CryCHRLoader@@QEAAXPEAVCSkel@@PEBD@Z 00000000315ec1f0 f   LoaderCHR.obj
 0001:000eb290       ?LoadNewCHR@CryCHRLoader@@QEAAPEAVCSkel@@PEBDI@Z 00000000315ec290 f   LoaderCHR.obj
 0001:000ed650       ?InMemory@CGlobalHeaderDBA@@QEAA_NXZ 00000000315ee650 f   LoaderDBA.obj
 0001:000ed660       ??_EIControllerRelocatableChain@@MEAAPEAXI@Z 00000000315ee660 f i LoaderDBA.obj
 0001:000ed660       ??_GIControllerRelocatableChain@@MEAAPEAXI@Z 00000000315ee660 f i LoaderDBA.obj
 0001:000ed690       ?Relocate@CInternalDatabaseInfo@@UEAAXPEAD0@Z 00000000315ee690 f   LoaderDBA.obj
 0001:000ed7a0       ?SizeOf_DBA@CGlobalHeaderDBA@@QEBA?B_KXZ 00000000315ee7a0 f   LoaderDBA.obj
 0001:000ed7f0       ??$__unguarded_linear_insert@PEAV?$_smart_ptr@VIController@@@@V1@VAnimCtrlSortPred@@@priv@stlpmtx_std@@YAXPEAV?$_smart_ptr@VIController@@@@V2@VAnimCtrlSortPred@@@Z 00000000315ee7f0 f i LoaderDBA.obj
 0001:000ed8a0       ??$__push_heap@PEAV?$_smart_ptr@VIController@@@@_JV1@VAnimCtrlSortPred@@@stlpmtx_std@@YAXPEAV?$_smart_ptr@VIController@@@@_J1V1@VAnimCtrlSortPred@@@Z 00000000315ee8a0 f i LoaderDBA.obj
 0001:000ed980       ?PhysicalizeAttachment@IAttachmentObject@@UEAA_NPEAUIAttachmentManager@@HHPEAUIPhysicalEntity@@AEBU?$Vec3_tpl@M@@@Z 00000000315ee980 f i AttachmentManager.obj
 0001:000ed980       ?GetS@CControllerPQLog@@UEBAEMAEAU?$Diag33_tpl@M@@@Z 00000000315ee980 f i ControllerPQLog.obj
 0001:000ed980       ?UpdatePhysicalizedAttachment@IAttachmentObject@@UEAA_NPEAUIAttachmentManager@@HPEAUIPhysicalEntity@@AEBU?$QuatT_tpl@M@@@Z 00000000315ee980 f i AttachmentManager.obj
 0001:000ed980       ?GetS@CController@@UEBAEMAEAU?$Diag33_tpl@M@@@Z 00000000315ee980 f i LoaderTCB.obj
 0001:000ed980       ?EnterScope@CDummyMemReplay@@UEAA_NW4Class@EMemReplayAllocClass@@GH@Z 00000000315ee980 f i AnimEventList.obj
 0001:000ed980       ?GetS@CControllerOptNonVirtual@@UEBAEMAEAU?$Diag33_tpl@M@@@Z 00000000315ee980 f i LoaderDBA.obj
 0001:000ed990       ?SetRotationKeyTimes@CControllerOptNonVirtual@@UEAAXIPEAD@Z 00000000315ee990 f i LoaderDBA.obj
 0001:000ed9b0       ?SetPositionKeyTimes@CControllerOptNonVirtual@@UEAAXIPEAD@Z 00000000315ee9b0 f i LoaderDBA.obj
 0001:000ed9d0       ?SetRotationKeys@CControllerOptNonVirtual@@UEAAXIPEAD@Z 00000000315ee9d0 f i LoaderDBA.obj
 0001:000ed9f0       ?SetPositionKeys@CControllerOptNonVirtual@@UEAAXIPEAD@Z 00000000315ee9f0 f i LoaderDBA.obj
 0001:000eda10       ?GetRotationFormat@CControllerOptNonVirtual@@UEBAIXZ 00000000315eea10 f i LoaderDBA.obj
 0001:000eda20       ?GetRotationKeyTimesFormat@CControllerOptNonVirtual@@UEBAIXZ 00000000315eea20 f i LoaderDBA.obj
 0001:000eda30       ?GetPositionFormat@CControllerOptNonVirtual@@UEBAIXZ 00000000315eea30 f i LoaderDBA.obj
 0001:000eda40       ?GetPositionKeyTimesFormat@CControllerOptNonVirtual@@UEBAIXZ 00000000315eea40 f i LoaderDBA.obj
 0001:000eda50       ?GetRotationKeyData@CControllerOptNonVirtual@@UEBAPEBDXZ 00000000315eea50 f i LoaderDBA.obj
 0001:000eda60       ?GetRotationKeyTimesData@CControllerOptNonVirtual@@UEBAPEBDXZ 00000000315eea60 f i LoaderDBA.obj
 0001:000eda70       ?GetPositionKeyData@CControllerOptNonVirtual@@UEBAPEBDXZ 00000000315eea70 f i LoaderDBA.obj
 0001:000eda80       ?GetPositionKeyTimesData@CControllerOptNonVirtual@@UEBAPEBDXZ 00000000315eea80 f i LoaderDBA.obj
 0001:000eda90       ?SizeOfController@CControllerOptNonVirtual@@UEBA_KXZ 00000000315eea90 f i LoaderDBA.obj
 0001:000edaa0       ?GetPosValueFromKey@CControllerOptNonVirtual@@QEBAXIAEAU?$Vec3_tpl@M@@@Z 00000000315eeaa0 f i LoaderDBA.obj
 0001:000edb10       ?ApproximateSizeOfThis@CControllerOptNonVirtual@@UEBA_KXZ 00000000315eeb10 f i LoaderDBA.obj
 0001:000edb80       ?GetRotationKeysNum@CControllerOptNonVirtual@@UEBA_KXZ 00000000315eeb80 f i LoaderDBA.obj
 0001:000edba0       ?GetPositionKeysNum@CControllerOptNonVirtual@@UEBA_KXZ 00000000315eeba0 f i LoaderDBA.obj
 0001:000edbc0       ??$GetKeyByteData@E@ControllerData@@QEBAIMAEAMPEBX@Z 00000000315eebc0 f i LoaderDBA.obj
 0001:000edcb0       ??$GetKeyByteData@G@ControllerData@@QEBAIMAEAMPEBX@Z 00000000315eecb0 f i LoaderDBA.obj
 0001:000eddb0       ??$GetKeyByteData@M@ControllerData@@QEBAIMAEAMPEBX@Z 00000000315eedb0 f i LoaderDBA.obj
 0001:000ede80       ?GetKeyBitData@ControllerData@@QEBAIMAEAM@Z 00000000315eee80 f i LoaderDBA.obj
 0001:000ee060       ??0CInternalDatabaseInfo@@QEAA@IAEBV?$CryStringT@D@@@Z 00000000315ef060 f   LoaderDBA.obj
 0001:000ee0c0       ??_ECInternalDatabaseInfo@@W7EAAPEAXI@Z 00000000315ef0c0 f i LoaderDBA.obj
 0001:000ee0d0       ??1CInternalDatabaseInfo@@UEAA@XZ 00000000315ef0d0 f   LoaderDBA.obj
 0001:000ee190       ?GetMemoryUsage@CGlobalHeaderDBA@@QEBAXPEAVICrySizer@@@Z 00000000315ef190 f   LoaderDBA.obj
 0001:000ee1f0       ??0CGlobalHeaderDBA@@QEAA@XZ 00000000315ef1f0 f   LoaderDBA.obj
 0001:000ee280       ??1CGlobalHeaderDBA@@QEAA@XZ 00000000315ef280 f   LoaderDBA.obj
 0001:000ee390       ??$copy_backward@PEAV?$_smart_ptr@VIController@@@@PEAV1@@stlpmtx_std@@YAPEAV?$_smart_ptr@VIController@@@@PEAV1@00@Z 00000000315ef390 f i LoaderDBA.obj
 0001:000ee410       ??$__adjust_heap@PEAV?$_smart_ptr@VIController@@@@_JV1@VAnimCtrlSortPred@@@stlpmtx_std@@YAXPEAV?$_smart_ptr@VIController@@@@_J1V1@VAnimCtrlSortPred@@@Z 00000000315ef410 f i LoaderDBA.obj
 0001:000ee530       ?GetPosValue@CControllerOptNonVirtual@@QEBA?AU?$Vec3_tpl@M@@M@Z 00000000315ef530 f i LoaderDBA.obj
 0001:000ee750       ?CreateDatabaseDBA@CGlobalHeaderDBA@@QEAAXPEBD@Z 00000000315ef750 f   LoaderDBA.obj
 0001:000ee960       ?StartStreamingDBA@CGlobalHeaderDBA@@QEAA_N_N@Z 00000000315ef960 f   LoaderDBA.obj
 0001:000eeaa0       ??_ECInternalDatabaseInfo@@UEAAPEAXI@Z 00000000315efaa0 f i LoaderDBA.obj
 0001:000eeaa0       ??_GCInternalDatabaseInfo@@UEAAPEAXI@Z 00000000315efaa0 f i LoaderDBA.obj
 0001:000eead0       ?ReportLoadError@CGlobalHeaderDBA@@QEAAXPEBD0@Z 00000000315efad0 f   LoaderDBA.obj
 0001:000eeb60       ??$__linear_insert@PEAV?$_smart_ptr@VIController@@@@V1@VAnimCtrlSortPred@@@priv@stlpmtx_std@@YAXPEAV?$_smart_ptr@VIController@@@@0V2@VAnimCtrlSortPred@@@Z 00000000315efb60 f i LoaderDBA.obj
 0001:000eec10       ??$__make_heap@PEAV?$_smart_ptr@VIController@@@@VAnimCtrlSortPred@@V1@_J@stlpmtx_std@@YAXPEAV?$_smart_ptr@VIController@@@@0VAnimCtrlSortPred@@0PEA_J@Z 00000000315efc10 f i LoaderDBA.obj
 0001:000eeca0       ?GetP@CControllerOptNonVirtual@@UEBAEMAEAU?$Vec3_tpl@M@@@Z 00000000315efca0 f i LoaderDBA.obj
 0001:000eece0       ?CompleteStreamingDBA@CGlobalHeaderDBA@@QEAAXPEAUCInternalDatabaseInfo@@@Z 00000000315efce0 f   LoaderDBA.obj
 0001:000eee50       ?StreamOnComplete@CInternalDatabaseInfo@@UEAAXPEAVIReadStream@@I@Z 00000000315efe50 f   LoaderDBA.obj
 0001:000eeea0       ?DeleteDatabaseDBA@CGlobalHeaderDBA@@QEAAXXZ 00000000315efea0 f   LoaderDBA.obj
 0001:000ef0c0       ??$__insertion_sort@PEAV?$_smart_ptr@VIController@@@@V1@VAnimCtrlSortPred@@@priv@stlpmtx_std@@YAXPEAV?$_smart_ptr@VIController@@@@00VAnimCtrlSortPred@@@Z 00000000315f00c0 f i LoaderDBA.obj
 0001:000ef140       ??$__final_insertion_sort@PEAV?$_smart_ptr@VIController@@@@VAnimCtrlSortPred@@@priv@stlpmtx_std@@YAXPEAV?$_smart_ptr@VIController@@@@0VAnimCtrlSortPred@@@Z 00000000315f0140 f i LoaderDBA.obj
 0001:000ef1d0       ??$sort_heap@PEAV?$_smart_ptr@VIController@@@@VAnimCtrlSortPred@@@stlpmtx_std@@YAXPEAV?$_smart_ptr@VIController@@@@0VAnimCtrlSortPred@@@Z 00000000315f01d0 f i LoaderDBA.obj
 0001:000ef2c0       ?resize@?$DynArray@IHU?$SmallDynStorage@IHUStandardAlloc@NAlloc@@@NArray@@@@QEAAXH@Z 00000000315f02c0 f i LoaderDBA.obj
 0001:000ef300       ??$__partial_sort@PEAV?$_smart_ptr@VIController@@@@V1@VAnimCtrlSortPred@@@priv@stlpmtx_std@@YAXPEAV?$_smart_ptr@VIController@@@@000VAnimCtrlSortPred@@@Z 00000000315f0300 f i LoaderDBA.obj
 0001:000ef410       ?InitControllerLookup@GlobalAnimationHeaderCAF@@QEAAXI@Z 00000000315f0410 f i LoaderDBA.obj
 0001:000ef4c0       ??$__introsort_loop@PEAV?$_smart_ptr@VIController@@@@V1@_JVAnimCtrlSortPred@@@priv@stlpmtx_std@@YAXPEAV?$_smart_ptr@VIController@@@@00_JVAnimCtrlSortPred@@@Z 00000000315f04c0 f i LoaderDBA.obj
 0001:000ef640       ??$sort@PEAV?$_smart_ptr@VIController@@@@VAnimCtrlSortPred@@@stlpmtx_std@@YAXPEAV?$_smart_ptr@VIController@@@@0VAnimCtrlSortPred@@@Z 00000000315f0640 f i LoaderDBA.obj
 0001:000ef6b0       ?ReadController905@CInternalDatabaseInfo@@QEAA_NPEAUChunkDesc@IChunkFile@@_N@Z 00000000315f06b0 f   LoaderDBA.obj
 0001:000f1530       ?LoadChunks@CInternalDatabaseInfo@@QEAA_NPEAUIChunkFile@@_N@Z 00000000315f2530 f   LoaderDBA.obj
 0001:000f1640       ?LoadDatabaseDBA@CGlobalHeaderDBA@@QEAAXPEBD@Z 00000000315f2640 f   LoaderDBA.obj
 0001:000f17f0       ?StreamAsyncOnComplete@CInternalDatabaseInfo@@UEAAXPEAVIReadStream@@I@Z 00000000315f27f0 f   LoaderDBA.obj
 0001:000f1b30       ??4?$_smart_ptr@VIKeyTimesInformation@@@@QEAAAEAV0@PEAVIKeyTimesInformation@@@Z 00000000315f2b30 f i LoaderTCB.obj
 0001:000f1bb0       ??$move_init@UCryTCB3Key@@@NArray@@YAXPEAUCryTCB3Key@@0_K@Z 00000000315f2bb0 f i LoaderTCB.obj
 0001:000f1c10       ?GetOPS@CControllerOptNonVirtual@@UEBAEMAEAU?$Quat_tpl@M@@AEAU?$Vec3_tpl@M@@AEAU?$Diag33_tpl@M@@@Z 00000000315f2c10 f i LoaderDBA.obj
 0001:000f1c10       ?GetOPS@CController@@UEBAEMAEAU?$Quat_tpl@M@@AEAU?$Vec3_tpl@M@@AEAU?$Diag33_tpl@M@@@Z 00000000315f2c10 f i LoaderTCB.obj
 0001:000f1c80       ?SizeOfController@CController@@UEBA_KXZ 00000000315f2c80 f i LoaderTCB.obj
 0001:000f1ce0       ?ApproximateSizeOfThis@CControllerTCB@@UEBA_KXZ 00000000315f2ce0 f i LoaderCGA.obj
 0001:000f1ce0       ?ApproximateSizeOfThis@CControllerPQLog@@UEBA_KXZ 00000000315f2ce0 f i ControllerPQLog.obj
 0001:000f1ce0       ?ApproximateSizeOfThis@CController@@UEBA_KXZ 00000000315f2ce0 f i LoaderTCB.obj
 0001:000f1cf0       ?GetO_numKey@CController@@UEBAHXZ 00000000315f2cf0 f i LoaderTCB.obj
 0001:000f1d10       ?GetP_numKey@CController@@UEBAHXZ 00000000315f2d10 f i LoaderTCB.obj
 0001:000f1d30       ?GetRotationKeysNum@CController@@UEBA_KXZ 00000000315f2d30 f i LoaderTCB.obj
 0001:000f1d60       ?GetPositionKeysNum@CController@@UEBA_KXZ 00000000315f2d60 f i LoaderTCB.obj
 0001:000f1d90       ??_ECController@@UEAAPEAXI@Z 00000000315f2d90 f i LoaderTCB.obj
 0001:000f1d90       ??_GCController@@UEAAPEAXI@Z 00000000315f2d90 f i LoaderTCB.obj
 0001:000f1e00       ??$move_init@UPQLog@@@NArray@@YAXPEAUPQLog@@0_K@Z 00000000315f2e00 f i LoaderTCB.obj
 0001:000f1e50       ?resize_raw@?$SmallDynStorage@PEAU?$DynArray@UCryTCB3Key@@HU?$SmallDynStorage@UCryTCB3Key@@HUStandardAlloc@NAlloc@@@NArray@@@@HUStandardAlloc@NAlloc@@@NArray@@QEAAXHH_N@Z 00000000315f2e50 f i LoaderTCB.obj
 0001:000f1fe0       ?resize_raw@?$SmallDynStorage@PEAU?$DynArray@UCryTCBQKey@@HU?$SmallDynStorage@UCryTCBQKey@@HUStandardAlloc@NAlloc@@@NArray@@@@HUStandardAlloc@NAlloc@@@NArray@@QEAAXHH_N@Z 00000000315f2fe0 f i LoaderTCB.obj
 0001:000f2170       ?set_size@?$SmallDynStorage@FHUStandardAlloc@NAlloc@@@NArray@@QEAAXH@Z 00000000315f3170 f i ParamLoader.obj
 0001:000f2170       ?set_size@?$SmallDynStorage@UTCBFlags@@HUStandardAlloc@NAlloc@@@NArray@@QEAAXH@Z 00000000315f3170 f i LoaderTCB.obj
 0001:000f2170       ?set_size@?$SmallDynStorage@GHUStandardAlloc@NAlloc@@@NArray@@QEAAXH@Z 00000000315f3170 f i LoaderCHR.obj
 0001:000f2210       ?resize_raw@?$SmallDynStorage@UTCBFlags@@HUStandardAlloc@NAlloc@@@NArray@@QEAAXHH_N@Z 00000000315f3210 f i LoaderTCB.obj
 0001:000f23a0       ?resize_raw@?$SmallDynStorage@UCryTCB3Key@@HUStandardAlloc@NAlloc@@@NArray@@QEAAXHH_N@Z 00000000315f33a0 f i LoaderTCB.obj
 0001:000f2520       ?SetKeyTimesInformation@ITrackInformation@@QEAAXAEAV?$_smart_ptr@VIKeyTimesInformation@@@@@Z 00000000315f3520 f i LoaderTCB.obj
 0001:000f25a0       ??_GITrackInformation@@UEAAPEAXI@Z 00000000315f35a0 f i LoaderTCB.obj
 0001:000f25a0       ??_EITrackInformation@@UEAAPEAXI@Z 00000000315f35a0 f i LoaderTCB.obj
 0001:000f2610       ??1IPositionController@@UEAA@XZ 00000000315f3610 f i LoaderTCB.obj
 0001:000f2680       ?SetRotationStorage@IRotationController@@UEAAXAEAPEAVITrackRotationStorage@@@Z 00000000315f3680 f i LoaderTCB.obj
 0001:000f2680       ?SetPositionStorage@IPositionController@@UEAAXAEAPEAVITrackPositionStorage@@@Z 00000000315f3680 f i LoaderTCB.obj
 0001:000f2690       ?GetData@IRotationController@@UEAAPEADXZ 00000000315f3690 f i LoaderTCB.obj
 0001:000f2690       ?GetData@IPositionController@@UEAAPEADXZ 00000000315f3690 f i LoaderTCB.obj
 0001:000f26a0       ?SizeOfPosController@IPositionController@@UEAA_KXZ 00000000315f36a0 f i LoaderTCB.obj
 0001:000f26f0       ??_GIPositionController@@UEAAPEAXI@Z 00000000315f36f0 f i LoaderTCB.obj
 0001:000f26f0       ??_EIPositionController@@UEAAPEAXI@Z 00000000315f36f0 f i LoaderTCB.obj
 0001:000f2720       ?GetFormat@IPositionController@@UEAAIXZ 00000000315f3720 f i LoaderTCB.obj
 0001:000f2720       ?GetFormat@IRotationController@@UEAAIXZ 00000000315f3720 f i LoaderTCB.obj
 0001:000f2730       ?SizeOfRotController@IRotationController@@UEAA_KXZ 00000000315f3730 f i LoaderTCB.obj
 0001:000f2770       ??1IRotationController@@UEAA@XZ 00000000315f3770 f i LoaderTCB.obj
 0001:000f27e0       ??_GIRotationController@@UEAAPEAXI@Z 00000000315f37e0 f i LoaderTCB.obj
 0001:000f27e0       ??_EIRotationController@@UEAAPEAXI@Z 00000000315f37e0 f i LoaderTCB.obj
 0001:000f2810       ?GetMemoryUsage@CController@@UEBAXPEAVICrySizer@@@Z 00000000315f3810 f i LoaderTCB.obj
 0001:000f2850       ?resize_raw@?$SmallDynStorage@UPQLog@@HUStandardAlloc@NAlloc@@@NArray@@QEAAXHH_N@Z 00000000315f3850 f i LoaderTCB.obj
 0001:000f29d0       ??0CLoaderTCB@@QEAA@XZ     00000000315f39d0 f   LoaderTCB.obj
 0001:000f2a00       ??1CLoaderTCB@@QEAA@XZ     00000000315f3a00 f   LoaderTCB.obj
 0001:000f2a90       ?ReadMotionParameters@CLoaderTCB@@AEAA_NPEAUChunkDesc@IChunkFile@@@Z 00000000315f3a90 f   LoaderTCB.obj
 0001:000f2b40       ?Blend@QuatLerp@@SAXAEAU?$Quat_tpl@M@@AEBU2@1M@Z 00000000315f3b40 f i LoaderTCB.obj
 0001:000f2ca0       ?GetValue@?$CAdvancedTrackInformation@U?$Quat_tpl@M@@UQuatLerp@@VIRotationController@@@@UEAAXMAEAU?$Quat_tpl@M@@@Z 00000000315f3ca0 f i LoaderTCB.obj
 0001:000f2d70       ?GetValue@?$CAdvancedTrackInformation@U?$Vec3_tpl@M@@UVec3Lerp@@VIPositionController@@@@UEAAXMAEAU?$Vec3_tpl@M@@@Z 00000000315f3d70 f i LoaderTCB.obj
 0001:000f2e70       ??_E?$CAdvancedTrackInformation@U?$Quat_tpl@M@@UQuatLerp@@VIRotationController@@@@UEAAPEAXI@Z 00000000315f3e70 f i LoaderTCB.obj
 0001:000f2e70       ??_G?$CAdvancedTrackInformation@U?$Quat_tpl@M@@UQuatLerp@@VIRotationController@@@@UEAAPEAXI@Z 00000000315f3e70 f i LoaderTCB.obj
 0001:000f2eb0       ??_E?$CAdvancedTrackInformation@U?$Vec3_tpl@M@@UVec3Lerp@@VIPositionController@@@@UEAAPEAXI@Z 00000000315f3eb0 f i LoaderTCB.obj
 0001:000f2eb0       ??_G?$CAdvancedTrackInformation@U?$Vec3_tpl@M@@UVec3Lerp@@VIPositionController@@@@UEAAPEAXI@Z 00000000315f3eb0 f i LoaderTCB.obj
 0001:000f2ef0       ?set_size@?$SmallDynStorage@UCryTCB3Key@@HUStandardAlloc@NAlloc@@@NArray@@QEAAXH@Z 00000000315f3ef0 f i LoaderTCB.obj
 0001:000f2fa0       ?set_size@?$SmallDynStorage@UGeomQuery@@HUStandardAlloc@NAlloc@@@NArray@@QEAAXH@Z 00000000315f3fa0 f i CharacterInstance.obj
 0001:000f2fa0       ?set_size@?$SmallDynStorage@UExtSkinVertex@@HUStandardAlloc@NAlloc@@@NArray@@QEAAXH@Z 00000000315f3fa0 f i LoaderSKIN.obj
 0001:000f2fa0       ?set_size@?$SmallDynStorage@UVirtualExample3D@@HUStandardAlloc@NAlloc@@@NArray@@QEAAXH@Z 00000000315f3fa0 f i ParametricSampler.obj
 0001:000f2fa0       ?set_size@?$SmallDynStorage@UDebugInstances@@HUStandardAlloc@NAlloc@@@NArray@@QEAAXH@Z 00000000315f3fa0 f i CharacterManager.obj
 0001:000f2fa0       ?set_size@?$SmallDynStorage@UADIKTarget@@HUStandardAlloc@NAlloc@@@NArray@@QEAAXH@Z 00000000315f3fa0 f i ParamLoader.obj
 0001:000f2fa0       ?set_size@?$SmallDynStorage@UCryTCBQKey@@HUStandardAlloc@NAlloc@@@NArray@@QEAAXH@Z 00000000315f3fa0 f i LoaderTCB.obj
 0001:000f3050       ?expand_raw@?$DynArray@UPQLog@@HU?$SmallDynStorage@UPQLog@@HUStandardAlloc@NAlloc@@@NArray@@@@IEAAPEAUPQLog@@PEAU2@H@Z 00000000315f4050 f i LoaderTCB.obj
 0001:000f3110       ?expand_raw@?$DynArray@UCryTCB3Key@@HU?$SmallDynStorage@UCryTCB3Key@@HUStandardAlloc@NAlloc@@@NArray@@@@IEAAPEAUCryTCB3Key@@PEAU2@H@Z 00000000315f4110 f i LoaderTCB.obj
 0001:000f31d0       ?append_raw@?$DynArray@UTCBFlags@@HU?$SmallDynStorage@UTCBFlags@@HUStandardAlloc@NAlloc@@@NArray@@@@QEAA?AU?$Array@UTCBFlags@@HU?$ArrayStorage@UTCBFlags@@H@NArray@@@@H@Z 00000000315f41d0 f i LoaderTCB.obj
 0001:000f3290       ?append_raw@?$DynArray@PEAU?$DynArray@UCryTCB3Key@@HU?$SmallDynStorage@UCryTCB3Key@@HUStandardAlloc@NAlloc@@@NArray@@@@HU?$SmallDynStorage@PEAU?$DynArray@UCryTCB3Key@@HU?$SmallDynStorage@UCryTCB3Key@@HUStandardAlloc@NAlloc@@@NArray@@@@HUStandardAlloc@NAlloc@@@NArray@@@@QEAA?AU?$Array@PEAU?$DynArray@UCryTCB3Key@@HU?$SmallDynStorage@UCryTCB3Key@@HUStandardAlloc@NAlloc@@@NArray@@@@HU?$ArrayStorage@PEAU?$DynArray@UCryTCB3Key@@HU?$SmallDynStorage@UCryTCB3Key@@HUStandardAlloc@NAlloc@@@NArray@@@@H@NArray@@@@H@Z 00000000315f4290 f i LoaderTCB.obj
 0001:000f3350       ?append_raw@?$DynArray@PEAU?$DynArray@UCryTCBQKey@@HU?$SmallDynStorage@UCryTCBQKey@@HUStandardAlloc@NAlloc@@@NArray@@@@HU?$SmallDynStorage@PEAU?$DynArray@UCryTCBQKey@@HU?$SmallDynStorage@UCryTCBQKey@@HUStandardAlloc@NAlloc@@@NArray@@@@HUStandardAlloc@NAlloc@@@NArray@@@@QEAA?AU?$Array@PEAU?$DynArray@UCryTCBQKey@@HU?$SmallDynStorage@UCryTCBQKey@@HUStandardAlloc@NAlloc@@@NArray@@@@HU?$ArrayStorage@PEAU?$DynArray@UCryTCBQKey@@HU?$SmallDynStorage@UCryTCBQKey@@HUStandardAlloc@NAlloc@@@NArray@@@@H@NArray@@@@H@Z 00000000315f4350 f i LoaderTCB.obj
 0001:000f3410       ??$move_init@UCryTCBQKey@@@NArray@@YAXPEAUCryTCBQKey@@0_K@Z 00000000315f4410 f i LoaderTCB.obj
 0001:000f3620       ?resize_raw@?$SmallDynStorage@UCryTCBQKey@@HUStandardAlloc@NAlloc@@@NArray@@QEAAXHH_N@Z 00000000315f4620 f i LoaderTCB.obj
 0001:000f37a0       ?push_back@?$DynArray@IHU?$SmallDynStorage@IHUStandardAlloc@NAlloc@@@NArray@@@@QEAAPEAIAEBI@Z 00000000315f47a0 f i LoaderTCB.obj
 0001:000f3800       ?resize@?$DynArray@UPQLog@@HU?$SmallDynStorage@UPQLog@@HUStandardAlloc@NAlloc@@@NArray@@@@QEAAXH@Z 00000000315f4800 f i LoaderTCB.obj
 0001:000f3840       ??0?$DynArray@UCryTCB3Key@@HU?$SmallDynStorage@UCryTCB3Key@@HUStandardAlloc@NAlloc@@@NArray@@@@QEAA@XZ 00000000315f4840 f i LoaderTCB.obj
 0001:000f38a0       ??0?$DynArray@UCryTCBQKey@@HU?$SmallDynStorage@UCryTCBQKey@@HUStandardAlloc@NAlloc@@@NArray@@@@QEAA@XZ 00000000315f48a0 f i LoaderTCB.obj
 0001:000f3900       ?expand_raw@?$DynArray@UCryTCBQKey@@HU?$SmallDynStorage@UCryTCBQKey@@HUStandardAlloc@NAlloc@@@NArray@@@@IEAAPEAUCryTCBQKey@@PEAU2@H@Z 00000000315f4900 f i LoaderTCB.obj
 0001:000f39c0       ??0CHeaderTCB@@QEAA@XZ     00000000315f49c0 f i LoaderTCB.obj
 0001:000f3c10       ??1CHeaderTCB@@UEAA@XZ     00000000315f4c10 f i LoaderTCB.obj
 0001:000f41c0       ??_ECHeaderTCB@@UEAAPEAXI@Z 00000000315f51c0 f i LoaderTCB.obj
 0001:000f41c0       ??_GCHeaderTCB@@UEAAPEAXI@Z 00000000315f51c0 f i LoaderTCB.obj
 0001:000f41f0       ?resize@?$DynArray@UCryTCBQKey@@HU?$SmallDynStorage@UCryTCBQKey@@HUStandardAlloc@NAlloc@@@NArray@@@@QEAAXH@Z 00000000315f51f0 f i LoaderTCB.obj
 0001:000f4230       ?ReadController@CLoaderTCB@@AEAA_NPEAUChunkDesc@IChunkFile@@@Z 00000000315f5230 f   LoaderTCB.obj
 0001:000f52e0       ?LoadChunksTCB@CLoaderTCB@@AEAA_NPEAUIChunkFile@@@Z 00000000315f62e0 f   LoaderTCB.obj
 0001:000f56d0       ?LoadTCB@CLoaderTCB@@QEAAPEAUCHeaderTCB@@PEBDPEAUIChunkFile@@PEAVILoaderCAFListener@@@Z 00000000315f66d0 f   LoaderTCB.obj
 0001:000f5990       ?LoadTCB@CLoaderTCB@@QEAAPEAUCHeaderTCB@@PEBDPEAVILoaderCAFListener@@@Z 00000000315f6990 f   LoaderTCB.obj
 0001:000f5a00       ?Warning@@YAXPEBDW4EValidatorSeverity@@0ZZ 00000000315f6a00 f   ParamLoader.obj
 0001:000f5a60       ??$__find_if@PEAUSAnimFile@@UFindByAliasName@?A0x32a97809@@@priv@stlpmtx_std@@YAPEAUSAnimFile@@PEAU2@0UFindByAliasName@?A0x32a97809@@AEBUrandom_access_iterator_tag@1@@Z 00000000315f6a60 f i ParamLoader.obj
 0001:000f5b70       ?GetFile@PathUtil@@YAPEBDPEBD@Z 00000000315f6b70 f i ParamLoader.obj
 0001:000f5bc0       ?MatchWildcard@PathUtil@@YA_NPEBD0@Z 00000000315f6bc0 f i ParamLoader.obj
 0001:000f5cb0       ??$move_init@UADIKTarget@@@NArray@@YAXPEAUADIKTarget@@0_K@Z 00000000315f6cb0 f i ParamLoader.obj
 0001:000f5d00       ?GetNameCStr@CSkel@@QEBAPEBDXZ 00000000315f6d00 f i ParamLoader.obj
 0001:000f5d50       ?ListProcessed@CParamLoader@@AEAAHPEBD@Z 00000000315f6d50 f   ParamLoader.obj
 0001:000f5de0       ?resize_raw@?$SmallDynStorage@USJointsAimIK_Rot@@HUStandardAlloc@NAlloc@@@NArray@@QEAAXHH_N@Z 00000000315f6de0 f i ParamLoader.obj
 0001:000f5fa0       ?resize_raw@?$SmallDynStorage@USJointsAimIK_Pos@@HUStandardAlloc@NAlloc@@@NArray@@QEAAXHH_N@Z 00000000315f6fa0 f i ParamLoader.obj
 0001:000f6140       ?resize_raw@?$SmallDynStorage@USRecoilJoints@@HUStandardAlloc@NAlloc@@@NArray@@QEAAXHH_N@Z 00000000315f7140 f i ParamLoader.obj
 0001:000f6300       ?resize_raw@?$SmallDynStorage@UProcAdjust@@HUStandardAlloc@NAlloc@@@NArray@@QEAAXHH_N@Z 00000000315f7300 f i ParamLoader.obj
 0001:000f64a0       ?resize_raw@?$SmallDynStorage@UADIKTarget@@HUStandardAlloc@NAlloc@@@NArray@@QEAAXHH_N@Z 00000000315f74a0 f i ParamLoader.obj
 0001:000f6620       ?set_size@?$SmallDynStorage@USJointProperty@@HUStandardAlloc@NAlloc@@@NArray@@QEAAXH@Z 00000000315f7620 f i Model.obj
 0001:000f6620       ?set_size@?$SmallDynStorage@UPQLog@@HUStandardAlloc@NAlloc@@@NArray@@QEAAXH@Z 00000000315f7620 f i LoaderTCB.obj
 0001:000f6620       ?set_size@?$SmallDynStorage@USRecoilJoints@@HUStandardAlloc@NAlloc@@@NArray@@QEAAXH@Z 00000000315f7620 f i ParamLoader.obj
 0001:000f6620       ?set_size@?$SmallDynStorage@USJointsAimIK_Rot@@HUStandardAlloc@NAlloc@@@NArray@@QEAAXH@Z 00000000315f7620 f i ParamLoader.obj
 0001:000f6620       ?set_size@?$SmallDynStorage@USEntry@CPoseModifierQueue@@HUStandardAlloc@NAlloc@@@NArray@@QEAAXH@Z 00000000315f7620 f i TransitionQueue.obj
 0001:000f66d0       ?set_size@?$SmallDynStorage@USAnimListInfo@@HUStandardAlloc@NAlloc@@@NArray@@QEAAXH@Z 00000000315f76d0 f i ParamLoader.obj
 0001:000f66d0       ?set_size@?$SmallDynStorage@VCAnimation@@HUStandardAlloc@NAlloc@@@NArray@@QEAAXH@Z 00000000315f76d0 f i TransitionQueue.obj
 0001:000f6780       ??$__find@PEAV?$CryStringT@D@@PEBD@priv@stlpmtx_std@@YAPEAV?$CryStringT@D@@PEAV2@0AEBQEBDAEBUrandom_access_iterator_tag@1@@Z 00000000315f7780 f i ParamLoader.obj
 0001:000f6960       ?NoAnimationAliasInDependencies@CParamLoader@@AEAA_NAEAUSAnimListInfo@@PEBD@Z 00000000315f7960 f   ParamLoader.obj
 0001:000f6a60       ?NoFacialAnimationAliasInDependencies@CParamLoader@@AEAA_NAEAUSAnimListInfo@@PEBD@Z 00000000315f7a60 f   ParamLoader.obj
 0001:000f6b60       ?set_size@?$SmallDynStorage@U?$Quat_tpl@M@@HUStandardAlloc@NAlloc@@@NArray@@QEAAXH@Z 00000000315f7b60 f i LoaderSKIN.obj
 0001:000f6b60       ?set_size@?$SmallDynStorage@UModelAnimationHeader@@HUStandardAlloc@NAlloc@@@NArray@@QEAAXH@Z 00000000315f7b60 f i LoaderCHR.obj
 0001:000f6b60       ?set_size@?$SmallDynStorage@UAimIKPose@@HUStandardAlloc@NAlloc@@@NArray@@QEAAXH@Z 00000000315f7b60 f i CharacterManager.obj
 0001:000f6b60       ?set_size@?$SmallDynStorage@USVertexFrameState@@HUStandardAlloc@NAlloc@@@NArray@@QEAAXH@Z 00000000315f7b60 f i VertexAnimation.obj
 0001:000f6b60       ?set_size@?$SmallDynStorage@URChunk@@HUStandardAlloc@NAlloc@@@NArray@@QEAAXH@Z 00000000315f7b60 f i LoaderSKIN.obj
 0001:000f6b60       ?set_size@?$SmallDynStorage@USCRCName@@HUStandardAlloc@NAlloc@@@NArray@@QEAAXH@Z 00000000315f7b60 f i CharacterManager.obj
 0001:000f6b60       ?set_size@?$SmallDynStorage@UProcAdjust@@HUStandardAlloc@NAlloc@@@NArray@@QEAAXH@Z 00000000315f7b60 f i ParamLoader.obj
 0001:000f6b60       ?set_size@?$SmallDynStorage@UIdxAndName@@HUStandardAlloc@NAlloc@@@NArray@@QEAAXH@Z 00000000315f7b60 f i ParamLoader.obj
 0001:000f6b60       ?set_size@?$SmallDynStorage@USJointInfo@CSkin@@HUStandardAlloc@NAlloc@@@NArray@@QEAAXH@Z 00000000315f7b60 f i LoaderSKIN.obj
 0001:000f6b60       ?set_size@?$SmallDynStorage@UBlendSpaceInfo@@HUStandardAlloc@NAlloc@@@NArray@@QEAAXH@Z 00000000315f7b60 f i CharacterManager.obj
 0001:000f6b60       ?set_size@?$SmallDynStorage@USJointsAimIK_Pos@@HUStandardAlloc@NAlloc@@@NArray@@QEAAXH@Z 00000000315f7b60 f i ParamLoader.obj
 0001:000f6c10       ?expand_raw@?$DynArray@UADIKTarget@@HU?$SmallDynStorage@UADIKTarget@@HUStandardAlloc@NAlloc@@@NArray@@@@IEAAPEAUADIKTarget@@PEAU2@H@Z 00000000315f7c10 f i ParamLoader.obj
 0001:000f6cd0       ?resize_raw@?$SmallDynStorage@FHUStandardAlloc@NAlloc@@@NArray@@QEAAXHH_N@Z 00000000315f7cd0 f i ParamLoader.obj
 0001:000f6e60       ?resize_raw@?$SmallDynStorage@UIdxAndName@@HUStandardAlloc@NAlloc@@@NArray@@QEAAXHH_N@Z 00000000315f7e60 f i ParamLoader.obj
 0001:000f7000       ?set_size@?$SmallDynStorage@USAnimFile@@HUStandardAlloc@NAlloc@@@NArray@@QEAAXH@Z 00000000315f8000 f i ParamLoader.obj
 0001:000f70c0       ??$GetParentDirectoryStackString@D$0CAA@@PathUtil@@YA?AV?$CryStackStringT@D$0CAA@@@AEBV1@H@Z 00000000315f80c0 f i ParamLoader.obj
 0001:000f7180       ?NoModelTracksDatabaseInDependencies@CParamLoader@@AEAA_NAEAUSAnimListInfo@@PEBD@Z 00000000315f8180 f   ParamLoader.obj
 0001:000f7260       ?LoadIKDefFeetLock@CParamLoader@@AEAA_NVXmlNodeRef@@@Z 00000000315f8260 f   ParamLoader.obj
 0001:000f73a0       ?clear@?$DynArray@USJointsAimIK_Rot@@HU?$SmallDynStorage@USJointsAimIK_Rot@@HUStandardAlloc@NAlloc@@@NArray@@@@QEAAXXZ 00000000315f83a0 f i ParamLoader.obj
 0001:000f7470       ?clear@?$DynArray@USJointsAimIK_Pos@@HU?$SmallDynStorage@USJointsAimIK_Pos@@HUStandardAlloc@NAlloc@@@NArray@@@@QEAAXXZ 00000000315f8470 f i ParamLoader.obj
 0001:000f7540       ?clear@?$DynArray@UProcAdjust@@HU?$SmallDynStorage@UProcAdjust@@HUStandardAlloc@NAlloc@@@NArray@@@@QEAAXXZ 00000000315f8540 f i ParamLoader.obj
 0001:000f7610       ?clear@?$DynArray@UADIKTarget@@HU?$SmallDynStorage@UADIKTarget@@HUStandardAlloc@NAlloc@@@NArray@@@@QEAAXXZ 00000000315f8610 f i ParamLoader.obj
 0001:000f76e0       ?expand_raw@?$DynArray@USAnimFile@@HU?$SmallDynStorage@USAnimFile@@HUStandardAlloc@NAlloc@@@NArray@@@@IEAAPEAUSAnimFile@@PEAU2@H@Z 00000000315f86e0 f i ParamLoader.obj
 0001:000f77a0       ??0?$_Vector_base@UFacialAnimationEntry@CAnimationSet@@V?$allocator@UFacialAnimationEntry@CAnimationSet@@@stlpmtx_std@@@priv@stlpmtx_std@@QEAA@_KAEBV?$allocator@UFacialAnimationEntry@CAnimationSet@@@2@@Z 00000000315f87a0 f i ParamLoader.obj
 0001:000f7880       ?TrimRight@?$CryStringT@D@@QEAAAEAV1@D@Z 00000000315f8880 f i ParamLoader.obj
 0001:000f7930       ??0SAnimFile@@QEAA@AEBV?$CryStackStringT@D$0CAA@@@0@Z 00000000315f8930 f i ParamLoader.obj
 0001:000f7c00       ?append_raw@?$DynArray@FHU?$SmallDynStorage@FHUStandardAlloc@NAlloc@@@NArray@@@@QEAA?AU?$Array@FHU?$ArrayStorage@FH@NArray@@@@H@Z 00000000315f8c00 f i ParamLoader.obj
 0001:000f7cc0       ?append_raw@?$DynArray@UIdxAndName@@HU?$SmallDynStorage@UIdxAndName@@HUStandardAlloc@NAlloc@@@NArray@@@@QEAA?AU?$Array@UIdxAndName@@HU?$ArrayStorage@UIdxAndName@@H@NArray@@@@H@Z 00000000315f8cc0 f i ParamLoader.obj
 0001:000f7d80       ?destroy@?$DynArray@UModelAnimationHeader@@HU?$SmallDynStorage@UModelAnimationHeader@@HUStandardAlloc@NAlloc@@@NArray@@@@IEAAXXZ 00000000315f8d80 f i ParamLoader.obj
 0001:000f7d80       ?destroy@?$DynArray@UBlendSpaceInfo@@HU?$SmallDynStorage@UBlendSpaceInfo@@HUStandardAlloc@NAlloc@@@NArray@@@@IEAAXXZ 00000000315f8d80 f i CharacterManager.obj
 0001:000f7e00       ??1IKLimbType@@QEAA@XZ     00000000315f8e00 f i ParamLoader.obj
 0001:000f7e90       ?MemFindFirst@CParamLoader@@AEAA?AUCAF_ID@@PEAPEBDPEBDIU2@@Z 00000000315f8e90 f   ParamLoader.obj
 0001:000f81b0       ?grow@?$DynArray@USAnimFile@@HU?$SmallDynStorage@USAnimFile@@HUStandardAlloc@NAlloc@@@NArray@@@@QEAAPEAUSAnimFile@@HAEBU2@@Z 00000000315f91b0 f i ParamLoader.obj
 0001:000f8240       ??0?$DynArray@FHU?$SmallDynStorage@FHUStandardAlloc@NAlloc@@@NArray@@@@QEAA@AEBU0@@Z 00000000315f9240 f i ParamLoader.obj
 0001:000f8300       ??0?$DynArray@HHU?$SmallDynStorage@HHUStandardAlloc@NAlloc@@@NArray@@@@QEAA@AEBU0@@Z 00000000315f9300 f i ParamLoader.obj
 0001:000f83c0       ??0?$DynArray@UIdxAndName@@HU?$SmallDynStorage@UIdxAndName@@HUStandardAlloc@NAlloc@@@NArray@@@@QEAA@AEBU0@@Z 00000000315f93c0 f i ParamLoader.obj
 0001:000f8480       ??0?$DynArray@USAnimFile@@HU?$SmallDynStorage@USAnimFile@@HUStandardAlloc@NAlloc@@@NArray@@@@QEAA@AEBU0@@Z 00000000315f9480 f i ParamLoader.obj
 0001:000f8570       ??$move_init@UDirectionalBlends@@@NArray@@YAXPEAUDirectionalBlends@@0_K@Z 00000000315f9570 f i ParamLoader.obj
 0001:000f8670       ??$__uninitialized_fill_n@PEAUFacialAnimationEntry@CAnimationSet@@_KU12@@priv@stlpmtx_std@@YAPEAUFacialAnimationEntry@CAnimationSet@@PEAU23@_KAEBU23@@Z 00000000315f9670 f i ParamLoader.obj
 0001:000f86f0       ?destroy@?$DynArray@UDirectionalBlends@@HU?$SmallDynStorage@UDirectionalBlends@@HUStandardAlloc@NAlloc@@@NArray@@@@IEAAXXZ 00000000315f96f0 f i ParamLoader.obj
 0001:000f8770       ?BuildDependencyList@CParamLoader@@AEAA_NHAEAU?$DynArray@IHU?$SmallDynStorage@IHUStandardAlloc@NAlloc@@@NArray@@@@@Z 00000000315f9770 f   ParamLoader.obj
 0001:000f8880       ?LoadIKDefAnimDrivenIKTargets@CParamLoader@@AEAA_NVXmlNodeRef@@@Z 00000000315f9880 f   ParamLoader.obj
 0001:000f8b40       ?LoadIKDefRecoil@CParamLoader@@AEAA_NVXmlNodeRef@@@Z 00000000315f9b40 f   ParamLoader.obj
 0001:000f8fe0       ?resize@?$DynArray@UIdxAndName@@HU?$SmallDynStorage@UIdxAndName@@HUStandardAlloc@NAlloc@@@NArray@@@@QEAAXH@Z 00000000315f9fe0 f i ParamLoader.obj
 0001:000f9050       ?resize_raw@?$SmallDynStorage@UDirectionalBlends@@HUStandardAlloc@NAlloc@@@NArray@@QEAAXHH_N@Z 00000000315fa050 f i ParamLoader.obj
 0001:000f91d0       ?init@?$DynArray@U?$DynArray@IHU?$SmallDynStorage@IHUStandardAlloc@NAlloc@@@NArray@@@@HU?$SmallDynStorage@U?$DynArray@IHU?$SmallDynStorage@IHUStandardAlloc@NAlloc@@@NArray@@@@HUStandardAlloc@NAlloc@@@NArray@@@@KAPEAU?$DynArray@IHU?$SmallDynStorage@IHUStandardAlloc@NAlloc@@@NArray@@@@U?$Array@U?$DynArray@IHU?$SmallDynStorage@IHUStandardAlloc@NAlloc@@@NArray@@@@HU?$ArrayStorage@U?$DynArray@IHU?$SmallDynStorage@IHUStandardAlloc@NAlloc@@@NArray@@@@H@NArray@@@@@Z 00000000315fa1d0 f i ParamLoader.obj
 0001:000f92f0       ??0?$_Impl_vector@UFacialAnimationEntry@CAnimationSet@@V?$allocator@UFacialAnimationEntry@CAnimationSet@@@stlpmtx_std@@@priv@stlpmtx_std@@QEAA@AEBV012@@Z 00000000315fa2f0 f i ParamLoader.obj
 0001:000f93e0       ??0IKLimbType@@QEAA@XZ     00000000315fa3e0 f i ParamLoader.obj
 0001:000f94f0       ?PrepareHeaderList@SAnimListInfo@@QEAAXXZ 00000000315fa4f0 f i ParamLoader.obj
 0001:000f9570       ?AddIfNewAnimationAlias@CParamLoader@@AEAA_NAEAUSAnimListInfo@@PEBD1@Z 00000000315fa570 f   ParamLoader.obj
 0001:000f9790       ?clear@?$DynArray@UDirectionalBlends@@HU?$SmallDynStorage@UDirectionalBlends@@HUStandardAlloc@NAlloc@@@NArray@@@@QEAAXXZ 00000000315fa790 f i ParamLoader.obj
 0001:000f9870       ?init@?$DynArray@UIKLimbType@@HU?$SmallDynStorage@UIKLimbType@@HUStandardAlloc@NAlloc@@@NArray@@@@KAPEAUIKLimbType@@U?$Array@UIKLimbType@@HU?$ArrayStorage@UIKLimbType@@H@NArray@@@@AEBU2@@Z 00000000315fa870 f i ParamLoader.obj
 0001:000f9920       ??0?$DynArray@UModelAnimationHeader@@HU?$SmallDynStorage@UModelAnimationHeader@@HUStandardAlloc@NAlloc@@@NArray@@@@QEAA@AEBU0@@Z 00000000315fa920 f i ParamLoader.obj
 0001:000f9a10       ??$move_init@UIKLimbType@@@NArray@@YAXPEAUIKLimbType@@0_K@Z 00000000315faa10 f i ParamLoader.obj
 0001:000f9ad0       ??$move_init@U?$DynArray@IHU?$SmallDynStorage@IHUStandardAlloc@NAlloc@@@NArray@@@@@NArray@@YAXPEAU?$DynArray@IHU?$SmallDynStorage@IHUStandardAlloc@NAlloc@@@NArray@@@@0_K@Z 00000000315faad0 f i ParamLoader.obj
 0001:000f9bd0       ?ExpandWildcardsForPath@CParamLoader@@AEAAXAEAUSAnimListInfo@@PEBDI11@Z 00000000315fabd0 f   ParamLoader.obj
 0001:000fa1c0       ?resize_raw@?$SmallDynStorage@UIKLimbType@@HUStandardAlloc@NAlloc@@@NArray@@QEAAXHH_N@Z 00000000315fb1c0 f i ParamLoader.obj
 0001:000fa350       ??0?$DynArray@V?$CryStringT@D@@HU?$SmallDynStorage@V?$CryStringT@D@@HUStandardAlloc@NAlloc@@@NArray@@@@QEAA@AEBU0@@Z 00000000315fb350 f i ParamLoader.obj
 0001:000fa420       ?expand_raw@?$DynArray@UIKLimbType@@HU?$SmallDynStorage@UIKLimbType@@HUStandardAlloc@NAlloc@@@NArray@@@@IEAAPEAUIKLimbType@@PEAU2@H@Z 00000000315fb420 f i ParamLoader.obj
 0001:000fa4e0       ?resize_raw@?$SmallDynStorage@U?$DynArray@IHU?$SmallDynStorage@IHUStandardAlloc@NAlloc@@@NArray@@@@HUStandardAlloc@NAlloc@@@NArray@@QEAAXHH_N@Z 00000000315fb4e0 f i ParamLoader.obj
 0001:000fa650       ?_M_insert_overflow_aux@?$_Impl_vector@UFacialAnimationEntry@CAnimationSet@@V?$allocator@UFacialAnimationEntry@CAnimationSet@@@stlpmtx_std@@@priv@stlpmtx_std@@AEAAXPEAUFacialAnimationEntry@CAnimationSet@@AEBU45@AEBU__false_type@3@_K_N@Z 00000000315fb650 f i ParamLoader.obj
 0001:000fa8a0       ??1SAnimListInfo@@QEAA@XZ  00000000315fb8a0 f i ParamLoader.obj
 0001:000faa80       ?clear@?$DynArray@UIKLimbType@@HU?$SmallDynStorage@UIKLimbType@@HUStandardAlloc@NAlloc@@@NArray@@@@QEAAXXZ 00000000315fba80 f i ParamLoader.obj
 0001:000fab20       ??0SAnimListInfo@@QEAA@AEBU0@@Z 00000000315fbb20 f i ParamLoader.obj
 0001:000fac10       ??0SAnimListInfo@@QEAA@PEBD@Z 00000000315fbc10 f i ParamLoader.obj
 0001:000fb010       ?AddIfNewModelTracksDatabase@CParamLoader@@AEAA_NAEAUSAnimListInfo@@PEBD@Z 00000000315fc010 f   ParamLoader.obj
 0001:000fb280       ?LoadIKDefLookIK@CParamLoader@@AEAA_NVXmlNodeRef@@@Z 00000000315fc280 f   ParamLoader.obj
 0001:000fbe60       ?LoadIKDefAimIK@CParamLoader@@AEAA_NVXmlNodeRef@@@Z 00000000315fce60 f   ParamLoader.obj
 0001:000fcbe0       ?init@?$DynArray@USAnimListInfo@@HU?$SmallDynStorage@USAnimListInfo@@HUStandardAlloc@NAlloc@@@NArray@@@@KAPEAUSAnimListInfo@@U?$Array@USAnimListInfo@@HU?$ArrayStorage@USAnimListInfo@@H@NArray@@@@AEBU2@@Z 00000000315fdbe0 f i ParamLoader.obj
 0001:000fcd20       ??$move_init@USAnimListInfo@@@NArray@@YAXPEAUSAnimListInfo@@0_K@Z 00000000315fdd20 f i ParamLoader.obj
 0001:000fcd90       ?ScanDirectoryFiles@SDirectoryEnumeratorHelper@@AEAAXAEBV?$CryStringT@D@@00AEAV?$vector@V?$CryStringT@D@@V?$allocator@V?$CryStringT@D@@@stlpmtx_std@@@stlpmtx_std@@@Z 00000000315fdd90 f i ParamLoader.obj
 0001:000fd4c0       ?resize_raw@?$SmallDynStorage@USAnimListInfo@@HUStandardAlloc@NAlloc@@@NArray@@QEAAXHH_N@Z 00000000315fe4c0 f i ParamLoader.obj
 0001:000fd650       ?expand_raw@?$DynArray@USAnimListInfo@@HU?$SmallDynStorage@USAnimListInfo@@HUStandardAlloc@NAlloc@@@NArray@@@@IEAAPEAUSAnimListInfo@@PEAU2@H@Z 00000000315fe650 f i ParamLoader.obj
 0001:000fd710       ?ScanDirectoryRecursive@SDirectoryEnumeratorHelper@@QEAAXAEBV?$CryStringT@D@@00AEAV?$vector@V?$CryStringT@D@@V?$allocator@V?$CryStringT@D@@@stlpmtx_std@@@stlpmtx_std@@@Z 00000000315fe710 f i ParamLoader.obj
 0001:000fde10       ?AddIfNewFacialAnimationAlias@CParamLoader@@AEAA_NAEAUSAnimListInfo@@PEBD1@Z 00000000315fee10 f   ParamLoader.obj
 0001:000fe090       ?LoadIKDefLimbIK@CParamLoader@@AEAA_NVXmlNodeRef@@@Z 00000000315ff090 f   ParamLoader.obj
 0001:000ff4a0       ??1?$DynArray@USAnimListInfo@@HU?$SmallDynStorage@USAnimListInfo@@HUStandardAlloc@NAlloc@@@NArray@@@@QEAA@XZ 00000000316004a0 f i ParamLoader.obj
 0001:000ff520       ??0CParamLoader@@QEAA@XZ   0000000031600520 f   ParamLoader.obj
 0001:000ff5e0       ?ExpandWildcards@CParamLoader@@QEAA_NI_N@Z 00000000316005e0 f   ParamLoader.obj
 0001:00102460       ?LoadLod@CParamLoader@@AEAA_NVXmlNodeRef@@@Z 0000000031603460 f   ParamLoader.obj
 0001:001029c0       ?ParseIKDef@CParamLoader@@AEAA_NVXmlNodeRef@@@Z 00000000316039c0 f   ParamLoader.obj
 0001:00102d40       ?LoadAnimList@CParamLoader@@AEAAHVXmlNodeRef@@PEBDV?$CryStringT@D@@AEA_N@Z 0000000031603d40 f   ParamLoader.obj
 0001:00104b30       ?LoadXML@CParamLoader@@QEAA_NPEAVCSkel@@V?$CryStringT@D@@QEBDAEAU?$DynArray@IHU?$SmallDynStorage@IHUStandardAlloc@NAlloc@@@NArray@@@@@Z 0000000031605b30 f   ParamLoader.obj
 0001:00104ee0       ?ClearLists@CParamLoader@@QEAAXXZ 0000000031605ee0 f   ParamLoader.obj
 0001:001055a0       ??1CParamLoader@@QEAA@XZ   00000000316065a0 f   ParamLoader.obj
 0001:001055f0       ?Release@CSkel@@UEAAXXZ    00000000316065f0 f   Model.obj
 0001:00105620       ??_GIFacialAnimSkeletonAnimationEntry@@UEAAPEAXI@Z 0000000031606620 f i FaceAnimSequence.obj
 0001:00105620       ??_GIFacialModel@@UEAAPEAXI@Z 0000000031606620 f i FacialModel.obj
 0001:00105620       ??_EIAnimEvents@@UEAAPEAXI@Z 0000000031606620 f i CharacterManager.obj
 0001:00105620       ??_GIAnimEventList@@UEAAPEAXI@Z 0000000031606620 f i AnimEventList.obj
 0001:00105620       ??_EICharacterModelSkeleton@@UEAAPEAXI@Z 0000000031606620 f i Model.obj
 0001:00105620       ??_GIAnimEvents@@UEAAPEAXI@Z 0000000031606620 f i CharacterManager.obj
 0001:00105620       ??_GICharacterModelSkeleton@@UEAAPEAXI@Z 0000000031606620 f i Model.obj
 0001:00105620       ??_EIFacialAnimSkeletonAnimationEntry@@UEAAPEAXI@Z 0000000031606620 f i FaceAnimSequence.obj
 0001:00105620       ??_EIAnimEventList@@UEAAPEAXI@Z 0000000031606620 f i AnimEventList.obj
 0001:00105620       ??_EIFacialModel@@UEAAPEAXI@Z 0000000031606620 f i FacialModel.obj
 0001:00105650       ??_GICharacterModel@@UEAAPEAXI@Z 0000000031606650 f i Model.obj
 0001:00105650       ??_EICharacterModel@@UEAAPEAXI@Z 0000000031606650 f i Model.obj
 0001:00105680       ?strnstr@CryStringUtils@@YAPEBDPEBD0H@Z 0000000031606680 f i Model.obj
 0001:00105720       ?GetMeshApproxFlags@@YAHPEBDH@Z 0000000031606720 f   Model.obj
 0001:001057f0       ?GetTextureMemoryUsage@CSkel@@UEBAIPEAVICrySizer@@@Z 00000000316067f0 f   Model.obj
 0001:001058a0       ?GetMeshMemoryUsage@CSkel@@UEBAIPEAVICrySizer@@@Z 00000000316068a0 f   Model.obj
 0001:001058f0       ?GetIRenderMesh@CSkel@@UEAAPEAUIRenderMesh@@H@Z 00000000316068f0 f   Model.obj
 0001:001058f0       ?GetIRenderMesh@CSkel@@UEBAPEBUIRenderMesh@@H@Z 00000000316068f0 f   Model.obj
 0001:00105910       ?GetNumLods@CSkel@@UEBAIXZ 0000000031606910 f   Model.obj
 0001:00105940       ?GetJointPhysGeom@CSkel@@UEBAPEBUphys_geometry@@IH@Z 0000000031606940 f   Model.obj
 0001:00105940       ?GetJointPhysGeom@CSkel@@UEAAPEAUphys_geometry@@IH@Z 0000000031606940 f   Model.obj
 0001:00105970       ?ParsePhysInfoProperties_ROPE@CSkel@@SA_NAEAUCryBonePhysics@@AEBU?$DynArray@USJointProperty@@HU?$SmallDynStorage@USJointProperty@@HUStandardAlloc@NAlloc@@@NArray@@@@@Z 0000000031606970 f   Model.obj
 0001:00105e80       ?resize_raw@?$SmallDynStorage@PEAVCCharInstance@@HUStandardAlloc@NAlloc@@@NArray@@QEAAXHH_N@Z 0000000031606e80 f i Model.obj
 0001:00106010       ?resize_raw@?$SmallDynStorage@USJointProperty@@HUStandardAlloc@NAlloc@@@NArray@@QEAAXHH_N@Z 0000000031607010 f i Model.obj
 0001:001061d0       ?set_size@?$SmallDynStorage@PEAVCCharInstance@@HUStandardAlloc@NAlloc@@@NArray@@QEAAXH@Z 00000000316071d0 f i Model.obj
 0001:001061d0       ?set_size@?$SmallDynStorage@PEAU?$DynArray@UCryTCBQKey@@HU?$SmallDynStorage@UCryTCBQKey@@HUStandardAlloc@NAlloc@@@NArray@@@@HUStandardAlloc@NAlloc@@@NArray@@QEAAXH@Z 00000000316071d0 f i LoaderTCB.obj
 0001:001061d0       ?set_size@?$SmallDynStorage@PEAVCAnimationSet@@HUStandardAlloc@NAlloc@@@NArray@@QEAAXH@Z 00000000316071d0 f i ModelAnimationSet.obj
 0001:001061d0       ?set_size@?$SmallDynStorage@V?$_smart_ptr@VIController@@@@HUStandardAlloc@NAlloc@@@NArray@@QEAAXH@Z 00000000316071d0 f i CharacterManager.obj
 0001:001061d0       ?set_size@?$SmallDynStorage@V?$_smart_ptr@UIAttachment@@@@HUStandardAlloc@NAlloc@@@NArray@@QEAAXH@Z 00000000316071d0 f i AttachmentManager.obj
 0001:001061d0       ?set_size@?$SmallDynStorage@UBoneIndices8@@HUStandardAlloc@NAlloc@@@NArray@@QEAAXH@Z 00000000316071d0 f i LoaderSKIN.obj
 0001:001061d0       ?set_size@?$SmallDynStorage@PEAVCAttachmentSKIN@@HUStandardAlloc@NAlloc@@@NArray@@QEAAXH@Z 00000000316071d0 f i ModelSkin.obj
 0001:001061d0       ?set_size@?$SmallDynStorage@V?$_smart_ptr@UCMorphTarget@@@@HUStandardAlloc@NAlloc@@@NArray@@QEAAXH@Z 00000000316071d0 f i LoaderSKIN.obj
 0001:001061d0       ?set_size@?$SmallDynStorage@V?$CryStringT@D@@HUStandardAlloc@NAlloc@@@NArray@@QEAAXH@Z 00000000316071d0 f i CharacterInstance.obj
 0001:001061d0       ?set_size@?$SmallDynStorage@U?$DynArray@IHU?$SmallDynStorage@IHUStandardAlloc@NAlloc@@@NArray@@@@HUStandardAlloc@NAlloc@@@NArray@@QEAAXH@Z 00000000316071d0 f i ParamLoader.obj
 0001:001061d0       ?set_size@?$SmallDynStorage@PEAU?$DynArray@UCryTCB3Key@@HU?$SmallDynStorage@UCryTCB3Key@@HUStandardAlloc@NAlloc@@@NArray@@@@HUStandardAlloc@NAlloc@@@NArray@@QEAAXH@Z 00000000316071d0 f i LoaderTCB.obj
 0001:00106270       ?CreateFacialInstance@CSkel@@QEAAXXZ 0000000031607270 f   Model.obj
 0001:001062c0       ?SetJointPhysProperties_ROPE@CSkel@@UEAA_NIHAEBU?$DynArray@USJointProperty@@HU?$SmallDynStorage@USJointProperty@@HUStandardAlloc@NAlloc@@@NArray@@@@@Z 00000000316072c0 f   Model.obj
 0001:001062f0       ?GetAttachmentTriangle@CSkel@@UEAA?AUClosestTri@@AEBU?$Vec3_tpl@M@@@Z 00000000316072f0 f   Model.obj
 0001:00106360       ?expand_raw@?$DynArray@USJointProperty@@HU?$SmallDynStorage@USJointProperty@@HUStandardAlloc@NAlloc@@@NArray@@@@IEAAPEAUSJointProperty@@PEAU2@H@Z 0000000031607360 f i Model.obj
 0001:00106420       ??$AddObject@HHU?$SmallDynStorage@HHUStandardAlloc@NAlloc@@@NArray@@@ICrySizer@@QEAAXAEBU?$DynArray@HHU?$SmallDynStorage@HHUStandardAlloc@NAlloc@@@NArray@@@@@Z 0000000031607420 f i ControllerPQLog.obj
 0001:00106420       ??$AddObject@IHU?$SmallDynStorage@IHUStandardAlloc@NAlloc@@@NArray@@@ICrySizer@@QEAAXAEBU?$DynArray@IHU?$SmallDynStorage@IHUStandardAlloc@NAlloc@@@NArray@@@@@Z 0000000031607420 f i Model.obj
 0001:00106420       ??$AddObject@MHU?$SmallDynStorage@MHUStandardAlloc@NAlloc@@@NArray@@@ICrySizer@@QEAAXAEBU?$DynArray@MHU?$SmallDynStorage@MHUStandardAlloc@NAlloc@@@NArray@@@@@Z 0000000031607420 f i CharacterInstance.obj
 0001:001064c0       ?SizeOfModelData@CSkel@@QEBAIXZ 00000000316074c0 f   Model.obj
 0001:00106770       ??$AddObject@U?$DynArray@IHU?$SmallDynStorage@IHUStandardAlloc@NAlloc@@@NArray@@@@HU?$SmallDynStorage@U?$DynArray@IHU?$SmallDynStorage@IHUStandardAlloc@NAlloc@@@NArray@@@@HUStandardAlloc@NAlloc@@@NArray@@@ICrySizer@@QEAAXAEBU?$DynArray@U?$DynArray@IHU?$SmallDynStorage@IHUStandardAlloc@NAlloc@@@NArray@@@@HU?$SmallDynStorage@U?$DynArray@IHU?$SmallDynStorage@IHUStandardAlloc@NAlloc@@@NArray@@@@HUStandardAlloc@NAlloc@@@NArray@@@@@Z 0000000031607770 f i Model.obj
 0001:001068c0       ?append_raw@?$DynArray@PEAVCCharInstance@@HU?$SmallDynStorage@PEAVCCharInstance@@HUStandardAlloc@NAlloc@@@NArray@@@@QEAA?AU?$Array@PEAVCCharInstance@@HU?$ArrayStorage@PEAVCCharInstance@@H@NArray@@@@H@Z 00000000316078c0 f i Model.obj
 0001:00106980       ?erase@?$DynArray@PEAVCAttachmentSKIN@@HU?$SmallDynStorage@PEAVCAttachmentSKIN@@HUStandardAlloc@NAlloc@@@NArray@@@@QEAAPEAPEAVCAttachmentSKIN@@PEAPEAV2@@Z 0000000031607980 f i ModelSkin.obj
 0001:00106980       ?erase@?$DynArray@PEAVCCharInstance@@HU?$SmallDynStorage@PEAVCCharInstance@@HUStandardAlloc@NAlloc@@@NArray@@@@QEAAPEAPEAVCCharInstance@@PEAPEAV2@@Z 0000000031607980 f i Model.obj
 0001:00106980       ?erase@?$DynArray@PEAVCAnimationSet@@HU?$SmallDynStorage@PEAVCAnimationSet@@HUStandardAlloc@NAlloc@@@NArray@@@@QEAAPEAPEAVCAnimationSet@@PEAPEAV2@@Z 0000000031607980 f i ModelAnimationSet.obj
 0001:001069f0       ??1?$DynArray@VCModelJoint@@HU?$SmallDynStorage@VCModelJoint@@HUStandardAlloc@NAlloc@@@NArray@@@@QEAA@XZ 00000000316079f0 f i Model.obj
 0001:00106a70       ??0?$DynArray@USJointProperty@@HU?$SmallDynStorage@USJointProperty@@HUStandardAlloc@NAlloc@@@NArray@@@@QEAA@XZ 0000000031607a70 f i Model.obj
 0001:00106ad0       ??1RecoilDesc@@QEAA@XZ     0000000031607ad0 f i Model.obj
 0001:00106b70       ?UnregisterInstance@CSkel@@QEAAXPEAVCCharInstance@@@Z 0000000031607b70 f   Model.obj
 0001:00106bc0       ?UpdatePhysBonePrimitives@CSkel@@QEAAXAEBU?$DynArray@UBONE_ENTITY@@HU?$SmallDynStorage@UBONE_ENTITY@@HUStandardAlloc@NAlloc@@@NArray@@@@H@Z 0000000031607bc0 f   Model.obj
 0001:00107250       ?GetPhysInfoProperties_ROPE@CSkel@@SA?AU?$DynArray@USJointProperty@@HU?$SmallDynStorage@USJointProperty@@HUStandardAlloc@NAlloc@@@NArray@@@@AEBUCryBonePhysics@@H@Z 0000000031608250 f   Model.obj
 0001:00107e70       ?destroy@?$DynArray@U?$DynArray@IHU?$SmallDynStorage@IHUStandardAlloc@NAlloc@@@NArray@@@@HU?$SmallDynStorage@U?$DynArray@IHU?$SmallDynStorage@IHUStandardAlloc@NAlloc@@@NArray@@@@HUStandardAlloc@NAlloc@@@NArray@@@@KAXU?$Array@U?$DynArray@IHU?$SmallDynStorage@IHUStandardAlloc@NAlloc@@@NArray@@@@HU?$ArrayStorage@U?$DynArray@IHU?$SmallDynStorage@IHUStandardAlloc@NAlloc@@@NArray@@@@H@NArray@@@@@Z 0000000031608e70 f i Model.obj
 0001:00107f60       ??$push_back_unique@U?$DynArray@PEAVCCharInstance@@HU?$SmallDynStorage@PEAVCCharInstance@@HUStandardAlloc@NAlloc@@@NArray@@@@PEAVCCharInstance@@@stl@@YA_NAEAU?$DynArray@PEAVCCharInstance@@HU?$SmallDynStorage@PEAVCCharInstance@@HUStandardAlloc@NAlloc@@@NArray@@@@AEBQEAVCCharInstance@@@Z 0000000031608f60 f i Model.obj
 0001:00108000       ??$AddObject@UMeshCollisionInfo@@HU?$SmallDynStorage@UMeshCollisionInfo@@HUStandardAlloc@NAlloc@@@NArray@@@ICrySizer@@QEAAXAEBU?$DynArray@UMeshCollisionInfo@@HU?$SmallDynStorage@UMeshCollisionInfo@@HUStandardAlloc@NAlloc@@@NArray@@@@@Z 0000000031609000 f i Model.obj
 0001:00108160       ??0RecoilDesc@@QEAA@XZ     0000000031609160 f i Model.obj
 0001:001081d0       ?destroy@?$DynArray@UMeshCollisionInfo@@HU?$SmallDynStorage@UMeshCollisionInfo@@HUStandardAlloc@NAlloc@@@NArray@@@@KAXU?$Array@UMeshCollisionInfo@@HU?$ArrayStorage@UMeshCollisionInfo@@H@NArray@@@@@Z 00000000316091d0 f i Model.obj
 0001:001082c0       ?RegisterInstance@CSkel@@QEAAXPEAVCCharInstance@@@Z 00000000316092c0 f   Model.obj
 0001:00108340       ?GetJointPhysProperties_ROPE@CSkel@@UEBA?AU?$DynArray@USJointProperty@@HU?$SmallDynStorage@USJointProperty@@HUStandardAlloc@NAlloc@@@NArray@@@@IH@Z 0000000031609340 f   Model.obj
 0001:001085b0       ?GetMemoryUsage@CSkel@@QEBAXPEAVICrySizer@@@Z 00000000316095b0 f   Model.obj
 0001:001086f0       ??0PoseBlenderLookDesc@@QEAA@XZ 00000000316096f0 f i Model.obj
 0001:00108800       ??1PoseBlenderLookDesc@@QEAA@XZ 0000000031609800 f i Model.obj
 0001:00108900       ??0PoseBlenderAimDesc@@QEAA@XZ 0000000031609900 f i Model.obj
 0001:00108a50       ??1PoseBlenderAimDesc@@QEAA@XZ 0000000031609a50 f i Model.obj
 0001:00108b20       ??1?$DynArray@UIKLimbType@@HU?$SmallDynStorage@UIKLimbType@@HUStandardAlloc@NAlloc@@@NArray@@@@QEAA@XZ 0000000031609b20 f i Model.obj
 0001:00108ba0       ??0CModelSkeleton@@QEAA@XZ 0000000031609ba0 f i Model.obj
 0001:00108d50       ??_ECModelSkeleton@@W7EAAPEAXI@Z 0000000031609d50 f i Model.obj
 0001:00108d60       ?GetJointParentIDByID@CModelSkeleton@@UEBAHH@Z 0000000031609d60 f i Model.obj
 0001:00108d90       ?GetLimbDefinitionIdx@CModelSkeleton@@UEBAH_K@Z 0000000031609d90 f i Model.obj
 0001:00108dc0       ??1CModelSkeleton@@UEAA@XZ 0000000031609dc0 f i Model.obj
 0001:00108ee0       ??_ECModelSkeleton@@UEAAPEAXI@Z 0000000031609ee0 f i Model.obj
 0001:00108ee0       ??_GCModelSkeleton@@UEAAPEAXI@Z 0000000031609ee0 f i Model.obj
 0001:00108f10       ??0CSkel@@QEAA@AEBV?$CryStringT@D@@IPEBD@Z 0000000031609f10 f   Model.obj
 0001:00109280       ?AddRef@CSkel@@UEAAXXZ     000000003160a280 f i Model.obj
 0001:00109290       ?DecRef@CSkel@@UEAAXXZ     000000003160a290 f i Model.obj
 0001:001092a0       ?GetICharacterModelSkeleton@CSkel@@UEAAPEAUICharacterModelSkeleton@@XZ 000000003160a2a0 f i Model.obj
 0001:001092a0       ?GetICharacterModelSkeleton@CSkel@@UEBAPEBUICharacterModelSkeleton@@XZ 000000003160a2a0 f i Model.obj
 0001:001092b0       ?GetNumJoints@CSkel@@UEBAIXZ 000000003160a2b0 f i Model.obj
 0001:001092c0       ?GetICharInstanceFromModel@CSkel@@UEBAPEBUICharacterInstance@@I@Z 000000003160a2c0 f i Model.obj
 0001:001092c0       ?GetICharInstanceFromModel@CSkel@@UEAAPEAUICharacterInstance@@I@Z 000000003160a2c0 f i Model.obj
 0001:00109300       ?GetNumInstances@CSkel@@UEBAIXZ 000000003160a300 f i Model.obj
 0001:00109310       ??1CSkel@@UEAA@XZ          000000003160a310 f   Model.obj
 0001:001095a0       ??_GCSkel@@UEAAPEAXI@Z     000000003160a5a0 f i Model.obj
 0001:001095a0       ??_ECSkel@@UEAAPEAXI@Z     000000003160a5a0 f i Model.obj
 0001:001095d0       ?GetAnimationDCCWorldSpaceLocation@CAnimationSet@@UEBA_NPEBDAEAU?$QuatT_tpl@M@@@Z 000000003160a5d0 f   ModelAnimationSet.obj
 0001:00109610       ?GetAnimationEndLocation@CAnimationSet@@UEBA_NPEBDAEAU?$QuatT_tpl@M@@@Z 000000003160a610 f   ModelAnimationSet.obj
 0001:00109650       ??_EIAnimationSet@@UEAAPEAXI@Z 000000003160a650 f i ModelAnimationSet.obj
 0001:00109650       ??_GIAnimationSet@@UEAAPEAXI@Z 000000003160a650 f i ModelAnimationSet.obj
 0001:00109680       ?GetModelAnimationHeader@CAnimationSet@@QEBAPEBUModelAnimationHeader@@H@Z 000000003160a680 f   ModelAnimationSet.obj
 0001:00109840       ?GetNameByAnimID@CAnimationSet@@UEBAPEBDH@Z 000000003160a840 f   ModelAnimationSet.obj
 0001:001098d0       ?GetCRCByAnimID@CAnimationSet@@UEBAIH@Z 000000003160a8d0 f   ModelAnimationSet.obj
 0001:00109900       ?GetFilePathCRCByAnimID@CAnimationSet@@UEBAIH@Z 000000003160a900 f   ModelAnimationSet.obj
 0001:00109990       ?IsAnimLoaded@CAnimationSet@@UEBA_NH@Z 000000003160a990 f   ModelAnimationSet.obj
 0001:00109b10       ?GetGAH_CAF@CAnimationSet@@QEBAPEAUGlobalAnimationHeaderCAF@@H@Z 000000003160ab10 f   ModelAnimationSet.obj
 0001:00109bb0       ?GetGAH_LMG@CAnimationSet@@QEAAPEAUGlobalAnimationHeaderLMG@@H@Z 000000003160abb0 f   ModelAnimationSet.obj
 0001:00109c50       ?GetDuration_sec@CAnimationSet@@UEBAMH@Z 000000003160ac50 f   ModelAnimationSet.obj
 0001:00109e40       ?GetAnimationFlags@CAnimationSet@@UEBAIH@Z 000000003160ae40 f   ModelAnimationSet.obj
 0001:00109f70       ?GetAnimationStatus@CAnimationSet@@UEBAPEBDH@Z 000000003160af70 f   ModelAnimationSet.obj
 0001:0010a040       ?GetStart@CAnimationSet@@UEAAMH@Z 000000003160b040 f   ModelAnimationSet.obj
 0001:0010a0f0       ?GetAnimationDCCWorldSpaceLocation@CAnimationSet@@UEBA_NHAEAU?$QuatT_tpl@M@@@Z 000000003160b0f0 f   ModelAnimationSet.obj
 0001:0010a210       ?GetFilePathByName@CAnimationSet@@UEBAPEBDPEBD@Z 000000003160b210 f   ModelAnimationSet.obj
 0001:0010a330       ?GetFilePathByID@CAnimationSet@@UEBAPEBDH@Z 000000003160b330 f   ModelAnimationSet.obj
 0001:0010a3d0       ?GetGlobalIDByName@CAnimationSet@@UEAAHPEBD@Z 000000003160b3d0 f   ModelAnimationSet.obj
 0001:0010a470       ?GetGlobalIDByAnimID@CAnimationSet@@UEAAHH@Z 000000003160b470 f   ModelAnimationSet.obj
 0001:0010a490       ?GetTotalPosKeys@CAnimationSet@@UEBAII@Z 000000003160b490 f   ModelAnimationSet.obj
 0001:0010a4d0       ?GetTotalRotKeys@CAnimationSet@@UEBAII@Z 000000003160b4d0 f   ModelAnimationSet.obj
 0001:0010a510       ?GetDBAFilePath@CAnimationSet@@UEBAPEBDI@Z 000000003160b510 f   ModelAnimationSet.obj
 0001:0010a540       ?VerifyLMGs@CAnimationSet@@QEAAXXZ 000000003160b540 f   ModelAnimationSet.obj
 0001:0010a690       ??$__lower_bound@PEAUFacialAnimationEntry@CAnimationSet@@PEBDU?$less_stricmp@PEBD@stl@@U34@_J@priv@stlpmtx_std@@YAPEAUFacialAnimationEntry@CAnimationSet@@PEAU23@0AEBQEBDU?$less_stricmp@PEBD@stl@@2PEA_J@Z 000000003160b690 f i ModelAnimationSet.obj
 0001:0010a740       ?resize_raw@?$SmallDynStorage@PEAVCAnimationSet@@HUStandardAlloc@NAlloc@@@NArray@@QEAAXHH_N@Z 000000003160b740 f i ModelAnimationSet.obj
 0001:0010a8d0       ?GetNumFacialAnimations@CAnimationSet@@UEAAHXZ 000000003160b8d0 f   ModelAnimationSet.obj
 0001:0010a8d0       ?GetEffectorCount@CFacialModel@@UEBAHXZ 000000003160b8d0 f   FacialModel.obj
 0001:0010a900       ?numMorphTargets@CAnimationSet@@UEBAIXZ 000000003160b900 f   ModelAnimationSet.obj
 0001:0010a930       ?GetNameMorphTarget@CAnimationSet@@UEAAPEBDH@Z 000000003160b930 f   ModelAnimationSet.obj
 0001:0010a9a0       ?GetJointStartLocation@CAnimationSet@@UEAA_NPEBDHAEAU?$QuatT_tpl@M@@@Z 000000003160b9a0 f   ModelAnimationSet.obj
 0001:0010aab0       ?GetAnimationDCCWorldSpaceLocation@CAnimationSet@@UEBA_NPEBVCAnimation@@AEAU?$QuatT_tpl@M@@@Z 000000003160bab0 f   ModelAnimationSet.obj
 0001:0010b2c0       ?GetClosestQuatInChannel@CAnimationSet@@UEAAMPEBDHAEBU?$Quat_tpl@M@@@Z 000000003160c2c0 f   ModelAnimationSet.obj
 0001:0010b580       ?ExportCAF2HTR@CAnimationSet@@UEAA_NPEBD0PEBUISkeletonAnim@@@Z 000000003160c580 f   ModelAnimationSet.obj
 0001:0010b690       ?ExportVGrid@CAnimationSet@@UEAA_NPEBD0PEBUISkeletonAnim@@@Z 000000003160c690 f   ModelAnimationSet.obj
 0001:0010b760       ?GetAnimationEndLocation@CAnimationSet@@UEBA_NHAEAU?$QuatT_tpl@M@@@Z 000000003160c760 f   ModelAnimationSet.obj
 0001:0010bc80       ??$AddObject@GHU?$SmallDynStorage@GHUStandardAlloc@NAlloc@@@NArray@@@ICrySizer@@QEAAXAEBU?$DynArray@GHU?$SmallDynStorage@GHUStandardAlloc@NAlloc@@@NArray@@@@@Z 000000003160cc80 f i ModelAnimationSet.obj
 0001:0010bc80       ??$AddObject@FHU?$SmallDynStorage@FHUStandardAlloc@NAlloc@@@NArray@@@ICrySizer@@QEAAXAEBU?$DynArray@FHU?$SmallDynStorage@FHUStandardAlloc@NAlloc@@@NArray@@@@@Z 000000003160cc80 f i Model.obj
 0001:0010bd20       ??$AddObject@IV?$CryStringT@D@@U?$less@I@stlpmtx_std@@V?$allocator@U?$pair@$$CBIV?$CryStringT@D@@@stlpmtx_std@@@3@@ICrySizer@@QEAAXAEBV?$map@IV?$CryStringT@D@@U?$less@I@stlpmtx_std@@V?$allocator@U?$pair@$$CBIV?$CryStringT@D@@@stlpmtx_std@@@3@@stlpmtx_std@@@Z 000000003160cd20 f i ModelAnimationSet.obj
 0001:0010bdf0       ?expand_raw@?$DynArray@PEAVCAnimationSet@@HU?$SmallDynStorage@PEAVCAnimationSet@@HUStandardAlloc@NAlloc@@@NArray@@@@IEAAPEAPEAVCAnimationSet@@PEAPEAV2@H@Z 000000003160cdf0 f i ModelAnimationSet.obj
 0001:0010be90       ?GetFacialAnimationPathByName@CAnimationSet@@UEAAPEBDPEBD@Z 000000003160ce90 f   ModelAnimationSet.obj
 0001:0010bf20       ?GetFacialAnimationName@CAnimationSet@@UEAAPEBDH@Z 000000003160cf20 f   ModelAnimationSet.obj
 0001:0010bf70       ?GetFacialAnimationPath@CAnimationSet@@UEAAPEBDH@Z 000000003160cf70 f   ModelAnimationSet.obj
 0001:0010bfc0       ?PrepareToReuseAnimations@CAnimationSet@@QEAAX_K@Z 000000003160cfc0 f   ModelAnimationSet.obj
 0001:0010c090       ?SizeOfAnimationSet@CAnimationSet@@QEBA_KXZ 000000003160d090 f   ModelAnimationSet.obj
 0001:0010c330       ??$AddObject@UModelAnimationHeader@@HU?$SmallDynStorage@UModelAnimationHeader@@HUStandardAlloc@NAlloc@@@NArray@@@ICrySizer@@QEAAXAEBU?$DynArray@UModelAnimationHeader@@HU?$SmallDynStorage@UModelAnimationHeader@@HUStandardAlloc@NAlloc@@@NArray@@@@@Z 000000003160d330 f i ModelAnimationSet.obj
 0001:0010c490       ??$AddObject@UFacialAnimationEntry@CAnimationSet@@V?$allocator@UFacialAnimationEntry@CAnimationSet@@@stlpmtx_std@@@ICrySizer@@QEAAXAEBV?$vector@UFacialAnimationEntry@CAnimationSet@@V?$allocator@UFacialAnimationEntry@CAnimationSet@@@stlpmtx_std@@@stlpmtx_std@@@Z 000000003160d490 f i ModelAnimationSet.obj
 0001:0010c580       ?SizeOfLMG@GlobalAnimationHeaderLMG@@QEBA_KXZ 000000003160d580 f i ModelAnimationSet.obj
 0001:0010c8a0       ?GetValueCRC@CAnimationSet@@AEBA_KI@Z 000000003160d8a0 f i ModelAnimationSet.obj
 0001:0010c930       ?GetValue@CAnimationSet@@AEBA_KPEBD@Z 000000003160d930 f i ModelAnimationSet.obj
 0001:0010ca00       ?insert_raw@?$DynArray@IHU?$SmallDynStorage@IHUStandardAlloc@NAlloc@@@NArray@@@@QEAA?AU?$Array@IHU?$ArrayStorage@IH@NArray@@@@PEAIH@Z 000000003160da00 f i ModelAnimationSet.obj
 0001:0010cac0       ?insert_raw@?$DynArray@PEAVCAnimationSet@@HU?$SmallDynStorage@PEAVCAnimationSet@@HUStandardAlloc@NAlloc@@@NArray@@@@QEAA?AU?$Array@PEAVCAnimationSet@@HU?$ArrayStorage@PEAVCAnimationSet@@H@NArray@@@@PEAPEAVCAnimationSet@@H@Z 000000003160dac0 f i ModelAnimationSet.obj
 0001:0010cb80       ?GetAnimIDByName@CAnimationSet@@UEBAHPEBD@Z 000000003160db80 f   ModelAnimationSet.obj
 0001:0010cbd0       ?GetAnimIDByCRC@CAnimationSet@@UEBAHI@Z 000000003160dbd0 f   ModelAnimationSet.obj
 0001:0010cbe0       ?GetAnimationSize@CAnimationSet@@UEBAII@Z 000000003160dbe0 f   ModelAnimationSet.obj
 0001:0010cc40       ?_M_create_node@?$_Rb_tree@IU?$less@I@stlpmtx_std@@U?$pair@$$CBIV?$CryStringT@D@@@2@U?$_Select1st@U?$pair@$$CBIV?$CryStringT@D@@@stlpmtx_std@@@priv@2@U?$_MapTraitsT@U?$pair@$$CBIV?$CryStringT@D@@@stlpmtx_std@@@52@V?$allocator@U?$pair@$$CBIV?$CryStringT@D@@@stlpmtx_std@@@2@@priv@stlpmtx_std@@IEAAPEAU_Rb_tree_node_base@23@AEBU?$pair@$$CBIV?$CryStringT@D@@@3@@Z 000000003160dc40 f i ModelAnimationSet.obj
 0001:0010ccd0       ?clear@?$DynArray@UModelAnimationHeader@@HU?$SmallDynStorage@UModelAnimationHeader@@HUStandardAlloc@NAlloc@@@NArray@@@@QEAAXXZ 000000003160dcd0 f i ModelAnimationSet.obj
 0001:0010cdb0       ?_M_erase@?$_Rb_tree@IU?$less@I@stlpmtx_std@@U?$pair@$$CBIV?$CryStringT@D@@@2@U?$_Select1st@U?$pair@$$CBIV?$CryStringT@D@@@stlpmtx_std@@@priv@2@U?$_MapTraitsT@U?$pair@$$CBIV?$CryStringT@D@@@stlpmtx_std@@@52@V?$allocator@U?$pair@$$CBIV?$CryStringT@D@@@stlpmtx_std@@@2@@priv@stlpmtx_std@@AEAAXPEAU_Rb_tree_node_base@23@@Z 000000003160ddb0 f i ModelAnimationSet.obj
 0001:0010ce30       ?Register@CAnimationManager@@QEAAXPEAVCAnimationSet@@@Z 000000003160de30 f i ModelAnimationSet.obj
 0001:0010ced0       ?Unregister@CAnimationManager@@QEAAXPEAVCAnimationSet@@@Z 000000003160ded0 f i ModelAnimationSet.obj
 0001:0010cf50       ?InsertHash@CAnimationSet@@AEAAXI_K@Z 000000003160df50 f i ModelAnimationSet.obj
 0001:0010d0a0       ?_M_insert@?$_Rb_tree@IU?$less@I@stlpmtx_std@@U?$pair@$$CBIV?$CryStringT@D@@@2@U?$_Select1st@U?$pair@$$CBIV?$CryStringT@D@@@stlpmtx_std@@@priv@2@U?$_MapTraitsT@U?$pair@$$CBIV?$CryStringT@D@@@stlpmtx_std@@@52@V?$allocator@U?$pair@$$CBIV?$CryStringT@D@@@stlpmtx_std@@@2@@priv@stlpmtx_std@@AEAA?AU?$_Rb_tree_iterator@U?$pair@$$CBIV?$CryStringT@D@@@stlpmtx_std@@U?$_MapTraitsT@U?$pair@$$CBIV?$CryStringT@D@@@stlpmtx_std@@@priv@2@@23@PEAU_Rb_tree_node_base@23@AEBU?$pair@$$CBIV?$CryStringT@D@@@3@00@Z 000000003160e0a0 f i ModelAnimationSet.obj
 0001:0010d160       ?insert_unique@?$_Rb_tree@IU?$less@I@stlpmtx_std@@U?$pair@$$CBIV?$CryStringT@D@@@2@U?$_Select1st@U?$pair@$$CBIV?$CryStringT@D@@@stlpmtx_std@@@priv@2@U?$_MapTraitsT@U?$pair@$$CBIV?$CryStringT@D@@@stlpmtx_std@@@52@V?$allocator@U?$pair@$$CBIV?$CryStringT@D@@@stlpmtx_std@@@2@@priv@stlpmtx_std@@QEAA?AU?$pair@U?$_Rb_tree_iterator@U?$pair@$$CBIV?$CryStringT@D@@@stlpmtx_std@@U?$_MapTraitsT@U?$pair@$$CBIV?$CryStringT@D@@@stlpmtx_std@@@priv@2@@priv@stlpmtx_std@@_N@3@AEBU?$pair@$$CBIV?$CryStringT@D@@@3@@Z 000000003160e160 f i ModelAnimationSet.obj
 0001:0010d360       ?Init@CAnimationSet@@QEAAXXZ 000000003160e360 f   ModelAnimationSet.obj
 0001:0010d380       ?prepareLoadCAFs@CAnimationSet@@QEAAXI@Z 000000003160e380 f   ModelAnimationSet.obj
 0001:0010d400       ?prepareLoadANMs@CAnimationSet@@QEAAXI@Z 000000003160e400 f   ModelAnimationSet.obj
 0001:0010d460       ?GetMemoryUsage@CAnimationSet@@QEBAXPEAVICrySizer@@@Z 000000003160e460 f   ModelAnimationSet.obj
 0001:0010d4c0       ?insert_unique@?$_Rb_tree@IU?$less@I@stlpmtx_std@@U?$pair@$$CBIV?$CryStringT@D@@@2@U?$_Select1st@U?$pair@$$CBIV?$CryStringT@D@@@stlpmtx_std@@@priv@2@U?$_MapTraitsT@U?$pair@$$CBIV?$CryStringT@D@@@stlpmtx_std@@@52@V?$allocator@U?$pair@$$CBIV?$CryStringT@D@@@stlpmtx_std@@@2@@priv@stlpmtx_std@@QEAA?AU?$_Rb_tree_iterator@U?$pair@$$CBIV?$CryStringT@D@@@stlpmtx_std@@U?$_MapTraitsT@U?$pair@$$CBIV?$CryStringT@D@@@stlpmtx_std@@@priv@2@@23@U423@AEBU?$pair@$$CBIV?$CryStringT@D@@@3@@Z 000000003160e4c0 f i ModelAnimationSet.obj
 0001:0010d900       ?ReuseAnimation@CAnimationSet@@QEAAXAEBUModelAnimationHeader@@@Z 000000003160e900 f   ModelAnimationSet.obj
 0001:0010d960       ?ReleaseAnimationData@CAnimationSet@@QEAAXXZ 000000003160e960 f   ModelAnimationSet.obj
 0001:0010dd40       ??$?AI@?$map@IV?$CryStringT@D@@U?$less@I@stlpmtx_std@@V?$allocator@U?$pair@$$CBIV?$CryStringT@D@@@stlpmtx_std@@@3@@stlpmtx_std@@QEAAAEAV?$CryStringT@D@@AEBI@Z 000000003160ed40 f i ModelAnimationSet.obj
 0001:0010de60       ??1CAnimationSet@@UEAA@XZ  000000003160ee60 f   ModelAnimationSet.obj
 0001:0010dfb0       ??0CAnimationSet@@QEAA@XZ  000000003160efb0 f   ModelAnimationSet.obj
 0001:0010e130       ??_ECAnimationSet@@UEAAPEAXI@Z 000000003160f130 f i ModelAnimationSet.obj
 0001:0010e130       ??_GCAnimationSet@@UEAAPEAXI@Z 000000003160f130 f i ModelAnimationSet.obj
 0001:0010e160       ?LoadFileCAF@CAnimationSet@@QEAAHPEBD0@Z 000000003160f160 f   ModelAnimationSet.obj
 0001:0010e4c0       ?LoadFileAIM@CAnimationSet@@QEAAHPEBD0@Z 000000003160f4c0 f   ModelAnimationSet.obj
 0001:0010e8f0       ?LoadFileANM@CAnimationSet@@QEAAHPEBD0AEAU?$DynArray@UCControllerTCB@@HU?$SmallDynStorage@UCControllerTCB@@HUStandardAlloc@NAlloc@@@NArray@@@@PEAVCryCGALoader@@@Z 000000003160f8f0 f   ModelAnimationSet.obj
 0001:0010ec10       ?LoadFileLMG@CAnimationSet@@QEAAHPEBD0@Z 000000003160fc10 f   ModelAnimationSet.obj
 0001:0010ef90       ?AddAnimationByPath@CAnimationSet@@UEAAHPEBD0@Z 000000003160ff90 f   ModelAnimationSet.obj
 0001:0010f0d0       ?TriExtent@@YAMW4EGeomForm@@AEBU?$Vec3_tpl@M@@11@Z 00000000316100d0 f i ModelMesh.obj
 0001:0010f300       ?GetAttachmentTriangle@CModelMesh@@QEAA?AUClosestTri@@PEAUIRenderMesh@@AEBU?$Vec3_tpl@M@@@Z 0000000031610300 f   ModelMesh.obj
 0001:0010f780       ??$AddObject@UBoneIndices8@@HU?$SmallDynStorage@UBoneIndices8@@HUStandardAlloc@NAlloc@@@NArray@@@ICrySizer@@QEAAXAEBU?$DynArray@UBoneIndices8@@HU?$SmallDynStorage@UBoneIndices8@@HUStandardAlloc@NAlloc@@@NArray@@@@@Z 0000000031610780 f i ModelMesh.obj
 0001:0010f820       ??$AddObject@UBoneWeights8@@HU?$SmallDynStorage@UBoneWeights8@@HUStandardAlloc@NAlloc@@@NArray@@@ICrySizer@@QEAAXAEBU?$DynArray@UBoneWeights8@@HU?$SmallDynStorage@UBoneWeights8@@HUStandardAlloc@NAlloc@@@NArray@@@@@Z 0000000031610820 f i ModelMesh.obj
 0001:0010f820       ??$AddObject@USPostProcess@@HU?$SmallDynStorage@USPostProcess@@HUStandardAlloc@NAlloc@@@NArray@@@ICrySizer@@QEAAXAEBU?$DynArray@USPostProcess@@HU?$SmallDynStorage@USPostProcess@@HUStandardAlloc@NAlloc@@@NArray@@@@@Z 0000000031610820 f i SkeletonPose_Debug.obj
 0001:0010f890       ??$AddObject@U?$Quat_tpl@M@@HU?$SmallDynStorage@U?$Quat_tpl@M@@HUStandardAlloc@NAlloc@@@NArray@@@ICrySizer@@QEAAXAEBU?$DynArray@U?$Quat_tpl@M@@HU?$SmallDynStorage@U?$Quat_tpl@M@@HUStandardAlloc@NAlloc@@@NArray@@@@@Z 0000000031610890 f i ModelMesh.obj
 0001:0010f900       ?get_alloc_size@?$SmallDynStorage@UMorphTargetVertex@@HUStandardAlloc@NAlloc@@@NArray@@QEBAHXZ 0000000031610900 f i ModelMesh.obj
 0001:0010f960       ?SizeOfModelMesh@CModelMesh@@QEBA_KXZ 0000000031610960 f   ModelMesh.obj
 0001:0010fd00       ?ComputeExtent@CModelMesh@@QEAAMAEAUGeomQuery@@W4EGeomForm@@PEAUIRenderMesh@@@Z 0000000031610d00 f   ModelMesh.obj
 0001:0010ffa0       ?InitSWSkinBuffer@CModelMesh@@QEAAIPEAUIRenderMesh@@@Z 0000000031610fa0 f   ModelMesh.obj
 0001:00110a60       ??$AddObject@URChunk@@HU?$SmallDynStorage@URChunk@@HUStandardAlloc@NAlloc@@@NArray@@@ICrySizer@@QEAAXAEBU?$DynArray@URChunk@@HU?$SmallDynStorage@URChunk@@HUStandardAlloc@NAlloc@@@NArray@@@@@Z 0000000031611a60 f i ModelMesh.obj
 0001:00110c40       ??$AddObject@V?$_smart_ptr@UCMorphTarget@@@@HU?$SmallDynStorage@V?$_smart_ptr@UCMorphTarget@@@@HUStandardAlloc@NAlloc@@@NArray@@@ICrySizer@@QEAAXAEBU?$DynArray@V?$_smart_ptr@UCMorphTarget@@@@HU?$SmallDynStorage@V?$_smart_ptr@UCMorphTarget@@@@HUStandardAlloc@NAlloc@@@NArray@@@@@Z 0000000031611c40 f i ModelMesh.obj
 0001:00110dc0       ?GetMemoryUsage@CModelMesh@@QEBAXPEAVICrySizer@@@Z 0000000031611dc0 f   ModelMesh.obj
 0001:00110e50       ?PostInitialize@CModelJoint@@QEAAXAEBVCPoseData@Skeleton@@@Z 0000000031611e50 f   ModelSkeleton.obj
 0001:001110e0       ?SetIKJointID@CModelSkeleton@@QEAAXXZ 00000000316120e0 f   ModelSkeleton.obj
 0001:00111240       ?GetJointIDByCRC32@CModelSkeleton@@UEBAHI@Z 0000000031612240 f   ModelSkeleton.obj
 0001:001112a0       ?GetJointNameByID@CModelSkeleton@@UEBAPEBDH@Z 00000000316122a0 f   ModelSkeleton.obj
 0001:001112d0       ?SizeOfEmptyPhysics@CModelSkeleton@@QEBAIXZ 00000000316122d0 f   ModelSkeleton.obj
 0001:00111310       ??1CModelJoint@@QEAA@XZ    0000000031612310 f   ModelSkeleton.obj
 0001:00111410       ?GetJointIDByName@CModelSkeleton@@UEBAHPEBD@Z 0000000031612410 f   ModelSkeleton.obj
 0001:001114a0       ?get_alloc_size@?$SmallDynStorage@VCModelJoint@@HUStandardAlloc@NAlloc@@@NArray@@QEBAHXZ 00000000316124a0 f i ModelSkeleton.obj
 0001:00111500       ?get_alloc_size@?$SmallDynStorage@UCGlobalHeaderDBA@@HUStandardAlloc@NAlloc@@@NArray@@QEBAHXZ 0000000031612500 f i AnimationManager.obj
 0001:00111500       ?get_alloc_size@?$SmallDynStorage@UIKLimbType@@HUStandardAlloc@NAlloc@@@NArray@@QEBAHXZ 0000000031612500 f i ModelSkeleton.obj
 0001:00111500       ?get_alloc_size@?$SmallDynStorage@UEffectEntry@CSkeletonEffectManager@@HUStandardAlloc@NAlloc@@@NArray@@QEBAHXZ 0000000031612500 f i CharacterInstance.obj
 0001:00111560       ?_M_create_node@?$_Rb_tree@IU?$less@I@stlpmtx_std@@U?$pair@$$CBIPEAVCModelJoint@@@2@U?$_Select1st@U?$pair@$$CBIPEAVCModelJoint@@@stlpmtx_std@@@priv@2@U?$_MapTraitsT@U?$pair@$$CBIPEAVCModelJoint@@@stlpmtx_std@@@52@V?$allocator@U?$pair@$$CBIPEAVCModelJoint@@@stlpmtx_std@@@2@@priv@stlpmtx_std@@IEAAPEAU_Rb_tree_node_base@23@AEBU?$pair@$$CBIPEAVCModelJoint@@@3@@Z 0000000031612560 f i ModelSkeleton.obj
 0001:00111560       ?_M_create_node@?$_Rb_tree@IU?$less@I@stlpmtx_std@@U?$pair@$$CBIPEAV?$vector@HV?$allocator@H@stlpmtx_std@@@stlpmtx_std@@@2@U?$_Select1st@U?$pair@$$CBIPEAV?$vector@HV?$allocator@H@stlpmtx_std@@@stlpmtx_std@@@stlpmtx_std@@@priv@2@U?$_MapTraitsT@U?$pair@$$CBIPEAV?$vector@HV?$allocator@H@stlpmtx_std@@@stlpmtx_std@@@stlpmtx_std@@@52@V?$allocator@U?$pair@$$CBIPEAV?$vector@HV?$allocator@H@stlpmtx_std@@@stlpmtx_std@@@stlpmtx_std@@@2@@priv@stlpmtx_std@@IEAAPEAU_Rb_tree_node_base@23@AEBU?$pair@$$CBIPEAV?$vector@HV?$allocator@H@stlpmtx_std@@@stlpmtx_std@@@3@@Z 0000000031612560 f i AnimationManager.obj
 0001:00111560       ?_M_create_node@?$_Rb_tree@IU?$less@I@stlpmtx_std@@U?$pair@$$CBIPEAV?$vector@IV?$allocator@I@stlpmtx_std@@@stlpmtx_std@@@2@U?$_Select1st@U?$pair@$$CBIPEAV?$vector@IV?$allocator@I@stlpmtx_std@@@stlpmtx_std@@@stlpmtx_std@@@priv@2@U?$_MapTraitsT@U?$pair@$$CBIPEAV?$vector@IV?$allocator@I@stlpmtx_std@@@stlpmtx_std@@@stlpmtx_std@@@52@V?$allocator@U?$pair@$$CBIPEAV?$vector@IV?$allocator@I@stlpmtx_std@@@stlpmtx_std@@@stlpmtx_std@@@2@@priv@stlpmtx_std@@IEAAPEAU_Rb_tree_node_base@23@AEBU?$pair@$$CBIPEAV?$vector@IV?$allocator@I@stlpmtx_std@@@stlpmtx_std@@@3@@Z 0000000031612560 f i AnimationManager.obj
 0001:00111560       ?_M_create_node@?$_Rb_tree@IU?$less@I@stlpmtx_std@@U?$pair@$$CBI_K@2@U?$_Select1st@U?$pair@$$CBI_K@stlpmtx_std@@@priv@2@U?$_MapTraitsT@U?$pair@$$CBI_K@stlpmtx_std@@@52@V?$allocator@U?$pair@$$CBI_K@stlpmtx_std@@@2@@priv@stlpmtx_std@@IEAAPEAU_Rb_tree_node_base@23@AEBU?$pair@$$CBI_K@3@@Z 0000000031612560 f i CharacterManager.obj
 0001:001115d0       ?SizeOfSkeleton@CModelSkeleton@@QEBAIXZ 00000000316125d0 f   ModelSkeleton.obj
 0001:00111bd0       ?insert_unique@?$_Rb_tree@IU?$less@I@stlpmtx_std@@U?$pair@$$CBIPEAVCModelJoint@@@2@U?$_Select1st@U?$pair@$$CBIPEAVCModelJoint@@@stlpmtx_std@@@priv@2@U?$_MapTraitsT@U?$pair@$$CBIPEAVCModelJoint@@@stlpmtx_std@@@52@V?$allocator@U?$pair@$$CBIPEAVCModelJoint@@@stlpmtx_std@@@2@@priv@stlpmtx_std@@QEAA?AU?$pair@U?$_Rb_tree_iterator@U?$pair@$$CBIPEAVCModelJoint@@@stlpmtx_std@@U?$_MapTraitsT@U?$pair@$$CBIPEAVCModelJoint@@@stlpmtx_std@@@priv@2@@priv@stlpmtx_std@@_N@3@AEBU?$pair@$$CBIPEAVCModelJoint@@@3@@Z 0000000031612bd0 f i ModelSkeleton.obj
 0001:00111bd0       ?insert_unique@?$_Rb_tree@IU?$less@I@stlpmtx_std@@U?$pair@$$CBIPEAV?$vector@IV?$allocator@I@stlpmtx_std@@@stlpmtx_std@@@2@U?$_Select1st@U?$pair@$$CBIPEAV?$vector@IV?$allocator@I@stlpmtx_std@@@stlpmtx_std@@@stlpmtx_std@@@priv@2@U?$_MapTraitsT@U?$pair@$$CBIPEAV?$vector@IV?$allocator@I@stlpmtx_std@@@stlpmtx_std@@@stlpmtx_std@@@52@V?$allocator@U?$pair@$$CBIPEAV?$vector@IV?$allocator@I@stlpmtx_std@@@stlpmtx_std@@@stlpmtx_std@@@2@@priv@stlpmtx_std@@QEAA?AU?$pair@U?$_Rb_tree_iterator@U?$pair@$$CBIPEAV?$vector@IV?$allocator@I@stlpmtx_std@@@stlpmtx_std@@@stlpmtx_std@@U?$_MapTraitsT@U?$pair@$$CBIPEAV?$vector@IV?$allocator@I@stlpmtx_std@@@stlpmtx_std@@@stlpmtx_std@@@priv@2@@priv@stlpmtx_std@@_N@3@AEBU?$pair@$$CBIPEAV?$vector@IV?$allocator@I@stlpmtx_std@@@stlpmtx_std@@@3@@Z 0000000031612bd0 f i AnimationManager.obj
 0001:00111bd0       ?insert_unique@?$_Rb_tree@IU?$less@I@stlpmtx_std@@U?$pair@$$CBIPEAV?$vector@HV?$allocator@H@stlpmtx_std@@@stlpmtx_std@@@2@U?$_Select1st@U?$pair@$$CBIPEAV?$vector@HV?$allocator@H@stlpmtx_std@@@stlpmtx_std@@@stlpmtx_std@@@priv@2@U?$_MapTraitsT@U?$pair@$$CBIPEAV?$vector@HV?$allocator@H@stlpmtx_std@@@stlpmtx_std@@@stlpmtx_std@@@52@V?$allocator@U?$pair@$$CBIPEAV?$vector@HV?$allocator@H@stlpmtx_std@@@stlpmtx_std@@@stlpmtx_std@@@2@@priv@stlpmtx_std@@QEAA?AU?$pair@U?$_Rb_tree_iterator@U?$pair@$$CBIPEAV?$vector@HV?$allocator@H@stlpmtx_std@@@stlpmtx_std@@@stlpmtx_std@@U?$_MapTraitsT@U?$pair@$$CBIPEAV?$vector@HV?$allocator@H@stlpmtx_std@@@stlpmtx_std@@@stlpmtx_std@@@priv@2@@priv@stlpmtx_std@@_N@3@AEBU?$pair@$$CBIPEAV?$vector@HV?$allocator@H@stlpmtx_std@@@stlpmtx_std@@@3@@Z 0000000031612bd0 f i AnimationManager.obj
 0001:00111bd0       ?insert_unique@?$_Rb_tree@IU?$less@I@stlpmtx_std@@U?$pair@$$CBI_K@2@U?$_Select1st@U?$pair@$$CBI_K@stlpmtx_std@@@priv@2@U?$_MapTraitsT@U?$pair@$$CBI_K@stlpmtx_std@@@52@V?$allocator@U?$pair@$$CBI_K@stlpmtx_std@@@2@@priv@stlpmtx_std@@QEAA?AU?$pair@U?$_Rb_tree_iterator@U?$pair@$$CBI_K@stlpmtx_std@@U?$_MapTraitsT@U?$pair@$$CBI_K@stlpmtx_std@@@priv@2@@priv@stlpmtx_std@@_N@3@AEBU?$pair@$$CBI_K@3@@Z 0000000031612bd0 f i CharacterManager.obj
 0001:00111dd0       ??$AddObject@VCModelJoint@@HU?$SmallDynStorage@VCModelJoint@@HUStandardAlloc@NAlloc@@@NArray@@@ICrySizer@@QEAAXAEBU?$DynArray@VCModelJoint@@HU?$SmallDynStorage@VCModelJoint@@HUStandardAlloc@NAlloc@@@NArray@@@@@Z 0000000031612dd0 f i ModelSkeleton.obj
 0001:00111ea0       ?PostInitPhysGeom@CModelJoint@@QEAA_NAEAV?$map@_JPEAUphys_geometry@@U?$less@_J@stlpmtx_std@@V?$allocator@U?$pair@$$CB_JPEAUphys_geometry@@@stlpmtx_std@@@3@@stlpmtx_std@@H_N@Z 0000000031612ea0 f   ModelSkeleton.obj
 0001:00111fc0       ?AddHierarchyToControllerIdMap@CModelJoint@@QEAAXAEAV?$map@IPEAVCModelJoint@@U?$less@I@stlpmtx_std@@V?$allocator@U?$pair@$$CBIPEAVCModelJoint@@@stlpmtx_std@@@3@@stlpmtx_std@@@Z 0000000031612fc0 f   ModelSkeleton.obj
 0001:00112050       ??$AddObject@UIKLimbType@@HU?$SmallDynStorage@UIKLimbType@@HUStandardAlloc@NAlloc@@@NArray@@@ICrySizer@@QEAAXAEBU?$DynArray@UIKLimbType@@HU?$SmallDynStorage@UIKLimbType@@HUStandardAlloc@NAlloc@@@NArray@@@@@Z 0000000031613050 f i ModelSkeleton.obj
 0001:00112190       ?UpdateHierarchyPhysics@CModelJoint@@QEAAXAEBU?$DynArray@UBONE_ENTITY@@HU?$SmallDynStorage@UBONE_ENTITY@@HUStandardAlloc@NAlloc@@@NArray@@@@H@Z 0000000031613190 f   ModelSkeleton.obj
 0001:00112710       ?GetMemoryUsage@CModelSkeleton@@QEBAXPEAVICrySizer@@@Z 0000000031613710 f   ModelSkeleton.obj
 0001:00112cd0       ?GetAnimEventList@CAnimationManager@@UEAAPEAUIAnimEventList@@PEBD@Z 0000000031613cd0 f   AnimationManager.obj
 0001:00112ce0       ?DestroyRunTimePools@CAnimationManager@@QEAAXXZ 0000000031613ce0 f   AnimationManager.obj
 0001:00112d20       ?AnimationReleaseCAF@CAnimationManager@@QEAAXAEAUGlobalAnimationHeaderCAF@@@Z 0000000031613d20 f   AnimationManager.obj
 0001:00112d40       ?AnimationReleaseLMG@CAnimationManager@@QEAAXAEAUGlobalAnimationHeaderLMG@@@Z 0000000031613d40 f   AnimationManager.obj
 0001:00112d50       ?InitialiseRunTimePools@CAnimationManager@@QEAAXXZ 0000000031613d50 f   AnimationManager.obj
 0001:00112ea0       ?FindGlobalHeaderByCRC_DBA@CAnimationManager@@QEAAPEAUCGlobalHeaderDBA@@I@Z 0000000031613ea0 f   AnimationManager.obj
 0001:00112ef0       ?SaveAnimEventToXml@CAnimationManager@@UEAA_NAEBVCAnimEventData@@AEAVXmlNodeRef@@@Z 0000000031613ef0 f   AnimationManager.obj
 0001:00112ff0       ?Unload_All_Animation@CAnimationManager@@QEAA_NXZ 0000000031613ff0 f   AnimationManager.obj
 0001:001130d0       ?DBA_Unload_All@CAnimationManager@@QEAA_NXZ 00000000316140d0 f   AnimationManager.obj
 0001:00113230       ?IsDatabaseInMemory@CAnimationManager@@QEAA_NI@Z 0000000031614230 f   AnimationManager.obj
 0001:00113280       ?GetGlobalIDbyFilePath_AIM@CAnimationManager@@QEBAHPEBD@Z 0000000031614280 f   AnimationManager.obj
 0001:001132f0       ?GetGlobalIDbyFilePath_LMG@CAnimationManager@@QEBAHPEBD@Z 00000000316142f0 f   AnimationManager.obj
 0001:00113360       ?DBA_LockStatus@CAnimationManager@@QEAA_NPEBDI_N@Z 0000000031614360 f   AnimationManager.obj
 0001:00113550       ?DBA_Unload@CAnimationManager@@QEAA_NPEBD@Z 0000000031614550 f   AnimationManager.obj
 0001:001137f0       ?ReloadCAF@CAnimationManager@@QEAAHPEBD@Z 00000000316147f0 f   AnimationManager.obj
 0001:00113b90       ?ReloadLMG@CAnimationManager@@QEAAHPEBD@Z 0000000031614b90 f   AnimationManager.obj
 0001:00113ca0       ?GetDBACRC32fromFilePath@CAnimationManager@@QEAAIPEBD@Z 0000000031614ca0 f   AnimationManager.obj
 0001:00113d00       ?get_alloc_size@?$SmallDynStorage@UGlobalAnimationHeaderCAF@@HUStandardAlloc@NAlloc@@@NArray@@QEBAHXZ 0000000031614d00 f i AnimationManager.obj
 0001:00113d60       ?get_alloc_size@?$SmallDynStorage@UGlobalAnimationHeaderAIM@@HUStandardAlloc@NAlloc@@@NArray@@QEBAHXZ 0000000031614d60 f i AnimationManager.obj
 0001:00113dc0       ?get_alloc_size@?$SmallDynStorage@UGlobalAnimationHeaderLMG@@HUStandardAlloc@NAlloc@@@NArray@@QEBAHXZ 0000000031614dc0 f i AnimationManager.obj
 0001:00113e20       ?erase@?$DynArray@V?$_smart_ptr@UCMorphTarget@@@@HU?$SmallDynStorage@V?$_smart_ptr@UCMorphTarget@@@@HUStandardAlloc@NAlloc@@@NArray@@@@QEAAPEAV?$_smart_ptr@UCMorphTarget@@@@PEAV2@0@Z 0000000031614e20 f i LoaderSKIN.obj
 0001:00113e20       ?erase@?$DynArray@V?$_smart_ptr@VIController@@@@HU?$SmallDynStorage@V?$_smart_ptr@VIController@@@@HUStandardAlloc@NAlloc@@@NArray@@@@QEAAPEAV?$_smart_ptr@VIController@@@@PEAV2@0@Z 0000000031614e20 f i AnimationManager.obj
 0001:00113ec0       ?set_size@?$SmallDynStorage@UCGlobalHeaderDBA@@HUStandardAlloc@NAlloc@@@NArray@@QEAAXH@Z 0000000031614ec0 f i AnimationManager.obj
 0001:00113ec0       ?set_size@?$SmallDynStorage@UEffectEntry@CSkeletonEffectManager@@HUStandardAlloc@NAlloc@@@NArray@@QEAAXH@Z 0000000031614ec0 f i SkeletonEffectManager.obj
 0001:00113ec0       ?set_size@?$SmallDynStorage@UIKLimbType@@HUStandardAlloc@NAlloc@@@NArray@@QEAAXH@Z 0000000031614ec0 f i ParamLoader.obj
 0001:00113f70       ?set_size@?$SmallDynStorage@UGlobalAnimationHeaderLMG@@HUStandardAlloc@NAlloc@@@NArray@@QEAAXH@Z 0000000031614f70 f i AnimationManager.obj
 0001:00114030       ??$AddObject@UGlobalAnimationHeaderCAF@@HU?$SmallDynStorage@UGlobalAnimationHeaderCAF@@HUStandardAlloc@NAlloc@@@NArray@@@ICrySizer@@QEAAXAEBU?$DynArray@UGlobalAnimationHeaderCAF@@HU?$SmallDynStorage@UGlobalAnimationHeaderCAF@@HUStandardAlloc@NAlloc@@@NArray@@@@@Z 0000000031615030 f i AnimationManager.obj
 0001:001140f0       ?SetFilePathCAF@GlobalAnimationHeaderCAF@@QEAAXAEBV?$CryStringT@D@@@Z 00000000316150f0 f i CharacterManager.obj
 0001:001140f0       ?SetFilePath@GlobalAnimationHeaderAIM@@QEAAXAEBV?$CryStringT@D@@@Z 00000000316150f0 f i AnimationManager.obj
 0001:001141e0       ??$AddObject@I_KU?$less@I@stlpmtx_std@@V?$allocator@U?$pair@$$CBI_K@stlpmtx_std@@@2@@ICrySizer@@QEAAXAEBV?$map@I_KU?$less@I@stlpmtx_std@@V?$allocator@U?$pair@$$CBI_K@stlpmtx_std@@@2@@stlpmtx_std@@@Z 00000000316151e0 f i AnimationManager.obj
 0001:00114280       ??$AddObject@UBSParameter@@HU?$SmallDynStorage@UBSParameter@@HUStandardAlloc@NAlloc@@@NArray@@@ICrySizer@@QEAAXAEBU?$DynArray@UBSParameter@@HU?$SmallDynStorage@UBSParameter@@HUStandardAlloc@NAlloc@@@NArray@@@@@Z 0000000031615280 f i AnimationManager.obj
 0001:001143f0       ??$AddObject@V?$_smart_ptr@VIController@@@@HU?$SmallDynStorage@V?$_smart_ptr@VIController@@@@HUStandardAlloc@NAlloc@@@NArray@@@ICrySizer@@QEAAXAEBU?$DynArray@V?$_smart_ptr@VIController@@@@HU?$SmallDynStorage@V?$_smart_ptr@VIController@@@@HUStandardAlloc@NAlloc@@@NArray@@@@@Z 00000000316153f0 f i AnimationManager.obj
 0001:00114540       ?GetSubFoldersVector@AnimSearchHelper@@QEAAPEAV?$vector@IV?$allocator@I@stlpmtx_std@@@stlpmtx_std@@I@Z 0000000031615540 f   AnimationManager.obj
 0001:00114580       ?GetAnimationsVector@AnimSearchHelper@@QEAAPEAV?$vector@HV?$allocator@H@stlpmtx_std@@@stlpmtx_std@@I@Z 0000000031615580 f   AnimationManager.obj
 0001:001145c0       ??4?$DynArray@V?$_smart_ptr@VIController@@@@HU?$SmallDynStorage@V?$_smart_ptr@VIController@@@@HUStandardAlloc@NAlloc@@@NArray@@@@QEAAAEAU0@U?$Array@$$CBV?$_smart_ptr@VIController@@@@HU?$ArrayStorage@$$CBV?$_smart_ptr@VIController@@@@H@NArray@@@@@Z 00000000316155c0 f i AnimationManager.obj
 0001:00114730       ?assign@?$Array@VCAnimEventData@@HU?$SmallDynStorage@VCAnimEventData@@HUStandardAlloc@NAlloc@@@NArray@@@@QEAAXU?$Array@$$CBVCAnimEventData@@HU?$ArrayStorage@$$CBVCAnimEventData@@H@NArray@@@@@Z 0000000031615730 f i AnimationManager.obj
 0001:00114800       ?erase@?$DynArray@IHU?$SmallDynStorage@IHUStandardAlloc@NAlloc@@@NArray@@@@QEAAPEAIPEAI0@Z 0000000031615800 f i AnimationManager.obj
 0001:00114800       ?erase@?$DynArray@UCControllerType@@HU?$SmallDynStorage@UCControllerType@@HUStandardAlloc@NAlloc@@@NArray@@@@QEAAPEAUCControllerType@@PEAU2@0@Z 0000000031615800 f i LoaderCGA.obj
 0001:00114860       ??$AddObject@UCGlobalHeaderDBA@@HU?$SmallDynStorage@UCGlobalHeaderDBA@@HUStandardAlloc@NAlloc@@@NArray@@@ICrySizer@@QEAAXAEBU?$DynArray@UCGlobalHeaderDBA@@HU?$SmallDynStorage@UCGlobalHeaderDBA@@HUStandardAlloc@NAlloc@@@NArray@@@@@Z 0000000031615860 f i AnimationManager.obj
 0001:00114910       ?_M_insert@?$_Rb_tree@IU?$less@I@stlpmtx_std@@U?$pair@$$CBIPEAV?$vector@IV?$allocator@I@stlpmtx_std@@@stlpmtx_std@@@2@U?$_Select1st@U?$pair@$$CBIPEAV?$vector@IV?$allocator@I@stlpmtx_std@@@stlpmtx_std@@@stlpmtx_std@@@priv@2@U?$_MapTraitsT@U?$pair@$$CBIPEAV?$vector@IV?$allocator@I@stlpmtx_std@@@stlpmtx_std@@@stlpmtx_std@@@52@V?$allocator@U?$pair@$$CBIPEAV?$vector@IV?$allocator@I@stlpmtx_std@@@stlpmtx_std@@@stlpmtx_std@@@2@@priv@stlpmtx_std@@AEAA?AU?$_Rb_tree_iterator@U?$pair@$$CBIPEAV?$vector@IV?$allocator@I@stlpmtx_std@@@stlpmtx_std@@@stlpmtx_std@@U?$_MapTraitsT@U?$pair@$$CBIPEAV?$vector@IV?$allocator@I@stlpmtx_std@@@stlpmtx_std@@@stlpmtx_std@@@priv@2@@23@PEAU_Rb_tree_node_base@23@AEBU?$pair@$$CBIPEAV?$vector@IV?$allocator@I@stlpmtx_std@@@stlpmtx_std@@@3@00@Z 0000000031615910 f i AnimationManager.obj
 0001:00114910       ?_M_insert@?$_Rb_tree@IU?$less@I@stlpmtx_std@@U?$pair@$$CBIPEAV?$vector@HV?$allocator@H@stlpmtx_std@@@stlpmtx_std@@@2@U?$_Select1st@U?$pair@$$CBIPEAV?$vector@HV?$allocator@H@stlpmtx_std@@@stlpmtx_std@@@stlpmtx_std@@@priv@2@U?$_MapTraitsT@U?$pair@$$CBIPEAV?$vector@HV?$allocator@H@stlpmtx_std@@@stlpmtx_std@@@stlpmtx_std@@@52@V?$allocator@U?$pair@$$CBIPEAV?$vector@HV?$allocator@H@stlpmtx_std@@@stlpmtx_std@@@stlpmtx_std@@@2@@priv@stlpmtx_std@@AEAA?AU?$_Rb_tree_iterator@U?$pair@$$CBIPEAV?$vector@HV?$allocator@H@stlpmtx_std@@@stlpmtx_std@@@stlpmtx_std@@U?$_MapTraitsT@U?$pair@$$CBIPEAV?$vector@HV?$allocator@H@stlpmtx_std@@@stlpmtx_std@@@stlpmtx_std@@@priv@2@@23@PEAU_Rb_tree_node_base@23@AEBU?$pair@$$CBIPEAV?$vector@HV?$allocator@H@stlpmtx_std@@@stlpmtx_std@@@3@00@Z 0000000031615910 f i AnimationManager.obj
 0001:00114910       ?_M_insert@?$_Rb_tree@IU?$less@I@stlpmtx_std@@U?$pair@$$CBI_K@2@U?$_Select1st@U?$pair@$$CBI_K@stlpmtx_std@@@priv@2@U?$_MapTraitsT@U?$pair@$$CBI_K@stlpmtx_std@@@52@V?$allocator@U?$pair@$$CBI_K@stlpmtx_std@@@2@@priv@stlpmtx_std@@AEAA?AU?$_Rb_tree_iterator@U?$pair@$$CBI_K@stlpmtx_std@@U?$_MapTraitsT@U?$pair@$$CBI_K@stlpmtx_std@@@priv@2@@23@PEAU_Rb_tree_node_base@23@AEBU?$pair@$$CBI_K@3@00@Z 0000000031615910 f i CharacterManager.obj
 0001:001149d0       ?SetName@CAnimEventData@@QEAAXPEBD@Z 00000000316159d0 f i AnimationManager.obj
 0001:00114a40       ?GetValue@CNameCRCMap@@QEBA_KPEBD@Z 0000000031615a40 f i AnimationManager.obj
 0001:00114b50       ?SizeOfAIM@GlobalAnimationHeaderAIM@@QEBA_KXZ 0000000031615b50 f i AnimationManager.obj
 0001:00114d90       ?GetGlobalIDbyFilePath_CAF@CAnimationManager@@QEBAHPEBD@Z 0000000031615d90 f   AnimationManager.obj
 0001:00114dd0       ?GetAnimEventList@CAnimationManager@@UEBAPEBUIAnimEventList@@PEBD@Z 0000000031615dd0 f   AnimationManager.obj
 0001:00114e60       ?LoadAnimEventFromXml@CAnimationManager@@UEAA_NAEBVXmlNodeRef@@AEAVCAnimEventData@@@Z 0000000031615e60 f   AnimationManager.obj
 0001:001157c0       ?InitializeSegmentationDataFromAnimEvents@CAnimationManager@@UEAAXPEBD@Z 00000000316167c0 f   AnimationManager.obj
 0001:00115a40       ?UnloadAnimationCAF@CAnimationManager@@QEAAXAEAUGlobalAnimationHeaderCAF@@@Z 0000000031616a40 f   AnimationManager.obj
 0001:00115ac0       ?DebugAnimUsage@CAnimationManager@@QEAAXI@Z 0000000031616ac0 f   AnimationManager.obj
 0001:00116c90       ??4?$DynArray@IHU?$SmallDynStorage@IHUStandardAlloc@NAlloc@@@NArray@@@@QEAAAEAU0@U?$Array@$$CBIHU?$ArrayStorage@$$CBIH@NArray@@@@@Z 0000000031617c90 f i AnimationManager.obj
 0001:00116da0       ?insert_unique@?$_Rb_tree@IU?$less@I@stlpmtx_std@@U?$pair@$$CBIPEAV?$vector@HV?$allocator@H@stlpmtx_std@@@stlpmtx_std@@@2@U?$_Select1st@U?$pair@$$CBIPEAV?$vector@HV?$allocator@H@stlpmtx_std@@@stlpmtx_std@@@stlpmtx_std@@@priv@2@U?$_MapTraitsT@U?$pair@$$CBIPEAV?$vector@HV?$allocator@H@stlpmtx_std@@@stlpmtx_std@@@stlpmtx_std@@@52@V?$allocator@U?$pair@$$CBIPEAV?$vector@HV?$allocator@H@stlpmtx_std@@@stlpmtx_std@@@stlpmtx_std@@@2@@priv@stlpmtx_std@@QEAA?AU?$_Rb_tree_iterator@U?$pair@$$CBIPEAV?$vector@HV?$allocator@H@stlpmtx_std@@@stlpmtx_std@@@stlpmtx_std@@U?$_MapTraitsT@U?$pair@$$CBIPEAV?$vector@HV?$allocator@H@stlpmtx_std@@@stlpmtx_std@@@stlpmtx_std@@@priv@2@@23@U423@AEBU?$pair@$$CBIPEAV?$vector@HV?$allocator@H@stlpmtx_std@@@stlpmtx_std@@@3@@Z 0000000031617da0 f i AnimationManager.obj
 0001:00116da0       ?insert_unique@?$_Rb_tree@IU?$less@I@stlpmtx_std@@U?$pair@$$CBI_K@2@U?$_Select1st@U?$pair@$$CBI_K@stlpmtx_std@@@priv@2@U?$_MapTraitsT@U?$pair@$$CBI_K@stlpmtx_std@@@52@V?$allocator@U?$pair@$$CBI_K@stlpmtx_std@@@2@@priv@stlpmtx_std@@QEAA?AU?$_Rb_tree_iterator@U?$pair@$$CBI_K@stlpmtx_std@@U?$_MapTraitsT@U?$pair@$$CBI_K@stlpmtx_std@@@priv@2@@23@U423@AEBU?$pair@$$CBI_K@3@@Z 0000000031617da0 f i CharacterManager.obj
 0001:00116da0       ?insert_unique@?$_Rb_tree@IU?$less@I@stlpmtx_std@@U?$pair@$$CBIPEAV?$vector@IV?$allocator@I@stlpmtx_std@@@stlpmtx_std@@@2@U?$_Select1st@U?$pair@$$CBIPEAV?$vector@IV?$allocator@I@stlpmtx_std@@@stlpmtx_std@@@stlpmtx_std@@@priv@2@U?$_MapTraitsT@U?$pair@$$CBIPEAV?$vector@IV?$allocator@I@stlpmtx_std@@@stlpmtx_std@@@stlpmtx_std@@@52@V?$allocator@U?$pair@$$CBIPEAV?$vector@IV?$allocator@I@stlpmtx_std@@@stlpmtx_std@@@stlpmtx_std@@@2@@priv@stlpmtx_std@@QEAA?AU?$_Rb_tree_iterator@U?$pair@$$CBIPEAV?$vector@IV?$allocator@I@stlpmtx_std@@@stlpmtx_std@@@stlpmtx_std@@U?$_MapTraitsT@U?$pair@$$CBIPEAV?$vector@IV?$allocator@I@stlpmtx_std@@@stlpmtx_std@@@stlpmtx_std@@@priv@2@@23@U423@AEBU?$pair@$$CBIPEAV?$vector@IV?$allocator@I@stlpmtx_std@@@stlpmtx_std@@@3@@Z 0000000031617da0 f i AnimationManager.obj
 0001:001171e0       ??$AddObject@UAimIKPose@@HU?$SmallDynStorage@UAimIKPose@@HUStandardAlloc@NAlloc@@@NArray@@@ICrySizer@@QEAAXAEBU?$DynArray@UAimIKPose@@HU?$SmallDynStorage@UAimIKPose@@HUStandardAlloc@NAlloc@@@NArray@@@@@Z 00000000316181e0 f i AnimationManager.obj
 0001:00117470       ?AnimationReleaseAIM@CAnimationManager@@QEAAXAEAUGlobalAnimationHeaderAIM@@@Z 0000000031618470 f   AnimationManager.obj
 0001:00117490       ?Clear@AnimSearchHelper@@QEAAXXZ 0000000031618490 f   AnimationManager.obj
 0001:00117770       ??$AddObject@UGlobalAnimationHeaderLMG@@HU?$SmallDynStorage@UGlobalAnimationHeaderLMG@@HUStandardAlloc@NAlloc@@@NArray@@@ICrySizer@@QEAAXAEBU?$DynArray@UGlobalAnimationHeaderLMG@@HU?$SmallDynStorage@UGlobalAnimationHeaderLMG@@HUStandardAlloc@NAlloc@@@NArray@@@@@Z 0000000031618770 f i AnimationManager.obj
 0001:001178f0       ?GetMemoryUsage@GlobalAnimationHeaderAIM@@QEBAXPEAVICrySizer@@@Z 00000000316188f0 f i AnimationManager.obj
 0001:00117990       ??4?$DynArray@VCAnimEventData@@HU?$SmallDynStorage@VCAnimEventData@@HUStandardAlloc@NAlloc@@@NArray@@@@QEAAAEAU0@U?$Array@$$CBVCAnimEventData@@HU?$ArrayStorage@$$CBVCAnimEventData@@H@NArray@@@@@Z 0000000031618990 f i AnimationManager.obj
 0001:00117ad0       ?AddAnimation@AnimSearchHelper@@QEAA_NII@Z 0000000031618ad0 f   AnimationManager.obj
 0001:00117d00       ?AddAnimation@AnimSearchHelper@@QEAAXAEBV?$CryStringT@D@@I@Z 0000000031618d00 f   AnimationManager.obj
 0001:00118280       ??$AddObject@UGlobalAnimationHeaderAIM@@HU?$SmallDynStorage@UGlobalAnimationHeaderAIM@@HUStandardAlloc@NAlloc@@@NArray@@@ICrySizer@@QEAAXAEBU?$DynArray@UGlobalAnimationHeaderAIM@@HU?$SmallDynStorage@UGlobalAnimationHeaderAIM@@HUStandardAlloc@NAlloc@@@NArray@@@@@Z 0000000031619280 f i AnimationManager.obj
 0001:00118330       ??0GlobalAnimationHeaderLMG@@QEAA@XZ 0000000031619330 f i AnimationManager.obj
 0001:00118790       ?GetMemoryUsage@CAnimationManager@@QEBAXPEAVICrySizer@@@Z 0000000031619790 f   AnimationManager.obj
 0001:00118800       ??4GlobalAnimationHeaderCAF@@QEAAAEAU0@AEBU0@@Z 0000000031619800 f i AnimationManager.obj
 0001:00118990       ?CreateGlobalHeaderDBA@CAnimationManager@@QEAA_NAEAU?$DynArray@V?$CryStringT@D@@HU?$SmallDynStorage@V?$CryStringT@D@@HUStandardAlloc@NAlloc@@@NArray@@@@@Z 0000000031619990 f   AnimationManager.obj
 0001:00118bf0       ?DBA_PreLoad@CAnimationManager@@QEAA_NPEBD_N@Z 0000000031619bf0 f   AnimationManager.obj
 0001:00118fb0       ?LoadAnimationTCB@CAnimationManager@@QEAA_NHAEAU?$DynArray@UCControllerTCB@@HU?$SmallDynStorage@UCControllerTCB@@HUStandardAlloc@NAlloc@@@NArray@@@@PEAVCryCGALoader@@PEBVCSkel@@@Z 0000000031619fb0 f   AnimationManager.obj
 0001:00119740       ?init@?$DynArray@UGlobalAnimationHeaderAIM@@HU?$SmallDynStorage@UGlobalAnimationHeaderAIM@@HUStandardAlloc@NAlloc@@@NArray@@@@KAPEAUGlobalAnimationHeaderAIM@@U?$Array@UGlobalAnimationHeaderAIM@@HU?$ArrayStorage@UGlobalAnimationHeaderAIM@@H@NArray@@@@AEBU2@@Z 000000003161a740 f i AnimationManager.obj
 0001:001198b0       ?expand_raw@?$DynArray@UGlobalAnimationHeaderLMG@@HU?$SmallDynStorage@UGlobalAnimationHeaderLMG@@HUStandardAlloc@NAlloc@@@NArray@@@@IEAAPEAUGlobalAnimationHeaderLMG@@PEAU2@H@Z 000000003161a8b0 f i AnimationManager.obj
 0001:00119970       ?grow@?$DynArray@UGlobalAnimationHeaderLMG@@HU?$SmallDynStorage@UGlobalAnimationHeaderLMG@@HUStandardAlloc@NAlloc@@@NArray@@@@QEAAPEAUGlobalAnimationHeaderLMG@@HAEBU2@@Z 000000003161a970 f i AnimationManager.obj
 0001:00119a00       ?push_back@?$DynArray@UGlobalAnimationHeaderCAF@@HU?$SmallDynStorage@UGlobalAnimationHeaderCAF@@HUStandardAlloc@NAlloc@@@NArray@@@@QEAAPEAUGlobalAnimationHeaderCAF@@XZ 000000003161aa00 f i AnimationManager.obj
 0001:00119a70       ?CreateGAH_CAF@CAnimationManager@@QEAAHAEBV?$CryStringT@D@@@Z 000000003161aa70 f   AnimationManager.obj
 0001:00119b80       ?CreateGAH_LMG@CAnimationManager@@QEAAHAEBV?$CryStringT@D@@@Z 000000003161ab80 f   AnimationManager.obj
 0001:00119c50       ?CreateGAH_AIM@CAnimationManager@@QEAAHAEBV?$CryStringT@D@@@Z 000000003161ac50 f   AnimationManager.obj
 0001:00119d30       ?GetPositionsFormatSizeOf@ControllerHelper@@YAII@Z 000000003161ad30 f   ControllerPQ.obj
 0001:00119d50       ?GetRotationFormatSizeOf@ControllerHelper@@YAII@Z 000000003161ad50 f   ControllerPQ.obj
 0001:00119d80       ?GetKeyTimesFormatSizeOf@ControllerHelper@@YAII@Z 000000003161ad80 f   ControllerPQ.obj
 0001:00119dd0       ?GetOP@CController@@UEBAEMAEAU?$Quat_tpl@M@@AEAU?$Vec3_tpl@M@@@Z 000000003161add0 f   ControllerPQ.obj
 0001:00119e30       ?GetO@CController@@UEBAEMAEAU?$Quat_tpl@M@@@Z 000000003161ae30 f   ControllerPQ.obj
 0001:00119e60       ?GetP@CController@@UEBAEMAEAU?$Vec3_tpl@M@@@Z 000000003161ae60 f   ControllerPQ.obj
 0001:00119e90       ?ToExternalType@SmallTree48BitQuat@@QEBAXAEAU?$Quat_tpl@M@@@Z 000000003161ae90 f i ControllerPQ.obj
 0001:00119fe0       ?ToExternalType@SmallTree64BitExtQuat@@QEBAXAEAU?$Quat_tpl@M@@@Z 000000003161afe0 f i ControllerPQ.obj
 0001:0011a110       ?AssignData@?$CTrackDataStorageInt@U?$Vec3_tpl@M@@UNoCompressVec3@@VITrackPositionStorage@@@@UEAAIPEBDI@Z 000000003161b110 f i ControllerPQ.obj
 0001:0011a200       ?GetDataRawSize@?$CTrackDataStorageInt@U?$Vec3_tpl@M@@UNoCompressVec3@@VITrackPositionStorage@@@@UEAAIXZ 000000003161b200 f i ControllerPQ.obj
 0001:0011a210       ?GetValue@?$CTrackDataStorageInt@U?$Vec3_tpl@M@@UNoCompressVec3@@VITrackPositionStorage@@@@UEAAXIAEAU?$Vec3_tpl@M@@@Z 000000003161b210 f i ControllerPQ.obj
 0001:0011a260       ?SizeOfPosController@?$CTrackDataStorageInt@U?$Vec3_tpl@M@@UNoCompressVec3@@VITrackPositionStorage@@@@UEAA_KXZ 000000003161b260 f i ControllerPQ.obj
 0001:0011a260       ?SizeOfRotController@?$CTrackDataStorageInt@U?$Vec3_tpl@M@@UNoCompressVec3@@VITrackPositionStorage@@@@UEAA_KXZ 000000003161b260 f i ControllerPQ.obj
 0001:0011a280       ?GetData@CKeyTimesInformationBitSet@@UEAAPEADXZ 000000003161b280 f i ControllerPQ.obj
 0001:0011a280       ?GetName@CFacialEffectorsLibrary@@UEAAPEBDXZ 000000003161b280 f i FaceEffectorLibrary.obj
 0001:0011a280       ?GetData@?$CTrackDataStorageInt@U?$Quat_tpl@M@@USmallTree64BitExtQuat@@VITrackRotationStorage@@@@UEAAPEADXZ 000000003161b280 f i ControllerPQ.obj
 0001:0011a280       ?GetName@CAttachmentBONE@@UEBAPEBDXZ 000000003161b280 f i AttachmentManager.obj
 0001:0011a280       ?GetReplacementMaterial@CCGFAttachment@@UEBAPEAUIMaterial@@XZ 000000003161b280 f i AttachmentManager.obj
 0001:0011a280       ?GetData@?$CTrackDataStorageInt@U?$Quat_tpl@M@@USmallTree48BitQuat@@VITrackRotationStorage@@@@UEAAPEADXZ 000000003161b280 f i ControllerPQ.obj
 0001:0011a280       ?GetName@CAttachmentFACE@@UEBAPEBDXZ 000000003161b280 f i AttachmentManager.obj
 0001:0011a280       ?GetICharacterModel@CCharInstance@@UEAAPEAUICharacterModel@@XZ 000000003161b280 f i CharacterInstance.obj
 0001:0011a280       ?GetData@?$CTrackDataStorageInt@U?$Vec3_tpl@M@@UNoCompressVec3@@VITrackPositionStorage@@@@UEAAPEADXZ 000000003161b280 f i ControllerPQ.obj
 0001:0011a280       ?GetReplacementMaterial@CSKELAttachment@@UEBAPEAUIMaterial@@XZ 000000003161b280 f i AttachmentManager.obj
 0001:0011a280       ?GetData@?$CTrackDataStorageInt@U?$Quat_tpl@M@@USmallTree64BitQuat@@VITrackRotationStorage@@@@UEAAPEADXZ 000000003161b280 f i ControllerPQ.obj
 0001:0011a280       ?GetSoundFile@CFacialAnimSoundEntry@@UEAAPEBDXZ 000000003161b280 f i FaceAnimSequence.obj
 0001:0011a280       ?GetName@CAttachmentSKIN@@UEBAPEBDXZ 000000003161b280 f i Attachment.obj
 0001:0011a280       ?GetSkelInstance@CAttachmentManager@@UEBAPEAUICharacterInstance@@XZ 000000003161b280 f i AttachmentManager.obj
 0001:0011a280       ?GetData@?$CTrackDataStorageInt@U?$Quat_tpl@M@@UNoCompressQuat@@VITrackRotationStorage@@@@UEAAPEADXZ 000000003161b280 f i ControllerPQ.obj
 0001:0011a280       ?GetReplacementMaterial@CSKINAttachment@@UEBAPEAUIMaterial@@XZ 000000003161b280 f i AttachmentManager.obj
 0001:0011a290       ?AssignData@?$CTrackDataStorageInt@U?$Quat_tpl@M@@UNoCompressQuat@@VITrackRotationStorage@@@@UEAAIPEBDI@Z 000000003161b290 f i ControllerPQ.obj
 0001:0011a380       ?GetDataRawSize@?$CTrackDataStorageInt@U?$Quat_tpl@M@@UNoCompressQuat@@VITrackRotationStorage@@@@UEAAIXZ 000000003161b380 f i ControllerPQ.obj
 0001:0011a390       ?GetValue@?$CTrackDataStorageInt@U?$Quat_tpl@M@@UNoCompressQuat@@VITrackRotationStorage@@@@UEAAXIAEAU?$Quat_tpl@M@@@Z 000000003161b390 f i ControllerPQ.obj
 0001:0011a400       ?SizeOfPosController@?$CTrackDataStorageInt@U?$Quat_tpl@M@@UNoCompressQuat@@VITrackRotationStorage@@@@UEAA_KXZ 000000003161b400 f i ControllerPQ.obj
 0001:0011a400       ?SizeOfRotController@?$CTrackDataStorageInt@U?$Quat_tpl@M@@UNoCompressQuat@@VITrackRotationStorage@@@@UEAA_KXZ 000000003161b400 f i ControllerPQ.obj
 0001:0011a410       ?Relocate@?$CTrackDataStorageInt@U?$Quat_tpl@M@@UNoCompressQuat@@VITrackRotationStorage@@@@UEAAXPEAD0@Z 000000003161b410 f i ControllerPQ.obj
 0001:0011a410       ?Relocate@?$CKeyTimesInformation@EUByteEncoder@@@@UEAAXPEAD0@Z 000000003161b410 f i ControllerPQ.obj
 0001:0011a410       ?Relocate@?$CTrackDataStorageInt@U?$Quat_tpl@M@@USmallTree64BitQuat@@VITrackRotationStorage@@@@UEAAXPEAD0@Z 000000003161b410 f i ControllerPQ.obj
 0001:0011a410       ?Relocate@?$CKeyTimesInformation@MUF32Encoder@@@@UEAAXPEAD0@Z 000000003161b410 f i ControllerPQ.obj
 0001:0011a410       ?Relocate@?$CKeyTimesInformation@GUUINT16Encoder@@@@UEAAXPEAD0@Z 000000003161b410 f i ControllerPQ.obj
 0001:0011a410       ?Relocate@?$CTrackDataStorageInt@U?$Quat_tpl@M@@USmallTree64BitExtQuat@@VITrackRotationStorage@@@@UEAAXPEAD0@Z 000000003161b410 f i ControllerPQ.obj
 0001:0011a410       ?Relocate@?$CTrackDataStorageInt@U?$Vec3_tpl@M@@UNoCompressVec3@@VITrackPositionStorage@@@@UEAAXPEAD0@Z 000000003161b410 f i ControllerPQ.obj
 0001:0011a410       ?Relocate@?$CTrackDataStorageInt@U?$Quat_tpl@M@@USmallTree48BitQuat@@VITrackRotationStorage@@@@UEAAXPEAD0@Z 000000003161b410 f i ControllerPQ.obj
 0001:0011a420       ?AssignData@?$CTrackDataStorageInt@U?$Quat_tpl@M@@USmallTree48BitQuat@@VITrackRotationStorage@@@@UEAAIPEBDI@Z 000000003161b420 f i ControllerPQ.obj
 0001:0011a510       ?GetDataRawSize@?$CTrackDataStorageInt@U?$Quat_tpl@M@@USmallTree48BitQuat@@VITrackRotationStorage@@@@UEAAIXZ 000000003161b510 f i ControllerPQ.obj
 0001:0011a520       ?GetValue@?$CTrackDataStorageInt@U?$Quat_tpl@M@@USmallTree48BitQuat@@VITrackRotationStorage@@@@UEAAXIAEAU?$Quat_tpl@M@@@Z 000000003161b520 f i ControllerPQ.obj
 0001:0011a560       ?SizeOfRotController@?$CTrackDataStorageInt@U?$Quat_tpl@M@@USmallTree48BitQuat@@VITrackRotationStorage@@@@UEAA_KXZ 000000003161b560 f i ControllerPQ.obj
 0001:0011a560       ?SizeOfPosController@?$CTrackDataStorageInt@U?$Quat_tpl@M@@USmallTree48BitQuat@@VITrackRotationStorage@@@@UEAA_KXZ 000000003161b560 f i ControllerPQ.obj
 0001:0011a580       ?GetDataRawSize@?$CTrackDataStorageInt@U?$Quat_tpl@M@@USmallTree64BitExtQuat@@VITrackRotationStorage@@@@UEAAIXZ 000000003161b580 f i ControllerPQ.obj
 0001:0011a580       ?GetDataRawSize@?$CTrackDataStorageInt@U?$Quat_tpl@M@@USmallTree64BitQuat@@VITrackRotationStorage@@@@UEAAIXZ 000000003161b580 f i ControllerPQ.obj
 0001:0011a590       ?GetValue@?$CTrackDataStorageInt@U?$Quat_tpl@M@@USmallTree64BitQuat@@VITrackRotationStorage@@@@UEAAXIAEAU?$Quat_tpl@M@@@Z 000000003161b590 f i ControllerPQ.obj
 0001:0011a5e0       ?GetFormat@CKeyTimesInformationBitSet@@UEAAIXZ 000000003161b5e0 f i ControllerPQ.obj
 0001:0011a5e0       ?GetFormat@?$CTrackDataStorageInt@U?$Quat_tpl@M@@USmallTree64BitQuat@@VITrackRotationStorage@@@@UEAAIXZ 000000003161b5e0 f i ControllerPQ.obj
 0001:0011a5f0       ?AssignData@?$CTrackDataStorageInt@U?$Quat_tpl@M@@USmallTree64BitQuat@@VITrackRotationStorage@@@@UEAAIPEBDI@Z 000000003161b5f0 f i ControllerPQ.obj
 0001:0011a5f0       ?AssignData@?$CTrackDataStorageInt@U?$Quat_tpl@M@@USmallTree64BitExtQuat@@VITrackRotationStorage@@@@UEAAIPEBDI@Z 000000003161b5f0 f i ControllerPQ.obj
 0001:0011a6e0       ?GetValue@?$CTrackDataStorageInt@U?$Quat_tpl@M@@USmallTree64BitExtQuat@@VITrackRotationStorage@@@@UEAAXIAEAU?$Quat_tpl@M@@@Z 000000003161b6e0 f i ControllerPQ.obj
 0001:0011a710       ?GetDataRawSize@?$CKeyTimesInformationStartStop@MUF32StartStopEncoder@@@@UEAAIXZ 000000003161b710 f i ControllerPQ.obj
 0001:0011a710       ?GetFormat@?$CTrackDataStorageInt@U?$Quat_tpl@M@@USmallTree64BitExtQuat@@VITrackRotationStorage@@@@UEAAIXZ 000000003161b710 f i ControllerPQ.obj
 0001:0011a720       ?SizeOfRotController@?$CTrackDataStorageInt@U?$Quat_tpl@M@@USmallTree64BitExtQuat@@VITrackRotationStorage@@@@UEAA_KXZ 000000003161b720 f i ControllerPQ.obj
 0001:0011a720       ?SizeOfPosController@?$CTrackDataStorageInt@U?$Quat_tpl@M@@USmallTree64BitQuat@@VITrackRotationStorage@@@@UEAA_KXZ 000000003161b720 f i ControllerPQ.obj
 0001:0011a720       ?SizeOfPosController@?$CTrackDataStorageInt@U?$Quat_tpl@M@@USmallTree64BitExtQuat@@VITrackRotationStorage@@@@UEAA_KXZ 000000003161b720 f i ControllerPQ.obj
 0001:0011a720       ?SizeOfRotController@?$CTrackDataStorageInt@U?$Quat_tpl@M@@USmallTree64BitQuat@@VITrackRotationStorage@@@@UEAA_KXZ 000000003161b720 f i ControllerPQ.obj
 0001:0011a730       ?GetKey@?$CKeyTimesInformation@MUF32Encoder@@@@UEAAIMAEAM@Z 000000003161b730 f i ControllerPQ.obj
 0001:0011a810       ?GetKey@?$CKeyTimesInformation@GUUINT16Encoder@@@@UEAAIMAEAM@Z 000000003161b810 f i ControllerPQ.obj
 0001:0011a950       ?GetKey@?$CKeyTimesInformation@EUByteEncoder@@@@UEAAIMAEAM@Z 000000003161b950 f i ControllerPQ.obj
 0001:0011aa90       ?GetDataRawSize@?$CKeyTimesInformation@EUByteEncoder@@@@UEAAIXZ 000000003161ba90 f i ControllerPQ.obj
 0001:0011aa90       ?GetNumKeys@?$CKeyTimesInformation@EUByteEncoder@@@@UEBAIXZ 000000003161ba90 f i ControllerPQ.obj
 0001:0011aa90       ?GetNumKeys@?$CKeyTimesInformation@GUUINT16Encoder@@@@UEBAIXZ 000000003161ba90 f i ControllerPQ.obj
 0001:0011aa90       ?GetNumKeys@?$CKeyTimesInformation@MUF32Encoder@@@@UEBAIXZ 000000003161ba90 f i ControllerPQ.obj
 0001:0011aaa0       ??_G?$CTrackDataStorageInt@U?$Vec3_tpl@M@@UNoCompressVec3@@VITrackPositionStorage@@@@UEAAPEAXI@Z 000000003161baa0 f i ControllerPQ.obj
 0001:0011aaa0       ??_E?$CTrackDataStorageInt@U?$Vec3_tpl@M@@UNoCompressVec3@@VITrackPositionStorage@@@@UEAAPEAXI@Z 000000003161baa0 f i ControllerPQ.obj
 0001:0011aaa0       ??_E?$CTrackDataStorage@U?$Vec3_tpl@M@@UNoCompressVec3@@VITrackPositionStorage@@@@UEAAPEAXI@Z 000000003161baa0 f i ControllerPQ.obj
 0001:0011aaa0       ??_G?$CTrackDataStorage@U?$Vec3_tpl@M@@UNoCompressVec3@@VITrackPositionStorage@@@@UEAAPEAXI@Z 000000003161baa0 f i ControllerPQ.obj
 0001:0011ab00       ?GetDataRawSize@CKeyTimesInformationBitSet@@UEAAIXZ 000000003161bb00 f i ControllerPQ.obj
 0001:0011ab10       ?GetKeyValueFloat@CKeyTimesInformationBitSet@@UEBAMI@Z 000000003161bb10 f i ControllerPQ.obj
 0001:0011abe0       ?GetKey@CKeyTimesInformationBitSet@@UEAAIMAEAM@Z 000000003161bbe0 f i ControllerPQ.obj
 0001:0011ade0       ?GetNumKeys@CKeyTimesInformationBitSet@@UEBAIXZ 000000003161bde0 f i ControllerPQ.obj
 0001:0011adf0       ?AssignKeyTime@CKeyTimesInformationBitSet@@UEAAIPEBDI@Z 000000003161bdf0 f i ControllerPQ.obj
 0001:0011ae80       ?GetMemoryUsage@CKeyTimesInformationBitSet@@UEBAXPEAVICrySizer@@@Z 000000003161be80 f i ControllerPQ.obj
 0001:0011aed0       ?GetRotValueFromKey@CControllerOptNonVirtual@@QEBAXIAEAU?$Quat_tpl@M@@@Z 000000003161bed0 f i ControllerPQ.obj
 0001:0011afa0       ??_ECKeyTimesInformationBitSet@@UEAAPEAXI@Z 000000003161bfa0 f i ControllerPQ.obj
 0001:0011b090       ?GetValueFromKey@IPositionController@@UEAAXIAEAU?$Vec3_tpl@M@@@Z 000000003161c090 f   ControllerPQ.obj
 0001:0011b090       ?GetValueFromKey@IRotationController@@UEAAXIAEAU?$Quat_tpl@M@@@Z 000000003161c090 f   ControllerPQ.obj
 0001:0011b0e0       ?GetMemoryUsage@?$CTrackDataStorage@U?$Quat_tpl@M@@UNoCompressQuat@@VITrackRotationStorage@@@@UEBAXPEAVICrySizer@@@Z 000000003161c0e0 f i ControllerPQ.obj
 0001:0011b0e0       ?GetMemoryUsage@?$CTrackDataStorage@U?$Quat_tpl@M@@USmallTree64BitQuat@@VITrackRotationStorage@@@@UEBAXPEAVICrySizer@@@Z 000000003161c0e0 f i ControllerPQ.obj
 0001:0011b0e0       ?GetMemoryUsage@?$CTrackDataStorage@U?$Vec3_tpl@M@@UNoCompressVec3@@VITrackPositionStorage@@@@UEBAXPEAVICrySizer@@@Z 000000003161c0e0 f i ControllerPQ.obj
 0001:0011b0e0       ?GetMemoryUsage@?$CTrackDataStorage@U?$Quat_tpl@M@@USmallTree64BitExtQuat@@VITrackRotationStorage@@@@UEBAXPEAVICrySizer@@@Z 000000003161c0e0 f i ControllerPQ.obj
 0001:0011b0e0       ?GetMemoryUsage@?$CTrackDataStorage@U?$Quat_tpl@M@@USmallTree48BitQuat@@VITrackRotationStorage@@@@UEBAXPEAVICrySizer@@@Z 000000003161c0e0 f i ControllerPQ.obj
 0001:0011b100       ?Release@?$CTrackDataStorage@U?$Quat_tpl@M@@USmallTree64BitExtQuat@@VITrackRotationStorage@@@@UEAAXXZ 000000003161c100 f i ControllerPQ.obj
 0001:0011b100       ?Release@?$CTrackDataStorage@U?$Vec3_tpl@M@@UNoCompressVec3@@VITrackPositionStorage@@@@UEAAXXZ 000000003161c100 f i ControllerPQ.obj
 0001:0011b100       ?Release@?$CTrackDataStorage@U?$Quat_tpl@M@@UNoCompressQuat@@VITrackRotationStorage@@@@UEAAXXZ 000000003161c100 f i ControllerPQ.obj
 0001:0011b100       ?Release@?$CTrackDataStorage@U?$Quat_tpl@M@@USmallTree48BitQuat@@VITrackRotationStorage@@@@UEAAXXZ 000000003161c100 f i ControllerPQ.obj
 0001:0011b100       ?Release@?$CTrackDataStorage@U?$Quat_tpl@M@@USmallTree64BitQuat@@VITrackRotationStorage@@@@UEAAXXZ 000000003161c100 f i ControllerPQ.obj
 0001:0011b120       ?GetKeyValueFloat@?$CKeyTimesInformation@MUF32Encoder@@@@UEBAMI@Z 000000003161c120 f i ControllerPQ.obj
 0001:0011b130       ?GetMemoryUsage@?$CKeyTimesInformation@EUByteEncoder@@@@UEBAXPEAVICrySizer@@@Z 000000003161c130 f i ControllerPQ.obj
 0001:0011b130       ?GetMemoryUsage@?$CKeyTimesInformation@GUUINT16Encoder@@@@UEBAXPEAVICrySizer@@@Z 000000003161c130 f i ControllerPQ.obj
 0001:0011b130       ?GetMemoryUsage@?$CKeyTimesInformation@MUF32Encoder@@@@UEBAXPEAVICrySizer@@@Z 000000003161c130 f i ControllerPQ.obj
 0001:0011b130       ?GetMemoryUsage@COperatorQueue@@UEBAXPEAVICrySizer@@@Z 000000003161c130 f i OperatorQueue.obj
 0001:0011b150       ?AssignKeyTime@?$CKeyTimesInformation@MUF32Encoder@@@@UEAAIPEBDI@Z 000000003161c150 f i ControllerPQ.obj
 0001:0011b250       ?GetDataRawSize@?$CKeyTimesInformation@MUF32Encoder@@@@UEAAIXZ 000000003161c250 f i ControllerPQ.obj
 0001:0011b260       ?GetKeyValueFloat@?$CKeyTimesInformation@GUUINT16Encoder@@@@UEBAMI@Z 000000003161c260 f i ControllerPQ.obj
 0001:0011b280       ?GetIAttachmentObject@CAttachmentFACE@@UEBAPEAUIAttachmentObject@@XZ 000000003161c280 f i AttachmentManager.obj
 0001:0011b280       ?GetIAttachmentObject@CAttachmentSKIN@@UEBAPEAUIAttachmentObject@@XZ 000000003161c280 f i Attachment.obj
 0001:0011b280       ?GetData@?$CKeyTimesInformation@GUUINT16Encoder@@@@UEAAPEADXZ 000000003161c280 f i ControllerPQ.obj
 0001:0011b280       ?GetData@?$CKeyTimesInformation@EUByteEncoder@@@@UEAAPEADXZ 000000003161c280 f i ControllerPQ.obj
 0001:0011b280       ?GetData@?$CKeyTimesInformation@MUF32Encoder@@@@UEAAPEADXZ 000000003161c280 f i ControllerPQ.obj
 0001:0011b280       ?GetIAttachmentObject@CAttachmentBONE@@UEBAPEAUIAttachmentObject@@XZ 000000003161c280 f i AttachmentManager.obj
 0001:0011b290       ?GetRelocateChain@?$CKeyTimesInformation@MUF32Encoder@@@@UEAAPEAVIControllerRelocatableChain@@XZ 000000003161c290 f i ControllerPQ.obj
 0001:0011b290       ?GetRelocateChain@?$CKeyTimesInformation@EUByteEncoder@@@@UEAAPEAVIControllerRelocatableChain@@XZ 000000003161c290 f i ControllerPQ.obj
 0001:0011b290       ?GetRelocateChain@?$CKeyTimesInformation@GUUINT16Encoder@@@@UEAAPEAVIControllerRelocatableChain@@XZ 000000003161c290 f i ControllerPQ.obj
 0001:0011b2a0       ?AssignKeyTime@?$CKeyTimesInformation@GUUINT16Encoder@@@@UEAAIPEBDI@Z 000000003161c2a0 f i ControllerPQ.obj
 0001:0011b3a0       ?GetDataRawSize@?$CKeyTimesInformation@GUUINT16Encoder@@@@UEAAIXZ 000000003161c3a0 f i ControllerPQ.obj
 0001:0011b3b0       ?GetKeyValueFloat@?$CKeyTimesInformation@EUByteEncoder@@@@UEBAMI@Z 000000003161c3b0 f i ControllerPQ.obj
 0001:0011b3d0       ?AssignKeyTime@?$CKeyTimesInformation@EUByteEncoder@@@@UEAAIPEBDI@Z 000000003161c3d0 f i ControllerPQ.obj
 0001:0011b4d0       ?GetKeyValueFloat@?$CKeyTimesInformationStartStop@MUF32StartStopEncoder@@@@UEBAMI@Z 000000003161c4d0 f i ControllerPQ.obj
 0001:0011b4f0       ?GetKey@?$CKeyTimesInformationStartStop@MUF32StartStopEncoder@@@@UEAAIMAEAM@Z 000000003161c4f0 f i ControllerPQ.obj
 0001:0011b530       ?GetNumKeys@?$CKeyTimesInformationStartStop@MUF32StartStopEncoder@@@@UEBAIXZ 000000003161c530 f i ControllerPQ.obj
 0001:0011b540       ?AssignKeyTime@?$CKeyTimesInformationStartStop@MUF32StartStopEncoder@@@@UEAAIPEBDI@Z 000000003161c540 f i ControllerPQ.obj
 0001:0011b550       ?GetKeyValueFloat@?$CKeyTimesInformationStartStop@GUUINT16StartStopEncoder@@@@UEBAMI@Z 000000003161c550 f i ControllerPQ.obj
 0001:0011b560       ?GetKey@?$CKeyTimesInformationStartStop@GUUINT16StartStopEncoder@@@@UEAAIMAEAM@Z 000000003161c560 f i ControllerPQ.obj
 0001:0011b5a0       ?GetNumKeys@?$CKeyTimesInformationStartStop@GUUINT16StartStopEncoder@@@@UEBAIXZ 000000003161c5a0 f i ControllerPQ.obj
 0001:0011b5b0       ?AssignKeyTime@?$CKeyTimesInformationStartStop@GUUINT16StartStopEncoder@@@@UEAAIPEBDI@Z 000000003161c5b0 f i ControllerPQ.obj
 0001:0011b5c0       ?GetDataRawSize@?$CKeyTimesInformationStartStop@GUUINT16StartStopEncoder@@@@UEAAIXZ 000000003161c5c0 f i ControllerPQ.obj
 0001:0011b5c0       ?GetNumDimensions@CFacialCameraPathOrientationInterpolator@@UEAAHXZ 000000003161c5c0 f i FaceAnimSequence.obj
 0001:0011b5c0       ?GetFormat@?$CKeyTimesInformationStartStop@GUUINT16StartStopEncoder@@@@UEAAIXZ 000000003161c5c0 f i ControllerPQ.obj
 0001:0011b5d0       ?GetKeyValueFloat@?$CKeyTimesInformationStartStop@EUByteStartStopEncoder@@@@UEBAMI@Z 000000003161c5d0 f i ControllerPQ.obj
 0001:0011b5e0       ?GetKey@?$CKeyTimesInformationStartStop@EUByteStartStopEncoder@@@@UEAAIMAEAM@Z 000000003161c5e0 f i ControllerPQ.obj
 0001:0011b620       ?GetNumKeys@?$CKeyTimesInformationStartStop@EUByteStartStopEncoder@@@@UEBAIXZ 000000003161c620 f i ControllerPQ.obj
 0001:0011b630       ?AssignKeyTime@?$CKeyTimesInformationStartStop@EUByteStartStopEncoder@@@@UEAAIPEBDI@Z 000000003161c630 f i ControllerPQ.obj
 0001:0011b640       ?GetData@?$CKeyTimesInformationStartStop@EUByteStartStopEncoder@@@@UEAAPEADXZ 000000003161c640 f i ControllerPQ.obj
 0001:0011b640       ?GetRotationStorage@IRotationController@@UEAAAEAPEAVITrackRotationStorage@@XZ 000000003161c640 f i LoaderTCB.obj
 0001:0011b640       ?GetPositionStorage@IPositionController@@UEAAAEAPEAVITrackPositionStorage@@XZ 000000003161c640 f i LoaderTCB.obj
 0001:0011b640       ?GetData@?$CKeyTimesInformationStartStop@GUUINT16StartStopEncoder@@@@UEAAPEADXZ 000000003161c640 f i ControllerPQ.obj
 0001:0011b640       ?GetData@?$CKeyTimesInformationStartStop@MUF32StartStopEncoder@@@@UEAAPEADXZ 000000003161c640 f i ControllerPQ.obj
 0001:0011b650       ?GetDataRawSize@?$CKeyTimesInformationStartStop@EUByteStartStopEncoder@@@@UEAAIXZ 000000003161c650 f i ControllerPQ.obj
 0001:0011b650       ?GetAttachmentType@CSKELAttachment@@UEAA?AW4EType@IAttachmentObject@@XZ 000000003161c650 f i AttachmentManager.obj
 0001:0011b650       ?GetType@CFacialMorphTarget@@UEAA?AW4EFacialEffectorType@@XZ 000000003161c650 f i FaceEffectorLibrary.obj
 0001:0011b650       ?GetSplineType@CFacialAnimChannelInterpolator@@UEAA?AW4ESplineType@@XZ 000000003161c650 f i FaceAnimSequence.obj
 0001:0011b650       ?GetType@CAttachmentSKIN@@UEBAIXZ 000000003161c650 f i Attachment.obj
 0001:0011b650       ?GetFormat@?$CKeyTimesInformation@EUByteEncoder@@@@UEAAIXZ 000000003161c650 f i ControllerPQ.obj
 0001:0011b650       ?GetFormat@?$CTrackDataStorageInt@U?$Vec3_tpl@M@@UNoCompressVec3@@VITrackPositionStorage@@@@UEAAIXZ 000000003161c650 f i ControllerPQ.obj
 0001:0011b660       ?GetMemoryUsage@?$CKeyTimesInformationStartStop@MUF32StartStopEncoder@@@@UEBAXPEAVICrySizer@@@Z 000000003161c660 f i ControllerPQ.obj
 0001:0011b660       ?GetMemoryUsage@?$CKeyTimesInformationStartStop@EUByteStartStopEncoder@@@@UEBAXPEAVICrySizer@@@Z 000000003161c660 f i ControllerPQ.obj
 0001:0011b660       ?GetMemoryUsage@?$CKeyTimesInformationStartStop@GUUINT16StartStopEncoder@@@@UEBAXPEAVICrySizer@@@Z 000000003161c660 f i ControllerPQ.obj
 0001:0011b660       ?GetMemoryUsage@CPoseMatching@@UEBAXPEAVICrySizer@@@Z 000000003161c660 f i PoseMatching.obj
 0001:0011b680       ??_G?$CTrackDataStorageInt@U?$Quat_tpl@M@@UNoCompressQuat@@VITrackRotationStorage@@@@UEAAPEAXI@Z 000000003161c680 f i ControllerPQ.obj
 0001:0011b680       ??_G?$CTrackDataStorage@U?$Quat_tpl@M@@UNoCompressQuat@@VITrackRotationStorage@@@@UEAAPEAXI@Z 000000003161c680 f i ControllerPQ.obj
 0001:0011b680       ??_E?$CTrackDataStorageInt@U?$Quat_tpl@M@@UNoCompressQuat@@VITrackRotationStorage@@@@UEAAPEAXI@Z 000000003161c680 f i ControllerPQ.obj
 0001:0011b680       ??_E?$CTrackDataStorage@U?$Quat_tpl@M@@UNoCompressQuat@@VITrackRotationStorage@@@@UEAAPEAXI@Z 000000003161c680 f i ControllerPQ.obj
 0001:0011b6e0       ??_G?$CTrackDataStorage@U?$Quat_tpl@M@@USmallTree48BitQuat@@VITrackRotationStorage@@@@UEAAPEAXI@Z 000000003161c6e0 f i ControllerPQ.obj
 0001:0011b6e0       ??_E?$CTrackDataStorage@U?$Quat_tpl@M@@USmallTree48BitQuat@@VITrackRotationStorage@@@@UEAAPEAXI@Z 000000003161c6e0 f i ControllerPQ.obj
 0001:0011b6e0       ??_G?$CTrackDataStorageInt@U?$Quat_tpl@M@@USmallTree48BitQuat@@VITrackRotationStorage@@@@UEAAPEAXI@Z 000000003161c6e0 f i ControllerPQ.obj
 0001:0011b6e0       ??_E?$CTrackDataStorageInt@U?$Quat_tpl@M@@USmallTree48BitQuat@@VITrackRotationStorage@@@@UEAAPEAXI@Z 000000003161c6e0 f i ControllerPQ.obj
 0001:0011b740       ??_E?$CTrackDataStorageInt@U?$Quat_tpl@M@@USmallTree64BitQuat@@VITrackRotationStorage@@@@UEAAPEAXI@Z 000000003161c740 f i ControllerPQ.obj
 0001:0011b740       ??_E?$CTrackDataStorage@U?$Quat_tpl@M@@USmallTree64BitQuat@@VITrackRotationStorage@@@@UEAAPEAXI@Z 000000003161c740 f i ControllerPQ.obj
 0001:0011b740       ??_G?$CTrackDataStorage@U?$Quat_tpl@M@@USmallTree64BitQuat@@VITrackRotationStorage@@@@UEAAPEAXI@Z 000000003161c740 f i ControllerPQ.obj
 0001:0011b740       ??_G?$CTrackDataStorageInt@U?$Quat_tpl@M@@USmallTree64BitQuat@@VITrackRotationStorage@@@@UEAAPEAXI@Z 000000003161c740 f i ControllerPQ.obj
 0001:0011b7a0       ??_G?$CTrackDataStorageInt@U?$Quat_tpl@M@@USmallTree64BitExtQuat@@VITrackRotationStorage@@@@UEAAPEAXI@Z 000000003161c7a0 f i ControllerPQ.obj
 0001:0011b7a0       ??_E?$CTrackDataStorage@U?$Quat_tpl@M@@USmallTree64BitExtQuat@@VITrackRotationStorage@@@@UEAAPEAXI@Z 000000003161c7a0 f i ControllerPQ.obj
 0001:0011b7a0       ??_E?$CTrackDataStorageInt@U?$Quat_tpl@M@@USmallTree64BitExtQuat@@VITrackRotationStorage@@@@UEAAPEAXI@Z 000000003161c7a0 f i ControllerPQ.obj
 0001:0011b7a0       ??_G?$CTrackDataStorage@U?$Quat_tpl@M@@USmallTree64BitExtQuat@@VITrackRotationStorage@@@@UEAAPEAXI@Z 000000003161c7a0 f i ControllerPQ.obj
 0001:0011b800       ??0CKeyTimesInformationBitSet@@QEAA@PEAGI@Z 000000003161c800 f i ControllerPQ.obj
 0001:0011b840       ?GetPositionControllerPtr@ControllerHelper@@YAPEAVITrackPositionStorage@@IPEAX_K@Z 000000003161c840 f   ControllerPQ.obj
 0001:0011b8b0       ?GetRotationControllerPtr@ControllerHelper@@YAPEAVITrackRotationStorage@@IPEAX_K@Z 000000003161c8b0 f   ControllerPQ.obj
 0001:0011b9c0       ?GetKeyTimesControllerPtr@ControllerHelper@@YAPEAVIKeyTimesInformation@@IPEAX_K@Z 000000003161c9c0 f   ControllerPQ.obj
 0001:0011bbe0       ??_E?$CKeyTimesInformation@MUF32Encoder@@@@UEAAPEAXI@Z 000000003161cbe0 f i ControllerPQ.obj
 0001:0011bd20       ??_E?$CKeyTimesInformation@GUUINT16Encoder@@@@UEAAPEAXI@Z 000000003161cd20 f i ControllerPQ.obj
 0001:0011be60       ??_E?$CKeyTimesInformation@EUByteEncoder@@@@UEAAPEAXI@Z 000000003161ce60 f i ControllerPQ.obj
 0001:0011bfa0       ??_E?$CKeyTimesInformationStartStop@GUUINT16StartStopEncoder@@@@UEAAPEAXI@Z 000000003161cfa0 f i ControllerPQ.obj
 0001:0011bfa0       ??_E?$CKeyTimesInformationStartStop@MUF32StartStopEncoder@@@@UEAAPEAXI@Z 000000003161cfa0 f i ControllerPQ.obj
 0001:0011bfa0       ??_E?$CKeyTimesInformationStartStop@EUByteStartStopEncoder@@@@UEAAPEAXI@Z 000000003161cfa0 f i ControllerPQ.obj
 0001:0011c020       ??_E?$CKeyTimesInformation@MUF32Encoder@@@@WBA@EAAPEAXI@Z 000000003161d020 f i ControllerPQ.obj
 0001:0011c030       ??_E?$CKeyTimesInformation@GUUINT16Encoder@@@@WBA@EAAPEAXI@Z 000000003161d030 f i ControllerPQ.obj
 0001:0011c040       ??_E?$CKeyTimesInformation@EUByteEncoder@@@@WBA@EAAPEAXI@Z 000000003161d040 f i ControllerPQ.obj
 0001:0011c050       ?GetRotValue@CControllerOptNonVirtual@@QEBA?AU?$Quat_tpl@M@@M@Z 000000003161d050 f i ControllerPQ.obj
 0001:0011c2f0       ?GetO@CControllerOptNonVirtual@@UEBAEMAEAU?$Quat_tpl@M@@@Z 000000003161d2f0 f   ControllerPQ.obj
 0001:0011c340       ?GetOP@CControllerOptNonVirtual@@UEBAEMAEAU?$Quat_tpl@M@@AEAU?$Vec3_tpl@M@@@Z 000000003161d340 f   ControllerPQ.obj
 0001:0011c3e0       ?AdjustLogRotations@@YAXAEAU?$Vec3_tpl@M@@0@Z 000000003161d3e0 f   ControllerPQLog.obj
 0001:0011c550       ?blendPQ@PQLog@@QEAAXAEBU1@0M@Z 000000003161d550 f   ControllerPQLog.obj
 0001:0011c8f0       ?GetOPS@CControllerPQLog@@UEBAEMAEAU?$Quat_tpl@M@@AEAU?$Vec3_tpl@M@@AEAU?$Diag33_tpl@M@@@Z 000000003161d8f0 f   ControllerPQLog.obj
 0001:0011cea0       ?GetOP@CControllerPQLog@@UEBAEMAEAU?$Quat_tpl@M@@AEAU?$Vec3_tpl@M@@@Z 000000003161dea0 f   ControllerPQLog.obj
 0001:0011d450       ?GetO@CControllerPQLog@@UEBAEMAEAU?$Quat_tpl@M@@@Z 000000003161e450 f   ControllerPQLog.obj
 0001:0011d960       ?GetP@CControllerPQLog@@UEBAEMAEAU?$Vec3_tpl@M@@@Z 000000003161e960 f   ControllerPQLog.obj
 0001:0011deb0       ??1CControllerPQLog@@UEAA@XZ 000000003161eeb0 f   ControllerPQLog.obj
 0001:0011df30       ?GetO_numKey@CControllerPQLog@@UEBAHXZ 000000003161ef30 f i ControllerPQLog.obj
 0001:0011df30       ?GetP_numKey@CControllerPQLog@@UEBAHXZ 000000003161ef30 f i ControllerPQLog.obj
 0001:0011df30       ?GetJointCount@CModelSkeleton@@UEBAIXZ 000000003161ef30 f i Model.obj
 0001:0011df40       ?get_alloc_size@?$SmallDynStorage@UPQLog@@HUStandardAlloc@NAlloc@@@NArray@@QEBAHXZ 000000003161ef40 f i ControllerPQLog.obj
 0001:0011dfa0       ?SizeOfController@CControllerPQLog@@UEBA_KXZ 000000003161efa0 f i ControllerPQLog.obj
 0001:0011e070       ?GetMemoryUsage@CControllerPQLog@@UEBAXPEAVICrySizer@@@Z 000000003161f070 f i ControllerPQLog.obj
 0001:0011e0d0       ??0CControllerPQLog@@QEAA@XZ 000000003161f0d0 f   ControllerPQLog.obj
 0001:0011e1a0       ??_GCControllerPQLog@@UEAAPEAXI@Z 000000003161f1a0 f i ControllerPQLog.obj
 0001:0011e1a0       ??_ECControllerPQLog@@UEAAPEAXI@Z 000000003161f1a0 f i ControllerPQLog.obj
 0001:0011e1d0       ??$__unguarded_linear_insert@PEAUTCBAngAxisKey@spline@@U12@U?$less@UTCBAngAxisKey@spline@@@stlpmtx_std@@@priv@stlpmtx_std@@YAXPEAUTCBAngAxisKey@spline@@U23@U?$less@UTCBAngAxisKey@spline@@@1@@Z 000000003161f1d0 f i ControllerTCB.obj
 0001:0011e2a0       ??$__push_heap@PEAUTCBAngAxisKey@spline@@_JU12@U?$less@UTCBAngAxisKey@spline@@@stlpmtx_std@@@stlpmtx_std@@YAXPEAUTCBAngAxisKey@spline@@_J1U12@U?$less@UTCBAngAxisKey@spline@@@0@@Z 000000003161f2a0 f i ControllerTCB.obj
 0001:0011e3d0       ??$__copy_backward@PEAUTCBAngAxisKey@spline@@PEAU12@_J@priv@stlpmtx_std@@YAPEAUTCBAngAxisKey@spline@@PEAU23@00AEBUrandom_access_iterator_tag@1@PEA_J@Z 000000003161f3d0 f i ControllerTCB.obj
 0001:0011e690       ?seek_key@?$TSpline@UTCBAngAxisKey@spline@@VHermitBasis@2@@spline@@IEAAHM@Z 000000003161f690 f i ControllerTCB.obj
 0001:0011e710       ??$__unguarded_insertion_sort_aux@PEAUTCBAngAxisKey@spline@@U12@U?$less@UTCBAngAxisKey@spline@@@stlpmtx_std@@@priv@stlpmtx_std@@YAXPEAUTCBAngAxisKey@spline@@00U?$less@UTCBAngAxisKey@spline@@@1@@Z 000000003161f710 f i ControllerTCB.obj
 0001:0011e860       ??$__adjust_heap@PEAUTCBAngAxisKey@spline@@_JU12@U?$less@UTCBAngAxisKey@spline@@@stlpmtx_std@@@stlpmtx_std@@YAXPEAUTCBAngAxisKey@spline@@_J1U12@U?$less@UTCBAngAxisKey@spline@@@0@@Z 000000003161f860 f i ControllerTCB.obj
 0001:0011eab0       ??$swap@UTCBAngAxisKey@spline@@@stlpmtx_std@@YAXAEAUTCBAngAxisKey@spline@@0@Z 000000003161fab0 f i ControllerTCB.obj
 0001:0011ecb0       ??$__pop_heap@PEAUTCBAngAxisKey@spline@@U12@U?$less@UTCBAngAxisKey@spline@@@stlpmtx_std@@_J@stlpmtx_std@@YAXPEAUTCBAngAxisKey@spline@@00U12@U?$less@UTCBAngAxisKey@spline@@@0@PEA_J@Z 000000003161fcb0 f i ControllerTCB.obj
 0001:0011ee60       ??$__make_heap@PEAUTCBAngAxisKey@spline@@U?$less@UTCBAngAxisKey@spline@@@stlpmtx_std@@U12@_J@stlpmtx_std@@YAXPEAUTCBAngAxisKey@spline@@0U?$less@UTCBAngAxisKey@spline@@@0@0PEA_J@Z 000000003161fe60 f i ControllerTCB.obj
 0001:0011f110       ??$__pop_heap_aux@PEAUTCBAngAxisKey@spline@@U12@U?$less@UTCBAngAxisKey@spline@@@stlpmtx_std@@@stlpmtx_std@@YAXPEAUTCBAngAxisKey@spline@@00U?$less@UTCBAngAxisKey@spline@@@0@@Z 0000000031620110 f i ControllerTCB.obj
 0001:0011f220       ??$__linear_insert@PEAUTCBAngAxisKey@spline@@U12@U?$less@UTCBAngAxisKey@spline@@@stlpmtx_std@@@priv@stlpmtx_std@@YAXPEAUTCBAngAxisKey@spline@@0U23@U?$less@UTCBAngAxisKey@spline@@@1@@Z 0000000031620220 f i ControllerTCB.obj
 0001:0011f3c0       ??$sort_heap@PEAUTCBAngAxisKey@spline@@U?$less@UTCBAngAxisKey@spline@@@stlpmtx_std@@@stlpmtx_std@@YAXPEAUTCBAngAxisKey@spline@@0U?$less@UTCBAngAxisKey@spline@@@0@@Z 00000000316203c0 f i ControllerTCB.obj
 0001:0011f470       ??$__insertion_sort@PEAUTCBAngAxisKey@spline@@U12@U?$less@UTCBAngAxisKey@spline@@@stlpmtx_std@@@priv@stlpmtx_std@@YAXPEAUTCBAngAxisKey@spline@@00U?$less@UTCBAngAxisKey@spline@@@1@@Z 0000000031620470 f i ControllerTCB.obj
 0001:0011f5d0       ??$__partial_sort@PEAUTCBAngAxisKey@spline@@U12@U?$less@UTCBAngAxisKey@spline@@@stlpmtx_std@@@priv@stlpmtx_std@@YAXPEAUTCBAngAxisKey@spline@@000U?$less@UTCBAngAxisKey@spline@@@1@@Z 00000000316205d0 f i ControllerTCB.obj
 0001:0011f760       ??$__final_insertion_sort@PEAUTCBAngAxisKey@spline@@U?$less@UTCBAngAxisKey@spline@@@stlpmtx_std@@@priv@stlpmtx_std@@YAXPEAUTCBAngAxisKey@spline@@0U?$less@UTCBAngAxisKey@spline@@@1@@Z 0000000031620760 f i ControllerTCB.obj
 0001:0011f7e0       ??$__introsort_loop@PEAUTCBAngAxisKey@spline@@U12@_JU?$less@UTCBAngAxisKey@spline@@@stlpmtx_std@@@priv@stlpmtx_std@@YAXPEAUTCBAngAxisKey@spline@@00_JU?$less@UTCBAngAxisKey@spline@@@1@@Z 00000000316207e0 f i ControllerTCB.obj
 0001:0011f960       ??$sort@PEAUTCBAngAxisKey@spline@@@stlpmtx_std@@YAXPEAUTCBAngAxisKey@spline@@0@Z 0000000031620960 f i ControllerTCB.obj
 0001:0011f9f0       ?GetP@CControllerTCB@@UEBAEMAEAU?$Vec3_tpl@M@@@Z 00000000316209f0 f   ControllerTCB.obj
 0001:0011fb20       ?GetS@CControllerTCB@@UEBAEMAEAU?$Diag33_tpl@M@@@Z 0000000031620b20 f   ControllerTCB.obj
 0001:0011fc20       ?interpolate@?$TSpline@UTCBAngAxisKey@spline@@VHermitBasis@2@@spline@@QEAA_NMAEAU?$Quat_tpl@M@@@Z 0000000031620c20 f i ControllerTCB.obj
 0001:0011fd80       ?GetOPS@CControllerTCB@@UEBAEMAEAU?$Quat_tpl@M@@AEAU?$Vec3_tpl@M@@AEAU?$Diag33_tpl@M@@@Z 0000000031620d80 f   ControllerTCB.obj
 0001:00120030       ?GetOP@CControllerTCB@@UEBAEMAEAU?$Quat_tpl@M@@AEAU?$Vec3_tpl@M@@@Z 0000000031621030 f   ControllerTCB.obj
 0001:00120230       ?GetO@CControllerTCB@@UEBAEMAEAU?$Quat_tpl@M@@@Z 0000000031621230 f   ControllerTCB.obj
 0001:00120350       ?AnnotateExamples@VExampleInit@@QEAAIIPEAUQuadIndices@@@Z 0000000031621350 f   GlobalAnimationHeaderAIM.obj
 0001:00120350       ?Debug_AnnotateExamples2@GlobalAnimationHeaderAIM@@QEAAIIPEAUQuadIndices@@@Z 0000000031621350 f   GlobalAnimationHeaderAIM.obj
 0001:00120ec0       ?Debug_PolarCoordinate@GlobalAnimationHeaderAIM@@QEAA?AU?$Vec3_tpl@M@@AEBU?$Quat_tpl@M@@@Z 0000000031621ec0 f   GlobalAnimationHeaderAIM.obj
 0001:00121070       ?ReadMotionParameters@GlobalAnimationHeaderAIM@@QEAA_NPEAUChunkDesc@IChunkFile@@@Z 0000000031622070 f   GlobalAnimationHeaderAIM.obj
 0001:00121190       ?Debug_NLerp2AimPose@GlobalAnimationHeaderAIM@@QEAAXPEAVCModelSkeleton@@PEAUSJointsAimIK_Rot@@IPEAUSJointsAimIK_Pos@@IPEAU?$QuatT_tpl@M@@3M3@Z 0000000031622190 f   GlobalAnimationHeaderAIM.obj
 0001:00121610       ?Debug_Blend4AimPose@GlobalAnimationHeaderAIM@@QEAAXPEAVCModelSkeleton@@PEAUSJointsAimIK_Rot@@IPEAUSJointsAimIK_Pos@@ICCCCAEBU?$Vec4_tpl@M@@PEAU?$QuatT_tpl@M@@4@Z 0000000031622610 f   GlobalAnimationHeaderAIM.obj
 0001:001221d0       ?CopyPoses2@VExampleInit@@QEAAXAEAU?$DynArray@USJointsAimIK_Rot@@HU?$SmallDynStorage@USJointsAimIK_Rot@@HUStandardAlloc@NAlloc@@@NArray@@@@AEAU?$DynArray@USJointsAimIK_Pos@@HU?$SmallDynStorage@USJointsAimIK_Pos@@HUStandardAlloc@NAlloc@@@NArray@@@@AEAUGlobalAnimationHeaderAIM@@II@Z 00000000316231d0 f   GlobalAnimationHeaderAIM.obj
 0001:00122650       ?ComputeAimPose@VExampleInit@@QEAAXAEAUGlobalAnimationHeaderAIM@@PEAVCModelSkeleton@@AEAU?$DynArray@USJointsAimIK_Rot@@HU?$SmallDynStorage@USJointsAimIK_Rot@@HUStandardAlloc@NAlloc@@@NArray@@@@AEAU?$DynArray@USJointsAimIK_Pos@@HU?$SmallDynStorage@USJointsAimIK_Pos@@HUStandardAlloc@NAlloc@@@NArray@@@@PEAU?$QuatT_tpl@N@@I@Z 0000000031623650 f   GlobalAnimationHeaderAIM.obj
 0001:00122ad0       ?NLerp2AimPose@VExampleInit@@QEAAXAEAU?$DynArray@USJointsAimIK_Rot@@HU?$SmallDynStorage@USJointsAimIK_Rot@@HUStandardAlloc@NAlloc@@@NArray@@@@AEAU?$DynArray@USJointsAimIK_Pos@@HU?$SmallDynStorage@USJointsAimIK_Pos@@HUStandardAlloc@NAlloc@@@NArray@@@@PEAU?$QuatT_tpl@N@@2N2@Z 0000000031623ad0 f   GlobalAnimationHeaderAIM.obj
 0001:00122fd0       ?PolarCoordinate@VExampleInit@@QEAA?AU?$Vec3_tpl@N@@AEBU?$Quat_tpl@N@@@Z 0000000031623fd0 f   GlobalAnimationHeaderAIM.obj
 0001:00123190       ?Blend4AimPose@VExampleInit@@QEAAXAEAUGlobalAnimationHeaderAIM@@AEAU?$DynArray@USJointsAimIK_Rot@@HU?$SmallDynStorage@USJointsAimIK_Rot@@HUStandardAlloc@NAlloc@@@NArray@@@@AEAU?$DynArray@USJointsAimIK_Pos@@HU?$SmallDynStorage@USJointsAimIK_Pos@@HUStandardAlloc@NAlloc@@@NArray@@@@CCCCAEBU?$Vec4_tpl@N@@PEAU?$QuatT_tpl@N@@4@Z 0000000031624190 f   GlobalAnimationHeaderAIM.obj
 0001:00123eb0       ?clear@?$DynArray@UVirtualExampleInit2@CHUNK_GAHAIM_INFO@@HU?$SmallDynStorage@UVirtualExampleInit2@CHUNK_GAHAIM_INFO@@HUStandardAlloc@NAlloc@@@NArray@@@@QEAAXXZ 0000000031624eb0 f i GlobalAnimationHeaderAIM.obj
 0001:00123f90       ?PointInQuat@VExampleInit@@QEAAIAEBU?$Vec2_tpl@N@@AEAUGlobalAnimationHeaderAIM@@AEAU?$DynArray@USJointsAimIK_Rot@@HU?$SmallDynStorage@USJointsAimIK_Rot@@HUStandardAlloc@NAlloc@@@NArray@@@@AEAU?$DynArray@USJointsAimIK_Pos@@HU?$SmallDynStorage@USJointsAimIK_Pos@@HUStandardAlloc@NAlloc@@@NArray@@@@HHHHHAEBU?$Vec4_tpl@N@@444@Z 0000000031624f90 f   GlobalAnimationHeaderAIM.obj
 0001:00125b00       ?RecursiveTest@VExampleInit@@QEAAXAEBU?$Vec2_tpl@N@@AEAUGlobalAnimationHeaderAIM@@AEAU?$DynArray@USJointsAimIK_Rot@@HU?$SmallDynStorage@USJointsAimIK_Rot@@HUStandardAlloc@NAlloc@@@NArray@@@@AEAU?$DynArray@USJointsAimIK_Pos@@HU?$SmallDynStorage@USJointsAimIK_Pos@@HUStandardAlloc@NAlloc@@@NArray@@@@HHHHHAEBU?$Vec4_tpl@N@@444@Z 0000000031626b00 f   GlobalAnimationHeaderAIM.obj
 0001:00127050       ?ReadController@GlobalAnimationHeaderAIM@@QEAA_NPEAUChunkDesc@IChunkFile@@I@Z 0000000031628050 f   GlobalAnimationHeaderAIM.obj
 0001:00127bf0       ?LoadChunks@GlobalAnimationHeaderAIM@@QEAA_NPEAUIChunkFile@@@Z 0000000031628bf0 f   GlobalAnimationHeaderAIM.obj
 0001:00127fd0       ?LoadAIM@GlobalAnimationHeaderAIM@@QEAAIXZ 0000000031628fd0 f   GlobalAnimationHeaderAIM.obj
 0001:00128370       ?Init@VExampleInit@@QEAAXPEAVCModelSkeleton@@AEAU?$DynArray@USJointsAimIK_Rot@@HU?$SmallDynStorage@USJointsAimIK_Rot@@HUStandardAlloc@NAlloc@@@NArray@@@@AEAU?$DynArray@USJointsAimIK_Pos@@HU?$SmallDynStorage@USJointsAimIK_Pos@@HUStandardAlloc@NAlloc@@@NArray@@@@AEAUGlobalAnimationHeaderAIM@@HI@Z 0000000031629370 f   GlobalAnimationHeaderAIM.obj
 0001:0012cb60       ?ProcessAimPoses@GlobalAnimationHeaderAIM@@QEAAXPEAVCSkel@@AEAU?$DynArray@UDirectionalBlends@@HU?$SmallDynStorage@UDirectionalBlends@@HUStandardAlloc@NAlloc@@@NArray@@@@AEAU?$DynArray@USJointsAimIK_Rot@@HU?$SmallDynStorage@USJointsAimIK_Rot@@HUStandardAlloc@NAlloc@@@NArray@@@@AEAU?$DynArray@USJointsAimIK_Pos@@HU?$SmallDynStorage@USJointsAimIK_Pos@@HUStandardAlloc@NAlloc@@@NArray@@@@@Z 000000003162db60 f   GlobalAnimationHeaderAIM.obj
 0001:0012ce70       ?ClearControllerData@GlobalAnimationHeaderCAF@@QEAAXXZ 000000003162de70 f   GlobalAnimationHeaderCAF.obj
 0001:0012cea0       ?FlagsSanityFilter@GlobalAnimationHeaderCAFStreamContent@@QEAAII@Z 000000003162dea0 f   GlobalAnimationHeaderCAF.obj
 0001:0012cee0       ??$fill@PEAUCryKeyPQLog@@U1@@stlpmtx_std@@YAXPEAUCryKeyPQLog@@0AEBU1@@Z 000000003162dee0 f i GlobalAnimationHeaderCAF.obj
 0001:0012cf50       ?DoesExistCAF@GlobalAnimationHeaderCAF@@QEAAIXZ 000000003162df50 f   GlobalAnimationHeaderCAF.obj
 0001:0012d030       ?GetTotalPosKeys@GlobalAnimationHeaderCAF@@QEBAIXZ 000000003162e030 f   GlobalAnimationHeaderCAF.obj
 0001:0012d0b0       ?GetTotalRotKeys@GlobalAnimationHeaderCAF@@QEBAIXZ 000000003162e0b0 f   GlobalAnimationHeaderCAF.obj
 0001:0012d130       ?ConnectCAFandDBA@GlobalAnimationHeaderCAF@@QEAAXXZ 000000003162e130 f   GlobalAnimationHeaderCAF.obj
 0001:0012d190       ?LoadDBA@GlobalAnimationHeaderCAF@@QEAAXXZ 000000003162e190 f   GlobalAnimationHeaderCAF.obj
 0001:0012d2c0       ?StreamOnNeedStorage@GlobalAnimationHeaderCAFStreamContent@@UEAAPEAXPEAVIReadStream@@I@Z 000000003162e2c0 f   GlobalAnimationHeaderCAF.obj
 0001:0012d380       ?ReadMotionParameters@GlobalAnimationHeaderCAFStreamContent@@QEAA_NPEAUChunkDesc@IChunkFile@@@Z 000000003162e380 f   GlobalAnimationHeaderCAF.obj
 0001:0012d530       ?CommitContent@GlobalAnimationHeaderCAF@@AEAAXAEAUGlobalAnimationHeaderCAFStreamContent@@@Z 000000003162e530 f   GlobalAnimationHeaderCAF.obj
 0001:0012d620       ??$__uninitialized_fill_n@PEAUCryKeyPQLog@@_KU1@@priv@stlpmtx_std@@YAPEAUCryKeyPQLog@@PEAU2@_KAEBU2@@Z 000000003162e620 f i GlobalAnimationHeaderCAF.obj
 0001:0012d6d0       ?SizeOfCAF@GlobalAnimationHeaderCAF@@QEBA_K_N@Z 000000003162e6d0 f   GlobalAnimationHeaderCAF.obj
 0001:0012d870       ?GetMemoryUsage@GlobalAnimationHeaderCAF@@QEBAXPEAVICrySizer@@@Z 000000003162e870 f   GlobalAnimationHeaderCAF.obj
 0001:0012d930       ?_M_fill_insert_aux@?$_Impl_vector@UCryKeyPQLog@@V?$allocator@UCryKeyPQLog@@@stlpmtx_std@@@priv@stlpmtx_std@@AEAAXPEAUCryKeyPQLog@@_KAEBU4@AEBU__false_type@3@@Z 000000003162e930 f i GlobalAnimationHeaderCAF.obj
 0001:0012dac0       ?erase@?$DynArray@U?$QuatT_tpl@M@@HU?$SmallDynStorage@U?$QuatT_tpl@M@@HUStandardAlloc@NAlloc@@@NArray@@@@QEAAPEAU?$QuatT_tpl@M@@PEAU2@0@Z 000000003162eac0 f i GlobalAnimationHeaderCAF.obj
 0001:0012dc90       ?ClearControllers@GlobalAnimationHeaderCAF@@QEAAXXZ 000000003162ec90 f   GlobalAnimationHeaderCAF.obj
 0001:0012dd60       ??4?$DynArray@U?$QuatT_tpl@M@@HU?$SmallDynStorage@U?$QuatT_tpl@M@@HUStandardAlloc@NAlloc@@@NArray@@@@QEAAAEAU0@U?$Array@$$CBU?$QuatT_tpl@M@@HU?$ArrayStorage@$$CBU?$QuatT_tpl@M@@H@NArray@@@@@Z 000000003162ed60 f i GlobalAnimationHeaderCAF.obj
 0001:0012dee0       ?SaveHTR@GlobalAnimationHeaderCAF@@SA_NPEBD0AEBV?$vector@V?$CryStringT@D@@V?$allocator@V?$CryStringT@D@@@stlpmtx_std@@@stlpmtx_std@@1AEBV?$vector@U?$DynArray@U?$QuatT_tpl@M@@HU?$SmallDynStorage@U?$QuatT_tpl@M@@HUStandardAlloc@NAlloc@@@NArray@@@@V?$allocator@U?$DynArray@U?$QuatT_tpl@M@@HU?$SmallDynStorage@U?$QuatT_tpl@M@@HUStandardAlloc@NAlloc@@@NArray@@@@@stlpmtx_std@@@3@PEBU?$QuatT_tpl@M@@@Z 000000003162eee0 f   GlobalAnimationHeaderCAF.obj
 0001:0012edd0       ??0GlobalAnimationHeaderCAFStreamContent@@QEAA@XZ 000000003162fdd0 f   GlobalAnimationHeaderCAF.obj
 0001:0012ee50       ??_EGlobalAnimationHeaderCAFStreamContent@@UEAAPEAXI@Z 000000003162fe50 f i GlobalAnimationHeaderCAF.obj
 0001:0012ee50       ??_GGlobalAnimationHeaderCAFStreamContent@@UEAAPEAXI@Z 000000003162fe50 f i GlobalAnimationHeaderCAF.obj
 0001:0012eec0       ?ParseChunkHeaders@GlobalAnimationHeaderCAFStreamContent@@QEAAIPEAUIChunkFile@@AEA_N1AEA_K@Z 000000003162fec0 f   GlobalAnimationHeaderCAF.obj
 0001:0012f340       ?ReadController@GlobalAnimationHeaderCAFStreamContent@@QEAA_NPEAUChunkDesc@IChunkFile@@_NAEAPEADAEAPEAVIControllerRelocatableChain@@@Z 0000000031630340 f   GlobalAnimationHeaderCAF.obj
 0001:001300a0       ??0?$DynArray@U?$QuatT_tpl@M@@HU?$SmallDynStorage@U?$QuatT_tpl@M@@HUStandardAlloc@NAlloc@@@NArray@@@@QEAA@AEBU0@@Z 00000000316310a0 f i GlobalAnimationHeaderCAF.obj
 0001:001301a0       ??$fill@PEAU?$DynArray@U?$QuatT_tpl@M@@HU?$SmallDynStorage@U?$QuatT_tpl@M@@HUStandardAlloc@NAlloc@@@NArray@@@@U1@@stlpmtx_std@@YAXPEAU?$DynArray@U?$QuatT_tpl@M@@HU?$SmallDynStorage@U?$QuatT_tpl@M@@HUStandardAlloc@NAlloc@@@NArray@@@@0AEBU1@@Z 00000000316311a0 f i GlobalAnimationHeaderCAF.obj
 0001:00130220       ??$__destroy_range_aux@V?$reverse_iterator@PEAU?$DynArray@U?$QuatT_tpl@M@@HU?$SmallDynStorage@U?$QuatT_tpl@M@@HUStandardAlloc@NAlloc@@@NArray@@@@@stlpmtx_std@@U?$DynArray@U?$QuatT_tpl@M@@HU?$SmallDynStorage@U?$QuatT_tpl@M@@HUStandardAlloc@NAlloc@@@NArray@@@@@stlpmtx_std@@YAXV?$reverse_iterator@PEAU?$DynArray@U?$QuatT_tpl@M@@HU?$SmallDynStorage@U?$QuatT_tpl@M@@HUStandardAlloc@NAlloc@@@NArray@@@@@0@0PEAU?$DynArray@U?$QuatT_tpl@M@@HU?$SmallDynStorage@U?$QuatT_tpl@M@@HUStandardAlloc@NAlloc@@@NArray@@@@AEBU__false_type@0@@Z 0000000031631220 f i GlobalAnimationHeaderCAF.obj
 0001:00130310       ??$__destroy_range_aux@PEAU?$DynArray@U?$QuatT_tpl@M@@HU?$SmallDynStorage@U?$QuatT_tpl@M@@HUStandardAlloc@NAlloc@@@NArray@@@@U1@@stlpmtx_std@@YAXPEAU?$DynArray@U?$QuatT_tpl@M@@HU?$SmallDynStorage@U?$QuatT_tpl@M@@HUStandardAlloc@NAlloc@@@NArray@@@@00AEBU__false_type@0@@Z 0000000031631310 f i GlobalAnimationHeaderCAF.obj
 0001:001303f0       ?ParseChunkRange@GlobalAnimationHeaderCAFStreamContent@@QEAA_NPEAUIChunkFile@@II_NAEAPEADAEAPEAVIControllerRelocatableChain@@@Z 00000000316313f0 f   GlobalAnimationHeaderCAF.obj
 0001:00130540       ?StreamAsyncOnComplete@GlobalAnimationHeaderCAFStreamContent@@UEAAXPEAVIReadStream@@I@Z 0000000031631540 f   GlobalAnimationHeaderCAF.obj
 0001:00130770       ?SaveCAF@GlobalAnimationHeaderCAF@@SA_NPEBD0AEBV?$vector@V?$CryStringT@D@@V?$allocator@V?$CryStringT@D@@@stlpmtx_std@@@stlpmtx_std@@AEBV?$vector@U?$DynArray@U?$QuatT_tpl@M@@HU?$SmallDynStorage@U?$QuatT_tpl@M@@HUStandardAlloc@NAlloc@@@NArray@@@@V?$allocator@U?$DynArray@U?$QuatT_tpl@M@@HU?$SmallDynStorage@U?$QuatT_tpl@M@@HUStandardAlloc@NAlloc@@@NArray@@@@@stlpmtx_std@@@3@@Z 0000000031631770 f   GlobalAnimationHeaderCAF.obj
 0001:00131390       ?_M_erase@?$_Impl_vector@U?$DynArray@U?$QuatT_tpl@M@@HU?$SmallDynStorage@U?$QuatT_tpl@M@@HUStandardAlloc@NAlloc@@@NArray@@@@V?$allocator@U?$DynArray@U?$QuatT_tpl@M@@HU?$SmallDynStorage@U?$QuatT_tpl@M@@HUStandardAlloc@NAlloc@@@NArray@@@@@stlpmtx_std@@@priv@stlpmtx_std@@AEAAPEAU?$DynArray@U?$QuatT_tpl@M@@HU?$SmallDynStorage@U?$QuatT_tpl@M@@HUStandardAlloc@NAlloc@@@NArray@@@@PEAU4@0AEBU__false_type@3@@Z 0000000031632390 f i GlobalAnimationHeaderCAF.obj
 0001:00131450       ??$__uninitialized_fill_n@PEAU?$DynArray@U?$QuatT_tpl@M@@HU?$SmallDynStorage@U?$QuatT_tpl@M@@HUStandardAlloc@NAlloc@@@NArray@@@@_KU1@@priv@stlpmtx_std@@YAPEAU?$DynArray@U?$QuatT_tpl@M@@HU?$SmallDynStorage@U?$QuatT_tpl@M@@HUStandardAlloc@NAlloc@@@NArray@@@@PEAU2@_KAEBU2@@Z 0000000031632450 f i GlobalAnimationHeaderCAF.obj
 0001:001314c0       ?StartStreamingCAF@GlobalAnimationHeaderCAF@@QEAAXXZ 00000000316324c0 f   GlobalAnimationHeaderCAF.obj
 0001:00131900       ?ControllerInit@GlobalAnimationHeaderCAF@@QEAAXXZ 0000000031632900 f   GlobalAnimationHeaderCAF.obj
 0001:001319e0       ?_M_fill_insert_aux@?$_Impl_vector@U?$DynArray@U?$QuatT_tpl@M@@HU?$SmallDynStorage@U?$QuatT_tpl@M@@HUStandardAlloc@NAlloc@@@NArray@@@@V?$allocator@U?$DynArray@U?$QuatT_tpl@M@@HU?$SmallDynStorage@U?$QuatT_tpl@M@@HUStandardAlloc@NAlloc@@@NArray@@@@@stlpmtx_std@@@priv@stlpmtx_std@@AEAAXPEAU?$DynArray@U?$QuatT_tpl@M@@HU?$SmallDynStorage@U?$QuatT_tpl@M@@HUStandardAlloc@NAlloc@@@NArray@@@@_KAEBU4@AEBU__false_type@3@@Z 00000000316329e0 f i GlobalAnimationHeaderCAF.obj
 0001:00131c40       ?LoadCAF@GlobalAnimationHeaderCAF@@QEAAIXZ 0000000031632c40 f   GlobalAnimationHeaderCAF.obj
 0001:00132040       ?LoadControllersCAF@GlobalAnimationHeaderCAF@@QEAAXXZ 0000000031633040 f   GlobalAnimationHeaderCAF.obj
 0001:00132060       ?FinishLoading@GlobalAnimationHeaderCAF@@AEAAXI@Z 0000000031633060 f   GlobalAnimationHeaderCAF.obj
 0001:00132170       ?_M_insert_overflow_aux@?$_Impl_vector@U?$DynArray@U?$QuatT_tpl@M@@HU?$SmallDynStorage@U?$QuatT_tpl@M@@HUStandardAlloc@NAlloc@@@NArray@@@@V?$allocator@U?$DynArray@U?$QuatT_tpl@M@@HU?$SmallDynStorage@U?$QuatT_tpl@M@@HUStandardAlloc@NAlloc@@@NArray@@@@@stlpmtx_std@@@priv@stlpmtx_std@@AEAAXPEAU?$DynArray@U?$QuatT_tpl@M@@HU?$SmallDynStorage@U?$QuatT_tpl@M@@HUStandardAlloc@NAlloc@@@NArray@@@@AEBU4@AEBU__false_type@3@_K_N@Z 0000000031633170 f i GlobalAnimationHeaderCAF.obj
 0001:00132370       ?StreamOnComplete@GlobalAnimationHeaderCAFStreamContent@@UEAAXPEAVIReadStream@@I@Z 0000000031633370 f   GlobalAnimationHeaderCAF.obj
 0001:00132570       ?Export2HTR@GlobalAnimationHeaderCAF@@QEAA_NPEBD0PEBVCSkel@@@Z 0000000031633570 f   GlobalAnimationHeaderCAF.obj
 0001:001332e0       ?ExportVGrid@GlobalAnimationHeaderLMG@@QEAA_NPEBD0PEBVCSkel@@PEAVCSkeletonAnim@@@Z 00000000316342e0 f   GlobalAnimationHeaderLMG.obj
 0001:001334e0       ?Init_TravelDist@GlobalAnimationHeaderLMG@@QEAAXPEBVCAnimationSet@@I@Z 00000000316344e0 f   GlobalAnimationHeaderLMG.obj
 0001:00133750       ?reserve@?$DynArray@UBSBlendable@@HU?$SmallDynStorage@UBSBlendable@@HUStandardAlloc@NAlloc@@@NArray@@@@QEAAXH@Z 0000000031634750 f i GlobalAnimationHeaderLMG.obj
 0001:001337b0       ?clear@?$DynArray@UBSBlendable@@HU?$SmallDynStorage@UBSBlendable@@HUStandardAlloc@NAlloc@@@NArray@@@@QEAAXXZ 00000000316347b0 f i GlobalAnimationHeaderLMG.obj
 0001:00133890       ?clear@?$DynArray@UVirtualExample1D@@HU?$SmallDynStorage@UVirtualExample1D@@HUStandardAlloc@NAlloc@@@NArray@@@@QEAAXXZ 0000000031634890 f i GlobalAnimationHeaderLMG.obj
 0001:00133970       ?clear@?$DynArray@UVirtualExample2D@@HU?$SmallDynStorage@UVirtualExample2D@@HUStandardAlloc@NAlloc@@@NArray@@@@QEAAXXZ 0000000031634970 f i GlobalAnimationHeaderLMG.obj
 0001:00133a50       ?clear@?$DynArray@UVirtualExample3D@@HU?$SmallDynStorage@UVirtualExample3D@@HUStandardAlloc@NAlloc@@@NArray@@@@QEAAXXZ 0000000031634a50 f i GlobalAnimationHeaderLMG.obj
 0001:00133b30       ?pop_back@?$DynArray@UBSParameter@@HU?$SmallDynStorage@UBSParameter@@HUStandardAlloc@NAlloc@@@NArray@@@@QEAAXH@Z 0000000031634b30 f i GlobalAnimationHeaderLMG.obj
 0001:00133be0       ?pop_back@?$DynArray@UBlendSpaceInfo@@HU?$SmallDynStorage@UBlendSpaceInfo@@HUStandardAlloc@NAlloc@@@NArray@@@@QEAAXH@Z 0000000031634be0 f i GlobalAnimationHeaderLMG.obj
 0001:00133c90       ?Init_MoveSpeed@GlobalAnimationHeaderLMG@@QEAAXPEBVCAnimationSet@@I@Z 0000000031634c90 f   GlobalAnimationHeaderLMG.obj
 0001:001342e0       ?Init_TurnSpeed@GlobalAnimationHeaderLMG@@QEAAXPEBVCAnimationSet@@I@Z 00000000316352e0 f   GlobalAnimationHeaderLMG.obj
 0001:00134a10       ?Init_TurnAngle@GlobalAnimationHeaderLMG@@QEAAXPEBVCAnimationSet@@I@Z 0000000031635a10 f   GlobalAnimationHeaderLMG.obj
 0001:00134f30       ?Init_TravelAngle@GlobalAnimationHeaderLMG@@QEAAXPEBVCAnimationSet@@I@Z 0000000031635f30 f   GlobalAnimationHeaderLMG.obj
 0001:00135720       ?Init_SlopeAngle@GlobalAnimationHeaderLMG@@QEAAXPEBVCAnimationSet@@I@Z 0000000031636720 f   GlobalAnimationHeaderLMG.obj
 0001:00135f20       ?clear@?$DynArray@UBSParameter@@HU?$SmallDynStorage@UBSParameter@@HUStandardAlloc@NAlloc@@@NArray@@@@QEAAXXZ 0000000031636f20 f i GlobalAnimationHeaderLMG.obj
 0001:00136000       ?clear@?$DynArray@UBlendSpaceInfo@@HU?$SmallDynStorage@UBlendSpaceInfo@@HUStandardAlloc@NAlloc@@@NArray@@@@QEAAXXZ 0000000031637000 f i GlobalAnimationHeaderLMG.obj
 0001:001360e0       ?init@?$DynArray@UBlendSpaceInfo@@HU?$SmallDynStorage@UBlendSpaceInfo@@HUStandardAlloc@NAlloc@@@NArray@@@@KAPEAUBlendSpaceInfo@@U?$Array@UBlendSpaceInfo@@HU?$ArrayStorage@UBlendSpaceInfo@@H@NArray@@@@@Z 00000000316370e0 f i GlobalAnimationHeaderLMG.obj
 0001:001361d0       ?ParameterExtraction@GlobalAnimationHeaderLMG@@QEAAXPEBVCAnimationSet@@II@Z 00000000316371d0 f   GlobalAnimationHeaderLMG.obj
 0001:00136240       ?resize@?$DynArray@USCRCName@@HU?$SmallDynStorage@USCRCName@@HUStandardAlloc@NAlloc@@@NArray@@@@QEAAXH@Z 0000000031637240 f i GlobalAnimationHeaderLMG.obj
 0001:001362b0       ?grow@?$DynArray@UBSParameter@@HU?$SmallDynStorage@UBSParameter@@HUStandardAlloc@NAlloc@@@NArray@@@@QEAAPEAUBSParameter@@H@Z 00000000316372b0 f i GlobalAnimationHeaderLMG.obj
 0001:00136330       ?LoadAndParseXML@GlobalAnimationHeaderLMG@@QEAA_NPEAVCAnimationSet@@_N@Z 0000000031637330 f   GlobalAnimationHeaderLMG.obj
 0001:00139080       ?CreateInternalType_Para1D@GlobalAnimationHeaderLMG@@QEAAXXZ 000000003163a080 f   GlobalAnimationHeaderLMG.obj
 0001:001393d0       ?Export2HTR@GlobalAnimationHeaderLMG@@QEAA_NPEBD0PEBVCSkel@@PEAVCSkeletonAnim@@@Z 000000003163a3d0 f   GlobalAnimationHeaderLMG.obj
 0001:0013b030       ??0CryLock_CritSection@@QEAA@XZ 000000003163c030 f   AnimationBase.obj
 0001:0013b050       ??1CryLock_CritSection@@QEAA@XZ 000000003163c050 f   AnimationBase.obj
 0001:0013b060       ?Lock@CryLock_CritSection@@QEAAXXZ 000000003163c060 f   AnimationBase.obj
 0001:0013b070       ?Unlock@CryLock_CritSection@@QEAAXXZ 000000003163c070 f   AnimationBase.obj
 0001:0013b080       ?cry_rand32@@YAIXZ         000000003163c080 f   AnimationBase.obj
 0001:0013b0a0       ?cry_rand@@YAIXZ           000000003163c0a0 f   AnimationBase.obj
 0001:0013b0d0       ?cry_frand@@YAMXZ          000000003163c0d0 f   AnimationBase.obj
 0001:0013b110       ?Init@_CryMemoryManagerPoolHelper@@SAXXZ 000000003163c110 f i AnimationBase.obj
 0001:0013b310       ?CryGetIMemoryManager@@YAPEAUIMemoryManager@@XZ 000000003163c310 f   AnimationBase.obj
 0001:0013b360       ?CrySleep@@YAXI@Z          000000003163c360 f   AnimationBase.obj
 0001:0013b370       ?CryInterlockedIncrement@@YAJPECH@Z 000000003163c370 f   AnimationBase.obj
 0001:0013b380       ?CryInterlockedDecrement@@YAJPECH@Z 000000003163c380 f   AnimationBase.obj
 0001:0013b390       ?CryInterlockedCompareExchangePointer@@YAPEAXPECREAXPEAX1@Z 000000003163c390 f   AnimationBase.obj
 0001:0013b3a0       ?CryCreateCriticalSectionInplace@@YAXPEAX@Z 000000003163c3a0 f   AnimationBase.obj
 0001:0013b3b0       ?CryGetCurrentThreadId@@YAIXZ 000000003163c3b0 f   AnimationBase.obj
 0001:0013b3c0       ?CryQueryPerformanceCounter@@YA_JXZ 000000003163c3c0 f   AnimationBase.obj
 0001:0013b3d0       ?CryPureCallHandler@@YAXXZ 000000003163c3d0 f   AnimationBase.obj
 0001:0013b3e0       ?CryInvalidParameterHandler@@YAXPEB_W00I_K@Z 000000003163c3e0 f   AnimationBase.obj
 0001:0013b3f0       ModuleInitISystem          000000003163c3f0 f   AnimationBase.obj
 0001:0013b4c0       CryGetMemoryInfoForModule  000000003163c4c0 f   AnimationBase.obj
 0001:0013b4c0       CryModuleGetMemoryInfo     000000003163c4c0 f   AnimationBase.obj
 0001:0013b500       ?CryDeleteCriticalSectionInplace@@YAXPEAX@Z 000000003163c500 f   AnimationBase.obj
 0001:0013b530       CryModuleMalloc            000000003163c530 f   AnimationBase.obj
 0001:0013b5d0       CryModuleRealloc           000000003163c5d0 f   AnimationBase.obj
 0001:0013b690       CryModuleFree              000000003163c690 f   AnimationBase.obj
 0001:0013b700       CryModuleMemalign          000000003163c700 f   AnimationBase.obj
 0001:0013b7b0       CryModuleMemalignFree      000000003163c7b0 f   AnimationBase.obj
 0001:0013b820       ??2@YAPEAX_K@Z             000000003163c820 f   AnimationBase.obj
 0001:0013b890       ??_U@YAPEAX_K@Z            000000003163c890 f   AnimationBase.obj
 0001:0013b900       ??3@YAXPEAX@Z              000000003163c900 f   AnimationBase.obj
 0001:0013b9a0       ??_V@YAXPEAX@Z             000000003163c9a0 f   AnimationBase.obj
 0001:0013ba40       ?OnSystemEvent@CSystemEventListner_Animation@@UEAAXW4ESystemEvent@@_K1@Z 000000003163ca40 f i AnimationBase.obj
 0001:0013bc50       ??_EISystemEventListener@@UEAAPEAXI@Z 000000003163cc50 f i AnimationBase.obj
 0001:0013bc50       ??_GJoystickSerializeContext@?4??BindJoystickSetToSequence@CFacialAnimation@@UEAAXPEAVIJoystickSet@@PEAUIFacialAnimSequence@@@Z@UEAAPEAXI@Z 000000003163cc50 f i FaceAnimation.obj
 0001:0013bc50       ??_GIFacialJoystickSerializeContext@@UEAAPEAXI@Z 000000003163cc50 f i FaceAnimation.obj
 0001:0013bc50       ??_GISystemEventListener@@UEAAPEAXI@Z 000000003163cc50 f i AnimationBase.obj
 0001:0013bc50       ??_GCSystemEventListner_Animation@@UEAAPEAXI@Z 000000003163cc50 f i AnimationBase.obj
 0001:0013bc50       ??_EJoystickSerializeContext@?4??BindJoystickSetToSequence@CFacialAnimation@@UEAAXPEAVIJoystickSet@@PEAUIFacialAnimSequence@@@Z@UEAAPEAXI@Z 000000003163cc50 f i FaceAnimation.obj
 0001:0013bc50       ??_ECSystemEventListner_Animation@@UEAAPEAXI@Z 000000003163cc50 f i AnimationBase.obj
 0001:0013bc50       ??_EIFacialJoystickSerializeContext@@UEAAPEAXI@Z 000000003163cc50 f i FaceAnimation.obj
 0001:0013bc80       ?GetFactory@CEngineModule_CryAnimation@@UEBAPEAUICryFactory@@XZ 000000003163cc80 f i AnimationBase.obj
 0001:0013bc90       ?GetName@CEngineModule_CryAnimation@@MEAAPEBDXZ 000000003163cc90 f i AnimationBase.obj
 0001:0013bca0       ?GetCategory@CEngineModule_CryAnimation@@MEAAPEBDXZ 000000003163cca0 f i AnimationBase.obj
 0001:0013bcb0       ?Initialize@CEngineModule_CryAnimation@@MEAA_NAEAUSSystemGlobalEnvironment@@AEBUSSystemInitParams@@@Z 000000003163ccb0 f i AnimationBase.obj
 0001:0013be50       ??_GCPoseMatching@@MEAAPEAXI@Z 000000003163ce50 f i PoseMatching.obj
 0001:0013be50       ??_GCLimbIk@@MEAAPEAXI@Z   000000003163ce50 f i LimbIk.obj
 0001:0013be50       ??_ECRecoil@PoseModifier@@MEAAPEAXI@Z 000000003163ce50 f i Recoil.obj
 0001:0013be50       ??_ECPoseBlenderAim@@MEAAPEAXI@Z 000000003163ce50 f i PoseBlenderAim.obj
 0001:0013be50       ??_ECPoseMatching@@MEAAPEAXI@Z 000000003163ce50 f i PoseMatching.obj
 0001:0013be50       ??_GCPoseBlenderAim@@MEAAPEAXI@Z 000000003163ce50 f i PoseBlenderAim.obj
 0001:0013be50       ??_GCRecoil@PoseModifier@@MEAAPEAXI@Z 000000003163ce50 f i Recoil.obj
 0001:0013be50       ??_GCFeetPoseRestore@@MEAAPEAXI@Z 000000003163ce50 f i FeetLock.obj
 0001:0013be50       ??_GCEngineModule_CryAnimation@@MEAAPEAXI@Z 000000003163ce50 f i AnimationBase.obj
 0001:0013be50       ??_ECEngineModule_CryAnimation@@MEAAPEAXI@Z 000000003163ce50 f i AnimationBase.obj
 0001:0013be50       ??_ECLimbIk@@MEAAPEAXI@Z   000000003163ce50 f i LimbIk.obj
 0001:0013be50       ??_ECFeetPoseRestore@@MEAAPEAXI@Z 000000003163ce50 f i FeetLock.obj
 0001:0013be80       ??0CFactory@CEngineModule_CryAnimation@@AEAA@XZ 000000003163ce80 f i AnimationBase.obj
 0001:0013bf20       ?GetClassName@CFactory@CEngineModule_CryAnimation@@UEBAPEBDXZ 000000003163cf20 f i AnimationBase.obj
 0001:0013bf30       ?GetClassID@CFactory@CEngineModule_CryAnimation@@UEBAAEBUCryGUID@@XZ 000000003163cf30 f i AnimationBase.obj
 0001:0013bf40       ??_GCFactory@CEngineModule_CryAnimation@@UEAAPEAXI@Z 000000003163cf40 f i AnimationBase.obj
 0001:0013bf40       ??_ECFactory@CEngineModule_CryAnimation@@UEAAPEAXI@Z 000000003163cf40 f i AnimationBase.obj
 0001:0013bf80       ??$?0VCEngineModule_CryAnimation@@@shared_count@detail@boost@@QEAA@PEAVCEngineModule_CryAnimation@@@Z 000000003163cf80 f i AnimationBase.obj
 0001:0013c090       ?QueryInterface@CEngineModule_CryAnimation@@MEBAPEAXAEBUCryGUID@@@Z 000000003163d090 f i AnimationBase.obj
 0001:0013c0e0       ?CreateClassInstance@CFactory@CEngineModule_CryAnimation@@UEBA?AV?$shared_ptr@UICryUnknown@@@boost@@XZ 000000003163d0e0 f i AnimationBase.obj
 0001:0013c1b0       ??0CAnimationThreadTask@@QEAA@XZ 000000003163d1b0 f   AnimationThreadTask.obj
 0001:0013c1d0       ??1CAnimationThreadTask@@UEAA@XZ 000000003163d1d0 f   AnimationThreadTask.obj
 0001:0013c1e0       ??_GCAnimationThreadTask@@UEAAPEAXI@Z 000000003163d1e0 f i AnimationThreadTask.obj
 0001:0013c1e0       ??_ECAnimationThreadTask@@UEAAPEAXI@Z 000000003163d1e0 f i AnimationThreadTask.obj
 0001:0013c210       ?Begin@CAnimationThreadTask@@QEAAXXZ 000000003163d210 f   AnimationThreadTask.obj
 0001:0013c240       ?DrawPose@Console@@QEAA_ND@Z 000000003163d240 f   cvars.obj
 0001:0013c3f0       ?Init@Console@@QEAAXXZ     000000003163d3f0 f   cvars.obj
 0001:0013e080       ?DeInitialize@?$Node_Alloc_Lock@$00$00@@SAXXZ 000000003163f080 f i stdafx.obj
 0001:0013e0f0       ??0CContext@Memory@@QEAA@XZ 000000003163f0f0 f   Memory.obj
 0001:0013e100       ?RemovePool@CContext@Memory@@QEAAXAEAVCPool@2@@Z 000000003163f100 f   Memory.obj
 0001:0013e150       ?Update@CAnimationContext@@QEAAXXZ 000000003163f150 f   Memory.obj
 0001:0013e180       ?AddPool@CContext@Memory@@QEAAXAEAVCPool@2@@Z 000000003163f180 f   Memory.obj
 0001:0013e1a0       ?GetMemoryUsage@CAnimationContext@@QEBAXPEAVICrySizer@@@Z 000000003163f1a0 f   Memory.obj
 0001:0013e200       ??_GCPool@Memory@@MEAAPEAXI@Z 000000003163f200 f i Pool.obj
 0001:0013e200       ??_ECPool@Memory@@MEAAPEAXI@Z 000000003163f200 f i Pool.obj
 0001:0013e240       ?Create@CBucket@CPoolFrameLocal@Memory@@SAPEAV123@I@Z 000000003163f240 f   Pool.obj
 0001:0013e2b0       ?Update@CPoolFrameLocal@Memory@@UEAAXXZ 000000003163f2b0 f   Pool.obj
 0001:0013e300       ??$AddObject@PEAVCBucket@CPoolFrameLocal@Memory@@V?$allocator@PEAVCBucket@CPoolFrameLocal@Memory@@@stlpmtx_std@@@ICrySizer@@QEAAXAEBV?$vector@PEAVCBucket@CPoolFrameLocal@Memory@@V?$allocator@PEAVCBucket@CPoolFrameLocal@Memory@@@stlpmtx_std@@@stlpmtx_std@@@Z 000000003163f300 f i Pool.obj
 0001:0013e390       ?GetMemoryUsage@CPoolFrameLocal@Memory@@UEBAXPEAVICrySizer@@@Z 000000003163f390 f   Pool.obj
 0001:0013e3d0       ??0CPoolFrameLocal@Memory@@AEAA@AEAVCContext@1@I@Z 000000003163f3d0 f   Pool.obj
 0001:0013e460       ?Create@CPoolFrameLocal@Memory@@SAPEAV12@AEAVCContext@2@I@Z 000000003163f460 f   Pool.obj
 0001:0013e4b0       ?CreateBucket@CPoolFrameLocal@Memory@@AEAAPEAVCBucket@12@XZ 000000003163f4b0 f   Pool.obj
 0001:0013e680       ?ReleaseBuckets@CPoolFrameLocal@Memory@@QEAAXXZ 000000003163f680 f   Pool.obj
 0001:0013e7a0       ?Allocate@CPoolFrameLocal@Memory@@UEAAPEAXI@Z 000000003163f7a0 f   Pool.obj
 0001:0013e880       ??_ECPoolFrameLocal@Memory@@EEAAPEAXI@Z 000000003163f880 f i Pool.obj
 0001:0013e880       ??_GCPoolFrameLocal@Memory@@EEAAPEAXI@Z 000000003163f880 f i Pool.obj
 0001:0013e900       ?SwSkinTangents@CAttachmentSKIN@@QEAAXPEAUSSkinningData@@PEAUSSoftwareSkinningData@@@Z 000000003163f900 f   _RenderSkinsSW.obj
 0001:0013f4a0       ?Invoke@?$SGenInvokerTSkinAttachmentTangents@VCAttachmentSKIN@@PEAUSSkinningData@@PEAUSSoftwareSkinningData@@USNullType@Detail@JobManager@@U456@U456@U456@U456@U456@U456@U456@U456@U456@@Detail@JobManager@@SAXPEAX@Z 00000000316404a0 f i _RenderSkinsSW.obj
 0001:0013f4b0       ?RegisterSoftwareSkinningJobs@CAttachmentSKIN@@SAXXZ 00000000316404b0 f   _RenderSkinsSW.obj
 0001:0013f500       ?InvokeSoftwareSkinning@CAttachmentSKIN@@SAXPEAUSSkinningData@@PEAUSSoftwareSkinningData@@@Z 0000000031640500 f   _RenderSkinsSW.obj
 0001:0013f606       _purecall                  0000000031640606 f   MSVCRT:MSVCR100.dll
 0001:0013f60c       _onexit                    000000003164060c f   MSVCRT:atonexit.obj
 0001:0013f6bc       atexit                     00000000316406bc f   MSVCRT:atonexit.obj
 0001:0013f6d4       cosf                       00000000316406d4 f   MSVCRT:MSVCR100.dll
 0001:0013f6da       sinf                       00000000316406da f   MSVCRT:MSVCR100.dll
 0001:0013f6e0       acosf                      00000000316406e0 f   MSVCRT:MSVCR100.dll
 0001:0013f700       __chkstk                   0000000031640700 f   MSVCRT:chkstk.obj
 0001:0013f700       _alloca_probe              0000000031640700     MSVCRT:chkstk.obj
 0001:0013f74e       memcpy                     000000003164074e f   MSVCRT:MSVCR100.dll
 0001:0013f754       memset                     0000000031640754 f   MSVCRT:MSVCR100.dll
 0001:0013f75a       sin                        000000003164075a f   MSVCRT:MSVCR100.dll
 0001:0013f760       cos                        0000000031640760 f   MSVCRT:MSVCR100.dll
 0001:0013f766       atan2                      0000000031640766 f   MSVCRT:MSVCR100.dll
 0001:0013f76c       atan2f                     000000003164076c f   MSVCRT:MSVCR100.dll
 0001:0013f772       ?what@exception@std@@UEBAPEBDXZ 0000000031640772 f   MSVCRT:MSVCR100.dll
 0001:0013f778       asinf                      0000000031640778 f   MSVCRT:MSVCR100.dll
 0001:0013f77e       powf                       000000003164077e f   MSVCRT:MSVCR100.dll
 0001:0013f784       fmodf                      0000000031640784 f   MSVCRT:MSVCR100.dll
 0001:0013f78a       expf                       000000003164078a f   MSVCRT:MSVCR100.dll
 0001:0013f790       acos                       0000000031640790 f   MSVCRT:MSVCR100.dll
 0001:0013f7f8       _CRT_INIT                  00000000316407f8 f   MSVCRT:crtdll.obj
 0001:0013fb90       _DllMainCRTStartup         0000000031640b90 f   MSVCRT:crtdll.obj
 0001:0013fbce       __C_specific_handler       0000000031640bce f   MSVCRT:MSVCR100.dll
 0001:0013fbd4       _unlock                    0000000031640bd4 f   MSVCRT:MSVCR100.dll
 0001:0013fbda       __dllonexit                0000000031640bda f   MSVCRT:MSVCR100.dll
 0001:0013fbe0       _lock                      0000000031640be0 f   MSVCRT:MSVCR100.dll
 0001:0013fbe8       __clean_type_info_names    0000000031640be8 f   MSVCRT:tncleanup.obj
 0001:0013fbf4       _RTC_Initialize            0000000031640bf4 f   MSVCRT:_initsect_.obj
 0001:0013fc2c       _RTC_Terminate             0000000031640c2c f   MSVCRT:_initsect_.obj
 0001:0013fc70       _ValidateImageBase         0000000031640c70 f   MSVCRT:pesect.obj
 0001:0013fca0       _FindPESection             0000000031640ca0 f   MSVCRT:pesect.obj
 0001:0013fcf0       _IsNonwritableInCurrentImage 0000000031640cf0 f   MSVCRT:pesect.obj
 0001:0013fd32       _initterm                  0000000031640d32 f   MSVCRT:MSVCR100.dll
 0001:0013fd38       _initterm_e                0000000031640d38 f   MSVCRT:MSVCR100.dll
 0001:0013fd3e       _amsg_exit                 0000000031640d3e f   MSVCRT:MSVCR100.dll
 0001:0013fd44       __CppXcptFilter            0000000031640d44 f   MSVCRT:MSVCR100.dll
 0001:0013fd4c       DllMain                    0000000031640d4c f   MSVCRT:dllmain.obj
 0001:0013fd70       __security_init_cookie     0000000031640d70 f   MSVCRT:gs_support.obj
 0001:0013fe24       __clean_type_info_names_internal 0000000031640e24 f   MSVCRT:MSVCR100.dll
 0001:00140450       ??__Fs_dummyMemReplay@?1??CryGetIMemReplay@@YAPEAUIMemReplay@@XZ@YAXXZ 0000000031641450 f i AnimEventList.obj
 0001:00140a20       ??__Fp@?1??CreateClassInstance@CFactory@CEngineModule_CryAnimation@@UEBA?AV?$shared_ptr@UICryUnknown@@@boost@@XZ@YAXXZ 0000000031641a20 f i AnimationBase.obj
 0002:00000000       __imp_InitializeCriticalSection 0000000031642000     kernel32:KERNEL32.dll
 0002:00000008       __imp_DeleteCriticalSection 0000000031642008     kernel32:KERNEL32.dll
 0002:00000010       __imp_EnterCriticalSection 0000000031642010     kernel32:KERNEL32.dll
 0002:00000018       __imp_LeaveCriticalSection 0000000031642018     kernel32:KERNEL32.dll
 0002:00000020       __imp_GetCurrentThreadId   0000000031642020     kernel32:KERNEL32.dll
 0002:00000028       __imp_LoadLibraryA         0000000031642028     kernel32:KERNEL32.dll
 0002:00000030       __imp_GetProcAddress       0000000031642030     kernel32:KERNEL32.dll
 0002:00000038       __imp_GetModuleHandleA     0000000031642038     kernel32:KERNEL32.dll
 0002:00000040       __imp_Sleep                0000000031642040     kernel32:KERNEL32.dll
 0002:00000048       __imp_GetCurrentProcessId  0000000031642048     kernel32:KERNEL32.dll
 0002:00000050       __imp_GetTickCount         0000000031642050     kernel32:KERNEL32.dll
 0002:00000058       __imp_QueryPerformanceCounter 0000000031642058     kernel32:KERNEL32.dll
 0002:00000060       __imp_DisableThreadLibraryCalls 0000000031642060     kernel32:KERNEL32.dll
 0002:00000068       __imp_DecodePointer        0000000031642068     kernel32:KERNEL32.dll
 0002:00000070       __imp_EncodePointer        0000000031642070     kernel32:KERNEL32.dll
 0002:00000078       __imp_GetSystemTimeAsFileTime 0000000031642078     kernel32:KERNEL32.dll
 0002:00000080       \177KERNEL32_NULL_THUNK_DATA 0000000031642080     kernel32:KERNEL32.dll
 0002:00000088       __imp_memcpy               0000000031642088     MSVCRT:MSVCR100.dll
 0002:00000090       __imp_memset               0000000031642090     MSVCRT:MSVCR100.dll
 0002:00000098       __imp_memmove              0000000031642098     MSVCRT:MSVCR100.dll
 0002:000000a0       __imp_abort                00000000316420a0     MSVCRT:MSVCR100.dll
 0002:000000a8       __imp_puts                 00000000316420a8     MSVCRT:MSVCR100.dll
 0002:000000b0       __imp_exit                 00000000316420b0     MSVCRT:MSVCR100.dll
 0002:000000b8       __imp_sin                  00000000316420b8     MSVCRT:MSVCR100.dll
 0002:000000c0       __imp_cos                  00000000316420c0     MSVCRT:MSVCR100.dll
 0002:000000c8       __imp_atan2                00000000316420c8     MSVCRT:MSVCR100.dll
 0002:000000d0       __imp_sprintf              00000000316420d0     MSVCRT:MSVCR100.dll
 0002:000000d8       __imp_strstr               00000000316420d8     MSVCRT:MSVCR100.dll
 0002:000000e0       __imp_fclose               00000000316420e0     MSVCRT:MSVCR100.dll
 0002:000000e8       __imp_fprintf              00000000316420e8     MSVCRT:MSVCR100.dll
 0002:000000f0       __imp_fopen                00000000316420f0     MSVCRT:MSVCR100.dll
 0002:000000f8       __imp_atan2f               00000000316420f8     MSVCRT:MSVCR100.dll
 0002:00000100       __imp_??0exception@std@@QEAA@AEBQEBDH@Z 0000000031642100     MSVCRT:MSVCR100.dll
 0002:00000108       __imp_acosf                0000000031642108     MSVCRT:MSVCR100.dll
 0002:00000110       __imp_??1exception@std@@UEAA@XZ 0000000031642110     MSVCRT:MSVCR100.dll
 0002:00000118       __imp_asinf                0000000031642118     MSVCRT:MSVCR100.dll
 0002:00000120       __imp_atof                 0000000031642120     MSVCRT:MSVCR100.dll
 0002:00000128       __imp_isdigit              0000000031642128     MSVCRT:MSVCR100.dll
 0002:00000130       __imp_strncmp              0000000031642130     MSVCRT:MSVCR100.dll
 0002:00000138       __imp_strchr               0000000031642138     MSVCRT:MSVCR100.dll
 0002:00000140       __imp_powf                 0000000031642140     MSVCRT:MSVCR100.dll
 0002:00000148       __imp_tolower              0000000031642148     MSVCRT:MSVCR100.dll
 0002:00000150       __imp__vscprintf           0000000031642150     MSVCRT:MSVCR100.dll
 0002:00000158       __imp__vsnprintf           0000000031642158     MSVCRT:MSVCR100.dll
 0002:00000158       __imp_vsnprintf            0000000031642158     MSVCRT:MSVCR100.dll
 0002:00000160       __imp_fmodf                0000000031642160     MSVCRT:MSVCR100.dll
 0002:00000168       __imp_strcspn              0000000031642168     MSVCRT:MSVCR100.dll
 0002:00000170       __imp_strspn               0000000031642170     MSVCRT:MSVCR100.dll
 0002:00000178       __imp_sscanf               0000000031642178     MSVCRT:MSVCR100.dll
 0002:00000180       __imp_expf                 0000000031642180     MSVCRT:MSVCR100.dll
 0002:00000188       __imp_strtod               0000000031642188     MSVCRT:MSVCR100.dll
 0002:00000190       __imp_strncpy              0000000031642190     MSVCRT:MSVCR100.dll
 0002:00000198       __imp_strtok               0000000031642198     MSVCRT:MSVCR100.dll
 0002:000001a0       __imp_fread                00000000316421a0     MSVCRT:MSVCR100.dll
 0002:000001a8       __imp_ftell                00000000316421a8     MSVCRT:MSVCR100.dll
 0002:000001b0       __imp_fseek                00000000316421b0     MSVCRT:MSVCR100.dll
 0002:000001b8       __imp_acos                 00000000316421b8     MSVCRT:MSVCR100.dll
 0002:000001c0       __imp_strrchr              00000000316421c0     MSVCRT:MSVCR100.dll
 0002:000001c8       __imp__set_invalid_parameter_handler 00000000316421c8     MSVCRT:MSVCR100.dll
 0002:000001d0       __imp__set_purecall_handler 00000000316421d0     MSVCRT:MSVCR100.dll
 0002:000001d8       __imp_atoi                 00000000316421d8     MSVCRT:MSVCR100.dll
 0002:000001e0       __imp___C_specific_handler 00000000316421e0     MSVCRT:MSVCR100.dll
 0002:000001e8       __imp__unlock              00000000316421e8     MSVCRT:MSVCR100.dll
 0002:000001f0       __imp___dllonexit          00000000316421f0     MSVCRT:MSVCR100.dll
 0002:000001f8       __imp__lock                00000000316421f8     MSVCRT:MSVCR100.dll
 0002:00000200       __imp__onexit              0000000031642200     MSVCRT:MSVCR100.dll
 0002:00000208       __imp__vsnprintf_s         0000000031642208     MSVCRT:MSVCR100.dll
 0002:00000208       __imp_vsnprintf_s          0000000031642208     MSVCRT:MSVCR100.dll
 0002:00000210       __imp__malloc_crt          0000000031642210     MSVCRT:MSVCR100.dll
 0002:00000218       __imp__initterm            0000000031642218     MSVCRT:MSVCR100.dll
 0002:00000220       __imp__initterm_e          0000000031642220     MSVCRT:MSVCR100.dll
 0002:00000228       __imp_free                 0000000031642228     MSVCRT:MSVCR100.dll
 0002:00000230       __imp__encoded_null        0000000031642230     MSVCRT:MSVCR100.dll
 0002:00000238       __imp__amsg_exit           0000000031642238     MSVCRT:MSVCR100.dll
 0002:00000240       __imp___CppXcptFilter      0000000031642240     MSVCRT:MSVCR100.dll
 0002:00000248       __imp___clean_type_info_names_internal 0000000031642248     MSVCRT:MSVCR100.dll
 0002:00000250       __imp_sinf                 0000000031642250     MSVCRT:MSVCR100.dll
 0002:00000258       __imp_cosf                 0000000031642258     MSVCRT:MSVCR100.dll
 0002:00000260       __imp__purecall            0000000031642260     MSVCRT:MSVCR100.dll
 0002:00000268       __imp_stricmp              0000000031642268     MSVCRT:MSVCR100.dll
 0002:00000268       __imp__stricmp             0000000031642268     MSVCRT:MSVCR100.dll
 0002:00000268       __imp_strcmpi              0000000031642268     MSVCRT:MSVCR100.dll
 0002:00000270       __imp__strnicmp            0000000031642270     MSVCRT:MSVCR100.dll
 0002:00000270       __imp_strnicmp             0000000031642270     MSVCRT:MSVCR100.dll
 0002:00000278       __imp_?what@exception@std@@UEBAPEBDXZ 0000000031642278     MSVCRT:MSVCR100.dll
 0002:00000280       \177MSVCR100_NULL_THUNK_DATA 0000000031642280     MSVCRT:MSVCR100.dll
 0002:00000288       __imp_MessageBoxA          0000000031642288     user32:USER32.dll
 0002:00000290       \177USER32_NULL_THUNK_DATA 0000000031642290     user32:USER32.dll
 0002:00000298       __xc_a                     0000000031642298     MSVCRT:cinitexe.obj
 0002:00000370       __xc_z                     0000000031642370     MSVCRT:cinitexe.obj
 0002:00000378       __xi_a                     0000000031642378     MSVCRT:cinitexe.obj
 0002:00000388       __xi_z                     0000000031642388     MSVCRT:cinitexe.obj
 0002:000003b0       ??_7IMemReplay@@6B@        00000000316423b0     AnimEventList.obj
 0002:000004e0       ??_7CDummyMemReplay@@6B@   00000000316424e0     AnimEventList.obj
 0002:00000610       ??_7CAnimEventList@@6B@    0000000031642610     AnimEventList.obj
 0002:00000650       __mask@@AbsFloat@          0000000031642650     Attachment.obj
 0002:00000660       __real@00000000            0000000031642660     Attachment.obj
 0002:00000664       __real@3f000000            0000000031642664     Attachment.obj
 0002:00000668       __real@3f800000            0000000031642668     Attachment.obj
 0002:0000066c       __real@bf800000            000000003164266c     Attachment.obj
 0002:00000670       __real@00800000            0000000031642670     Attachment.obj
 0002:00000674       __real@42652ee1            0000000031642674     Attachment.obj
 0002:00000678       __real@40000000            0000000031642678     Attachment.obj
 0002:0000067c       ??_C@_02DKCKIIND@?$CFs?$AA@ 000000003164267c     Attachment.obj
 0002:00000680       __real@46fffe00            0000000031642680     Attachment.obj
 0002:00000684       __real@38000100            0000000031642684     Attachment.obj
 0002:00000690       ??_7IAttachment@@6B@       0000000031642690     Attachment.obj
 0002:000007b0       ??_7IAttachmentSkin@@6B@   00000000316427b0     Attachment.obj
 0002:000007f0       __mask@@NegFloat@          00000000316427f0     Attachment.obj
 0002:00000800       ??_C@_0LJ@MJDPKDNI@AttachObjectToBone?5is?5called?5for@ 0000000031642800     Attachment.obj
 0002:000008bc       __real@1e3ce508            00000000316428bc     Attachment.obj
 0002:000008c0       __real@bf000000            00000000316428c0     Attachment.obj
 0002:000008c4       __real@3f4f5c28            00000000316428c4     Attachment.obj
 0002:000008c8       __real@38d1b717            00000000316428c8     Attachment.obj
 0002:000008d0       ??_C@_0P@OFCFADAK@HideInMainPass?$AA@ 00000000316428d0     Attachment.obj
 0002:000008e0       ??_C@_0BA@KIHOGAB@CAttachmentSKIN?$AA@ 00000000316428e0     Attachment.obj
 0002:000008f0       __real@3e4ccccd            00000000316428f0     Attachment.obj
 0002:000008f8       __real@3f1a36e2eb1c432d    00000000316428f8     Attachment.obj
 0002:00000900       __real@3c8efa35            0000000031642900     Attachment.obj
 0002:00000908       ??_C@_0CI@POBBGDGM@vertex?5stream?5declarations?5have?5@ 0000000031642908     Attachment.obj
 0002:00000930       ??_C@_09EDIHJNKH@Character?$AA@ 0000000031642930     Attachment.obj
 0002:00000940       ??_C@_0BG@KLDDMFMG@cloned?5for?5swskinning?$AA@ 0000000031642940     Attachment.obj
 0002:00000958       __real@41800000            0000000031642958     Attachment.obj
 0002:00000960       ??_C@_0BA@HAKOGMIL@SW?9Skinning?3?5?$CFs?$AA@ 0000000031642960     Attachment.obj
 0002:00000970       __real@3fa66666            0000000031642970     Attachment.obj
 0002:00000974       __real@3cf5c28f            0000000031642974     Attachment.obj
 0002:00000978       __real@3d23d70a            0000000031642978     Attachment.obj
 0002:0000097c       __real@3d4ccccd            000000003164297c     Attachment.obj
 0002:00000980       __real@40490fdb            0000000031642980     Attachment.obj
 0002:00000984       __real@3c23d70a            0000000031642984     Attachment.obj
 0002:00000988       __real@c0490fdb            0000000031642988     Attachment.obj
 0002:0000098c       __real@c11cf5c3            000000003164298c     Attachment.obj
 0002:00000990       __real@3ba3d70a            0000000031642990     Attachment.obj
 0002:00000994       __real@3ca3d70a            0000000031642994     Attachment.obj
 0002:00000998       __real@bcf5c28f            0000000031642998     Attachment.obj
 0002:0000099c       __real@bca3d70a            000000003164299c     Attachment.obj
 0002:000009a0       __real@3eaaaaab            00000000316429a0     Attachment.obj
 0002:000009b0       ??_7CAttachmentSKIN@@6BIAttachment@@@ 00000000316429b0     Attachment.obj
 0002:00000ad0       ??_7CAttachmentSKIN@@6BIAttachmentSkin@@@ 0000000031642ad0     Attachment.obj
 0002:00000b10       ??_C@_0BD@HKEJKAJE@?$CF03d?5JointName?3?5?$CFs?$AA@ 0000000031642b10     Attachment.obj
 0002:00000b28       ??_C@_0BK@BIGEPFME@SLAVE?5?5SKELETON?3?5path?3?5?$CFs?$AA@ 0000000031642b28     Attachment.obj
 0002:00000b48       ??_C@_0BK@CNDDAMJA@MASTER?5SKELETON?3?5path?3?5?$CFs?$AA@ 0000000031642b48     Attachment.obj
 0002:00000b70       ??_C@_0FB@JGGJBAML@Bone?9names?5of?5SLAVE?9skeleton?5don@ 0000000031642b70     Attachment.obj
 0002:00000bd0       ??_C@_0FB@OCMIBIFK@SLAVE?9skeleton?5needs?5to?5have?5les@ 0000000031642bd0     Attachment.obj
 0002:00000c30       ??_C@_0HF@NPAHMHBP@CryAnimation?3?5if?5you?5create?5the?5@ 0000000031642c30     Attachment.obj
 0002:00000ca8       ??_7IDefragAllocatorPolicy@@6B@ 0000000031642ca8     ControllerDefragHeap.obj
 0002:00000cd0       ??_C@_0P@PCJPAHLM@out?5of?5memory?6?$AA@ 0000000031642cd0     ControllerDefragHeap.obj
 0002:00000ce0       ??_C@_06NBFPPGEG@vector?$AA@ 0000000031642ce0     ControllerDefragHeap.obj
 0002:00000ce8       ??_7CControllerDefragHeap@@6B@ 0000000031642ce8     ControllerDefragHeap.obj
 0002:00000d10       ??_C@_00CNPNBAHC@?$AA@     0000000031642d10     ControllerDefragHeap.obj
 0002:00000d18       ??_C@_0BB@OMBAPGD@Anim?5Defrag?5Heap?$AA@ 0000000031642d18     ControllerDefragHeap.obj
 0002:00000d30       ??_C@_0BO@ECPGPOHM@CControllerDefragHeap?3?3Update?$AA@ 0000000031642d30     ControllerDefragHeap.obj
 0002:00000d50       __real@3ff0000000000000    0000000031642d50     DrawHelper.obj
 0002:00000d58       __real@3f666666            0000000031642d58     DrawHelper.obj
 0002:00000d5c       __real@3f400000            0000000031642d5c     DrawHelper.obj
 0002:00000d60       __real@4000000000000000    0000000031642d60     DrawHelper.obj
 0002:00000d70       __mask@@NegDouble@         0000000031642d70     DrawHelper.obj
 0002:00000d80       __real@3f7d70a4            0000000031642d80     DrawHelper.obj
 0002:00000d84       __real@3e19999a            0000000031642d84     DrawHelper.obj
 0002:00000d88       __real@3c1374bc            0000000031642d88     DrawHelper.obj
 0002:00000d90       __real@3f8eb851eb851eb8    0000000031642d90     DrawHelper.obj
 0002:00000d98       __real@3fe0000000000000    0000000031642d98     DrawHelper.obj
 0002:00000da0       __real@3f947ae147ae147b    0000000031642da0     DrawHelper.obj
 0002:00000da8       __real@3d99999a            0000000031642da8     DrawHelper.obj
 0002:00000dac       __real@3e800000            0000000031642dac     DrawHelper.obj
 0002:00000db8       ??_C@_0CI@IOKCCNHB@Deleting?5Reference?5Counted?5Objec@ 0000000031642db8     LoaderSKIN.obj
 0002:00000de0       __real@d8635fa9            0000000031642de0     LoaderSKIN.obj
 0002:00000de4       __real@58635fa9            0000000031642de4     LoaderSKIN.obj
 0002:00000df0       ??_C@_0EL@JEKIGBJA@Character?5LOD?5mismatch?4?5The?5bone@ 0000000031642df0     LoaderSKIN.obj
 0002:00000e40       ??_C@_0BD@GAJPFAIO@Hierarchy?5of?5LOD?$CFi?$AA@ 0000000031642e40     LoaderSKIN.obj
 0002:00000e60       ??_C@_0ED@EMLDLHGL@?9?9?9?9?9?9?9?9?9?9?9?9?9?9?9?9?9?9?9?9?9?9?9?9?9?9?9?9?9?9?9?9@ 0000000031642e60     LoaderSKIN.obj
 0002:00000ea8       ??_C@_0BD@JKBIHFBO@Joint?5ID?5?3?5?$CF02d?5?$CFs?$AA@ 0000000031642ea8     LoaderSKIN.obj
 0002:00000ec0       ??_C@_0BC@CMAFGEHH@Hierarchy?5of?5LOD0?$AA@ 0000000031642ec0     LoaderSKIN.obj
 0002:00000ee0       ??_C@_0EC@CDOMHHGC@Failed?5to?5Load?5Character?0?5Differ@ 0000000031642ee0     LoaderSKIN.obj
 0002:00000f24       __real@3dcccccd            0000000031642f24     LoaderSKIN.obj
 0002:00000f28       ??_C@_02GMHACPFF@?$CFu?$AA@ 0000000031642f28     LoaderSKIN.obj
 0002:00000f2c       ??_C@_04NHPAFEHJ@skin?$AA@ 0000000031642f2c     LoaderSKIN.obj
 0002:00000f34       ??_C@_01LFCBOECM@?4?$AA@   0000000031642f34     LoaderSKIN.obj
 0002:00000f38       ??_C@_04LAHEDKPN@_lod?$AA@ 0000000031642f38     LoaderSKIN.obj
 0002:00000f40       ??_C@_0EG@EBKKPPLH@Failed?5to?5Load?5Character?5file?4?5S@ 0000000031642f40     LoaderSKIN.obj
 0002:00000f88       ??_C@_0DB@FJJGDDBE@Failed?5to?5Load?5Character?5file?4?5G@ 0000000031642f88     LoaderSKIN.obj
 0002:00000fc0       ??_C@_0BM@PPPNKEGO@Invalid?5vertex?5?$CFd?5in?5lod?5?$CFd?$AA@ 0000000031642fc0     LoaderSKIN.obj
 0002:00000fe0       ??_7CMorphTarget@@6B@      0000000031642fe0     LoaderSKIN.obj
 0002:00000ff8       ??_C@_0CB@EIMOFNGE@arrExtMorph?$FL?$FN?5is?5empty?5in?5lod?5?$CFd@ 0000000031642ff8     LoaderSKIN.obj
 0002:00001020       ??_C@_0CF@ELPJCGJF@Vertex?5extension?5x?5is?5zero?5in?5lo@ 0000000031643020     LoaderSKIN.obj
 0002:00001048       ??_C@_0CF@COJOBNND@Vertex?5extension?5y?5is?5zero?5in?5lo@ 0000000031643048     LoaderSKIN.obj
 0002:00001070       ??_C@_0CF@IBDHFABJ@Vertex?5extension?5z?5is?5zero?5in?5lo@ 0000000031643070     LoaderSKIN.obj
 0002:00001098       ??_C@_0CB@NMCAMOME@Bound?5box?5is?5too?5small?5in?5lod?5?$CFd@ 0000000031643098     LoaderSKIN.obj
 0002:000010c0       ??_C@_0CE@KGCDEIAK@Vertex?5id?50x?$CFx?5is?5too?5big?5in?5lod@ 00000000316430c0     LoaderSKIN.obj
 0002:000010e4       __real@41700000            00000000316430e4     LoaderSKIN.obj
 0002:000010e8       __real@3a83126f            00000000316430e8     LoaderSKIN.obj
 0002:000010ec       __real@437f0000            00000000316430ec     LoaderSKIN.obj
 0002:000010f0       __real@c7c34f80            00000000316430f0     LoaderSKIN.obj
 0002:000010f4       __real@47c34f80            00000000316430f4     LoaderSKIN.obj
 0002:000010f8       ??_C@_0CN@IPOFNMHK@Bone?5?$CFd?3?5B2W?5is?5not?5orthonormal?5@ 00000000316430f8     LoaderSKIN.obj
 0002:00001128       ??_C@_0BF@JHCFNCDB@Model?5has?5no?5Joints?4?$AA@ 0000000031643128     LoaderSKIN.obj
 0002:00001140       ??_C@_0CP@JEJKDKLN@Too?5many?5Joints?5in?5model?4?5Curren@ 0000000031643140     LoaderSKIN.obj
 0002:00001170       ??_C@_0BP@OOOCOAFP@Duplicated?5morph?5mask?5found?5?$CFs?$AA@ 0000000031643170     LoaderSKIN.obj
 0002:00001190       ??_C@_0BO@KMGPEDAO@Base?5skinned?5model?5is?5missing?$AA@ 0000000031643190     LoaderSKIN.obj
 0002:000011b0       ??_C@_0CK@FPIIFKJK@The?5Chunk?9Loader?5failed?5to?5load?5@ 00000000316431b0     LoaderSKIN.obj
 0002:000011e0       ??_C@_0CD@BBJOEHHB@Skinning?5info?5is?5missing?5in?5lod?5@ 00000000316431e0     LoaderSKIN.obj
 0002:00001208       ??_C@_0BP@CMMDHOGJ@Ext2Int?5map?5is?5empty?5in?5lod?5?$CFd?$AA@ 0000000031643208     LoaderSKIN.obj
 0002:00001228       ??_C@_0BG@JBIGAFMF@No?5material?5in?5lod?5?$CFd?$AA@ 0000000031643228     LoaderSKIN.obj
 0002:00001240       ??_C@_0BM@JOPKNICB@No?5internal?5faces?5in?5lod?5?$CFd?$AA@ 0000000031643240     LoaderSKIN.obj
 0002:00001260       ??_C@_0CI@LFMLLEBF@Failed?5to?5create?5render?5mesh?5for@ 0000000031643260     LoaderSKIN.obj
 0002:00001290       ??_C@_0FF@BMNHAGLP@external?5and?5internal?5face?9amoun@ 0000000031643290     LoaderSKIN.obj
 0002:000012e8       ??_C@_0N@EGPCGIEE@e_CharLodMin?$AA@ 00000000316432e8     LoaderSKIN.obj
 0002:000012f8       ??_C@_0N@MAGOOHJD@e_charLodMin?$AA@ 00000000316432f8     LoaderSKIN.obj
 0002:00001308       ??_C@_0O@NMCPHDFF@consoles_lod0?$AA@ 0000000031643308     LoaderSKIN.obj
 0002:00001318       ??_C@_0BG@EFLJKDCI@ca_UseAssetDefinedLod?$AA@ 0000000031643318     LoaderSKIN.obj
 0002:00001330       ??_C@_0BJ@BIICHPJO@Wrong?5character?5filename?$AA@ 0000000031643330     LoaderSKIN.obj
 0002:0000134c       ??_C@_03KMOFPJOC@chr?$AA@  000000003164334c     LoaderSKIN.obj
 0002:00001350       ??_C@_0BB@CGHIGGGM@LoadCharacter?5?$CFs?$AA@ 0000000031643350     LoaderSKIN.obj
 0002:00001368       ??_C@_0BK@HNKMOAFK@CryCHRLoader?3?3LoadNewSKIN?$AA@ 0000000031643368     LoaderSKIN.obj
 0002:00001388       __real@3727c5ac            0000000031643388     ModelMesh_DebugPC.obj
 0002:00001388       ?minPosArea@?1???$ComputeTexMappingAreas@U?$Vec3_tpl@M@@USMeshTexCoord@@@CMeshHelpers@@SA_N_KPEBG0PEBU?$Vec3_tpl@M@@0PEBUSMeshTexCoord@@0AEAM4AEAPEBD@Z@4MB 0000000031643388     LoaderCGA.obj
 0002:0000138c       __real@47c35000            000000003164338c     ModelMesh_DebugPC.obj
 0002:00001390       ??_C@_02DPKJAMEF@?$CFd?$AA@ 0000000031643390     ModelMesh_DebugPC.obj
 0002:00001394       ??_C@_04GEFJINEE@?$CF?42f?$AA@ 0000000031643394     ModelMesh_DebugPC.obj
 0002:000013a0       ??_C@_08GDAMKODC@?$CFd?0?$CFd?0?$CFd?$AA@ 00000000316433a0     ModelMesh_DebugPC.obj
 0002:000013b0       ??_C@_0M@MLCONGPP@?$CFd?0?$CFd?0?$CFd?0?$CFd?$AA@ 00000000316433b0     ModelMesh_DebugPC.obj
 0002:000013bc       ??_C@_05LCKIIOJE@?$CFd?1?$CFd?$AA@ 00000000316433bc     ModelMesh_DebugPC.obj
 0002:000013c4       __real@42f00000            00000000316433c4     ModelMesh_DebugPC.obj
 0002:000013c8       __real@40c90fdb            00000000316433c8     ModelMesh_DebugPC.obj
 0002:000013d0       ??_C@_0BB@CDDPHBIK@?$CFs?6?$CFd?5LOD?$CI?$CFi?2?$CFi?$CJ?$AA@ 00000000316433d0     ModelMesh_DebugPC.obj
 0002:000013e4       ??_C@_02PCIJFNDE@?$AN?6?$AA@ 00000000316433e4     ModelMesh_DebugPC.obj
 0002:000013e8       ??_C@_03ELIABIOC@w?$CLb?$AA@ 00000000316433e8     ModelMesh_DebugPC.obj
 0002:000013ec       __real@3b808081            00000000316433ec     ModelMesh_DebugPC.obj
 0002:000013f0       ??_C@_0BD@KNEHJKOE@SoftwareSkinningDQ?$AA@ 00000000316433f0     ModelMesh_DebugPC.obj
 0002:00001408       ??_C@_0BP@KJMNBCEI@CModelMesh?3?3SoftwareSkinningDQ?$AA@ 0000000031643408     ModelMesh_DebugPC.obj
 0002:00001430       ??_7IFacialSentence@@6B@   0000000031643430     LipSync.obj
 0002:00001430       ??_7ISkin@@6B@             0000000031643430     ModelSkin.obj
 0002:00001498       ??_C@_0L@JGFNFNNF@CModelMesh?$AA@ 0000000031643498     ModelSkin.obj
 0002:000014b0       ??_7CSkin@@6B@             00000000316434b0     ModelSkin.obj
 0002:00001528       ??_C@_0BP@NOKONOFF@?$CBMORPH?5TARGET?5ID?5OUT?5OF?5RANGE?$CB?$AA@ 0000000031643528     ModelSkin.obj
 0002:00001548       ??_C@_0BC@LGKPNEPG@CSkin?5Release?3?5?$CFs?$AA@ 0000000031643548     ModelSkin.obj
 0002:00001560       ??_C@_0FJ@LKDGMGOG@The?5model?5?8?$CFs?8?5still?5has?5?$CFd?5skin@ 0000000031643560     ModelSkin.obj
 0002:000015c8       ??_C@_08IFJOJHOO@e_Clouds?$AA@ 00000000316435c8     ParametricSampler.obj
 0002:000015d8       ??_C@_07EFDJIHNI@e_Roads?$AA@ 00000000316435d8     ParametricSampler.obj
 0002:000015e0       ??_C@_0P@GLJFAGLA@e_WaterVolumes?$AA@ 00000000316435e0     ParametricSampler.obj
 0002:000015f0       ??_C@_0N@DNCIPFKM@e_WaterWaves?$AA@ 00000000316435f0     ParametricSampler.obj
 0002:00001600       ??_C@_08HDKOIENJ@e_Decals?$AA@ 0000000031643600     ParametricSampler.obj
 0002:00001610       ??_C@_0M@BBFEECFK@e_Particles?$AA@ 0000000031643610     ParametricSampler.obj
 0002:00001620       ??_C@_0N@BCKEBKIL@e_WaterOcean?$AA@ 0000000031643620     ParametricSampler.obj
 0002:00001630       ??_C@_09HEKIHBOB@e_Terrain?$AA@ 0000000031643630     ParametricSampler.obj
 0002:00001640       ??_C@_0L@JLCOCKLP@e_Entities?$AA@ 0000000031643640     ParametricSampler.obj
 0002:00001650       ??_C@_0N@IDHCJDNJ@e_Vegetation?$AA@ 0000000031643650     ParametricSampler.obj
 0002:00001660       ??_C@_09MHBOCIPH@e_Brushes?$AA@ 0000000031643660     ParametricSampler.obj
 0002:00001670       ??_C@_09HMFDJOHK@e_Shadows?$AA@ 0000000031643670     ParametricSampler.obj
 0002:00001680       ??_C@_08OEHLIOJG@e_VoxTer?$AA@ 0000000031643680     ParametricSampler.obj
 0002:00001690       ??_C@_07DPCBLJHC@e_Voxel?$AA@ 0000000031643690     ParametricSampler.obj
 0002:00001698       ??_C@_0BC@BEKKKHMP@e_DefaultMaterial?$AA@ 0000000031643698     ParametricSampler.obj
 0002:000016ac       __real@3f333333            00000000316436ac     ParametricSampler.obj
 0002:000016b0       __real@3f4ccccd            00000000316436b0     ParametricSampler.obj
 0002:000016b4       __real@3c888889            00000000316436b4     ParametricSampler.obj
 0002:000016b8       ??_C@_0P@IINHJLIF@e_CameraFreeze?$AA@ 00000000316436b8     ParametricSampler.obj
 0002:000016c8       __real@42200000            00000000316436c8     ParametricSampler.obj
 0002:000016d0       ??_C@_0BC@BOLHFEBM@Inside?5Block1?3?5?$CFd?$AA@ 00000000316436d0     ParametricSampler.obj
 0002:000016e4       __real@40800000            00000000316436e4     ParametricSampler.obj
 0002:000016e8       __real@40166666            00000000316436e8     ParametricSampler.obj
 0002:000016ec       __real@40600000            00000000316436ec     ParametricSampler.obj
 0002:000016f0       ??_C@_0P@ONCKKLGM@InternalPara1D?$AA@ 00000000316436f0     ParametricSampler.obj
 0002:00001700       ??_C@_0BE@PBKONPHH@Not?5an?5Internal?5LMG?$AA@ 0000000031643700     ParametricSampler.obj
 0002:00001714       __real@3fc00000            0000000031643714     ParametricSampler.obj
 0002:00001718       ??_C@_0DH@CPEAIGHN@CryAnimation?3?5more?5then?53?5dimens@ 0000000031643718     ParametricSampler.obj
 0002:00001750       __real@3d8f5c29            0000000031643750     ParametricSampler.obj
 0002:00001754       __real@41a00000            0000000031643754     ParametricSampler.obj
 0002:00001758       ??_C@_09HJKJEFNK@?$CFs?3?5?$CFf?5?$CFd?$AA@ 0000000031643758     ParametricSampler.obj
 0002:00001768       ??_C@_0BA@KLKAAMJI@invalid?5sum?3?5?$CFf?$AA@ 0000000031643768     ParametricSampler.obj
 0002:00001778       ??_C@_0BA@PJAEBMKK@Invalid?5Weights?$AA@ 0000000031643778     ParametricSampler.obj
 0002:00001788       __real@41f80000            0000000031643788     ParametricSampler.obj
 0002:0000178c       __real@40400000            000000003164378c     ParametricSampler.obj
 0002:00001790       ??_C@_0CG@CCCLNGHK@CryAnimation?3?5nParaID?5not?5initia@ 0000000031643790     ParametricSampler.obj
 0002:000017b8       __real@41a80000            00000000316437b8     ParametricSampler.obj
 0002:000017c0       ??_C@_07MIGDMPIL@mem?3?5?$CFd?$AA@ 00000000316437c0     ParametricSampler.obj
 0002:000017c8       __real@42c80000            00000000316437c8     ParametricSampler.obj
 0002:000017cc       __real@c2c80000            00000000316437cc     ParametricSampler.obj
 0002:000017d0       ??_C@_0BH@KPHNFGHL@CryAnimation?3?5negative?$AA@ 00000000316437d0     ParametricSampler.obj
 0002:000017e8       __real@41f00000            00000000316437e8     ParametricSampler.obj
 0002:000017ec       __real@3d088889            00000000316437ec     ParametricSampler.obj
 0002:000017f0       ??_C@_0BI@BNNPNGGM@Sum?5of?5weights?5is?5wrong?$AA@ 00000000316437f0     ParametricSampler.obj
 0002:00001808       __real@40a66666            0000000031643808     ParametricSampler.obj
 0002:0000180c       __real@c0a66666            000000003164380c     ParametricSampler.obj
 0002:00001810       ??_C@_0BH@KFJNBPEB@CryAnimation?3?5?$CFs?3?5?8?$CFs?8?$AA@ 0000000031643810     ParametricSampler.obj
 0002:00001828       ??_7CPlaceholderCharacter@@6B@ 0000000031643828     PlaceholderCharacter.obj
 0002:0000184c       __real@34000000            000000003164384c     DirectionalBlender.obj
 0002:00001850       __real@3e70a3d7            0000000031643850     DirectionalBlender.obj
 0002:00001854       __real@3ef5c28f            0000000031643854     DirectionalBlender.obj
 0002:00001858       __real@39000000            0000000031643858     DirectionalBlender.obj
 0002:0000185c       __real@4022f983            000000003164385c     DirectionalBlender.obj
 0002:00001860       __real@3fc90fdb            0000000031643860     DirectionalBlender.obj
 0002:00001864       __real@3e051eb8            0000000031643864     DirectionalBlender.obj
 0002:00001868       __real@3da3d70a            0000000031643868     DirectionalBlender.obj
 0002:0000186c       __real@3fb33333            000000003164386c     DirectionalBlender.obj
 0002:00001870       __real@bfb33333            0000000031643870     DirectionalBlender.obj
 0002:00001874       __real@41d00000            0000000031643874     DirectionalBlender.obj
 0002:00001878       __real@c0486c04            0000000031643878     DirectionalBlender.obj
 0002:0000187c       __real@40486c04            000000003164387c     DirectionalBlender.obj
 0002:00001880       __real@3fcccccd            0000000031643880     DirectionalBlender.obj
 0002:00001884       __real@bfc90fdb            0000000031643884     DirectionalBlender.obj
 0002:00001888       __real@3feff7ced916872b    0000000031643888     DirectionalBlender.obj
 0002:00001890       __real@3f8ccccd            0000000031643890     DirectionalBlender.obj
 0002:00001894       __real@3fc9309f            0000000031643894     DirectionalBlender.obj
 0002:00001898       __real@4049203d            0000000031643898     DirectionalBlender.obj
 0002:0000189c       __real@ba83126f            000000003164389c     DirectionalBlender.obj
 0002:000018a0       __real@3ec90fdb            00000000316438a0     DirectionalBlender.obj
 0002:000018a4       __real@41600000            00000000316438a4     DirectionalBlender.obj
 0002:000018a8       ??_C@_0BD@GFPCDKCE@fAimPoseWeight?3?5?$CFf?$AA@ 00000000316438a8     DirectionalBlender.obj
 0002:000018bc       __real@3f99999a            00000000316438bc     DirectionalBlender.obj
 0002:000018c0       __real@4019999a            00000000316438c0     DirectionalBlender.obj
 0002:000018c8       ??_C@_0BM@HHDJLNNF@final?5polar?3?5?$CFf?5?$CFf?5?5?5wR?3?5?$CFf?$AA@ 00000000316438c8     DirectionalBlender.obj
 0002:000018e4       __real@41200000            00000000316438e4     DirectionalBlender.obj
 0002:000018e8       ?iid@?1??IID@ICryUnknown@@CAAEBUCryGUID@@XZ@4U3@B 00000000316438e8     OperatorQueue.obj
 0002:000018f8       ?iid@?1??IID@IAnimationPoseModifier@@CAAEBUCryGUID@@XZ@4U3@B 00000000316438f8     OperatorQueue.obj
 0002:00001908       ?iid@?1??IID@IAnimationOperatorQueue@@CAAEBUCryGUID@@XZ@4U3@B 0000000031643908     OperatorQueue.obj
 0002:00001918       ??_7ICryFactory@@6B@       0000000031643918     OperatorQueue.obj
 0002:00001948       ??_7CFactory@COperatorQueue@@6B@ 0000000031643948     OperatorQueue.obj
 0002:00001978       ??_C@_0CE@INMPALAM@AnimationPoseModifier_OperatorQu@ 0000000031643978     OperatorQueue.obj
 0002:000019a0       ?cid@?1??GetClassID@CFactory@COperatorQueue@@UEBAAEBUCryGUID@@XZ@4U4@B 00000000316439a0     OperatorQueue.obj
 0002:000019b0       ??_7bad_alloc@std@@6B@     00000000316439b0     OperatorQueue.obj
 0002:000019c0       ??_C@_0P@GHFPNOJB@bad?5allocation?$AA@ 00000000316439c0     OperatorQueue.obj
 0002:000019d0       ??_7sp_counted_base@detail@boost@@6B@ 00000000316439d0     OperatorQueue.obj
 0002:000019f0       ??_C@_0BN@FOKPCDPC@Boost?5threw?5an?5exception?3?5?$CFs?$AA@ 00000000316439f0     OperatorQueue.obj
 0002:00001a10       ??_7COperatorQueue@@6B@    0000000031643a10     OperatorQueue.obj
 0002:00001a88       ?iid@?1??IID@IAnimationPoseAlignerChain@@CAAEBUCryGUID@@XZ@4U3@B 0000000031643a88     PoseAlignerChain.obj
 0002:00001a98       __real@322bcc77            0000000031643a98     PoseAlignerChain.obj
 0002:00001a9c       __real@3f19999a            0000000031643a9c     PoseAlignerChain.obj
 0002:00001aa0       __real@3fd9999a            0000000031643aa0     PoseAlignerChain.obj
 0002:00001ab0       ??_7CPoseAlignerChain@@6B@ 0000000031643ab0     PoseAlignerChain.obj
 0002:00001b00       __real@3e000000            0000000031643b00     PoseAlignerChain.obj
 0002:00001b04       __real@c0000000            0000000031643b04     PoseAlignerChain.obj
 0002:00001b08       ??_C@_0BH@ILEOFMKI@a_poseAlignerDebugDraw?$AA@ 0000000031643b08     PoseAlignerChain.obj
 0002:00001b20       ??_7CFactory@CPoseAlignerChain@@6B@ 0000000031643b20     PoseAlignerChain.obj
 0002:00001b50       ??_C@_0CH@JHIPBLIP@AnimationPoseModifier_PoseAligne@ 0000000031643b50     PoseAlignerChain.obj
 0002:00001b78       ?cid@?1??GetClassID@CFactory@CPoseAlignerChain@@UEBAAEBUCryGUID@@XZ@4U4@B 0000000031643b78     PoseAlignerChain.obj
 0002:00001b98       ?iid@?1??IID@IAnimationPoseMatching@@CAAEBUCryGUID@@XZ@4U3@B 0000000031643b98     PoseMatching.obj
 0002:00001bb0       ??_7CPoseMatching@@6B@     0000000031643bb0     PoseMatching.obj
 0002:00001c00       __real@501502f9            0000000031643c00     PoseMatching.obj
 0002:00001c08       ??_7CFactory@CPoseMatching@@6B@ 0000000031643c08     PoseMatching.obj
 0002:00001c38       ??_C@_0CD@KLIGADKD@AnimationPoseModifier_PoseMatchi@ 0000000031643c38     PoseMatching.obj
 0002:00001c60       ?cid@?1??GetClassID@CFactory@CPoseMatching@@UEBAAEBUCryGUID@@XZ@4U4@B 0000000031643c60     PoseMatching.obj
 0002:00001c78       ??_C@_0CC@CNAFILPC@CryAnimation?3?5VEG?9ID?5out?5of?5rang@ 0000000031643c78     SkeletonAnim_Locator.obj
 0002:00001ca0       ??_C@_0BF@PLHLAKMB@CryAnimation?3?5no?5VEG?$AA@ 0000000031643ca0     SkeletonAnim_Locator.obj
 0002:00001cb8       ??_C@_0CC@CBGNOEAD@No?5Controllers?5found?5in?5Asset?3?5?$CF@ 0000000031643cb8     SkeletonAnim_Locator.obj
 0002:00001ce0       ??_C@_0DA@KHBKMFJG@CryAnimation?3?5No?5Controllers?5fou@ 0000000031643ce0     SkeletonAnim_Locator.obj
 0002:00001d10       ??_C@_0EH@DPPJCECM@CryAnimation?3?5reverse?5playback?5o@ 0000000031643d10     SkeletonAnim_Locator.obj
 0002:00001d58       __real@40133333            0000000031643d58     SkeletonAnim_Locator.obj
 0002:00001d60       ??_C@_0DL@MFPHNIBP@fMoveSpeed?3?5?$CFf?5?5fTurnSpeed?3?5?$CFf?5?5@ 0000000031643d60     SkeletonAnim_Locator.obj
 0002:00001d9c       __real@80000000            0000000031643d9c     SkeletonAnim_Locator.obj
 0002:00001db0       ??_7IVertexAnimation@@6B@  0000000031643db0     VertexAnimation.obj
 0002:00001db0       ??_7Validator@pe_action_batch_parts_update@@6B@ 0000000031643db0     SkeletonPhysics.obj
 0002:00001db0       ??_7ISplineBackup@@6B@     0000000031643db0     FaceAnimSequence.obj
 0002:00001db0       ??_7IFaceState@@6B@        0000000031643db0     FacialModel.obj
 0002:00001dc8       ??_7SBatchUpdateValidator@@6B@ 0000000031643dc8     SkeletonPhysics.obj
 0002:00001de0       ??_C@_04NHHOEEHI@Calf?$AA@ 0000000031643de0     SkeletonPhysics.obj
 0002:00001de8       ??_C@_05NGPCKMLC@Thigh?$AA@ 0000000031643de8     SkeletonPhysics.obj
 0002:00001df0       ??_C@_05CBBIAFIL@Spine?$AA@ 0000000031643df0     SkeletonPhysics.obj
 0002:00001df8       ??_C@_04BFCCBDOP@Head?$AA@ 0000000031643df8     SkeletonPhysics.obj
 0002:00001e00       ??_C@_06EIPNOIEJ@Pelvis?$AA@ 0000000031643e00     SkeletonPhysics.obj
 0002:00001e08       ??_C@_07BLFFLKLF@Forearm?$AA@ 0000000031643e08     SkeletonPhysics.obj
 0002:00001e10       __real@42100000            0000000031643e10     SkeletonPhysics.obj
 0002:00001e14       ??_C@_04IJEANHEE@mass?$AA@ 0000000031643e14     SkeletonPhysics.obj
 0002:00001e1c       __real@40a00000            0000000031643e1c     SkeletonPhysics.obj
 0002:00001e20       __real@3eb33333            0000000031643e20     SkeletonPhysics.obj
 0002:00001e24       ??_C@_06LMBGEFBP@Spine1?$AA@ 0000000031643e24     SkeletonPhysics.obj
 0002:00001e2c       ??_C@_04JBBMMDIF@Hand?$AA@ 0000000031643e2c     SkeletonPhysics.obj
 0002:00001e38       ??_C@_08BOKOBFBJ@UpperArm?$AA@ 0000000031643e38     SkeletonPhysics.obj
 0002:00001e48       ??_C@_0CN@BCDMNCJF@CSkeletonPhysics?3?3SynchronizeWit@ 0000000031643e48     SkeletonPhysics.obj
 0002:00001e78       ??_C@_0BN@NGOFJCFL@rope_stiffness_controller_?$CFd?$AA@ 0000000031643e78     SkeletonPhysics.obj
 0002:00001e98       ??_C@_0M@KOHNAGAB@attach_?$CF?4?$CKs?$AA@ 0000000031643e98     SkeletonPhysics.obj
 0002:00001ea4       __real@44480000            0000000031643ea4     SkeletonPhysics.obj
 0002:00001ea8       ??_C@_04GKOOIABA@loop?$AA@ 0000000031643ea8     SkeletonPhysics.obj
 0002:00001eb0       ??_C@_04JFPBKLKK@rope?$AA@ 0000000031643eb0     SkeletonPhysics.obj
 0002:00001eb8       __real@c2b40000            0000000031643eb8     SkeletonPhysics.obj
 0002:00001ebc       __real@43340000            0000000031643ebc     SkeletonPhysics.obj
 0002:00001ec0       ??_C@_0CO@KCAIEJIE@CSkeletonPhysics?3?3Physics_Synchr@ 0000000031643ec0     SkeletonPhysics.obj
 0002:00001ef0       __real@44610000            0000000031643ef0     SkeletonPhysics.obj
 0002:00001ef8       ??_C@_0CJ@FPNKAHEM@CSkeletonPhysics?3?3SynchronizeWit@ 0000000031643ef8     SkeletonPhysics.obj
 0002:00001f24       __real@c0c00000            0000000031643f24     SkeletonPhysics.obj
 0002:00001f38       ??_C@_0BH@MKEGFDBH@GetStatus?$CI?$CJ?5returned?50?$AA@ 0000000031643f38     SkeletonPhysics_SPU.obj
 0002:00001f50       ??_C@_0DL@KNAAJKGE@CSkeletonPhysics?3?3SPU_Physics_Sy@ 0000000031643f50     SkeletonPhysics_SPU.obj
 0002:00001f90       ??_C@_0DE@DMBPAOJG@CSkeletonPhysics?3?3SPU_Physics_Sy@ 0000000031643f90     SkeletonPhysics_SPU.obj
 0002:00001fc8       ??_C@_0CO@IEFCAFMK@CSkeletonPhysics?3?3SPU_Physics_Sy@ 0000000031643fc8     SkeletonPhysics_SPU.obj
 0002:00002000       ??_C@_0EL@MHNLDCI@Too?5many?5?$CI?5?$DO?52?5?$CJ?5animations?5in?5t@ 0000000031644000     TransitionQueue.obj
 0002:00002050       ??_C@_07NBCGADJA@Unknown?$AA@ 0000000031644050     TransitionQueue.obj
 0002:00002058       ??_7CVertexAnimation@@6B@  0000000031644058     VertexAnimation.obj
 0002:00002078       ??_C@_0DI@LJBCAOEA@CCharInstance?3?3RenderCGA?3?5object@ 0000000031644078     _Render.obj
 0002:000020b0       ??_C@_0EA@HOEPBFKF@CryAnimation?3?5CGA?5should?5not?5hav@ 00000000316440b0     _Render.obj
 0002:000020f0       ??_C@_0BP@EKHBKMOH@CCharInstance?3?3GetSkinningData?$AA@ 00000000316440f0     _Render.obj
 0002:00002110       ??_C@_0M@CCHJNHEL@e_DebugDraw?$AA@ 0000000031644110     _Render.obj
 0002:00002120       ??_C@_0BO@HOAMFGDG@model?5?8?$CFs?8?5has?5no?5render?5mesh?$AA@ 0000000031644120     _Render.obj
 0002:00002140       __real@3d6147ae            0000000031644140     _Render.obj
 0002:00002148       ??_C@_08EALJILLJ@e_LodMin?$AA@ 0000000031644148     _Render.obj
 0002:00002158       ??_C@_0BO@FHEBEPB@CryAnimation?3?5pMaster?5is?5zero?$AA@ 0000000031644158     _RenderSkins.obj
 0002:00002178       ??_C@_0CB@BAMEGJJA@CAttachmentSKIN?3?3GetSkinningData@ 0000000031644178     _RenderSkins.obj
 0002:000021a0       ??_7IAttachmentObject@@6B@ 00000000316441a0     AttachmentManager.obj
 0002:00002220       ??_7CCGFAttachment@@6B@    0000000031644220     AttachmentManager.obj
 0002:000022a0       ??_C@_0BD@NEBKDNEB@CAttachmentManager?$AA@ 00000000316442a0     AttachmentManager.obj
 0002:000022c0       ??_7CSKELAttachment@@6B@   00000000316442c0     AttachmentManager.obj
 0002:00002340       ??_7CSKINAttachment@@6B@   0000000031644340     AttachmentManager.obj
 0002:000023c0       ??_C@_0DC@OPCJEBHN@CAttachmentManager?3?3ProcessAllAt@ 00000000316443c0     AttachmentManager.obj
 0002:000023f8       ??_C@_0CE@IKGEDBIL@CAttachmentManager?3?3DrawAttachme@ 00000000316443f8     AttachmentManager.obj
 0002:00002420       ??_C@_0DN@LIGJMAJA@CryAnimation?3?5skin?9attachment?5no@ 0000000031644420     AttachmentManager.obj
 0002:00002460       ??_C@_0DL@MILMPAAL@CryAnimation?3?5skin?9attachment?5mu@ 0000000031644460     AttachmentManager.obj
 0002:000024a0       ??_C@_0CH@GBLCFAEO@CryAnimation?3?5no?5character?5creat@ 00000000316444a0     AttachmentManager.obj
 0002:000024c8       ??_C@_0DJ@BOJDPIMN@CryAnimation?3?5no?5static?5object?5a@ 00000000316444c8     AttachmentManager.obj
 0002:00002508       ??_C@_0DF@FBPKFMKG@CryAnimation?3?5no?5character?5as?5at@ 0000000031644508     AttachmentManager.obj
 0002:00002540       ??_C@_03IJBHGJIK@cgf?$AA@  0000000031644540     AttachmentManager.obj
 0002:00002544       ??_C@_03MGFGPPEN@cga?$AA@  0000000031644544     AttachmentManager.obj
 0002:00002548       ??_C@_03ILFBNHND@cdf?$AA@  0000000031644548     AttachmentManager.obj
 0002:00002550       ??_7CAttachmentBONE@@6B@   0000000031644550     AttachmentManager.obj
 0002:00002670       ??_7CAttachmentFACE@@6B@   0000000031644670     AttachmentManager.obj
 0002:00002790       ??_C@_07HMJPJE@CA_SKIN?$AA@ 0000000031644790     AttachmentManager.obj
 0002:00002798       ??_C@_07CJKCDLBP@CA_FACE?$AA@ 0000000031644798     AttachmentManager.obj
 0002:000027a0       ??_C@_05BOOEKJH@Flags?$AA@ 00000000316447a0     AttachmentManager.obj
 0002:000027a8       ??_C@_08EHLKLHMC@lod?$CFd_?$CFs?$AA@ 00000000316447a8     AttachmentManager.obj
 0002:000027b8       ??_C@_0N@DCGKFBOO@PhysPropType?$AA@ 00000000316447b8     AttachmentManager.obj
 0002:000027c8       ??_C@_0BC@HKBCGBAC@PA_PendulumOffset?$AA@ 00000000316447c8     AttachmentManager.obj
 0002:000027e0       ??_C@_0P@BFNFOLOJ@PA_PivotOffset?$AA@ 00000000316447e0     AttachmentManager.obj
 0002:000027f0       ??_C@_0L@NDCAKFMA@PA_Damping?$AA@ 00000000316447f0     AttachmentManager.obj
 0002:00002800       ??_C@_0N@EIIFNMLH@PA_HRotation?$AA@ 0000000031644800     AttachmentManager.obj
 0002:00002810       ??_C@_0M@BGCDNALG@PA_MaxAngle?$AA@ 0000000031644810     AttachmentManager.obj
 0002:00002820       ??_C@_0BA@BKMCDHKE@PA_PendulumType?$AA@ 0000000031644820     AttachmentManager.obj
 0002:00002830       ??_C@_08CPBFELGP@Material?$AA@ 0000000031644830     AttachmentManager.obj
 0002:00002840       ??_C@_07JPNMPAFE@Binding?$AA@ 0000000031644840     AttachmentManager.obj
 0002:00002848       ??_C@_08FPDFGKEJ@BoneName?$AA@ 0000000031644848     AttachmentManager.obj
 0002:00002858       ??_C@_08GCJNLIKG@Position?$AA@ 0000000031644858     AttachmentManager.obj
 0002:00002868       ??_C@_08GFJPCMMD@Rotation?$AA@ 0000000031644868     AttachmentManager.obj
 0002:00002874       ??_C@_05LGOFDGEK@AName?$AA@ 0000000031644874     AttachmentManager.obj
 0002:0000287c       ??_C@_04KOACHJEN@Type?$AA@ 000000003164487c     AttachmentManager.obj
 0002:00002888       ??_C@_07DECFHJLP@CA_BONE?$AA@ 0000000031644888     AttachmentManager.obj
 0002:00002890       ??_C@_0L@PHKLKKHI@Attachment?$AA@ 0000000031644890     AttachmentManager.obj
 0002:000028a0       ??_C@_0P@NCIHDFGC@AttachmentList?$AA@ 00000000316448a0     AttachmentManager.obj
 0002:000028b0       ??_C@_0JE@JIFLDKKB@CryAnimation?3?5Attachment?5CRC32?5f@ 00000000316448b0     AttachmentManager.obj
 0002:00002950       ??_C@_0FF@DBCAHCGP@CryAnimation?3?5Attachment?5name?5?8?$CF@ 0000000031644950     AttachmentManager.obj
 0002:000029a8       ??_C@_05GKKHKKE@Cloth?$AA@ 00000000316449a8     AttachmentManager.obj
 0002:000029b0       ??_C@_04FEDAIEKO@Rope?$AA@ 00000000316449b0     AttachmentManager.obj
 0002:000029bc       __real@41000000            00000000316449bc     CharacterInstance.obj
 0002:000029c0       ??_7ICharacterInstance@@6B@ 00000000316449c0     CharacterInstance.obj
 0002:00002b90       ??_C@_0BE@HJMAHGKO@g_useSinglePosition?$AA@ 0000000031644b90     CharacterInstance.obj
 0002:00002ba8       ??_C@_0CI@LCECAICE@CCharInstance?3?3StartAnimationPro@ 0000000031644ba8     CharacterInstance.obj
 0002:00002bd0       ??_C@_0P@KLIDNMJ@fPlaybackScale?$AA@ 0000000031644bd0     CharacterInstance.obj
 0002:00002be0       ??_C@_0O@IJLABJDO@CCharInstance?$AA@ 0000000031644be0     CharacterInstance.obj
 0002:00002bf0       ??_C@_0CB@GOEOGGKH@Character?5instance?5serialization@ 0000000031644bf0     CharacterInstance.obj
 0002:00002c18       ??_C@_0DC@BOFAPKML@CCharInstance?3?3SkinningTransform@ 0000000031644c18     CharacterInstance.obj
 0002:00002c50       ??_C@_0CA@CNAELFJE@CCharInstance?3?3UpdatePhysicsCGA?$AA@ 0000000031644c50     CharacterInstance.obj
 0002:00002c70       ??_C@_0CD@IALEGKJH@SkinningTransformationsComputati@ 0000000031644c70     CharacterInstance.obj
 0002:00002c98       ??_C@_0N@JDNGJMJC@SkeletonPose?$AA@ 0000000031644c98     CharacterInstance.obj
 0002:00002ca8       ??_C@_0N@KPICOJGL@SkeletonAnim?$AA@ 0000000031644ca8     CharacterInstance.obj
 0002:00002cb8       ??_C@_0BG@NNIDJJEH@skeletonEffectManager?$AA@ 0000000031644cb8     CharacterInstance.obj
 0002:00002cd0       ??_C@_0P@FKGPMGCF@FacialInstance?$AA@ 0000000031644cd0     CharacterInstance.obj
 0002:00002ce0       ??_C@_0N@IMBLMJCA@DecalManager?$AA@ 0000000031644ce0     CharacterInstance.obj
 0002:00002cf0       ??_7CAttachmentManager@@6B@ 0000000031644cf0     CharacterInstance.obj
 0002:00002d90       ??_C@_0N@NBFDINLK@Reloading?5?$CFs?$AA@ 0000000031644d90     CharacterInstance.obj
 0002:00002da0       ??_C@_04FPMBEGCJ@?4cga?$AA@ 0000000031644da0     CharacterInstance.obj
 0002:00002da8       ??_C@_04DFHCEAIG@?4chr?$AA@ 0000000031644da8     CharacterInstance.obj
 0002:00002db0       ??_C@_0L@BINJLNLL@?4chrparams?$AA@ 0000000031644db0     CharacterInstance.obj
 0002:00002dc0       ??_C@_0P@MPKEIAAE@eye_right_bone?$AA@ 0000000031644dc0     CharacterInstance.obj
 0002:00002dd0       ??_C@_0O@LEMMFOGJ@eye_left_bone?$AA@ 0000000031644dd0     CharacterInstance.obj
 0002:00002de0       ??_C@_0L@GHIHOBPC@Bip01?5Head?$AA@ 0000000031644de0     CharacterInstance.obj
 0002:00002df0       ??_C@_0BD@GILDFHIJ@Character?5Instance?$AA@ 0000000031644df0     CharacterInstance.obj
 0002:00002e08       ??_C@_0BN@LKLKFLMP@CCharInstance?3?3CCharInstance?$AA@ 0000000031644e08     CharacterInstance.obj
 0002:00002e30       ??_7CCharInstance@@6B@     0000000031644e30     CharacterInstance.obj
 0002:00003018       ??_C@_0BH@GOPGBEEC@CSkelInstance?3?3Release?$AA@ 0000000031645018     CharacterInstance.obj
 0002:00003038       __real@3bb60b61            0000000031645038     SkeletonEffectManager.obj
 0002:0000303c       __real@40490fd0            000000003164503c     SkeletonEffectManager.obj
 0002:00003040       ??_C@_0HL@DKCIOAAC@CSkeletonEffectManager?3?3KillAllE@ 0000000031645040     SkeletonEffectManager.obj
 0002:000030c0       ??_C@_0O@EDBNCENI@?$DMEFFECT?5NULL?$DO?$AA@ 00000000316450c0     SkeletonEffectManager.obj
 0002:000030d0       ??_C@_0EJ@CFHONEBF@CSkeletonEffectManager?3?3Update?$CIt@ 00000000316450d0     SkeletonEffectManager.obj
 0002:00003120       ??_C@_0BB@EAGAEMEP@effect?5has?5ended?$AA@ 0000000031645120     SkeletonEffectManager.obj
 0002:00003138       ??_C@_0BE@INGNAFEN@animation?5has?5ended?$AA@ 0000000031645138     SkeletonEffectManager.obj
 0002:00003150       ??_C@_0GB@KCJFBAAL@CSkeletonEffectManager?3?3SpawnEff@ 0000000031645150     SkeletonEffectManager.obj
 0002:000031c0       ??_C@_0EC@OODFIMGA@Anim?5events?5cannot?5find?5effect?5?$CC@ 00000000316451c0     SkeletonEffectManager.obj
 0002:00003208       ??_C@_0BE@GBHJILEN@?$DMMISSING?5ANIM?5NAME?$DO?$AA@ 0000000031645208     SkeletonEffectManager.obj
 0002:00003220       ??_C@_0GP@PLKJKPDM@CSkeletonEffectManager?3?3SpawnEff@ 0000000031645220     SkeletonEffectManager.obj
 0002:00003290       ??_C@_0BG@OBHJPKFK@?$DMMISSING?5EFFECT?5NAME?$DO?$AA@ 0000000031645290     SkeletonEffectManager.obj
 0002:000032b0       ??_7ISkeletonPhysics@@6B@  00000000316452b0     SkeletonPose.obj
 0002:00003368       ?iid@?1??IID@IAnimationPoseBlenderDir@@CAAEBUCryGUID@@XZ@4U3@B 0000000031645368     SkeletonPose.obj
 0002:00003380       ??_7CSkeletonPose@@6B@     0000000031645380     SkeletonPose.obj
 0002:000034f8       ??_C@_0BN@FJGLIONO@AnimationPoseModifier_LimbIk?$AA@ 00000000316454f8     SkeletonPose.obj
 0002:00003518       ??_C@_0BN@CDBOBPKN@AnimationPoseModifier_Recoil?$AA@ 0000000031645518     SkeletonPose.obj
 0002:00003538       ??_C@_0CF@FNOFOMKI@AnimationPoseModifier_PoseBlende@ 0000000031645538     SkeletonPose.obj
 0002:00003560       ??_C@_0CG@IACGDDFJ@AnimationPoseModifier_PoseBlende@ 0000000031645560     SkeletonPose.obj
 0002:0000358c       __real@3be56041            000000003164558c     SkeletonPose_Debug.obj
 0002:00003590       __real@3bfc5048            0000000031645590     SkeletonPose_Debug.obj
 0002:00003598       ??_C@_0BA@MOHPKELD@ca_filterJoints?$AA@ 0000000031645598     SkeletonPose_Debug.obj
 0002:000035b0       ??_C@_0FP@NMBIDECH@CryAnimation?3?5Invalid?5BBox?5?$CI?$CF?43f@ 00000000316455b0     SkeletonPose_Process.obj
 0002:00003610       __real@be4ccccd            0000000031645610     SkeletonPose_Process.obj
 0002:00003614       __real@3ecccccd            0000000031645614     SkeletonPose_Process.obj
 0002:00003620       ??_C@_0HG@JKDPDHGB@CryAnimation?3?5Invalid?5BBox?5of?5eA@ 0000000031645620     SkeletonPose_Process.obj
 0002:000036a0       ??_C@_0HI@CDNHHDIC@CryAnimation?3?5Invalid?5BBox?5of?5eA@ 00000000316456a0     SkeletonPose_Process.obj
 0002:00003720       ??_C@_0GF@BNBINMGD@CryAnimation?3?5Invalid?5BBox?5of?5eA@ 0000000031645720     SkeletonPose_Process.obj
 0002:00003790       ??_C@_0HF@DMFLBKPI@CryAnimation?3?5Invalid?5BBox?5of?5eA@ 0000000031645790     SkeletonPose_Process.obj
 0002:00003808       ??_C@_0DC@KCEBGHKH@CryAnimation?3?5Invalid?5BBox?5of?5eA@ 0000000031645808     SkeletonPose_Process.obj
 0002:00003840       ??_C@_0DD@PFPHELGK@CryAnimation?3?5Invalid?5BBox?5of?5eA@ 0000000031645840     SkeletonPose_Process.obj
 0002:00003878       ??_C@_0DB@KGEJIDDH@CryAnimation?3?5Invalid?5BBox?5of?5eA@ 0000000031645878     SkeletonPose_Process.obj
 0002:000038ac       ??_C@_01EOFPKCAF@?$EA?$AA@ 00000000316458ac     SkeletonPose_Process.obj
 0002:000038b0       __real@464b2000            00000000316458b0     SkeletonPose_Process.obj
 0002:000038b4       __real@c64b2000            00000000316458b4     SkeletonPose_Process.obj
 0002:000038b8       ??_C@_0BK@FEFLJLDB@CSkeletonPose?3?3UpdateBBox?$AA@ 00000000316458b8     SkeletonPose_Process.obj
 0002:000038d8       ??_C@_0CB@JFODNIDJ@CSkeletonPose?3?3UpdateAttachments@ 00000000316458d8     SkeletonPose_Process.obj
 0002:00003900       ??_C@_0CD@NNGGBPBL@CSkeletonPose?3?3SkeletonPostProce@ 0000000031645900     SkeletonPose_Process.obj
 0002:00003928       ??_7CSkeletonAnimTask@@6B@ 0000000031645928     SkeletonAnim.obj
 0002:00003940       ??_7ISkeletonAnim@@6B@     0000000031645940     SkeletonAnim.obj
 0002:00003a60       ??_C@_0EM@NCIMOGPO@Trying?5to?5set?5manual?5mixing?5weig@ 0000000031645a60     SkeletonAnim.obj
 0002:00003ab0       ??_C@_0HN@OAMMIFAP@Run?5out?5of?5free?5parametric?5slots@ 0000000031645ab0     SkeletonAnim.obj
 0002:00003b30       ??_C@_0BB@JDCEONKJ@nSegmentCounter0?$AA@ 0000000031645b30     SkeletonAnim.obj
 0002:00003b48       ??_C@_08GICNLBFM@nAnimIDs?$AA@ 0000000031645b48     SkeletonAnim.obj
 0002:00003b54       ??_C@_02OLOABKKD@ID?$AA@   0000000031645b54     SkeletonAnim.obj
 0002:00003b58       ??_C@_0O@OBKBEJFL@m_numExamples?$AA@ 0000000031645b58     SkeletonAnim.obj
 0002:00003b68       ??_C@_0BI@EPLIHMDK@m_MotionParameterFlags3?$AA@ 0000000031645b68     SkeletonAnim.obj
 0002:00003b80       ??_C@_0BI@FGKDENHL@m_MotionParameterFlags2?$AA@ 0000000031645b80     SkeletonAnim.obj
 0002:00003b98       ??_C@_0BI@HNIOBOLI@m_MotionParameterFlags1?$AA@ 0000000031645b98     SkeletonAnim.obj
 0002:00003bb0       ??_C@_0BI@GEJFCPPJ@m_MotionParameterFlags0?$AA@ 0000000031645bb0     SkeletonAnim.obj
 0002:00003bc8       ??_C@_0BD@FNMPMFCO@MotionParameterID3?$AA@ 0000000031645bc8     SkeletonAnim.obj
 0002:00003be0       ??_C@_0BD@EENEPEGP@MotionParameterID2?$AA@ 0000000031645be0     SkeletonAnim.obj
 0002:00003bf8       ??_C@_0BD@GPPJKHKM@MotionParameterID1?$AA@ 0000000031645bf8     SkeletonAnim.obj
 0002:00003c10       ??_C@_0BD@HGOCJGON@MotionParameterID0?$AA@ 0000000031645c10     SkeletonAnim.obj
 0002:00003c28       ??_C@_0BB@BNGLIPCC@MotionParameter3?$AA@ 0000000031645c28     SkeletonAnim.obj
 0002:00003c40       ??_C@_0BB@EHALOGD@MotionParameter2?$AA@ 0000000031645c40     SkeletonAnim.obj
 0002:00003c58       ??_C@_0BB@CPFNONKA@MotionParameter1?$AA@ 0000000031645c58     SkeletonAnim.obj
 0002:00003c70       ??_C@_0BB@DGEGNMOB@MotionParameter0?$AA@ 0000000031645c70     SkeletonAnim.obj
 0002:00003c88       ??_C@_0BC@HODPFOO@m_nParametricType?$AA@ 0000000031645c88     SkeletonAnim.obj
 0002:00003ca0       ??_C@_0BA@DGHJNPFJ@m_numDimensions?$AA@ 0000000031645ca0     SkeletonAnim.obj
 0002:00003cb0       ??_C@_0BD@GDFFJPDJ@SParametricSampler?$AA@ 0000000031645cb0     SkeletonAnim.obj
 0002:00003cc8       ??_C@_0BI@KOCPMHMM@CSkeletonAnimTask?3?3Wait?$AA@ 0000000031645cc8     SkeletonAnim.obj
 0002:00003ce0       ??_C@_0CG@PKLKOFJC@CSkeletonAnim?3?3ProcessAnimationU@ 0000000031645ce0     SkeletonAnim.obj
 0002:00003d08       ??_C@_0BF@LBMBDMEN@CommandBufferExecute?$AA@ 0000000031645d08     SkeletonAnim.obj
 0002:00003d20       ??_C@_0CL@KIKELEAM@CSkeletonAnim?3?3FinishAnimationCo@ 0000000031645d20     SkeletonAnim.obj
 0002:00003d50       ??_C@_0M@FBNCIMKH@BlenderLook?$AA@ 0000000031645d50     SkeletonAnim.obj
 0002:00003d60       ??_C@_0L@BCDNODAM@BlenderAim?$AA@ 0000000031645d60     SkeletonAnim.obj
 0002:00003d6c       ??_C@_06LNHJHIDK@Recoil?$AA@ 0000000031645d6c     SkeletonAnim.obj
 0002:00003d74       ??_C@_06FCIIMNOL@LimbIK?$AA@ 0000000031645d74     SkeletonAnim.obj
 0002:00003d80       ??_C@_0CO@BDOOGFON@Animation?5Task?5started?5while?5alr@ 0000000031645d80     SkeletonAnim.obj
 0002:00003db0       ??_C@_0CB@KNFFGCC@several?5pre?9updates?3?5FrameID?3?5?$CFx@ 0000000031645db0     SkeletonAnim.obj
 0002:00003de0       ??_C@_0EN@CHENBBIP@CSkeletonAnim?3?3ProcessAnimations@ 0000000031645de0     SkeletonAnim.obj
 0002:00003e30       ??_C@_0M@NJMOOCJK@fUserData?$CFi?$AA@ 0000000031645e30     SkeletonAnim.obj
 0002:00003e40       ??_C@_0L@DGANLLHB@nUserToken?$AA@ 0000000031645e40     SkeletonAnim.obj
 0002:00003e50       ??_C@_0P@LEFAENAC@fPlaybackSpeed?$AA@ 0000000031645e50     SkeletonAnim.obj
 0002:00003e60       ??_C@_0L@PHEIIFBJ@fStartTime?$AA@ 0000000031645e60     SkeletonAnim.obj
 0002:00003e70       ??_C@_0BA@NAJHGMIJ@fTransitionTime?$AA@ 0000000031645e70     SkeletonAnim.obj
 0002:00003e80       ??_C@_06PGMJADPC@nFlags?$AA@ 0000000031645e80     SkeletonAnim.obj
 0002:00003e88       ??_C@_09NIOBDIMK@DynFlags1?$AA@ 0000000031645e88     SkeletonAnim.obj
 0002:00003e98       ??_C@_09MBPKAJIL@DynFlags0?$AA@ 0000000031645e98     SkeletonAnim.obj
 0002:00003ea8       ??_C@_0BH@IFGILKFJ@segmentNormalizedTime1?$AA@ 0000000031645ea8     SkeletonAnim.obj
 0002:00003ec0       ??_C@_0BH@JMHDILBI@segmentNormalizedTime0?$AA@ 0000000031645ec0     SkeletonAnim.obj
 0002:00003ed8       ??_C@_0BL@JEFJNGNP@segmentNormalizedTimePrev1?$AA@ 0000000031645ed8     SkeletonAnim.obj
 0002:00003ef8       ??_C@_0BL@INECOHJO@segmentNormalizedTimePrev0?$AA@ 0000000031645ef8     SkeletonAnim.obj
 0002:00003f18       ??_C@_0BF@ILDLBJEJ@currentSegmentIndex1?$AA@ 0000000031645f18     SkeletonAnim.obj
 0002:00003f30       ??_C@_0BF@JCCACIAI@currentSegmentIndex0?$AA@ 0000000031645f30     SkeletonAnim.obj
 0002:00003f48       ??_C@_0BN@LADPHNKL@expectedTotalDurationSeconds?$AA@ 0000000031645f48     SkeletonAnim.obj
 0002:00003f68       ??_C@_0CG@HBMDHLAE@currentSegmentExpectedDurationSe@ 0000000031645f68     SkeletonAnim.obj
 0002:00003f90       ??_C@_0BB@NDJBDEPO@transitionWeight?$AA@ 0000000031645f90     SkeletonAnim.obj
 0002:00003fa8       ??_C@_0BD@HAOBDOND@transitionPriority?$AA@ 0000000031645fa8     SkeletonAnim.obj
 0002:00003fc0       ??_C@_0BL@BKOJBLHA@segmentNormalizedTimeDelta?$AA@ 0000000031645fc0     SkeletonAnim.obj
 0002:00003fe0       ??_C@_0M@CAHNJPEP@animationId?$AA@ 0000000031645fe0     SkeletonAnim.obj
 0002:00003ff0       ??_C@_0L@CKOPHJKN@CAnimation?$AA@ 0000000031645ff0     SkeletonAnim.obj
 0002:00004000       ??_7CSkeletonAnim@@6B@     0000000031646000     SkeletonAnim.obj
 0002:00004128       ??_C@_0N@NOMPLAGO@nAnimsInFIFO?$AA@ 0000000031646128     SkeletonAnim.obj
 0002:00004138       ??_C@_04LIEBAAE@FIFO?$AA@  0000000031646138     SkeletonAnim.obj
 0002:00004140       ??_C@_0BE@OCLDLCOI@ForceSkeletonUpdate?$AA@ 0000000031646140     SkeletonAnim.obj
 0002:00004158       ??_C@_0BG@IDEPGADK@AnimationDrivenMotion?$AA@ 0000000031646158     SkeletonAnim.obj
 0002:00004170       ??_C@_0O@EMJFAEAE@CSkeletonAnim?$AA@ 0000000031646170     SkeletonAnim.obj
 0002:00004188       ??_C@_0BB@LBPDIKEH@?$CLybVFx3nSIAKTRLM?$AA@ 0000000031646188     SkeletonAnim_BlendMan.obj
 0002:000041a0       ??_C@_0BF@PAKPFLEL@invalid?5layer?5id?3?5?$CFd?$AA@ 00000000316461a0     SkeletonAnim_BlendMan.obj
 0002:000041b8       ??_C@_0DH@EADFOBJA@SetLayerPlaybackScale?$CI?$CJ?5was?5usin@ 00000000316461b8     SkeletonAnim_BlendMan.obj
 0002:000041f0       __real@bf490fdb            00000000316461f0     SkeletonAnim_BlendMan.obj
 0002:000041f8       ??_C@_0BK@OFNKCMHP@CryAnimation?3?5weird?5error?$AA@ 00000000316461f8     SkeletonAnim_BlendMan.obj
 0002:00004218       __real@3f50624dd2f1a9fc    0000000031646218     SkeletonAnim_BlendMan.obj
 0002:00004220       __real@3ffffcb9            0000000031646220     SkeletonAnim_BlendMan.obj
 0002:00004228       ??_C@_0BG@DJGEAONA@PM?5class?3?5?$CFs?0?5name?5?$CFs?$AA@ 0000000031646228     SkeletonAnim_BlendMan.obj
 0002:00004240       ??_C@_0BH@CCCIPAEE@LayerBlendWeight?3?5?$CF?42f?$AA@ 0000000031646240     SkeletonAnim_BlendMan.obj
 0002:00004258       ??_C@_0BK@HCHOIMBG@TurnAngle?3?5?$CFf?5?5locked?3?5?$CFd?$AA@ 0000000031646258     SkeletonAnim_BlendMan.obj
 0002:00004278       ??_C@_0BL@PCPKINMJ@TravelDist?3?5?$CFf?5?5locked?3?5?$CFd?$AA@ 0000000031646278     SkeletonAnim_BlendMan.obj
 0002:00004298       ??_C@_0BM@MODFLBDB@TravelAngle?3?5?$CFf?5?5locked?3?5?$CFd?$AA@ 0000000031646298     SkeletonAnim_BlendMan.obj
 0002:000042b8       ??_C@_0BH@GFJBEPIE@Slope?3?5?$CFf?5?5?5locked?3?5?$CFd?$AA@ 00000000316462b8     SkeletonAnim_BlendMan.obj
 0002:000042d0       ??_C@_0BK@JGCNEMDL@TurnSpeed?3?5?$CFf?5?5locked?3?5?$CFd?$AA@ 00000000316462d0     SkeletonAnim_BlendMan.obj
 0002:000042f0       ??_C@_0BK@HFGLOKKI@MoveSpeed?3?5?$CFf?5?5locked?3?5?$CFd?$AA@ 00000000316462f0     SkeletonAnim_BlendMan.obj
 0002:00004310       ??_C@_0BJ@PKAHMHPG@StopLeg?3?5?$CFf?5?5?5locked?3?5?$CFd?$AA@ 0000000031646310     SkeletonAnim_BlendMan.obj
 0002:00004330       ??_C@_0DK@EHGNKBIP@?$CITry?$CJUseAimIK?3?5?$CFd?5?5AimIKBlend?3?5?$CF@ 0000000031646330     SkeletonAnim_BlendMan.obj
 0002:00004370       ??_C@_0HG@KFADONL@AnimInAFIFO?5?$CF02d?3?5t?3?$CFd?5?5?$CFs?5?5ATim@ 0000000031646370     SkeletonAnim_BlendMan.obj
 0002:000043e8       ??_C@_0CJ@JAGHNNHF@CryAnimation?3?5I2M?5without?5Turn?9P@ 00000000316463e8     SkeletonAnim_BlendMan.obj
 0002:00004418       ??_C@_0CB@GENKLKFL@CryAnimation?3?5streaming?5file?3?5?$CFs@ 0000000031646418     SkeletonAnim_BlendMan.obj
 0002:00004440       ??_C@_0BG@BNBLDCEC@Streaming?5Assets?3?5?$CFs?5?$AA@ 0000000031646440     SkeletonAnim_BlendMan.obj
 0002:00004458       __real@40266666            0000000031646458     SkeletonAnim_BlendMan.obj
 0002:0000445c       __real@358637bd            000000003164645c     SkeletonAnim_BlendMan.obj
 0002:00004460       ??_C@_0DI@BLFGLGHC@CryAnimation?3?5sum?5of?5transition?9@ 0000000031646460     SkeletonAnim_BlendMan.obj
 0002:00004498       ??_C@_0BM@MAMIHPIG@CSkeletonAnim?3?3BlendManager?$AA@ 0000000031646498     SkeletonAnim_BlendMan.obj
 0002:000044b8       ??_C@_0CG@ENFHLLOI@CryAnimation?3?5CommandBuffer?5over@ 00000000316464b8     SkeletonAnim_Commands.obj
 0002:000044e0       __real@3ee66666            00000000316464e0     SkeletonAnim_Commands.obj
 0002:000044e8       ??_C@_0DK@MAHKPBIL@CryAnimation?3?5LMG?5asset?5sorting?5@ 00000000316464e8     SkeletonAnim_Commands.obj
 0002:00004530       ??_C@_0EH@KGLPLNGH@CryAnimation?3?5LMG?5weights?5don?8t?5@ 0000000031646530     SkeletonAnim_Commands.obj
 0002:00004578       __real@3db851ec            0000000031646578     SkeletonAnim_Commands.obj
 0002:00004580       ??_C@_0BP@HKBDNLIE@CSkeletonAnim?3?3Commands_Create?$AA@ 0000000031646580     SkeletonAnim_Commands.obj
 0002:000045a8       ??_C@_0DD@LGCDNMMN@animation?9name?5?8?$CFs?8?5not?5in?5CAL?9f@ 00000000316465a8     SkeletonAnim_Queue.obj
 0002:000045dc       ??_C@_04HIBGFPH@NULL?$AA@  00000000316465dc     SkeletonAnim_Queue.obj
 0002:000045e4       ??_C@_04MLLLIHIP@null?$AA@ 00000000316465e4     SkeletonAnim_Queue.obj
 0002:000045f0       ??_C@_0CA@IHMAKIHG@No?5name?5for?5animation?5specified?$AA@ 00000000316465f0     SkeletonAnim_Queue.obj
 0002:00004610       ??_C@_0EP@MOCENKPM@illegal?5layer?5index?5used?5in?5func@ 0000000031646610     SkeletonAnim_Queue.obj
 0002:00004660       ??_C@_0CF@LPDMCJ@Exceeding?5max?5examples?5in?5?$CFs?0?5CR@ 0000000031646660     SkeletonAnim_Queue.obj
 0002:00004688       ??_C@_0BN@CEPHBKBJ@CryAnimation?3?5not?5initalized?$AA@ 0000000031646688     SkeletonAnim_Queue.obj
 0002:000046b0       ??_C@_0GB@OIDNMHKB@Animation?9queue?5overflow?4?5More?5t@ 00000000316466b0     SkeletonAnim_Queue.obj
 0002:00004718       ??_C@_0BF@EIDJGIHD@LMG?5is?5invalid?3?5?8?$CFs?8?$AA@ 0000000031646718     SkeletonAnim_Queue.obj
 0002:00004730       ??_C@_0BM@MJDBPANO@Anim?5asset?5error?3?5?$CFs?5failed?$AA@ 0000000031646730     SkeletonAnim_Queue.obj
 0002:00004750       ??_C@_0BM@JJOGJBAO@rLMG?4IsAssetLMGValid?$CI?$CJ?5?$CB?$DN?50?$AA@ 0000000031646750     SkeletonAnim_Queue.obj
 0002:00004770       ??_C@_0DL@KFFEMKAN@Asset?5for?5animation?9name?5?8?$CFs?8?5do@ 0000000031646770     SkeletonAnim_Queue.obj
 0002:000047b0       ??_C@_0DI@GLLODHOF@trying?5to?5play?5an?5unloaded?5Look?9@ 00000000316467b0     SkeletonAnim_Queue.obj
 0002:000047e8       ??_C@_0DH@PMBKPGAO@trying?5to?5play?5an?5unloaded?5Aim?9P@ 00000000316467e8     SkeletonAnim_Queue.obj
 0002:00004820       ??_C@_0DK@ECPNMJGD@Asset?5for?5animation?9name?5?8?$CFs?8?5do@ 0000000031646820     SkeletonAnim_Queue.obj
 0002:00004860       ??_C@_0CC@PLKNFGEP@CSkeletonAnim?3?3StartAnimationByI@ 0000000031646860     SkeletonAnim_Queue.obj
 0002:00004888       ??_C@_0BF@GGEMLKGC@Eye_right_lower_left?$AA@ 0000000031646888     EyeMovementFaceAnim.obj
 0002:000048a0       ??_C@_0BG@KHLAEODP@Eye_right_middle_left?$AA@ 00000000316468a0     EyeMovementFaceAnim.obj
 0002:000048b8       ??_C@_0BF@BDDPHIA@Eye_right_upper_left?$AA@ 00000000316468b8     EyeMovementFaceAnim.obj
 0002:000048d0       ??_C@_0BH@LKHBJMFB@Eye_right_upper_middle?$AA@ 00000000316468d0     EyeMovementFaceAnim.obj
 0002:000048e8       ??_C@_0BG@PHEGLPLO@Eye_right_upper_right?$AA@ 00000000316468e8     EyeMovementFaceAnim.obj
 0002:00004900       ??_C@_0BH@KMDOJCBK@Eye_right_middle_right?$AA@ 0000000031646900     EyeMovementFaceAnim.obj
 0002:00004918       ??_C@_0BG@LJCFEDKH@Eye_right_lower_right?$AA@ 0000000031646918     EyeMovementFaceAnim.obj
 0002:00004930       ??_C@_0BH@NOFEFHGN@Eye_right_lower_middle?$AA@ 0000000031646930     EyeMovementFaceAnim.obj
 0002:00004948       ??_C@_0BE@MPOBEKFA@Eye_left_lower_left?$AA@ 0000000031646948     EyeMovementFaceAnim.obj
 0002:00004960       ??_C@_0BF@GPMOLCEP@Eye_left_middle_left?$AA@ 0000000031646960     EyeMovementFaceAnim.obj
 0002:00004978       ??_C@_0BE@KIJOAHLC@Eye_left_upper_left?$AA@ 0000000031646978     EyeMovementFaceAnim.obj
 0002:00004990       ??_C@_0BG@OKLMJDJB@Eye_left_upper_middle?$AA@ 0000000031646990     EyeMovementFaceAnim.obj
 0002:000049a8       ??_C@_0BF@DPDIEDMO@Eye_left_upper_right?$AA@ 00000000316469a8     EyeMovementFaceAnim.obj
 0002:000049c0       ??_C@_0BG@PMPDJNNK@Eye_left_middle_right?$AA@ 00000000316469c0     EyeMovementFaceAnim.obj
 0002:000049d8       ??_C@_0BF@HBFLLPNH@Eye_left_lower_right?$AA@ 00000000316469d8     EyeMovementFaceAnim.obj
 0002:000049f0       ??_C@_0BG@IOJJFIKN@Eye_left_lower_middle?$AA@ 00000000316469f0     EyeMovementFaceAnim.obj
 0002:00004a08       ??_7CEyeMovementFaceAnim@@6B@ 0000000031646a08     EyeMovementFaceAnim.obj
 0002:00004a08       ??_7?$_i_reference_target@H@@6B@ 0000000031646a08     LoaderSKIN.obj
 0002:00004a20       __real@3ea2f98c            0000000031646a20     EyeMovementFaceAnim.obj
 0002:00004a24       __real@3d888889            0000000031646a24     EyeMovementFaceAnim.obj
 0002:00004a28       ??_C@_09EDIDEKJE@eye_right?$AA@ 0000000031646a28     EyeMovementFaceAnim.obj
 0002:00004a38       ??_C@_08MPHIOKHM@eye_left?$AA@ 0000000031646a38     EyeMovementFaceAnim.obj
 0002:00004a48       ??_C@_0BB@LHAAIHLB@?$CF?43f?0?5?$CF?43f?0?5?$CF?43f?$AA@ 0000000031646a48     EyeMovementFaceAnim.obj
 0002:00004a5c       __real@3e22f983            0000000031646a5c     EyeMovementFaceAnim.obj
 0002:00004a68       ??_7JoystickSerializeContext@?4??BindJoystickSetToSequence@CFacialAnimation@@UEAAXPEAVIJoystickSet@@PEAUIFacialAnimSequence@@@Z@6B@ 0000000031646a68     FaceAnimation.obj
 0002:00004a78       ??_C@_09KJHOEFNK@?$CFs?3?$CF?42f?0?5?$AA@ 0000000031646a78     FaceAnimation.obj
 0002:00004a88       ??_C@_0CD@PCKJDCCB@Failed?5to?5load?5facial?5joysticks?5@ 0000000031646a88     FaceAnimation.obj
 0002:00004aac       ??_C@_03DHFGHJCG@joy?$AA@  0000000031646aac     FaceAnimation.obj
 0002:00004ab0       ??_C@_0BI@MKDILCDF@Stop?5Facial?5Sequence?5?$CFs?$AA@ 0000000031646ab0     FaceAnimation.obj
 0002:00004ac8       ??_7CFacialAnimSequenceInstance@@6B@ 0000000031646ac8     FaceAnimation.obj
 0002:00004ae0       ??_7CFacialAnimationContext@@6B@ 0000000031646ae0     FaceAnimation.obj
 0002:00004af8       ??_C@_0BB@KCOAIOFL@?$CFs?5?3?5?$CItime?$DN?$CF?42f?$CJ?$AA@ 0000000031646af8     FaceAnimation.obj
 0002:00004b0c       __real@bdcccccd            0000000031646b0c     FaceAnimation.obj
 0002:00004b10       ??_C@_0BK@HDFLJAGF@Stop?5All?5Facial?5Sequences?$AA@ 0000000031646b10     FaceAnimation.obj
 0002:00004b30       ??_7CFacialAnimation@@6BIJoystickContext@@@ 0000000031646b30     FaceAnimation.obj
 0002:00004b50       ??_7CFacialAnimation@@6BIFacialAnimation@@@ 0000000031646b50     FaceAnimation.obj
 0002:00004bc0       ??_C@_0EM@OJIBBPNJ@CFacialAnimationContext?3?3Update?$CI@ 0000000031646bc0     FaceAnimation.obj
 0002:00004c10       ??_C@_0CA@JFHDHLDA@CFacialAnimationContext?3?3Update?$AA@ 0000000031646c10     FaceAnimation.obj
 0002:00004c30       ??_C@_0BI@OCHHCIBP@Play?5Facial?5Sequence?5?$CFs?$AA@ 0000000031646c30     FaceAnimation.obj
 0002:00004c48       ??_C@_0CH@HGMAHIPL@Failed?5to?5allocate?5memory?5for?5se@ 0000000031646c48     FaceAnimation.obj
 0002:00004c70       ??_C@_0BP@BPEJPION@Failed?5to?5load?5facial?5sequence?$AA@ 0000000031646c70     FaceAnimation.obj
 0002:00004c90       ??_C@_03KAGFBGIC@fsq?$AA@  0000000031646c90     FaceAnimation.obj
 0002:00004c94       ??_C@_02MOLJINC@?3?3?$AA@  0000000031646c94     FaceAnimation.obj
 0002:00004ca0       ??_7ISplineInterpolator@@6B@ 0000000031646ca0     FaceAnimSequence.obj
 0002:00004ca0       ??_7IFacialAnimChannel@@6B@ 0000000031646ca0     FaceAnimSequence.obj
 0002:00004d50       ??_7IFacialAnimSoundEntry@@6B@ 0000000031646d50     FaceAnimSequence.obj
 0002:00004d80       ??_7IFacialAnimSequence@@6B@ 0000000031646d80     FaceAnimSequence.obj
 0002:00004e88       ??_7IStreamCallback@@6B@   0000000031646e88     FaceAnimSequence.obj
 0002:00004ea8       ??_C@_06DLKDIFGH@Spline?$AA@ 0000000031646ea8     FaceAnimSequence.obj
 0002:00004eb0       ??_C@_07DMJBFPJJ@Channel?$AA@ 0000000031646eb0     FaceAnimSequence.obj
 0002:00004eb8       ??_C@_04FABLJDN@Name?$AA@  0000000031646eb8     FaceAnimSequence.obj
 0002:00004ec0       ??_C@_0FG@JCOJGMCK@CFacialAnimSequence?3?5Getting?5ske@ 0000000031646ec0     FaceAnimSequence.obj
 0002:00004f18       __real@bdf5c28f            0000000031646f18     FaceAnimSequence.obj
 0002:00004f1c       __real@3df5c28f            0000000031646f1c     FaceAnimSequence.obj
 0002:00004f20       ??_7CFacialAnimSoundEntry@@6B@ 0000000031646f20     FaceAnimSequence.obj
 0002:00004f50       ??_7CFacialAnimSkeletalAnimationEntry@@6B@ 0000000031646f50     FaceAnimSequence.obj
 0002:00004f88       ??_7CFacialAnimChannel@@6B?$_i_reference_target@H@@@ 0000000031646f88     FaceAnimSequence.obj
 0002:00004fa0       ??_7CFacialAnimChannel@@6BIFacialAnimChannel@@@ 0000000031646fa0     FaceAnimSequence.obj
 0002:00005050       ??_7?$TSpline@U?$SplineKey@U?$Quat_tpl@M@@@spline@@VHermitBasis@2@@spline@@6B@ 0000000031647050     FaceAnimSequence.obj
 0002:00005070       ??_7?$TSpline@U?$TCBSplineKey@U?$Vec3_tpl@M@@@spline@@VHermitBasis@2@@spline@@6B@ 0000000031647070     FaceAnimSequence.obj
 0002:00005090       ??_C@_09BLOICCGF@?$CFg?3?$CFg?3?$CFd?0?$AA@ 0000000031647090     FaceAnimSequence.obj
 0002:000050a0       ??_C@_08NLFPHCLG@?$CFg?3?$CFg?3?$CFd?$AA@ 00000000316470a0     FaceAnimSequence.obj
 0002:000050ac       ??_C@_01IHBHIGKO@?0?$AA@   00000000316470ac     FaceAnimSequence.obj
 0002:000050b0       ??_C@_04EFDEBPGB@Keys?$AA@ 00000000316470b0     FaceAnimSequence.obj
 0002:000050b8       ??_C@_0BA@KMFEKME@?$CFg?3?$CFg?1?$CFg?1?$CFg?3?$CFd?0?$AA@ 00000000316470b8     FaceAnimSequence.obj
 0002:000050c8       ??_C@_0P@PHDMIPGN@?$CFg?3?$CFg?1?$CFg?1?$CFg?3?$CFd?$AA@ 00000000316470c8     FaceAnimSequence.obj
 0002:000050d8       ??_C@_0BD@MLFCNHLL@?$CFg?3?$CFg?1?$CFg?1?$CFg?1?$CFg?3?$CFd?0?$AA@ 00000000316470d8     FaceAnimSequence.obj
 0002:000050f0       ??_C@_0BC@BLMFLFD@?$CFg?3?$CFg?1?$CFg?1?$CFg?1?$CFg?3?$CFd?$AA@ 00000000316470f0     FaceAnimSequence.obj
 0002:00005108       ??_7?$TCBSpline@U?$Vec3_tpl@M@@U?$TCBSplineKey@U?$Vec3_tpl@M@@@spline@@@spline@@6B@ 0000000031647108     FaceAnimSequence.obj
 0002:00005128       ??_7?$SSplineBackup@V?$HermitSplineEx@U?$Quat_tpl@M@@U?$SplineKey@U?$Quat_tpl@M@@@spline@@@spline@@@spline@@6B?$HermitSplineEx@U?$Quat_tpl@M@@U?$SplineKey@U?$Quat_tpl@M@@@spline@@@1@@ 0000000031647128     FaceAnimSequence.obj
 0002:00005148       ??_7?$SSplineBackup@V?$HermitSplineEx@U?$Quat_tpl@M@@U?$SplineKey@U?$Quat_tpl@M@@@spline@@@spline@@@spline@@6BISplineBackup@@@ 0000000031647148     FaceAnimSequence.obj
 0002:00005160       ??_7?$SSplineBackup@V?$HermitSplineEx@MU?$SplineKey@M@spline@@@spline@@@spline@@6B?$HermitSplineEx@MU?$SplineKey@M@spline@@@1@@ 0000000031647160     FaceAnimSequence.obj
 0002:00005180       ??_7?$SSplineBackup@V?$HermitSplineEx@MU?$SplineKey@M@spline@@@spline@@@spline@@6BISplineBackup@@@ 0000000031647180     FaceAnimSequence.obj
 0002:000051a0       ??_C@_0ED@ECEILDBO@CFacialAnimSequence?3?5Deleting?5no@ 00000000316471a0     FaceAnimSequence.obj
 0002:000051f0       ??_C@_0FH@FIIKLAIH@CFacialAnimSequence?3?5Deleting?5sk@ 00000000316471f0     FaceAnimSequence.obj
 0002:00005248       ??_7?$SSplineBackup@V?$TCBSpline@U?$Vec3_tpl@M@@U?$TCBSplineKey@U?$Vec3_tpl@M@@@spline@@@spline@@@spline@@6B?$TCBSpline@U?$Vec3_tpl@M@@U?$TCBSplineKey@U?$Vec3_tpl@M@@@spline@@@1@@ 0000000031647248     FaceAnimSequence.obj
 0002:00005268       ??_7?$SSplineBackup@V?$TCBSpline@U?$Vec3_tpl@M@@U?$TCBSplineKey@U?$Vec3_tpl@M@@@spline@@@spline@@@spline@@6BISplineBackup@@@ 0000000031647268     FaceAnimSequence.obj
 0002:00005280       ??_7CFacialCameraPathPositionInterpolator@@6B?$TCBSpline@U?$Vec3_tpl@M@@U?$TCBSplineKey@U?$Vec3_tpl@M@@@spline@@@spline@@@ 0000000031647280     FaceAnimSequence.obj
 0002:000052a0       ??_7CFacialCameraPathPositionInterpolator@@6BISplineInterpolator@@@ 00000000316472a0     FaceAnimSequence.obj
 0002:00005350       ??_7CFacialCameraPathOrientationInterpolator@@6B?$HermitSplineEx@U?$Quat_tpl@M@@U?$SplineKey@U?$Quat_tpl@M@@@spline@@@spline@@@ 0000000031647350     FaceAnimSequence.obj
 0002:00005370       ??_7CFacialCameraPathOrientationInterpolator@@6BISplineInterpolator@@@ 0000000031647370     FaceAnimSequence.obj
 0002:00005420       ??_7CFacialAnimChannelInterpolator@@6B?$HermitSplineEx@MU?$SplineKey@M@spline@@@spline@@@ 0000000031647420     FaceAnimSequence.obj
 0002:00005440       ??_7CFacialAnimChannelInterpolator@@6BISplineInterpolator@@@ 0000000031647440     FaceAnimSequence.obj
 0002:000054f0       ??_7CFacialAnimSequence@@6BIStreamCallback@@@ 00000000316474f0     FaceAnimSequence.obj
 0002:00005510       ??_7CFacialAnimSequence@@6BIFacialAnimSequence@@@ 0000000031647510     FaceAnimSequence.obj
 0002:00005620       ??_C@_0CG@GNBPJBKH@Failed?5to?5stream?5facial?5sequence@ 0000000031647620     FaceAnimSequence.obj
 0002:00005648       ??_C@_0CG@HGLPGDO@CFacialAnimSequence?3?3StreamOnCom@ 0000000031647648     FaceAnimSequence.obj
 0002:00005670       ??_C@_0BA@PNDICABG@Neck_left_right?$AA@ 0000000031647670     FaceAnimSequence.obj
 0002:00005680       ??_C@_0N@BKPMEFLO@Neck_up_down?$AA@ 0000000031647680     FaceAnimSequence.obj
 0002:00005690       ??_C@_0BB@LLGBCJAO@Default?5Sequence?$AA@ 0000000031647690     FaceAnimSequence.obj
 0002:000056b0       ??_C@_0EL@OGGFCGGC@CFacialAnimSequence?3?5Inserting?5s@ 00000000316476b0     FaceAnimSequence.obj
 0002:00005700       ??_C@_0FI@GCHEDGEC@CFacialAnimSequence?3?5Inserting?5s@ 0000000031647700     FaceAnimSequence.obj
 0002:00005758       ??_C@_07LDICNKFK@?$CFs?$EA?3?$EA?$CFs?$AA@ 0000000031647758     FaceAnimSequence.obj
 0002:00005760       ??_C@_0DF@PIOFEMFB@Attempting?5to?5merge?5sequence?5wit@ 0000000031647760     FaceAnimSequence.obj
 0002:00005798       ??_C@_0N@NFDKOEAM@BakedLipSync?$AA@ 0000000031647798     FaceAnimSequence.obj
 0002:000057a8       ??_C@_0BH@EKOBJLKB@SkeletonAnimationStart?$AA@ 00000000316477a8     FaceAnimSequence.obj
 0002:000057c0       ??_C@_0BC@LPJKMPGL@SkeletonAnimation?$AA@ 00000000316477c0     FaceAnimSequence.obj
 0002:000057d8       ??_C@_0O@IGGNDABF@CameraPathFOV?$AA@ 00000000316477d8     FaceAnimSequence.obj
 0002:000057e8       ??_C@_0BH@HAKIDAOD@CameraPathOrientations?$AA@ 00000000316477e8     FaceAnimSequence.obj
 0002:00005800       ??_C@_0BE@PILIAEOL@CameraPathPositions?$AA@ 0000000031647800     FaceAnimSequence.obj
 0002:00005818       ??_C@_0O@HEOGOAJ@AnimationName?$AA@ 0000000031647818     FaceAnimSequence.obj
 0002:00005828       ??_C@_0BH@GHFHCMOE@SkeletonAnimationEntry?$AA@ 0000000031647828     FaceAnimSequence.obj
 0002:00005840       ??_C@_05MAHMNMLO@Sound?$AA@ 0000000031647840     FaceAnimSequence.obj
 0002:00005848       ??_C@_0L@GBCGONJH@SoundEntry?$AA@ 0000000031647848     FaceAnimSequence.obj
 0002:00005858       ??_C@_08FJCINCME@Sentence?$AA@ 0000000031647858     FaceAnimSequence.obj
 0002:00005868       ??_C@_09BFDKACGK@Joysticks?$AA@ 0000000031647868     FaceAnimSequence.obj
 0002:00005878       ??_C@_07GAHEIAPI@EndTime?$AA@ 0000000031647878     FaceAnimSequence.obj
 0002:00005880       ??_C@_09MHCEAAPI@StartTime?$AA@ 0000000031647880     FaceAnimSequence.obj
 0002:00005894       __real@40c90fd0            0000000031647894     FaceChannelSmoothing.obj
 0002:000058a0       ??_7IFacialEffector@@6B@   00000000316478a0     FaceEffector.obj
 0002:00005950       ??_7IFacialEffCtrl@@6B@    0000000031647950     FaceEffector.obj
 0002:00005950       ??_7IJoystickSet@@6B@      0000000031647950     FaceJoystick.obj
 0002:000059b0       ??_C@_08EPGFEOCM@Effector?$AA@ 00000000316479b0     FaceEffector.obj
 0002:000059bc       ??_C@_06ODJMJFLN@Weight?$AA@ 00000000316479bc     FaceEffector.obj
 0002:000059c8       ??_C@_09MANMBJC@RotOffset?$AA@ 00000000316479c8     FaceEffector.obj
 0002:000059d8       ??_C@_09CDNBILG@PosOffset?$AA@ 00000000316479d8     FaceEffector.obj
 0002:000059e4       ??_C@_06OCDDEAHI@?$CFg?3?$CFg?0?$AA@ 00000000316479e4     FaceEffector.obj
 0002:000059f0       ??_7?$TSpline@U?$SplineKey@M@spline@@VHermitBasis@2@@spline@@6B@ 00000000316479f0     FaceAnimSequence.obj
 0002:000059f0       ??_7?$TSpline@U?$SplineKey@M@spline@@U?$TCoeffBasis@M@2@@spline@@6B@ 00000000316479f0     FaceEffector.obj
 0002:00005a10       ??_7CFacialEffector@@6BIFacialEffector@@@ 0000000031647a10     FaceEffector.obj
 0002:00005ae0       ??_7CFacialEffectorAttachment@@6BIFacialEffector@@@ 0000000031647ae0     FaceEffector.obj
 0002:00005bc0       ??_7CFacialEffectorBone@@6B?$_i_reference_target@H@@@ 0000000031647bc0     FaceEffectorLibrary.obj
 0002:00005bc0       ??_7CFacialEffectorAttachment@@6B?$_i_reference_target@H@@@ 0000000031647bc0     FaceEffector.obj
 0002:00005bd8       ??_7?$CatmullRomSpline@MU?$SplineKey@M@spline@@$0A@@spline@@6B@ 0000000031647bd8     FaceEffector.obj
 0002:00005c00       ??_7?$CBaseSplineInterpolator@MV?$CatmullRomSpline@MU?$SplineKey@M@spline@@$0A@@spline@@@spline@@6BISplineInterpolator@@@ 0000000031647c00     FaceEffector.obj
 0002:00005cb0       ??_7?$SSplineBackup@V?$CatmullRomSpline@MU?$SplineKey@M@spline@@$0A@@spline@@@spline@@6BISplineBackup@@@ 0000000031647cb0     FaceEffector.obj
 0002:00005cc8       ??_7?$SSplineBackup@V?$CatmullRomSpline@MU?$SplineKey@M@spline@@$0A@@spline@@@spline@@6B?$CatmullRomSpline@MU?$SplineKey@M@spline@@$0A@@1@@ 0000000031647cc8     FaceEffector.obj
 0002:00005cf0       ??_7CFacialEffCtrlSplineInterpolator@@6BISplineInterpolator@@@ 0000000031647cf0     FaceEffector.obj
 0002:00005da0       ??_7?$CBaseSplineInterpolator@MV?$CatmullRomSpline@MU?$SplineKey@M@spline@@$0A@@spline@@@spline@@6B?$CatmullRomSpline@MU?$SplineKey@M@spline@@$0A@@1@@ 0000000031647da0     FaceEffector.obj
 0002:00005da0       ??_7CFacialEffCtrlSplineInterpolator@@6B?$CatmullRomSpline@MU?$SplineKey@M@spline@@$0A@@spline@@@ 0000000031647da0     FaceEffector.obj
 0002:00005dc0       ??_7CFacialEffCtrl@@6B?$_i_reference_target@H@@@ 0000000031647dc0     FaceEffector.obj
 0002:00005de0       ??_7CFacialEffCtrl@@6BIFacialEffCtrl@@@ 0000000031647de0     FaceEffector.obj
 0002:00005e58       ??_C@_07CIFAGBMG@unknown?$AA@ 0000000031647e58     FaceEffectorLibrary.obj
 0002:00005e60       ??_C@_08KNOEMJMM@material?$AA@ 0000000031647e60     FaceEffectorLibrary.obj
 0002:00005e70       ??_C@_0L@HBDHCFKP@attachment?$AA@ 0000000031647e70     FaceEffectorLibrary.obj
 0002:00005e7c       ??_C@_04ODKJLCFC@bone?$AA@ 0000000031647e7c     FaceEffectorLibrary.obj
 0002:00005e84       ??_C@_05NJNGEDKM@morph?$AA@ 0000000031647e84     FaceEffectorLibrary.obj
 0002:00005e90       ??_C@_0L@FKCCBALC@expression?$AA@ 0000000031647e90     FaceEffectorLibrary.obj
 0002:00005e9c       ??_C@_05MGJOOGAJ@group?$AA@ 0000000031647e9c     FaceEffectorLibrary.obj
 0002:00005ea8       ??_C@_07NPCLAIKJ@SubCtrl?$AA@ 0000000031647ea8     FaceEffectorLibrary.obj
 0002:00005eb0       ??_7CFacialEffectorsLibrary@@6B@ 0000000031647eb0     FaceEffectorLibrary.obj
 0002:00005f30       ??_C@_0EF@BALMIJNF@Attachment?5Effectors?5no?5longer?5s@ 0000000031647f30     FaceEffectorLibrary.obj
 0002:00005f80       ??_7CFacialMorphTarget@@6BIFacialEffector@@@ 0000000031647f80     FaceEffectorLibrary.obj
 0002:00006048       ??_7CFacialMorphTarget@@6B?$_i_reference_target@H@@@ 0000000031648048     FaceEffectorLibrary.obj
 0002:00006048       ??_7CFacialEffector@@6B?$_i_reference_target@H@@@ 0000000031648048     FaceEffector.obj
 0002:00006048       ??_7CFacialEffectorExpression@@6B?$_i_reference_target@H@@@ 0000000031648048     FaceEffectorLibrary.obj
 0002:00006060       ??_C@_04BAJDEDPD@Root?$AA@ 0000000031648060     FaceEffectorLibrary.obj
 0002:00006070       ??_7CFacialEffectorExpression@@6BIFacialEffector@@@ 0000000031648070     FaceEffectorLibrary.obj
 0002:00006140       ??_7CFacialEffectorBone@@6BIFacialEffector@@@ 0000000031648140     FaceEffectorLibrary.obj
 0002:00006220       ??_C@_0DE@HHGOBIHP@Attempting?5to?5merge?5library?5with@ 0000000031648220     FaceEffectorLibrary.obj
 0002:00006258       ??_C@_0M@INHKPGMC@Controllers?$AA@ 0000000031648258     FaceEffectorLibrary.obj
 0002:00006268       ??_C@_0N@MNPGGADE@AllEffectors?$AA@ 0000000031648268     FaceEffectorLibrary.obj
 0002:00006278       ??_C@_0CE@HJAMLKEC@Effector?5with?5name?5?$CFs?5already?5ex@ 0000000031648278     FaceEffectorLibrary.obj
 0002:000062a0       ??_7IFacialAnimation@@6B@  00000000316482a0     FaceAnimation.obj
 0002:000062a0       ??_7IJoystick@@6B@         00000000316482a0     FaceJoystick.obj
 0002:000062a0       ??_7IJoystickChannel@@6B@  00000000316482a0     FaceJoystick.obj
 0002:000062a0       ??_7IFacialEffectorsLibrary@@6B@ 00000000316482a0     FaceEffectorLibrary.obj
 0002:00006310       ??_7CFacialJoystickChannel@@6B@ 0000000031648310     FaceJoystick.obj
 0002:00006380       ??_7CFacialJoystick@@6B@   0000000031648380     FaceJoystick.obj
 0002:000063f0       ??_7CFacialJoystickSet@@6B@ 00000000316483f0     FaceJoystick.obj
 0002:00006450       ??_C@_01EANLCPLP@y?$AA@    0000000031648450     FaceJoystick.obj
 0002:00006454       ??_C@_01FJMABOPO@x?$AA@    0000000031648454     FaceJoystick.obj
 0002:00006458       ??_C@_0M@LNJPGNEG@VideoOffset?$AA@ 0000000031648458     FaceJoystick.obj
 0002:00006468       ??_C@_0L@EDKOHOLB@VideoScale?$AA@ 0000000031648468     FaceJoystick.obj
 0002:00006478       ??_C@_07MLKCHEME@Flipped?$AA@ 0000000031648478     FaceJoystick.obj
 0002:00006480       ??_C@_08FGBNDLMK@Vertical?$AA@ 0000000031648480     FaceJoystick.obj
 0002:00006490       ??_C@_0L@DKFGPADG@Horizontal?$AA@ 0000000031648490     FaceJoystick.obj
 0002:0000649c       ??_C@_04LBNBCLPC@Axis?$AA@ 000000003164849c     FaceJoystick.obj
 0002:000064a4       ??_C@_05PDOBBJNA@Color?$AA@ 00000000316484a4     FaceJoystick.obj
 0002:000064b0       ??_C@_08CJCDADNL@Joystick?$AA@ 00000000316484b0     FaceJoystick.obj
 0002:000064c0       ??_C@_0L@NDPLFEJ@Dimensions?$AA@ 00000000316484c0     FaceJoystick.obj
 0002:000064cc       ??_C@_06MCOJAMLH@Centre?$AA@ 00000000316484cc     FaceJoystick.obj
 0002:000064e0       ??_7IFacialInstance@@6B@   00000000316484e0     FacialInstance.obj
 0002:000064e0       ??_7IAttachmentManager@@6B@ 00000000316484e0     CharacterInstance.obj
 0002:00006580       ??_C@_0GI@FNHCCAAL@Loading?5facial?5animation?5sequenc@ 0000000031648580     FacialInstance.obj
 0002:000065f0       ??_C@_0GD@LMLLHIE@Loading?5facial?5animation?5sequenc@ 00000000316485f0     FacialInstance.obj
 0002:00006658       ??_C@_0BK@DLLBCJKE@Invalid?5layer?5passed?5?9?5?$CFd?$AA@ 0000000031648658     FacialInstance.obj
 0002:00006674       __real@3b03126f            0000000031648674     FacialInstance.obj
 0002:00006678       __real@3c9374bc            0000000031648678     FacialInstance.obj
 0002:00006680       ??_C@_0GF@FLEPIFBF@CFacialInstance?3?3TemporarilyEnab@ 0000000031648680     FacialInstance.obj
 0002:000066f0       ??_C@_0FE@MOCEADPK@CFacialInstance?3?3UpdateCurrentSe@ 00000000316486f0     FacialInstance.obj
 0002:00006750       ??_C@_0EK@LLJKCLIA@CFacialInstance?3?3UpdateCurrentSe@ 0000000031648750     FacialInstance.obj
 0002:000067a0       ??_C@_0EK@ELPDFMFO@CFacialInstance?3?3UpdateCurrentSe@ 00000000316487a0     FacialInstance.obj
 0002:000067f0       ??_C@_0ED@FDFFFADK@CFacialInstance?3?3UpdateCurrentSe@ 00000000316487f0     FacialInstance.obj
 0002:00006840       ??_C@_0FJ@KLEIDDPM@CFacialInstance?3?3UpdateCurrentSe@ 0000000031648840     FacialInstance.obj
 0002:000068a0       ??_C@_0DL@NALGPHFE@CFacialInstance?3?3Update?5?9?5?$CIthis?$DN@ 00000000316488a0     FacialInstance.obj
 0002:000068e0       ??_C@_0EA@HHOENHDP@CFacialInstance?3?3PlaySequence?$CIth@ 00000000316488e0     FacialInstance.obj
 0002:00006920       ??_C@_0EA@NGPEOLAA@CFacialInstance?3?3StopSequence?$CIth@ 0000000031648920     FacialInstance.obj
 0002:00006960       ??_C@_05NCABIDLI@Blink?$AA@ 0000000031648960     FacialInstance.obj
 0002:00006968       ??_C@_0CA@IIJMAECO@CFacialInstance?3?3Reset?$CIthis?$DN?$CFp?$CJ?$AA@ 0000000031648968     FacialInstance.obj
 0002:00006988       ??_C@_01KMDKNFGN@?1?$AA@   0000000031648988     FacialInstance.obj
 0002:00006990       ??_C@_0BA@HMOFIHLL@g_languageAudio?$AA@ 0000000031648990     FacialInstance.obj
 0002:000069a0       ??_7CFacialInstance@@6B?$_i_reference_target@H@@@ 00000000316489a0     FacialInstance.obj
 0002:000069c0       ??_7CFacialInstance@@6BIFacialInstance@@@ 00000000316489c0     FacialInstance.obj
 0002:00006a68       ??_7CFaceState@@6B?$_i_reference_target@H@@@ 0000000031648a68     FacialModel.obj
 0002:00006a80       ??_7CFaceState@@6BIFaceState@@@ 0000000031648a80     FacialModel.obj
 0002:00006a98       ??_C@_0CL@BGMIDNDI@Attachment?5Effectors?5not?5longer?5@ 0000000031648a98     FacialModel.obj
 0002:00006ac8       ??_C@_0CH@IOKJKNBL@CFacialModel?3?3FillInfoMapFromFac@ 0000000031648ac8     FacialModel.obj
 0002:00006af0       ??_7CFacialModel@@6B?$_i_reference_target@H@@@ 0000000031648af0     FacialModel.obj
 0002:00006b08       ??_7CFacialModel@@6BIFacialModel@@@ 0000000031648b08     FacialModel.obj
 0002:00006b40       ??_C@_08NJFLMLKA@pleasure?$AA@ 0000000031648b40     LipSync.obj
 0002:00006b4c       ??_C@_02PEPMCKME@zh?$AA@   0000000031648b4c     LipSync.obj
 0002:00006b50       ??_C@_03LMBDLIPK@zap?$AA@  0000000031648b50     LipSync.obj
 0002:00006b54       ??_C@_01GLPGHMHM@z?$AA@    0000000031648b54     LipSync.obj
 0002:00006b58       ??_C@_04BIGBAIKH@yard?$AA@ 0000000031648b58     LipSync.obj
 0002:00006b60       ??_C@_04MKNNKNJH@with?$AA@ 0000000031648b60     LipSync.obj
 0002:00006b68       ??_C@_01NOFIACDB@w?$AA@    0000000031648b68     LipSync.obj
 0002:00006b6c       ??_C@_03JCKJMCEG@vat?$AA@  0000000031648b6c     LipSync.obj
 0002:00006b70       ??_C@_01MHEDDDHA@v?$AA@    0000000031648b70     LipSync.obj
 0002:00006b74       ??_C@_03JLAIOMFN@too?$AA@  0000000031648b74     LipSync.obj
 0002:00006b78       ??_C@_02DCPKGDGH@uw?$AA@   0000000031648b78     LipSync.obj
 0002:00006b7c       ??_C@_04HMOIPFOL@book?$AA@ 0000000031648b7c     LipSync.obj
 0002:00006b84       ??_C@_02PPKAGNPJ@uh?$AA@   0000000031648b84     LipSync.obj
 0002:00006b88       ??_C@_04HHGFCHIH@thin?$AA@ 0000000031648b88     LipSync.obj
 0002:00006b90       ??_C@_02POGCAHMO@th?$AA@   0000000031648b90     LipSync.obj
 0002:00006b94       ??_C@_04HBNBFOKD@talk?$AA@ 0000000031648b94     LipSync.obj
 0002:00006b9c       ??_C@_01PFHFFBPC@t?$AA@    0000000031648b9c     LipSync.obj
 0002:00006ba0       ??_C@_03PJHPCKOL@she?$AA@  0000000031648ba0     LipSync.obj
 0002:00006ba4       ??_C@_02PLCNBBEL@sh?$AA@   0000000031648ba4     LipSync.obj
 0002:00006ba8       ??_C@_03KLGEGDMM@sit?$AA@  0000000031648ba8     LipSync.obj
 0002:00006bac       ??_C@_01LKDEMHDF@s?$AA@    0000000031648bac     LipSync.obj
 0002:00006bb0       ??_C@_03FAAAOPJM@red?$AA@  0000000031648bb0     LipSync.obj
 0002:00006bb4       ??_C@_01KDCPPGHE@r?$AA@    0000000031648bb4     LipSync.obj
 0002:00006bb8       ??_C@_03KMONJGDG@put?$AA@  0000000031648bb8     LipSync.obj
 0002:00006bbc       ??_C@_01JBBJJEPG@p?$AA@    0000000031648bbc     LipSync.obj
 0002:00006bc0       ??_C@_03IHJAFJIK@toy?$AA@  0000000031648bc0     LipSync.obj
 0002:00006bc4       ??_C@_02LNMIGIEP@oy?$AA@   0000000031648bc4     LipSync.obj
 0002:00006bc8       ??_C@_02KPEDIMCA@go?$AA@   0000000031648bc8     LipSync.obj
 0002:00006bcc       ??_C@_02CDELEFMB@ow?$AA@   0000000031648bcc     LipSync.obj
 0002:00006bd0       ??_C@_04KJHEDBDO@sing?$AA@ 0000000031648bd0     LipSync.obj
 0002:00006bd8       ??_C@_02GIELDNKH@ng?$AA@   0000000031648bd8     LipSync.obj
 0002:00006bdc       ??_C@_02KAJCLHKP@no?$AA@   0000000031648bdc     LipSync.obj
 0002:00006be0       ??_C@_01EFFIKLCJ@n?$AA@    0000000031648be0     LipSync.obj
 0002:00006be4       ??_C@_03BFLBBCNI@mat?$AA@  0000000031648be4     LipSync.obj
 0002:00006be8       ??_C@_01GOHFPIOK@m?$AA@    0000000031648be8     LipSync.obj
 0002:00006bec       ??_C@_03OJNMDGFE@lid?$AA@  0000000031648bec     LipSync.obj
 0002:00006bf0       ??_C@_01HHGOMJKL@l?$AA@    0000000031648bf0     LipSync.obj
 0002:00006bf4       ??_C@_01DICPFPGM@k?$AA@    0000000031648bf4     LipSync.obj
 0002:00006bf8       ??_C@_02OINKIJLE@jh?$AA@   0000000031648bf8     LipSync.obj
 0002:00006bfc       ??_C@_04KEADKAFO@feel?$AA@ 0000000031648bfc     LipSync.obj
 0002:00006c04       ??_C@_02LJEFBEPN@iy?$AA@   0000000031648c04     LipSync.obj
 0002:00006c08       ??_C@_04OBAECEGJ@fill?$AA@ 0000000031648c08     LipSync.obj
 0002:00006c10       ??_C@_02OKJMDHON@ih?$AA@   0000000031648c10     LipSync.obj
 0002:00006c14       ??_C@_04PCJFHION@help?$AA@ 0000000031648c14     LipSync.obj
 0002:00006c1c       ??_C@_01BDACAMKP@h?$AA@    0000000031648c1c     LipSync.obj
 0002:00006c20       ??_C@_03GBCDPJBA@gut?$AA@  0000000031648c20     LipSync.obj
 0002:00006c24       ??_C@_01JEJKBAGA@g?$AA@    0000000031648c24     LipSync.obj
 0002:00006c28       ??_C@_04JNJGGDAI@fork?$AA@ 0000000031648c28     LipSync.obj
 0002:00006c30       ??_C@_01INIBCBCB@f?$AA@    0000000031648c30     LipSync.obj
 0002:00006c34       ??_C@_03BGFDOPOL@ate?$AA@  0000000031648c34     LipSync.obj
 0002:00006c38       ??_C@_02LAFPONJJ@ey?$AA@   0000000031648c38     LipSync.obj
 0002:00006c3c       ??_C@_03IPMFDJPD@fur?$AA@  0000000031648c3c     LipSync.obj
 0002:00006c40       ??_C@_02FDKLDEFC@er?$AA@   0000000031648c40     LipSync.obj
 0002:00006c44       ??_C@_03LAMLDFEG@pet?$AA@  0000000031648c44     LipSync.obj
 0002:00006c48       ??_C@_02ODIGMOIJ@eh?$AA@   0000000031648c48     LipSync.obj
 0002:00006c4c       ??_C@_04HOHPNOOD@then?$AA@ 0000000031648c4c     LipSync.obj
 0002:00006c54       ??_C@_02OCEEKELO@dh?$AA@   0000000031648c54     LipSync.obj
 0002:00006c58       ??_C@_03HEFENHI@dig?$AA@   0000000031648c58     LipSync.obj
 0002:00006c5c       ??_C@_01LPLHEDKD@d?$AA@    0000000031648c5c     LipSync.obj
 0002:00006c60       ??_C@_04KFKFGMBF@chin?$AA@ 0000000031648c60     LipSync.obj
 0002:00006c68       ??_C@_02OHALLCDL@ch?$AA@   0000000031648c68     LipSync.obj
 0002:00006c6c       ??_C@_03CCCOBCKE@big?$AA@  0000000031648c6c     LipSync.obj
 0002:00006c70       ??_C@_01OJONOECF@b?$AA@    0000000031648c70     LipSync.obj
 0002:00006c74       ??_C@_04NHHDMLCI@bite?$AA@ 0000000031648c74     LipSync.obj
 0002:00006c7c       ??_C@_02LHFGEFEF@ay?$AA@   0000000031648c7c     LipSync.obj
 0002:00006c80       ??_C@_03PCNMBKEI@ago?$AA@  0000000031648c80     LipSync.obj
 0002:00006c84       ??_C@_02KOENHEAE@ax?$AA@   0000000031648c84     LipSync.obj
 0002:00006c88       ??_C@_04NHJIODEK@foul?$AA@ 0000000031648c88     LipSync.obj
 0002:00006c90       ??_C@_02CJNFGIML@aw?$AA@   0000000031648c90     LipSync.obj
 0002:00006c94       ??_C@_03DMIDBMK@dog?$AA@   0000000031648c94     LipSync.obj
 0002:00006c98       ??_C@_02KLMOPAJC@ao?$AA@   0000000031648c98     LipSync.obj
 0002:00006c9c       ??_C@_03OOEBGOEH@cut?$AA@  0000000031648c9c     LipSync.obj
 0002:00006ca0       ??_C@_02OEIPGGFF@ah?$AA@   0000000031648ca0     LipSync.obj
 0002:00006ca4       ??_C@_03PFGOGFOL@cat?$AA@  0000000031648ca4     LipSync.obj
 0002:00006ca8       ??_C@_02FBCBBIBI@ae?$AA@   0000000031648ca8     LipSync.obj
 0002:00006cac       ??_C@_06OIIIAOPN@father?$AA@ 0000000031648cac     LipSync.obj
 0002:00006cb4       ??_C@_02DFENNNBM@aa?$AA@   0000000031648cb4     LipSync.obj
 0002:00006cb8       ??_C@_0BF@EPOMEAHF@Silence?5?$CIunderscore?$CJ?$AA@ 0000000031648cb8     LipSync.obj
 0002:00006cd0       ??_C@_01IDAFKMJL@_?$AA@    0000000031648cd0     LipSync.obj
 0002:00006cd8       ??_C@_0CE@DOKFPDIK@Sentence?5terminator?5?$CIquestion?5ma@ 0000000031648cd8     LipSync.obj
 0002:00006cfc       ??_C@_01OGPIMHDM@?$DP?$AA@ 0000000031648cfc     LipSync.obj
 0002:00006d00       ??_C@_0BN@EKGECIKE@Sentence?5terminator?5?$CIperiod?$CJ?$AA@ 0000000031648d00     LipSync.obj
 0002:00006d20       ??_C@_0BM@CMAJFDHL@Sentence?5terminator?5?$CIcomma?$CJ?$AA@ 0000000031648d20     LipSync.obj
 0002:00006d3c       ??_C@_01HNPIGOCE@?$CG?$AA@ 0000000031648d3c     LipSync.obj
 0002:00006d40       ??_C@_0BE@PPDGDKBH@Sentence?5terminator?$AA@ 0000000031648d40     LipSync.obj
 0002:00006d54       ??_C@_01DCLJPIOD@?$CB?$AA@ 0000000031648d54     LipSync.obj
 0002:00006d58       ??_C@_08DMNNLLJJ@syllable?$AA@ 0000000031648d58     LipSync.obj
 0002:00006d64       ??_C@_01JOAMLHOP@?9?$AA@   0000000031648d64     LipSync.obj
 0002:00006d70       ??_7IJoystickContext@@6B@  0000000031648d70     FaceAnimation.obj
 0002:00006d70       ??_7IPlaceholderCharacter@@6B@ 0000000031648d70     PlaceholderCharacter.obj
 0002:00006d70       ??_7ICryUnknown@@6B@       0000000031648d70     OperatorQueue.obj
 0002:00006d70       ??_7IPhonemeLibrary@@6B@   0000000031648d70     LipSync.obj
 0002:00006d90       ??_7?$_reference_target@H@@6B@ 0000000031648d90     LipSync.obj
 0002:00006d98       __real@447a0000            0000000031648d98     LipSync.obj
 0002:00006da0       ??_C@_07OKOCHHP@?$CFs?3?$CF?42f?$AA@ 0000000031648da0     LipSync.obj
 0002:00006da8       ??_7CFacialSentence@@6B?$_reference_target@H@@@ 0000000031648da8     LipSync.obj
 0002:00006db0       ??_7CFacialSentence@@6BIFacialSentence@@@ 0000000031648db0     LipSync.obj
 0002:00006e18       ??_7CPhonemesLibrary@@6B@  0000000031648e18     LipSync.obj
 0002:00006e38       ??_C@_08BHPDILBD@?$CFd?3?$CFd?3?$CFs?$AA@ 0000000031648e38     LipSync.obj
 0002:00006e44       ??_C@_03DBKJMAGF@End?$AA@  0000000031648e44     LipSync.obj
 0002:00006e48       ??_C@_05FHMJPCKA@Start?$AA@ 0000000031648e48     LipSync.obj
 0002:00006e50       ??_C@_04IGEPOOPB@Word?$AA@ 0000000031648e50     LipSync.obj
 0002:00006e58       ??_C@_08PFDKLHBC@Phonemes?$AA@ 0000000031648e58     LipSync.obj
 0002:00006e64       ??_C@_05MOCOKHFB@Words?$AA@ 0000000031648e64     LipSync.obj
 0002:00006e6c       ??_C@_04OJAHODMC@Text?$AA@ 0000000031648e6c     LipSync.obj
 0002:00006e80       ??_7CFeetPoseRestore@@6B@  0000000031648e80     FeetLock.obj
 0002:00006ec0       ??_7CFeetPoseStore@@6B@    0000000031648ec0     FeetLock.obj
 0002:00006f00       ??_7CFactory@CFeetPoseStore@@6B@ 0000000031648f00     FeetLock.obj
 0002:00006f30       ??_C@_0CE@FIJHOGBC@AnimationPoseModifier_FeetPoseSt@ 0000000031648f30     FeetLock.obj
 0002:00006f58       ?cid@?1??GetClassID@CFactory@CFeetPoseStore@@UEBAAEBUCryGUID@@XZ@4U4@B 0000000031648f58     FeetLock.obj
 0002:00006f68       ??_7CFactory@CFeetPoseRestore@@6B@ 0000000031648f68     FeetLock.obj
 0002:00006f98       ??_C@_0CG@OHIIAMBF@AnimationPoseModifier_FeetPoseRe@ 0000000031648f98     FeetLock.obj
 0002:00006fc0       ?cid@?1??GetClassID@CFactory@CFeetPoseRestore@@UEBAAEBUCryGUID@@XZ@4U4@B 0000000031648fc0     FeetLock.obj
 0002:00006fd0       ??_C@_08OKNEMAIJ@RgtLeg01?$AA@ 0000000031648fd0     GroundAlignment.obj
 0002:00006fe0       ??_C@_08ECHMFJPE@LftLeg01?$AA@ 0000000031648fe0     GroundAlignment.obj
 0002:00006ff0       ??_C@_06DCFKOEPA@R?5Heel?$AA@ 0000000031648ff0     GroundAlignment.obj
 0002:00006ff8       ??_C@_06FLLADGD@L?5Heel?$AA@ 0000000031648ff8     GroundAlignment.obj
 0002:00007000       ?iid@?1??IID@IAnimationGroundAlignment@@CAAEBUCryGUID@@XZ@4U3@B 0000000031649000     GroundAlignment.obj
 0002:00007010       ??_7CGroundAlignment@@6B@  0000000031649010     GroundAlignment.obj
 0002:00007058       ??_7CFactory@CGroundAlignment@@6B@ 0000000031649058     GroundAlignment.obj
 0002:00007088       ??_C@_0CG@DDGGKLBL@AnimationPoseModifier_GroundAlig@ 0000000031649088     GroundAlignment.obj
 0002:000070b0       ?cid@?1??GetClassID@CFactory@CGroundAlignment@@UEBAAEBUCryGUID@@XZ@4U4@B 00000000316490b0     GroundAlignment.obj
 0002:000070d0       ??_7CLimbIk@@6B@           00000000316490d0     LimbIk.obj
 0002:00007110       ??_7CFactory@CLimbIk@@6B@  0000000031649110     LimbIk.obj
 0002:00007140       ?cid@?1??GetClassID@CFactory@CLimbIk@@UEBAAEBUCryGUID@@XZ@4U4@B 0000000031649140     LimbIk.obj
 0002:00007160       ??_7CPoseBlenderAim@@6B@   0000000031649160     PoseBlenderAim.obj
 0002:000071e8       __real@7f7fffff            00000000316491e8     PoseBlenderAim.obj
 0002:000071f0       ??_C@_0DF@INPOJLLI@CryAnimation?3?5No?5weapon?9bone?5spe@ 00000000316491f0     PoseBlenderAim.obj
 0002:00007228       ??_C@_0CL@CGDELOPI@CryAnimation?3?5No?5AimIK?9Setup?5for@ 0000000031649228     PoseBlenderAim.obj
 0002:00007258       ??_7CFactory@CPoseBlenderAim@@6B@ 0000000031649258     PoseBlenderAim.obj
 0002:00007288       ?cid@?1??GetClassID@CFactory@CPoseBlenderAim@@UEBAAEBUCryGUID@@XZ@4U4@B 0000000031649288     PoseBlenderAim.obj
 0002:0000729c       __real@3f3504f3            000000003164929c     PoseBlenderLook.obj
 0002:000072a0       ??_7CPoseBlenderLook@@6B@  00000000316492a0     PoseBlenderLook.obj
 0002:00007328       ??_C@_0DF@EGJAADOE@CryAnimation?3?5Right?5Eyeball?5atta@ 0000000031649328     PoseBlenderLook.obj
 0002:00007360       ??_C@_0DE@NBIDDDLC@CryAnimation?3?5Left?5Eyeball?5attac@ 0000000031649360     PoseBlenderLook.obj
 0002:00007398       ??_C@_0DD@CIEFHBDA@CryAnimation?3?5No?5look?9bone?5speci@ 0000000031649398     PoseBlenderLook.obj
 0002:000073d0       ??_C@_0CM@LFPKMBEO@CryAnimation?3?5No?5LookIK?9Setup?5fo@ 00000000316493d0     PoseBlenderLook.obj
 0002:00007400       ??_C@_0CF@OOHODMO@EyeRight?3?5?$CFf?5?$CFf?5?$CFf?5?$CFf?5?5m_IKBlend@ 0000000031649400     PoseBlenderLook.obj
 0002:00007428       ??_C@_0CE@DNOEJCJM@EyeLeft?3?5?$CFf?5?$CFf?5?$CFf?5?$CFf?5?5m_IKBlend?3@ 0000000031649428     PoseBlenderLook.obj
 0002:00007450       ??_7CFactory@CPoseBlenderLook@@6B@ 0000000031649450     PoseBlenderLook.obj
 0002:00007480       ?cid@?1??GetClassID@CFactory@CPoseBlenderLook@@UEBAAEBUCryGUID@@XZ@4U4@B 0000000031649480     PoseBlenderLook.obj
 0002:00007494       __real@bf7d70a4            0000000031649494     PoseModifierHelper.obj
 0002:00007498       __real@461c4000            0000000031649498     PoseModifierHelper.obj
 0002:0000749c       __real@3fa00000            000000003164949c     PoseModifierHelper.obj
 0002:000074a0       __real@3f7fff58            00000000316494a0     PoseModifierHelper.obj
 0002:000074a4       __real@2edbe6ff            00000000316494a4     PoseModifierHelper.obj
 0002:000074a8       __real@bf7ae148            00000000316494a8     PoseModifierHelper.obj
 0002:000074ac       __real@3e947ae1            00000000316494ac     PoseModifierHelper.obj
 0002:000074b0       __real@bf666666            00000000316494b0     PoseModifierHelper.obj
 0002:000074b4       __real@3f733333            00000000316494b4     PoseModifierHelper.obj
 0002:000074b8       __real@3f0ccccd            00000000316494b8     PoseModifierHelper.obj
 0002:000074bc       __real@3e99999a            00000000316494bc     PoseModifierHelper.obj
 0002:000074d0       ??_7CRecoil@PoseModifier@@6B@ 00000000316494d0     Recoil.obj
 0002:00007510       ??_7CFactory@CRecoil@PoseModifier@@6B@ 0000000031649510     Recoil.obj
 0002:00007540       ?cid@?1??GetClassID@CFactory@CRecoil@PoseModifier@@UEBAAEBUCryGUID@@XZ@4U5@B 0000000031649540     Recoil.obj
 0002:00007558       ??_C@_0DM@PBEMGCIH@CryAnimation?3?5Command?9Buffer?5Inv@ 0000000031649558     Command_Buffer.obj
 0002:00007598       ??_C@_0CB@ODGLIDOL@PartPose_FETCH_ADD?3?5w?3?$CFf?5t?3?$CFf?5?$CFs@ 0000000031649598     Command_Buffer.obj
 0002:000075c0       ??_C@_0CB@BFCOJGGE@BasePose_FETCH_ADD?3?5w?3?$CFf?5t?3?$CFf?5?$CFs@ 00000000316495c0     Command_Buffer.obj
 0002:000075e8       ??_C@_0CB@BDNGEMDG@PartAnim_FETCH_ADD?3?5w?3?$CFf?5t?3?$CFf?5?$CFs@ 00000000316495e8     Command_Buffer.obj
 0002:00007610       ??_C@_0BB@LGPJFNKO@Proc_POSEMOD?3?5?$CFs?$AA@ 0000000031649610     Command_Buffer.obj
 0002:00007628       ??_C@_0CB@OFJDFJLJ@BaseAnim_FETCH_ADD?3?5w?3?$CFf?5t?3?$CFf?5?$CFs@ 0000000031649628     Command_Buffer.obj
 0002:00007650       ??_C@_0BA@INCLFOHP@State_JOINTMASK?$AA@ 0000000031649650     Command_Buffer.obj
 0002:00007660       ??_C@_0BA@FCLDIGAF@BaseAnim_USCALE?$AA@ 0000000031649660     Command_Buffer.obj
 0002:00007670       ??_C@_0BD@GAMGPJMH@BaseAnim_NORMALIZE?$AA@ 0000000031649670     Command_Buffer.obj
 0002:00007688       ??_C@_0BC@HPHFEMMB@BaseAnim_COPY_ADD?$AA@ 0000000031649688     Command_Buffer.obj
 0002:000076a0       ??_C@_0BG@BNPBJNAD@BaseAnim_CLEAR_BUFFER?$AA@ 00000000316496a0     Command_Buffer.obj
 0002:000076b8       ??_C@_0BE@MKAOLHMH@BaseAnim_CLEAR_ROOT?$AA@ 00000000316496b8     Command_Buffer.obj
 0002:000076d0       ??_C@_0CI@DDCDLAMD@m_CommandBufferCounter?5?$CFd?5?5Comma@ 00000000316496d0     Command_Buffer.obj
 0002:000076f8       __real@3c75c28f            00000000316496f8     Command_Buffer.obj
 0002:00007700       ??_C@_0EI@GABFMADP@LHand_IKTarget?3?5name?3?5?$CFs?5?5rot?3?5?$CI@ 0000000031649700     Command_Buffer.obj
 0002:00007748       ??_C@_0BJ@OGGKAMHL@ProcessAnimationDrivenIk?$AA@ 0000000031649748     Command_Buffer.obj
 0002:00007768       ??_C@_0BK@OJHNFMAM@Command?3?3CBuffer?3?3Execute?$AA@ 0000000031649768     Command_Buffer.obj
 0002:00007788       ??_C@_09NEDHICLM@cryMemcpy?$AA@ 0000000031649788     Command_Commands.obj
 0002:000077a0       ??_C@_0EF@DIMOALKN@CryAnimation?3?5Asset?5Not?5Loaded?3?5@ 00000000316497a0     Command_Commands.obj
 0002:000077e8       ??_C@_0DJ@GIJGEOJH@illegal?5index?5in?5RSingleEvaluati@ 00000000316497e8     Command_Commands.obj
 0002:00007830       ??_7IAnimationPoseData@@6B@ 0000000031649830     Skeleton.obj
 0002:00007880       ??_7CPoseData@Skeleton@@6B@ 0000000031649880     Skeleton.obj
 0002:000078d0       ??_C@_0BE@BNBLBEIO@Character?5Pose?5Data?$AA@ 00000000316498d0     Skeleton.obj
 0002:000078e8       ??_C@_0BL@IJJIPNKE@Character?5Pose?5Data?5Cloned?$AA@ 00000000316498e8     Skeleton.obj
 0002:00007904       ??_C@_06HOPIODND@effect?$AA@ 0000000031649904     AnimEventLoader.obj
 0002:0000790c       ??_C@_04MEMAJGDJ@name?$AA@ 000000003164990c     AnimEventLoader.obj
 0002:00007918       ??_C@_09KCBFNMAJ@animation?$AA@ 0000000031649918     AnimEventLoader.obj
 0002:00007928       ??_C@_0L@OBDHBINM@AnimEvents?$AA@ 0000000031649928     AnimEventLoader.obj
 0002:00007934       ??_C@_06HPGEIPLA@?$DMnull?$DO?$AA@ 0000000031649934     CharacterManager.obj
 0002:00007940       ??_C@_07KAALEJHI@?$DMlocal?$DO?$AA@ 0000000031649940     CharacterManager.obj
 0002:00007950       ??_7ICharacterManager@@6B@ 0000000031649950     CharacterManager.obj
 0002:00007ac0       ??_C@_04PBAHLACE@File?$AA@ 0000000031649ac0     CharacterManager.obj
 0002:00007ac8       ??_C@_05NFIJOKEG@Model?$AA@ 0000000031649ac8     CharacterManager.obj
 0002:00007ad0       ??_C@_0DH@OHPBLIHM@CryAnimation?3?5character?9definiti@ 0000000031649ad0     CharacterManager.obj
 0002:00007b08       ??_C@_0BE@OLDKOMJJ@CharacterDefinition?$AA@ 0000000031649b08     CharacterManager.obj
 0002:00007b20       ??_C@_0BE@NPEDKBDG@Character?5instances?$AA@ 0000000031649b20     CharacterManager.obj
 0002:00007b34       __real@42000000            0000000031649b34     CharacterManager.obj
 0002:00007b38       ??_C@_0DG@FKBAHALH@nSkinningPoolSize?3?5?$CFd?5?5?5nTotalSk@ 0000000031649b38     CharacterManager.obj
 0002:00007b70       ??_C@_0BO@LHHDLBCA@TotalModelMemory?5?$CIMem?3?5?$CF4dKB?$CJ?$AA@ 0000000031649b70     CharacterManager.obj
 0002:00007b90       ??_C@_0EF@KLPBKCHC@nTotalModelSkeletonMemory?3?5?5?$CF4dK@ 0000000031649b90     CharacterManager.obj
 0002:00007bd8       ??_C@_0BG@NGMNAJGJ@nAnimationSet?3?5?5?$CF4dKB?$AA@ 0000000031649bd8     CharacterManager.obj
 0002:00007bf0       ??_C@_0DO@PPBPJBDK@nTotalAttachmentMemory?3?5?5?$CF4dKB?5?5@ 0000000031649bf0     CharacterManager.obj
 0002:00007c30       ??_C@_0FK@NEDBHHJB@?9?9?9?9?9?9?9?9?9?9?9?9?9?9?9?9?9?9?9?9?9?9?9?9?9?9?9?9?9?9?9?9@ 0000000031649c30     CharacterManager.obj
 0002:00007c90       ??_C@_0EJ@GCNGJGJK@SKINInstancesCounter?3?$CF3d?5?$CIMem?3?5?$CF@ 0000000031649c90     CharacterManager.obj
 0002:00007ce0       ??_C@_0DI@OOFGLCFP@Model?3?5?$CF3d?5?5Skin?3?5?$CF2d?5imem?3?5?$CF7d?5@ 0000000031649ce0     CharacterManager.obj
 0002:00007d20       ??_C@_0FC@DGAPPCGC@Model?3?5?$CF3d?5?5?5Skin?3?5?$CF2d?5imem?3?5?$CF7d@ 0000000031649d20     CharacterManager.obj
 0002:00007d80       ??_C@_0EE@PDECEPPA@Model?3?5?$CF3d?5?5?5Skel?3?5?$CF2d?5?5imem?3?5?$CF7@ 0000000031649d80     CharacterManager.obj
 0002:00007dd0       ??_C@_0ED@JOJCFEF@Model?3?5?$CF3d?5?5?5Skel?3?5?$CF2d?5imem?3?5?$CF7d@ 0000000031649dd0     CharacterManager.obj
 0002:00007e20       ??_C@_0EJ@GJGEHJGL@SKELInstancesCounter?3?$CF3d?5?$CIMem?3?5?$CF@ 0000000031649e20     CharacterManager.obj
 0002:00007e70       ??_C@_0BN@PLJJFMHL@CryAnimation?3?5mem?5corruption?$AA@ 0000000031649e70     CharacterManager.obj
 0002:00007e90       ??_C@_0CP@PHGEPJJL@No?3?$CF04d?5DBA?3?5?$CF08x?5p?3?$CF02x?5q?3?$CF02x?5@ 0000000031649e90     CharacterManager.obj
 0002:00007ec0       ??_C@_02BKFDOEMK@wt?$AA@   0000000031649ec0     CharacterManager.obj
 0002:00007ec8       ??_C@_0BH@FONECNPF@No?3?$CF04d?5use?3?$CF05d?5?5?5?$CFs?6?$AA@ 0000000031649ec8     CharacterManager.obj
 0002:00007ee0       ??_C@_07OANIALAE@chr?4pak?$AA@ 0000000031649ee0     CharacterManager.obj
 0002:00007ee8       ??_C@_0DN@FEBKIFHJ@?$DN?$DN?$DN?$DN?$DN?5Finished?5Preloading?5?$CFd?5Cha@ 0000000031649ee8     CharacterManager.obj
 0002:00007f28       ??_C@_0CB@FCAIPGCG@?$DN?$DN?$DN?$DN?$DN?5Preloading?5Characters?5?$DN?$DN?$DN?$DN@ 0000000031649f28     CharacterManager.obj
 0002:00007f50       ??_C@_0M@JKINLGFJ@Preload?5CHR?$AA@ 0000000031649f50     CharacterManager.obj
 0002:00007f60       ??_C@_0CD@PDHBIC@CharacterManager?3?3PreloadModelsC@ 0000000031649f60     CharacterManager.obj
 0002:00007f88       ??_C@_0CE@BFGBHKLO@CharacterManager?3?3RegisterModelS@ 0000000031649f88     CharacterManager.obj
 0002:00007fb0       ??_C@_0CE@COENOBFI@CharacterManager?3?3RegisterModelS@ 0000000031649fb0     CharacterManager.obj
 0002:00007fd8       ??_C@_0DA@INOLIAEE@CryAnimation?3?5Reloading?5CHRPARAM@ 0000000031649fd8     CharacterManager.obj
 0002:00008008       ??_C@_02JDPG@rb?$AA@       000000003164a008     CharacterManager.obj
 0002:00008010       ??_C@_0DH@NAEANFNA@?$DN?$DN?$DN?$DN?$DN?5Finished?5Preloading?5?$CFd?5CGA@ 000000003164a010     CharacterManager.obj
 0002:00008048       ??_C@_07JDNCALNI@cga?4pak?$AA@ 000000003164a048     CharacterManager.obj
 0002:00008050       ??_C@_0M@ECJONIAD@e_StreamCgf?$AA@ 000000003164a050     CharacterManager.obj
 0002:00008060       ??_C@_0BL@FJEOOLEB@?$DN?$DN?$DN?$DN?$DN?5Preloading?5CGAs?5?$DN?$DN?$DN?$DN?$AA@ 000000003164a060     CharacterManager.obj
 0002:00008080       ??_C@_0M@PADOLAPG@Preload?5CGA?$AA@ 000000003164a080     CharacterManager.obj
 0002:00008090       ??_C@_0CD@GKEAHHCN@CharacterManager?3?3PreloadModelsC@ 000000003164a090     CharacterManager.obj
 0002:000080b8       ??_C@_0BC@MGOEEFL@Animation?5Context?$AA@ 000000003164a0b8     CharacterManager.obj
 0002:000080d0       ??_C@_0BE@KJDJFMJA@STL?5Allocator?5Waste?$AA@ 000000003164a0d0     CharacterManager.obj
 0002:000080e8       ??_C@_0L@HKIBOMFD@Model?5Data?$AA@ 000000003164a0e8     CharacterManager.obj
 0002:000080f8       ??_C@_0BB@KDBPHKIO@Facial?5Animation?$AA@ 000000003164a0f8     CharacterManager.obj
 0002:00008110       ??_7CharacterDefinition@@6B@ 000000003164a110     CharacterManager.obj
 0002:00008120       ??_C@_0EN@FCGGFBPH@CryAnimation?3?5no?5valid?5character@ 000000003164a120     CharacterManager.obj
 0002:00008170       ??_C@_0CA@DDELBMIL@CharacterManager?3?3LoadModelSKIN?$AA@ 000000003164a170     CharacterManager.obj
 0002:00008190       ??_C@_0L@EMODJLOD@Characters?$AA@ 000000003164a190     CharacterManager.obj
 0002:000081a0       ??_C@_0BK@GOFBGCI@AnimStats_NotUsed_LMG?4txt?$AA@ 000000003164a1a0     CharacterManager.obj
 0002:000081c0       ??_C@_0BH@KNBMFCMI@AnimStats_Used_LMG?4txt?$AA@ 000000003164a1c0     CharacterManager.obj
 0002:000081d8       ??_C@_0BK@NDDJLNFF@AnimStats_NotUsed_CAF?4txt?$AA@ 000000003164a1d8     CharacterManager.obj
 0002:000081f8       ??_C@_0BH@HIMAPJLF@AnimStats_Used_CAF?4txt?$AA@ 000000003164a1f8     CharacterManager.obj
 0002:00008210       ??_C@_0DD@FOOMPIDA@Anim?3?$CI?$CFd?$CJ?5?5Force?3?$CI?$CFd?$CJ?5?5Visible?3?$CI@ 000000003164a210     CharacterManager.obj
 0002:00008248       ??_C@_0CL@PHOJHIIJ@Instances?5with?5?8Force?5Skeleton?5U@ 000000003164a248     CharacterManager.obj
 0002:00008278       ??_C@_0BE@IOBGFPOI@SkeletonUpdates?3?5?$CFd?$AA@ 000000003164a278     CharacterManager.obj
 0002:00008290       ??_C@_0BF@GGOPHLKB@AnimationUpdates?3?5?$CFd?$AA@ 000000003164a290     CharacterManager.obj
 0002:000082a8       ??_C@_0DE@NJMNECHC@nAnimsPerFrame?3?5?$CF4d?5?5nAnimsMax?3?5@ 000000003164a2a8     CharacterManager.obj
 0002:000082e0       ??_C@_0BD@GAAEDFAB@arrModelCache?3?5?$CF4d?$AA@ 000000003164a2e0     CharacterManager.obj
 0002:000082f8       ??_C@_0BM@MAHCAFAA@arrModelCache_CharEdit?3?5?$CF4d?$AA@ 000000003164a2f8     CharacterManager.obj
 0002:00008318       ??_C@_0BJ@CDDMONIK@CharacterManager?3?3Update?$AA@ 000000003164a318     CharacterManager.obj
 0002:00008338       ??_7CAnimationManager@@6B@ 000000003164a338     CharacterManager.obj
 0002:00008370       ??_C@_0FF@MKPLPECI@m_arrModelCacheSKEL?5is?5supposed?5@ 000000003164a370     CharacterManager.obj
 0002:000083c8       ??_C@_0BN@NPJPGGNA@m_arrModelCacheSKEL?$FL?$CFi?$FN?5?$DN?5?$CFs?$AA@ 000000003164a3c8     CharacterManager.obj
 0002:000083f0       ??_C@_0FF@JBCJLFOE@m_arrModelCacheSKIN?5is?5supposed?5@ 000000003164a3f0     CharacterManager.obj
 0002:00008448       ??_C@_0BN@ICPJJCJA@m_arrModelCacheSKIN?$FL?$CFi?$FN?5?$DN?5?$CFs?$AA@ 000000003164a448     CharacterManager.obj
 0002:00008468       ??_C@_0DM@MHCCPBPK@CharacterManager?3CleanModelCache@ 000000003164a468     CharacterManager.obj
 0002:000084b0       ??_C@_0IA@BDKJANBB@?$CKERROR?$CK?5CharacterManager?3?5?$CFu?5bod@ 000000003164a4b0     CharacterManager.obj
 0002:00008530       ??_7CharacterManager@@6B@  000000003164a530     CharacterManager.obj
 0002:000086a0       ??_C@_0EK@FKCNNNGO@CryAnimation?3?5Assets?5has?5no?5cont@ 000000003164a6a0     CharacterManager.obj
 0002:000086f0       ??_C@_0ED@MKCPEGIJ@CryAnimation?3?5m_arrController?5re@ 000000003164a6f0     CharacterManager.obj
 0002:00008740       ??_C@_0FA@NJADGAO@CryAnimation?3?5CRC32?5Invalid?$CB?5Mos@ 000000003164a740     CharacterManager.obj
 0002:00008790       ??_C@_0CP@INOEFHAC@Badly?5exported?5animation?9asset?3?5@ 000000003164a790     CharacterManager.obj
 0002:000087c0       ??_C@_0DO@NPPJMPBB@CryAnimation?3?5the?5list?5with?5Glob@ 000000003164a7c0     CharacterManager.obj
 0002:00008800       ??_C@_0CM@LCFLJELM@CharacterManager?3?3LoadAnimationI@ 000000003164a800     CharacterManager.obj
 0002:00008830       ??_C@_0BD@HNEEBJGG@InternalPara1D?4LMG?$AA@ 000000003164a830     CharacterManager.obj
 0002:00008844       ??_C@_03IGKKBKKP@CDF?$AA@  000000003164a844     CharacterManager.obj
 0002:00008848       ??_C@_0BK@JFFBIKHL@CharacterManager?3?3LoadCDF?$AA@ 000000003164a848     CharacterManager.obj
 0002:00008868       ??_C@_0DB@BLBFJBND@CryAnimation?3?5character?9definiti@ 000000003164a868     CharacterManager.obj
 0002:000088a0       ??_C@_0DH@NELFFEPE@?$DN?$DN?$DN?$DN?$DN?5Finished?5Preloading?5?$CFd?5CDF@ 000000003164a8a0     CharacterManager.obj
 0002:000088d8       ??_C@_04BCMGGOLH@?4cdf?$AA@ 000000003164a8d8     CharacterManager.obj
 0002:000088e0       ??_C@_0BL@GKAGNOJN@?$DN?$DN?$DN?$DN?$DN?5Preloading?5CDFs?5?$DN?$DN?$DN?$DN?$AA@ 000000003164a8e0     CharacterManager.obj
 0002:00008900       ??_C@_0M@LNDJJIGI@Preload?5CDF?$AA@ 000000003164a900     CharacterManager.obj
 0002:00008910       ??_C@_0CD@CHEHFPLD@CharacterManager?3?3PreloadModelsC@ 000000003164a910     CharacterManager.obj
 0002:00008938       ??_C@_0BI@HJHCIGLK@CDF?4?5Finish?4?5Memstat?5?$CFi?$AA@ 000000003164a938     CharacterManager.obj
 0002:00008950       ??_C@_0CD@BPIDLBGP@Couldn?8t?5create?5base?9character?3?5@ 000000003164a950     CharacterManager.obj
 0002:00008980       ??_C@_0EG@MOMOBCLL@CryAnimation?3?5base?9character?5mus@ 000000003164a980     CharacterManager.obj
 0002:000089c8       ??_C@_0BK@KNHFHPBF@CDF?5?$CFs?4?5Start?4?5Memstat?5?$CFi?$AA@ 000000003164a9c8     CharacterManager.obj
 0002:000089e8       ??_C@_0CK@IOKDEHCE@CharacterManager?3?3LoadCharacterD@ 000000003164a9e8     CharacterManager.obj
 0002:00008a18       ??_C@_0BD@KHKNKNFF@Preload?5Characters?$AA@ 000000003164aa18     CharacterManager.obj
 0002:00008a30       ??_C@_0CF@NAMGPPIA@CharacterManager?3?3PreloadLevelMo@ 000000003164aa30     CharacterManager.obj
 0002:00008a58       ??_C@_0CI@JGBNBLAB@Badly?5exported?5aim?9pose?3?5flags?3?5@ 000000003164aa58     CharacterManager.obj
 0002:00008a80       ??_C@_0CJ@JOOFGFDA@CharacterManager?3?3LoadAnimationI@ 000000003164aa80     CharacterManager.obj
 0002:00008ab0       ??_C@_0BK@HHIKGHID@animations?1animations?4img?$AA@ 000000003164aab0     CharacterManager.obj
 0002:00008ad0       ??_C@_0CB@NMEJACKB@animations?1DirectionalBlends?4img@ 000000003164aad0     CharacterManager.obj
 0002:00008b00       ??_C@_0GM@HDENCGKJ@CryAnimation?3FetchPlaceHolderCha@ 000000003164ab00     CharacterManager.obj
 0002:00008b70       ??_C@_0GM@DALBFNHC@CryAnimation?3FetchPlaceHolderCha@ 000000003164ab70     CharacterManager.obj
 0002:00008be0       ??_C@_0GM@EHJLEEIM@CryAnimation?3FetchPlaceHolderCha@ 000000003164abe0     CharacterManager.obj
 0002:00008c50       ??_C@_0GO@DIGNOCFO@CryAnimation?3FetchPlaceHolderCha@ 000000003164ac50     CharacterManager.obj
 0002:00008cc0       ??_C@_0GI@BKIDNJII@CryAnimation?3FetchPlaceHolderCha@ 000000003164acc0     CharacterManager.obj
 0002:00008d28       ??_C@_0BF@COJDDOIE@Instances?5Memstat?5?$CFi?$AA@ 000000003164ad28     CharacterManager.obj
 0002:00008d40       ??_C@_0BP@OLGKDIDE@InitCGAInstance?5?$CFs?4?5Memstat?5?$CFi?$AA@ 000000003164ad40     CharacterManager.obj
 0002:00008d60       ??_C@_0P@DIBCHGHO@Loading?5CGA?5?$CFs?$AA@ 000000003164ad60     CharacterManager.obj
 0002:00008d70       ??_C@_0CE@KMAAOPHC@CharacterManager?3?3CreateCGAInsta@ 000000003164ad70     CharacterManager.obj
 0002:00008d98       ??_C@_09EEDOMAPA@chrparams?$AA@ 000000003164ad98     CharacterManager.obj
 0002:00008da8       ??_C@_0CF@KCPFIJAI@CharacterManager?3?3CreateSKELInst@ 000000003164ada8     CharacterManager.obj
 0002:00008dd0       ??_C@_0CA@IGHIHGN@CharacterManager?3?3LoadModelSKEL?$AA@ 000000003164add0     CharacterManager.obj
 0002:00008df0       ??_C@_0DD@LHBEEHJA@CharacterManager?3?3FetchPlaceHold@ 000000003164adf0     CharacterManager.obj
 0002:00008e30       ??_C@_0FI@LOPBNJDN@CPF?5file?5allowed?5for?5use?5only?5in@ 000000003164ae30     CharacterManager.obj
 0002:00008e88       ??_C@_04BHIIPFEC@base?$AA@ 000000003164ae88     CharacterManager.obj
 0002:00008e90       ??_C@_0EB@CIMONDIL@CryAnimation?3?5no?5valid?5character@ 000000003164ae90     CharacterManager.obj
 0002:00008ed4       ??_C@_03JAHONMHP@cpf?$AA@  000000003164aed4     CharacterManager.obj
 0002:00008ed8       ??_C@_0DM@JCMOKGDP@CryAnimation?3PrefetchCharacterRe@ 000000003164aed8     CharacterManager.obj
 0002:00008f14       ??_C@_04DOHGOLCD@$lod?$AA@ 000000003164af14     LoaderCGA.obj
 0002:00008f20       ??_C@_0CK@PIMHCPOB@Animation?5could?5not?5be?5read?5for?5@ 000000003164af20     LoaderCGA.obj
 0002:00008f50       ??_7IController@@6B@       000000003164af50     LoaderCGA.obj
 0002:00008fc8       ??_C@_0CC@LPDMFHBH@indices?5and?1or?5positions?5are?5NUL@ 000000003164afc8     LoaderCGA.obj
 0002:00008ff0       ??_C@_0CO@BKPCLEDN@faces?5are?5too?5small?5or?5have?5stre@ 000000003164aff0     LoaderCGA.obj
 0002:00009020       ??_C@_0BK@MMDPIIJG@bad?5vertex?5index?5detected?$AA@ 000000003164b020     LoaderCGA.obj
 0002:0000903c       ?minTexArea@?1???$ComputeTexMappingAreas@U?$Vec3_tpl@M@@USMeshTexCoord@@@CMeshHelpers@@SA_N_KPEBG0PEBU?$Vec3_tpl@M@@0PEBUSMeshTexCoord@@0AEAM4AEAPEBD@Z@4MB 000000003164b03c     LoaderCGA.obj
 0002:0000903c       __real@33d6bf95            000000003164b03c     SkeletonAnim_Locator.obj
 0002:00009040       ??_C@_0BG@BDLCLLKE@bad?5number?5of?5indices?$AA@ 000000003164b040     LoaderCGA.obj
 0002:00009058       ??_C@_0BN@KFBFLIPO@texture?5coordinates?5are?5NULL?$AA@ 000000003164b058     LoaderCGA.obj
 0002:00009078       ??_C@_0BC@HPECBPJJ@vertex?5count?5is?50?$AA@ 000000003164b078     LoaderCGA.obj
 0002:00009090       ??_C@_0BB@IGNNBDOM@index?5count?5is?50?$AA@ 000000003164b090     LoaderCGA.obj
 0002:000090a8       ??_C@_0BB@ELKAEEPN@missing?5vertices?$AA@ 000000003164b0a8     LoaderCGA.obj
 0002:000090c0       ??_C@_0BM@IFOLHLJG@missing?5texture?5coordinates?$AA@ 000000003164b0c0     LoaderCGA.obj
 0002:000090e0       ??_C@_0CB@HMHDCALB@missing?5or?5bad?5indices?5in?5subset@ 000000003164b0e0     LoaderCGA.obj
 0002:00009108       ??_C@_0BA@PAFHHGGK@missing?5indices?$AA@ 000000003164b108     LoaderCGA.obj
 0002:00009118       ??_C@_0BE@KHFBNAHK@subset?5index?5is?5bad?$AA@ 000000003164b118     LoaderCGA.obj
 0002:00009130       ??_C@_0L@CPDIKD@L?5UpperArm?$AA@ 000000003164b130     LoaderCGA.obj
 0002:00009140       ??_C@_0L@PMKPNHGO@R?5UpperArm?$AA@ 000000003164b140     LoaderCGA.obj
 0002:00009150       ??_C@_07LDJNDMEG@L?5Thigh?$AA@ 000000003164b150     LoaderCGA.obj
 0002:00009158       ??_C@_07NKKMBPFP@R?5Thigh?$AA@ 000000003164b158     LoaderCGA.obj
 0002:00009160       ??_7?$TSpline@UTCBAngAxisKey@spline@@VHermitBasis@2@@spline@@6B@ 000000003164b160     LoaderCGA.obj
 0002:00009180       ??_7TCBAngleAxisSpline@spline@@6B@ 000000003164b180     LoaderCGA.obj
 0002:000091a8       __real@3f7ff972            000000003164b1a8     LoaderCGA.obj
 0002:000091ac       __real@40c90fbb            000000003164b1ac     LoaderCGA.obj
 0002:000091b0       __real@3ea2f983            000000003164b1b0     LoaderCGA.obj
 0002:000091b4       __real@40490fb1            000000003164b1b4     LoaderCGA.obj
 0002:000091c0       ??_7CControllerTCB@@6B@    000000003164b1c0     LoaderCGA.obj
 0002:00009238       ??_C@_0BE@OMJLCPFJ@Should?5never?5happen?$AA@ 000000003164b238     LoaderCGA.obj
 0002:00009250       ??_C@_0N@HOBCLLKA@CharacterCGA?$AA@ 000000003164b250     LoaderCGA.obj
 0002:00009260       ??_C@_0CG@HICNHCLM@Cannot?5be?5merged?5to?5one?5skin?5ins@ 000000003164b260     LoaderCGA.obj
 0002:00009288       __real@3bcccccd            000000003164b288     LoaderCGA.obj
 0002:00009290       ??_C@_0BM@PFEDBNEJ@Failed?5to?5load?5ANM?9file?3?5?$CFs?$AA@ 000000003164b290     LoaderCGA.obj
 0002:000092b0       ??_C@_0L@KIBGKOJH@animevents?$AA@ 000000003164b2b0     LoaderCGA.obj
 0002:000092bc       ??_C@_04BEANKMFM@?4caf?$AA@ 000000003164b2bc     LoaderCGA.obj
 0002:000092c4       ??_C@_04FGKMPKCB@?4anm?$AA@ 000000003164b2c4     LoaderCGA.obj
 0002:000092cc       ??_C@_02FNAGIBCP@?4?$CK?$AA@ 000000003164b2cc     LoaderCGA.obj
 0002:000092d0       ??_C@_02IDFIDEI@_?$CK?$AA@ 000000003164b2d0     LoaderCGA.obj
 0002:000092d8       ??_C@_0BN@DPJAHDFM@CryCGALoader?3?3LoadAnimations?$AA@ 000000003164b2d8     LoaderCGA.obj
 0002:000092f8       ??_C@_07MCAEODGB@Default?$AA@ 000000003164b2f8     LoaderCGA.obj
 0002:00009300       ??_C@_0BK@LLFPEIEJ@Failed?5to?5load?5CGA?9Object?$AA@ 000000003164b300     LoaderCGA.obj
 0002:0000931c       ??_C@_03MLKNDCDB@CGA?$AA@  000000003164b31c     LoaderCGA.obj
 0002:00009330       __mask@@AbsDouble@         000000003164b330     LoaderCHR.obj
 0002:00009340       ??_C@_0CC@GEHLENNH@CryCHRLoader?3?3ReuseAnimationFile@ 000000003164b340     LoaderCHR.obj
 0002:00009368       ??_C@_0L@HNGMIHEN@animations?$AA@ 000000003164b368     LoaderCHR.obj
 0002:00009378       ??_C@_0M@HJLLEEH@?1animations?$AA@ 000000003164b378     LoaderCHR.obj
 0002:00009390       ??_C@_0FE@LAHILELP@CryAnimation?3?5Matrix?9Tangents?5ar@ 000000003164b390     LoaderCHR.obj
 0002:000093e8       ??_C@_0DL@PNJAKJAP@Facial?5Effector?5Library?5?$CFs?5not?5f@ 000000003164b3e8     LoaderCHR.obj
 0002:00009428       ??_C@_0BK@HAILMHKA@CryCHRLoader?3?3LoadFaceLib?$AA@ 000000003164b428     LoaderCHR.obj
 0002:00009448       ??_C@_0CO@KOEOJBCH@Physics?3?5Failed?5to?5create?5phys?5m@ 000000003164b448     LoaderCHR.obj
 0002:00009478       ??_C@_0BP@DMCHIPGL@Physics?3?5No?5material?5in?5lod?5?$CFd?$AA@ 000000003164b478     LoaderCHR.obj
 0002:000094a0       ??_C@_0EL@JHAFEIHE@Animation?5?$CIcaf?$CJ?5file?5?$CC?$CFs?$CC?5could?5@ 000000003164b4a0     LoaderCHR.obj
 0002:000094ec       ??_C@_04JDMOLDHM@comb?$AA@ 000000003164b4ec     LoaderCHR.obj
 0002:000094f4       ??_C@_06NLFPJIBA@bspace?$AA@ 000000003164b4f4     LoaderCHR.obj
 0002:000094fc       ??_C@_03MFPIMNEL@lmg?$AA@  000000003164b4fc     LoaderCHR.obj
 0002:00009500       ??_C@_03INJKBFDI@caf?$AA@  000000003164b500     LoaderCHR.obj
 0002:00009508       ??_C@_0CN@IKHFBIPF@The?5GlobalID?5of?5the?5default?5Para@ 000000003164b508     LoaderCHR.obj
 0002:00009538       ??_C@_0CB@KOBLDDLL@CryCHRLoader?3?3LoadAnimationFiles@ 000000003164b538     LoaderCHR.obj
 0002:0000955c       ??_C@_04MKMLCMBL@?4fxl?$AA@ 000000003164b55c     LoaderCHR.obj
 0002:00009568       ??_C@_0L@MMMPLAFM@Memstat?5?$CFi?$AA@ 000000003164b568     LoaderCHR.obj
 0002:00009578       ??_C@_0DA@OMGLPLED@?5?5?$CFd?5animation?9assets?5loaded?5?$CIto@ 000000003164b578     LoaderCHR.obj
 0002:000095a8       ??_C@_0BN@PKLOMKFG@CryCHRLoader?3?3LoadAnimations?$AA@ 000000003164b5a8     LoaderCHR.obj
 0002:000095d0       ??_C@_0GD@BIOBFDCL@Default?9Skeleton?5has?5wrong?5orien@ 000000003164b5d0     LoaderCHR.obj
 0002:00009638       __real@3fc1eb8520000000    000000003164b638     LoaderCHR.obj
 0002:00009640       ??_C@_0BO@NBIMBHLL@CryAnimation?3?5assetDefinedLOD?$AA@ 000000003164b640     LoaderCHR.obj
 0002:00009660       ??_C@_0CF@CFMJFCCB@CryAnimation?3?5m_nBaseLOD?5should?5@ 000000003164b660     LoaderCHR.obj
 0002:00009688       ??_C@_0BJ@MBHDKFEE@CryCHRLoader?3?3LoadNewCHR?$AA@ 000000003164b688     LoaderCHR.obj
 0002:000096a8       ??_7IControllerRelocatableChain@@6B@ 000000003164b6a8     LoaderDBA.obj
 0002:000096c0       ??_7CControllerOptNonVirtual@@6B@ 000000003164b6c0     LoaderDBA.obj
 0002:00009798       ??_7CInternalDatabaseInfo@@6BIControllerRelocatableChain@@@ 000000003164b798     LoaderDBA.obj
 0002:000097a8       ??_7CInternalDatabaseInfo@@6BIStreamCallback@@@ 000000003164b7a8     LoaderDBA.obj
 0002:000097c8       ??_C@_0DO@PFPEONFD@Failed?5To?5Load?5Animation?5DBA?5?8?$CFs@ 000000003164b7c8     LoaderDBA.obj
 0002:00009808       ??_C@_0CO@KBAEHNDD@ERROR?0?5controller?5array?5size?5to?5@ 000000003164b808     LoaderDBA.obj
 0002:00009838       ??_C@_0N@BCCFIHEB@ALL?5DBAs?5?$CFli?$AA@ 000000003164b838     LoaderDBA.obj
 0002:00009848       ??_C@_0BJ@PIMHMAGK@Current?5DBA?4?5Memstat?5?$CFli?$AA@ 000000003164b848     LoaderDBA.obj
 0002:00009868       ??_C@_0CJ@FLLKFPPC@ReadController903?4?5Finished?4?5Mem@ 000000003164b868     LoaderDBA.obj
 0002:00009898       ??_C@_0P@JDIHECOA@Invalid?5GAH?5ID?$AA@ 000000003164b898     LoaderDBA.obj
 0002:000098a8       ??_C@_0BH@EOMBJNOG@DBA?1CAF?5mismatch?5in?5?$CFs?$AA@ 000000003164b8a8     LoaderDBA.obj
 0002:000098c0       ??_C@_0BD@GOOKFDHB@GAH?5does?5not?5exist?$AA@ 000000003164b8c0     LoaderDBA.obj
 0002:000098e0       ??_C@_0EM@EGJGGEMM@Going?5to?5create?5a?5CAF?5header?5on?5@ 000000003164b8e0     LoaderDBA.obj
 0002:00009930       ??_C@_0DI@FCIOEJBO@ReadController905?4?5All?5dynamic?5d@ 000000003164b930     LoaderDBA.obj
 0002:00009968       ??_C@_0BH@MGGDIFFJ@Empty?5controller?5found?$AA@ 000000003164b968     LoaderDBA.obj
 0002:00009980       ??_C@_0CN@JCHDIHHA@ReadController905?4?5TracksResize?4@ 000000003164b980     LoaderDBA.obj
 0002:000099b0       ??_C@_0CF@NHHPDLLA@ReadController905?4?5Init?4?5Memstat@ 000000003164b9b0     LoaderDBA.obj
 0002:000099d8       ??_C@_0CD@MLCMJLOB@error?3?5could?5not?5allocate?5?$CFd?5byt@ 000000003164b9d8     LoaderDBA.obj
 0002:00009a00       ??_C@_0CJ@JICLBEBF@CInternalDatabaseInfo?3?3ReadContr@ 000000003164ba00     LoaderDBA.obj
 0002:00009a30       ??_C@_0FE@CEPIMKIH@CryAnimation?3?5unknown?5chunk?9vers@ 000000003164ba30     LoaderDBA.obj
 0002:00009a90       ??_C@_0FN@ECGHOMFI@CryAnimation?3?5ReadController904?5@ 000000003164ba90     LoaderDBA.obj
 0002:00009af0       ??_C@_0FN@CKAOPOAN@CryAnimation?3?5ReadController903?5@ 000000003164baf0     LoaderDBA.obj
 0002:00009b50       ??_C@_0FN@HKLNJENB@CryAnimation?3?5ReadController902?5@ 000000003164bb50     LoaderDBA.obj
 0002:00009bb0       ??_C@_0FN@NLNLEBGJ@CryAnimation?3?5ReadController900?5@ 000000003164bbb0     LoaderDBA.obj
 0002:00009c10       ??_C@_0BG@GCJJICEA@Failed?5to?5load?5chunks?$AA@ 000000003164bc10     LoaderDBA.obj
 0002:00009c28       ??_C@_0CA@EIBOCEEG@Illegal?5File?5Type?5for?5?4dba?5file?$AA@ 000000003164bc28     LoaderDBA.obj
 0002:00009c48       ??_C@_0BF@EDAFHOON@Bad?5DBA?5file?5version?$AA@ 000000003164bc48     LoaderDBA.obj
 0002:00009c60       ??_C@_0BN@NCKMPNBB@Failed?5to?5stream?5DBA?9file?5?$CFx?$AA@ 000000003164bc60     LoaderDBA.obj
 0002:00009c80       ??_C@_0CN@IKNFBJGB@CInternalDatabaseInfo?3?3StreamAsy@ 000000003164bc80     LoaderDBA.obj
 0002:00009cb0       ??_7CController@@6B@       000000003164bcb0     LoaderTCB.obj
 0002:00009d28       ??_7ITrackInformation@@6B@ 000000003164bd28     LoaderTCB.obj
 0002:00009d40       ??_7IPositionController@@6B@ 000000003164bd40     LoaderTCB.obj
 0002:00009d90       ??_7IRotationController@@6B@ 000000003164bd90     LoaderTCB.obj
 0002:00009de0       ??_C@_0ED@CKLAKBPH@Data?5Error?5in?5Win32?5Build?3?5CAF?5f@ 000000003164bde0     LoaderTCB.obj
 0002:00009e28       ??_C@_0BF@GKLLIPEB@ReadMotionParameters?$AA@ 000000003164be28     LoaderTCB.obj
 0002:00009e40       ??_7?$CAdvancedTrackInformation@U?$Quat_tpl@M@@UQuatLerp@@VIRotationController@@@@6B@ 000000003164be40     LoaderTCB.obj
 0002:00009e90       ??_7?$CAdvancedTrackInformation@U?$Vec3_tpl@M@@UVec3Lerp@@VIPositionController@@@@6B@ 000000003164be90     LoaderTCB.obj
 0002:00009ed8       ??_7CHeaderTCB@@6B@        000000003164bed8     LoaderTCB.obj
 0002:00009ee0       ??_C@_0EB@MAFIPHCH@animation?5not?5loaded?3?5found?5unsu@ 000000003164bee0     LoaderTCB.obj
 0002:00009f30       ??_C@_0EB@DGECOHO@animation?5not?5loaded?3?5controller@ 000000003164bf30     LoaderTCB.obj
 0002:00009f80       ??_C@_0EB@CPCKOGLC@animation?5not?5loaded?3?5controller@ 000000003164bf80     LoaderTCB.obj
 0002:00009fc8       ??_C@_0BL@HNEFPEED@CONTROLLER_CHUNK_DESC_0828?$AA@ 000000003164bfc8     LoaderTCB.obj
 0002:00009fe8       ??_C@_0CE@HPJMHPKM@Illegal?5File?5Type?5for?5?4caf?5file?3@ 000000003164bfe8     LoaderTCB.obj
 0002:0000a010       ??_C@_0BJ@BFJPNJCO@Bad?5CAF?5file?5version?3?5?$CFs?$AA@ 000000003164c010     LoaderTCB.obj
 0002:0000a030       ??_C@_06BNNOMDLO@Handle?$AA@ 000000003164c030     ParamLoader.obj
 0002:0000a038       ??_C@_09OBHIPIHP@LIKHandle?$AA@ 000000003164c038     ParamLoader.obj
 0002:0000a048       ??_C@_09NIBPEJCE@RIKHandle?$AA@ 000000003164c048     ParamLoader.obj
 0002:0000a058       ??_C@_08GAHNGDIJ@IKHandle?$AA@ 000000003164c058     ParamLoader.obj
 0002:0000a068       ??_C@_0BL@DCAKIFLJ@CParamLoader?3?3MemFindFirst?$AA@ 000000003164c068     ParamLoader.obj
 0002:0000a088       ??_C@_0BG@PLFGIMMI@Failure?5for?5weight?5?$CFs?$AA@ 000000003164c088     ParamLoader.obj
 0002:0000a0a0       ??_C@_0N@HIPKJGLI@nWeightIdx?$DO0?$AA@ 000000003164c0a0     ParamLoader.obj
 0002:0000a0b0       ??_C@_0BG@NAMCFIGE@Failure?5for?5target?5?$CFs?$AA@ 000000003164c0b0     ParamLoader.obj
 0002:0000a0c8       ??_C@_0N@PLPGFIAE@nTargetIdx?$DO0?$AA@ 000000003164c0c8     ParamLoader.obj
 0002:0000a0d8       ??_C@_06FGANPIPG@Target?$AA@ 000000003164c0d8     ParamLoader.obj
 0002:0000a0e0       ??_C@_0L@CGLHJMHG@ADIKTarget?$AA@ 000000003164c0e0     ParamLoader.obj
 0002:0000a0ec       ??_C@_05ENDOMFAI@Delay?$AA@ 000000003164c0ec     ParamLoader.obj
 0002:0000a0f4       ??_C@_03HKDFLGGP@Arm?$AA@  000000003164c0f4     ParamLoader.obj
 0002:0000a0f8       ??_C@_0M@LDCHAHBG@ImpactJoint?$AA@ 000000003164c0f8     ParamLoader.obj
 0002:0000a108       ??_C@_0N@PAHFLIGD@ImpactJoints?$AA@ 000000003164c108     ParamLoader.obj
 0002:0000a118       ??_C@_0N@FIINBKCH@LWeaponJoint?$AA@ 000000003164c118     ParamLoader.obj
 0002:0000a128       ??_C@_09KOHFDMLF@JointName?$AA@ 000000003164c128     ParamLoader.obj
 0002:0000a138       ??_C@_0N@BGGMLAEN@RWeaponJoint?$AA@ 000000003164c138     ParamLoader.obj
 0002:0000a148       ??_C@_0CI@NKKGJNAP@CryAnimation?5Error?3?5Look?9Poses?5d@ 000000003164c148     ParamLoader.obj
 0002:0000a170       ??_C@_0EL@DBLACMEL@Look?9Pose?5Error?3?5Reference?5Joint@ 000000003164c170     ParamLoader.obj
 0002:0000a1c0       ??_C@_0P@GAPEMHIJ@ReferenceJoint?$AA@ 000000003164c1c0     ParamLoader.obj
 0002:0000a1d0       ??_C@_0EI@MLODPBJP@Look?9Pose?5Error?3?5?5Start?5JointNam@ 000000003164c1d0     ParamLoader.obj
 0002:0000a218       ??_C@_0L@MNFJAMCB@StartJoint?$AA@ 000000003164c218     ParamLoader.obj
 0002:0000a230       ??_C@_0EB@NBLLANHO@Look?9Pose?5Error?3?5JointName?5?8?$CFs?8?5@ 000000003164c230     ParamLoader.obj
 0002:0000a278       ??_C@_0P@MGJAFNBF@ParameterJoint?$AA@ 000000003164c278     ParamLoader.obj
 0002:0000a288       ??_C@_09JFBKCAJ@AnimToken?$AA@ 000000003164c288     ParamLoader.obj
 0002:0000a294       ??_C@_05LEKIHFJL@Joint?$AA@ 000000003164c294     ParamLoader.obj
 0002:0000a2a0       ??_C@_0BC@IAPMCPPH@DirectionalBlends?$AA@ 000000003164c2a0     ParamLoader.obj
 0002:0000a2b8       ??_C@_0N@CNHHKGI@PositionList?$AA@ 000000003164c2b8     ParamLoader.obj
 0002:0000a2c8       ??_C@_08NGDGBBLG@Additive?$AA@ 000000003164c2c8     ParamLoader.obj
 0002:0000a2d8       ??_C@_07NAEHBBNL@Primary?$AA@ 000000003164c2d8     ParamLoader.obj
 0002:0000a2e0       ??_C@_0DA@BNADLPKC@JointName?5?8?$CFs?8?5for?5Look?9Pose?5not@ 000000003164c2e0     ParamLoader.obj
 0002:0000a310       ??_C@_0N@FIGHJKFE@RotationList?$AA@ 000000003164c310     ParamLoader.obj
 0002:0000a320       ??_C@_04GIAGJOJD@para?$AA@ 000000003164c320     ParamLoader.obj
 0002:0000a328       ??_C@_03PHODBHCN@FOV?$AA@  000000003164c328     ParamLoader.obj
 0002:0000a330       ??_C@_0P@CFGKLJDI@REyeAttachment?$AA@ 000000003164c330     ParamLoader.obj
 0002:0000a340       ??_C@_0P@IMHLDOAC@LEyeAttachment?$AA@ 000000003164c340     ParamLoader.obj
 0002:0000a350       ??_C@_0CH@OGOIEFLC@CryAnimation?5Error?3?5Aim?9Poses?5di@ 000000003164c350     ParamLoader.obj
 0002:0000a380       ??_C@_0EO@GJJJEFKH@Aim?9Pose?5Error?3?5ProcAdjustment?5J@ 000000003164c380     ParamLoader.obj
 0002:0000a3d0       ??_C@_0BA@HINOHKMB@ProcAdjustments?$AA@ 000000003164c3d0     ParamLoader.obj
 0002:0000a3e0       ??_C@_0EJ@PPFJJBLB@Aim?9Pose?5Error?3?5Reference?5JointN@ 000000003164c3e0     ParamLoader.obj
 0002:0000a430       ??_C@_0EE@PGDKGCKI@Aim?9Pose?5Error?3?5StartJointName?5?8@ 000000003164c430     ParamLoader.obj
 0002:0000a478       ??_C@_0DP@LDLOABDK@Aim?9Pose?5Error?3?5JointName?5?8?$CFs?8?5f@ 000000003164c478     ParamLoader.obj
 0002:0000a4b8       ??_C@_03EMIMMIHL@?$CK?4?$CK?$AA@ 000000003164c4b8     ParamLoader.obj
 0002:0000a4c0       ??_C@_0BC@KHIBCMBD@Failure?5for?5J4?5?$CFs?$AA@ 000000003164c4c0     ParamLoader.obj
 0002:0000a4d8       ??_C@_08HCPLBCDA@nJ4Idx?$DO0?$AA@ 000000003164c4d8     ParamLoader.obj
 0002:0000a4e4       ??_C@_02MGJJNNAM@J4?$AA@   000000003164c4e4     ParamLoader.obj
 0002:0000a4e8       ??_C@_0BC@BFKBPAAD@Failure?5for?5J3?5?$CFs?$AA@ 000000003164c4e8     ParamLoader.obj
 0002:0000a500       ??_C@_08LHFMCMLO@nJ3Idx?$DO0?$AA@ 000000003164c500     ParamLoader.obj
 0002:0000a50c       ??_C@_02IJNIELML@J3?$AA@   000000003164c50c     ParamLoader.obj
 0002:0000a510       ??_C@_09MCEHMCIG@For?5J2?5?$CFs?$AA@ 000000003164c510     ParamLoader.obj
 0002:0000a520       ??_C@_08BBCLCHAK@nJ2Idx?$DO0?$AA@ 000000003164c520     ParamLoader.obj
 0002:0000a52c       ??_C@_02JAMDHKIK@J2?$AA@   000000003164c52c     ParamLoader.obj
 0002:0000a530       ??_C@_09IFOHLIFG@For?5J1?5?$CFs?$AA@ 000000003164c530     ParamLoader.obj
 0002:0000a540       ??_C@_08CAMDDNJH@nJ1Idx?$DO0?$AA@ 000000003164c540     ParamLoader.obj
 0002:0000a54c       ??_C@_02LLOOCJEJ@J1?$AA@   000000003164c54c     ParamLoader.obj
 0002:0000a550       ??_C@_09LIIHJBOG@For?5J0?5?$CFs?$AA@ 000000003164c550     ParamLoader.obj
 0002:0000a560       ??_C@_08IGLEDGCD@nJ0Idx?$DO0?$AA@ 000000003164c560     ParamLoader.obj
 0002:0000a56c       ??_C@_02KCPFBIAI@J0?$AA@   000000003164c56c     ParamLoader.obj
 0002:0000a570       ??_C@_0P@JNLINEBF@nMaxInteration?$AA@ 000000003164c570     ParamLoader.obj
 0002:0000a580       ??_C@_0L@ELELNKBI@fThreshold?$AA@ 000000003164c580     ParamLoader.obj
 0002:0000a590       ??_C@_09JJEBABC@fStepSize?$AA@ 000000003164c590     ParamLoader.obj
 0002:0000a5a0       ??_C@_0M@KANHEFDJ@EndEffector?$AA@ 000000003164c5a0     ParamLoader.obj
 0002:0000a5ac       ??_C@_06MIIPBJJH@Solver?$AA@ 000000003164c5ac     ParamLoader.obj
 0002:0000a5b4       ??_C@_02GMHIAGGM@IK?$AA@   000000003164c5b4     ParamLoader.obj
 0002:0000a5b8       ??_C@_0BO@JNONGKEO@CParamLoader?3?3ExpandWildcards?$AA@ 000000003164c5b8     ParamLoader.obj
 0002:0000a5d8       ??_C@_05KJNJLLGA@level?$AA@ 000000003164c5d8     ParamLoader.obj
 0002:0000a5e0       ??_C@_09FEGAOKFA@JointList?$AA@ 000000003164c5e0     ParamLoader.obj
 0002:0000a5f0       ??_C@_0BB@PKMHEMPI@AimIK_Definition?$AA@ 000000003164c5f0     ParamLoader.obj
 0002:0000a608       ??_C@_0BC@OMKLAMBI@LookIK_Definition?$AA@ 000000003164c608     ParamLoader.obj
 0002:0000a620       ??_C@_0BC@MHDOBOAO@Recoil_Definition?$AA@ 000000003164c620     ParamLoader.obj
 0002:0000a638       ??_C@_0BE@HPIABMHN@FeetLock_Definition?$AA@ 000000003164c638     ParamLoader.obj
 0002:0000a650       ??_C@_0BM@JLBGLKEH@Animation_Driven_IK_Targets?$AA@ 000000003164c650     ParamLoader.obj
 0002:0000a670       ??_C@_0BC@LKENIJBM@LimbIK_Definition?$AA@ 000000003164c670     ParamLoader.obj
 0002:0000a688       ??_C@_0O@GCHJNOID@IK_Definition?$AA@ 000000003164c688     ParamLoader.obj
 0002:0000a698       ??_C@_07DHMEHIPB@?5?7?6?$AN?0?$CI?$CJ?$AA@ 000000003164c698     ParamLoader.obj
 0002:0000a6a0       ??_C@_06EDBFFAMA@?5?7?6?$AN?$DN?$CI?$AA@ 000000003164c6a0     ParamLoader.obj
 0002:0000a6b0       ??_C@_0FB@CKLBBPDE@Failed?5to?5create?5animation?5alias@ 000000003164c6b0     ParamLoader.obj
 0002:0000a704       ??_C@_05GFOLEBJA@?$CFs?1?$CFs?$AA@ 000000003164c704     ParamLoader.obj
 0002:0000a710       ??_C@_0BK@FGLKMAKN@Deprecated?5directive?5?$CC?$CFs?$CC?$AA@ 000000003164c710     ParamLoader.obj
 0002:0000a730       ??_C@_0BK@PIIOJFFC@Unknown?5directive?5in?5?8?$CFs?8?$AA@ 000000003164c730     ParamLoader.obj
 0002:0000a750       ??_C@_0DN@FAJPOACF@Failed?5to?5set?5face?5lib?5?$CC?$CFs?$CC?4?5Fac@ 000000003164c750     ParamLoader.obj
 0002:0000a790       ??_C@_08BKGFCPAD@$FaceLib?$AA@ 000000003164c790     ParamLoader.obj
 0002:0000a7a0       ??_C@_0O@PNFLLIOM@AnimationList?$AA@ 000000003164c7a0     ParamLoader.obj
 0002:0000a7b0       ??_C@_06MGHLEEEG@Params?$AA@ 000000003164c7b0     ParamLoader.obj
 0002:0000a7b8       ??_C@_08PCKHJNII@$Include?$AA@ 000000003164c7b8     ParamLoader.obj
 0002:0000a7c8       ??_C@_0L@DLDGMDEL@persistent?$AA@ 000000003164c7c8     ParamLoader.obj
 0002:0000a7d4       ??_C@_05GECEPKB@flags?$AA@ 000000003164c7d4     ParamLoader.obj
 0002:0000a7e0       ??_C@_0CO@HDNFLOKE@Duplicate?5model?5tracks?5database?5@ 000000003164c7e0     ParamLoader.obj
 0002:0000a810       ??_C@_0BA@FHGJMAGE@$TracksDatabase?$AA@ 000000003164c810     ParamLoader.obj
 0002:0000a820       ??_C@_0BD@CPBAAOIB@$AnimEventDatabase?$AA@ 000000003164c820     ParamLoader.obj
 0002:0000a838       ??_C@_0P@DEBICNIP@$AnimDirectory?$AA@ 000000003164c838     ParamLoader.obj
 0002:0000a848       ??_C@_0BE@CDPOIOIF@$AnimationDirectory?$AA@ 000000003164c848     ParamLoader.obj
 0002:0000a860       ??_C@_08PIHFAEOK@$AnimDir?$AA@ 000000003164c860     ParamLoader.obj
 0002:0000a870       ??_C@_0O@LIIBPCBH@$AnimationDir?$AA@ 000000003164c870     ParamLoader.obj
 0002:0000a880       ??_C@_04LOAJBDKD@true?$AA@ 000000003164c880     ParamLoader.obj
 0002:0000a888       ??_C@_0BB@JJMFGJMC@?$CDParseSubFolders?$AA@ 000000003164c888     ParamLoader.obj
 0002:0000a8a0       ??_C@_09MIHJIFBG@?$CDfilepath?$AA@ 000000003164c8a0     ParamLoader.obj
 0002:0000a8ac       ??_C@_05EJAMACJC@?5?7?6?$AN?$DN?$AA@ 000000003164c8ac     ParamLoader.obj
 0002:0000a8b4       ??_C@_04LNEJFJGI@path?$AA@ 000000003164c8b4     ParamLoader.obj
 0002:0000a8c0       ??_C@_09ONEINPNJ@Animation?$AA@ 000000003164c8c0     ParamLoader.obj
 0002:0000a8cc       ??_C@_05GPNABNFL@null?1?$AA@ 000000003164c8cc     ParamLoader.obj
 0002:0000a8d8       ??_C@_0BL@PPLFDBBD@CParamLoader?3?3LoadAnimList?$AA@ 000000003164c8d8     ParamLoader.obj
 0002:0000a8f8       ??_C@_0BO@DIJIECID@Failed?5to?5load?5animations?3?5?$CFs?$AA@ 000000003164c8f8     ParamLoader.obj
 0002:0000a918       ??_C@_03ENGDOFNI@Lod?$AA@  000000003164c918     ParamLoader.obj
 0002:0000a920       ??_C@_0BG@CANMHDPD@CParamLoader?3?3LoadXML?$AA@ 000000003164c920     ParamLoader.obj
 0002:0000a938       __real@5f800000            000000003164c938     Compression.obj
 0002:0000a940       ??_C@_0M@FAGLBHGK@mat_default?$AA@ 000000003164c940     Model.obj
 0002:0000a950       ??_7ICharacterModel@@6B@   000000003164c950     Model.obj
 0002:0000a9f8       ??_7IFacialAnimSkeletonAnimationEntry@@6B@ 000000003164c9f8     FaceAnimSequence.obj
 0002:0000a9f8       ??_7IAnimEventList@@6B@    000000003164c9f8     AnimEventList.obj
 0002:0000a9f8       ??_7ICharacterModelSkeleton@@6B@ 000000003164c9f8     Model.obj
 0002:0000a9f8       ??_7IAnimEvents@@6B@       000000003164c9f8     CharacterManager.obj
 0002:0000a9f8       ??_7IFacialModel@@6B@      000000003164c9f8     FacialModel.obj
 0002:0000aa30       ??_C@_06FOHEPPJH@sphere?$AA@ 000000003164ca30     Model.obj
 0002:0000aa38       ??_C@_07FJIOKKEJ@capsule?$AA@ 000000003164ca38     Model.obj
 0002:0000aa40       ??_C@_08GNLJBPEP@cylinder?$AA@ 000000003164ca40     Model.obj
 0002:0000aa4c       ??_C@_03OLPJGAII@box?$AA@  000000003164ca4c     Model.obj
 0002:0000aa50       ??_C@_0M@NKEMBHLE@DampingAnim?$AA@ 000000003164ca50     Model.obj
 0002:0000aa60       ??_C@_0BD@JFPAJNFL@StiffnessDecayAnim?$AA@ 000000003164ca60     Model.obj
 0002:0000aa78       ??_C@_0O@KLKDFFAF@StiffnessAnim?$AA@ 000000003164ca78     Model.obj
 0002:0000aa88       ??_C@_0O@MCPAABAE@AirResistance?$AA@ 000000003164ca88     Model.obj
 0002:0000aa98       ??_C@_0O@KEGAKDKO@StiffnessTang?$AA@ 000000003164ca98     Model.obj
 0002:0000aaa8       ??_C@_0O@IBDMOJCA@StiffnessNorm?$AA@ 000000003164caa8     Model.obj
 0002:0000aab8       ??_C@_0L@CLKEODIP@MaxStretch?$AA@ 000000003164cab8     Model.obj
 0002:0000aac8       ??_C@_0BF@JLJEJDNJ@StiffnessControlBone?$AA@ 000000003164cac8     Model.obj
 0002:0000aae0       ??_C@_09CEKHLCFH@Thickness?$AA@ 000000003164cae0     Model.obj
 0002:0000aaec       ??_C@_04EIIBPIEA@Mass?$AA@ 000000003164caec     Model.obj
 0002:0000aaf8       ??_C@_0P@JHEAKJPO@BodyCollisions?$AA@ 000000003164caf8     Model.obj
 0002:0000ab08       ??_C@_0O@KEMNECCG@EnvCollisions?$AA@ 000000003164cb08     Model.obj
 0002:0000ab18       ??_C@_0P@ELOPBDHG@SimpleBlending?$AA@ 000000003164cb18     Model.obj
 0002:0000ab28       ??_C@_08DIMMEHEB@Friction?$AA@ 000000003164cb28     Model.obj
 0002:0000ab38       ??_C@_07HJKIPEFI@Damping?$AA@ 000000003164cb38     Model.obj
 0002:0000ab40       ??_C@_0P@MPIGCMMH@StiffnessDecay?$AA@ 000000003164cb40     Model.obj
 0002:0000ab50       ??_C@_09GCCJCEDC@Stiffness?$AA@ 000000003164cb50     Model.obj
 0002:0000ab60       ??_C@_0M@DHGMMGNF@MaxTimestep?$AA@ 000000003164cb60     Model.obj
 0002:0000ab70       ??_C@_0BD@NEJDDAMA@JointLimitIncrease?$AA@ 000000003164cb70     Model.obj
 0002:0000ab88       ??_C@_0L@IEFEJNGD@JointLimit?$AA@ 000000003164cb88     Model.obj
 0002:0000ab98       ??_C@_07JMGDFJEK@Gravity?$AA@ 000000003164cb98     Model.obj
 0002:0000aba0       ??_C@_0M@JFHCMOIP@cloth_proxy?$AA@ 000000003164cba0     Model.obj
 0002:0000abb0       ??_C@_0O@JNEDNOB@CollisionInfo?$AA@ 000000003164cbb0     Model.obj
 0002:0000abc0       ??_C@_0M@MLNNNIFK@FacialModel?$AA@ 000000003164cbc0     Model.obj
 0002:0000abd0       ??_C@_0O@BPDDIHEF@AnimationSets?$AA@ 000000003164cbd0     Model.obj
 0002:0000abe0       ??_C@_0O@FNBEOPPF@ModelSkeleton?$AA@ 000000003164cbe0     Model.obj
 0002:0000abf0       ??_7CModelSkeleton@@6B?$_reference_target@H@@@ 000000003164cbf0     Model.obj
 0002:0000abf8       ??_7CModelSkeleton@@6BICharacterModelSkeleton@@@ 000000003164cbf8     Model.obj
 0002:0000ac30       ??_7CSkel@@6B@             000000003164cc30     Model.obj
 0002:0000ace0       ??_C@_0BC@BCDELJLP@CSkel?5Release?3?5?$CFs?$AA@ 000000003164cce0     Model.obj
 0002:0000ad00       ??_C@_0FH@BFCNOANF@The?5model?5?8?$CFs?8?5still?5has?5?$CFd?5skel@ 000000003164cd00     Model.obj
 0002:0000ad60       ??_7IAnimationSet@@6B@     000000003164cd60     ModelAnimationSet.obj
 0002:0000ae88       ??_C@_0CH@KKJIOKKC@Invalid?5Animation?5ID?3?5?$CFd?5for?5Mod@ 000000003164ce88     ModelAnimationSet.obj
 0002:0000aeb0       ??_C@_0CH@GBJHKOKG@CAnimationSet?3?3GetModelAnimation@ 000000003164ceb0     ModelAnimationSet.obj
 0002:0000aed8       ??_C@_0BI@FLFIHPFJ@?$CBNEGATIVE?5ANIMATION?5ID?$CB?$AA@ 000000003164ced8     ModelAnimationSet.obj
 0002:0000aef0       ??_C@_0BM@ICDIPNOO@?$CBANIMATION?5ID?5OUT?5OF?5RANGE?$CB?$AA@ 000000003164cef0     ModelAnimationSet.obj
 0002:0000af10       ??_C@_0CL@CAADJKCO@illegal?5animation?5index?5?8?$CFd?8?5for@ 000000003164cf10     ModelAnimationSet.obj
 0002:0000af40       ??_C@_0EL@IGFMDGNC@illegal?5animation?5index?5used?5in?5@ 000000003164cf40     ModelAnimationSet.obj
 0002:0000af90       ??_C@_0EO@LPMHKCIG@illegal?5animation?5index?5used?5in?5@ 000000003164cf90     ModelAnimationSet.obj
 0002:0000afe0       ??_C@_0EG@LPAFCHLM@illegal?5animation?5index?5used?5in?5@ 000000003164cfe0     ModelAnimationSet.obj
 0002:0000b028       ??_C@_0DB@IBBOCMGJ@animation?9name?5not?5in?5cal?9file?3?5@ 000000003164d028     ModelAnimationSet.obj
 0002:0000b060       ??_C@_0BL@HBHKFCBB@?$CBNEGATIVE?5MORPH?5TARGET?5ID?$CB?$AA@ 000000003164d060     ModelAnimationSet.obj
 0002:0000b080       ??_C@_0EE@HMPGHNOG@CAnimationSet?3?3GetAnimationDCCWo@ 000000003164d080     ModelAnimationSet.obj
 0002:0000b0d0       ??_C@_0EA@LJNOOANO@CAnimationSet?3?3GetAnimationDCCWo@ 000000003164d0d0     ModelAnimationSet.obj
 0002:0000b110       ??_C@_0CG@ECBPIFCO@illegal?5joint?5index?3?5?$CFd?5for?5Mode@ 000000003164d110     ModelAnimationSet.obj
 0002:0000b138       ??_C@_0DC@BICBPBBO@animation?9name?5?8?$CFs?8?5not?5in?5CAL?9f@ 000000003164d138     ModelAnimationSet.obj
 0002:0000b170       ??_C@_0EG@GLAOHHAM@?$CL?$CL?$CL?$CL?5Trying?5to?5get?5StartLocation@ 000000003164d170     ModelAnimationSet.obj
 0002:0000b1b8       ??_C@_0CE@KIHHODMM@CryAnimation?3?5CAL?9file?5loaded?5tw@ 000000003164d1b8     ModelAnimationSet.obj
 0002:0000b1e0       ??_7CAnimationSet@@6B@     000000003164d1e0     ModelAnimationSet.obj
 0002:0000b310       ??_C@_0EH@FLFJJNIB@Unnecessary?5Loading?5of?5CAF?9files@ 000000003164d310     ModelAnimationSet.obj
 0002:0000b360       ??_C@_0EH@OEMEILP@Unnecessary?5Loading?5of?5CAF?9files@ 000000003164d360     ModelAnimationSet.obj
 0002:0000b3b0       ??_C@_0MB@DLLCPOOG@CryAnimation?3?3?5Trying?5to?5load?5an@ 000000003164d3b0     ModelAnimationSet.obj
 0002:0000b478       ??_C@_0CC@DGFFKLPE@Failed?5to?5load?5animation?5CAF?5fil@ 000000003164d478     ModelAnimationSet.obj
 0002:0000b4a0       ??_C@_0CI@MFGAAJDC@CryAnimation?3?3?5weird?5access?5of?5A@ 000000003164d4a0     ModelAnimationSet.obj
 0002:0000b4c8       ??_C@_0CI@DKHEGOPL@CryAnimation?3?3?5weird?5access?5of?5C@ 000000003164d4c8     ModelAnimationSet.obj
 0002:0000b4f4       __real@3e2aaaab            000000003164d4f4     ModelMesh.obj
 0002:0000b4f8       ??_C@_0BJ@DPHJOGLI@FindClosestPointOnMesh?3?5?$AA@ 000000003164d4f8     ModelMesh.obj
 0002:0000b514       __real@4cbebc20            000000003164d514     ModelMesh.obj
 0002:0000b518       ??_C@_0N@ECCGOBMG@Bip01?5R?5Toe0?$AA@ 000000003164d518     ModelSkeleton.obj
 0002:0000b528       ??_C@_0N@JOIFGJHJ@Bip01?5R?5Heel?$AA@ 000000003164d528     ModelSkeleton.obj
 0002:0000b538       ??_C@_0N@MBIECKPD@Bip01?5R?5Foot?$AA@ 000000003164d538     ModelSkeleton.obj
 0002:0000b548       ??_C@_0N@JDAJBMDK@Bip01?5R?5Calf?$AA@ 000000003164d548     ModelSkeleton.obj
 0002:0000b558       ??_C@_0N@HFMHAGFF@Bip01?5L?5Toe0?$AA@ 000000003164d558     ModelSkeleton.obj
 0002:0000b568       ??_C@_0N@KJGEIOOK@Bip01?5L?5Heel?$AA@ 000000003164d568     ModelSkeleton.obj
 0002:0000b578       ??_C@_0N@PGGFMNGA@Bip01?5L?5Foot?$AA@ 000000003164d578     ModelSkeleton.obj
 0002:0000b588       ??_C@_0N@KEOIPLKJ@Bip01?5L?5Calf?$AA@ 000000003164d588     ModelSkeleton.obj
 0002:0000b598       ??_C@_0BI@IDONHEOJ@todo?3?5delete?5bones?5phys?$AA@ 000000003164d598     ModelSkeleton.obj
 0002:0000b5b0       ??_C@_0M@OHJCPMGN@active_phys?$AA@ 000000003164d5b0     ModelSkeleton.obj
 0002:0000b5c0       ??_C@_07GFBFDLBM@gravity?$AA@ 000000003164d5c0     ModelSkeleton.obj
 0002:0000b5c8       ??_C@_05NCCFOPHA@model?$AA@ 000000003164d5c8     AnimationManager.obj
 0002:0000b5d0       ??_C@_03DAPAKLGM@dir?$AA@  000000003164d5d0     AnimationManager.obj
 0002:0000b5d4       ??_C@_06KLHHMIGM@offset?$AA@ 000000003164d5d4     AnimationManager.obj
 0002:0000b5e0       ??_C@_09DAGAJHIH@parameter?$AA@ 000000003164d5e0     AnimationManager.obj
 0002:0000b5f0       ??_C@_07JJACOCKO@endTime?$AA@ 000000003164d5f0     AnimationManager.obj
 0002:0000b5f8       ??_C@_04CLCEDBPF@time?$AA@ 000000003164d5f8     AnimationManager.obj
 0002:0000b600       ??_C@_05GFHEIIDD@event?$AA@ 000000003164d600     AnimationManager.obj
 0002:0000b608       ??_C@_0BJ@FBLMMOEB@CAF?5Reloading?5failed?3?5?$CFs?$AA@ 000000003164d608     AnimationManager.obj
 0002:0000b628       ??_C@_0CC@IBDFJLNA@Hot?5loaded?5animation?5CAF?9file?3?5?$CF@ 000000003164d628     AnimationManager.obj
 0002:0000b650       ??_C@_0FH@GLDCLENN@Could?5not?5process?5aim?5poses?5from@ 000000003164d650     AnimationManager.obj
 0002:0000b6a8       ??_C@_0BL@PEJBPCKA@Re?9Processed?5Look?9Pose?3?5?$CFs?$AA@ 000000003164d6a8     AnimationManager.obj
 0002:0000b6c8       ??_C@_0BK@KIKPHPJP@Re?9Processed?5Aim?9Pose?3?5?$CFs?$AA@ 000000003164d6c8     AnimationManager.obj
 0002:0000b6e8       ??_C@_0DK@CLFMPEFJ@Hot?5loaded?5animation?5CAF?9file?5fo@ 000000003164d6e8     AnimationManager.obj
 0002:0000b728       ??_C@_0DK@BABPPFII@CAF?5Reloading?5failed?0?5asset?5wasn@ 000000003164d728     AnimationManager.obj
 0002:0000b768       ??_C@_0CC@GCMBNMKE@Hot?5loaded?5animation?5LMG?9file?3?5?$CF@ 000000003164d768     AnimationManager.obj
 0002:0000b790       ??_C@_0BJ@JDJPOJGL@LMG?5Reloading?5failed?3?5?$CFs?$AA@ 000000003164d790     AnimationManager.obj
 0002:0000b7b0       ??_C@_0M@EGNNJIMG@__unnamed__?$AA@ 000000003164d7b0     AnimationManager.obj
 0002:0000b7c0       ??_C@_08NAFBJPAH@segment4?$AA@ 000000003164d7c0     AnimationManager.obj
 0002:0000b7d0       ??_C@_08JPBAAJMA@segment3?$AA@ 000000003164d7d0     AnimationManager.obj
 0002:0000b7e0       ??_C@_08IGALDIIB@segment2?$AA@ 000000003164d7e0     AnimationManager.obj
 0002:0000b7f0       ??_C@_08KNCGGLEC@segment1?$AA@ 000000003164d7f0     AnimationManager.obj
 0002:0000b800       ??_C@_0N@HLEDPIHE@Total?3?5?$CF4dKB?$AA@ 000000003164d800     AnimationManager.obj
 0002:0000b810       ??_C@_0FH@MOAGBIJJ@CharInstances?3?$CF3d?5?$CIMem?3?5?$CF4dKB?$CJ?5S@ 000000003164d810     AnimationManager.obj
 0002:0000b868       __real@41c80000            000000003164d868     AnimationManager.obj
 0002:0000b86c       __real@400ccccd            000000003164d86c     AnimationManager.obj
 0002:0000b870       ??_C@_0DC@DAFNBAKF@Defrag?5heap?3?5?$CFiKB?5moveable?5?$CFiKB?5@ 000000003164d870     AnimationManager.obj
 0002:0000b8a8       ??_C@_0DN@HMBLBPBC@LMG?3?5?$CF04d?5?5?5?5Loaded?3?5?$CF04d?5?5?5?5Use@ 000000003164d8a8     AnimationManager.obj
 0002:0000b8e8       ??_C@_0DO@OFMPJGHE@AIM?3?5?$CF04d?5?5?5?5Loaded?3?5?$CF04d?5?5?5?5Use@ 000000003164d8e8     AnimationManager.obj
 0002:0000b930       ??_C@_0EF@DIODCEKM@CAF?3?5?$CF04d?5?5?5?5Loaded?3?5?$CF04d?5?5?5?5Use@ 000000003164d930     AnimationManager.obj
 0002:0000b978       ??_C@_0BI@DFAHFJLE@nSizeOfLoadedKeys?3?5?$CF07d?$AA@ 000000003164d978     AnimationManager.obj
 0002:0000b990       ??_C@_0BP@JGLJADPL@CafInMemory?3?5?$CF07d?5FilePath?3?5?$CFs?$AA@ 000000003164d990     AnimationManager.obj
 0002:0000b9b0       ??_C@_0CH@CJCBCHLJ@CafInMemory?3?5?$CF7d?5ref?3?5?$CF5d?5FilePa@ 000000003164d9b0     AnimationManager.obj
 0002:0000b9d8       ??_C@_0DE@FGOCMMFD@DBA?3?5?$CFd?5KBytes?5?5?5Clients?3?5?$CFd?5KBy@ 000000003164d9d8     AnimationManager.obj
 0002:0000ba10       ??_C@_0DJ@IAMGMGNJ@size?5of?5path?5names?3?5?$CFd?5bytes?5?5?5?5@ 000000003164da10     AnimationManager.obj
 0002:0000ba50       ??_C@_0DL@HJBFHPHA@UsedAssets?3?5?$CF04d?5?5nTCount?3?5?$CFu?5?5S@ 000000003164da50     AnimationManager.obj
 0002:0000ba8c       __real@41300000            000000003164da8c     AnimationManager.obj
 0002:0000ba90       ??_C@_0CC@DMIIEABE@CAnimationManager?3?3DebugAnimUsag@ 000000003164da90     AnimationManager.obj
 0002:0000bab8       ??_C@_0O@EHHLMIFF@AnimationKeys?$AA@ 000000003164dab8     AnimationManager.obj
 0002:0000bac8       ??_C@_0CE@CGKHFNED@CAnimationManager?3?3LoadAnimation@ 000000003164dac8     AnimationManager.obj
 0002:0000baf0       ?m_byteTable@ControllerHelper@@3QBEB 000000003164daf0     ControllerPQ.obj
 0002:0000bbf0       ?m_byteLowBit@ControllerHelper@@3QBEB 000000003164dbf0     ControllerPQ.obj
 0002:0000bcf0       ?m_byteHighBit@ControllerHelper@@3QBEB 000000003164dcf0     ControllerPQ.obj
 0002:0000bdf0       __real@383505e6            000000003164ddf0     ControllerPQ.obj
 0002:0000bdf4       __real@35b50506            000000003164ddf4     ControllerPQ.obj
 0002:0000bdf8       __real@353504fe            000000003164ddf8     ControllerPQ.obj
 0002:0000be00       ??_7?$CTrackDataStorageInt@U?$Vec3_tpl@M@@UNoCompressVec3@@VITrackPositionStorage@@@@6B@ 000000003164de00     ControllerPQ.obj
 0002:0000be50       ??_7?$CTrackDataStorageInt@U?$Quat_tpl@M@@UNoCompressQuat@@VITrackRotationStorage@@@@6B@ 000000003164de50     ControllerPQ.obj
 0002:0000bea0       ??_7?$CTrackDataStorageInt@U?$Quat_tpl@M@@USmallTree48BitQuat@@VITrackRotationStorage@@@@6B@ 000000003164dea0     ControllerPQ.obj
 0002:0000bef0       ??_7?$CTrackDataStorageInt@U?$Quat_tpl@M@@USmallTree64BitQuat@@VITrackRotationStorage@@@@6B@ 000000003164def0     ControllerPQ.obj
 0002:0000bf40       ??_7?$CTrackDataStorageInt@U?$Quat_tpl@M@@USmallTree64BitExtQuat@@VITrackRotationStorage@@@@6B@ 000000003164df40     ControllerPQ.obj
 0002:0000bf90       ??_7CKeyTimesInformationBitSet@@6B@ 000000003164df90     ControllerPQ.obj
 0002:0000bfe0       ??_C@_0CI@NIMGLEEI@Unknown?5Rotation?5Compression?5for@ 000000003164dfe0     ControllerPQ.obj
 0002:0000c010       ??_7?$CTrackDataStorage@U?$Vec3_tpl@M@@UNoCompressVec3@@VITrackPositionStorage@@@@6B@ 000000003164e010     ControllerPQ.obj
 0002:0000c070       ??_7?$CTrackDataStorage@U?$Quat_tpl@M@@UNoCompressQuat@@VITrackRotationStorage@@@@6B@ 000000003164e070     ControllerPQ.obj
 0002:0000c0d0       ??_7?$CTrackDataStorage@U?$Quat_tpl@M@@USmallTree48BitQuat@@VITrackRotationStorage@@@@6B@ 000000003164e0d0     ControllerPQ.obj
 0002:0000c130       ??_7?$CTrackDataStorage@U?$Quat_tpl@M@@USmallTree64BitQuat@@VITrackRotationStorage@@@@6B@ 000000003164e130     ControllerPQ.obj
 0002:0000c190       ??_7?$CTrackDataStorage@U?$Quat_tpl@M@@USmallTree64BitExtQuat@@VITrackRotationStorage@@@@6B@ 000000003164e190     ControllerPQ.obj
 0002:0000c1f0       ??_7?$CKeyTimesInformation@MUF32Encoder@@@@6BIControllerRelocatableChain@@@ 000000003164e1f0     ControllerPQ.obj
 0002:0000c200       ??_7?$CKeyTimesInformation@MUF32Encoder@@@@6BIKeyTimesInformation@@@ 000000003164e200     ControllerPQ.obj
 0002:0000c250       ??_7?$CKeyTimesInformation@GUUINT16Encoder@@@@6BIControllerRelocatableChain@@@ 000000003164e250     ControllerPQ.obj
 0002:0000c260       ??_7?$CKeyTimesInformation@GUUINT16Encoder@@@@6BIKeyTimesInformation@@@ 000000003164e260     ControllerPQ.obj
 0002:0000c2b0       ??_7?$CKeyTimesInformation@EUByteEncoder@@@@6BIControllerRelocatableChain@@@ 000000003164e2b0     ControllerPQ.obj
 0002:0000c2c0       ??_7?$CKeyTimesInformation@EUByteEncoder@@@@6BIKeyTimesInformation@@@ 000000003164e2c0     ControllerPQ.obj
 0002:0000c310       ??_7?$CKeyTimesInformationStartStop@MUF32StartStopEncoder@@@@6B@ 000000003164e310     ControllerPQ.obj
 0002:0000c360       ??_7?$CKeyTimesInformationStartStop@GUUINT16StartStopEncoder@@@@6B@ 000000003164e360     ControllerPQ.obj
 0002:0000c3b0       ??_7?$CKeyTimesInformationStartStop@EUByteStartStopEncoder@@@@6B@ 000000003164e3b0     ControllerPQ.obj
 0002:0000c400       __real@3eb0c6f7a0000000    000000003164e400     ControllerPQLog.obj
 0002:0000c408       __real@3ff921fb54442d18    000000003164e408     ControllerPQLog.obj
 0002:0000c410       __real@400921fb54442d18    000000003164e410     ControllerPQLog.obj
 0002:0000c420       ??_7CControllerPQLog@@6B@  000000003164e420     ControllerPQLog.obj
 0002:0000c4a0       __real@bff0000000000000    000000003164e4a0     GlobalAnimationHeaderAIM.obj
 0002:0000c4a8       __real@0010000000000000    000000003164e4a8     GlobalAnimationHeaderAIM.obj
 0002:0000c4b0       __real@3ddb7cdfd9d7bdbb    000000003164e4b0     GlobalAnimationHeaderAIM.obj
 0002:0000c4b8       __real@4024000000000000    000000003164e4b8     GlobalAnimationHeaderAIM.obj
 0002:0000c4c0       __real@3f847ae140000000    000000003164e4c0     GlobalAnimationHeaderAIM.obj
 0002:0000c4c8       __real@4008000000000000    000000003164e4c8     GlobalAnimationHeaderAIM.obj
 0002:0000c4d0       __real@3fd0000000000000    000000003164e4d0     GlobalAnimationHeaderAIM.obj
 0002:0000c4d8       __real@403e000000000000    000000003164e4d8     GlobalAnimationHeaderAIM.obj
 0002:0000c4e0       __real@3f847ae147ae147b    000000003164e4e0     GlobalAnimationHeaderAIM.obj
 0002:0000c4e8       __real@3f80a3d7            000000003164e4e8     GlobalAnimationHeaderAIM.obj
 0002:0000c4f0       ??_C@_0BL@ODMGNJMN@CONTROLLER_CHUNK_DESC_0826?$AA@ 000000003164e4f0     GlobalAnimationHeaderAIM.obj
 0002:0000c510       ??_C@_0CG@HDJMEILE@Animation?5file?5has?5no?5compressed@ 000000003164e510     GlobalAnimationHeaderAIM.obj
 0002:0000c538       ??_C@_0CF@OGCHLH@Animation?5file?5has?5uncompressed?5@ 000000003164e538     GlobalAnimationHeaderAIM.obj
 0002:0000c560       ??_C@_0BB@HBALHEOC@weird?5controller?$AA@ 000000003164e560     GlobalAnimationHeaderAIM.obj
 0002:0000c578       ??_C@_0BL@KNEFCFDN@CONTROLLER_CHUNK_DESC_0831?$AA@ 000000003164e578     GlobalAnimationHeaderAIM.obj
 0002:0000c598       ??_C@_0BL@LEFOBEHM@CONTROLLER_CHUNK_DESC_0830?$AA@ 000000003164e598     GlobalAnimationHeaderAIM.obj
 0002:0000c5b8       ??_C@_0L@NECCCPPF@TCB?5chunks?$AA@ 000000003164e5b8     GlobalAnimationHeaderAIM.obj
 0002:0000c5c8       ??_C@_0CE@FCEPGAHG@Illegal?5File?5Type?5for?5?4CAF?5file?3@ 000000003164e5c8     GlobalAnimationHeaderAIM.obj
 0002:0000c5f0       __real@40c0000000000000    000000003164e5f0     GlobalAnimationHeaderAIM.obj
 0002:0000c5f8       __real@461c3c00            000000003164e5f8     GlobalAnimationHeaderAIM.obj
 0002:0000c600       __real@3ff00068db8bac71    000000003164e600     GlobalAnimationHeaderAIM.obj
 0002:0000c608       __real@3ff004189374bc6a    000000003164e608     GlobalAnimationHeaderAIM.obj
 0002:0000c610       __real@3fa999999999999a    000000003164e610     GlobalAnimationHeaderAIM.obj
 0002:0000c618       __real@3fd921fb54442d18    000000003164e618     GlobalAnimationHeaderAIM.obj
 0002:0000c620       ??_C@_0EM@OIFELHKN@CryAnimation?3?5Aimpose?5?8?$CFs?8?5disab@ 000000003164e620     GlobalAnimationHeaderAIM.obj
 0002:0000c670       ??_C@_0ED@KBHGCNDO@CryAnimation?3?5Parameter?5joint?5?8?$CF@ 000000003164e670     GlobalAnimationHeaderAIM.obj
 0002:0000c6b8       ??_C@_0DN@PJFOJMDA@CryAnimation?3?5Parameter?5joint?5?8?$CF@ 000000003164e6b8     GlobalAnimationHeaderAIM.obj
 0002:0000c6f8       ??_C@_0CD@LDOKNDOJ@CryAnimation?3?5process?5Aimpose?5?8?$CF@ 000000003164e6f8     GlobalAnimationHeaderAIM.obj
 0002:0000c71c       ??_C@_01LOCGONAA@?$AA?$AA@ 000000003164e71c     GlobalAnimationHeaderAIM.obj
 0002:0000c728       ??_C@_0CH@FGLCCHPF@GlobalAnimationHeaderCAF?3?3DoesEx@ 000000003164e728     GlobalAnimationHeaderCAF.obj
 0002:0000c750       ??_C@_0O@HEFJBIFC@Animation?5DBA?$AA@ 000000003164e750     GlobalAnimationHeaderCAF.obj
 0002:0000c760       ??_C@_0CK@PCKLFE@SPEED_CHUNK_DESC_1?5not?5supported@ 000000003164e760     GlobalAnimationHeaderCAF.obj
 0002:0000c790       ??_C@_0CI@CHBFAPGJ@SPEED_CHUNK_DESC?5not?5supported?5a@ 000000003164e790     GlobalAnimationHeaderCAF.obj
 0002:0000c7b8       ??_7GlobalAnimationHeaderCAFStreamContent@@6B@ 000000003164e7b8     GlobalAnimationHeaderCAF.obj
 0002:0000c7d8       ??_C@_0BJ@CLIKGAMM@?$CFd?5?$CFf?5?$CFf?5?$CFf?5?$CFf?5?$CFf?5?$CFf?5?$CFf?6?$AA@ 000000003164e7d8     GlobalAnimationHeaderCAF.obj
 0002:0000c7f4       ??_C@_05MGFEFMAH@?$FL?$CFs?$FN?6?$AA@ 000000003164e7f4     GlobalAnimationHeaderCAF.obj
 0002:0000c800       ??_C@_0BK@GMCOOBCN@?$CDFr?7Tx?7Ty?7Tz?7Rx?7Ry?7Rz?7SF?6?$AA@ 000000003164e800     GlobalAnimationHeaderCAF.obj
 0002:0000c820       ??_C@_0CH@HOGCBNHO@?$CDBeginning?5of?5Data?4?5Separated?5by@ 000000003164e820     GlobalAnimationHeaderCAF.obj
 0002:0000c848       ??_C@_0BK@MLILPEIB@?$CFs?5?$CFf?5?$CFf?5?$CFf?5?$CFf?5?$CFf?5?$CFf?5?$CFf?5?6?$AA@ 000000003164e848     GlobalAnimationHeaderCAF.obj
 0002:0000c868       ??_C@_0DB@GOIDDDLG@?$CDSegmentName?5Tx?0?5Ty?0?5Tz?0?5Rx?0?5Ry?0@ 000000003164e868     GlobalAnimationHeaderCAF.obj
 0002:0000c8a0       ??_C@_0BA@HCLCKBKE@?$FLBasePosition?$FN?6?$AA@ 000000003164e8a0     GlobalAnimationHeaderCAF.obj
 0002:0000c8b0       ??_C@_06IINFAHFO@?$CFs?5?$CFs?6?$AA@ 000000003164e8b0     GlobalAnimationHeaderCAF.obj
 0002:0000c8b8       ??_C@_06FNIPBJLB@GLOBAL?$AA@ 000000003164e8b8     GlobalAnimationHeaderCAF.obj
 0002:0000c8c0       ??_C@_07DNODLGKM@INVALID?$AA@ 000000003164e8c0     GlobalAnimationHeaderCAF.obj
 0002:0000c8c8       ??_C@_0P@KNDGJNPN@?$CDCHILD?7PARENT?6?$AA@ 000000003164e8c8     GlobalAnimationHeaderCAF.obj
 0002:0000c8d8       ??_C@_0BK@FIEHECJB@?$FLSegmentNames?$CGHierarchy?$FN?6?$AA@ 000000003164e8d8     GlobalAnimationHeaderCAF.obj
 0002:0000c8f8       ??_C@_0BC@PLMODGGP@ScaleFactor?51?400?6?$AA@ 000000003164e8f8     GlobalAnimationHeaderCAF.obj
 0002:0000c910       ??_C@_0BC@LACMDAJF@BoneLengthAxis?5Y?6?$AA@ 000000003164e910     GlobalAnimationHeaderCAF.obj
 0002:0000c928       ??_C@_0BH@IBIJNGBE@GlobalAxisofGravity?5Y?6?$AA@ 000000003164e928     GlobalAnimationHeaderCAF.obj
 0002:0000c940       ??_C@_0BH@DGLENGCE@RotationUnits?5Degrees?6?$AA@ 000000003164e940     GlobalAnimationHeaderCAF.obj
 0002:0000c958       ??_C@_0BF@OKDFJOBC@CalibrationUnits?5mm?6?$AA@ 000000003164e958     GlobalAnimationHeaderCAF.obj
 0002:0000c970       ??_C@_0BI@LACHBPJI@EulerRotationOrder?5ZYX?6?$AA@ 000000003164e970     GlobalAnimationHeaderCAF.obj
 0002:0000c988       ??_C@_0DK@GLCCHHDF@DataFrameRate?5?$CFd?7?7?$CDinteger?0?5data@ 000000003164e988     GlobalAnimationHeaderCAF.obj
 0002:0000c9c8       ??_C@_0BI@FJIJOOIN@NumFrames?5?$CFd?7?7?$CDinteger?6?$AA@ 000000003164e9c8     GlobalAnimationHeaderCAF.obj
 0002:0000c9e0       ??_C@_0BK@BFNNFED@NumSegments?5?$CFd?7?7?$CDinteger?6?$AA@ 000000003164e9e0     GlobalAnimationHeaderCAF.obj
 0002:0000ca00       ??_C@_0BJ@IBCLPNKG@FileVersion?51?7?7?$CDinteger?6?$AA@ 000000003164ea00     GlobalAnimationHeaderCAF.obj
 0002:0000ca20       ??_C@_0EB@PEACHJMM@DataType?5HTRS?7?7?$CDTranslation?5foll@ 000000003164ea20     GlobalAnimationHeaderCAF.obj
 0002:0000ca68       ??_C@_0CD@PNOAEFKH@FileType?5HTR?7?7?$CDSingle?5word?5strin@ 000000003164ea68     GlobalAnimationHeaderCAF.obj
 0002:0000ca90       ??_C@_0DC@IACPGBAE@?$CDHeader?5keywords?5are?5followed?5by@ 000000003164ea90     GlobalAnimationHeaderCAF.obj
 0002:0000cac8       ??_C@_0L@CALEHGCD@?$FLHeader?$FN?7?6?$AA@ 000000003164eac8     GlobalAnimationHeaderCAF.obj
 0002:0000cad8       ??_C@_0DF@OKGHBAIO@?$CDHierarchical?5Translation?5and?5Ro@ 000000003164ead8     GlobalAnimationHeaderCAF.obj
 0002:0000cb10       ??_C@_0DG@DKOOKMLC@?$CDComment?5line?5ignore?5any?5data?5fo@ 000000003164eb10     GlobalAnimationHeaderCAF.obj
 0002:0000cb48       ??_C@_04PHEPJNJD@?4htr?$AA@ 000000003164eb48     GlobalAnimationHeaderCAF.obj
 0002:0000cb50       ??_C@_0CA@GHFHHAOC@Illegal?5File?5Type?5for?5?4caf?5file?$AA@ 000000003164eb50     GlobalAnimationHeaderCAF.obj
 0002:0000cb70       ??_C@_0BF@NBFOLJEO@Bad?5CAF?5file?5version?$AA@ 000000003164eb70     GlobalAnimationHeaderCAF.obj
 0002:0000cb90       ??_C@_0HL@BICADCBF@GlobalAnimationHeaderCAF?5is?5not?5@ 000000003164eb90     GlobalAnimationHeaderCAF.obj
 0002:0000cc10       ??_C@_0EO@DNGKKJGM@CryAnimation?5CAF?3?5Assets?5has?5no?5@ 000000003164ec10     GlobalAnimationHeaderCAF.obj
 0002:0000cc60       ??_C@_0BH@KADPCBAF@CAF?9File?5Not?5Found?3?5?$CFs?$AA@ 000000003164ec60     GlobalAnimationHeaderCAF.obj
 0002:0000cc78       ??_C@_0BB@LGNCGFD@CAF?5Animation?5?$CFs?$AA@ 000000003164ec78     GlobalAnimationHeaderCAF.obj
 0002:0000cc90       ??_C@_0CI@CEIBOAIJ@Animation?9asset?5not?5in?5Animation@ 000000003164ec90     GlobalAnimationHeaderCAF.obj
 0002:0000ccb8       ??_C@_0CC@OFOPDEKN@GlobalAnimationHeaderCAF?3?3LoadCA@ 000000003164ecb8     GlobalAnimationHeaderCAF.obj
 0002:0000cce0       ??_C@_0BM@JEBLFMNF@Failed?5to?5parse?5CAF?9file?5?$CFx?$AA@ 000000003164ece0     GlobalAnimationHeaderCAF.obj
 0002:0000cd00       ??_C@_0DI@GIACGBCH@GlobalAnimationHeaderCAFStreamCo@ 000000003164ed00     GlobalAnimationHeaderCAF.obj
 0002:0000cd40       ??_C@_09JDIBPAEJ@?$DM?1VGrid?$DO?6?$AA@ 000000003164ed40     GlobalAnimationHeaderLMG.obj
 0002:0000cd50       ??_C@_0LJ@NKMLEKDJ@?7?$DMVExample?5i0?$DN?$CC?$CF2d?$CC?5i1?$DN?$CC?$CF2d?$CC?5i2?$DN@ 000000003164ed50     GlobalAnimationHeaderLMG.obj
 0002:0000ce10       ??_C@_08HBIAJAJD@?$DMVGrid?$DO?6?$AA@ 000000003164ee10     GlobalAnimationHeaderLMG.obj
 0002:0000ce20       ??_C@_0DP@CFNOMPCL@CryAnimation?3?5asset?5for?5paramete@ 000000003164ee20     GlobalAnimationHeaderLMG.obj
 0002:0000ce60       ??_C@_0CL@EDKCNNKH@Error?3?5ParaGroup?5has?5no?5examples@ 000000003164ee60     GlobalAnimationHeaderLMG.obj
 0002:0000ce90       ??_C@_0CN@LMDFKGDA@Error?3?5ParaGroup?5has?5no?5dimensio@ 000000003164ee90     GlobalAnimationHeaderLMG.obj
 0002:0000cec0       ??_C@_0BA@IJGNAHAN@?8?5was?5not?5found?$AA@ 000000003164eec0     GlobalAnimationHeaderLMG.obj
 0002:0000ced0       ??_C@_0BL@JDPLPDDI@Error?3?5The?5included?5file?5?8?$AA@ 000000003164eed0     GlobalAnimationHeaderLMG.obj
 0002:0000cef0       ??_C@_0P@EPLPMDPH@?8?5is?5not?5valid?$AA@ 000000003164eef0     GlobalAnimationHeaderLMG.obj
 0002:0000cf00       ??_C@_0CC@BNBCGHJD@Error?3?5The?5included?5blend?9space?5@ 000000003164ef00     GlobalAnimationHeaderLMG.obj
 0002:0000cf30       ??_C@_0EG@HMKJJPIC@Error?3?5More?5then?54?5additional?5ex@ 000000003164ef30     GlobalAnimationHeaderLMG.obj
 0002:0000cf78       ??_C@_0DO@GDICJIMA@Error?3?5More?5then?54?5dimensions?5pe@ 000000003164ef78     GlobalAnimationHeaderLMG.obj
 0002:0000cfb8       ??_C@_05HAIIBMHI@aname?$AA@ 000000003164efb8     GlobalAnimationHeaderLMG.obj
 0002:0000cfc0       ??_C@_0L@NPKCPEDM@BlendSpace?$AA@ 000000003164efc0     GlobalAnimationHeaderLMG.obj
 0002:0000cfd0       ??_C@_0M@CLKCPEEG@BlendSpaces?$AA@ 000000003164efd0     GlobalAnimationHeaderLMG.obj
 0002:0000cfe0       ??_C@_0BB@ECHECOCG@ChooseBlendSpace?$AA@ 000000003164efe0     GlobalAnimationHeaderLMG.obj
 0002:0000cff8       ??_C@_09KDJIBPJO@ParaScale?$AA@ 000000003164eff8     GlobalAnimationHeaderLMG.obj
 0002:0000d008       ??_C@_0BF@JMFFNCEF@Error?3?5The?5XML?9Tag?5?8?$AA@ 000000003164f008     GlobalAnimationHeaderLMG.obj
 0002:0000d020       ??_C@_0CC@BLKFDNDD@?8?4?5It?5is?5expected?5to?5be?5?8Example@ 000000003164f020     GlobalAnimationHeaderLMG.obj
 0002:0000d048       ??_C@_0CK@FPFCGPOG@Error?3?5The?5ExampleTAG?5for?5an?5exa@ 000000003164f048     GlobalAnimationHeaderLMG.obj
 0002:0000d080       ??_C@_0FE@DOPPMCAJ@The?5ParaGroup?5?8?$CFs?8?5is?5invalid?$CB?5T@ 000000003164f080     GlobalAnimationHeaderLMG.obj
 0002:0000d0d8       ??_C@_0BJ@DCBDEEAK@?8?5is?5not?5in?5the?5CAL?9file?$AA@ 000000003164f0d8     GlobalAnimationHeaderLMG.obj
 0002:0000d0f8       ??_C@_0BH@BIDNBJJH@Error?3?5The?5animation?5?8?$AA@ 000000003164f0f8     GlobalAnimationHeaderLMG.obj
 0002:0000d110       ??_C@_0FK@KEJALHHG@The?5ParaGroup?5?8?$CFs?8?5is?5invalid?$CB?5T@ 000000003164f110     GlobalAnimationHeaderLMG.obj
 0002:0000d170       ??_C@_0BB@JKIDKOJK@?8?5does?5not?5exist?$AA@ 000000003164f170     GlobalAnimationHeaderLMG.obj
 0002:0000d188       ??_C@_0CF@JNIHMDHP@Error?3?5The?5asset?5for?5the?5animati@ 000000003164f188     GlobalAnimationHeaderLMG.obj
 0002:0000d1b0       ??_C@_0EA@NACDAFHJ@Error?3?5More?5then?53?5dimensions?5pe@ 000000003164f1b0     GlobalAnimationHeaderLMG.obj
 0002:0000d1f0       ??_C@_0BN@EPHGHLEL@?8?5is?5currently?5not?5supported?$AA@ 000000003164f1f0     GlobalAnimationHeaderLMG.obj
 0002:0000d210       ??_C@_0BH@FMDDKGDP@Error?3?5The?5parameter?5?8?$AA@ 000000003164f210     GlobalAnimationHeaderLMG.obj
 0002:0000d228       ??_C@_05IHAFCALK@Style?$AA@ 000000003164f228     GlobalAnimationHeaderLMG.obj
 0002:0000d230       ??_C@_08HHFKANFI@NewStyle?$AA@ 000000003164f230     GlobalAnimationHeaderLMG.obj
 0002:0000d240       ??_C@_0BC@ICLDOOLI@MotionCombination?$AA@ 000000003164f240     GlobalAnimationHeaderLMG.obj
 0002:0000d254       ??_C@_02MBAHPIAM@w7?$AA@   000000003164f254     GlobalAnimationHeaderLMG.obj
 0002:0000d258       ??_C@_02NIBMMJEN@w6?$AA@   000000003164f258     GlobalAnimationHeaderLMG.obj
 0002:0000d25c       ??_C@_02PDDBJKIO@w5?$AA@   000000003164f25c     GlobalAnimationHeaderLMG.obj
 0002:0000d260       ??_C@_02OKCKKLMP@w4?$AA@   000000003164f260     GlobalAnimationHeaderLMG.obj
 0002:0000d264       ??_C@_02KFGLDNAI@w3?$AA@   000000003164f264     GlobalAnimationHeaderLMG.obj
 0002:0000d268       ??_C@_02LMHAAMEJ@w2?$AA@   000000003164f268     GlobalAnimationHeaderLMG.obj
 0002:0000d26c       ??_C@_02NHLPHGHG@i7?$AA@   000000003164f26c     GlobalAnimationHeaderLMG.obj
 0002:0000d270       ??_C@_02MOKEEHDH@i6?$AA@   000000003164f270     GlobalAnimationHeaderLMG.obj
 0002:0000d274       ??_C@_02OFIJBEPE@i5?$AA@   000000003164f274     GlobalAnimationHeaderLMG.obj
 0002:0000d278       ??_C@_02PMJCCFLF@i4?$AA@   000000003164f278     GlobalAnimationHeaderLMG.obj
 0002:0000d27c       ??_C@_02LDNDLDHC@i3?$AA@   000000003164f27c     GlobalAnimationHeaderLMG.obj
 0002:0000d280       ??_C@_02KKMIICDD@i2?$AA@   000000003164f280     GlobalAnimationHeaderLMG.obj
 0002:0000d284       ??_C@_02IBOFNBPA@i1?$AA@   000000003164f284     GlobalAnimationHeaderLMG.obj
 0002:0000d288       ??_C@_02JIPOOALB@i0?$AA@   000000003164f288     GlobalAnimationHeaderLMG.obj
 0002:0000d290       ??_C@_08DGDGODFB@VExample?$AA@ 000000003164f290     GlobalAnimationHeaderLMG.obj
 0002:0000d29c       ??_C@_05PJJIAHPE@VGrid?$AA@ 000000003164f29c     GlobalAnimationHeaderLMG.obj
 0002:0000d2a4       ??_C@_02MEEIOOIJ@p7?$AA@   000000003164f2a4     GlobalAnimationHeaderLMG.obj
 0002:0000d2a8       ??_C@_02NNFDNPMI@p6?$AA@   000000003164f2a8     GlobalAnimationHeaderLMG.obj
 0002:0000d2ac       ??_C@_02PGHOIMAL@p5?$AA@   000000003164f2ac     GlobalAnimationHeaderLMG.obj
 0002:0000d2b0       ??_C@_02OPGFLNEK@p4?$AA@   000000003164f2b0     GlobalAnimationHeaderLMG.obj
 0002:0000d2b4       ??_C@_02KACECLIN@p3?$AA@   000000003164f2b4     GlobalAnimationHeaderLMG.obj
 0002:0000d2b8       ??_C@_02LJDPBKMM@p2?$AA@   000000003164f2b8     GlobalAnimationHeaderLMG.obj
 0002:0000d2bc       ??_C@_04DPOPNPPG@Face?$AA@ 000000003164f2bc     GlobalAnimationHeaderLMG.obj
 0002:0000d2c8       ??_C@_09IALACKFM@Blendable?$AA@ 000000003164f2c8     GlobalAnimationHeaderLMG.obj
 0002:0000d2d4       ??_C@_02JHFNFPIK@w1?$AA@   000000003164f2d4     GlobalAnimationHeaderLMG.obj
 0002:0000d2d8       ??_C@_02IOEGGOML@w0?$AA@   000000003164f2d8     GlobalAnimationHeaderLMG.obj
 0002:0000d2dc       ??_C@_02JCBCEJAP@p1?$AA@   000000003164f2dc     GlobalAnimationHeaderLMG.obj
 0002:0000d2e0       ??_C@_02ILAJHIEO@p0?$AA@   000000003164f2e0     GlobalAnimationHeaderLMG.obj
 0002:0000d2e4       ??_C@_06GMHIAKFO@Pseudo?$AA@ 000000003164f2e4     GlobalAnimationHeaderLMG.obj
 0002:0000d2f0       ??_C@_0BL@BKKBLDIH@UseDirectlyForDeltaMotion3?$AA@ 000000003164f2f0     GlobalAnimationHeaderLMG.obj
 0002:0000d310       ??_C@_0BL@DLKICMG@UseDirectlyForDeltaMotion2?$AA@ 000000003164f310     GlobalAnimationHeaderLMG.obj
 0002:0000d330       ??_C@_0BL@CIJHNBAF@UseDirectlyForDeltaMotion1?$AA@ 000000003164f330     GlobalAnimationHeaderLMG.obj
 0002:0000d350       ??_C@_0BL@DBIMOAEE@UseDirectlyForDeltaMotion0?$AA@ 000000003164f350     GlobalAnimationHeaderLMG.obj
 0002:0000d370       ??_C@_08GJBDGDP@SetPara3?$AA@ 000000003164f370     GlobalAnimationHeaderLMG.obj
 0002:0000d380       ??_C@_08BPIKAHHO@SetPara2?$AA@ 000000003164f380     GlobalAnimationHeaderLMG.obj
 0002:0000d390       ??_C@_08DEKHFELN@SetPara1?$AA@ 000000003164f390     GlobalAnimationHeaderLMG.obj
 0002:0000d3a0       ??_C@_08CNLMGFPM@SetPara0?$AA@ 000000003164f3a0     GlobalAnimationHeaderLMG.obj
 0002:0000d3b0       ??_C@_0O@GMBENGPI@PlaybackScale?$AA@ 000000003164f3b0     GlobalAnimationHeaderLMG.obj
 0002:0000d3c0       ??_C@_07LEFFBAGK@Example?$AA@ 000000003164f3c0     GlobalAnimationHeaderLMG.obj
 0002:0000d3c8       ??_C@_0BF@CFNNMGLO@AdditionalExtraction?$AA@ 000000003164f3c8     GlobalAnimationHeaderLMG.obj
 0002:0000d3e0       ??_C@_06KKBPGBGI@locked?$AA@ 000000003164f3e0     GlobalAnimationHeaderLMG.obj
 0002:0000d3e8       ??_C@_04DEMJELKJ@ekey?$AA@ 000000003164f3e8     GlobalAnimationHeaderLMG.obj
 0002:0000d3f0       ??_C@_04NLGJCJIL@skey?$AA@ 000000003164f3f0     GlobalAnimationHeaderLMG.obj
 0002:0000d3f8       ??_C@_05MHMEBBGO@scale?$AA@ 000000003164f3f8     GlobalAnimationHeaderLMG.obj
 0002:0000d400       ??_C@_05KFKAILFP@cells?$AA@ 000000003164f400     GlobalAnimationHeaderLMG.obj
 0002:0000d408       ??_C@_03LJAEFNNE@max?$AA@  000000003164f408     GlobalAnimationHeaderLMG.obj
 0002:0000d40c       ??_C@_03KLIPLJLL@min?$AA@  000000003164f40c     GlobalAnimationHeaderLMG.obj
 0002:0000d410       ??_C@_07OMEBGOOF@StopLeg?$AA@ 000000003164f410     GlobalAnimationHeaderLMG.obj
 0002:0000d418       ??_C@_0M@HEHNJKHP@BlendWeight?$AA@ 000000003164f418     GlobalAnimationHeaderLMG.obj
 0002:0000d428       ??_C@_09DOPCOEIN@TurnAngle?$AA@ 000000003164f428     GlobalAnimationHeaderLMG.obj
 0002:0000d438       ??_C@_0L@NPIFDIHI@TravelDist?$AA@ 000000003164f438     GlobalAnimationHeaderLMG.obj
 0002:0000d448       ??_C@_0M@GJCIJMHH@TravelAngle?$AA@ 000000003164f448     GlobalAnimationHeaderLMG.obj
 0002:0000d458       ??_C@_0M@INHOBOHM@TravelSlope?$AA@ 000000003164f458     GlobalAnimationHeaderLMG.obj
 0002:0000d468       ??_C@_09BDPPKMLL@TurnSpeed?$AA@ 000000003164f468     GlobalAnimationHeaderLMG.obj
 0002:0000d478       ??_C@_09HHOHJEHG@MoveSpeed?$AA@ 000000003164f478     GlobalAnimationHeaderLMG.obj
 0002:0000d484       ??_C@_05LOJBNELM@Param?$AA@ 000000003164f484     GlobalAnimationHeaderLMG.obj
 0002:0000d490       ??_C@_09ODPNOLPG@Idle2Move?$AA@ 000000003164f490     GlobalAnimationHeaderLMG.obj
 0002:0000d4a0       ??_C@_09HAFMGPLD@VEGPARAMS?$AA@ 000000003164f4a0     GlobalAnimationHeaderLMG.obj
 0002:0000d4ac       ??_C@_02IGJGHHBN@tz?$AA@   000000003164f4ac     GlobalAnimationHeaderLMG.obj
 0002:0000d4b0       ??_C@_09EILGBNO@THRESHOLD?$AA@ 000000003164f4b0     GlobalAnimationHeaderLMG.obj
 0002:0000d4c0       ??_C@_0CG@DOEGIGK@Error?3?5no?5examples?5in?5this?5ParaG@ 000000003164f4c0     GlobalAnimationHeaderLMG.obj
 0002:0000d4f0       ??_C@_0EL@GBNGEHGE@Error?3?5too?5many?5examples?5in?5one?5@ 000000003164f4f0     GlobalAnimationHeaderLMG.obj
 0002:0000d540       ??_C@_0O@PJOADIDN@ExamplePseudo?$AA@ 000000003164f540     GlobalAnimationHeaderLMG.obj
 0002:0000d550       ??_C@_0M@IFLEANKJ@ExampleList?$AA@ 000000003164f550     GlobalAnimationHeaderLMG.obj
 0002:0000d560       ??_C@_0BE@GIKNGEKK@CryAnimation?5?$CFs?3?5?$CFs?$AA@ 000000003164f560     GlobalAnimationHeaderLMG.obj
 0002:0000d578       ??_C@_0DM@GGNNFPCH@?8?4?5It?5is?5expected?5to?5be?5?8ParaGro@ 000000003164f578     GlobalAnimationHeaderLMG.obj
 0002:0000d5b8       ??_C@_0BH@MALMLOBG@Error?3?5The?5XMLTAG?5is?5?8?$AA@ 000000003164f5b8     GlobalAnimationHeaderLMG.obj
 0002:0000d5d0       ??_C@_0BD@FPPGAOB@CombinedBlendSpace?$AA@ 000000003164f5d0     GlobalAnimationHeaderLMG.obj
 0002:0000d5e8       ??_C@_09KCMCOIPJ@ParaGroup?$AA@ 000000003164f5e8     GlobalAnimationHeaderLMG.obj
 0002:0000d5f8       ??_C@_0CC@GGJPBFGD@Error?3?5Parametric?9Group?5not?5foun@ 000000003164f5f8     GlobalAnimationHeaderLMG.obj
 0002:0000d620       ??_C@_0EI@PNPGPCFE@Error?3?5Parametric?9Group?5loaded?5f@ 000000003164f620     GlobalAnimationHeaderLMG.obj
 0002:0000d670       ??_C@_0EJ@PGHDDIJ@Error?3?5Parametric?9Group?5loaded?5f@ 000000003164f670     GlobalAnimationHeaderLMG.obj
 0002:0000d6c0       ??_C@_0GA@FLLAOKLL@CryAnimation?3?5?5LMGs?5not?5supporte@ 000000003164f6c0     GlobalAnimationHeaderLMG.obj
 0002:0000d720       ??_C@_0BM@CDIMEJKN@CryAnimation?3?5data?5mismatch?$AA@ 000000003164f720     GlobalAnimationHeaderLMG.obj
 0002:0000d740       ??_C@_01GBGANLPD@0?$AA@    000000003164f740     AnimationBase.obj
 0002:0000d744       __real@2f800000            000000003164f744     AnimationBase.obj
 0002:0000d748       ??_C@_0DJ@DLJMMMP@Could?5not?5access?5CrySystem?4dll?5?$CI@ 000000003164f748     AnimationBase.obj
 0002:0000d788       ??_C@_0P@NHEMOHAI@Memory?5Manager?$AA@ 000000003164f788     AnimationBase.obj
 0002:0000d798       ??_C@_0O@FFDHMLKN@CrySystem?4dll?$AA@ 000000003164f798     AnimationBase.obj
 0002:0000d7a8       ??_C@_0BO@JDKBDPNB@CryGetIMemoryManagerInterface?$AA@ 000000003164f7a8     AnimationBase.obj
 0002:0000d7c8       ??_C@_0BB@PNKHDABP@CrySystemCrtFree?$AA@ 000000003164f7c8     AnimationBase.obj
 0002:0000d7e0       ??_C@_0BB@MFMFBMDO@CrySystemCrtSize?$AA@ 000000003164f7e0     AnimationBase.obj
 0002:0000d7f8       ??_C@_0BD@BBIFHONI@CrySystemCrtMalloc?$AA@ 000000003164f7f8     AnimationBase.obj
 0002:0000d810       ??_C@_0O@LCCIKADF@CryGetMemSize?$AA@ 000000003164f810     AnimationBase.obj
 0002:0000d820       ??_C@_07CKAGCLEE@CryFree?$AA@ 000000003164f820     AnimationBase.obj
 0002:0000d828       ??_C@_0L@FICCDMFO@CryRealloc?$AA@ 000000003164f828     AnimationBase.obj
 0002:0000d838       ??_C@_09MCKPOEAK@CryMalloc?$AA@ 000000003164f838     AnimationBase.obj
 0002:0000d848       ?iid@?1??IID@IEngineModule@@CAAEBUCryGUID@@XZ@4U3@B 000000003164f848     AnimationBase.obj
 0002:0000d858       ??_7IFacialJoystickSerializeContext@@6B@ 000000003164f858     FaceAnimation.obj
 0002:0000d858       ??_7ISystemEventListener@@6B@ 000000003164f858     AnimationBase.obj
 0002:0000d868       __real@40c00000            000000003164f868     AnimationBase.obj
 0002:0000d870       ??_C@_0BD@PJOKHJBB@Pure?5function?5call?$AA@ 000000003164f870     AnimationBase.obj
 0002:0000d888       ??_C@_0CL@LKHBOBAH@Invalid?5parameter?5detected?5in?5CR@ 000000003164f888     AnimationBase.obj
 0002:0000d8b8       ??_C@_0BO@HAMEIFMK@Critical?5Section?5hanging?5lock?$AA@ 000000003164f8b8     AnimationBase.obj
 0002:0000d8d8       ??_7CSystemEventListner_Animation@@6B@ 000000003164f8d8     AnimationBase.obj
 0002:0000d8e8       ??_7CEngineModule_CryAnimation@@6B@ 000000003164f8e8     AnimationBase.obj
 0002:0000d920       ??_C@_0N@EMOPHPFF@CryAnimation?$AA@ 000000003164f920     AnimationBase.obj
 0002:0000d930       ??_C@_09BHIABECK@CryEngine?$AA@ 000000003164f930     AnimationBase.obj
 0002:0000d940       ??_7CFactory@CEngineModule_CryAnimation@@6B@ 000000003164f940     AnimationBase.obj
 0002:0000d970       ??_C@_0BK@PCOPBKHN@EngineModule_CryAnimation?$AA@ 000000003164f970     AnimationBase.obj
 0002:0000d990       ?cid@?1??GetClassID@CFactory@CEngineModule_CryAnimation@@UEBAAEBUCryGUID@@XZ@4U4@B 000000003164f990     AnimationBase.obj
 0002:0000d9a0       ??_7?$sp_counted_impl_p@VCEngineModule_CryAnimation@@@detail@boost@@6B@ 000000003164f9a0     AnimationBase.obj
 0002:0000d9a0       ??_7?$sp_counted_impl_p@VCOperatorQueue@@@detail@boost@@6B@ 000000003164f9a0     OperatorQueue.obj
 0002:0000d9a0       ??_7?$sp_counted_impl_p@VCPoseBlenderLook@@@detail@boost@@6B@ 000000003164f9a0     PoseBlenderLook.obj
 0002:0000d9a0       ??_7?$sp_counted_impl_p@VCFeetPoseStore@@@detail@boost@@6B@ 000000003164f9a0     FeetLock.obj
 0002:0000d9a0       ??_7?$sp_counted_impl_p@VCLimbIk@@@detail@boost@@6B@ 000000003164f9a0     LimbIk.obj
 0002:0000d9a0       ??_7?$sp_counted_impl_p@VCPoseMatching@@@detail@boost@@6B@ 000000003164f9a0     PoseMatching.obj
 0002:0000d9a0       ??_7?$sp_counted_impl_p@VCGroundAlignment@@@detail@boost@@6B@ 000000003164f9a0     GroundAlignment.obj
 0002:0000d9a0       ??_7?$sp_counted_impl_p@VCRecoil@PoseModifier@@@detail@boost@@6B@ 000000003164f9a0     Recoil.obj
 0002:0000d9a0       ??_7?$sp_counted_impl_p@VCPoseAlignerChain@@@detail@boost@@6B@ 000000003164f9a0     PoseAlignerChain.obj
 0002:0000d9a0       ??_7?$sp_counted_impl_p@VCPoseBlenderAim@@@detail@boost@@6B@ 000000003164f9a0     PoseBlenderAim.obj
 0002:0000d9a0       ??_7?$sp_counted_impl_p@VCFeetPoseRestore@@@detail@boost@@6B@ 000000003164f9a0     FeetLock.obj
 0002:0000d9c0       ??_7CAnimationThreadTask@@6B@ 000000003164f9c0     AnimationThreadTask.obj
 0002:0000d9d0       ??_C@_0M@EBCFMMOO@ca_DrawPose?$AA@ 000000003164f9d0     cvars.obj
 0002:0000d9e0       ??_C@_0BE@JOJOEEHJ@Character?5LOD?5ratio?$AA@ 000000003164f9e0     cvars.obj
 0002:0000d9f8       ??_C@_0N@HBLINJMH@ca_lod_ratio?$AA@ 000000003164f9f8     cvars.obj
 0002:0000da08       ??_C@_0BJ@EFBPDBDN@ca_FacialAnimationRadius?$AA@ 000000003164fa08     cvars.obj
 0002:0000da30       ??_C@_0FE@PMLLDBLE@Maximum?5distance?5at?5which?5facial@ 000000003164fa30     cvars.obj
 0002:0000da88       ??_C@_0BI@JIEFPKKN@ca_cloth_air_resistance?$AA@ 000000003164fa88     cvars.obj
 0002:0000daa0       ??_C@_0CN@OHMALND@?$CCadvanced?$CC?5?$CImore?5correct?$CJ?5versio@ 000000003164faa0     cvars.obj
 0002:0000dad0       ??_C@_0BB@FOEHFOJF@ca_cloth_damping?$AA@ 000000003164fad0     cvars.obj
 0002:0000dae8       ??_C@_0BI@MCPNLIO@ca_cloth_stiffness_tang?$AA@ 000000003164fae8     cvars.obj
 0002:0000db00       ??_C@_0DB@ONEEGFBO@stiffness?5for?5shape?5preservation@ 000000003164fb00     cvars.obj
 0002:0000db38       ??_C@_0BI@CJHDJBAA@ca_cloth_stiffness_norm?$AA@ 000000003164fb38     cvars.obj
 0002:0000db50       ??_C@_0EK@DDGLJPG@stiffness?5for?5shape?5preservation@ 000000003164fb50     cvars.obj
 0002:0000dba0       ??_C@_0BC@NNDOBGOG@ca_cloth_friction?$AA@ 000000003164fba0     cvars.obj
 0002:0000dbb8       ??_C@_0BD@GMPAHGEN@ca_cloth_thickness?$AA@ 000000003164fbb8     cvars.obj
 0002:0000dbd0       ??_C@_0BP@NJANAPLJ@thickness?5for?5collision?5checks?$AA@ 000000003164fbd0     cvars.obj
 0002:0000dbf0       ??_C@_0BD@CKHOOACI@ca_cloth_stiffness?$AA@ 000000003164fbf0     cvars.obj
 0002:0000dc08       ??_C@_0BJ@FAIMJLEO@stiffness?5for?5stretching?$AA@ 000000003164fc08     cvars.obj
 0002:0000dc28       ??_C@_0BH@LJCFFBDO@ca_cloth_max_safe_step?$AA@ 000000003164fc28     cvars.obj
 0002:0000dc40       ??_C@_0FG@KEFONKLH@if?5a?5segment?5stretches?5more?5than@ 000000003164fc40     cvars.obj
 0002:0000dc98       ??_C@_0BG@BFLELBCD@ca_cloth_max_timestep?$AA@ 000000003164fc98     cvars.obj
 0002:0000dcb0       ??_C@_0BL@OAGPEHCI@ca_AttachmentCullingRation?$AA@ 000000003164fcb0     cvars.obj
 0002:0000dcd0       ??_C@_0DJ@OHMCHNBH@ration?5between?5size?5of?5attachmen@ 000000003164fcd0     cvars.obj
 0002:0000dd0c       __real@43480000            000000003164fd0c     cvars.obj
 0002:0000dd10       ??_C@_0BM@DHENNHLO@ca_lipsync_phoneme_strength?$AA@ 000000003164fd10     cvars.obj
 0002:0000dd30       ??_C@_0BJ@JEKMPDAK@LipSync?5phoneme?5strength?$AA@ 000000003164fd30     cvars.obj
 0002:0000dd50       ??_C@_0BH@FPKPCHNI@ca_lipsync_vertex_drag?$AA@ 000000003164fd50     cvars.obj
 0002:0000dd68       ??_C@_0DE@MGCDNDAD@Vertex?5drag?5coefficient?5when?5ble@ 000000003164fd68     cvars.obj
 0002:0000dda0       ??_C@_0BC@FCFJEAPB@ca_DeathBlendTime?$AA@ 000000003164fda0     cvars.obj
 0002:0000ddc0       ??_C@_0FH@NFBJKPON@Specifies?5the?5blending?5time?5betw@ 000000003164fdc0     cvars.obj
 0002:0000de18       ??_C@_0BP@IMGGOJJB@ca_MotionBlurMovementThreshold?$AA@ 000000003164fe18     cvars.obj
 0002:0000de40       ??_C@_0EM@LCCEBGGB@?$CCadvanced?$CC?5Set?5motion?5blur?5movem@ 000000003164fe40     cvars.obj
 0002:0000de90       ??_C@_0BG@BMEEJOGJ@ca_ParametricPoolSize?$AA@ 000000003164fe90     cvars.obj
 0002:0000dea8       ??_C@_0BM@IDPDBJFB@Size?5of?5the?5parametric?5pool?$AA@ 000000003164fea8     cvars.obj
 0002:0000dec8       ??_C@_0BH@INCACHFD@ca_MemoryDefragEnabled?$AA@ 000000003164fec8     cvars.obj
 0002:0000dee0       ??_C@_0CF@IHFPNJPB@Enables?5defragmentation?5of?5anim?5@ 000000003164fee0     cvars.obj
 0002:0000df08       ??_C@_0BI@NFLCLMJD@ca_MemoryDefragPoolSize?$AA@ 000000003164ff08     cvars.obj
 0002:0000df20       ??_C@_0CN@LMOEMFHO@Sets?5the?5upper?5limit?5on?5the?5defr@ 000000003164ff20     cvars.obj
 0002:0000df50       ??_C@_0BC@GNNEHGKD@ca_MemoryUsageLog?$AA@ 000000003164ff50     cvars.obj
 0002:0000df68       ??_C@_0BL@HFBKIPEK@enables?5a?5memory?5usage?5log?$AA@ 000000003164ff68     cvars.obj
 0002:0000df88       ??_C@_0BI@FJMAFHBD@ca_physicsProcessImpact?$AA@ 000000003164ff88     cvars.obj
 0002:0000dfa0       ??_C@_0BP@BOCAJCHI@Process?5physics?5impact?5pulses?4?$AA@ 000000003164ffa0     cvars.obj
 0002:0000dfc0       ??_C@_0BH@FNDDEFNL@ca_DecalSizeMultiplier?$AA@ 000000003164ffc0     cvars.obj
 0002:0000dfd8       ??_C@_0CD@HKOANJDA@The?5multiplier?5for?5the?5decal?5siz@ 000000003164ffd8     cvars.obj
 0002:0000e000       ??_C@_0P@MMIJBJMP@ca_DrawVEGInfo?$AA@ 0000000031650000     cvars.obj
 0002:0000e010       ??_C@_0CJ@JONDKHCD@if?5set?5to?51?0?5the?5VEG?5debug?5info?5@ 0000000031650010     cvars.obj
 0002:0000e040       ??_C@_0BN@FLHDGLEO@ca_DisableAnimationUnloading?$AA@ 0000000031650040     cvars.obj
 0002:0000e060       ??_C@_0BN@PCALLINP@Disable?5Animation?5Unloading?4?$AA@ 0000000031650060     cvars.obj
 0002:0000e080       ??_C@_0BJ@ECNHADFF@ca_PrecacheAnimationSets?$AA@ 0000000031650080     cvars.obj
 0002:0000e0a0       ??_C@_0DD@JJEHANKB@Enable?5Precaching?5of?5Animation?5S@ 00000000316500a0     cvars.obj
 0002:0000e0d8       ??_C@_0BH@HIIBGPEN@ca_DBAUnloadRemoveTime?$AA@ 00000000316500d8     cvars.obj
 0002:0000e0f0       ??_C@_0CE@LLCCBPLI@DBA?5Unload?5Timing?3?5DBA?5Remove?5Ti@ 00000000316500f0     cvars.obj
 0002:0000e118       ??_C@_0BL@HBKEKJMC@ca_DBAUnloadUnregisterTime?$AA@ 0000000031650118     cvars.obj
 0002:0000e138       ??_C@_0CI@CFJDCLLO@DBA?5Unload?5Timing?3?5CAF?5Unregiste@ 0000000031650138     cvars.obj
 0002:0000e160       ??_C@_0BD@PGAODFMP@ca_thread1Affinity?$AA@ 0000000031650160     cvars.obj
 0002:0000e178       ??_C@_0CF@HFPHNJC@Affinity?5of?5second?5Animation?5Thr@ 0000000031650178     cvars.obj
 0002:0000e1a0       ??_C@_0BD@BJMMFOPB@ca_thread0Affinity?$AA@ 00000000316501a0     cvars.obj
 0002:0000e1b8       ??_C@_0CE@ILFKAAMM@Affinity?5of?5first?5Animation?5Thre@ 00000000316501b8     cvars.obj
 0002:0000e1e0       ??_C@_09NKFFJOFC@ca_thread?$AA@ 00000000316501e0     cvars.obj
 0002:0000e1f0       ??_C@_0CJ@ILBOOLCK@If?5?$DO0?5enables?5Animation?5Multi?9Th@ 00000000316501f0     cvars.obj
 0002:0000e220       ??_C@_0BC@BLCGFKPE@ca_disable_thread?$AA@ 0000000031650220     cvars.obj
 0002:0000e238       ??_C@_0BP@HOGKGLKJ@TEMP?5Disable?5Animation?5Thread?4?$AA@ 0000000031650238     cvars.obj
 0002:0000e258       ??_C@_0BD@ICEENPMF@ca_UseJointMasking?$AA@ 0000000031650258     cvars.obj
 0002:0000e270       ??_C@_0CP@JFBGPMJI@Use?5Joint?5Masking?5to?5speed?5up?5mo@ 0000000031650270     cvars.obj
 0002:0000e2a0       ??_C@_0M@NIBNONAK@ca_Validate?$AA@ 00000000316502a0     cvars.obj
 0002:0000e2b0       ??_C@_0DD@OGEBBLJF@if?5set?5to?51?0?5will?5run?5validation@ 00000000316502b0     cvars.obj
 0002:0000e2f0       ??_C@_0GL@CKPBEHGA@Lowers?5render?5LODs?5for?5character@ 00000000316502f0     cvars.obj
 0002:0000e360       ??_C@_0CC@ELAFCBEH@ca_AllowMultipleEffectsOfSameNam@ 0000000031650360     cvars.obj
 0002:0000e390       ??_C@_0HB@BPKNANN@Allow?5a?5skeleton?5animation?5to?5sp@ 0000000031650390     cvars.obj
 0002:0000e408       ??_C@_0BM@JGBPONLD@ca_FacialAnimationFramerate?$AA@ 0000000031650408     cvars.obj
 0002:0000e430       ??_C@_0GP@JJBJNLJN@Update?5facial?5system?5at?5a?5maximu@ 0000000031650430     cvars.obj
 0002:0000e4a0       ??_C@_0BJ@DLDLGCNK@ca_SerializeSkeletonAnim?$AA@ 00000000316504a0     cvars.obj
 0002:0000e4c0       ??_C@_0CF@IPALCDKO@Turn?5on?5CSkeletonAnim?5Serializat@ 00000000316504c0     cvars.obj
 0002:0000e4e8       ??_C@_0BE@IFJGJCEG@ca_cloth_vars_reset?$AA@ 00000000316504e8     cvars.obj
 0002:0000e500       ??_C@_0EI@LIDOPPLP@1?5?9?5load?5the?5values?5from?5the?5nex@ 0000000031650500     cvars.obj
 0002:0000e548       ??_C@_0BL@JPIFKACH@ca_MinInPlaceCAFStreamSize?$AA@ 0000000031650548     cvars.obj
 0002:0000e568       ??_C@_0DA@KAGFHHNF@min?5size?5a?5caf?5should?5be?5for?5in?9@ 0000000031650568     cvars.obj
 0002:0000e598       ??_C@_0BG@FKJHEGLJ@ca_UnloadAnimationDBA?$AA@ 0000000031650598     cvars.obj
 0002:0000e5b0       ??_C@_0CC@GHFLMPAJ@if?51?0?5then?5unload?5DBA?5if?5not?5use@ 00000000316505b0     cvars.obj
 0002:0000e5d8       ??_C@_0BG@IKEHFGJO@ca_UnloadAnimationCAF?$AA@ 00000000316505d8     cvars.obj
 0002:0000e5f0       ??_C@_0DF@NHCELDFK@unloading?5streamed?5CAFs?5as?5soon?5@ 00000000316505f0     cvars.obj
 0002:0000e628       ??_C@_0O@ODDFHGJE@ca_UseIMG_AIM?$AA@ 0000000031650628     cvars.obj
 0002:0000e638       ??_C@_0O@KENLDGGM@ca_UseIMG_CAF?$AA@ 0000000031650638     cvars.obj
 0002:0000e650       ??_C@_0EM@LEHOJILF@if?51?0?5then?5we?5use?5the?5IMG?5file?4?5@ 0000000031650650     cvars.obj
 0002:0000e6a0       ??_C@_0BH@ICIDFFCH@ca_DebugCriticalErrors?$AA@ 00000000316506a0     cvars.obj
 0002:0000e6c0       ??_C@_0ED@IHNECKBD@if?51?0?5then?5we?5stop?5with?5a?5Fatal?9@ 00000000316506c0     cvars.obj
 0002:0000e708       ??_C@_0M@HFNGIPLD@ca_SaveAABB?$AA@ 0000000031650708     cvars.obj
 0002:0000e718       ??_C@_0DH@LDGHIGLM@if?5the?5AABB?5is?5invalid?0?5replace?5@ 0000000031650718     cvars.obj
 0002:0000e750       ??_C@_0BE@NGCNMBH@ca_DebugADIKTargets?$AA@ 0000000031650750     cvars.obj
 0002:0000e770       ??_C@_0FB@HHNKIAKE@If?51?0?5then?5it?5will?5show?5if?5there@ 0000000031650770     cvars.obj
 0002:0000e7c8       ??_C@_0BC@KOCIPNFH@ca_useADIKTargets?$AA@ 00000000316507c8     cvars.obj
 0002:0000e7e0       ??_C@_0CB@JPJDCCLB@Use?5Animation?5Driven?5Ik?5Targets?4@ 00000000316507e0     cvars.obj
 0002:0000e808       ??_C@_0BD@JJBPFNOD@ca_SkipLoadThinFat?$AA@ 0000000031650808     cvars.obj
 0002:0000e820       ??_C@_0CG@KNEIJJLF@Skip?5loading?5fat?7hin?5stuff?5if?5en@ 0000000031650820     cvars.obj
 0002:0000e848       ??_C@_0BD@EADKPCNL@ca_DebugFacialEyes?$AA@ 0000000031650848     cvars.obj
 0002:0000e860       ??_C@_0BH@BMFMOOJN@Debug?5facial?5eyes?5info?$AA@ 0000000031650860     cvars.obj
 0002:0000e878       ??_C@_0P@BPDLLOAN@ca_DebugFacial?$AA@ 0000000031650878     cvars.obj
 0002:0000e888       ??_C@_0BL@IAGGECCM@Debug?5facial?5playback?5info?$AA@ 0000000031650888     cvars.obj
 0002:0000e8a8       ??_C@_0BB@JIJFFIF@ca_lipsync_debug?$AA@ 00000000316508a8     cvars.obj
 0002:0000e8c0       ??_C@_0CE@HJKBKFCI@Enables?5facial?5animation?5debug?5d@ 00000000316508c0     cvars.obj
 0002:0000e8e8       ??_C@_0BD@PACKHAKI@ca_eyes_procedural?$AA@ 00000000316508e8     cvars.obj
 0002:0000e900       ??_C@_0CL@JEGBKNKL@Enables?1Disables?5procedural?5eyes@ 0000000031650900     cvars.obj
 0002:0000e930       ??_C@_0BN@GPJFFPOO@ca_lipsync_phoneme_crossfade?$AA@ 0000000031650930     cvars.obj
 0002:0000e950       ??_C@_0DB@CMGMAGFM@Cross?5fade?5time?5between?5phonemes@ 0000000031650950     cvars.obj
 0002:0000e988       ??_C@_0BK@GHKEBONN@ca_lipsync_phoneme_offset?$AA@ 0000000031650988     cvars.obj
 0002:0000e9a8       ??_C@_0DI@KHLBKNAK@Offset?5phoneme?5start?5time?5by?5thi@ 00000000316509a8     cvars.obj
 0002:0000e9e0       ??_C@_0BI@KPCIAMFN@ca_DebugSkeletonEffects?$AA@ 00000000316509e0     cvars.obj
 0002:0000e9f8       ??_C@_0DO@JINKPBJJ@If?5true?0?5dump?5log?5messages?5when?5@ 00000000316509f8     cvars.obj
 0002:0000ea38       ??_C@_0O@MCJKIJHD@ca_KeepModels?$AA@ 0000000031650a38     cvars.obj
 0002:0000ea50       ??_C@_0GP@BADIOIKE@If?5set?5to?51?0?5will?5prevent?5models@ 0000000031650a50     cvars.obj
 0002:0000eac0       ??_C@_0BE@FHGGOKBM@ca_AnimWarningLevel?$AA@ 0000000031650ac0     cvars.obj
 0002:0000eae0       ??_C@_0FF@LOGLEDBK@if?5you?5set?5this?5to?50?0?5there?5won?8@ 0000000031650ae0     cvars.obj
 0002:0000eb38       ??_C@_0BB@HNJCBPAG@ca_DumpUsedAnims?$AA@ 0000000031650b38     cvars.obj
 0002:0000eb50       ??_C@_0CO@IKBCLPFN@writes?5animation?5asset?5statistic@ 0000000031650b50     cvars.obj
 0002:0000eb80       ??_C@_0BI@PDMPAFEP@ca_StoreAnimNamesOnLoad?$AA@ 0000000031650b80     cvars.obj
 0002:0000eba0       ??_C@_0EO@EOFGBPOE@stores?5the?5names?5of?5animations?5d@ 0000000031650ba0     cvars.obj
 0002:0000ebf0       ??_C@_0BO@HPFFLABM@ca_DebugAnimUsageOnFileAccess?$AA@ 0000000031650bf0     cvars.obj
 0002:0000ec10       ??_C@_0FG@NHLJNPAJ@shows?5what?5animation?5assets?5are?5@ 0000000031650c10     cvars.obj
 0002:0000ec68       ??_C@_0BC@DAKMICOE@ca_DebugAnimUsage?$AA@ 0000000031650c68     cvars.obj
 0002:0000ec80       ??_C@_0DC@KNJOJOPG@shows?5what?5animation?5assets?5are?5@ 0000000031650c80     cvars.obj
 0002:0000ecb8       ??_C@_0BE@HFGKIJMC@ca_DebugAnimUpdates?$AA@ 0000000031650cb8     cvars.obj
 0002:0000ecd0       ??_C@_0CF@EKFABEPM@shows?5the?5amount?5of?5skeleton?9upd@ 0000000031650cd0     cvars.obj
 0002:0000ecf8       ??_C@_0BG@BADHPGJH@ca_ReloadAllCHRPARAMS?$AA@ 0000000031650cf8     cvars.obj
 0002:0000ed10       ??_C@_0BF@KHBHJIJP@realod?5all?5CHRPARAMS?$AA@ 0000000031650d10     cvars.obj
 0002:0000ed28       ??_C@_0BI@EMMOJMOM@ca_TrackSkinTransMemory?$AA@ 0000000031650d28     cvars.obj
 0002:0000ed40       ??_C@_0DI@IMICCPNO@shows?5how?5much?5memory?5the?5Skinni@ 0000000031650d40     cvars.obj
 0002:0000ed78       ??_C@_0BD@MGJEPDDC@ca_DebugModelCache?$AA@ 0000000031650d78     cvars.obj
 0002:0000ed90       ??_C@_0EF@DJBHIAFJ@shows?5what?5models?5are?5currently?5@ 0000000031650d90     cvars.obj
 0002:0000edd8       ??_C@_0N@OFLBFAKC@ca_UseDecals?$AA@ 0000000031650dd8     cvars.obj
 0002:0000edf0       ??_C@_0HN@KMILDOJK@if?5set?5to?50?0?5effectively?5disable@ 0000000031650df0     cvars.obj
 0002:0000ee70       ??_C@_0BM@HPCOFAEL@ca_ApplyJointVelocitiesMode?$AA@ 0000000031650e70     cvars.obj
 0002:0000ee90       ??_C@_0FI@MPAFKAPI@Joint?5velocity?5preservation?5code@ 0000000031650e90     cvars.obj
 0002:0000eee8       ??_C@_0BI@PFJEMCOI@ca_ForceUpdateSkeletons?$AA@ 0000000031650ee8     cvars.obj
 0002:0000ef00       ??_C@_0DC@NELAHNFF@Always?5update?5all?5skeletons?0?5eve@ 0000000031650f00     cvars.obj
 0002:0000ef38       ??_C@_0BC@PILFPGJD@ca_LockFeetWithIK?$AA@ 0000000031650f38     cvars.obj
 0002:0000ef50       ??_C@_0GA@GOGDMLA@If?5this?5is?5set?5to?51?0?5then?5we?5loc@ 0000000031650f50     cvars.obj
 0002:0000efb0       ??_C@_0BG@FKLMHNFH@ca_UseFacialAnimation?$AA@ 0000000031650fb0     cvars.obj
 0002:0000efc8       ??_C@_0DD@CHNCAAIJ@If?5this?5is?5set?5to?51?0?5we?5can?5play@ 0000000031650fc8     cvars.obj
 0002:0000f000       ??_C@_0BD@DLIDBMDO@ca_DrawAimIKVEGrid?$AA@ 0000000031651000     cvars.obj
 0002:0000f018       ??_C@_0DM@IAKBDCDE@if?5set?5to?51?0?5we?5will?5the?5the?5gri@ 0000000031651018     cvars.obj
 0002:0000f058       ??_C@_0M@DEJLCBPH@ca_UseAimIK?$AA@ 0000000031651058     cvars.obj
 0002:0000f068       ??_C@_0N@PEJBAIDG@ca_UseLookIK?$AA@ 0000000031651068     cvars.obj
 0002:0000f080       ??_C@_0EM@MHHKLIJM@If?5this?5is?5set?5to?51?0?5then?5we?5are@ 0000000031651080     cvars.obj
 0002:0000f0d0       ??_C@_0O@DGJMLBON@ca_UsePhysics?$AA@ 00000000316510d0     cvars.obj
 0002:0000f0e0       ??_C@_0DA@COLJGECI@the?5physics?5is?5not?5applied?5?$CIeffe@ 00000000316510e0     cvars.obj
 0002:0000f110       ??_C@_09CFBCPLFA@ca_NoAnim?$AA@ 0000000031651110     cvars.obj
 0002:0000f120       ??_C@_0EF@HCMHNOKH@the?5animation?5isn?8t?5updated?5?$CIthe@ 0000000031651120     cvars.obj
 0002:0000f168       ??_C@_0M@FBHAPKJL@ca_UseMorph?$AA@ 0000000031651168     cvars.obj
 0002:0000f180       ??_C@_0FE@IAIFCBEP@the?5morph?5skinning?5step?5is?5skipp@ 0000000031651180     cvars.obj
 0002:0000f1d8       ??_C@_0BK@MPBPEBJP@ca_LoadUncompressedChunks?$AA@ 00000000316511d8     cvars.obj
 0002:0000f200       ??_C@_0EE@NHPHCLII@If?5this?51?0?5then?5uncompressed?5chu@ 0000000031651200     cvars.obj
 0002:0000f248       ??_C@_0BL@OKMLDGKP@ca_DebugAnimationStreaming?$AA@ 0000000031651248     cvars.obj
 0002:0000f268       ??_C@_0DM@DAIEEMPF@if?5this?5is?51?0?5then?5it?5shows?5what@ 0000000031651268     cvars.obj
 0002:0000f2a8       ??_C@_0BG@BBDHFJLC@ca_DebugCommandBuffer?$AA@ 00000000316512a8     cvars.obj
 0002:0000f2c0       ??_C@_0EI@OMBFEIBM@if?5this?5is?51?0?5it?5will?5print?5the?5@ 00000000316512c0     cvars.obj
 0002:0000f308       ??_C@_0N@HDBDOJNB@ca_DebugText?$AA@ 0000000031651308     cvars.obj
 0002:0000f320       ??_C@_0JG@OKJGDI@if?5this?5is?51?0?5it?5will?5print?5some@ 0000000031651320     cvars.obj
 0002:0000f3b8       ??_C@_0BI@DBBEJHFA@ca_DebugAnimMemTracking?$AA@ 00000000316513b8     cvars.obj
 0002:0000f3d0       ??_C@_0DG@JDKMHCEB@if?5this?5is?51?0?5then?5its?5shows?5the@ 00000000316513d0     cvars.obj
 0002:0000f408       ??_C@_0BD@CMLGDBNA@ca_DebugSWSkinning?$AA@ 0000000031651408     cvars.obj
 0002:0000f420       ??_C@_0FD@KLENFGMF@if?5this?5is?51?0?5then?5we?5will?5see?5a@ 0000000031651420     cvars.obj
 0002:0000f478       ??_C@_0BB@NHGLINGA@ca_DrawCGAAsSkin?$AA@ 0000000031651478     cvars.obj
 0002:0000f490       ??_C@_0EL@HPAKLPED@if?5this?5is?51?0?5will?5draw?5the?5CGA?5@ 0000000031651490     cvars.obj
 0002:0000f4e0       ??_C@_09OMCHEIFA@ca_DrawCC?$AA@ 00000000316514e0     cvars.obj
 0002:0000f4f0       ??_C@_0CO@CCJDMHEB@if?5this?5is?50?0?5will?5not?5draw?5the?5@ 00000000316514f0     cvars.obj
 0002:0000f520       ??_C@_0L@OPFPKGIL@ca_DrawCHR?$AA@ 0000000031651520     cvars.obj
 0002:0000f530       ??_C@_0CP@HHALCDAN@if?5this?5is?50?0?5will?5not?5draw?5the?5@ 0000000031651530     cvars.obj
 0002:0000f560       ??_C@_0L@IFOMKACE@ca_DrawCGA?$AA@ 0000000031651560     cvars.obj
 0002:0000f570       ??_C@_0CP@CIFCFNOP@if?5this?5is?50?0?5will?5not?5draw?5the?5@ 0000000031651570     cvars.obj
 0002:0000f5a0       ??_C@_0P@OIKKJBHD@ca_DrawLocator?$AA@ 00000000316515a0     cvars.obj
 0002:0000f5b0       ??_C@_0HA@LKFLMFEA@if?5this?5is?51?0?5we?5will?5draw?5the?5b@ 00000000316515b0     cvars.obj
 0002:0000f620       ??_C@_0BA@IHIJCMGE@ca_DrawBaseMesh?$AA@ 0000000031651620     cvars.obj
 0002:0000f630       ??_C@_0CL@LLDIBBLG@if?5this?5is?50?0?5will?5not?5draw?5the?5@ 0000000031651630     cvars.obj
 0002:0000f660       ??_C@_0BF@OJMPMHBN@ca_DrawAttachmentOBB?$AA@ 0000000031651660     cvars.obj
 0002:0000f678       ??_C@_0BD@DFPABPCK@ca_DrawAttachments?$AA@ 0000000031651678     cvars.obj
 0002:0000f690       ??_C@_0DE@GKAJOCDP@if?5this?5is?50?0?5will?5not?5draw?5the?5@ 0000000031651690     cvars.obj
 0002:0000f6c8       ??_C@_0P@NLGPICIE@ca_DrawNormals?$AA@ 00000000316516c8     cvars.obj
 0002:0000f6d8       ??_C@_0CM@PHOOPKHH@draws?5the?5normals?5of?5the?5rendere@ 00000000316516d8     cvars.obj
 0002:0000f708       ??_C@_0BB@IOBJBGIF@ca_DrawBinormals?$AA@ 0000000031651708     cvars.obj
 0002:0000f720       ??_C@_0CO@DAEPAFP@draws?5the?5binormals?5of?5the?5rende@ 0000000031651720     cvars.obj
 0002:0000f750       ??_C@_0BA@JJFLHFEB@ca_DrawTangents?$AA@ 0000000031651750     cvars.obj
 0002:0000f760       ??_C@_0CN@OIDHNMMA@draws?5the?5tangents?5of?5the?5render@ 0000000031651760     cvars.obj
 0002:0000f790       ??_C@_0O@NLFIMKFH@ca_DrawLookIK?$AA@ 0000000031651790     cvars.obj
 0002:0000f7a0       ??_C@_0CB@BMHNHPOO@draws?5a?5visualization?5of?5look?5ik@ 00000000316517a0     cvars.obj
 0002:0000f7c8       ??_C@_0BA@HBFJBKOG@ca_DrawAimPoses?$AA@ 00000000316517c8     cvars.obj
 0002:0000f7d8       ??_C@_0CF@GBEFKEKH@draws?5the?5wireframe?5of?5the?5aim?5p@ 00000000316517d8     cvars.obj
 0002:0000f800       ??_C@_0BB@KHFHLIDN@ca_DrawWireframe?$AA@ 0000000031651800     cvars.obj
 0002:0000f818       ??_C@_0DD@NFCANLL@draws?5a?5wireframe?5on?5top?5of?5the?5@ 0000000031651818     cvars.obj
 0002:0000f850       ??_C@_0BI@HGFGBAN@ca_DrawEmptyAttachments?$AA@ 0000000031651850     cvars.obj
 0002:0000f870       ??_C@_0EF@ONPLPOJD@draws?5a?5wireframe?5cube?5if?5there?5@ 0000000031651870     cvars.obj
 0002:0000f8b8       ??_C@_0BE@NOHAPOFE@ca_DrawPositionPost?$AA@ 00000000316518b8     cvars.obj
 0002:0000f8d0       ??_C@_0DJ@EDKKDGKP@draws?5the?5world?5position?5of?5the?5@ 00000000316518d0     cvars.obj
 0002:0000f910       ??_C@_0BE@GAOKAHKJ@ca_DrawDecalsBBoxes?$AA@ 0000000031651910     cvars.obj
 0002:0000f928       ??_C@_0CJ@CMAGMJDF@if?5set?5to?51?0?5the?5decals?5bboxes?5a@ 0000000031651928     cvars.obj
 0002:0000f958       ??_C@_0BA@NEIBDHAP@ca_DrawSkeleton?$AA@ 0000000031651958     cvars.obj
 0002:0000f968       ??_C@_0CD@BAIOFGGC@if?5set?5to?51?0?5the?5skeleton?5is?5dra@ 0000000031651968     cvars.obj
 0002:0000f990       ??_C@_0M@ODANEJOH@ca_DrawBBox?$AA@ 0000000031651990     cvars.obj
 0002:0000f9a0       ??_C@_0DM@HALBLLMA@if?5set?5to?51?0?5the?5own?5bounding?5bo@ 00000000316519a0     cvars.obj
 0002:0000f9e0       ??_C@_0BB@FGCINMPC@ca_usePhysicsLOD?$AA@ 00000000316519e0     cvars.obj
 0002:0000f9f8       ??_C@_0DP@OALMMENO@If?5set?5to?50?5it?5loads?5only?5LOD0?4?5@ 00000000316519f8     cvars.obj
 0002:0000fa38       ??_C@_0BA@HNABOPEG@ca_FilterJoints?$AA@ 0000000031651a38     cvars.obj
 0002:0000fa48       ??_C@_0BB@BCONMOMD@ca_CharEditModel?$AA@ 0000000031651a48     cvars.obj
 0002:0000fa60       ??_C@_0DI@MGGBHHJD@objects?1characters?1human?1us?1nano@ 0000000031651a60     cvars.obj
 0002:0000faa0       ??_7CPool@Memory@@6B@      0000000031651aa0     Pool.obj
 0002:0000fac8       ??_C@_05FHGOFLKH@Fatal?$AA@ 0000000031651ac8     Pool.obj
 0002:0000fad0       ??_7CPoolFrameLocal@Memory@@6B@ 0000000031651ad0     Pool.obj
 0002:0000faf8       ??_C@_0BH@MCAFGJEB@SkinAttachmentTangents?$AA@ 0000000031651af8     _RenderSkinsSW.obj
 0002:0000fb10       _pDefaultRawDllMain        0000000031651b10     MSVCRT:crtdll.obj
 0002:0000fb10       _pRawDllMain               0000000031651b10     MSVCRT:crtdll.obj
 0002:0000fb70       __rtc_iaa                  0000000031651b70     MSVCRT:_initsect_.obj
 0002:0000fb78       __rtc_izz                  0000000031651b78     MSVCRT:_initsect_.obj
 0002:0000fb80       __rtc_taa                  0000000031651b80     MSVCRT:_initsect_.obj
 0002:0000fb88       __rtc_tzz                  0000000031651b88     MSVCRT:_initsect_.obj
 0002:0002094c       __IMPORT_DESCRIPTOR_KERNEL32 000000003166294c     kernel32:KERNEL32.dll
 0002:00020960       __IMPORT_DESCRIPTOR_USER32 0000000031662960     user32:USER32.dll
 0002:00020974       __IMPORT_DESCRIPTOR_MSVCR100 0000000031662974     MSVCRT:MSVCR100.dll
 0002:00020988       __NULL_IMPORT_DESCRIPTOR   0000000031662988     kernel32:KERNEL32.dll
 0003:00000000       ?sEmptyStringBuffer@?1??_emptyHeader@?$CryStringT@D@@KAPEAUStrHeader@2@XZ@4PAU32@A 0000000031664000     AnimEventList.obj
 0003:00000018       ?g_firstValidator@SBatchUpdateValidator@@2U1@A 0000000031664018     SkeletonPhysics.obj
 0003:00000040       ?szEyeBoneNames@CEyeMovementFaceAnim@@0PAPEBDA 0000000031664040     EyeMovementFaceAnim.obj
 0003:000004b8       ?s_factory@CFactory@CFeetPoseStore@@0V12@A 00000000316644b8     FeetLock.obj
 0003:000004e0       ?s_factory@CFactory@CFeetPoseRestore@@0V12@A 00000000316644e0     FeetLock.obj
 0003:00000508       ?g_leftLeg@@3PEBDEB        0000000031664508     GroundAlignment.obj
 0003:00000510       ?g_rightLeg@@3PEBDEB       0000000031664510     GroundAlignment.obj
 0003:00000518       ?fVec3_OneZ@?$Vec3Constants@M@@2U?$Vec3_tpl@M@@B 0000000031664518     GroundAlignment.obj
 0003:00000528       ?s_factory@CFactory@CLimbIk@@0V12@A 0000000031664528     LimbIk.obj
 0003:00000550       ?s_factory@CFactory@CRecoil@PoseModifier@@0V123@A 0000000031664550     Recoil.obj
 0003:00000590       ?g_arrLimbNames@?1??SetJointName@CModelJoint@@QEAAXPEBD@Z@4PAPEBDA 0000000031664590     LoaderCGA.obj
 0003:00002448       ?strEmpty@@3PEBDEB         0000000031666448     ModelAnimationSet.obj
 0003:00002460       ?m_seed@CLCGRndGen@@0_KA   0000000031666460     AnimationBase.obj
 0003:00002490       ?g_DefaultAnim@@3VCAnimation@@A 0000000031666490     AnimationBase.obj
 0003:00002500       ?g_IdentityQuatT@@3U?$QuatT_tpl@M@@A 0000000031666500     AnimationBase.obj
 0003:00002520       ?g_Consoleself@@3UConsole@@A 0000000031666520     cvars.obj
 0003:000026f8       ?fVec3_Zero@?$Vec3Constants@M@@2U?$Vec3_tpl@M@@B 00000000316666f8     stdafx.obj
 0003:00002708       ?fVec3_One@?$Vec3Constants@M@@2U?$Vec3_tpl@M@@B 0000000031666708     stdafx.obj
 0003:00002718       ?fVec2_Zero@?$Vec2Constants@M@@2U?$Vec2_tpl@M@@A 0000000031666718     stdafx.obj
 0003:00002720       ?fVec2_OneX@?$Vec2Constants@M@@2U?$Vec2_tpl@M@@A 0000000031666720     stdafx.obj
 0003:00002728       ?fVec2_OneY@?$Vec2Constants@M@@2U?$Vec2_tpl@M@@A 0000000031666728     stdafx.obj
 0003:00002730       ?fVec2_One@?$Vec2Constants@M@@2U?$Vec2_tpl@M@@A 0000000031666730     stdafx.obj
 0003:00002738       _fltused                   0000000031666738     MSVCRT:dllsupp.obj
 0003:00002740       __native_dllmain_reason    0000000031666740     MSVCRT:natstart.obj
 0003:00002744       __native_vcclrit_reason    0000000031666744     MSVCRT:natstart.obj
 0003:00002748       __security_cookie          0000000031666748     MSVCRT:gs_cookie.obj
 0003:00002750       __security_cookie_complement 0000000031666750     MSVCRT:gs_cookie.obj
 0003:00002760       ?s_used_memory@?1??_usedMemory@?$CryStringT@D@@SA_K_J@Z@4_KA 0000000031666760     AnimEventList.obj
 0003:00002768       ?s_EmptyElems@?1??set_null@?$SmallDynStorage@VCAnimEventData@@HUStandardAlloc@NAlloc@@@NArray@@IEAAXXZ@4PEAVCAnimEventData@@EA 0000000031666768     AnimEventList.obj
 0003:00002770       ?s_EmptyHeader@?1??set_null@?$SmallDynStorage@VCAnimEventData@@HUStandardAlloc@NAlloc@@@NArray@@IEAAXXZ@4UEmptyHeader@23@A 0000000031666770     AnimEventList.obj
 0003:0000277c       ??_B?1??set_null@?$SmallDynStorage@VCAnimEventData@@HUStandardAlloc@NAlloc@@@NArray@@IEAAXXZ@51 000000003166677c     AnimEventList.obj
 0003:00002780       ?s_pMemReplay@?1??CryGetIMemReplay@@YAPEAUIMemReplay@@XZ@4PEAU2@EA 0000000031666780     AnimEventList.obj
 0003:00002788       ?s_dummyMemReplay@?1??CryGetIMemReplay@@YAPEAUIMemReplay@@XZ@4UCDummyMemReplay@@A 0000000031666788     AnimEventList.obj
 0003:00002790       ??_B?1??CryGetIMemReplay@@YAPEAUIMemReplay@@XZ@51 0000000031666790     AnimEventList.obj
 0003:00002798       ?s_EmptyElems@?1??set_null@?$SmallDynStorage@EHUStandardAlloc@NAlloc@@@NArray@@IEAAXXZ@4PEAEEA 0000000031666798     Attachment.obj
 0003:000027a0       ?s_EmptyHeader@?1??set_null@?$SmallDynStorage@EHUStandardAlloc@NAlloc@@@NArray@@IEAAXXZ@4UEmptyHeader@23@A 00000000316667a0     Attachment.obj
 0003:000027a8       ??_B?1??set_null@?$SmallDynStorage@EHUStandardAlloc@NAlloc@@@NArray@@IEAAXXZ@51 00000000316667a8     Attachment.obj
 0003:00002bd0       ?s_used_memory@?1??_usedMemory@?$CryStackStringT@D$0CAA@@@SA_K_K@Z@4_KA 0000000031666bd0     LoaderSKIN.obj
 0003:00002bd8       ?s_EmptyElems@?1??set_null@?$SmallDynStorage@UMorphTargetVertex@@HUStandardAlloc@NAlloc@@@NArray@@IEAAXXZ@4PEAUMorphTargetVertex@@EA 0000000031666bd8     LoaderSKIN.obj
 0003:00002be0       ?s_EmptyHeader@?1??set_null@?$SmallDynStorage@UMorphTargetVertex@@HUStandardAlloc@NAlloc@@@NArray@@IEAAXXZ@4UEmptyHeader@23@A 0000000031666be0     LoaderSKIN.obj
 0003:00002be8       ??_B?1??set_null@?$SmallDynStorage@UMorphTargetVertex@@HUStandardAlloc@NAlloc@@@NArray@@IEAAXXZ@51 0000000031666be8     LoaderSKIN.obj
 0003:00002bf0       ?s_EmptyElems@?1??set_null@?$SmallDynStorage@UExtSkinVertex@@HUStandardAlloc@NAlloc@@@NArray@@IEAAXXZ@4PEAUExtSkinVertex@@EA 0000000031666bf0     LoaderSKIN.obj
 0003:00002bf8       ?s_EmptyHeader@?1??set_null@?$SmallDynStorage@UExtSkinVertex@@HUStandardAlloc@NAlloc@@@NArray@@IEAAXXZ@4UEmptyHeader@23@A 0000000031666bf8     LoaderSKIN.obj
 0003:00002c00       ??_B?1??set_null@?$SmallDynStorage@UExtSkinVertex@@HUStandardAlloc@NAlloc@@@NArray@@IEAAXXZ@51 0000000031666c00     LoaderSKIN.obj
 0003:00002c08       ?s_EmptyElems@?1??set_null@?$SmallDynStorage@VCModelMesh@@HUStandardAlloc@NAlloc@@@NArray@@IEAAXXZ@4PEAVCModelMesh@@EA 0000000031666c08     LoaderSKIN.obj
 0003:00002c10       ?s_EmptyHeader@?1??set_null@?$SmallDynStorage@VCModelMesh@@HUStandardAlloc@NAlloc@@@NArray@@IEAAXXZ@4UEmptyHeader@23@A 0000000031666c10     LoaderSKIN.obj
 0003:00002c1c       ??_B?1??set_null@?$SmallDynStorage@VCModelMesh@@HUStandardAlloc@NAlloc@@@NArray@@IEAAXXZ@51 0000000031666c1c     LoaderSKIN.obj
 0003:00002c20       ?s_EmptyElems@?1??set_null@?$SmallDynStorage@USJointInfo@CSkin@@HUStandardAlloc@NAlloc@@@NArray@@IEAAXXZ@4PEAUSJointInfo@CSkin@@EA 0000000031666c20     LoaderSKIN.obj
 0003:00002c28       ?s_EmptyHeader@?1??set_null@?$SmallDynStorage@USJointInfo@CSkin@@HUStandardAlloc@NAlloc@@@NArray@@IEAAXXZ@4UEmptyHeader@23@A 0000000031666c28     LoaderSKIN.obj
 0003:00002c34       ??_B?1??set_null@?$SmallDynStorage@USJointInfo@CSkin@@HUStandardAlloc@NAlloc@@@NArray@@IEAAXXZ@51 0000000031666c34     LoaderSKIN.obj
 0003:00002c38       ?s_EmptyElems@?1??set_null@?$SmallDynStorage@U?$Vec3_tpl@M@@HUStandardAlloc@NAlloc@@@NArray@@IEAAXXZ@4PEAU?$Vec3_tpl@M@@EA 0000000031666c38     LoaderSKIN.obj
 0003:00002c40       ?s_EmptyHeader@?1??set_null@?$SmallDynStorage@U?$Vec3_tpl@M@@HUStandardAlloc@NAlloc@@@NArray@@IEAAXXZ@4UEmptyHeader@23@A 0000000031666c40     LoaderSKIN.obj
 0003:00002c48       ??_B?1??set_null@?$SmallDynStorage@U?$Vec3_tpl@M@@HUStandardAlloc@NAlloc@@@NArray@@IEAAXXZ@51 0000000031666c48     LoaderSKIN.obj
 0003:00002c50       ?s_EmptyElems@?1??set_null@?$SmallDynStorage@U?$Quat_tpl@M@@HUStandardAlloc@NAlloc@@@NArray@@IEAAXXZ@4PEAU?$Quat_tpl@M@@EA 0000000031666c50     LoaderSKIN.obj
 0003:00002c58       ?s_EmptyHeader@?1??set_null@?$SmallDynStorage@U?$Quat_tpl@M@@HUStandardAlloc@NAlloc@@@NArray@@IEAAXXZ@4UEmptyHeader@23@A 0000000031666c58     LoaderSKIN.obj
 0003:00002c60       ??_B?1??set_null@?$SmallDynStorage@U?$Quat_tpl@M@@HUStandardAlloc@NAlloc@@@NArray@@IEAAXXZ@51 0000000031666c60     LoaderSKIN.obj
 0003:00002c68       ?s_EmptyElems@?1??set_null@?$SmallDynStorage@URChunk@@HUStandardAlloc@NAlloc@@@NArray@@IEAAXXZ@4PEAURChunk@@EA 0000000031666c68     LoaderSKIN.obj
 0003:00002c70       ?s_EmptyHeader@?1??set_null@?$SmallDynStorage@URChunk@@HUStandardAlloc@NAlloc@@@NArray@@IEAAXXZ@4UEmptyHeader@23@A 0000000031666c70     LoaderSKIN.obj
 0003:00002c7c       ??_B?1??set_null@?$SmallDynStorage@URChunk@@HUStandardAlloc@NAlloc@@@NArray@@IEAAXXZ@51 0000000031666c7c     LoaderSKIN.obj
 0003:00002c80       ?s_EmptyElems@?1??set_null@?$SmallDynStorage@UBoneIndices8@@HUStandardAlloc@NAlloc@@@NArray@@IEAAXXZ@4PEAUBoneIndices8@@EA 0000000031666c80     LoaderSKIN.obj
 0003:00002c88       ?s_EmptyHeader@?1??set_null@?$SmallDynStorage@UBoneIndices8@@HUStandardAlloc@NAlloc@@@NArray@@IEAAXXZ@4UEmptyHeader@23@A 0000000031666c88     LoaderSKIN.obj
 0003:00002c90       ??_B?1??set_null@?$SmallDynStorage@UBoneIndices8@@HUStandardAlloc@NAlloc@@@NArray@@IEAAXXZ@51 0000000031666c90     LoaderSKIN.obj
 0003:00002c98       ?s_EmptyElems@?1??set_null@?$SmallDynStorage@UBoneWeights8@@HUStandardAlloc@NAlloc@@@NArray@@IEAAXXZ@4PEAUBoneWeights8@@EA 0000000031666c98     LoaderSKIN.obj
 0003:00002ca0       ?s_EmptyHeader@?1??set_null@?$SmallDynStorage@UBoneWeights8@@HUStandardAlloc@NAlloc@@@NArray@@IEAAXXZ@4UEmptyHeader@23@A 0000000031666ca0     LoaderSKIN.obj
 0003:00002ca8       ??_B?1??set_null@?$SmallDynStorage@UBoneWeights8@@HUStandardAlloc@NAlloc@@@NArray@@IEAAXXZ@51 0000000031666ca8     LoaderSKIN.obj
 0003:00002cb0       ?s_EmptyElems@?1??set_null@?$SmallDynStorage@V?$_smart_ptr@UCMorphTarget@@@@HUStandardAlloc@NAlloc@@@NArray@@IEAAXXZ@4PEAV?$_smart_ptr@UCMorphTarget@@@@EA 0000000031666cb0     LoaderSKIN.obj
 0003:00002cb8       ?s_EmptyHeader@?1??set_null@?$SmallDynStorage@V?$_smart_ptr@UCMorphTarget@@@@HUStandardAlloc@NAlloc@@@NArray@@IEAAXXZ@4UEmptyHeader@23@A 0000000031666cb8     LoaderSKIN.obj
 0003:00002cc4       ??_B?1??set_null@?$SmallDynStorage@V?$_smart_ptr@UCMorphTarget@@@@HUStandardAlloc@NAlloc@@@NArray@@IEAAXXZ@51 0000000031666cc4     LoaderSKIN.obj
 0003:00002cc8       ?BIAS_SCALE_16BIT@?6??FromFrameReflection@QTangent@@YA?AU?$Quat_tpl@M@@U3@M@Z@4MB 0000000031666cc8     LoaderSKIN.obj
 0003:00002ccc       ??_B?6??FromFrameReflection@QTangent@@YA?AU?$Quat_tpl@M@@U2@M@Z@56 0000000031666ccc     LoaderSKIN.obj
 0003:00003150       ?s_EmptyElems@?1??set_null@?$SmallDynStorage@PEAVCAttachmentSKIN@@HUStandardAlloc@NAlloc@@@NArray@@IEAAXXZ@4PEAPEAVCAttachmentSKIN@@EA 0000000031667150     ModelSkin.obj
 0003:00003158       ?s_EmptyHeader@?1??set_null@?$SmallDynStorage@PEAVCAttachmentSKIN@@HUStandardAlloc@NAlloc@@@NArray@@IEAAXXZ@4UEmptyHeader@23@A 0000000031667158     ModelSkin.obj
 0003:00003164       ??_B?1??set_null@?$SmallDynStorage@PEAVCAttachmentSKIN@@HUStandardAlloc@NAlloc@@@NArray@@IEAAXXZ@51 0000000031667164     ModelSkin.obj
 0003:00003168       ?pClouds@?1??InitRenderingFlags@SRenderingPassInfo@@AEAAXI@Z@4PEAUICVar@@EA 0000000031667168     ParametricSampler.obj
 0003:00003170       ?pRoads@?1??InitRenderingFlags@SRenderingPassInfo@@AEAAXI@Z@4PEAUICVar@@EA 0000000031667170     ParametricSampler.obj
 0003:00003178       ?pWaterVolumes@?1??InitRenderingFlags@SRenderingPassInfo@@AEAAXI@Z@4PEAUICVar@@EA 0000000031667178     ParametricSampler.obj
 0003:00003180       ?pWaterWaves@?1??InitRenderingFlags@SRenderingPassInfo@@AEAAXI@Z@4PEAUICVar@@EA 0000000031667180     ParametricSampler.obj
 0003:00003188       ?pDecals@?1??InitRenderingFlags@SRenderingPassInfo@@AEAAXI@Z@4PEAUICVar@@EA 0000000031667188     ParametricSampler.obj
 0003:00003190       ?pParticles@?1??InitRenderingFlags@SRenderingPassInfo@@AEAAXI@Z@4PEAUICVar@@EA 0000000031667190     ParametricSampler.obj
 0003:00003198       ?pWaterOcean@?1??InitRenderingFlags@SRenderingPassInfo@@AEAAXI@Z@4PEAUICVar@@EA 0000000031667198     ParametricSampler.obj
 0003:000031a0       ?pTerrain@?1??InitRenderingFlags@SRenderingPassInfo@@AEAAXI@Z@4PEAUICVar@@EA 00000000316671a0     ParametricSampler.obj
 0003:000031a8       ?pEntities@?1??InitRenderingFlags@SRenderingPassInfo@@AEAAXI@Z@4PEAUICVar@@EA 00000000316671a8     ParametricSampler.obj
 0003:000031b0       ?pVegetation@?1??InitRenderingFlags@SRenderingPassInfo@@AEAAXI@Z@4PEAUICVar@@EA 00000000316671b0     ParametricSampler.obj
 0003:000031b8       ?pBrushes@?1??InitRenderingFlags@SRenderingPassInfo@@AEAAXI@Z@4PEAUICVar@@EA 00000000316671b8     ParametricSampler.obj
 0003:000031c0       ?pShadows@?1??InitRenderingFlags@SRenderingPassInfo@@AEAAXI@Z@4PEAUICVar@@EA 00000000316671c0     ParametricSampler.obj
 0003:000031c8       ?pVoxTer@?1??InitRenderingFlags@SRenderingPassInfo@@AEAAXI@Z@4PEAUICVar@@EA 00000000316671c8     ParametricSampler.obj
 0003:000031d0       ?pVoxel@?1??InitRenderingFlags@SRenderingPassInfo@@AEAAXI@Z@4PEAUICVar@@EA 00000000316671d0     ParametricSampler.obj
 0003:000031d8       ?pDefaultMaterial@?1??InitRenderingFlags@SRenderingPassInfo@@AEAAXI@Z@4PEAUICVar@@EA 00000000316671d8     ParametricSampler.obj
 0003:000031e0       ??_B?1??InitRenderingFlags@SRenderingPassInfo@@AEAAXI@Z@51 00000000316671e0     ParametricSampler.obj
 0003:000031e8       ?pCameraFreeze@?1??CreateGeneralPassRenderingInfo@SRenderingPassInfo@@SA?AU2@AEBVCCamera@@I@Z@4PEAUICVar@@EA 00000000316671e8     ParametricSampler.obj
 0003:000031f0       ??_B?1??CreateGeneralPassRenderingInfo@SRenderingPassInfo@@SA?AU1@AEBVCCamera@@I@Z@51 00000000316671f0     ParametricSampler.obj
 0003:000031f8       ?s_EmptyElems@?1??set_null@?$SmallDynStorage@UVirtualExample1D@@HUStandardAlloc@NAlloc@@@NArray@@IEAAXXZ@4PEAUVirtualExample1D@@EA 00000000316671f8     ParametricSampler.obj
 0003:00003200       ?s_EmptyHeader@?1??set_null@?$SmallDynStorage@UVirtualExample1D@@HUStandardAlloc@NAlloc@@@NArray@@IEAAXXZ@4UEmptyHeader@23@A 0000000031667200     ParametricSampler.obj
 0003:00003208       ??_B?1??set_null@?$SmallDynStorage@UVirtualExample1D@@HUStandardAlloc@NAlloc@@@NArray@@IEAAXXZ@51 0000000031667208     ParametricSampler.obj
 0003:00003210       ?s_EmptyElems@?1??set_null@?$SmallDynStorage@UVirtualExample2D@@HUStandardAlloc@NAlloc@@@NArray@@IEAAXXZ@4PEAUVirtualExample2D@@EA 0000000031667210     ParametricSampler.obj
 0003:00003218       ?s_EmptyHeader@?1??set_null@?$SmallDynStorage@UVirtualExample2D@@HUStandardAlloc@NAlloc@@@NArray@@IEAAXXZ@4UEmptyHeader@23@A 0000000031667218     ParametricSampler.obj
 0003:00003220       ??_B?1??set_null@?$SmallDynStorage@UVirtualExample2D@@HUStandardAlloc@NAlloc@@@NArray@@IEAAXXZ@51 0000000031667220     ParametricSampler.obj
 0003:00003228       ?s_EmptyElems@?1??set_null@?$SmallDynStorage@UVirtualExample3D@@HUStandardAlloc@NAlloc@@@NArray@@IEAAXXZ@4PEAUVirtualExample3D@@EA 0000000031667228     ParametricSampler.obj
 0003:00003230       ?s_EmptyHeader@?1??set_null@?$SmallDynStorage@UVirtualExample3D@@HUStandardAlloc@NAlloc@@@NArray@@IEAAXXZ@4UEmptyHeader@23@A 0000000031667230     ParametricSampler.obj
 0003:00003238       ??_B?1??set_null@?$SmallDynStorage@UVirtualExample3D@@HUStandardAlloc@NAlloc@@@NArray@@IEAAXXZ@51 0000000031667238     ParametricSampler.obj
 0003:00003298       ?s_globalObjectCount@CPlaceholderCharacter@@0HA 0000000031667298     PlaceholderCharacter.obj
 0003:000032a0       ?s_EmptyElems@?1??set_null@?$SmallDynStorage@V?$_smart_ptr@VIController@@@@HUStandardAlloc@NAlloc@@@NArray@@IEAAXXZ@4PEAV?$_smart_ptr@VIController@@@@EA 00000000316672a0     DirectionalBlender.obj
 0003:000032a8       ?s_EmptyHeader@?1??set_null@?$SmallDynStorage@V?$_smart_ptr@VIController@@@@HUStandardAlloc@NAlloc@@@NArray@@IEAAXXZ@4UEmptyHeader@23@A 00000000316672a8     DirectionalBlender.obj
 0003:000032b4       ??_B?1??set_null@?$SmallDynStorage@V?$_smart_ptr@VIController@@@@HUStandardAlloc@NAlloc@@@NArray@@IEAAXXZ@51 00000000316672b4     DirectionalBlender.obj
 0003:000032b8       ?s_EmptyElems@?1??set_null@?$SmallDynStorage@UAimIKPose@@HUStandardAlloc@NAlloc@@@NArray@@IEAAXXZ@4PEAUAimIKPose@@EA 00000000316672b8     DirectionalBlender.obj
 0003:000032c0       ?s_EmptyHeader@?1??set_null@?$SmallDynStorage@UAimIKPose@@HUStandardAlloc@NAlloc@@@NArray@@IEAAXXZ@4UEmptyHeader@23@A 00000000316672c0     DirectionalBlender.obj
 0003:000032cc       ??_B?1??set_null@?$SmallDynStorage@UAimIKPose@@HUStandardAlloc@NAlloc@@@NArray@@IEAAXXZ@51 00000000316672cc     DirectionalBlender.obj
 0003:000032d0       ?s_EmptyElems@?1??set_null@?$SmallDynStorage@UVirtualExampleInit2@CHUNK_GAHAIM_INFO@@HUStandardAlloc@NAlloc@@@NArray@@IEAAXXZ@4PEAUVirtualExampleInit2@CHUNK_GAHAIM_INFO@@EA 00000000316672d0     DirectionalBlender.obj
 0003:000032d8       ?s_EmptyHeader@?1??set_null@?$SmallDynStorage@UVirtualExampleInit2@CHUNK_GAHAIM_INFO@@HUStandardAlloc@NAlloc@@@NArray@@IEAAXXZ@4UEmptyHeader@23@A 00000000316672d8     DirectionalBlender.obj
 0003:000032e0       ??_B?1??set_null@?$SmallDynStorage@UVirtualExampleInit2@CHUNK_GAHAIM_INFO@@HUStandardAlloc@NAlloc@@@NArray@@IEAAXXZ@51 00000000316672e0     DirectionalBlender.obj
 0003:00003318       ?supportedIIDs@?1???0CFactory@COperatorQueue@@AEAA@XZ@4PAUCryGUID@@A 0000000031667318     OperatorQueue.obj
 0003:00003348       ?s_factory@CFactory@COperatorQueue@@0V12@A 0000000031667348     OperatorQueue.obj
 0003:00003380       ?supportedIIDs@?1???0CFactory@CPoseAlignerChain@@AEAA@XZ@4PAUCryGUID@@A 0000000031667380     PoseAlignerChain.obj
 0003:000033b0       ?s_factory@CFactory@CPoseAlignerChain@@0V12@A 00000000316673b0     PoseAlignerChain.obj
 0003:000033d8       ?supportedIIDs@?1???0CFactory@CPoseMatching@@AEAA@XZ@4PAUCryGUID@@A 00000000316673d8     PoseMatching.obj
 0003:00003408       ?s_factory@CFactory@CPoseMatching@@0V12@A 0000000031667408     PoseMatching.obj
 0003:00003430       ?g_lockList@SBatchUpdateValidator@@2HC 0000000031667430     SkeletonPhysics.obj
 0003:00003438       ?s_EmptyElems@?1??set_null@?$SmallDynStorage@U?$QuatT_tpl@M@@HUStandardAlloc@NAlloc@@@NArray@@IEAAXXZ@4PEAU?$QuatT_tpl@M@@EA 0000000031667438     SkeletonPhysics.obj
 0003:00003440       ?s_EmptyHeader@?1??set_null@?$SmallDynStorage@U?$QuatT_tpl@M@@HUStandardAlloc@NAlloc@@@NArray@@IEAAXXZ@4UEmptyHeader@23@A 0000000031667440     SkeletonPhysics.obj
 0003:00003448       ??_B?1??set_null@?$SmallDynStorage@U?$QuatT_tpl@M@@HUStandardAlloc@NAlloc@@@NArray@@IEAAXXZ@51 0000000031667448     SkeletonPhysics.obj
 0003:00003450       ?s_EmptyElems@?1??set_null@?$SmallDynStorage@HHUStandardAlloc@NAlloc@@@NArray@@IEAAXXZ@4PEAHEA 0000000031667450     SkeletonPhysics.obj
 0003:00003458       ?s_EmptyHeader@?1??set_null@?$SmallDynStorage@HHUStandardAlloc@NAlloc@@@NArray@@IEAAXXZ@4UEmptyHeader@23@A 0000000031667458     SkeletonPhysics.obj
 0003:00003460       ??_B?1??set_null@?$SmallDynStorage@HHUStandardAlloc@NAlloc@@@NArray@@IEAAXXZ@51 0000000031667460     SkeletonPhysics.obj
 0003:00003810       ?s_EmptyElems@?1??set_null@?$SmallDynStorage@UCPhysicsJoint@@HUStandardAlloc@NAlloc@@@NArray@@IEAAXXZ@4PEAUCPhysicsJoint@@EA 0000000031667810     SkeletonPhysics.obj
 0003:00003818       ?s_EmptyHeader@?1??set_null@?$SmallDynStorage@UCPhysicsJoint@@HUStandardAlloc@NAlloc@@@NArray@@IEAAXXZ@4UEmptyHeader@23@A 0000000031667818     SkeletonPhysics.obj
 0003:00003820       ??_B?1??set_null@?$SmallDynStorage@UCPhysicsJoint@@HUStandardAlloc@NAlloc@@@NArray@@IEAAXXZ@51 0000000031667820     SkeletonPhysics.obj
 0003:00004a50       ?s_EmptyElems@?1??set_null@?$SmallDynStorage@USEntry@CPoseModifierQueue@@HUStandardAlloc@NAlloc@@@NArray@@IEAAXXZ@4PEAUSEntry@CPoseModifierQueue@@EA 0000000031668a50     TransitionQueue.obj
 0003:00004a58       ?s_EmptyHeader@?1??set_null@?$SmallDynStorage@USEntry@CPoseModifierQueue@@HUStandardAlloc@NAlloc@@@NArray@@IEAAXXZ@4UEmptyHeader@23@A 0000000031668a58     TransitionQueue.obj
 0003:00004a64       ??_B?1??set_null@?$SmallDynStorage@USEntry@CPoseModifierQueue@@HUStandardAlloc@NAlloc@@@NArray@@IEAAXXZ@51 0000000031668a64     TransitionQueue.obj
 0003:00004a68       ?s_EmptyElems@?1??set_null@?$SmallDynStorage@VCAnimation@@HUStandardAlloc@NAlloc@@@NArray@@IEAAXXZ@4PEAVCAnimation@@EA 0000000031668a68     TransitionQueue.obj
 0003:00004a70       ?s_EmptyHeader@?1??set_null@?$SmallDynStorage@VCAnimation@@HUStandardAlloc@NAlloc@@@NArray@@IEAAXXZ@4UEmptyHeader@23@A 0000000031668a70     TransitionQueue.obj
 0003:00004a7c       ??_B?1??set_null@?$SmallDynStorage@VCAnimation@@HUStandardAlloc@NAlloc@@@NArray@@IEAAXXZ@51 0000000031668a7c     TransitionQueue.obj
 0003:00004a80       ?s_EmptyElems@?1??set_null@?$SmallDynStorage@USVertexFrameState@@HUStandardAlloc@NAlloc@@@NArray@@IEAAXXZ@4PEAUSVertexFrameState@@EA 0000000031668a80     VertexAnimation.obj
 0003:00004a88       ?s_EmptyHeader@?1??set_null@?$SmallDynStorage@USVertexFrameState@@HUStandardAlloc@NAlloc@@@NArray@@IEAAXXZ@4UEmptyHeader@23@A 0000000031668a88     VertexAnimation.obj
 0003:00004a94       ??_B?1??set_null@?$SmallDynStorage@USVertexFrameState@@HUStandardAlloc@NAlloc@@@NArray@@IEAAXXZ@51 0000000031668a94     VertexAnimation.obj
 0003:00004a98       ?s_EmptyElems@?1??set_null@?$SmallDynStorage@USVF_P3F@@HUStandardAlloc@NAlloc@@@NArray@@IEAAXXZ@4PEAUSVF_P3F@@EA 0000000031668a98     VertexData.obj
 0003:00004aa0       ?s_EmptyHeader@?1??set_null@?$SmallDynStorage@USVF_P3F@@HUStandardAlloc@NAlloc@@@NArray@@IEAAXXZ@4UEmptyHeader@23@A 0000000031668aa0     VertexData.obj
 0003:00004aa8       ??_B?1??set_null@?$SmallDynStorage@USVF_P3F@@HUStandardAlloc@NAlloc@@@NArray@@IEAAXXZ@51 0000000031668aa8     VertexData.obj
 0003:00005288       ?s_EmptyElems@?1??set_null@?$SmallDynStorage@V?$_smart_ptr@UIAttachment@@@@HUStandardAlloc@NAlloc@@@NArray@@IEAAXXZ@4PEAV?$_smart_ptr@UIAttachment@@@@EA 0000000031669288     AttachmentManager.obj
 0003:00005290       ?s_EmptyHeader@?1??set_null@?$SmallDynStorage@V?$_smart_ptr@UIAttachment@@@@HUStandardAlloc@NAlloc@@@NArray@@IEAAXXZ@4UEmptyHeader@23@A 0000000031669290     AttachmentManager.obj
 0003:0000529c       ??_B?1??set_null@?$SmallDynStorage@V?$_smart_ptr@UIAttachment@@@@HUStandardAlloc@NAlloc@@@NArray@@IEAAXXZ@51 000000003166929c     AttachmentManager.obj
 0003:000052a0       ?s_EmptyElems@?1??set_null@?$SmallDynStorage@UCharacterAttachment@@HUStandardAlloc@NAlloc@@@NArray@@IEAAXXZ@4PEAUCharacterAttachment@@EA 00000000316692a0     AttachmentManager.obj
 0003:000052a8       ?s_EmptyHeader@?1??set_null@?$SmallDynStorage@UCharacterAttachment@@HUStandardAlloc@NAlloc@@@NArray@@IEAAXXZ@4UEmptyHeader@23@A 00000000316692a8     AttachmentManager.obj
 0003:000052b4       ??_B?1??set_null@?$SmallDynStorage@UCharacterAttachment@@HUStandardAlloc@NAlloc@@@NArray@@IEAAXXZ@51 00000000316692b4     AttachmentManager.obj
 0003:00005a00       ?gJobHandleTSkinningTransformationsComputation@Detail@JobManager@@3PEAUSJobStringHandle@2@EA 0000000031669a00     CharacterInstance.obj
 0003:00005a08       ?s_EmptyElems@?1??set_null@?$SmallDynStorage@MHUStandardAlloc@NAlloc@@@NArray@@IEAAXXZ@4PEAMEA 0000000031669a08     CharacterInstance.obj
 0003:00005a10       ?s_EmptyHeader@?1??set_null@?$SmallDynStorage@MHUStandardAlloc@NAlloc@@@NArray@@IEAAXXZ@4UEmptyHeader@23@A 0000000031669a10     CharacterInstance.obj
 0003:00005a18       ??_B?1??set_null@?$SmallDynStorage@MHUStandardAlloc@NAlloc@@@NArray@@IEAAXXZ@51 0000000031669a18     CharacterInstance.obj
 0003:00005a20       ?s_EmptyElems@?1??set_null@?$SmallDynStorage@UGeomQuery@@HUStandardAlloc@NAlloc@@@NArray@@IEAAXXZ@4PEAUGeomQuery@@EA 0000000031669a20     CharacterInstance.obj
 0003:00005a28       ?s_EmptyHeader@?1??set_null@?$SmallDynStorage@UGeomQuery@@HUStandardAlloc@NAlloc@@@NArray@@IEAAXXZ@4UEmptyHeader@23@A 0000000031669a28     CharacterInstance.obj
 0003:00005a34       ??_B?1??set_null@?$SmallDynStorage@UGeomQuery@@HUStandardAlloc@NAlloc@@@NArray@@IEAAXXZ@51 0000000031669a34     CharacterInstance.obj
 0003:00005a38       ?s_EmptyElems@?1??set_null@?$SmallDynStorage@_NHUStandardAlloc@NAlloc@@@NArray@@IEAAXXZ@4PEA_NEA 0000000031669a38     CharacterInstance.obj
 0003:00005a40       ?s_EmptyHeader@?1??set_null@?$SmallDynStorage@_NHUStandardAlloc@NAlloc@@@NArray@@IEAAXXZ@4UEmptyHeader@23@A 0000000031669a40     CharacterInstance.obj
 0003:00005a48       ??_B?1??set_null@?$SmallDynStorage@_NHUStandardAlloc@NAlloc@@@NArray@@IEAAXXZ@51 0000000031669a48     CharacterInstance.obj
 0003:00005a50       ?s_EmptyElems@?1??set_null@?$SmallDynStorage@IHUStandardAlloc@NAlloc@@@NArray@@IEAAXXZ@4PEAIEA 0000000031669a50     CharacterInstance.obj
 0003:00005a58       ?s_EmptyHeader@?1??set_null@?$SmallDynStorage@IHUStandardAlloc@NAlloc@@@NArray@@IEAAXXZ@4UEmptyHeader@23@A 0000000031669a58     CharacterInstance.obj
 0003:00005a60       ??_B?1??set_null@?$SmallDynStorage@IHUStandardAlloc@NAlloc@@@NArray@@IEAAXXZ@51 0000000031669a60     CharacterInstance.obj
 0003:00005a68       ?s_EmptyElems@?1??set_null@?$SmallDynStorage@V?$CryStringT@D@@HUStandardAlloc@NAlloc@@@NArray@@IEAAXXZ@4PEAV?$CryStringT@D@@EA 0000000031669a68     CharacterInstance.obj
 0003:00005a70       ?s_EmptyHeader@?1??set_null@?$SmallDynStorage@V?$CryStringT@D@@HUStandardAlloc@NAlloc@@@NArray@@IEAAXXZ@4UEmptyHeader@23@A 0000000031669a70     CharacterInstance.obj
 0003:00005a7c       ??_B?1??set_null@?$SmallDynStorage@V?$CryStringT@D@@HUStandardAlloc@NAlloc@@@NArray@@IEAAXXZ@51 0000000031669a7c     CharacterInstance.obj
 0003:00006570       ?g_arrVerticesBS@@3V?$vector@U?$Vec3_tpl@M@@V?$allocator@U?$Vec3_tpl@M@@@stlpmtx_std@@@stlpmtx_std@@A 000000003166a570     DecalManager.obj
 0003:00006588       ?g_arrDecalVertexMapping@@3V?$vector@HV?$allocator@H@stlpmtx_std@@@stlpmtx_std@@A 000000003166a588     DecalManager.obj
 0003:000065a0       ?g_arrDecalFaceMapping@@3V?$vector@HV?$allocator@H@stlpmtx_std@@@stlpmtx_std@@A 000000003166a5a0     DecalManager.obj
 0003:000065b8       ?s_EmptyElems@?1??set_null@?$SmallDynStorage@UEffectEntry@CSkeletonEffectManager@@HUStandardAlloc@NAlloc@@@NArray@@IEAAXXZ@4PEAUEffectEntry@CSkeletonEffectManager@@EA 000000003166a5b8     SkeletonEffectManager.obj
 0003:000065c0       ?s_EmptyHeader@?1??set_null@?$SmallDynStorage@UEffectEntry@CSkeletonEffectManager@@HUStandardAlloc@NAlloc@@@NArray@@IEAAXXZ@4UEmptyHeader@23@A 000000003166a5c0     SkeletonEffectManager.obj
 0003:000065cc       ??_B?1??set_null@?$SmallDynStorage@UEffectEntry@CSkeletonEffectManager@@HUStandardAlloc@NAlloc@@@NArray@@IEAAXXZ@51 000000003166a5cc     SkeletonEffectManager.obj
 0003:000065d0       ?s_EmptyElems@?1??set_null@?$SmallDynStorage@UCCGAJoint@@HUStandardAlloc@NAlloc@@@NArray@@IEAAXXZ@4PEAUCCGAJoint@@EA 000000003166a5d0     SkeletonPose.obj
 0003:000065d8       ?s_EmptyHeader@?1??set_null@?$SmallDynStorage@UCCGAJoint@@HUStandardAlloc@NAlloc@@@NArray@@IEAAXXZ@4UEmptyHeader@23@A 000000003166a5d8     SkeletonPose.obj
 0003:000065e4       ??_B?1??set_null@?$SmallDynStorage@UCCGAJoint@@HUStandardAlloc@NAlloc@@@NArray@@IEAAXXZ@51 000000003166a5e4     SkeletonPose.obj
 0003:000065e8       ?s_EmptyElems@?1??set_null@?$SmallDynStorage@USPostProcess@@HUStandardAlloc@NAlloc@@@NArray@@IEAAXXZ@4PEAUSPostProcess@@EA 000000003166a5e8     SkeletonPose.obj
 0003:000065f0       ?s_EmptyHeader@?1??set_null@?$SmallDynStorage@USPostProcess@@HUStandardAlloc@NAlloc@@@NArray@@IEAAXXZ@4UEmptyHeader@23@A 000000003166a5f0     SkeletonPose.obj
 0003:000065f8       ??_B?1??set_null@?$SmallDynStorage@USPostProcess@@HUStandardAlloc@NAlloc@@@NArray@@IEAAXXZ@51 000000003166a5f8     SkeletonPose.obj
 0003:00007130       ?gJobHandleTCommandBufferExecuteJob@Detail@JobManager@@3PEAUSJobStringHandle@2@EA 000000003166b130     SkeletonAnim.obj
 0003:00007138       ?s_pMemoryPool@CSkeletonAnimTask@@0PEAVCPoolFrameLocal@Memory@@EA 000000003166b138     SkeletonAnim.obj
 0003:00007140       ?GUID_AnimationPoseModifier_TransformationPin@@3UCryGUID@@A 000000003166b140     SkeletonAnim.obj
 0003:00007150       ?instance@?1??Instance@CAnimationContext@@SAAEAV2@XZ@4V2@A 000000003166b150     SkeletonAnim.obj
 0003:00007158       ??_B?1??Instance@CAnimationContext@@SAAEAV1@XZ@51 000000003166b158     SkeletonAnim.obj
 0003:00008c00       ?s_EmptyElems@?1??set_null@?$SmallDynStorage@U?$SplineKey@M@spline@@HUStandardAlloc@NAlloc@@@NArray@@IEAAXXZ@4PEAU?$SplineKey@M@spline@@EA 000000003166cc00     FaceAnimSequence.obj
 0003:00008c08       ?s_EmptyHeader@?1??set_null@?$SmallDynStorage@U?$SplineKey@M@spline@@HUStandardAlloc@NAlloc@@@NArray@@IEAAXXZ@4UEmptyHeader@23@A 000000003166cc08     FaceAnimSequence.obj
 0003:00008c10       ??_B?1??set_null@?$SmallDynStorage@U?$SplineKey@M@spline@@HUStandardAlloc@NAlloc@@@NArray@@IEAAXXZ@51 000000003166cc10     FaceAnimSequence.obj
 0003:00008c18       ?s_EmptyElems@?1??set_null@?$SmallDynStorage@U?$SplineKey@U?$Quat_tpl@M@@@spline@@HUStandardAlloc@NAlloc@@@NArray@@IEAAXXZ@4PEAU?$SplineKey@U?$Quat_tpl@M@@@spline@@EA 000000003166cc18     FaceAnimSequence.obj
 0003:00008c20       ?s_EmptyHeader@?1??set_null@?$SmallDynStorage@U?$SplineKey@U?$Quat_tpl@M@@@spline@@HUStandardAlloc@NAlloc@@@NArray@@IEAAXXZ@4UEmptyHeader@23@A 000000003166cc20     FaceAnimSequence.obj
 0003:00008c28       ??_B?1??set_null@?$SmallDynStorage@U?$SplineKey@U?$Quat_tpl@M@@@spline@@HUStandardAlloc@NAlloc@@@NArray@@IEAAXXZ@51 000000003166cc28     FaceAnimSequence.obj
 0003:00008c30       ?s_EmptyElems@?1??set_null@?$SmallDynStorage@U?$TCBSplineKey@U?$Vec3_tpl@M@@@spline@@HUStandardAlloc@NAlloc@@@NArray@@IEAAXXZ@4PEAU?$TCBSplineKey@U?$Vec3_tpl@M@@@spline@@EA 000000003166cc30     FaceAnimSequence.obj
 0003:00008c38       ?s_EmptyHeader@?1??set_null@?$SmallDynStorage@U?$TCBSplineKey@U?$Vec3_tpl@M@@@spline@@HUStandardAlloc@NAlloc@@@NArray@@IEAAXXZ@4UEmptyHeader@23@A 000000003166cc38     FaceAnimSequence.obj
 0003:00008c40       ??_B?1??set_null@?$SmallDynStorage@U?$TCBSplineKey@U?$Vec3_tpl@M@@@spline@@HUStandardAlloc@NAlloc@@@NArray@@IEAAXXZ@51 000000003166cc40     FaceAnimSequence.obj
 0003:00008ff8       ?s_EmptyElems@?1??set_null@?$SmallDynStorage@VCFacialAnimForcedRotationEntry@@HUStandardAlloc@NAlloc@@@NArray@@IEAAXXZ@4PEAVCFacialAnimForcedRotationEntry@@EA 000000003166cff8     FacialInstance.obj
 0003:00009000       ?s_EmptyHeader@?1??set_null@?$SmallDynStorage@VCFacialAnimForcedRotationEntry@@HUStandardAlloc@NAlloc@@@NArray@@IEAAXXZ@4UEmptyHeader@23@A 000000003166d000     FacialInstance.obj
 0003:00009008       ??_B?1??set_null@?$SmallDynStorage@VCFacialAnimForcedRotationEntry@@HUStandardAlloc@NAlloc@@@NArray@@IEAAXXZ@51 000000003166d008     FacialInstance.obj
 0003:000093c0       ?supportedIIDs@?1???0CFactory@CFeetPoseStore@@AEAA@XZ@4PAUCryGUID@@A 000000003166d3c0     FeetLock.obj
 0003:000093e0       ?supportedIIDs@?1???0CFactory@CFeetPoseRestore@@AEAA@XZ@4PAUCryGUID@@A 000000003166d3e0     FeetLock.obj
 0003:00009400       ?supportedIIDs@?1???0CFactory@CGroundAlignment@@AEAA@XZ@4PAUCryGUID@@A 000000003166d400     GroundAlignment.obj
 0003:00009430       ?s_factory@CFactory@CGroundAlignment@@0V12@A 000000003166d430     GroundAlignment.obj
 0003:00009458       ?supportedIIDs@?1???0CFactory@CLimbIk@@AEAA@XZ@4PAUCryGUID@@A 000000003166d458     LimbIk.obj
 0003:00009488       ?supportedIIDs@?1???0CFactory@CPoseBlenderAim@@AEAA@XZ@4PAUCryGUID@@A 000000003166d488     PoseBlenderAim.obj
 0003:000094b8       ?s_factory@CFactory@CPoseBlenderAim@@0V12@A 000000003166d4b8     PoseBlenderAim.obj
 0003:000094f0       ?supportedIIDs@?1???0CFactory@CPoseBlenderLook@@AEAA@XZ@4PAUCryGUID@@A 000000003166d4f0     PoseBlenderLook.obj
 0003:00009520       ?s_factory@CFactory@CPoseBlenderLook@@0V12@A 000000003166d520     PoseBlenderLook.obj
 0003:00009548       ?supportedIIDs@?1???0CFactory@CRecoil@PoseModifier@@AEAA@XZ@4PAUCryGUID@@A 000000003166d548     Recoil.obj
 0003:0000a05c       ?g_result@Skeleton@@3IA    000000003166e05c     Skeleton.obj
 0003:0000a068       ?g_YLine@@3MA              000000003166e068     CharacterManager.obj
 0003:0000a06c       ?s_bPaused@CharacterManager@@2_NA 000000003166e06c     CharacterManager.obj
 0003:0000a070       ?s_renderFrameIdLocal@CharacterManager@@2IA 000000003166e070     CharacterManager.obj
 0003:0000a0a0       ?s_EmptyElems@?1??set_null@?$SmallDynStorage@UDebugInstances@@HUStandardAlloc@NAlloc@@@NArray@@IEAAXXZ@4PEAUDebugInstances@@EA 000000003166e0a0     CharacterManager.obj
 0003:0000a0a8       ?s_EmptyHeader@?1??set_null@?$SmallDynStorage@UDebugInstances@@HUStandardAlloc@NAlloc@@@NArray@@IEAAXXZ@4UEmptyHeader@23@A 000000003166e0a8     CharacterManager.obj
 0003:0000a0b4       ??_B?1??set_null@?$SmallDynStorage@UDebugInstances@@HUStandardAlloc@NAlloc@@@NArray@@IEAAXXZ@51 000000003166e0b4     CharacterManager.obj
 0003:0000a0b8       ?s_EmptyElems@?1??set_null@?$SmallDynStorage@V?$TCBSpline@U?$Vec3_tpl@M@@U?$TCBSplineKey@U?$Vec3_tpl@M@@@spline@@@spline@@HUStandardAlloc@NAlloc@@@NArray@@IEAAXXZ@4PEAV?$TCBSpline@U?$Vec3_tpl@M@@U?$TCBSplineKey@U?$Vec3_tpl@M@@@spline@@@spline@@EA 000000003166e0b8     CharacterManager.obj
 0003:0000a0c0       ?s_EmptyHeader@?1??set_null@?$SmallDynStorage@V?$TCBSpline@U?$Vec3_tpl@M@@U?$TCBSplineKey@U?$Vec3_tpl@M@@@spline@@@spline@@HUStandardAlloc@NAlloc@@@NArray@@IEAAXXZ@4UEmptyHeader@23@A 000000003166e0c0     CharacterManager.obj
 0003:0000a0cc       ??_B?1??set_null@?$SmallDynStorage@V?$TCBSpline@U?$Vec3_tpl@M@@U?$TCBSplineKey@U?$Vec3_tpl@M@@@spline@@@spline@@HUStandardAlloc@NAlloc@@@NArray@@IEAAXXZ@51 000000003166e0cc     CharacterManager.obj
 0003:0000a0d0       ?s_EmptyElems@?1??set_null@?$SmallDynStorage@VTCBAngleAxisSpline@spline@@HUStandardAlloc@NAlloc@@@NArray@@IEAAXXZ@4PEAVTCBAngleAxisSpline@spline@@EA 000000003166e0d0     CharacterManager.obj
 0003:0000a0d8       ?s_EmptyHeader@?1??set_null@?$SmallDynStorage@VTCBAngleAxisSpline@spline@@HUStandardAlloc@NAlloc@@@NArray@@IEAAXXZ@4UEmptyHeader@23@A 000000003166e0d8     CharacterManager.obj
 0003:0000a0e4       ??_B?1??set_null@?$SmallDynStorage@VTCBAngleAxisSpline@spline@@HUStandardAlloc@NAlloc@@@NArray@@IEAAXXZ@51 000000003166e0e4     CharacterManager.obj
 0003:0000a0e8       ?s_EmptyElems@?1??set_null@?$SmallDynStorage@UCControllerType@@HUStandardAlloc@NAlloc@@@NArray@@IEAAXXZ@4PEAUCControllerType@@EA 000000003166e0e8     CharacterManager.obj
 0003:0000a0f0       ?s_EmptyHeader@?1??set_null@?$SmallDynStorage@UCControllerType@@HUStandardAlloc@NAlloc@@@NArray@@IEAAXXZ@4UEmptyHeader@23@A 000000003166e0f0     CharacterManager.obj
 0003:0000a0f8       ??_B?1??set_null@?$SmallDynStorage@UCControllerType@@HUStandardAlloc@NAlloc@@@NArray@@IEAAXXZ@51 000000003166e0f8     CharacterManager.obj
 0003:0000a100       ?s_EmptyElems@?1??set_null@?$SmallDynStorage@UNodeDesc@@HUStandardAlloc@NAlloc@@@NArray@@IEAAXXZ@4PEAUNodeDesc@@EA 000000003166e100     CharacterManager.obj
 0003:0000a108       ?s_EmptyHeader@?1??set_null@?$SmallDynStorage@UNodeDesc@@HUStandardAlloc@NAlloc@@@NArray@@IEAAXXZ@4UEmptyHeader@23@A 000000003166e108     CharacterManager.obj
 0003:0000a110       ??_B?1??set_null@?$SmallDynStorage@UNodeDesc@@HUStandardAlloc@NAlloc@@@NArray@@IEAAXXZ@51 000000003166e110     CharacterManager.obj
 0003:0000a118       ?s_EmptyElems@?1??set_null@?$SmallDynStorage@UCControllerTCB@@HUStandardAlloc@NAlloc@@@NArray@@IEAAXXZ@4PEAUCControllerTCB@@EA 000000003166e118     CharacterManager.obj
 0003:0000a120       ?s_EmptyHeader@?1??set_null@?$SmallDynStorage@UCControllerTCB@@HUStandardAlloc@NAlloc@@@NArray@@IEAAXXZ@4UEmptyHeader@23@A 000000003166e120     CharacterManager.obj
 0003:0000a12c       ??_B?1??set_null@?$SmallDynStorage@UCControllerTCB@@HUStandardAlloc@NAlloc@@@NArray@@IEAAXXZ@51 000000003166e12c     CharacterManager.obj
 0003:0000a130       ?s_EmptyElems@?1??set_null@?$SmallDynStorage@UCGlobalHeaderDBA@@HUStandardAlloc@NAlloc@@@NArray@@IEAAXXZ@4PEAUCGlobalHeaderDBA@@EA 000000003166e130     CharacterManager.obj
 0003:0000a138       ?s_EmptyHeader@?1??set_null@?$SmallDynStorage@UCGlobalHeaderDBA@@HUStandardAlloc@NAlloc@@@NArray@@IEAAXXZ@4UEmptyHeader@23@A 000000003166e138     CharacterManager.obj
 0003:0000a144       ??_B?1??set_null@?$SmallDynStorage@UCGlobalHeaderDBA@@HUStandardAlloc@NAlloc@@@NArray@@IEAAXXZ@51 000000003166e144     CharacterManager.obj
 0003:0000a148       ?s_EmptyElems@?1??set_null@?$SmallDynStorage@UGlobalAnimationHeaderCAF@@HUStandardAlloc@NAlloc@@@NArray@@IEAAXXZ@4PEAUGlobalAnimationHeaderCAF@@EA 000000003166e148     CharacterManager.obj
 0003:0000a150       ?s_EmptyHeader@?1??set_null@?$SmallDynStorage@UGlobalAnimationHeaderCAF@@HUStandardAlloc@NAlloc@@@NArray@@IEAAXXZ@4UEmptyHeader@23@A 000000003166e150     CharacterManager.obj
 0003:0000a15c       ??_B?1??set_null@?$SmallDynStorage@UGlobalAnimationHeaderCAF@@HUStandardAlloc@NAlloc@@@NArray@@IEAAXXZ@51 000000003166e15c     CharacterManager.obj
 0003:0000a160       ?s_EmptyElems@?1??set_null@?$SmallDynStorage@UGlobalAnimationHeaderAIM@@HUStandardAlloc@NAlloc@@@NArray@@IEAAXXZ@4PEAUGlobalAnimationHeaderAIM@@EA 000000003166e160     CharacterManager.obj
 0003:0000a168       ?s_EmptyHeader@?1??set_null@?$SmallDynStorage@UGlobalAnimationHeaderAIM@@HUStandardAlloc@NAlloc@@@NArray@@IEAAXXZ@4UEmptyHeader@23@A 000000003166e168     CharacterManager.obj
 0003:0000a174       ??_B?1??set_null@?$SmallDynStorage@UGlobalAnimationHeaderAIM@@HUStandardAlloc@NAlloc@@@NArray@@IEAAXXZ@51 000000003166e174     CharacterManager.obj
 0003:0000a178       ?s_EmptyElems@?1??set_null@?$SmallDynStorage@UGlobalAnimationHeaderLMG@@HUStandardAlloc@NAlloc@@@NArray@@IEAAXXZ@4PEAUGlobalAnimationHeaderLMG@@EA 000000003166e178     CharacterManager.obj
 0003:0000a180       ?s_EmptyHeader@?1??set_null@?$SmallDynStorage@UGlobalAnimationHeaderLMG@@HUStandardAlloc@NAlloc@@@NArray@@IEAAXXZ@4UEmptyHeader@23@A 000000003166e180     CharacterManager.obj
 0003:0000a18c       ??_B?1??set_null@?$SmallDynStorage@UGlobalAnimationHeaderLMG@@HUStandardAlloc@NAlloc@@@NArray@@IEAAXXZ@51 000000003166e18c     CharacterManager.obj
 0003:0000a190       ?s_EmptyElems@?1??set_null@?$SmallDynStorage@UBSParameter@@HUStandardAlloc@NAlloc@@@NArray@@IEAAXXZ@4PEAUBSParameter@@EA 000000003166e190     CharacterManager.obj
 0003:0000a198       ?s_EmptyHeader@?1??set_null@?$SmallDynStorage@UBSParameter@@HUStandardAlloc@NAlloc@@@NArray@@IEAAXXZ@4UEmptyHeader@23@A 000000003166e198     CharacterManager.obj
 0003:0000a1a4       ??_B?1??set_null@?$SmallDynStorage@UBSParameter@@HUStandardAlloc@NAlloc@@@NArray@@IEAAXXZ@51 000000003166e1a4     CharacterManager.obj
 0003:0000a1a8       ?s_EmptyElems@?1??set_null@?$SmallDynStorage@UBSBlendable@@HUStandardAlloc@NAlloc@@@NArray@@IEAAXXZ@4PEAUBSBlendable@@EA 000000003166e1a8     CharacterManager.obj
 0003:0000a1b0       ?s_EmptyHeader@?1??set_null@?$SmallDynStorage@UBSBlendable@@HUStandardAlloc@NAlloc@@@NArray@@IEAAXXZ@4UEmptyHeader@23@A 000000003166e1b0     CharacterManager.obj
 0003:0000a1b8       ??_B?1??set_null@?$SmallDynStorage@UBSBlendable@@HUStandardAlloc@NAlloc@@@NArray@@IEAAXXZ@51 000000003166e1b8     CharacterManager.obj
 0003:0000a1c0       ?s_EmptyElems@?1??set_null@?$SmallDynStorage@UBlendSpaceInfo@@HUStandardAlloc@NAlloc@@@NArray@@IEAAXXZ@4PEAUBlendSpaceInfo@@EA 000000003166e1c0     CharacterManager.obj
 0003:0000a1c8       ?s_EmptyHeader@?1??set_null@?$SmallDynStorage@UBlendSpaceInfo@@HUStandardAlloc@NAlloc@@@NArray@@IEAAXXZ@4UEmptyHeader@23@A 000000003166e1c8     CharacterManager.obj
 0003:0000a1d4       ??_B?1??set_null@?$SmallDynStorage@UBlendSpaceInfo@@HUStandardAlloc@NAlloc@@@NArray@@IEAAXXZ@51 000000003166e1d4     CharacterManager.obj
 0003:0000a1d8       ?s_EmptyElems@?1??set_null@?$SmallDynStorage@USCRCName@@HUStandardAlloc@NAlloc@@@NArray@@IEAAXXZ@4PEAUSCRCName@@EA 000000003166e1d8     CharacterManager.obj
 0003:0000a1e0       ?s_EmptyHeader@?1??set_null@?$SmallDynStorage@USCRCName@@HUStandardAlloc@NAlloc@@@NArray@@IEAAXXZ@4UEmptyHeader@23@A 000000003166e1e0     CharacterManager.obj
 0003:0000a1ec       ??_B?1??set_null@?$SmallDynStorage@USCRCName@@HUStandardAlloc@NAlloc@@@NArray@@IEAAXXZ@51 000000003166e1ec     CharacterManager.obj
 0003:0000a1f0       ?s_EmptyElems@?1??set_null@?$SmallDynStorage@PEAVCAnimationSet@@HUStandardAlloc@NAlloc@@@NArray@@IEAAXXZ@4PEAPEAVCAnimationSet@@EA 000000003166e1f0     CharacterManager.obj
 0003:0000a1f8       ?s_EmptyHeader@?1??set_null@?$SmallDynStorage@PEAVCAnimationSet@@HUStandardAlloc@NAlloc@@@NArray@@IEAAXXZ@4UEmptyHeader@23@A 000000003166e1f8     CharacterManager.obj
 0003:0000a204       ??_B?1??set_null@?$SmallDynStorage@PEAVCAnimationSet@@HUStandardAlloc@NAlloc@@@NArray@@IEAAXXZ@51 000000003166e204     CharacterManager.obj
 0003:0000a5c8       ?s_EmptyElems@?1??set_null@?$SmallDynStorage@USMeshSubset@@HUStandardAlloc@NAlloc@@@NArray@@IEAAXXZ@4PEAUSMeshSubset@@EA 000000003166e5c8     LoaderCGA.obj
 0003:0000a5d0       ?s_EmptyHeader@?1??set_null@?$SmallDynStorage@USMeshSubset@@HUStandardAlloc@NAlloc@@@NArray@@IEAAXXZ@4UEmptyHeader@23@A 000000003166e5d0     LoaderCGA.obj
 0003:0000a5dc       ??_B?1??set_null@?$SmallDynStorage@USMeshSubset@@HUStandardAlloc@NAlloc@@@NArray@@IEAAXXZ@51 000000003166e5dc     LoaderCGA.obj
 0003:0000a5e0       ?s_EmptyElems@?1??set_null@?$SmallDynStorage@VCModelJoint@@HUStandardAlloc@NAlloc@@@NArray@@IEAAXXZ@4PEAVCModelJoint@@EA 000000003166e5e0     LoaderCGA.obj
 0003:0000a5e8       ?s_EmptyHeader@?1??set_null@?$SmallDynStorage@VCModelJoint@@HUStandardAlloc@NAlloc@@@NArray@@IEAAXXZ@4UEmptyHeader@23@A 000000003166e5e8     LoaderCGA.obj
 0003:0000a5f4       ??_B?1??set_null@?$SmallDynStorage@VCModelJoint@@HUStandardAlloc@NAlloc@@@NArray@@IEAAXXZ@51 000000003166e5f4     LoaderCGA.obj
 0003:0000a5f8       ?s_EmptyElems@?1??set_null@?$SmallDynStorage@UTCBAngAxisKey@spline@@HUStandardAlloc@NAlloc@@@NArray@@IEAAXXZ@4PEAUTCBAngAxisKey@spline@@EA 000000003166e5f8     LoaderCGA.obj
 0003:0000a600       ?s_EmptyHeader@?1??set_null@?$SmallDynStorage@UTCBAngAxisKey@spline@@HUStandardAlloc@NAlloc@@@NArray@@IEAAXXZ@4UEmptyHeader@23@A 000000003166e600     LoaderCGA.obj
 0003:0000a608       ??_B?1??set_null@?$SmallDynStorage@UTCBAngAxisKey@spline@@HUStandardAlloc@NAlloc@@@NArray@@IEAAXXZ@51 000000003166e608     LoaderCGA.obj
 0003:0000a610       ?s_used_memory@?1??_usedMemory@?$CryStackStringT@D$0BAA@@@SA_K_K@Z@4_KA 000000003166e610     LoaderCHR.obj
 0003:0000a618       ?s_EmptyElems@?1??set_null@?$SmallDynStorage@UModelAnimationHeader@@HUStandardAlloc@NAlloc@@@NArray@@IEAAXXZ@4PEAUModelAnimationHeader@@EA 000000003166e618     LoaderCHR.obj
 0003:0000a620       ?s_EmptyHeader@?1??set_null@?$SmallDynStorage@UModelAnimationHeader@@HUStandardAlloc@NAlloc@@@NArray@@IEAAXXZ@4UEmptyHeader@23@A 000000003166e620     LoaderCHR.obj
 0003:0000a62c       ??_B?1??set_null@?$SmallDynStorage@UModelAnimationHeader@@HUStandardAlloc@NAlloc@@@NArray@@IEAAXXZ@51 000000003166e62c     LoaderCHR.obj
 0003:0000a630       ?s_EmptyElems@?1??set_null@?$SmallDynStorage@USAnimFile@@HUStandardAlloc@NAlloc@@@NArray@@IEAAXXZ@4PEAUSAnimFile@@EA 000000003166e630     LoaderCHR.obj
 0003:0000a638       ?s_EmptyHeader@?1??set_null@?$SmallDynStorage@USAnimFile@@HUStandardAlloc@NAlloc@@@NArray@@IEAAXXZ@4UEmptyHeader@23@A 000000003166e638     LoaderCHR.obj
 0003:0000a640       ??_B?1??set_null@?$SmallDynStorage@USAnimFile@@HUStandardAlloc@NAlloc@@@NArray@@IEAAXXZ@51 000000003166e640     LoaderCHR.obj
 0003:0000a648       ?s_EmptyElems@?1??set_null@?$SmallDynStorage@DHUStandardAlloc@NAlloc@@@NArray@@IEAAXXZ@4PEADEA 000000003166e648     LoaderCHR.obj
 0003:0000a650       ?s_EmptyHeader@?1??set_null@?$SmallDynStorage@DHUStandardAlloc@NAlloc@@@NArray@@IEAAXXZ@4UEmptyHeader@23@A 000000003166e650     LoaderCHR.obj
 0003:0000a658       ??_B?1??set_null@?$SmallDynStorage@DHUStandardAlloc@NAlloc@@@NArray@@IEAAXXZ@51 000000003166e658     LoaderCHR.obj
 0003:0000a660       ?s_EmptyElems@?1??set_null@?$SmallDynStorage@GHUStandardAlloc@NAlloc@@@NArray@@IEAAXXZ@4PEAGEA 000000003166e660     LoaderCHR.obj
 0003:0000a668       ?s_EmptyHeader@?1??set_null@?$SmallDynStorage@GHUStandardAlloc@NAlloc@@@NArray@@IEAAXXZ@4UEmptyHeader@23@A 000000003166e668     LoaderCHR.obj
 0003:0000a670       ??_B?1??set_null@?$SmallDynStorage@GHUStandardAlloc@NAlloc@@@NArray@@IEAAXXZ@51 000000003166e670     LoaderCHR.obj
 0003:0000adc0       ?s_EmptyElems@?1??set_null@?$SmallDynStorage@PEAU?$DynArray@UCryTCB3Key@@HU?$SmallDynStorage@UCryTCB3Key@@HUStandardAlloc@NAlloc@@@NArray@@@@HUStandardAlloc@NAlloc@@@NArray@@IEAAXXZ@4PEAPEAU?$DynArray@UCryTCB3Key@@HU?$SmallDynStorage@UCryTCB3Key@@HUStandardAlloc@NAlloc@@@NArray@@@@EA 000000003166edc0     LoaderTCB.obj
 0003:0000adc8       ?s_EmptyHeader@?1??set_null@?$SmallDynStorage@PEAU?$DynArray@UCryTCB3Key@@HU?$SmallDynStorage@UCryTCB3Key@@HUStandardAlloc@NAlloc@@@NArray@@@@HUStandardAlloc@NAlloc@@@NArray@@IEAAXXZ@4UEmptyHeader@23@A 000000003166edc8     LoaderTCB.obj
 0003:0000add4       ??_B?1??set_null@?$SmallDynStorage@PEAU?$DynArray@UCryTCB3Key@@HU?$SmallDynStorage@UCryTCB3Key@@HUStandardAlloc@NAlloc@@@NArray@@@@HUStandardAlloc@NAlloc@@@NArray@@IEAAXXZ@51 000000003166edd4     LoaderTCB.obj
 0003:0000add8       ?s_EmptyElems@?1??set_null@?$SmallDynStorage@PEAU?$DynArray@UCryTCBQKey@@HU?$SmallDynStorage@UCryTCBQKey@@HUStandardAlloc@NAlloc@@@NArray@@@@HUStandardAlloc@NAlloc@@@NArray@@IEAAXXZ@4PEAPEAU?$DynArray@UCryTCBQKey@@HU?$SmallDynStorage@UCryTCBQKey@@HUStandardAlloc@NAlloc@@@NArray@@@@EA 000000003166edd8     LoaderTCB.obj
 0003:0000ade0       ?s_EmptyHeader@?1??set_null@?$SmallDynStorage@PEAU?$DynArray@UCryTCBQKey@@HU?$SmallDynStorage@UCryTCBQKey@@HUStandardAlloc@NAlloc@@@NArray@@@@HUStandardAlloc@NAlloc@@@NArray@@IEAAXXZ@4UEmptyHeader@23@A 000000003166ede0     LoaderTCB.obj
 0003:0000adec       ??_B?1??set_null@?$SmallDynStorage@PEAU?$DynArray@UCryTCBQKey@@HU?$SmallDynStorage@UCryTCBQKey@@HUStandardAlloc@NAlloc@@@NArray@@@@HUStandardAlloc@NAlloc@@@NArray@@IEAAXXZ@51 000000003166edec     LoaderTCB.obj
 0003:0000adf0       ?s_EmptyElems@?1??set_null@?$SmallDynStorage@UTCBFlags@@HUStandardAlloc@NAlloc@@@NArray@@IEAAXXZ@4PEAUTCBFlags@@EA 000000003166edf0     LoaderTCB.obj
 0003:0000adf8       ?s_EmptyHeader@?1??set_null@?$SmallDynStorage@UTCBFlags@@HUStandardAlloc@NAlloc@@@NArray@@IEAAXXZ@4UEmptyHeader@23@A 000000003166edf8     LoaderTCB.obj
 0003:0000ae00       ??_B?1??set_null@?$SmallDynStorage@UTCBFlags@@HUStandardAlloc@NAlloc@@@NArray@@IEAAXXZ@51 000000003166ee00     LoaderTCB.obj
 0003:0000ae08       ?s_EmptyElems@?1??set_null@?$SmallDynStorage@UCryTCB3Key@@HUStandardAlloc@NAlloc@@@NArray@@IEAAXXZ@4PEAUCryTCB3Key@@EA 000000003166ee08     LoaderTCB.obj
 0003:0000ae10       ?s_EmptyHeader@?1??set_null@?$SmallDynStorage@UCryTCB3Key@@HUStandardAlloc@NAlloc@@@NArray@@IEAAXXZ@4UEmptyHeader@23@A 000000003166ee10     LoaderTCB.obj
 0003:0000ae18       ??_B?1??set_null@?$SmallDynStorage@UCryTCB3Key@@HUStandardAlloc@NAlloc@@@NArray@@IEAAXXZ@51 000000003166ee18     LoaderTCB.obj
 0003:0000ae20       ?s_EmptyElems@?1??set_null@?$SmallDynStorage@UCryTCBQKey@@HUStandardAlloc@NAlloc@@@NArray@@IEAAXXZ@4PEAUCryTCBQKey@@EA 000000003166ee20     LoaderTCB.obj
 0003:0000ae28       ?s_EmptyHeader@?1??set_null@?$SmallDynStorage@UCryTCBQKey@@HUStandardAlloc@NAlloc@@@NArray@@IEAAXXZ@4UEmptyHeader@23@A 000000003166ee28     LoaderTCB.obj
 0003:0000ae30       ??_B?1??set_null@?$SmallDynStorage@UCryTCBQKey@@HUStandardAlloc@NAlloc@@@NArray@@IEAAXXZ@51 000000003166ee30     LoaderTCB.obj
 0003:0000ae38       ?s_EmptyElems@?1??set_null@?$SmallDynStorage@UPQLog@@HUStandardAlloc@NAlloc@@@NArray@@IEAAXXZ@4PEAUPQLog@@EA 000000003166ee38     LoaderTCB.obj
 0003:0000ae40       ?s_EmptyHeader@?1??set_null@?$SmallDynStorage@UPQLog@@HUStandardAlloc@NAlloc@@@NArray@@IEAAXXZ@4UEmptyHeader@23@A 000000003166ee40     LoaderTCB.obj
 0003:0000ae48       ??_B?1??set_null@?$SmallDynStorage@UPQLog@@HUStandardAlloc@NAlloc@@@NArray@@IEAAXXZ@51 000000003166ee48     LoaderTCB.obj
 0003:0000ae50       ?s_EmptyElems@?1??set_null@?$SmallDynStorage@USAnimListInfo@@HUStandardAlloc@NAlloc@@@NArray@@IEAAXXZ@4PEAUSAnimListInfo@@EA 000000003166ee50     ParamLoader.obj
 0003:0000ae58       ?s_EmptyHeader@?1??set_null@?$SmallDynStorage@USAnimListInfo@@HUStandardAlloc@NAlloc@@@NArray@@IEAAXXZ@4UEmptyHeader@23@A 000000003166ee58     ParamLoader.obj
 0003:0000ae64       ??_B?1??set_null@?$SmallDynStorage@USAnimListInfo@@HUStandardAlloc@NAlloc@@@NArray@@IEAAXXZ@51 000000003166ee64     ParamLoader.obj
 0003:0000ae68       ?s_EmptyElems@?1??set_null@?$SmallDynStorage@U?$DynArray@IHU?$SmallDynStorage@IHUStandardAlloc@NAlloc@@@NArray@@@@HUStandardAlloc@NAlloc@@@NArray@@IEAAXXZ@4PEAU?$DynArray@IHU?$SmallDynStorage@IHUStandardAlloc@NAlloc@@@NArray@@@@EA 000000003166ee68     ParamLoader.obj
 0003:0000ae70       ?s_EmptyHeader@?1??set_null@?$SmallDynStorage@U?$DynArray@IHU?$SmallDynStorage@IHUStandardAlloc@NAlloc@@@NArray@@@@HUStandardAlloc@NAlloc@@@NArray@@IEAAXXZ@4UEmptyHeader@23@A 000000003166ee70     ParamLoader.obj
 0003:0000ae7c       ??_B?1??set_null@?$SmallDynStorage@U?$DynArray@IHU?$SmallDynStorage@IHUStandardAlloc@NAlloc@@@NArray@@@@HUStandardAlloc@NAlloc@@@NArray@@IEAAXXZ@51 000000003166ee7c     ParamLoader.obj
 0003:0000ae80       ?s_EmptyElems@?1??set_null@?$SmallDynStorage@FHUStandardAlloc@NAlloc@@@NArray@@IEAAXXZ@4PEAFEA 000000003166ee80     ParamLoader.obj
 0003:0000ae88       ?s_EmptyHeader@?1??set_null@?$SmallDynStorage@FHUStandardAlloc@NAlloc@@@NArray@@IEAAXXZ@4UEmptyHeader@23@A 000000003166ee88     ParamLoader.obj
 0003:0000ae90       ??_B?1??set_null@?$SmallDynStorage@FHUStandardAlloc@NAlloc@@@NArray@@IEAAXXZ@51 000000003166ee90     ParamLoader.obj
 0003:0000ae98       ?s_EmptyElems@?1??set_null@?$SmallDynStorage@USJointsAimIK_Rot@@HUStandardAlloc@NAlloc@@@NArray@@IEAAXXZ@4PEAUSJointsAimIK_Rot@@EA 000000003166ee98     ParamLoader.obj
 0003:0000aea0       ?s_EmptyHeader@?1??set_null@?$SmallDynStorage@USJointsAimIK_Rot@@HUStandardAlloc@NAlloc@@@NArray@@IEAAXXZ@4UEmptyHeader@23@A 000000003166eea0     ParamLoader.obj
 0003:0000aeac       ??_B?1??set_null@?$SmallDynStorage@USJointsAimIK_Rot@@HUStandardAlloc@NAlloc@@@NArray@@IEAAXXZ@51 000000003166eeac     ParamLoader.obj
 0003:0000aeb0       ?s_EmptyElems@?1??set_null@?$SmallDynStorage@USJointsAimIK_Pos@@HUStandardAlloc@NAlloc@@@NArray@@IEAAXXZ@4PEAUSJointsAimIK_Pos@@EA 000000003166eeb0     ParamLoader.obj
 0003:0000aeb8       ?s_EmptyHeader@?1??set_null@?$SmallDynStorage@USJointsAimIK_Pos@@HUStandardAlloc@NAlloc@@@NArray@@IEAAXXZ@4UEmptyHeader@23@A 000000003166eeb8     ParamLoader.obj
 0003:0000aec4       ??_B?1??set_null@?$SmallDynStorage@USJointsAimIK_Pos@@HUStandardAlloc@NAlloc@@@NArray@@IEAAXXZ@51 000000003166eec4     ParamLoader.obj
 0003:0000aec8       ?s_EmptyElems@?1??set_null@?$SmallDynStorage@UDirectionalBlends@@HUStandardAlloc@NAlloc@@@NArray@@IEAAXXZ@4PEAUDirectionalBlends@@EA 000000003166eec8     ParamLoader.obj
 0003:0000aed0       ?s_EmptyHeader@?1??set_null@?$SmallDynStorage@UDirectionalBlends@@HUStandardAlloc@NAlloc@@@NArray@@IEAAXXZ@4UEmptyHeader@23@A 000000003166eed0     ParamLoader.obj
 0003:0000aedc       ??_B?1??set_null@?$SmallDynStorage@UDirectionalBlends@@HUStandardAlloc@NAlloc@@@NArray@@IEAAXXZ@51 000000003166eedc     ParamLoader.obj
 0003:0000aee0       ?s_EmptyElems@?1??set_null@?$SmallDynStorage@UIdxAndName@@HUStandardAlloc@NAlloc@@@NArray@@IEAAXXZ@4PEAUIdxAndName@@EA 000000003166eee0     ParamLoader.obj
 0003:0000aee8       ?s_EmptyHeader@?1??set_null@?$SmallDynStorage@UIdxAndName@@HUStandardAlloc@NAlloc@@@NArray@@IEAAXXZ@4UEmptyHeader@23@A 000000003166eee8     ParamLoader.obj
 0003:0000aef4       ??_B?1??set_null@?$SmallDynStorage@UIdxAndName@@HUStandardAlloc@NAlloc@@@NArray@@IEAAXXZ@51 000000003166eef4     ParamLoader.obj
 0003:0000aef8       ?s_EmptyElems@?1??set_null@?$SmallDynStorage@USRecoilJoints@@HUStandardAlloc@NAlloc@@@NArray@@IEAAXXZ@4PEAUSRecoilJoints@@EA 000000003166eef8     ParamLoader.obj
 0003:0000af00       ?s_EmptyHeader@?1??set_null@?$SmallDynStorage@USRecoilJoints@@HUStandardAlloc@NAlloc@@@NArray@@IEAAXXZ@4UEmptyHeader@23@A 000000003166ef00     ParamLoader.obj
 0003:0000af0c       ??_B?1??set_null@?$SmallDynStorage@USRecoilJoints@@HUStandardAlloc@NAlloc@@@NArray@@IEAAXXZ@51 000000003166ef0c     ParamLoader.obj
 0003:0000af10       ?s_EmptyElems@?1??set_null@?$SmallDynStorage@UProcAdjust@@HUStandardAlloc@NAlloc@@@NArray@@IEAAXXZ@4PEAUProcAdjust@@EA 000000003166ef10     ParamLoader.obj
 0003:0000af18       ?s_EmptyHeader@?1??set_null@?$SmallDynStorage@UProcAdjust@@HUStandardAlloc@NAlloc@@@NArray@@IEAAXXZ@4UEmptyHeader@23@A 000000003166ef18     ParamLoader.obj
 0003:0000af24       ??_B?1??set_null@?$SmallDynStorage@UProcAdjust@@HUStandardAlloc@NAlloc@@@NArray@@IEAAXXZ@51 000000003166ef24     ParamLoader.obj
 0003:0000af28       ?s_EmptyElems@?1??set_null@?$SmallDynStorage@UIKLimbType@@HUStandardAlloc@NAlloc@@@NArray@@IEAAXXZ@4PEAUIKLimbType@@EA 000000003166ef28     ParamLoader.obj
 0003:0000af30       ?s_EmptyHeader@?1??set_null@?$SmallDynStorage@UIKLimbType@@HUStandardAlloc@NAlloc@@@NArray@@IEAAXXZ@4UEmptyHeader@23@A 000000003166ef30     ParamLoader.obj
 0003:0000af3c       ??_B?1??set_null@?$SmallDynStorage@UIKLimbType@@HUStandardAlloc@NAlloc@@@NArray@@IEAAXXZ@51 000000003166ef3c     ParamLoader.obj
 0003:0000af40       ?s_EmptyElems@?1??set_null@?$SmallDynStorage@UADIKTarget@@HUStandardAlloc@NAlloc@@@NArray@@IEAAXXZ@4PEAUADIKTarget@@EA 000000003166ef40     ParamLoader.obj
 0003:0000af48       ?s_EmptyHeader@?1??set_null@?$SmallDynStorage@UADIKTarget@@HUStandardAlloc@NAlloc@@@NArray@@IEAAXXZ@4UEmptyHeader@23@A 000000003166ef48     ParamLoader.obj
 0003:0000af54       ??_B?1??set_null@?$SmallDynStorage@UADIKTarget@@HUStandardAlloc@NAlloc@@@NArray@@IEAAXXZ@51 000000003166ef54     ParamLoader.obj
 0003:0000af58       ?s_EmptyElems@?1??set_null@?$SmallDynStorage@PEAVCCharInstance@@HUStandardAlloc@NAlloc@@@NArray@@IEAAXXZ@4PEAPEAVCCharInstance@@EA 000000003166ef58     Model.obj
 0003:0000af60       ?s_EmptyHeader@?1??set_null@?$SmallDynStorage@PEAVCCharInstance@@HUStandardAlloc@NAlloc@@@NArray@@IEAAXXZ@4UEmptyHeader@23@A 000000003166ef60     Model.obj
 0003:0000af6c       ??_B?1??set_null@?$SmallDynStorage@PEAVCCharInstance@@HUStandardAlloc@NAlloc@@@NArray@@IEAAXXZ@51 000000003166ef6c     Model.obj
 0003:0000af70       ?s_EmptyElems@?1??set_null@?$SmallDynStorage@USJointProperty@@HUStandardAlloc@NAlloc@@@NArray@@IEAAXXZ@4PEAUSJointProperty@@EA 000000003166ef70     Model.obj
 0003:0000af78       ?s_EmptyHeader@?1??set_null@?$SmallDynStorage@USJointProperty@@HUStandardAlloc@NAlloc@@@NArray@@IEAAXXZ@4UEmptyHeader@23@A 000000003166ef78     Model.obj
 0003:0000af84       ??_B?1??set_null@?$SmallDynStorage@USJointProperty@@HUStandardAlloc@NAlloc@@@NArray@@IEAAXXZ@51 000000003166ef84     Model.obj
 0003:0000af88       ?s_EmptyElems@?1??set_null@?$SmallDynStorage@UMeshCollisionInfo@@HUStandardAlloc@NAlloc@@@NArray@@IEAAXXZ@4PEAUMeshCollisionInfo@@EA 000000003166ef88     Model.obj
 0003:0000af90       ?s_EmptyHeader@?1??set_null@?$SmallDynStorage@UMeshCollisionInfo@@HUStandardAlloc@NAlloc@@@NArray@@IEAAXXZ@4UEmptyHeader@23@A 000000003166ef90     Model.obj
 0003:0000af9c       ??_B?1??set_null@?$SmallDynStorage@UMeshCollisionInfo@@HUStandardAlloc@NAlloc@@@NArray@@IEAAXXZ@51 000000003166ef9c     Model.obj
 0003:0000baa0       ?g_pCharacterManager@@3PEAVCharacterManager@@EA 000000003166faa0     AnimationBase.obj
 0003:0000baa8       ?numAllocations@_CryMemoryManagerPoolHelper@@2HC 000000003166faa8     AnimationBase.obj
 0003:0000baac       ?requestedMemory@_CryMemoryManagerPoolHelper@@2JC 000000003166faac     AnimationBase.obj
 0003:0000bab0       ?freedMemory@_CryMemoryManagerPoolHelper@@2JC 000000003166fab0     AnimationBase.obj
 0003:0000bab4       ?allocatedMemory@_CryMemoryManagerPoolHelper@@2JC 000000003166fab4     AnimationBase.obj
 0003:0000bab8       ?gEnv@@3PEAUSSystemGlobalEnvironment@@EA 000000003166fab8     AnimationBase.obj
 0003:0000bac0       ?m_pFirst@Test@CryUnitTest@@2PEAU12@EA 000000003166fac0     AnimationBase.obj
 0003:0000bac8       ?m_pLast@Test@CryUnitTest@@2PEAU12@EA 000000003166fac8     AnimationBase.obj
 0003:0000bad0       ?g_pHeadToRegFactories@@3PEAUSRegFactoryNode@@EA 000000003166fad0     AnimationBase.obj
 0003:0000bad8       ?g_bProfilerEnabled@@3_NA  000000003166fad8     AnimationBase.obj
 0003:0000bad9       ?g_bForceLOD@@3_NA         000000003166fad9     AnimationBase.obj
 0003:0000bada       ?g_bProfilerOn@@3_NA       000000003166fada     AnimationBase.obj
 0003:0000badc       ?g_iTraceAllocations@@3HA  000000003166fadc     AnimationBase.obj
 0003:0000bae0       ?_CryMalloc@_CryMemoryManagerPoolHelper@@2P6APEAX_KAEA_K0@ZEA 000000003166fae0     AnimationBase.obj
 0003:0000bae8       ?_CryGetMemSize@_CryMemoryManagerPoolHelper@@2P6A_KPEAX_K@ZEA 000000003166fae8     AnimationBase.obj
 0003:0000baf0       ?_CryRealloc@_CryMemoryManagerPoolHelper@@2P6APEAXPEAX_KAEA_K21@ZEA 000000003166faf0     AnimationBase.obj
 0003:0000baf8       ?_CryFree@_CryMemoryManagerPoolHelper@@2P6A_KPEAX_K@ZEA 000000003166faf8     AnimationBase.obj
 0003:0000bb00       ?_CryCrtMalloc@_CryMemoryManagerPoolHelper@@2P6APEAX_K@ZEA 000000003166fb00     AnimationBase.obj
 0003:0000bb08       ?_CryCrtRealloc@_CryMemoryManagerPoolHelper@@2P6APEAXPEAX_K@ZEA 000000003166fb08     AnimationBase.obj
 0003:0000bb10       ?_CryCrtFree@_CryMemoryManagerPoolHelper@@2P6A_KPEAX@ZEA 000000003166fb10     AnimationBase.obj
 0003:0000bb18       ?_CryCrtSize@_CryMemoryManagerPoolHelper@@2P6A_KPEAX@ZEA 000000003166fb18     AnimationBase.obj
 0003:0000bb20       ?_CryGetIMemoryManagerInterface@_CryMemoryManagerPoolHelper@@2P6AXPEAPEAX@ZEA 000000003166fb20     AnimationBase.obj
 0003:0000bb28       ?m_bInitialized@_CryMemoryManagerPoolHelper@@2HA 000000003166fb28     AnimationBase.obj
 0003:0000bb2c       ?g_AverageFrameTime@@3MA   000000003166fb2c     AnimationBase.obj
 0003:0000bb30       ?g_pISystem@@3PEAUISystem@@EA 000000003166fb30     AnimationBase.obj
 0003:0000bb38       ?g_pITimer@@3PEAUITimer@@EA 000000003166fb38     AnimationBase.obj
 0003:0000bb40       ?g_pILog@@3PEAUILog@@EA    000000003166fb40     AnimationBase.obj
 0003:0000bb48       ?g_pIConsole@@3PEAUIConsole@@EA 000000003166fb48     AnimationBase.obj
 0003:0000bb50       ?g_pIPak@@3PEAUICryPak@@EA 000000003166fb50     AnimationBase.obj
 0003:0000bb58       ?g_pIStreamEngine@@3PEAUIStreamEngine@@EA 000000003166fb58     AnimationBase.obj
 0003:0000bb60       ?g_pCrc32Gen@@3PEAVCrc32Gen@@EA 000000003166fb60     AnimationBase.obj
 0003:0000bb68       ?g_pIRenderer@@3PEAUIRenderer@@EA 000000003166fb68     AnimationBase.obj
 0003:0000bb70       ?g_pAuxGeom@@3PEAUIRenderAuxGeom@@EA 000000003166fb70     AnimationBase.obj
 0003:0000bb78       ?g_pIPhysicalWorld@@3PEAUIPhysicalWorld@@EA 000000003166fb78     AnimationBase.obj
 0003:0000bb80       ?g_pI3DEngine@@3PEAUI3DEngine@@EA 000000003166fb80     AnimationBase.obj
 0003:0000bb88       ?g_nRenderThreadUpdateID@@3HA 000000003166fb88     AnimationBase.obj
 0003:0000bb8c       ?g_totalParametrics@@3HA   000000003166fb8c     AnimationBase.obj
 0003:0000bb90       ?g_parametricPool@@3PEAUSParametricSamplerInternal@@EA 000000003166fb90     AnimationBase.obj
 0003:0000bb98       ?g_usedParametrics@@3PEA_NEA 000000003166fb98     AnimationBase.obj
 0003:0000bba0       ?g_ForcedLODNum@@3HA       000000003166fba0     AnimationBase.obj
 0003:0000bba4       ?g_fCurrTime@@3MA          000000003166fba4     AnimationBase.obj
 0003:0000bba8       ?g_CpuFlags@@3HA           000000003166fba8     AnimationBase.obj
 0003:0000bbac       ?g_random_generator@@3VCLCGRndGen@@A 000000003166fbac     AnimationBase.obj
 0003:0000bbb0       ?s_factory@CFactory@CEngineModule_CryAnimation@@0V12@A 000000003166fbb0     AnimationBase.obj
 0003:0000bc00       ?g_DataMismatch@@3U?$DynArray@V?$CryStringT@D@@HU?$SmallDynStorage@V?$CryStringT@D@@HUStandardAlloc@NAlloc@@@NArray@@@@A 000000003166fc00     AnimationBase.obj
 0003:0000bc08       ?g_IdentityAABB@@3UAABB@@A 000000003166fc08     AnimationBase.obj
 0003:0000bc20       ?g_controllerHeap@@3VCControllerDefragHeap@@A 000000003166fc20     AnimationBase.obj
 0003:0000c558       ?g_AnimStatisticsInfo@@3UAnimStatisticsInfo@@A 0000000031670558     AnimationBase.obj
 0003:0000c580       ?s_used_memory@?1??_usedMemory@?$CryStringT@_W@@SA_K_J@Z@4_KA 0000000031670580     AnimationBase.obj
 0003:0000c588       ?supportedIIDs@?1???0CFactory@CEngineModule_CryAnimation@@AEAA@XZ@4PAUCryGUID@@A 0000000031670588     AnimationBase.obj
 0003:0000c5a8       ?p@?1??CreateClassInstance@CFactory@CEngineModule_CryAnimation@@UEBA?AV?$shared_ptr@UICryUnknown@@@boost@@XZ@4V?$shared_ptr@VCEngineModule_CryAnimation@@@5@A 00000000316705a8     AnimationBase.obj
 0003:0000c5b8       ??_B?1??CreateClassInstance@CFactory@CEngineModule_CryAnimation@@UEBA?AV?$shared_ptr@UICryUnknown@@@boost@@XZ@51 00000000316705b8     AnimationBase.obj
 0003:0000c5bc       ?g_ConsoleInstanceCount@?A0xe26663e7@@3HA 00000000316705bc     cvars.obj
 0003:0000c5e0       ?g_globalSections@?$Node_Alloc_Lock@$00$00@@2PAUInternalCriticalSectionDummy@@A 00000000316705e0     stdafx.obj
 0003:0000d660       ?m_bInitialized@?$Node_Alloc_Lock@$00$00@@2_NA 0000000031671660     stdafx.obj
 0003:0000d668       ?gJobHandleTSkinAttachmentTangents@Detail@JobManager@@3PEAUSJobStringHandle@2@EA 0000000031671668     _RenderSkinsSW.obj
 0003:0000d670       ?gJobHandleTSkinAttachmentQtangents@Detail@JobManager@@3PEAUSJobStringHandle@2@EA 0000000031671670     _RenderSkinsSW.obj
 0003:0000d680       ?__type_info_root_node@@3U__type_info_node@@A 0000000031671680     MSVCRT:tncleanup.obj
 0003:0000d690       __native_startup_state     0000000031671690     <common>
 0003:0000d698       __native_startup_lock      0000000031671698     <common>
 0003:0000d6a0       __dyn_tls_init_callback    00000000316716a0     <common>
 0003:0000d6a8       __onexitend                00000000316716a8     <common>
 0003:0000d6b0       __onexitbegin              00000000316716b0     <common>
 0005:00000000       ?m_Self@CrySimpleThreadSelf@@1PEAV1@EA 0000000031680000     AnimationBase.obj

 entry point at        0001:0013fb90

 Static symbols

 0001:00011fa0       ?ValidateLodSkeleton@CryCHRLoader_LoadNewSKIN_Helpers@@YA_NPEAUCSkinningInfo@@0HPEBD@Z 0000000031512fa0 f   LoaderSKIN.obj
 0001:00011fa0       ?ValidateLodSkeleton@CryCHRLoader_LoadNewCHR_Helpers@@YA_NPEAUCSkinningInfo@@0HPEBD@Z 0000000031512fa0 f   LoaderSKIN.obj
 0001:00015550       ?GetLODName@CryCHRLoader_LoadNewSKIN_Helpers@@YA?AV?$CryStringT@D@@AEBV2@PEBDI@Z 0000000031516550 f   LoaderSKIN.obj
 0001:00015f50       ?FindFirstMeshAndMaterial@CryCHRLoader_LoadNewCHR_Helpers@@YA_NAEAPEAVCMesh@@AEAPEAUCNodeCGF@@AEAV?$_smart_ptr@UIMaterial@@@@PEAVCContentCGF@@PEBDH@Z 0000000031516f50 f   LoaderSKIN.obj
 0001:00015f50       ?FindFirstMeshAndMaterial@CryCHRLoader_LoadNewSKIN_Helpers@@YA_NAEAPEAVCMesh@@AEAPEAUCNodeCGF@@AEAV?$_smart_ptr@UIMaterial@@@@PEAVCContentCGF@@PEBDH@Z 0000000031516f50 f   LoaderSKIN.obj
 0001:00016120       ?release@ContentCgfs@?6??LoadNewSKIN@CryCHRLoader@@QEAAPEAVCSkin@@PEBDI@Z@QEAAXXZ 0000000031517120 f   LoaderSKIN.obj
 0001:00016120       ?release@ContentCgfs@?4??LoadNewCHR@CryCHRLoader@@QEAAPEAVCSkel@@PEBDI@Z@QEAAXXZ 0000000031517120 f   LoaderSKIN.obj
 0001:00016ba0       ?ExtractExternalVertices@CryCHRLoader_LoadNewSKIN_Helpers@@YA_NAEAU?$DynArray@UExtSkinVertex@@HU?$SmallDynStorage@UExtSkinVertex@@HUStandardAlloc@NAlloc@@@NArray@@@@PEBVCModelMesh@@IPEBVCMesh@@PEBDH@Z 0000000031517ba0 f   LoaderSKIN.obj
 0001:00018360       ?InitializeBones@CryCHRLoader_LoadNewSKIN_Helpers@@YA_NPEAVCSkin@@PEAUCSkinningInfo@@PEBD@Z 0000000031519360 f   LoaderSKIN.obj
 0001:00018c60       ?CreateMorphNameToIndexMap@CryCHRLoader_LoadNewCHR_Helpers@@YA_NAEAV?$VectorMap@V?$CryStringT@D@@HU?$less@V?$CryStringT@D@@@stlpmtx_std@@V?$allocator@U?$pair@V?$CryStringT@D@@H@stlpmtx_std@@@3@@@PEAPEAVCContentCGF@@HPEBD@Z 0000000031519c60 f   LoaderSKIN.obj
 0001:00018c60       ?CreateMorphNameToIndexMap@CryCHRLoader_LoadNewSKIN_Helpers@@YA_NAEAV?$VectorMap@V?$CryStringT@D@@HU?$less@V?$CryStringT@D@@@stlpmtx_std@@V?$allocator@U?$pair@V?$CryStringT@D@@H@stlpmtx_std@@@3@@@PEAPEAVCContentCGF@@HPEBD@Z 0000000031519c60 f   LoaderSKIN.obj
 0001:0006d0e0       ?strstri@@YAPEBDPEBD0@Z    000000003156e0e0 f   SkeletonPose_Debug.obj
 0001:0007b510       ?FindChannel@JoystickSerializeContext@?4??BindJoystickSetToSequence@CFacialAnimation@@UEAAXPEAVIJoystickSet@@PEAUIFacialAnimSequence@@@Z@UEAAPEAUIFacialAnimChannel@@PEBD@Z 000000003157c510 f   FaceAnimation.obj
 0001:000876b0       ??RRecurser@?CL@??BindChannels@CFacialAnimSequenceInstance@@QEAAXPEAVCFacialAnimationContext@@PEAVCFacialAnimSequence@@@Z@QEAAXPEAUIFacialEffector@@@Z 00000000315886b0 f   FaceAnimSequence.obj
 0001:0009be60       ?Recurse@Recurser@?M@??RemoveEffector@CFacialEffectorsLibrary@@UEAAXPEAUIFacialEffector@@@Z@AEAAX0@Z 000000003159ce60 f   FaceEffectorLibrary.obj
 0001:0009bef0       ?CopyController@Recurser@?4??MergeLibrary@CFacialEffectorsLibrary@@UEAAXPEAUIFacialEffectorsLibrary@@AEBV?$Functor1wRet@PEBDW4MergeCollisionAction@@@@@Z@AEAAXPEAUIFacialEffCtrl@@2@Z 000000003159cef0 f   FaceEffectorLibrary.obj
 0001:0009c130       ?Recurse@Recurser@?M@??ReplaceEffector@CFacialEffectorsLibrary@@AEAAXPEAVCFacialEffector@@0@Z@AEAAXPEAUIFacialEffector@@@Z 000000003159d130 f   FaceEffectorLibrary.obj
 0001:0009dd90       ?Recurse@Recurser@?4??MergeLibrary@CFacialEffectorsLibrary@@UEAAXPEAUIFacialEffectorsLibrary@@AEBV?$Functor1wRet@PEBDW4MergeCollisionAction@@@@@Z@AEAAXPEAUIFacialEffector@@2@Z 000000003159ed90 f   FaceEffectorLibrary.obj
 0001:000d56f0       ?GetLodIndex@CryCGALoaderHelper@@YAHQEBD@Z 00000000315d66f0 f   LoaderCGA.obj
 0001:000e5420       ?GetLODName@CryCHRLoader_LoadNewCHR_Helpers@@YA?AV?$CryStringT@D@@AEBV2@PEBDI@Z 00000000315e6420 f   LoaderCHR.obj
 0001:000e65a0       ?ExtractExternalVertices@CryCHRLoader_LoadNewCHR_Helpers@@YA_NAEAU?$DynArray@UExtSkinVertex@@HU?$SmallDynStorage@UExtSkinVertex@@HUStandardAlloc@NAlloc@@@NArray@@@@PEBVCModelMesh@@IPEBVCMesh@@PEBDH@Z 00000000315e75a0 f   LoaderCHR.obj
 0001:000e6e00       ?SetupPhysicalProxies@CryCHRLoader_LoadNewCHR_Helpers@@YA_NPEAUIGeomManager@@PEAVCSkel@@PEAUIMaterial@@PEBUCSkinningInfo@@PEBDH@Z 00000000315e7e00 f   LoaderCHR.obj
 0001:000e7b30       ?CopyMorphTargets@CryCHRLoader_LoadNewCHR_Helpers@@YA_NPEAVCModelMesh@@IPEAUCSkinningInfo@@AEBU?$DynArray@UExtSkinVertex@@HU?$SmallDynStorage@UExtSkinVertex@@HUStandardAlloc@NAlloc@@@NArray@@@@AEBV?$VectorMap@V?$CryStringT@D@@HU?$less@V?$CryStringT@D@@@stlpmtx_std@@V?$allocator@U?$pair@V?$CryStringT@D@@H@stlpmtx_std@@@3@@@PEBDH@Z 00000000315e8b30 f   LoaderCHR.obj
 0001:000e7b30       ?CopyMorphTargets@CryCHRLoader_LoadNewSKIN_Helpers@@YA_NPEAVCModelMesh@@IPEAUCSkinningInfo@@AEBU?$DynArray@UExtSkinVertex@@HU?$SmallDynStorage@UExtSkinVertex@@HUStandardAlloc@NAlloc@@@NArray@@@@AEBV?$VectorMap@V?$CryStringT@D@@HU?$less@V?$CryStringT@D@@@stlpmtx_std@@V?$allocator@U?$pair@V?$CryStringT@D@@H@stlpmtx_std@@@3@@@PEBDH@Z 00000000315e8b30 f   LoaderCHR.obj
 0001:000e96c0       ?InitializeBones@CryCHRLoader_LoadNewCHR_Helpers@@YA_NPEAVCModelSkeleton@@PEAUCSkinningInfo@@PEBD@Z 00000000315ea6c0 f   LoaderCHR.obj
 0001:0013c2d0       ?CADebugText@@YAXPEAUIConsoleCmdArgs@@@Z 000000003163d2d0 f   cvars.obj
 0001:0013f798       pre_c_init                 0000000031640798 f   MSVCRT:crtdll.obj
 0001:0013fa54       __DllMainCRTStartup        0000000031640a54 f   MSVCRT:crtdll.obj
 0001:0013fe30       _onexit$fin$0              0000000031640e30 f   MSVCRT:atonexit.obj
 0001:0013fe4b       __DllMainCRTStartup$filt$0 0000000031640e4b f   MSVCRT:crtdll.obj
 0001:0013fe7b       __DllMainCRTStartup$fin$1  0000000031640e7b f   MSVCRT:crtdll.obj
 0001:0013fea0       _IsNonwritableInCurrentImage$filt$0 0000000031640ea0 f   MSVCRT:pesect.obj
 0001:0013fed0       ??__E?s_factory@CFactory@COperatorQueue@@0V12@A@@YAXXZ 0000000031640ed0 f   OperatorQueue.obj
 0001:0013fef0       ??__E?s_factory@CFactory@CPoseAlignerChain@@0V12@A@@YAXXZ 0000000031640ef0 f   PoseAlignerChain.obj
 0001:0013ff10       ??__E?s_factory@CFactory@CPoseMatching@@0V12@A@@YAXXZ 0000000031640f10 f   PoseMatching.obj
 0001:0013ff30       ??__E?g_firstValidator@SBatchUpdateValidator@@2U1@A@@YAXXZ 0000000031640f30 f   SkeletonPhysics.obj
 0001:0013ff90       ??__Eg_arrVerticesBS@@YAXXZ 0000000031640f90 f   DecalManager.obj
 0001:0013ffc0       ??__Eg_arrDecalVertexMapping@@YAXXZ 0000000031640fc0 f   DecalManager.obj
 0001:0013fff0       ??__Eg_arrDecalFaceMapping@@YAXXZ 0000000031640ff0 f   DecalManager.obj
 0001:00140020       ??__EGUID_AnimationPoseModifier_TransformationPin@@YAXXZ 0000000031641020 f   SkeletonAnim.obj
 0001:00140050       ??__E?s_factory@CFactory@CFeetPoseStore@@0V12@A@@YAXXZ 0000000031641050 f   FeetLock.obj
 0001:001400b0       ??__E?s_factory@CFactory@CFeetPoseRestore@@0V12@A@@YAXXZ 00000000316410b0 f   FeetLock.obj
 0001:00140110       ??__E?s_factory@CFactory@CGroundAlignment@@0V12@A@@YAXXZ 0000000031641110 f   GroundAlignment.obj
 0001:00140130       ??__E?s_factory@CFactory@CLimbIk@@0V12@A@@YAXXZ 0000000031641130 f   LimbIk.obj
 0001:00140190       ??__E?s_factory@CFactory@CPoseBlenderAim@@0V12@A@@YAXXZ 0000000031641190 f   PoseBlenderAim.obj
 0001:001401b0       ??__E?s_factory@CFactory@CPoseBlenderLook@@0V12@A@@YAXXZ 00000000316411b0 f   PoseBlenderLook.obj
 0001:001401d0       ??__E?s_factory@CFactory@CRecoil@PoseModifier@@0V123@A@@YAXXZ 00000000316411d0 f   Recoil.obj
 0001:00140230       ??__ECryUserInvalidID@@YAXXZ 0000000031641230 f   CharacterManager.obj
 0001:00140240       ??__ECrySessionInvalidID@@YAXXZ 0000000031641240 f   CharacterManager.obj
 0001:00140250       ??__Eg_random_generator@@YAXXZ 0000000031641250 f   AnimationBase.obj
 0001:00140260       ??__Eg_system_event_listener_anim@@YAXXZ 0000000031641260 f   AnimationBase.obj
 0001:00140270       ??__E?s_factory@CFactory@CEngineModule_CryAnimation@@0V12@A@@YAXXZ 0000000031641270 f   AnimationBase.obj
 0001:00140290       ??__Eg_DefaultAnim@@YAXXZ  0000000031641290 f   AnimationBase.obj
 0001:001402c0       ??__Eg_DataMismatch@@YAXXZ 00000000316412c0 f   AnimationBase.obj
 0001:00140330       ??__Eg_IdentityAABB@@YAXXZ 0000000031641330 f   AnimationBase.obj
 0001:001403a0       ??__Eg_controllerHeap@@YAXXZ 00000000316413a0 f   AnimationBase.obj
 0001:001403c0       ??__Eg_Consoleself@@YAXXZ  00000000316413c0 f   cvars.obj
 0001:001403f0       ??__EautoInitializer@@YAXXZ 00000000316413f0 f   stdafx.obj
 0001:00140460       ??__FarrExtSkinnedStream@?1??DrawWireframeStatic@CModelMesh@@QEAAXAEBU?$Matrix34_tpl@M@@PEAUIRenderMesh@@I@Z@YAXXZ 0000000031641460 f   ModelMesh_DebugPC.obj
 0001:001404a0       ??__FarrExtSkinnedStream@?EI@??SoftwareSkinningDQ@CModelMesh@@QEAAXPEAUIRenderMesh@@PEAVCCharInstance@@PEAVCAttachmentSKIN@@U?$Matrix34_tpl@M@@EEEEPEAU?$DualQuat_tpl@M@@@Z@YAXXZ 00000000316414a0 f   ModelMesh_DebugPC.obj
 0001:001404e0       ??__FarrExtVColors@?EE@??SoftwareSkinningDQ@CModelMesh@@QEAAXPEAUIRenderMesh@@PEAVCCharInstance@@PEAVCAttachmentSKIN@@U?$Matrix34_tpl@M@@EEEEPEAU?$DualQuat_tpl@M@@@Z@YAXXZ 00000000316414e0 f   ModelMesh_DebugPC.obj
 0001:00140520       ??__FarrExtSkinnedStream@?DN@??SoftwareSkinningDQ@CModelMesh@@QEAAXPEAUIRenderMesh@@PEAVCCharInstance@@PEAVCAttachmentSKIN@@U?$Matrix34_tpl@M@@EEEEPEAU?$DualQuat_tpl@M@@@Z@YAXXZ 0000000031641520 f   ModelMesh_DebugPC.obj
 0001:00140560       ??__FarrExtVColors@?DJ@??SoftwareSkinningDQ@CModelMesh@@QEAAXPEAUIRenderMesh@@PEAVCCharInstance@@PEAVCAttachmentSKIN@@U?$Matrix34_tpl@M@@EEEEPEAU?$DualQuat_tpl@M@@@Z@YAXXZ 0000000031641560 f   ModelMesh_DebugPC.obj
 0001:001405a0       ??__FarrExtSkinnedStream@?DC@??SoftwareSkinningDQ@CModelMesh@@QEAAXPEAUIRenderMesh@@PEAVCCharInstance@@PEAVCAttachmentSKIN@@U?$Matrix34_tpl@M@@EEEEPEAU?$DualQuat_tpl@M@@@Z@YAXXZ 00000000316415a0 f   ModelMesh_DebugPC.obj
 0001:001405e0       ??__FarrExtVColors@?CO@??SoftwareSkinningDQ@CModelMesh@@QEAAXPEAUIRenderMesh@@PEAVCCharInstance@@PEAVCAttachmentSKIN@@U?$Matrix34_tpl@M@@EEEEPEAU?$DualQuat_tpl@M@@@Z@YAXXZ 00000000316415e0 f   ModelMesh_DebugPC.obj
 0001:00140620       ??__Fg_arrQTangents@?1??SoftwareSkinningDQ@CModelMesh@@QEAAXPEAUIRenderMesh@@PEAVCCharInstance@@PEAVCAttachmentSKIN@@U?$Matrix34_tpl@M@@EEEEPEAU?$DualQuat_tpl@M@@@Z@YAXXZ 0000000031641620 f   ModelMesh_DebugPC.obj
 0001:00140660       ??__Fg_arrExtSkinnedStream@?1??SoftwareSkinningDQ@CModelMesh@@QEAAXPEAUIRenderMesh@@PEAVCCharInstance@@PEAVCAttachmentSKIN@@U?$Matrix34_tpl@M@@EEEEPEAU?$DualQuat_tpl@M@@@Z@YAXXZ 0000000031641660 f   ModelMesh_DebugPC.obj
 0001:001406a0       ??__F?s_factory@CFactory@COperatorQueue@@0V12@A@@YAXXZ 00000000316416a0 f   OperatorQueue.obj
 0001:001406b0       ??__F?s_factory@CFactory@CPoseAlignerChain@@0V12@A@@YAXXZ 00000000316416b0 f   PoseAlignerChain.obj
 0001:001406c0       ??__F?s_factory@CFactory@CPoseMatching@@0V12@A@@YAXXZ 00000000316416c0 f   PoseMatching.obj
 0001:001406d0       ??__F?g_firstValidator@SBatchUpdateValidator@@2U1@A@@YAXXZ 00000000316416d0 f   SkeletonPhysics.obj
 0001:00140730       ??__FarrExtSkinnedStream@?GA@??DrawAttachment@CAttachmentSKIN@@UEAAXAEAUSRendParams@@AEBUSRenderingPassInfo@@AEBU?$Matrix34_tpl@M@@M@Z@YAXXZ 0000000031641730 f   _RenderSkins.obj
 0001:00140770       ??__FarrExtVColors@?FM@??DrawAttachment@CAttachmentSKIN@@UEAAXAEAUSRendParams@@AEBUSRenderingPassInfo@@AEBU?$Matrix34_tpl@M@@M@Z@YAXXZ 0000000031641770 f   _RenderSkins.obj
 0001:001407b0       ??__FarrDstPositions@?FD@??DrawAttachment@CAttachmentSKIN@@UEAAXAEAUSRendParams@@AEBUSRenderingPassInfo@@AEBU?$Matrix34_tpl@M@@M@Z@YAXXZ 00000000316417b0 f   _RenderSkins.obj
 0001:001407f0       ??__Fg_arrDecalFaceMapping@@YAXXZ 00000000316417f0 f   DecalManager.obj
 0001:00140830       ??__Fg_arrVerticesBS@@YAXXZ 0000000031641830 f   DecalManager.obj
 0001:00140870       ??__Fg_arrDecalVertexMapping@@YAXXZ 0000000031641870 f   DecalManager.obj
 0001:001408b0       ??__F?s_factory@CFactory@CFeetPoseStore@@0V12@A@@YAXXZ 00000000316418b0 f   FeetLock.obj
 0001:001408c0       ??__F?s_factory@CFactory@CFeetPoseRestore@@0V12@A@@YAXXZ 00000000316418c0 f   FeetLock.obj
 0001:001408d0       ??__F?s_factory@CFactory@CGroundAlignment@@0V12@A@@YAXXZ 00000000316418d0 f   GroundAlignment.obj
 0001:001408e0       ??__F?s_factory@CFactory@CLimbIk@@0V12@A@@YAXXZ 00000000316418e0 f   LimbIk.obj
 0001:001408f0       ??__F?s_factory@CFactory@CPoseBlenderAim@@0V12@A@@YAXXZ 00000000316418f0 f   PoseBlenderAim.obj
 0001:00140900       ??__F?s_factory@CFactory@CPoseBlenderLook@@0V12@A@@YAXXZ 0000000031641900 f   PoseBlenderLook.obj
 0001:00140910       ??__F?s_factory@CFactory@CRecoil@PoseModifier@@0V123@A@@YAXXZ 0000000031641910 f   Recoil.obj
 0001:00140920       ??__FCrySessionInvalidID@@YAXXZ 0000000031641920 f   CharacterManager.obj
 0001:00140970       ??__FCryUserInvalidID@@YAXXZ 0000000031641970 f   CharacterManager.obj
 0001:001409c0       ??__Fg_controllerHeap@@YAXXZ 00000000316419c0 f   AnimationBase.obj
 0001:001409d0       ??__F?s_factory@CFactory@CEngineModule_CryAnimation@@0V12@A@@YAXXZ 00000000316419d0 f   AnimationBase.obj
 0001:00140a00       ??__Fg_DefaultAnim@@YAXXZ  0000000031641a00 f   AnimationBase.obj
 0001:00140a10       ??__Fg_system_event_listener_anim@@YAXXZ 0000000031641a10 f   AnimationBase.obj
 0001:00140a60       ??__Fg_DataMismatch@@YAXXZ 0000000031641a60 f   AnimationBase.obj
 0001:00140ad0       ??__Fg_Consoleself@@YAXXZ  0000000031641ad0 f   cvars.obj
 0001:00140b10       ??__FautoInitializer@@YAXXZ 0000000031641b10 f   stdafx.obj
